 config_alm_db_output

 Timestamp is 614c80f9 (Thu Sep 23 13:28:25 2021)

 Preferred load address is 10000000

 Start         Length     Name                   Class
 0001:00000000 00000134H .text$di                CODE
 0001:00000140 0001feacH .text$mn                CODE
 0001:0001fff0 00004ecdH .text$x                 CODE
 0001:00024ec0 0000008fH .text$yd                CODE
 0002:00000000 0000167cH .idata$5                DATA
 0002:0000167c 00000004H .CRT$XCA                DATA
 0002:00001680 0000002cH .CRT$XCU                DATA
 0002:000016ac 00000004H .CRT$XCZ                DATA
 0002:000016b0 00000004H .CRT$XIA                DATA
 0002:000016b4 00000004H .CRT$XIAA               DATA
 0002:000016b8 00000004H .CRT$XIC                DATA
 0002:000016bc 00000004H .CRT$XIZ                DATA
 0002:000016c0 00008990H .rdata                  DATA
 0002:0000a050 00001f50H .rdata$r                DATA
 0002:0000bfa0 00000004H .rtc$IAA                DATA
 0002:0000bfa4 00000004H .rtc$IZZ                DATA
 0002:0000bfa8 00000004H .rtc$TAA                DATA
 0002:0000bfac 00000004H .rtc$TZZ                DATA
 0002:0000bfb0 0000483cH .xdata$x                DATA
 0002:000107f0 00000068H .edata                  DATA
 0002:00010858 00000078H .idata$2                DATA
 0002:000108d0 00000014H .idata$3                DATA
 0002:000108e4 0000167cH .idata$4                DATA
 0002:00011f60 0000e660H .idata$6                DATA
 0003:00000000 00000194H .data                   DATA
 0003:00000194 00000a14H .data$r                 DATA
 0003:00000ba8 000003dcH .bss                    DATA
 0004:00000000 000000a0H .rsrc$01                DATA
 0004:000000a0 00000630H .rsrc$02                DATA

  Address         Publics by Value              Rva+Base       Lib:Object

 0000:00000000       ___guard_flags             00000000     <absolute>
 0000:00000000       ___guard_fids_count        00000000     <absolute>
 0000:00000000       ___safe_se_handler_count   00000000     <absolute>
 0000:00000000       __except_list              00000000     <absolute>
 0000:00000000       ___guard_fids_table        00000000     <absolute>
 0000:00000000       ___safe_se_handler_table   00000000     <absolute>
 0000:00009876       __ldused                   00009876     <absolute>
 0000:00009876       __fltused                  00009876     <absolute>
 0000:00000000       ___ImageBase               10000000     <linker-defined>
 0001:00000140       ??$_Allocate@D@std@@YAPADIPAD@Z 10001140 f i alm_db_output.obj
 0001:00000168       ??0?$QGuardedPtr@VQDockWindow@@@@QAE@XZ 10001168 f i alm_db_output.obj
 0001:00000168       ??0?$QGuardedPtr@VQPopupMenu@@@@QAE@XZ 10001168 f i alm_db_output.obj
 0001:000001a9       ??0?$QMap@VQString@@PAVcProcess@@@@QAE@XZ 100011a9 f i alm_db_output.obj
 0001:000001dc       ??0?$QMapNode@VQString@@PAVcProcess@@@@QAE@ABU0@@Z 100011dc f i alm_db_output.obj
 0001:0000021a       ??0?$QMapNode@VQString@@PAVcProcess@@@@QAE@ABVQString@@@Z 1000121a f i alm_db_output.obj
 0001:0000024e       ??0?$QMapPrivate@VQString@@PAVcProcess@@@@QAE@PBV0@@Z 1000124e f i alm_db_output.obj
 0001:00000300       ??0?$QMapPrivate@VQString@@PAVcProcess@@@@QAE@XZ 10001300 f i alm_db_output.obj
 0001:0000035c       ??0?$basic_string@DU?$char_traits@D@std@@V?$allocator@D@2@@std@@QAE@PBD@Z 1000135c f i alm_db_output.obj
 0001:0000038b       ??0FileLoad_BncsSystem@alm_db_output@@QAE@PAV1@@Z 1000138b f   alm_db_output.obj
 0001:000003fc       ??0alm_db_output@@QAE@ABVQString@@00@Z 100013fc f   alm_db_output.obj
 0001:0000114f       ??0config_plugin_base@@QAE@ABVQString@@00@Z 1000214f f i alm_db_output.obj
 0001:000011dc       ??1?$QDict@VQAction@@@@UAE@XZ 100021dc f i alm_db_output.obj
 0001:0000120f       ??1?$QGuardedPtr@VQPopupMenu@@@@QAE@XZ 1000220f f i alm_db_output.obj
 0001:0000120f       ??1?$QGuardedPtr@VQDockWindow@@@@QAE@XZ 1000220f f i alm_db_output.obj
 0001:00001214       ??1?$QMap@VQString@@PAVcProcess@@@@QAE@XZ 10002214 f i alm_db_output.obj
 0001:00001231       ??1?$QMapPrivate@VQString@@PAVcProcess@@@@QAE@XZ 10002231 f i alm_db_output.obj
 0001:00001252       ??1?$QPtrList@VQPopupMenu@@@@UAE@XZ 10002252 f i alm_db_output.obj
 0001:00001285       ??1?$QPtrList@VcOutputFile@@@@UAE@XZ 10002285 f i alm_db_output.obj
 0001:000012b8       ??1?$QPtrList@VcProcess@@@@UAE@XZ 100022b8 f i alm_db_output.obj
 0001:000012eb       ??1FileLoad_BncsSystem@alm_db_output@@UAE@XZ 100022eb f   alm_db_output.obj
 0001:00001324       ??1QDockWindowList@@UAE@XZ 10002324 f i alm_db_output.obj
 0001:0000136d       ??1QPopupMenuList@@UAE@XZ  1000236d f i alm_db_output.obj
 0001:0000139f       ??1alm_db_output@@UAE@XZ   1000239f f   alm_db_output.obj
 0001:0000154c       ??1config_plugin_base@@UAE@XZ 1000254c f i alm_db_output.obj
 0001:000015a6       ??4?$QGuardedPtr@VQDockWindow@@@@QAEAAV0@PAVQDockWindow@@@Z 100025a6 f i alm_db_output.obj
 0001:000015a6       ??4?$QGuardedPtr@VQPopupMenu@@@@QAEAAV0@PAVQPopupMenu@@@Z 100025a6 f i alm_db_output.obj
 0001:00001604       ??8error_condition@std@@QBE_NABV01@@Z 10002604 f i alm_db_output.obj
 0001:00001623       ??A?$QMap@VQString@@PAVcProcess@@@@QAEAAPAVcProcess@@ABVQString@@@Z 10002623 f i alm_db_output.obj
 0001:00001676       ??_ECAlm_sys_select@@WCI@AEPAXI@Z 10002676 f i alm_db_output.obj
 0001:0000167e       ??_EQBoxLayout@@WCI@AEPAXI@Z 1000267e f i alm_db_output.obj
 0001:00001686       ??_EQDockWindow@@WCI@AEPAXI@Z 10002686 f i alm_db_output.obj
 0001:0000168e       ??_EQListView@@WCI@AEPAXI@Z 1000268e f i alm_db_output.obj
 0001:00001696       ??_EQPopupMenu@@WCI@AEPAXI@Z 10002696 f i alm_db_output.obj
 0001:0000169e       ??_EQPopupMenu@@WIM@AEPAXI@Z 1000269e f i alm_db_output.obj
 0001:000016a9       ??_EQTabWidget@@WCI@AEPAXI@Z 100026a9 f i alm_db_output.obj
 0001:000016b1       ??_EQToolBar@@WCI@AEPAXI@Z 100026b1 f i alm_db_output.obj
 0001:000016b9       ??_EQWidget@@WCI@AEPAXI@Z  100026b9 f i alm_db_output.obj
 0001:000016c1       ??_Ealm_db_output@@WCI@AEPAXI@Z 100026c1 f i alm_db_output.obj
 0001:000016c9       ??_Econfig_plugin_base@@WCI@AEPAXI@Z 100026c9 f i alm_db_output.obj
 0001:000016d1       ??_G?$QDict@VQAction@@@@UAEPAXI@Z 100026d1 f i alm_db_output.obj
 0001:000016d1       ??_E?$QDict@VQAction@@@@UAEPAXI@Z 100026d1 f i alm_db_output.obj
 0001:000016f0       ??_G?$QPtrList@VQPopupMenu@@@@UAEPAXI@Z 100026f0 f i alm_db_output.obj
 0001:000016f0       ??_E?$QPtrList@VQPopupMenu@@@@UAEPAXI@Z 100026f0 f i alm_db_output.obj
 0001:0000170f       ??_G?$QPtrList@VcOutputFile@@@@UAEPAXI@Z 1000270f f i alm_db_output.obj
 0001:0000170f       ??_E?$QPtrList@VcOutputFile@@@@UAEPAXI@Z 1000270f f i alm_db_output.obj
 0001:0000172e       ??_E?$QPtrList@VcProcess@@@@UAEPAXI@Z 1000272e f i alm_db_output.obj
 0001:0000172e       ??_G?$QPtrList@VcProcess@@@@UAEPAXI@Z 1000272e f i alm_db_output.obj
 0001:0000174d       ??_ECAlm_sys_select@@UAEPAXI@Z 1000274d f i alm_db_output.obj
 0001:0000174d       ??_GCAlm_sys_select@@UAEPAXI@Z 1000274d f i alm_db_output.obj
 0001:0000176d       ??_EFileLoad_BncsSystem@alm_db_output@@UAEPAXI@Z 1000276d f i alm_db_output.obj
 0001:0000176d       ??_GFileLoad_BncsSystem@alm_db_output@@UAEPAXI@Z 1000276d f i alm_db_output.obj
 0001:0000178c       ??_EQAction@@UAEPAXI@Z     1000278c f i alm_db_output.obj
 0001:0000178c       ??_GQAction@@UAEPAXI@Z     1000278c f i alm_db_output.obj
 0001:000017ac       ??_GQBoxLayout@@UAEPAXI@Z  100027ac f i alm_db_output.obj
 0001:000017ac       ??_EQBoxLayout@@UAEPAXI@Z  100027ac f i alm_db_output.obj
 0001:000017cc       ??_EQDockWindow@@UAEPAXI@Z 100027cc f i alm_db_output.obj
 0001:000017cc       ??_GQDockWindow@@UAEPAXI@Z 100027cc f i alm_db_output.obj
 0001:000017ec       ??_EQDockWindowList@@UAEPAXI@Z 100027ec f i alm_db_output.obj
 0001:000017ec       ??_GQDockWindowList@@UAEPAXI@Z 100027ec f i alm_db_output.obj
 0001:0000180b       ??_GQFile@@UAEPAXI@Z       1000280b f i alm_db_output.obj
 0001:0000180b       ??_EQFile@@UAEPAXI@Z       1000280b f i alm_db_output.obj
 0001:0000182b       ??_GQGuardedPtrPrivate@@UAEPAXI@Z 1000282b f i alm_db_output.obj
 0001:0000182b       ??_EQGuardedPtrPrivate@@UAEPAXI@Z 1000282b f i alm_db_output.obj
 0001:0000184b       ??_GQListView@@UAEPAXI@Z   1000284b f i alm_db_output.obj
 0001:0000184b       ??_EQListView@@UAEPAXI@Z   1000284b f i alm_db_output.obj
 0001:0000186b       ??_EQListViewItem@@UAEPAXI@Z 1000286b f i alm_db_output.obj
 0001:0000186b       ??_GQListViewItem@@UAEPAXI@Z 1000286b f i alm_db_output.obj
 0001:0000188b       ??_GQPopupMenu@@UAEPAXI@Z  1000288b f i alm_db_output.obj
 0001:0000188b       ??_EQPopupMenu@@UAEPAXI@Z  1000288b f i alm_db_output.obj
 0001:000018ab       ??_EQPopupMenuList@@UAEPAXI@Z 100028ab f i alm_db_output.obj
 0001:000018ab       ??_GQPopupMenuList@@UAEPAXI@Z 100028ab f i alm_db_output.obj
 0001:000018ca       ??_EQTabWidget@@UAEPAXI@Z  100028ca f i alm_db_output.obj
 0001:000018ca       ??_GQTabWidget@@UAEPAXI@Z  100028ca f i alm_db_output.obj
 0001:000018ea       ??_GQToolBar@@UAEPAXI@Z    100028ea f i alm_db_output.obj
 0001:000018ea       ??_EQToolBar@@UAEPAXI@Z    100028ea f i alm_db_output.obj
 0001:0000190a       ??_GQWidget@@UAEPAXI@Z     1000290a f i alm_db_output.obj
 0001:0000190a       ??_EQWidget@@UAEPAXI@Z     1000290a f i alm_db_output.obj
 0001:0000192a       ??_G_System_error_category@std@@UAEPAXI@Z 1000292a f i alm_db_output.obj
 0001:0000192a       ??_Eerror_category@std@@UAEPAXI@Z 1000292a f i alm_db_output.obj
 0001:0000192a       ??_G_Iostream_error_category@std@@UAEPAXI@Z 1000292a f i alm_db_output.obj
 0001:0000192a       ??_E_Iostream_error_category@std@@UAEPAXI@Z 1000292a f i alm_db_output.obj
 0001:0000192a       ??_E_System_error_category@std@@UAEPAXI@Z 1000292a f i alm_db_output.obj
 0001:0000192a       ??_Gerror_category@std@@UAEPAXI@Z 1000292a f i alm_db_output.obj
 0001:0000192a       ??_G_Generic_error_category@std@@UAEPAXI@Z 1000292a f i alm_db_output.obj
 0001:0000192a       ??_E_Generic_error_category@std@@UAEPAXI@Z 1000292a f i alm_db_output.obj
 0001:0000194a       ??_Galm_db_output@@UAEPAXI@Z 1000294a f i alm_db_output.obj
 0001:0000194a       ??_Ealm_db_output@@UAEPAXI@Z 1000294a f i alm_db_output.obj
 0001:00001969       ??_Gconfig_plugin_base@@UAEPAXI@Z 10002969 f i alm_db_output.obj
 0001:00001969       ??_Econfig_plugin_base@@UAEPAXI@Z 10002969 f i alm_db_output.obj
 0001:00001988       ?AllocateCfgFileName@alm_db_output@@AAEXAAVQString@@0AAH@Z 10002988 f   alm_db_output.obj
 0001:00001b31       ?EditProcess@alm_db_output@@AAEXXZ 10002b31 f   alm_db_output.obj
 0001:00001b84       ?GetBncsSystem@alm_db_output@@EBEPAVDocument_BncsSystem@@XZ 10002b84 f   alm_db_output.obj
 0001:00001b8b       ?GetInstances@alm_db_output@@EBEPAVDocument_Instances@@XZ 10002b8b f   alm_db_output.obj
 0001:00001b8b       ?GetLaunch@alm_db_output@@EBEPAVDocument_Launch@@XZ 10002b8b f   alm_db_output.obj
 0001:00001b8b       ?GetDeviceDescriptions@alm_db_output@@EBEPAVDocumentSet_DeviceDescription@@XZ 10002b8b f   alm_db_output.obj
 0001:00001b8b       ?GetDevicetypes@alm_db_output@@EBEPAVDocument_Devicetypes@@XZ 10002b8b f   alm_db_output.obj
 0001:00001b8b       ?GetComplexSpecs@alm_db_output@@EBEPAVDocumentSet_ComplexSpec@@XZ 10002b8b f   alm_db_output.obj
 0001:00001b8e       ?_Copy@?$basic_string@DU?$char_traits@D@std@@V?$allocator@D@2@@std@@QAEXII@Z 10002b8e f i alm_db_output.obj
 0001:00001c85       ?_Grow@?$basic_string@DU?$char_traits@D@std@@V?$allocator@D@2@@std@@QAE_NI_N@Z 10002c85 f i alm_db_output.obj
 0001:00001ce8       ?_Inside@?$basic_string@DU?$char_traits@D@std@@V?$allocator@D@2@@std@@QAE_NPBD@Z 10002ce8 f i alm_db_output.obj
 0001:00001d23       ?_Tidy@?$basic_string@DU?$char_traits@D@std@@V?$allocator@D@2@@std@@QAEX_NI@Z 10002d23 f i alm_db_output.obj
 0001:00001d67       ?about@alm_db_output@@UAE?AVQString@@XZ 10002d67 f   alm_db_output.obj
 0001:00001db3       ?about@config_plugin_base@@UAE?AVQString@@XZ 10002db3 f i alm_db_output.obj
 0001:00001e09       ?activate@alm_db_output@@UAEX_N@Z 10002e09 f   alm_db_output.obj
 0001:00001f32       ?addProcSetting@alm_db_output@@AAEXPAVcProcess@@ABVQString@@@Z 10002f32 f   alm_db_output.obj
 0001:000020a3       ?allocateSystemName@alm_db_output@@AAEXAAVQString@@@Z 100030a3 f   alm_db_output.obj
 0001:00002171       ?apply@alm_db_output@@EAEXXZ 10003171 f   alm_db_output.obj
 0001:00002207       ?apply@config_plugin_base@@UAEXXZ 10003207 f i alm_db_output.obj
 0001:00002208       ?assign@?$basic_string@DU?$char_traits@D@std@@V?$allocator@D@2@@std@@QAEAAV12@ABV12@II@Z 10003208 f i alm_db_output.obj
 0001:0000229c       ?assign@?$basic_string@DU?$char_traits@D@std@@V?$allocator@D@2@@std@@QAEAAV12@PBDI@Z 1000329c f i alm_db_output.obj
 0001:00002315       ?begin@?$QMap@VQString@@PAVcProcess@@@@QAE?AV?$QMapIterator@VQString@@PAVcProcess@@@@XZ 10003315 f i alm_db_output.obj
 0001:00002338       ?clear@?$QDict@VQAction@@@@UAEXXZ 10003338 f i alm_db_output.obj
 0001:0000233e       ?clear@?$QMap@VQString@@PAVcProcess@@@@QAEXXZ 1000333e f i alm_db_output.obj
 0001:00002381       ?clear@?$QMapPrivate@VQString@@PAVcProcess@@@@QAEXPAU?$QMapNode@VQString@@PAVcProcess@@@@@Z 10003381 f i alm_db_output.obj
 0001:000023b9       ?clear@?$QMapPrivate@VQString@@PAVcProcess@@@@QAEXXZ 100033b9 f i alm_db_output.obj
 0001:000023e8       ?clearProcMap@alm_db_output@@AAEXXZ 100033e8 f   alm_db_output.obj
 0001:00002439       ?closeEvent@alm_db_output@@UAEXPAVQCloseEvent@@@Z 10003439 f   alm_db_output.obj
 0001:000024be       ?closeEvent@config_plugin_base@@UAEXPAVQCloseEvent@@@Z 100034be f i alm_db_output.obj
 0001:000024cc       ?contains@?$QMap@VQString@@PAVcProcess@@@@QBE_NABVQString@@@Z 100034cc f i alm_db_output.obj
 0001:000024ee       ?copy@?$QMapPrivate@VQString@@PAVcProcess@@@@QAEPAU?$QMapNode@VQString@@PAVcProcess@@@@PAU2@@Z 100034ee f i alm_db_output.obj
 0001:00002570       ?copyToClipBoard@alm_db_output@@AAEXXZ 10003570 f   alm_db_output.obj
 0001:000028cc       ?count@?$QDict@VQAction@@@@UBEIXZ 100038cc f i alm_db_output.obj
 0001:000028d0       ?count@?$QPtrList@VFileLoad@@@@UBEIXZ 100038d0 f i config_alarm_utilities:Loaders.obj
 0001:000028d0       ?count@?$QPtrList@VcOutputFile@@@@UBEIXZ 100038d0 f i alm_db_output.obj
 0001:000028d0       ?count@?$QPtrList@VcProcess@@@@UBEIXZ 100038d0 f i alm_db_output.obj
 0001:000028d0       ?count@?$QPtrList@VQPopupMenu@@@@UBEIXZ 100038d0 f i alm_db_output.obj
 0001:000028d0       ?count@?$QPtrList@VDirLoad@@@@UBEIXZ 100038d0 f i config_alarm_utilities:Loaders.obj
 0001:000028d4       ?dec@?$QMapIterator@VQString@@PAVcProcess@@@@AAEHXZ 100038d4 f i alm_db_output.obj
 0001:00002913       ?decodeSystem@alm_db_output@@AAEXABVQString@@@Z 10003913 f   alm_db_output.obj
 0001:00002c9a       ?default_error_condition@_System_error_category@std@@UBE?AVerror_condition@2@H@Z 10003c9a f i alm_db_output.obj
 0001:00002cc7       ?default_error_condition@error_category@std@@UBE?AVerror_condition@2@H@Z 10003cc7 f i alm_db_output.obj
 0001:00002cd9       ?deleteItem@?$QPtrList@VQPopupMenu@@@@EAEXPAX@Z 10003cd9 f i alm_db_output.obj
 0001:00002cd9       ?deleteItem@?$QDict@VQAction@@@@EAEXPAX@Z 10003cd9 f i alm_db_output.obj
 0001:00002cf4       ?deleteItem@?$QPtrList@VcOutputFile@@@@EAEXPAX@Z 10003cf4 f i alm_db_output.obj
 0001:00002cf4       ?deleteItem@?$QPtrList@VcProcess@@@@EAEXPAX@Z 10003cf4 f i alm_db_output.obj
 0001:00002d0e       ?deref@?$QGuardedPtr@VQPopupMenu@@@@AAEXXZ 10003d0e f i alm_db_output.obj
 0001:00002d0e       ?deref@?$QGuardedPtr@VQDockWindow@@@@AAEXXZ 10003d0e f i alm_db_output.obj
 0001:00002d23       ?detachInternal@?$QMap@VQString@@PAVcProcess@@@@AAEXXZ 10003d23 f i alm_db_output.obj
 0001:00002d5c       ?doDone@alm_db_output@@AAEXPAVresponse@@@Z 10003d5c f   alm_db_output.obj
 0001:0000319b       ?doDownload@alm_db_output@@AAEXPAVresponse@@@Z 1000419b f   alm_db_output.obj
 0001:0000323f       ?doDownloadRead@alm_db_output@@AAEXPAVresponse@@@Z 1000423f f   alm_db_output.obj
 0001:000039a1       ?doLock@alm_db_output@@AAEXPAVresponse@@@Z 100049a1 f   alm_db_output.obj
 0001:00003d14       ?doUpload@alm_db_output@@AAEXPAVresponse@@@Z 10004d14 f   alm_db_output.obj
 0001:00003d84       ?editSelectedProcs@alm_db_output@@AAEXXZ 10004d84 f   alm_db_output.obj
 0001:0000475c       ?equivalent@error_category@std@@UBE_NABVerror_code@2@H@Z 1000575c f i alm_db_output.obj
 0001:00004779       ?equivalent@error_category@std@@UBE_NHABVerror_condition@2@@Z 10005779 f i alm_db_output.obj
 0001:0000479a       ?erase@?$basic_string@DU?$char_traits@D@std@@V?$allocator@D@2@@std@@QAEAAV12@I@Z 1000579a f i alm_db_output.obj
 0001:000047c9       ?erase@?$basic_string@DU?$char_traits@D@std@@V?$allocator@D@2@@std@@QAEAAV12@II@Z 100057c9 f i alm_db_output.obj
 0001:0000484c       ?fileListContextMenu@alm_db_output@@AAEXPAVQListViewItem@@ABVQPoint@@H@Z 1000584c f   alm_db_output.obj
 0001:00004867       ?filterChange@alm_db_output@@AAEXXZ 10005867 f   alm_db_output.obj
 0001:000049ef       ?find@?$QMapPrivate@VQString@@PAVcProcess@@@@QBE?AV?$QMapConstIterator@VQString@@PAVcProcess@@@@ABVQString@@@Z 100059ef f i alm_db_output.obj
 0001:00004a4d       ?getKey@config_plugin_base@@QAE?AVQString@@XZ 10005a4d f i alm_db_output.obj
 0001:00004a6b       ?insert@?$QMap@VQString@@PAVcProcess@@@@QAE?AV?$QMapIterator@VQString@@PAVcProcess@@@@ABVQString@@ABQAVcProcess@@_N@Z 10005a6b f i alm_db_output.obj
 0001:00004ab0       ?insert@?$QMapPrivate@VQString@@PAVcProcess@@@@QAE?AV?$QMapIterator@VQString@@PAVcProcess@@@@PAUQMapNodeBase@@0ABVQString@@@Z 10005ab0 f i alm_db_output.obj
 0001:00004b57       ?insertSingle@?$QMapPrivate@VQString@@PAVcProcess@@@@QAE?AV?$QMapIterator@VQString@@PAVcProcess@@@@ABVQString@@@Z 10005b57 f i alm_db_output.obj
 0001:00004be4       ?isDirty@alm_db_output@@UAE_NXZ 10005be4 f   alm_db_output.obj
 0001:00004beb       ?isDirty@config_plugin_base@@UAE_NXZ 10005beb f i alm_db_output.obj
 0001:00004beb       ?validate@config_plugin_base@@UAE_NXZ 10005beb f i alm_db_output.obj
 0001:00004bee       ?length@?$char_traits@D@std@@SAIPBD@Z 10005bee f i alm_db_output.obj
 0001:00004c06       ?load@FileLoad_BncsSystem@alm_db_output@@UAEXABVQString@@@Z 10005c06 f   alm_db_output.obj
 0001:00004c2c       ?loadFile@alm_db_output@@AAE_NABVQString@@@Z 10005c2c f   alm_db_output.obj
 0001:00005340       ?loadProcesses@alm_db_output@@AAE_NABVQString@@@Z 10006340 f   alm_db_output.obj
 0001:00005964       ?markDirty@alm_db_output@@AAEXXZ 10006964 f   alm_db_output.obj
 0001:000059cd       ?menuDeleteFile@alm_db_output@@AAEXXZ 100069cd f   alm_db_output.obj
 0001:00005ad9       ?menuDuplicateFile@alm_db_output@@AAEXXZ 10006ad9 f   alm_db_output.obj
 0001:00005cdf       ?menuNewFile@alm_db_output@@AAEXXZ 10006cdf f   alm_db_output.obj
 0001:00005d2d       ?menuRename@alm_db_output@@AAEXXZ 10006d2d f   alm_db_output.obj
 0001:00005d47       ?menus@alm_db_output@@UAE?AVQPopupMenuList@@XZ 10006d47 f   alm_db_output.obj
 0001:00005d94       ?menus@config_plugin_base@@UAE?AVQPopupMenuList@@XZ 10006d94 f i alm_db_output.obj
 0001:00005db7       ?message@_Generic_error_category@std@@UBE?AV?$basic_string@DU?$char_traits@D@std@@V?$allocator@D@2@@2@H@Z 10006db7 f i alm_db_output.obj
 0001:00005de5       ?message@_Iostream_error_category@std@@UBE?AV?$basic_string@DU?$char_traits@D@std@@V?$allocator@D@2@@2@H@Z 10006de5 f i alm_db_output.obj
 0001:00005e16       ?message@_System_error_category@std@@UBE?AV?$basic_string@DU?$char_traits@D@std@@V?$allocator@D@2@@2@H@Z 10006e16 f i alm_db_output.obj
 0001:00005e44       ?metaObject@alm_db_output@@UBEPAVQMetaObject@@XZ 10006e44 f i alm_db_output.obj
 0001:00005e49       ?name@_Generic_error_category@std@@UBEPBDXZ 10006e49 f i alm_db_output.obj
 0001:00005e4f       ?name@_Iostream_error_category@std@@UBEPBDXZ 10006e4f f i alm_db_output.obj
 0001:00005e55       ?name@_System_error_category@std@@UBEPBDXZ 10006e55 f i alm_db_output.obj
 0001:00005e5b       ?navigate@alm_db_output@@UAEXABVQString@@0@Z 10006e5b f   alm_db_output.obj
 0001:00006203       ?navigate@config_plugin_base@@UAEXABVQString@@0@Z 10007203 f i alm_db_output.obj
 0001:00006206       ?newFile@alm_db_output@@AAEXABVQString@@@Z 10007206 f   alm_db_output.obj
 0001:0000650a       ?pasteAllProcs@alm_db_output@@AAEXXZ 1000750a f   alm_db_output.obj
 0001:00006512       ?pasteOptions@alm_db_output@@AAEXXZ 10007512 f   alm_db_output.obj
 0001:000065e9       ?pasteSelectedProcs@alm_db_output@@AAEX_N@Z 100075e9 f   alm_db_output.obj
 0001:00006a3f       ?procSelection@alm_db_output@@AAEXXZ 10007a3f f   alm_db_output.obj
 0001:00006b99       ?renameModule@alm_db_output@@AAEXPAVQListViewItem@@HABVQString@@@Z 10007b99 f   alm_db_output.obj
 0001:00006d0b       ?reply@alm_db_output@@UAEXPAVresponse@@@Z 10007d0b f   alm_db_output.obj
 0001:00006ddf       ?resizeEvent@alm_db_output@@UAEXPAVQResizeEvent@@@Z 10007ddf f   alm_db_output.obj
 0001:00006e14       ?saveFile@alm_db_output@@AAE_NPAVcOutputFile@@@Z 10007e14 f   alm_db_output.obj
 0001:00007c04       ?selectFile@alm_db_output@@AAEXPAVQListViewItem@@@Z 10008c04 f   alm_db_output.obj
 0001:00007f03       ?selectProcess@alm_db_output@@AAEXABVQString@@@Z 10008f03 f   alm_db_output.obj
 0001:00007fda       ?selectSystem@alm_db_output@@AAEXABVQString@@@Z 10008fda f   alm_db_output.obj
 0001:00008437       ?sendCommand@alm_db_output@@UAEXABVQString@@0@Z 10009437 f   alm_db_output.obj
 0001:00008478       ?templateProcess@alm_db_output@@AAEXXZ 10009478 f   alm_db_output.obj
 0001:00008b73       ?toolbars@alm_db_output@@UAE?AVQDockWindowList@@XZ 10009b73 f   alm_db_output.obj
 0001:00008bce       ?toolbars@config_plugin_base@@UAE?AVQDockWindowList@@XZ 10009bce f i alm_db_output.obj
 0001:00008bf4       ?updateFileList@alm_db_output@@AAEXXZ 10009bf4 f   alm_db_output.obj
 0001:000097eb       ?updateList@alm_db_output@@AAEXXZ 1000a7eb f   alm_db_output.obj
 0001:000099b9       ?useAltId@alm_db_output@@AAE?AVQString@@V2@ABV2@_N@Z 1000a9b9 f   alm_db_output.obj
 0001:00009a55       ??0cOutputFile@@QAE@XZ     1000aa55 f   cOutputFile.obj
 0001:00009aa1       ??1cOutputFile@@UAE@XZ     1000aaa1 f   cOutputFile.obj
 0001:00009ae8       ??_GcOutputFile@@UAEPAXI@Z 1000aae8 f i cOutputFile.obj
 0001:00009ae8       ??_EcOutputFile@@UAEPAXI@Z 1000aae8 f i cOutputFile.obj
 0001:00009b07       ??0cProcess@@QAE@VQString@@@Z 1000ab07 f   cProcess.obj
 0001:00009bbf       ??1cProcess@@UAE@XZ        1000abbf f   cProcess.obj
 0001:00009c54       ??_GcProcess@@UAEPAXI@Z    1000ac54 f i cProcess.obj
 0001:00009c54       ??_EcProcess@@UAEPAXI@Z    1000ac54 f i cProcess.obj
 0001:00009c73       ??0dbConnection@@QAE@XZ    1000ac73 f   DBCONNECTION.obj
 0001:00009d58       ??1dbConnection@@UAE@XZ    1000ad58 f   DBCONNECTION.obj
 0001:00009ddf       ??_EdbConnection@@UAEPAXI@Z 1000addf f i DBCONNECTION.obj
 0001:00009ddf       ??_GdbConnection@@UAEPAXI@Z 1000addf f i DBCONNECTION.obj
 0001:00009dfe       ?close@dbConnection@@QAEXXZ 1000adfe f   DBCONNECTION.obj
 0001:00009e07       ?connected@dbConnection@@QBE_NXZ 1000ae07 f   DBCONNECTION.obj
 0001:00009e10       ?getDbase@dbConnection@@QAEPAVQSqlDatabase@@XZ 1000ae10 f   DBCONNECTION.obj
 0001:00009e7e       ?lastError@dbConnection@@QAE?AVQString@@XZ 1000ae7e f   DBCONNECTION.obj
 0001:0000a17e       ?run@dbConnection@@UAEXXZ  1000b17e f   DBCONNECTION.obj
 0001:0000a3fe       ??0dialog@@QAE@PAVIGetDocuments@@PAVQWidget@@PBDI@Z 1000b3fe f   dialogimpl.obj
 0001:0000b1d3       ??1dialog@@UAE@XZ          1000c1d3 f   dialogimpl.obj
 0001:0000b881       ??_EQSqlCursor@@W7AEPAXI@Z 1000c881 f i dialogimpl.obj
 0001:0000b889       ??_Edialog@@WCI@AEPAXI@Z   1000c889 f i dialogimpl.obj
 0001:0000b891       ??_GQSqlCursor@@UAEPAXI@Z  1000c891 f i dialogimpl.obj
 0001:0000b891       ??_EQSqlCursor@@UAEPAXI@Z  1000c891 f i dialogimpl.obj
 0001:0000b8b1       ??_EQTimer@@UAEPAXI@Z      1000c8b1 f i dialogimpl.obj
 0001:0000b8b1       ??_GQTimer@@UAEPAXI@Z      1000c8b1 f i dialogimpl.obj
 0001:0000b8d1       ??_Edialog@@UAEPAXI@Z      1000c8d1 f i dialogimpl.obj
 0001:0000b8d1       ??_Gdialog@@UAEPAXI@Z      1000c8d1 f i dialogimpl.obj
 0001:0000b8f0       ?clearAllLogs@dialog@@QAEXXZ 1000c8f0 f   dialogimpl.obj
 0001:0000b988       ?clearAllProcesses@dialog@@QAEXXZ 1000c988 f   dialogimpl.obj
 0001:0000ba20       ?clearAllText@dialog@@QAEXXZ 1000ca20 f   dialogimpl.obj
 0001:0000bb7c       ?clearLogsBefore@dialog@@QAEXXZ 1000cb7c f   dialogimpl.obj
 0001:0000bc95       ?clearProcess@dialog@@QAEXXZ 1000cc95 f   dialogimpl.obj
 0001:0000bd0b       ?clearProcessesBefore@dialog@@QAEXXZ 1000cd0b f   dialogimpl.obj
 0001:0000be24       ?clearSystem@dialog@@QAEXXZ 1000ce24 f   dialogimpl.obj
 0001:0000bf0a       ?connectDb@dialog@@AAEPAVQSqlDatabase@@XZ 1000cf0a f   dialogimpl.obj
 0001:0000c070       ?copyData@dialog@@QAEXXZ   1000d070 f   dialogimpl.obj
 0001:0000c199       ?createNewLogTable@dialog@@QAEXXZ 1000d199 f   dialogimpl.obj
 0001:0000c5ba       ?createNewProcTable@dialog@@QAEXXZ 1000d5ba f   dialogimpl.obj
 0001:0000c999       ?dbDriverChanged@dialog@@QAEXABVQString@@@Z 1000d999 f   dialogimpl.obj
 0001:0000ca5c       ?dbDriverChanged_reserve@dialog@@QAEXABVQString@@@Z 1000da5c f   dialogimpl.obj
 0001:0000cb1f       ?dbEditStart@dialog@@QAEXXZ 1000db1f f   dialogimpl.obj
 0001:0000ccbe       ?dbStartConnect@dialog@@AAEXXZ 1000dcbe f   dialogimpl.obj
 0001:0000cfb3       ?dbToolUpdate@dialog@@QAEXXZ 1000dfb3 f   dialogimpl.obj
 0001:0000d28f       ?dbToolsEnd@dialog@@QAEXXZ 1000e28f f   dialogimpl.obj
 0001:0000d2ba       ?dbToolsStart@dialog@@QAEXXZ 1000e2ba f   dialogimpl.obj
 0001:0000d3ed       ?defaultText@dialog@@AAE?AVQString@@W4AlarmStates@Alarms@@@Z 1000e3ed f   dialogimpl.obj
 0001:0000d60d       ?fillDataTable@dialog@@QAEXXZ 1000e60d f   dialogimpl.obj
 0001:0000d72c       ?fillDataTableEdit@dialog@@QAEXH@Z 1000e72c f   dialogimpl.obj
 0001:0000d755       ?fillDataTableTools@dialog@@QAEXH@Z 1000e755 f   dialogimpl.obj
 0001:0000d77e       ?getSep@dialog@@QAE?AVQString@@H@Z 1000e77e f   dialogimpl.obj
 0001:0000d8a1       ?itemChanged@dialog@@QAEXABVQString@@@Z 1000e8a1 f   dialogimpl.obj
 0001:0000da37       ?itemChanged@dialog@@QAEXH@Z 1000ea37 f   dialogimpl.obj
 0001:0000da77       ?levelChanged@dialog@@QAEXH@Z 1000ea77 f   dialogimpl.obj
 0001:0000dae2       ?metaObject@dialog@@UBEPAVQMetaObject@@XZ 1000eae2 f i dialogimpl.obj
 0001:0000dae7       ?pasteData@dialog@@QAEXXZ  1000eae7 f   dialogimpl.obj
 0001:0000dfca       ?resetDefaults@dialog@@QAEXXZ 1000efca f   dialogimpl.obj
 0001:0000e13c       ?saveProcess@dialog@@QAE_NPAVcProcess@@@Z 1000f13c f   dialogimpl.obj
 0001:0000e2c5       ?setAckDefaultText@dialog@@QAEXXZ 1000f2c5 f   dialogimpl.obj
 0001:0000e331       ?setAllDefaultText@dialog@@QAEXXZ 1000f331 f   dialogimpl.obj
 0001:0000e482       ?setBncsSystemValues@dialog@@QAEXXZ 1000f482 f   dialogimpl.obj
 0001:0000e4b5       ?setFailDefaultText@dialog@@QAEXXZ 1000f4b5 f   dialogimpl.obj
 0001:0000e521       ?setGroupDefaultText@dialog@@QAEXXZ 1000f521 f   dialogimpl.obj
 0001:0000e5a7       ?setIgnoreDefaultText@dialog@@QAEXXZ 1000f5a7 f   dialogimpl.obj
 0001:0000e613       ?setLatchedDefaultText@dialog@@QAEXXZ 1000f613 f   dialogimpl.obj
 0001:0000e67f       ?setOkDefaultText@dialog@@QAEXXZ 1000f67f f   dialogimpl.obj
 0001:0000e6eb       ?setProcess@dialog@@QAE_NPAVcProcess@@@Z 1000f6eb f   dialogimpl.obj
 0001:0000e7f8       ?setUnknownDefaultText@dialog@@QAEXXZ 1000f7f8 f   dialogimpl.obj
 0001:0000e864       ?showingWidget@dialog@@QAEXPAVQWidget@@@Z 1000f864 f   dialogimpl.obj
 0001:0000e8be       ?useAltId@dialog@@AAE?AVQString@@V2@0_N@Z 1000f8be f   dialogimpl.obj
 0001:0000e9be       ?value@QSqlCursor@@W7BE?AVQVariant@@H@Z 1000f9be f i dialogimpl.obj
 0001:0000e9c7       ??0manage_temp@@QAE@QAV?$QMap@VQString@@PAVcProcess@@@@PAVdialog@@@Z 1000f9c7 f   manage_tempimpl.obj
 0001:0000ecfc       ??1manage_temp@@UAE@XZ     1000fcfc f   manage_tempimpl.obj
 0001:0000eeb4       ??_Emanage_temp@@WCI@AEPAXI@Z 1000feb4 f i manage_tempimpl.obj
 0001:0000eebc       ??_GQCheckTableItem@@UAEPAXI@Z 1000febc f i manage_tempimpl.obj
 0001:0000eebc       ??_EQCheckTableItem@@UAEPAXI@Z 1000febc f i manage_tempimpl.obj
 0001:0000eedc       ??_Emanage_temp@@UAEPAXI@Z 1000fedc f i manage_tempimpl.obj
 0001:0000eedc       ??_Gmanage_temp@@UAEPAXI@Z 1000fedc f i manage_tempimpl.obj
 0001:0000eefb       ?clearAllParamsText@manage_temp@@QAEXXZ 1000fefb f   manage_tempimpl.obj
 0001:0000ef92       ?clearAllText@manage_temp@@QAEXXZ 1000ff92 f   manage_tempimpl.obj
 0001:0000f13b       ?defaultText@manage_temp@@AAE?AVQString@@W4AlarmStates@Alarms@@@Z 1001013b f   manage_tempimpl.obj
 0001:0000f460       ?deselectAllInstances@manage_temp@@QAEXXZ 10010460 f   manage_tempimpl.obj
 0001:0000f4a8       ?deselectSelectedInstances@manage_temp@@QAEXXZ 100104a8 f   manage_tempimpl.obj
 0001:0000f513       ?inc@?$QMapConstIterator@VQString@@PAVcProcess@@@@AAEHXZ 10010513 f i manage_tempimpl.obj
 0001:0000f513       ?inc@?$QMapIterator@VQString@@PAVcProcess@@@@AAEHXZ 10010513 f i alm_db_output.obj
 0001:0000f513       ?inc@?$QMapIterator@VQString@@H@@AAEHXZ 10010513 f i alm_db_output.obj
 0001:0000f544       ?itemChanged@manage_temp@@QAEXXZ 10010544 f   manage_tempimpl.obj
 0001:0000f716       ?metaObject@manage_temp@@UBEPAVQMetaObject@@XZ 10010716 f i manage_tempimpl.obj
 0001:0000f71b       ?prefixChanged@manage_temp@@QAEXABVQString@@@Z 1001071b f   manage_tempimpl.obj
 0001:0000fcf9       ?selectAllInstances@manage_temp@@QAEXXZ 10010cf9 f   manage_tempimpl.obj
 0001:0000fd41       ?selectProcess@manage_temp@@QAEXPAVQListViewItem@@@Z 10010d41 f   manage_tempimpl.obj
 0001:0001005b       ?selectSelectedInstances@manage_temp@@QAEXXZ 1001105b f   manage_tempimpl.obj
 0001:000100c6       ?setAckDefaultText@manage_temp@@QAEXXZ 100110c6 f   manage_tempimpl.obj
 0001:00010105       ?setAllDefaultText@manage_temp@@QAEXXZ 10011105 f   manage_tempimpl.obj
 0001:00010268       ?setAllParamsDefaultText@manage_temp@@QAEXXZ 10011268 f   manage_tempimpl.obj
 0001:000102fe       ?setDefaultGroup@manage_temp@@QAEXVQString@@@Z 100112fe f   manage_tempimpl.obj
 0001:00010333       ?setDeviceDefaultText@manage_temp@@QAEXXZ 10011333 f   manage_tempimpl.obj
 0001:000103cc       ?setFailDefaultText@manage_temp@@QAEXXZ 100113cc f   manage_tempimpl.obj
 0001:0001040b       ?setGroupDefaultText@manage_temp@@QAEXXZ 1001140b f   manage_tempimpl.obj
 0001:00010425       ?setIgnoreDefaultText@manage_temp@@QAEXXZ 10011425 f   manage_tempimpl.obj
 0001:00010464       ?setLatchedDefaultText@manage_temp@@QAEXXZ 10011464 f   manage_tempimpl.obj
 0001:000104a3       ?setLevelDefaultText@manage_temp@@QAEXXZ 100114a3 f   manage_tempimpl.obj
 0001:000104d7       ?setOkDefaultText@manage_temp@@QAEXXZ 100114d7 f   manage_tempimpl.obj
 0001:00010516       ?setProcess@manage_temp@@AAEXPAVQListViewItem@@@Z 10011516 f   manage_tempimpl.obj
 0001:00010695       ?setUnknownDefaultText@manage_temp@@QAEXXZ 10011695 f   manage_tempimpl.obj
 0001:000106d4       ?className@setDefaultsBase@@UBEPBDXZ 100116d4 f   moc_setdefaults.obj
 0001:000106da       ?qt_cast@setDefaultsBase@@UAEPAXPBD@Z 100116da f   moc_setdefaults.obj
 0001:00010708       ?qt_invoke@setDefaultsBase@@UAE_NHPAUQUObject@@@Z 10011708 f   moc_setdefaults.obj
 0001:0001073a       ?staticMetaObject@setDefaultsBase@@SAPAVQMetaObject@@XZ 1001173a f   moc_setdefaults.obj
 0001:00010784       ?tr@setDefaultsBase@@SA?AVQString@@PBD0@Z 10011784 f   moc_setdefaults.obj
 0001:000107c7       ?className@setDefaults@@UBEPBDXZ 100117c7 f   moc_setdefaultsimpl.obj
 0001:000107cd       ?qt_cast@setDefaults@@UAEPAXPBD@Z 100117cd f   moc_setdefaultsimpl.obj
 0001:000107fa       ?qt_invoke@setDefaults@@UAE_NHPAUQUObject@@@Z 100117fa f   moc_setdefaultsimpl.obj
 0001:00010803       ?staticMetaObject@setDefaults@@SAPAVQMetaObject@@XZ 10011803 f   moc_setdefaultsimpl.obj
 0001:00010847       ??_Eplugindesc@@UAEPAXI@Z  10011847 f i plugindesc.obj
 0001:00010847       ??_Gconfig_plugin_desc_base@@UAEPAXI@Z 10011847 f i plugindesc.obj
 0001:00010847       ??_Gplugindesc@@UAEPAXI@Z  10011847 f i plugindesc.obj
 0001:00010847       ??_Econfig_plugin_desc_base@@UAEPAXI@Z 10011847 f i plugindesc.obj
 0001:00010867       ?create@plugindesc@@UAEPAVconfig_plugin_base@@ABVQString@@00@Z 10011867 f   plugindesc.obj
 0001:000108a2       ?keys@plugindesc@@UAE?AVQStringList@@ABVQString@@0@Z 100118a2 f   plugindesc.obj
 0001:000108fd       ?pixmap@plugindesc@@UAE?AVQPixmap@@ABVQString@@@Z 100118fd f   plugindesc.obj
 0001:0001091c       _load_bncs_config_plugin_desc 1001191c f   plugindesc.obj
 0001:00010932       ??0processList@@QAE@XZ     10011932 f   processList.obj
 0001:00010950       ??1processList@@UAE@XZ     10011950 f   processList.obj
 0001:0001095f       ??_GprocessList@@UAEPAXI@Z 1001195f f i processList.obj
 0001:0001095f       ??_EprocessList@@UAEPAXI@Z 1001195f f i processList.obj
 0001:00010984       ??0setDefaultsBase@@QAE@PAVQWidget@@PBD_NI@Z 10011984 f   setdefaults.obj
 0001:000121f1       ??1setDefaultsBase@@UAE@XZ 100131f1 f   setdefaults.obj
 0001:00012204       ??_EQComboBox@@WCI@AEPAXI@Z 10013204 f i setdefaults.obj
 0001:0001220c       ??_EQGridLayout@@WCI@AEPAXI@Z 1001320c f i setdefaults.obj
 0001:00012214       ??_EQGroupBox@@WCI@AEPAXI@Z 10013214 f i setdefaults.obj
 0001:0001221c       ??_EQHBoxLayout@@WCI@AEPAXI@Z 1001321c f i setdefaults.obj
 0001:00012224       ??_EQLabel@@WCI@AEPAXI@Z   10013224 f i setdefaults.obj
 0001:0001222c       ??_EQLineEdit@@WCI@AEPAXI@Z 1001322c f i setdefaults.obj
 0001:00012234       ??_EQPushButton@@WCI@AEPAXI@Z 10013234 f i setdefaults.obj
 0001:0001223c       ??_EQVBoxLayout@@WCI@AEPAXI@Z 1001323c f i setdefaults.obj
 0001:00012244       ??_EsetDefaultsBase@@WCI@AEPAXI@Z 10013244 f i setdefaults.obj
 0001:0001224c       ??_GQComboBox@@UAEPAXI@Z   1001324c f i setdefaults.obj
 0001:0001224c       ??_EQComboBox@@UAEPAXI@Z   1001324c f i setdefaults.obj
 0001:0001226c       ??_GQGridLayout@@UAEPAXI@Z 1001326c f i setdefaults.obj
 0001:0001226c       ??_EQGridLayout@@UAEPAXI@Z 1001326c f i setdefaults.obj
 0001:0001228c       ??_GQGroupBox@@UAEPAXI@Z   1001328c f i setdefaults.obj
 0001:0001228c       ??_EQGroupBox@@UAEPAXI@Z   1001328c f i setdefaults.obj
 0001:000122ac       ??_EQHBoxLayout@@UAEPAXI@Z 100132ac f i setdefaults.obj
 0001:000122ac       ??_GQHBoxLayout@@UAEPAXI@Z 100132ac f i setdefaults.obj
 0001:000122cc       ??_GQLabel@@UAEPAXI@Z      100132cc f i setdefaults.obj
 0001:000122cc       ??_EQLabel@@UAEPAXI@Z      100132cc f i setdefaults.obj
 0001:000122ec       ??_EQLineEdit@@UAEPAXI@Z   100132ec f i setdefaults.obj
 0001:000122ec       ??_GQLineEdit@@UAEPAXI@Z   100132ec f i setdefaults.obj
 0001:0001230c       ??_EQPushButton@@UAEPAXI@Z 1001330c f i setdefaults.obj
 0001:0001230c       ??_GQPushButton@@UAEPAXI@Z 1001330c f i setdefaults.obj
 0001:0001232c       ??_EQSpacerItem@@UAEPAXI@Z 1001332c f i setdefaults.obj
 0001:0001232c       ??_GQSpacerItem@@UAEPAXI@Z 1001332c f i setdefaults.obj
 0001:0001234c       ??_EQVBoxLayout@@UAEPAXI@Z 1001334c f i setdefaults.obj
 0001:0001234c       ??_GQVBoxLayout@@UAEPAXI@Z 1001334c f i setdefaults.obj
 0001:0001236c       ??_GsetDefaultsBase@@UAEPAXI@Z 1001336c f i setdefaults.obj
 0001:0001236c       ??_EsetDefaultsBase@@UAEPAXI@Z 1001336c f i setdefaults.obj
 0001:0001238b       ?languageChange@setDefaultsBase@@MAEXXZ 1001338b f   setdefaults.obj
 0001:00012cdc       ?metaObject@setDefaultsBase@@UBEPAVQMetaObject@@XZ 10013cdc f i setdefaults.obj
 0001:00012ce1       ??0setDefaults@@QAE@PAVQWidget@@PBD_NI@Z 10013ce1 f   setdefaultsimpl.obj
 0001:00012e20       ??1setDefaults@@UAE@XZ     10013e20 f   setdefaultsimpl.obj
 0001:00012e32       ??_EsetDefaults@@WCI@AEPAXI@Z 10013e32 f i setdefaultsimpl.obj
 0001:00012e3a       ??_EsetDefaults@@UAEPAXI@Z 10013e3a f i setdefaultsimpl.obj
 0001:00012e3a       ??_GsetDefaults@@UAEPAXI@Z 10013e3a f i setdefaultsimpl.obj
 0001:00012e59       ?metaObject@setDefaults@@UBEPAVQMetaObject@@XZ 10013e59 f i setdefaultsimpl.obj
 0001:00012e5e       ??0dialogBase@@QAE@PAVQWidget@@PBDI@Z 10013e5e f   dialog.obj
 0001:000176b8       ??1dialogBase@@UAE@XZ      100186b8 f   dialog.obj
 0001:000176cb       ??_EQButtonGroup@@WCI@AEPAXI@Z 100186cb f i dialog.obj
 0001:000176d3       ??_EQDataTable@@WCI@AEPAXI@Z 100186d3 f i dialog.obj
 0001:000176db       ??_EQDateEdit@@WCI@AEPAXI@Z 100186db f i dialog.obj
 0001:000176e3       ??_EQRadioButton@@WCI@AEPAXI@Z 100186e3 f i dialog.obj
 0001:000176e3       ??_EQCheckBox@@WCI@AEPAXI@Z 100186e3 f i setdefaults.obj
 0001:000176eb       ??_EQSpinBox@@WCI@AEPAXI@Z 100186eb f i dialog.obj
 0001:000176f3       ??_EQSpinBox@@WGM@AEPAXI@Z 100186f3 f i dialog.obj
 0001:000176fb       ??_EQSplitter@@WCI@AEPAXI@Z 100186fb f i dialog.obj
 0001:00017703       ??_EdialogBase@@WCI@AEPAXI@Z 10018703 f i dialog.obj
 0001:0001770b       ??_GQButtonGroup@@UAEPAXI@Z 1001870b f i dialog.obj
 0001:0001770b       ??_EQButtonGroup@@UAEPAXI@Z 1001870b f i dialog.obj
 0001:0001772b       ??_EQDataTable@@UAEPAXI@Z  1001872b f i dialog.obj
 0001:0001772b       ??_GQDataTable@@UAEPAXI@Z  1001872b f i dialog.obj
 0001:0001774b       ??_GQDateEdit@@UAEPAXI@Z   1001874b f i dialog.obj
 0001:0001774b       ??_EQDateEdit@@UAEPAXI@Z   1001874b f i dialog.obj
 0001:0001776b       ??_GQCheckBox@@UAEPAXI@Z   1001876b f i setdefaults.obj
 0001:0001776b       ??_EQRadioButton@@UAEPAXI@Z 1001876b f i dialog.obj
 0001:0001776b       ??_GQRadioButton@@UAEPAXI@Z 1001876b f i dialog.obj
 0001:0001776b       ??_EQCheckBox@@UAEPAXI@Z   1001876b f i setdefaults.obj
 0001:0001778b       ??_EQSpinBox@@UAEPAXI@Z    1001878b f i dialog.obj
 0001:0001778b       ??_GQSpinBox@@UAEPAXI@Z    1001878b f i dialog.obj
 0001:000177ab       ??_EQSplitter@@UAEPAXI@Z   100187ab f i dialog.obj
 0001:000177ab       ??_GQSplitter@@UAEPAXI@Z   100187ab f i dialog.obj
 0001:000177cb       ??_GdialogBase@@UAEPAXI@Z  100187cb f i dialog.obj
 0001:000177cb       ??_EdialogBase@@UAEPAXI@Z  100187cb f i dialog.obj
 0001:000177ea       ?languageChange@dialogBase@@MAEXXZ 100187ea f   dialog.obj
 0001:000194a6       ?metaObject@dialogBase@@UBEPAVQMetaObject@@XZ 1001a4a6 f i dialog.obj
 0001:000194ab       ?polish@dialogBase@@UAEXXZ 1001a4ab f   dialog.obj
 0001:000194b1       ??0manage_tempBase@@QAE@PAVQWidget@@PBD_NI@Z 1001a4b1 f   manage_temp.obj
 0001:0001b0a0       ??1manage_tempBase@@UAE@XZ 1001c0a0 f   manage_temp.obj
 0001:0001b0b3       ??_EQTable@@WCI@AEPAXI@Z   1001c0b3 f i manage_temp.obj
 0001:0001b0bb       ??_Emanage_tempBase@@WCI@AEPAXI@Z 1001c0bb f i manage_temp.obj
 0001:0001b0c3       ??_EQTable@@UAEPAXI@Z      1001c0c3 f i manage_temp.obj
 0001:0001b0c3       ??_GQTable@@UAEPAXI@Z      1001c0c3 f i manage_temp.obj
 0001:0001b0e3       ??_Gmanage_tempBase@@UAEPAXI@Z 1001c0e3 f i manage_temp.obj
 0001:0001b0e3       ??_Emanage_tempBase@@UAEPAXI@Z 1001c0e3 f i manage_temp.obj
 0001:0001b102       ?languageChange@manage_tempBase@@MAEXXZ 1001c102 f   manage_temp.obj
 0001:0001bd06       ?metaObject@manage_tempBase@@UBEPAVQMetaObject@@XZ 1001cd06 f i manage_temp.obj
 0001:0001bd0b       ?className@alm_db_output@@UBEPBDXZ 1001cd0b f   moc_alm_db_output.obj
 0001:0001bd11       ?command@alm_db_output@@IAEXVQString@@0@Z 1001cd11 f   moc_alm_db_output.obj
 0001:0001bdd1       ?qt_cast@alm_db_output@@UAEPAXPBD@Z 1001cdd1 f   moc_alm_db_output.obj
 0001:0001be3d       ?qt_emit@alm_db_output@@UAE_NHPAUQUObject@@@Z 1001ce3d f   moc_alm_db_output.obj
 0001:0001bea4       ?qt_invoke@alm_db_output@@UAE_NHPAUQUObject@@@Z 1001cea4 f   moc_alm_db_output.obj
 0001:0001c024       ?qt_property@dialogBase@@UAE_NHHPAVQVariant@@@Z 1001d024 f   moc_dialog.obj
 0001:0001c024       ?qt_property@alm_db_output@@UAE_NHHPAVQVariant@@@Z 1001d024 f   moc_alm_db_output.obj
 0001:0001c02e       ?staticMetaObject@alm_db_output@@SAPAVQMetaObject@@XZ 1001d02e f   moc_alm_db_output.obj
 0001:0001c21b       ?className@dialogBase@@UBEPBDXZ 1001d21b f   moc_dialog.obj
 0001:0001c221       ?qt_cast@dialogBase@@UAEPAXPBD@Z 1001d221 f   moc_dialog.obj
 0001:0001c24f       ?qt_emit@dialogBase@@UAE_NHPAUQUObject@@@Z 1001d24f f   moc_dialog.obj
 0001:0001c259       ?qt_invoke@dialogBase@@UAE_NHPAUQUObject@@@Z 1001d259 f   moc_dialog.obj
 0001:0001c29d       ?staticMetaObject@dialogBase@@SAPAVQMetaObject@@XZ 1001d29d f   moc_dialog.obj
 0001:0001c2e7       ?tr@dialogBase@@SA?AVQString@@PBD0@Z 1001d2e7 f   moc_dialog.obj
 0001:0001c32a       ?className@dialog@@UBEPBDXZ 1001d32a f   moc_dialogimpl.obj
 0001:0001c330       ?itemsChanged@dialog@@IAEXXZ 1001d330 f   moc_dialogimpl.obj
 0001:0001c345       ?qt_cast@dialog@@UAEPAXPBD@Z 1001d345 f   moc_dialogimpl.obj
 0001:0001c372       ?qt_emit@dialog@@UAE_NHPAUQUObject@@@Z 1001d372 f   moc_dialogimpl.obj
 0001:0001c3a0       ?qt_invoke@dialog@@UAE_NHPAUQUObject@@@Z 1001d3a0 f   moc_dialogimpl.obj
 0001:0001c600       ?qt_property@dialog@@UAE_NHHPAVQVariant@@@Z 1001d600 f   moc_dialogimpl.obj
 0001:0001c609       ?staticMetaObject@dialog@@SAPAVQMetaObject@@XZ 1001d609 f   moc_dialogimpl.obj
 0001:0001c77a       ?className@manage_tempBase@@UBEPBDXZ 1001d77a f   moc_manage_temp.obj
 0001:0001c780       ?qt_cast@manage_tempBase@@UAEPAXPBD@Z 1001d780 f   moc_manage_temp.obj
 0001:0001c7ae       ?qt_emit@manage_tempBase@@UAE_NHPAUQUObject@@@Z 1001d7ae f   moc_manage_temp.obj
 0001:0001c7ae       ?qt_emit@setDefaultsBase@@UAE_NHPAUQUObject@@@Z 1001d7ae f   moc_setdefaults.obj
 0001:0001c7b8       ?qt_invoke@manage_tempBase@@UAE_NHPAUQUObject@@@Z 1001d7b8 f   moc_manage_temp.obj
 0001:0001c7ea       ?qt_property@manage_tempBase@@UAE_NHHPAVQVariant@@@Z 1001d7ea f   moc_manage_temp.obj
 0001:0001c7ea       ?qt_property@setDefaultsBase@@UAE_NHHPAVQVariant@@@Z 1001d7ea f   moc_setdefaults.obj
 0001:0001c7f4       ?staticMetaObject@manage_tempBase@@SAPAVQMetaObject@@XZ 1001d7f4 f   moc_manage_temp.obj
 0001:0001c83e       ?tr@manage_tempBase@@SA?AVQString@@PBD0@Z 1001d83e f   moc_manage_temp.obj
 0001:0001c881       ?className@manage_temp@@UBEPBDXZ 1001d881 f   moc_manage_tempimpl.obj
 0001:0001c887       ?qt_cast@manage_temp@@UAEPAXPBD@Z 1001d887 f   moc_manage_tempimpl.obj
 0001:0001c8b4       ?qt_emit@setDefaults@@UAE_NHPAUQUObject@@@Z 1001d8b4 f   moc_setdefaultsimpl.obj
 0001:0001c8b4       ?qt_emit@manage_temp@@UAE_NHPAUQUObject@@@Z 1001d8b4 f   moc_manage_tempimpl.obj
 0001:0001c8bd       ?qt_invoke@manage_temp@@UAE_NHPAUQUObject@@@Z 1001d8bd f   moc_manage_tempimpl.obj
 0001:0001ca2d       ?qt_property@setDefaults@@UAE_NHHPAVQVariant@@@Z 1001da2d f   moc_setdefaultsimpl.obj
 0001:0001ca2d       ?qt_property@manage_temp@@UAE_NHHPAVQVariant@@@Z 1001da2d f   moc_manage_tempimpl.obj
 0001:0001ca36       ?staticMetaObject@manage_temp@@SAPAVQMetaObject@@XZ 1001da36 f   moc_manage_tempimpl.obj
 0001:0001cb04       ?setName@QWidget@@UAEXPBD@Z 1001db04 f   qt-mt323:qt-mt323.dll
 0001:0001cb0a       ?open@QFile@@UAE_NH@Z      1001db0a f   qt-mt323:qt-mt323.dll
 0001:0001cb10       ?close@QFile@@UAEXXZ       1001db10 f   qt-mt323:qt-mt323.dll
 0001:0001cb16       ?acceptDrop@QListViewItem@@UBE_NPBVQMimeSource@@@Z 1001db16 f   qt-mt323:qt-mt323.dll
 0001:0001cb1c       ?activate@QListViewItem@@MAEXXZ 1001db1c f   qt-mt323:qt-mt323.dll
 0001:0001cb22       ?activateItemAt@QPopupMenu@@UAEXH@Z 1001db22 f   qt-mt323:qt-mt323.dll
 0001:0001cb28       ?addChild@QScrollView@@UAEXPAVQWidget@@HH@Z 1001db28 f   qt-mt323:qt-mt323.dll
 0001:0001cb2e       ?addColumn@QListView@@UAEHABVQIconSet@@ABVQString@@H@Z 1001db2e f   qt-mt323:qt-mt323.dll
 0001:0001cb34       ?addColumn@QListView@@UAEHABVQString@@H@Z 1001db34 f   qt-mt323:qt-mt323.dll
 0001:0001cb3a       ?addItem@QBoxLayout@@UAEXPAVQLayoutItem@@@Z 1001db3a f   qt-mt323:qt-mt323.dll
 0001:0001cb40       ?addTab@QTabWidget@@UAEXPAVQWidget@@ABVQIconSet@@ABVQString@@@Z 1001db40 f   qt-mt323:qt-mt323.dll
 0001:0001cb46       ?addTab@QTabWidget@@UAEXPAVQWidget@@ABVQString@@@Z 1001db46 f   qt-mt323:qt-mt323.dll
 0001:0001cb4c       ?addTab@QTabWidget@@UAEXPAVQWidget@@PAVQTab@@@Z 1001db4c f   qt-mt323:qt-mt323.dll
 0001:0001cb52       ?addTo@QAction@@UAE_NPAVQWidget@@@Z 1001db52 f   qt-mt323:qt-mt323.dll
 0001:0001cb58       ?addedTo@QAction@@MAEXHPAVQPopupMenu@@@Z 1001db58 f   qt-mt323:qt-mt323.dll
 0001:0001cb5e       ?addedTo@QAction@@MAEXPAVQWidget@@0@Z 1001db5e f   qt-mt323:qt-mt323.dll
 0001:0001cb64       ?adjustSize@QWidget@@UAEXXZ 1001db64 f   qt-mt323:qt-mt323.dll
 0001:0001cb6a       ?at@QFile@@UAE_NK@Z        1001db6a f   qt-mt323:qt-mt323.dll
 0001:0001cb70       ?at@QFile@@UBEKXZ          1001db70 f   qt-mt323:qt-mt323.dll
 0001:0001cb76       ?atEnd@QFile@@UBE_NXZ      1001db76 f   qt-mt323:qt-mt323.dll
 0001:0001cb7c       ?cancelRename@QListViewItem@@MAEXH@Z 1001db7c f   qt-mt323:qt-mt323.dll
 0001:0001cb82       ?checkConnectArgs@QObject@@MAE_NPBDPBV1@0@Z 1001db82 f   qt-mt323:qt-mt323.dll
 0001:0001cb88       ?childEvent@QLayout@@MAEXPAVQChildEvent@@@Z 1001db88 f   qt-mt323:qt-mt323.dll
 0001:0001cb8e       ?childEvent@QObject@@MAEXPAVQChildEvent@@@Z 1001db8e f   qt-mt323:qt-mt323.dll
 0001:0001cb94       ?className@QAction@@UBEPBDXZ 1001db94 f   qt-mt323:qt-mt323.dll
 0001:0001cb9a       ?className@QBoxLayout@@UBEPBDXZ 1001db9a f   qt-mt323:qt-mt323.dll
 0001:0001cba0       ?className@QDockWindow@@UBEPBDXZ 1001dba0 f   qt-mt323:qt-mt323.dll
 0001:0001cba6       ?className@QGuardedPtrPrivate@@UBEPBDXZ 1001dba6 f   qt-mt323:qt-mt323.dll
 0001:0001cbac       ?className@QListView@@UBEPBDXZ 1001dbac f   qt-mt323:qt-mt323.dll
 0001:0001cbb2       ?className@QPopupMenu@@UBEPBDXZ 1001dbb2 f   qt-mt323:qt-mt323.dll
 0001:0001cbb8       ?className@QTabWidget@@UBEPBDXZ 1001dbb8 f   qt-mt323:qt-mt323.dll
 0001:0001cbbe       ?className@QToolBar@@UBEPBDXZ 1001dbbe f   qt-mt323:qt-mt323.dll
 0001:0001cbc4       ?className@QWidget@@UBEPBDXZ 1001dbc4 f   qt-mt323:qt-mt323.dll
 0001:0001cbca       ?clear@?$QPtrList@VQDockWindow@@@@UAEXXZ 1001dbca f   qt-mt323:qt-mt323.dll
 0001:0001cbd0       ?clear@QListView@@UAEXXZ   1001dbd0 f   qt-mt323:qt-mt323.dll
 0001:0001cbd6       ?clear@QToolBar@@UAEXXZ    1001dbd6 f   qt-mt323:qt-mt323.dll
 0001:0001cbdc       ?clearSelection@QListView@@UAEXXZ 1001dbdc f   qt-mt323:qt-mt323.dll
 0001:0001cbe2       ?close@QWidget@@UAE_N_N@Z  1001dbe2 f   qt-mt323:qt-mt323.dll
 0001:0001cbe8       ?closeEvent@QPopupMenu@@MAEXPAVQCloseEvent@@@Z 1001dbe8 f   qt-mt323:qt-mt323.dll
 0001:0001cbee       ?closeEvent@QWidget@@MAEXPAVQCloseEvent@@@Z 1001dbee f   qt-mt323:qt-mt323.dll
 0001:0001cbf4       ?cmd@QPaintDevice@@MAE_NHPAVQPainter@@PATQPDevCmdParam@@@Z 1001dbf4 f   qt-mt323:qt-mt323.dll
 0001:0001cbfa       ?compare@QListViewItem@@UBEHPAV1@H_N@Z 1001dbfa f   qt-mt323:qt-mt323.dll
 0001:0001cc00       ?compareItems@QGList@@MAEHPAX0@Z 1001dc00 f   qt-mt323:qt-mt323.dll
 0001:0001cc06       ?connectNotify@QObject@@MAEXPBD@Z 1001dc06 f   qt-mt323:qt-mt323.dll
 0001:0001cc0c       ?contentsContextMenuEvent@QListView@@MAEXPAVQContextMenuEvent@@@Z 1001dc0c f   qt-mt323:qt-mt323.dll
 0001:0001cc12       ?contentsDragEnterEvent@QListView@@MAEXPAVQDragEnterEvent@@@Z 1001dc12 f   qt-mt323:qt-mt323.dll
 0001:0001cc18       ?contentsDragLeaveEvent@QListView@@MAEXPAVQDragLeaveEvent@@@Z 1001dc18 f   qt-mt323:qt-mt323.dll
 0001:0001cc1e       ?contentsDragMoveEvent@QListView@@MAEXPAVQDragMoveEvent@@@Z 1001dc1e f   qt-mt323:qt-mt323.dll
 0001:0001cc24       ?contentsDropEvent@QListView@@MAEXPAVQDropEvent@@@Z 1001dc24 f   qt-mt323:qt-mt323.dll
 0001:0001cc2a       ?contentsMouseDoubleClickEvent@QListView@@MAEXPAVQMouseEvent@@@Z 1001dc2a f   qt-mt323:qt-mt323.dll
 0001:0001cc30       ?contentsMouseMoveEvent@QListView@@MAEXPAVQMouseEvent@@@Z 1001dc30 f   qt-mt323:qt-mt323.dll
 0001:0001cc36       ?contentsMousePressEvent@QListView@@MAEXPAVQMouseEvent@@@Z 1001dc36 f   qt-mt323:qt-mt323.dll
 0001:0001cc3c       ?contentsMouseReleaseEvent@QListView@@MAEXPAVQMouseEvent@@@Z 1001dc3c f   qt-mt323:qt-mt323.dll
 0001:0001cc42       ?contentsWheelEvent@QScrollView@@MAEXPAVQWheelEvent@@@Z 1001dc42 f   qt-mt323:qt-mt323.dll
 0001:0001cc48       ?contextMenuEvent@QDockWindow@@MAEXPAVQContextMenuEvent@@@Z 1001dc48 f   qt-mt323:qt-mt323.dll
 0001:0001cc4e       ?contextMenuEvent@QScrollView@@MAEXPAVQContextMenuEvent@@@Z 1001dc4e f   qt-mt323:qt-mt323.dll
 0001:0001cc54       ?contextMenuEvent@QWidget@@MAEXPAVQContextMenuEvent@@@Z 1001dc54 f   qt-mt323:qt-mt323.dll
 0001:0001cc5a       ?count@?$QPtrList@VQDockWindow@@@@UBEIXZ 1001dc5a f   qt-mt323:qt-mt323.dll
 0001:0001cc60       ?create@QWidget@@MAEXPAUHWND__@@_N1@Z 1001dc60 f   qt-mt323:qt-mt323.dll
 0001:0001cc66       ?customEvent@QObject@@MAEXPAVQCustomEvent@@@Z 1001dc66 f   qt-mt323:qt-mt323.dll
 0001:0001cc6c       ?customWhatsThis@QPopupMenu@@UBE_NXZ 1001dc6c f   qt-mt323:qt-mt323.dll
 0001:0001cc72       ?customWhatsThis@QWidget@@UBE_NXZ 1001dc72 f   qt-mt323:qt-mt323.dll
 0001:0001cc78       ?deleteItem@?$QPtrList@VQDockWindow@@@@EAEXPAX@Z 1001dc78 f   qt-mt323:qt-mt323.dll
 0001:0001cc7e       ?destroy@QWidget@@MAEX_N0@Z 1001dc7e f   qt-mt323:qt-mt323.dll
 0001:0001cc84       ?disconnectNotify@QObject@@MAEXPBD@Z 1001dc84 f   qt-mt323:qt-mt323.dll
 0001:0001cc8a       ?dock@QDockWindow@@UAEXXZ  1001dc8a f   qt-mt323:qt-mt323.dll
 0001:0001cc90       ?dragEnterEvent@QWidget@@MAEXPAVQDragEnterEvent@@@Z 1001dc90 f   qt-mt323:qt-mt323.dll
 0001:0001cc96       ?dragEntered@QListViewItem@@MAEXXZ 1001dc96 f   qt-mt323:qt-mt323.dll
 0001:0001cc9c       ?dragLeaveEvent@QWidget@@MAEXPAVQDragLeaveEvent@@@Z 1001dc9c f   qt-mt323:qt-mt323.dll
 0001:0001cca2       ?dragLeft@QListViewItem@@MAEXXZ 1001dca2 f   qt-mt323:qt-mt323.dll
 0001:0001cca8       ?dragMoveEvent@QWidget@@MAEXPAVQDragMoveEvent@@@Z 1001dca8 f   qt-mt323:qt-mt323.dll
 0001:0001ccae       ?dragObject@QListView@@MAEPAVQDragObject@@XZ 1001dcae f   qt-mt323:qt-mt323.dll
 0001:0001ccb4       ?drawContents@QDockWindow@@MAEXPAVQPainter@@@Z 1001dcb4 f   qt-mt323:qt-mt323.dll
 0001:0001ccba       ?drawContents@QFrame@@MAEXPAVQPainter@@@Z 1001dcba f   qt-mt323:qt-mt323.dll
 0001:0001ccc0       ?drawContents@QPopupMenu@@MAEXPAVQPainter@@@Z 1001dcc0 f   qt-mt323:qt-mt323.dll
 0001:0001ccc6       ?drawContents@QScrollView@@EAEXPAVQPainter@@@Z 1001dcc6 f   qt-mt323:qt-mt323.dll
 0001:0001cccc       ?drawContents@QScrollView@@MAEXPAVQPainter@@HHHH@Z 1001dccc f   qt-mt323:qt-mt323.dll
 0001:0001ccd2       ?drawContentsOffset@QListView@@MAEXPAVQPainter@@HHHHHH@Z 1001dcd2 f   qt-mt323:qt-mt323.dll
 0001:0001ccd8       ?drawFrame@QDockWindow@@MAEXPAVQPainter@@@Z 1001dcd8 f   qt-mt323:qt-mt323.dll
 0001:0001ccde       ?drawFrame@QFrame@@MAEXPAVQPainter@@@Z 1001dcde f   qt-mt323:qt-mt323.dll
 0001:0001cce4       ?dropEvent@QWidget@@MAEXPAVQDropEvent@@@Z 1001dce4 f   qt-mt323:qt-mt323.dll
 0001:0001ccea       ?dropped@QListViewItem@@MAEXPAVQDropEvent@@@Z 1001dcea f   qt-mt323:qt-mt323.dll
 0001:0001ccf0       ?enabledChange@QPopupMenu@@MAEX_N@Z 1001dcf0 f   qt-mt323:qt-mt323.dll
 0001:0001ccf6       ?enabledChange@QWidget@@MAEX_N@Z 1001dcf6 f   qt-mt323:qt-mt323.dll
 0001:0001ccfc       ?enforceSortOrder@QListViewItem@@MBEXXZ 1001dcfc f   qt-mt323:qt-mt323.dll
 0001:0001cd02       ?enterEvent@QWidget@@MAEXPAVQEvent@@@Z 1001dd02 f   qt-mt323:qt-mt323.dll
 0001:0001cd08       ?event@QDockWindow@@MAE_NPAVQEvent@@@Z 1001dd08 f   qt-mt323:qt-mt323.dll
 0001:0001cd0e       ?event@QObject@@UAE_NPAVQEvent@@@Z 1001dd0e f   qt-mt323:qt-mt323.dll
 0001:0001cd14       ?event@QToolBar@@UAE_NPAVQEvent@@@Z 1001dd14 f   qt-mt323:qt-mt323.dll
 0001:0001cd1a       ?event@QWidget@@MAE_NPAVQEvent@@@Z 1001dd1a f   qt-mt323:qt-mt323.dll
 0001:0001cd20       ?eventFilter@QDockWindow@@UAE_NPAVQObject@@PAVQEvent@@@Z 1001dd20 f   qt-mt323:qt-mt323.dll
 0001:0001cd26       ?eventFilter@QLayout@@MAE_NPAVQObject@@PAVQEvent@@@Z 1001dd26 f   qt-mt323:qt-mt323.dll
 0001:0001cd2c       ?eventFilter@QListView@@UAE_NPAVQObject@@PAVQEvent@@@Z 1001dd2c f   qt-mt323:qt-mt323.dll
 0001:0001cd32       ?eventFilter@QObject@@UAE_NPAV1@PAVQEvent@@@Z 1001dd32 f   qt-mt323:qt-mt323.dll
 0001:0001cd38       ?eventFilter@QTabWidget@@MAE_NPAVQObject@@PAVQEvent@@@Z 1001dd38 f   qt-mt323:qt-mt323.dll
 0001:0001cd3e       ?expanding@QBoxLayout@@UBE?AW4ExpandData@QSizePolicy@@XZ 1001dd3e f   qt-mt323:qt-mt323.dll
 0001:0001cd44       ?flush@QFile@@UAEXXZ       1001dd44 f   qt-mt323:qt-mt323.dll
 0001:0001cd4a       ?focusInEvent@QListView@@MAEXPAVQFocusEvent@@@Z 1001dd4a f   qt-mt323:qt-mt323.dll
 0001:0001cd50       ?focusInEvent@QPopupMenu@@MAEXPAVQFocusEvent@@@Z 1001dd50 f   qt-mt323:qt-mt323.dll
 0001:0001cd56       ?focusInEvent@QWidget@@MAEXPAVQFocusEvent@@@Z 1001dd56 f   qt-mt323:qt-mt323.dll
 0001:0001cd5c       ?focusNextPrevChild@QPopupMenu@@MAE_N_N@Z 1001dd5c f   qt-mt323:qt-mt323.dll
 0001:0001cd62       ?focusNextPrevChild@QScrollView@@MAE_N_N@Z 1001dd62 f   qt-mt323:qt-mt323.dll
 0001:0001cd68       ?focusNextPrevChild@QWidget@@MAE_N_N@Z 1001dd68 f   qt-mt323:qt-mt323.dll
 0001:0001cd6e       ?focusOutEvent@QListView@@MAEXPAVQFocusEvent@@@Z 1001dd6e f   qt-mt323:qt-mt323.dll
 0001:0001cd74       ?focusOutEvent@QPopupMenu@@MAEXPAVQFocusEvent@@@Z 1001dd74 f   qt-mt323:qt-mt323.dll
 0001:0001cd7a       ?focusOutEvent@QWidget@@MAEXPAVQFocusEvent@@@Z 1001dd7a f   qt-mt323:qt-mt323.dll
 0001:0001cd80       ?fontChange@QScrollView@@MAEXABVQFont@@@Z 1001dd80 f   qt-mt323:qt-mt323.dll
 0001:0001cd86       ?fontChange@QWidget@@MAEXABVQFont@@@Z 1001dd86 f   qt-mt323:qt-mt323.dll
 0001:0001cd8c       ?fontInf@QPaintDevice@@MBEHPAVQFont@@H@Z 1001dd8c f   qt-mt323:qt-mt323.dll
 0001:0001cd92       ?fontMet@QPaintDevice@@MBEHPAVQFont@@HPBDH@Z 1001dd92 f   qt-mt323:qt-mt323.dll
 0001:0001cd98       ?frameChanged@QFrame@@MAEXXZ 1001dd98 f   qt-mt323:qt-mt323.dll
 0001:0001cd9e       ?frameChanged@QHBox@@MAEXXZ 1001dd9e f   qt-mt323:qt-mt323.dll
 0001:0001cda4       ?frameChanged@QPopupMenu@@EAEXXZ 1001dda4 f   qt-mt323:qt-mt323.dll
 0001:0001cdaa       ?frameChanged@QScrollView@@MAEXXZ 1001ddaa f   qt-mt323:qt-mt323.dll
 0001:0001cdb0       ?geometry@QLayout@@UBE?AVQRect@@XZ 1001ddb0 f   qt-mt323:qt-mt323.dll
 0001:0001cdb6       ?getch@QFile@@UAEHXZ       1001ddb6 f   qt-mt323:qt-mt323.dll
 0001:0001cdbc       ?handle@QPaintDevice@@UBEPAUHDC__@@XZ 1001ddbc f   qt-mt323:qt-mt323.dll
 0001:0001cdc2       ?hasHeightForWidth@QBoxLayout@@UBE_NXZ 1001ddc2 f   qt-mt323:qt-mt323.dll
 0001:0001cdc8       ?heightForWidth@QBoxLayout@@UBEHH@Z 1001ddc8 f   qt-mt323:qt-mt323.dll
 0001:0001cdce       ?heightForWidth@QWidget@@UBEHH@Z 1001ddce f   qt-mt323:qt-mt323.dll
 0001:0001cdd4       ?hide@QPopupMenu@@UAEXXZ   1001ddd4 f   qt-mt323:qt-mt323.dll
 0001:0001cdda       ?hide@QToolBar@@UAEXXZ     1001ddda f   qt-mt323:qt-mt323.dll
 0001:0001cde0       ?hide@QWidget@@UAEXXZ      1001dde0 f   qt-mt323:qt-mt323.dll
 0001:0001cde6       ?hideEvent@QDockWindow@@MAEXPAVQHideEvent@@@Z 1001dde6 f   qt-mt323:qt-mt323.dll
 0001:0001cdec       ?hideEvent@QWidget@@MAEXPAVQHideEvent@@@Z 1001ddec f   qt-mt323:qt-mt323.dll
 0001:0001cdf2       ?imComposeEvent@QWidget@@MAEXPAVQIMEvent@@@Z 1001ddf2 f   qt-mt323:qt-mt323.dll
 0001:0001cdf8       ?imEndEvent@QWidget@@MAEXPAVQIMEvent@@@Z 1001ddf8 f   qt-mt323:qt-mt323.dll
 0001:0001cdfe       ?imStartEvent@QWidget@@MAEXPAVQIMEvent@@@Z 1001ddfe f   qt-mt323:qt-mt323.dll
 0001:0001ce04       ?insertChild@QObject@@UAEXPAV1@@Z 1001de04 f   qt-mt323:qt-mt323.dll
 0001:0001ce0a       ?insertItem@QListView@@UAEXPAVQListViewItem@@@Z 1001de0a f   qt-mt323:qt-mt323.dll
 0001:0001ce10       ?insertItem@QListViewItem@@UAEXPAV1@@Z 1001de10 f   qt-mt323:qt-mt323.dll
 0001:0001ce16       ?insertTab@QTabWidget@@UAEXPAVQWidget@@ABVQIconSet@@ABVQString@@H@Z 1001de16 f   qt-mt323:qt-mt323.dll
 0001:0001ce1c       ?insertTab@QTabWidget@@UAEXPAVQWidget@@ABVQString@@H@Z 1001de1c f   qt-mt323:qt-mt323.dll
 0001:0001ce22       ?insertTab@QTabWidget@@UAEXPAVQWidget@@PAVQTab@@H@Z 1001de22 f   qt-mt323:qt-mt323.dll
 0001:0001ce28       ?invalidate@QBoxLayout@@UAEXXZ 1001de28 f   qt-mt323:qt-mt323.dll
 0001:0001ce2e       ?invalidateHeight@QListViewItem@@UAEXXZ 1001de2e f   qt-mt323:qt-mt323.dll
 0001:0001ce34       ?invertSelection@QListView@@UAEXXZ 1001de34 f   qt-mt323:qt-mt323.dll
 0001:0001ce3a       ?isEmpty@QLayout@@UBE_NXZ  1001de3a f   qt-mt323:qt-mt323.dll
 0001:0001ce40       ?iterator@QBoxLayout@@UAE?AVQLayoutIterator@@XZ 1001de40 f   qt-mt323:qt-mt323.dll
 0001:0001ce46       ?key@QListViewItem@@UBE?AVQString@@H_N@Z 1001de46 f   qt-mt323:qt-mt323.dll
 0001:0001ce4c       ?keyPressEvent@QListView@@MAEXPAVQKeyEvent@@@Z 1001de4c f   qt-mt323:qt-mt323.dll
 0001:0001ce52       ?keyPressEvent@QPopupMenu@@MAEXPAVQKeyEvent@@@Z 1001de52 f   qt-mt323:qt-mt323.dll
 0001:0001ce58       ?keyPressEvent@QWidget@@MAEXPAVQKeyEvent@@@Z 1001de58 f   qt-mt323:qt-mt323.dll
 0001:0001ce5e       ?keyReleaseEvent@QWidget@@MAEXPAVQKeyEvent@@@Z 1001de5e f   qt-mt323:qt-mt323.dll
 0001:0001ce64       ?layout@QLayout@@UAEPAV1@XZ 1001de64 f   qt-mt323:qt-mt323.dll
 0001:0001ce6a       ?leaveEvent@QPopupMenu@@MAEXPAVQEvent@@@Z 1001de6a f   qt-mt323:qt-mt323.dll
 0001:0001ce70       ?leaveEvent@QWidget@@MAEXPAVQEvent@@@Z 1001de70 f   qt-mt323:qt-mt323.dll
 0001:0001ce76       ?maximumSize@QBoxLayout@@UBE?AVQSize@@XZ 1001de76 f   qt-mt323:qt-mt323.dll
 0001:0001ce7c       ?menuContentsChanged@QPopupMenu@@EAEXXZ 1001de7c f   qt-mt323:qt-mt323.dll
 0001:0001ce82       ?menuDelPopup@QPopupMenu@@EAEXPAV1@@Z 1001de82 f   qt-mt323:qt-mt323.dll
 0001:0001ce88       ?menuInsPopup@QPopupMenu@@EAEXPAV1@@Z 1001de88 f   qt-mt323:qt-mt323.dll
 0001:0001ce8e       ?menuStateChanged@QPopupMenu@@EAEXXZ 1001de8e f   qt-mt323:qt-mt323.dll
 0001:0001ce94       ?metaObject@QAction@@UBEPAVQMetaObject@@XZ 1001de94 f   qt-mt323:qt-mt323.dll
 0001:0001ce9a       ?metaObject@QBoxLayout@@UBEPAVQMetaObject@@XZ 1001de9a f   qt-mt323:qt-mt323.dll
 0001:0001cea0       ?metaObject@QDockWindow@@UBEPAVQMetaObject@@XZ 1001dea0 f   qt-mt323:qt-mt323.dll
 0001:0001cea6       ?metaObject@QGuardedPtrPrivate@@UBEPAVQMetaObject@@XZ 1001dea6 f   qt-mt323:qt-mt323.dll
 0001:0001ceac       ?metaObject@QListView@@UBEPAVQMetaObject@@XZ 1001deac f   qt-mt323:qt-mt323.dll
 0001:0001ceb2       ?metaObject@QPopupMenu@@UBEPAVQMetaObject@@XZ 1001deb2 f   qt-mt323:qt-mt323.dll
 0001:0001ceb8       ?metaObject@QTabWidget@@UBEPAVQMetaObject@@XZ 1001deb8 f   qt-mt323:qt-mt323.dll
 0001:0001cebe       ?metaObject@QToolBar@@UBEPAVQMetaObject@@XZ 1001debe f   qt-mt323:qt-mt323.dll
 0001:0001cec4       ?metaObject@QWidget@@UBEPAVQMetaObject@@XZ 1001dec4 f   qt-mt323:qt-mt323.dll
 0001:0001ceca       ?metric@QWidget@@MBEHH@Z   1001deca f   qt-mt323:qt-mt323.dll
 0001:0001ced0       ?minimumSize@QBoxLayout@@UBE?AVQSize@@XZ 1001ded0 f   qt-mt323:qt-mt323.dll
 0001:0001ced6       ?minimumSizeHint@QDockWindow@@UBE?AVQSize@@XZ 1001ded6 f   qt-mt323:qt-mt323.dll
 0001:0001cedc       ?minimumSizeHint@QListView@@UBE?AVQSize@@XZ 1001dedc f   qt-mt323:qt-mt323.dll
 0001:0001cee2       ?minimumSizeHint@QTabWidget@@UBE?AVQSize@@XZ 1001dee2 f   qt-mt323:qt-mt323.dll
 0001:0001cee8       ?minimumSizeHint@QToolBar@@UBE?AVQSize@@XZ 1001dee8 f   qt-mt323:qt-mt323.dll
 0001:0001ceee       ?minimumSizeHint@QWidget@@UBE?AVQSize@@XZ 1001deee f   qt-mt323:qt-mt323.dll
 0001:0001cef4       ?mouseDoubleClickEvent@QScrollView@@MAEXPAVQMouseEvent@@@Z 1001def4 f   qt-mt323:qt-mt323.dll
 0001:0001cefa       ?mouseDoubleClickEvent@QWidget@@MAEXPAVQMouseEvent@@@Z 1001defa f   qt-mt323:qt-mt323.dll
 0001:0001cf00       ?mouseMoveEvent@QPopupMenu@@MAEXPAVQMouseEvent@@@Z 1001df00 f   qt-mt323:qt-mt323.dll
 0001:0001cf06       ?mouseMoveEvent@QScrollView@@MAEXPAVQMouseEvent@@@Z 1001df06 f   qt-mt323:qt-mt323.dll
 0001:0001cf0c       ?mouseMoveEvent@QWidget@@MAEXPAVQMouseEvent@@@Z 1001df0c f   qt-mt323:qt-mt323.dll
 0001:0001cf12       ?mousePressEvent@QPopupMenu@@MAEXPAVQMouseEvent@@@Z 1001df12 f   qt-mt323:qt-mt323.dll
 0001:0001cf18       ?mousePressEvent@QScrollView@@MAEXPAVQMouseEvent@@@Z 1001df18 f   qt-mt323:qt-mt323.dll
 0001:0001cf1e       ?mousePressEvent@QWidget@@MAEXPAVQMouseEvent@@@Z 1001df1e f   qt-mt323:qt-mt323.dll
 0001:0001cf24       ?mouseReleaseEvent@QPopupMenu@@MAEXPAVQMouseEvent@@@Z 1001df24 f   qt-mt323:qt-mt323.dll
 0001:0001cf2a       ?mouseReleaseEvent@QScrollView@@MAEXPAVQMouseEvent@@@Z 1001df2a f   qt-mt323:qt-mt323.dll
 0001:0001cf30       ?mouseReleaseEvent@QWidget@@MAEXPAVQMouseEvent@@@Z 1001df30 f   qt-mt323:qt-mt323.dll
 0001:0001cf36       ?move@QWidget@@UAEXHH@Z    1001df36 f   qt-mt323:qt-mt323.dll
 0001:0001cf3c       ?moveChild@QScrollView@@UAEXPAVQWidget@@HH@Z 1001df3c f   qt-mt323:qt-mt323.dll
 0001:0001cf42       ?moveEvent@QWidget@@MAEXPAVQMoveEvent@@@Z 1001df42 f   qt-mt323:qt-mt323.dll
 0001:0001cf48       ?newItem@QPtrCollection@@MAEPAXPAX@Z 1001df48 f   qt-mt323:qt-mt323.dll
 0001:0001cf4e       ?okRename@QListViewItem@@MAEXH@Z 1001df4e f   qt-mt323:qt-mt323.dll
 0001:0001cf54       ?paintBranches@QListViewItem@@UAEXPAVQPainter@@ABVQColorGroup@@HHH@Z 1001df54 f   qt-mt323:qt-mt323.dll
 0001:0001cf5a       ?paintCell@QListViewItem@@UAEXPAVQPainter@@ABVQColorGroup@@HHH@Z 1001df5a f   qt-mt323:qt-mt323.dll
 0001:0001cf60       ?paintEmptyArea@QListView@@MAEXPAVQPainter@@ABVQRect@@@Z 1001df60 f   qt-mt323:qt-mt323.dll
 0001:0001cf66       ?paintEvent@QFrame@@MAEXPAVQPaintEvent@@@Z 1001df66 f   qt-mt323:qt-mt323.dll
 0001:0001cf6c       ?paintEvent@QPopupMenu@@MAEXPAVQPaintEvent@@@Z 1001df6c f   qt-mt323:qt-mt323.dll
 0001:0001cf72       ?paintEvent@QWidget@@MAEXPAVQPaintEvent@@@Z 1001df72 f   qt-mt323:qt-mt323.dll
 0001:0001cf78       ?paintFocus@QListViewItem@@UAEXPAVQPainter@@ABVQColorGroup@@ABVQRect@@@Z 1001df78 f   qt-mt323:qt-mt323.dll
 0001:0001cf7e       ?paletteChange@QWidget@@MAEXABVQPalette@@@Z 1001df7e f   qt-mt323:qt-mt323.dll
 0001:0001cf84       ?pixmap@QListViewItem@@UBEPBVQPixmap@@H@Z 1001df84 f   qt-mt323:qt-mt323.dll
 0001:0001cf8a       ?polish@QWidget@@UAEXXZ    1001df8a f   qt-mt323:qt-mt323.dll
 0001:0001cf90       ?property@QObject@@UBE?AVQVariant@@PBD@Z 1001df90 f   qt-mt323:qt-mt323.dll
 0001:0001cf96       ?putch@QFile@@UAEHH@Z      1001df96 f   qt-mt323:qt-mt323.dll
 0001:0001cf9c       ?qt_cast@QAction@@UAEPAXPBD@Z 1001df9c f   qt-mt323:qt-mt323.dll
 0001:0001cfa2       ?qt_cast@QBoxLayout@@UAEPAXPBD@Z 1001dfa2 f   qt-mt323:qt-mt323.dll
 0001:0001cfa8       ?qt_cast@QDockWindow@@UAEPAXPBD@Z 1001dfa8 f   qt-mt323:qt-mt323.dll
 0001:0001cfae       ?qt_cast@QGuardedPtrPrivate@@UAEPAXPBD@Z 1001dfae f   qt-mt323:qt-mt323.dll
 0001:0001cfb4       ?qt_cast@QListView@@UAEPAXPBD@Z 1001dfb4 f   qt-mt323:qt-mt323.dll
 0001:0001cfba       ?qt_cast@QPopupMenu@@UAEPAXPBD@Z 1001dfba f   qt-mt323:qt-mt323.dll
 0001:0001cfc0       ?qt_cast@QTabWidget@@UAEPAXPBD@Z 1001dfc0 f   qt-mt323:qt-mt323.dll
 0001:0001cfc6       ?qt_cast@QToolBar@@UAEPAXPBD@Z 1001dfc6 f   qt-mt323:qt-mt323.dll
 0001:0001cfcc       ?qt_cast@QWidget@@UAEPAXPBD@Z 1001dfcc f   qt-mt323:qt-mt323.dll
 0001:0001cfd2       ?qt_emit@QAction@@UAE_NHPAUQUObject@@@Z 1001dfd2 f   qt-mt323:qt-mt323.dll
 0001:0001cfd8       ?qt_emit@QBoxLayout@@UAE_NHPAUQUObject@@@Z 1001dfd8 f   qt-mt323:qt-mt323.dll
 0001:0001cfde       ?qt_emit@QDockWindow@@UAE_NHPAUQUObject@@@Z 1001dfde f   qt-mt323:qt-mt323.dll
 0001:0001cfe4       ?qt_emit@QGuardedPtrPrivate@@UAE_NHPAUQUObject@@@Z 1001dfe4 f   qt-mt323:qt-mt323.dll
 0001:0001cfea       ?qt_emit@QListView@@UAE_NHPAUQUObject@@@Z 1001dfea f   qt-mt323:qt-mt323.dll
 0001:0001cff0       ?qt_emit@QPopupMenu@@UAE_NHPAUQUObject@@@Z 1001dff0 f   qt-mt323:qt-mt323.dll
 0001:0001cff6       ?qt_emit@QTabWidget@@UAE_NHPAUQUObject@@@Z 1001dff6 f   qt-mt323:qt-mt323.dll
 0001:0001cffe       ?qt_emit@QToolBar@@UAE_NHPAUQUObject@@@Z 1001dffe f   qt-mt323:qt-mt323.dll
 0001:0001d004       ?qt_emit@QWidget@@UAE_NHPAUQUObject@@@Z 1001e004 f   qt-mt323:qt-mt323.dll
 0001:0001d00a       ?qt_invoke@QAction@@UAE_NHPAUQUObject@@@Z 1001e00a f   qt-mt323:qt-mt323.dll
 0001:0001d010       ?qt_invoke@QBoxLayout@@UAE_NHPAUQUObject@@@Z 1001e010 f   qt-mt323:qt-mt323.dll
 0001:0001d016       ?qt_invoke@QDockWindow@@UAE_NHPAUQUObject@@@Z 1001e016 f   qt-mt323:qt-mt323.dll
 0001:0001d01c       ?qt_invoke@QGuardedPtrPrivate@@UAE_NHPAUQUObject@@@Z 1001e01c f   qt-mt323:qt-mt323.dll
 0001:0001d022       ?qt_invoke@QListView@@UAE_NHPAUQUObject@@@Z 1001e022 f   qt-mt323:qt-mt323.dll
 0001:0001d028       ?qt_invoke@QPopupMenu@@UAE_NHPAUQUObject@@@Z 1001e028 f   qt-mt323:qt-mt323.dll
 0001:0001d02e       ?qt_invoke@QTabWidget@@UAE_NHPAUQUObject@@@Z 1001e02e f   qt-mt323:qt-mt323.dll
 0001:0001d034       ?qt_invoke@QToolBar@@UAE_NHPAUQUObject@@@Z 1001e034 f   qt-mt323:qt-mt323.dll
 0001:0001d03a       ?qt_invoke@QWidget@@UAE_NHPAUQUObject@@@Z 1001e03a f   qt-mt323:qt-mt323.dll
 0001:0001d040       ?qt_property@QAction@@UAE_NHHPAVQVariant@@@Z 1001e040 f   qt-mt323:qt-mt323.dll
 0001:0001d046       ?qt_property@QBoxLayout@@UAE_NHHPAVQVariant@@@Z 1001e046 f   qt-mt323:qt-mt323.dll
 0001:0001d04c       ?qt_property@QDockWindow@@UAE_NHHPAVQVariant@@@Z 1001e04c f   qt-mt323:qt-mt323.dll
 0001:0001d052       ?qt_property@QGuardedPtrPrivate@@UAE_NHHPAVQVariant@@@Z 1001e052 f   qt-mt323:qt-mt323.dll
 0001:0001d058       ?qt_property@QListView@@UAE_NHHPAVQVariant@@@Z 1001e058 f   qt-mt323:qt-mt323.dll
 0001:0001d05e       ?qt_property@QPopupMenu@@UAE_NHHPAVQVariant@@@Z 1001e05e f   qt-mt323:qt-mt323.dll
 0001:0001d064       ?qt_property@QTabWidget@@UAE_NHHPAVQVariant@@@Z 1001e064 f   qt-mt323:qt-mt323.dll
 0001:0001d06a       ?qt_property@QToolBar@@UAE_NHHPAVQVariant@@@Z 1001e06a f   qt-mt323:qt-mt323.dll
 0001:0001d070       ?qt_property@QWidget@@UAE_NHHPAVQVariant@@@Z 1001e070 f   qt-mt323:qt-mt323.dll
 0001:0001d076       ?read@QGDict@@MAEAAVQDataStream@@AAV2@AAPAX@Z 1001e076 f   qt-mt323:qt-mt323.dll
 0001:0001d07c       ?read@QGList@@MAEAAVQDataStream@@AAV2@AAPAX@Z 1001e07c f   qt-mt323:qt-mt323.dll
 0001:0001d082       ?readAll@QIODevice@@UAE?AV?$QMemArray@D@@XZ 1001e082 f   qt-mt323:qt-mt323.dll
 0001:0001d088       ?readBlock@QFile@@UAEJPADK@Z 1001e088 f   qt-mt323:qt-mt323.dll
 0001:0001d08e       ?readLine@QFile@@UAEJPADK@Z 1001e08e f   qt-mt323:qt-mt323.dll
 0001:0001d094       ?removeChild@QObject@@UAEXPAV1@@Z 1001e094 f   qt-mt323:qt-mt323.dll
 0001:0001d09a       ?removeChild@QScrollView@@UAEXPAVQObject@@@Z 1001e09a f   qt-mt323:qt-mt323.dll
 0001:0001d0a0       ?removeColumn@QListView@@UAEXH@Z 1001e0a0 f   qt-mt323:qt-mt323.dll
 0001:0001d0a6       ?removeFrom@QAction@@UAE_NPAVQWidget@@@Z 1001e0a6 f   qt-mt323:qt-mt323.dll
 0001:0001d0ac       ?removeItem@QListView@@UAEXPAVQListViewItem@@@Z 1001e0ac f   qt-mt323:qt-mt323.dll
 0001:0001d0b2       ?removeItem@QListViewItem@@UAEXPAV1@@Z 1001e0b2 f   qt-mt323:qt-mt323.dll
 0001:0001d0b8       ?removePage@QTabWidget@@UAEXPAVQWidget@@@Z 1001e0b8 f   qt-mt323:qt-mt323.dll
 0001:0001d0be       ?reparent@QWidget@@UAEXPAV1@IABVQPoint@@_N@Z 1001e0be f   qt-mt323:qt-mt323.dll
 0001:0001d0c4       ?resize@QScrollView@@UAEXHH@Z 1001e0c4 f   qt-mt323:qt-mt323.dll
 0001:0001d0ca       ?resize@QWidget@@UAEXHH@Z  1001e0ca f   qt-mt323:qt-mt323.dll
 0001:0001d0d0       ?resizeContents@QScrollView@@UAEXHH@Z 1001e0d0 f   qt-mt323:qt-mt323.dll
 0001:0001d0d6       ?resizeEvent@QDockWindow@@MAEXPAVQResizeEvent@@@Z 1001e0d6 f   qt-mt323:qt-mt323.dll
 0001:0001d0dc       ?resizeEvent@QFrame@@MAEXPAVQResizeEvent@@@Z 1001e0dc f   qt-mt323:qt-mt323.dll
 0001:0001d0e2       ?resizeEvent@QListView@@MAEXPAVQResizeEvent@@@Z 1001e0e2 f   qt-mt323:qt-mt323.dll
 0001:0001d0e8       ?resizeEvent@QTabWidget@@MAEXPAVQResizeEvent@@@Z 1001e0e8 f   qt-mt323:qt-mt323.dll
 0001:0001d0ee       ?resizeEvent@QToolBar@@MAEXPAVQResizeEvent@@@Z 1001e0ee f   qt-mt323:qt-mt323.dll
 0001:0001d0f4       ?resizeEvent@QWidget@@MAEXPAVQResizeEvent@@@Z 1001e0f4 f   qt-mt323:qt-mt323.dll
 0001:0001d0fa       ?resolution@QPaintDevice@@UBEHXZ 1001e0fa f   qt-mt323:qt-mt323.dll
 0001:0001d100       ?rtti@QListViewItem@@UBEHXZ 1001e100 f   qt-mt323:qt-mt323.dll
 0001:0001d106       ?selectAll@QListView@@UAEX_N@Z 1001e106 f   qt-mt323:qt-mt323.dll
 0001:0001d10c       ?setAccel@QAction@@UAEXABVQKeySequence@@@Z 1001e10c f   qt-mt323:qt-mt323.dll
 0001:0001d112       ?setAcceptDrops@QWidget@@UAEX_N@Z 1001e112 f   qt-mt323:qt-mt323.dll
 0001:0001d118       ?setActiveItem@QPopupMenu@@UAEXH@Z 1001e118 f   qt-mt323:qt-mt323.dll
 0001:0001d11e       ?setActiveWindow@QWidget@@UAEXXZ 1001e11e f   qt-mt323:qt-mt323.dll
 0001:0001d124       ?setAlignment@QLayoutItem@@UAEXH@Z 1001e124 f   qt-mt323:qt-mt323.dll
 0001:0001d12a       ?setAllColumnsShowFocus@QListView@@UAEX_N@Z 1001e12a f   qt-mt323:qt-mt323.dll
 0001:0001d130       ?setAutoAdd@QLayout@@UAEX_N@Z 1001e130 f   qt-mt323:qt-mt323.dll
 0001:0001d136       ?setAutoMask@QWidget@@UAEX_N@Z 1001e136 f   qt-mt323:qt-mt323.dll
 0001:0001d13c       ?setBackgroundColor@QWidget@@UAEXABVQColor@@@Z 1001e13c f   qt-mt323:qt-mt323.dll
 0001:0001d142       ?setBackgroundMode@QWidget@@UAEXW4BackgroundMode@Qt@@@Z 1001e142 f   qt-mt323:qt-mt323.dll
 0001:0001d148       ?setBackgroundOrigin@QWidget@@UAEXW4BackgroundOrigin@1@@Z 1001e148 f   qt-mt323:qt-mt323.dll
 0001:0001d14e       ?setBackgroundPixmap@QWidget@@UAEXABVQPixmap@@@Z 1001e14e f   qt-mt323:qt-mt323.dll
 0001:0001d154       ?setCaption@QDockWindow@@UAEXABVQString@@@Z 1001e154 f   qt-mt323:qt-mt323.dll
 0001:0001d15a       ?setCaption@QWidget@@UAEXABVQString@@@Z 1001e15a f   qt-mt323:qt-mt323.dll
 0001:0001d160       ?setCheckable@QPopupMenu@@UAEX_N@Z 1001e160 f   qt-mt323:qt-mt323.dll
 0001:0001d166       ?setCloseMode@QDockWindow@@UAEXH@Z 1001e166 f   qt-mt323:qt-mt323.dll
 0001:0001d16c       ?setColumnAlignment@QListView@@UAEXHH@Z 1001e16c f   qt-mt323:qt-mt323.dll
 0001:0001d172       ?setColumnText@QListView@@UAEXHABVQIconSet@@ABVQString@@@Z 1001e172 f   qt-mt323:qt-mt323.dll
 0001:0001d178       ?setColumnText@QListView@@UAEXHABVQString@@@Z 1001e178 f   qt-mt323:qt-mt323.dll
 0001:0001d17e       ?setColumnWidth@QListView@@UAEXHH@Z 1001e17e f   qt-mt323:qt-mt323.dll
 0001:0001d184       ?setColumnWidthMode@QListView@@UAEXHW4WidthMode@1@@Z 1001e184 f   qt-mt323:qt-mt323.dll
 0001:0001d18a       ?setContentsPos@QListView@@UAEXHH@Z 1001e18a f   qt-mt323:qt-mt323.dll
 0001:0001d190       ?setCornerWidget@QScrollView@@UAEXPAVQWidget@@@Z 1001e190 f   qt-mt323:qt-mt323.dll
 0001:0001d196       ?setCurrentItem@QListView@@UAEXPAVQListViewItem@@@Z 1001e196 f   qt-mt323:qt-mt323.dll
 0001:0001d19c       ?setCursor@QWidget@@UAEXABVQCursor@@@Z 1001e19c f   qt-mt323:qt-mt323.dll
 0001:0001d1a2       ?setDefaultRenameAction@QListView@@UAEXW4RenameAction@1@@Z 1001e1a2 f   qt-mt323:qt-mt323.dll
 0001:0001d1a8       ?setDragAutoScroll@QScrollView@@UAEX_N@Z 1001e1a8 f   qt-mt323:qt-mt323.dll
 0001:0001d1ae       ?setDragEnabled@QListViewItem@@UAEX_N@Z 1001e1ae f   qt-mt323:qt-mt323.dll
 0001:0001d1b4       ?setDropEnabled@QListViewItem@@UAEX_N@Z 1001e1b4 f   qt-mt323:qt-mt323.dll
 0001:0001d1ba       ?setEnabled@QAction@@UAEX_N@Z 1001e1ba f   qt-mt323:qt-mt323.dll
 0001:0001d1c0       ?setEnabled@QListViewItem@@UAEX_N@Z 1001e1c0 f   qt-mt323:qt-mt323.dll
 0001:0001d1c6       ?setEnabled@QScrollView@@UAEX_N@Z 1001e1c6 f   qt-mt323:qt-mt323.dll
 0001:0001d1cc       ?setEnabled@QWidget@@UAEX_N@Z 1001e1cc f   qt-mt323:qt-mt323.dll
 0001:0001d1d2       ?setEraseColor@QWidget@@UAEXABVQColor@@@Z 1001e1d2 f   qt-mt323:qt-mt323.dll
 0001:0001d1d8       ?setErasePixmap@QWidget@@UAEXABVQPixmap@@@Z 1001e1d8 f   qt-mt323:qt-mt323.dll
 0001:0001d1de       ?setExpandable@QListViewItem@@UAEX_N@Z 1001e1de f   qt-mt323:qt-mt323.dll
 0001:0001d1e4       ?setFirstItemActive@QPopupMenu@@EAEXXZ 1001e1e4 f   qt-mt323:qt-mt323.dll
 0001:0001d1ea       ?setFixedExtentHeight@QDockWindow@@UAEXH@Z 1001e1ea f   qt-mt323:qt-mt323.dll
 0001:0001d1f0       ?setFixedExtentWidth@QDockWindow@@UAEXH@Z 1001e1f0 f   qt-mt323:qt-mt323.dll
 0001:0001d1f6       ?setFocus@QWidget@@UAEXXZ  1001e1f6 f   qt-mt323:qt-mt323.dll
 0001:0001d1fc       ?setFocusPolicy@QWidget@@UAEXW4FocusPolicy@1@@Z 1001e1fc f   qt-mt323:qt-mt323.dll
 0001:0001d202       ?setFocusProxy@QWidget@@UAEXPAV1@@Z 1001e202 f   qt-mt323:qt-mt323.dll
 0001:0001d208       ?setFont@QListView@@UAEXABVQFont@@@Z 1001e208 f   qt-mt323:qt-mt323.dll
 0001:0001d20e       ?setFont@QPopupMenu@@UAEXABVQFont@@@Z 1001e20e f   qt-mt323:qt-mt323.dll
 0001:0001d214       ?setFont@QWidget@@UAEXABVQFont@@@Z 1001e214 f   qt-mt323:qt-mt323.dll
 0001:0001d21a       ?setFrameRect@QFrame@@UAEXABVQRect@@@Z 1001e21a f   qt-mt323:qt-mt323.dll
 0001:0001d220       ?setFrameStyle@QFrame@@UAEXH@Z 1001e220 f   qt-mt323:qt-mt323.dll
 0001:0001d226       ?setGeometry@QBoxLayout@@UAEXABVQRect@@@Z 1001e226 f   qt-mt323:qt-mt323.dll
 0001:0001d22c       ?setGeometry@QWidget@@UAEXABVQRect@@@Z 1001e22c f   qt-mt323:qt-mt323.dll
 0001:0001d232       ?setGeometry@QWidget@@UAEXHHHH@Z 1001e232 f   qt-mt323:qt-mt323.dll
 0001:0001d238       ?setHBarGeometry@QScrollView@@MAEXAAVQScrollBar@@HHHH@Z 1001e238 f   qt-mt323:qt-mt323.dll
 0001:0001d23e       ?setHScrollBarMode@QScrollView@@UAEXW4ScrollBarMode@1@@Z 1001e23e f   qt-mt323:qt-mt323.dll
 0001:0001d244       ?setHeight@QListViewItem@@MAEXH@Z 1001e244 f   qt-mt323:qt-mt323.dll
 0001:0001d24a       ?setHorizontallyStretchable@QDockWindow@@UAEX_N@Z 1001e24a f   qt-mt323:qt-mt323.dll
 0001:0001d250       ?setIcon@QWidget@@UAEXABVQPixmap@@@Z 1001e250 f   qt-mt323:qt-mt323.dll
 0001:0001d256       ?setIconSet@QAction@@UAEXABVQIconSet@@@Z 1001e256 f   qt-mt323:qt-mt323.dll
 0001:0001d25c       ?setIconText@QWidget@@UAEXABVQString@@@Z 1001e25c f   qt-mt323:qt-mt323.dll
 0001:0001d262       ?setId@QMenuData@@UAEXHH@Z 1001e262 f   qt-mt323:qt-mt323.dll
 0001:0001d268       ?setItemMargin@QListView@@UAEXH@Z 1001e268 f   qt-mt323:qt-mt323.dll
 0001:0001d26e       ?setKeyCompression@QWidget@@MAEX_N@Z 1001e26e f   qt-mt323:qt-mt323.dll
 0001:0001d274       ?setLabel@QToolBar@@UAEXABVQString@@@Z 1001e274 f   qt-mt323:qt-mt323.dll
 0001:0001d27a       ?setLineWidth@QFrame@@UAEXH@Z 1001e27a f   qt-mt323:qt-mt323.dll
 0001:0001d280       ?setMargin@QFrame@@UAEXH@Z 1001e280 f   qt-mt323:qt-mt323.dll
 0001:0001d286       ?setMargin@QLayout@@UAEXH@Z 1001e286 f   qt-mt323:qt-mt323.dll
 0001:0001d28c       ?setMargins@QScrollView@@MAEXHHHH@Z 1001e28c f   qt-mt323:qt-mt323.dll
 0001:0001d292       ?setMask@QWidget@@UAEXABVQBitmap@@@Z 1001e292 f   qt-mt323:qt-mt323.dll
 0001:0001d298       ?setMask@QWidget@@UAEXABVQRegion@@@Z 1001e298 f   qt-mt323:qt-mt323.dll
 0001:0001d29e       ?setMaximumSize@QWidget@@UAEXHH@Z 1001e29e f   qt-mt323:qt-mt323.dll
 0001:0001d2a4       ?setMenuBar@QLayout@@UAEXPAVQMenuBar@@@Z 1001e2a4 f   qt-mt323:qt-mt323.dll
 0001:0001d2aa       ?setMenuText@QAction@@UAEXABVQString@@@Z 1001e2aa f   qt-mt323:qt-mt323.dll
 0001:0001d2b0       ?setMicroFocusHint@QWidget@@MAEXHHHH_NPAVQFont@@@Z 1001e2b0 f   qt-mt323:qt-mt323.dll
 0001:0001d2b6       ?setMidLineWidth@QFrame@@UAEXH@Z 1001e2b6 f   qt-mt323:qt-mt323.dll
 0001:0001d2bc       ?setMinimumSize@QToolBar@@UAEXHH@Z 1001e2bc f   qt-mt323:qt-mt323.dll
 0001:0001d2c2       ?setMinimumSize@QWidget@@UAEXHH@Z 1001e2c2 f   qt-mt323:qt-mt323.dll
 0001:0001d2c8       ?setMouseTracking@QWidget@@UAEX_N@Z 1001e2c8 f   qt-mt323:qt-mt323.dll
 0001:0001d2ce       ?setMovingEnabled@QDockWindow@@UAEX_N@Z 1001e2ce f   qt-mt323:qt-mt323.dll
 0001:0001d2d4       ?setMultiLinesEnabled@QListViewItem@@UAEX_N@Z 1001e2d4 f   qt-mt323:qt-mt323.dll
 0001:0001d2da       ?setMultiSelection@QListView@@UAEX_N@Z 1001e2da f   qt-mt323:qt-mt323.dll
 0001:0001d2e0       ?setName@QObject@@UAEXPBD@Z 1001e2e0 f   qt-mt323:qt-mt323.dll
 0001:0001d2e6       ?setNewLine@QDockWindow@@UAEX_N@Z 1001e2e6 f   qt-mt323:qt-mt323.dll
 0001:0001d2ec       ?setOffset@QDockWindow@@UAEXH@Z 1001e2ec f   qt-mt323:qt-mt323.dll
 0001:0001d2f2       ?setOn@QAction@@UAEX_N@Z   1001e2f2 f   qt-mt323:qt-mt323.dll
 0001:0001d2f8       ?setOpaqueMoving@QDockWindow@@UAEX_N@Z 1001e2f8 f   qt-mt323:qt-mt323.dll
 0001:0001d2fe       ?setOpen@QListView@@UAEXPAVQListViewItem@@_N@Z 1001e2fe f   qt-mt323:qt-mt323.dll
 0001:0001d304       ?setOpen@QListViewItem@@UAEX_N@Z 1001e304 f   qt-mt323:qt-mt323.dll
 0001:0001d30a       ?setOrientation@QDockWindow@@UAEXW4Orientation@Qt@@@Z 1001e30a f   qt-mt323:qt-mt323.dll
 0001:0001d310       ?setOrientation@QToolBar@@UAEXW4Orientation@Qt@@@Z 1001e310 f   qt-mt323:qt-mt323.dll
 0001:0001d316       ?setPalette@QListView@@UAEXABVQPalette@@@Z 1001e316 f   qt-mt323:qt-mt323.dll
 0001:0001d31c       ?setPalette@QWidget@@UAEXABVQPalette@@@Z 1001e31c f   qt-mt323:qt-mt323.dll
 0001:0001d322       ?setPaletteBackgroundColor@QWidget@@UAEXABVQColor@@@Z 1001e322 f   qt-mt323:qt-mt323.dll
 0001:0001d328       ?setPaletteBackgroundPixmap@QWidget@@UAEXABVQPixmap@@@Z 1001e328 f   qt-mt323:qt-mt323.dll
 0001:0001d32e       ?setPixmap@QListViewItem@@UAEXHABVQPixmap@@@Z 1001e32e f   qt-mt323:qt-mt323.dll
 0001:0001d334       ?setProperty@QObject@@UAE_NPBDABVQVariant@@@Z 1001e334 f   qt-mt323:qt-mt323.dll
 0001:0001d33a       ?setRenameEnabled@QListViewItem@@UAEXH_N@Z 1001e33a f   qt-mt323:qt-mt323.dll
 0001:0001d340       ?setResizeEnabled@QDockWindow@@UAEX_N@Z 1001e340 f   qt-mt323:qt-mt323.dll
 0001:0001d346       ?setResizeMode@QListView@@UAEXW4ResizeMode@1@@Z 1001e346 f   qt-mt323:qt-mt323.dll
 0001:0001d34c       ?setResizePolicy@QScrollView@@UAEXW4ResizePolicy@1@@Z 1001e34c f   qt-mt323:qt-mt323.dll
 0001:0001d352       ?setResolution@QPaintDevice@@UAEXH@Z 1001e352 f   qt-mt323:qt-mt323.dll
 0001:0001d358       ?setRootIsDecorated@QListView@@UAEX_N@Z 1001e358 f   qt-mt323:qt-mt323.dll
 0001:0001d35e       ?setSelectable@QListViewItem@@UAEX_N@Z 1001e35e f   qt-mt323:qt-mt323.dll
 0001:0001d364       ?setSelected@QListView@@UAEXPAVQListViewItem@@_N@Z 1001e364 f   qt-mt323:qt-mt323.dll
 0001:0001d36a       ?setSelected@QListViewItem@@UAEX_N@Z 1001e36a f   qt-mt323:qt-mt323.dll
 0001:0001d370       ?setShowSortIndicator@QListView@@UAEX_N@Z 1001e370 f   qt-mt323:qt-mt323.dll
 0001:0001d376       ?setShowToolTips@QListView@@UAEX_N@Z 1001e376 f   qt-mt323:qt-mt323.dll
 0001:0001d37c       ?setSizeIncrement@QWidget@@UAEXHH@Z 1001e37c f   qt-mt323:qt-mt323.dll
 0001:0001d382       ?setSizePolicy@QWidget@@UAEXVQSizePolicy@@@Z 1001e382 f   qt-mt323:qt-mt323.dll
 0001:0001d388       ?setSorting@QListView@@UAEXH_N@Z 1001e388 f   qt-mt323:qt-mt323.dll
 0001:0001d38e       ?setSpacing@QLayout@@UAEXH@Z 1001e38e f   qt-mt323:qt-mt323.dll
 0001:0001d394       ?setStatusTip@QAction@@UAEXABVQString@@@Z 1001e394 f   qt-mt323:qt-mt323.dll
 0001:0001d39a       ?setStretchableWidget@QToolBar@@UAEXPAVQWidget@@@Z 1001e39a f   qt-mt323:qt-mt323.dll
 0001:0001d3a0       ?setText@QAction@@UAEXABVQString@@@Z 1001e3a0 f   qt-mt323:qt-mt323.dll
 0001:0001d3a6       ?setText@QListViewItem@@UAEXHABVQString@@@Z 1001e3a6 f   qt-mt323:qt-mt323.dll
 0001:0001d3ac       ?setToggleAction@QAction@@UAEX_N@Z 1001e3ac f   qt-mt323:qt-mt323.dll
 0001:0001d3b2       ?setToolTip@QAction@@UAEXABVQString@@@Z 1001e3b2 f   qt-mt323:qt-mt323.dll
 0001:0001d3b8       ?setTreeStepSize@QListView@@UAEXH@Z 1001e3b8 f   qt-mt323:qt-mt323.dll
 0001:0001d3be       ?setUpdatesEnabled@QWidget@@UAEX_N@Z 1001e3be f   qt-mt323:qt-mt323.dll
 0001:0001d3c4       ?setVBarGeometry@QScrollView@@MAEXAAVQScrollBar@@HHHH@Z 1001e3c4 f   qt-mt323:qt-mt323.dll
 0001:0001d3ca       ?setVScrollBarMode@QScrollView@@UAEXW4ScrollBarMode@1@@Z 1001e3ca f   qt-mt323:qt-mt323.dll
 0001:0001d3d0       ?setVerticallyStretchable@QDockWindow@@UAEX_N@Z 1001e3d0 f   qt-mt323:qt-mt323.dll
 0001:0001d3d6       ?setWFlags@QWidget@@MAEXI@Z 1001e3d6 f   qt-mt323:qt-mt323.dll
 0001:0001d3dc       ?setWState@QWidget@@MAEXI@Z 1001e3dc f   qt-mt323:qt-mt323.dll
 0001:0001d3e2       ?setWhatsThis@QAction@@UAEXABVQString@@@Z 1001e3e2 f   qt-mt323:qt-mt323.dll
 0001:0001d3e8       ?setWidget@QDockWindow@@UAEXPAVQWidget@@@Z 1001e3e8 f   qt-mt323:qt-mt323.dll
 0001:0001d3ee       ?setup@QListViewItem@@UAEXXZ 1001e3ee f   qt-mt323:qt-mt323.dll
 0001:0001d3f4       ?show@QListView@@UAEXXZ    1001e3f4 f   qt-mt323:qt-mt323.dll
 0001:0001d3fa       ?show@QPopupMenu@@UAEXXZ   1001e3fa f   qt-mt323:qt-mt323.dll
 0001:0001d400       ?show@QToolBar@@UAEXXZ     1001e400 f   qt-mt323:qt-mt323.dll
 0001:0001d406       ?show@QWidget@@UAEXXZ      1001e406 f   qt-mt323:qt-mt323.dll
 0001:0001d40c       ?showEvent@QDockWindow@@MAEXPAVQShowEvent@@@Z 1001e40c f   qt-mt323:qt-mt323.dll
 0001:0001d412       ?showEvent@QListView@@MAEXPAVQShowEvent@@@Z 1001e412 f   qt-mt323:qt-mt323.dll
 0001:0001d418       ?showEvent@QTabWidget@@MAEXPAVQShowEvent@@@Z 1001e418 f   qt-mt323:qt-mt323.dll
 0001:0001d41e       ?showEvent@QWidget@@MAEXPAVQShowEvent@@@Z 1001e41e f   qt-mt323:qt-mt323.dll
 0001:0001d424       ?showMaximized@QWidget@@UAEXXZ 1001e424 f   qt-mt323:qt-mt323.dll
 0001:0001d42a       ?showMinimized@QWidget@@UAEXXZ 1001e42a f   qt-mt323:qt-mt323.dll
 0001:0001d430       ?showNormal@QWidget@@UAEXXZ 1001e430 f   qt-mt323:qt-mt323.dll
 0001:0001d436       ?showPage@QTabWidget@@UAEXPAVQWidget@@@Z 1001e436 f   qt-mt323:qt-mt323.dll
 0001:0001d43c       ?size@QFile@@UBEKXZ        1001e43c f   qt-mt323:qt-mt323.dll
 0001:0001d442       ?sizeHint@QBoxLayout@@UBE?AVQSize@@XZ 1001e442 f   qt-mt323:qt-mt323.dll
 0001:0001d448       ?sizeHint@QDockWindow@@UBE?AVQSize@@XZ 1001e448 f   qt-mt323:qt-mt323.dll
 0001:0001d44e       ?sizeHint@QHBox@@UBE?AVQSize@@XZ 1001e44e f   qt-mt323:qt-mt323.dll
 0001:0001d454       ?sizeHint@QListView@@UBE?AVQSize@@XZ 1001e454 f   qt-mt323:qt-mt323.dll
 0001:0001d45a       ?sizeHint@QPopupMenu@@UBE?AVQSize@@XZ 1001e45a f   qt-mt323:qt-mt323.dll
 0001:0001d460       ?sizeHint@QTabWidget@@UBE?AVQSize@@XZ 1001e460 f   qt-mt323:qt-mt323.dll
 0001:0001d466       ?sizeHint@QWidget@@UBE?AVQSize@@XZ 1001e466 f   qt-mt323:qt-mt323.dll
 0001:0001d46c       ?sizePolicy@QWidget@@UBE?AVQSizePolicy@@XZ 1001e46c f   qt-mt323:qt-mt323.dll
 0001:0001d472       ?sort@QListView@@UAEXXZ    1001e472 f   qt-mt323:qt-mt323.dll
 0001:0001d478       ?sort@QListViewItem@@UAEXXZ 1001e478 f   qt-mt323:qt-mt323.dll
 0001:0001d47e       ?sortChildItems@QListViewItem@@UAEXH_N@Z 1001e47e f   qt-mt323:qt-mt323.dll
 0001:0001d484       ?spacerItem@QLayoutItem@@UAEPAVQSpacerItem@@XZ 1001e484 f   qt-mt323:qt-mt323.dll
 0001:0001d48a       ?startDrag@QListView@@MAEXXZ 1001e48a f   qt-mt323:qt-mt323.dll
 0001:0001d490       ?startRename@QListViewItem@@UAEXH@Z 1001e490 f   qt-mt323:qt-mt323.dll
 0001:0001d496       ?styleChange@QFrame@@MAEXAAVQStyle@@@Z 1001e496 f   qt-mt323:qt-mt323.dll
 0001:0001d49c       ?styleChange@QListView@@MAEXAAVQStyle@@@Z 1001e49c f   qt-mt323:qt-mt323.dll
 0001:0001d4a2       ?styleChange@QPopupMenu@@MAEXAAVQStyle@@@Z 1001e4a2 f   qt-mt323:qt-mt323.dll
 0001:0001d4a8       ?styleChange@QTabWidget@@MAEXAAVQStyle@@@Z 1001e4a8 f   qt-mt323:qt-mt323.dll
 0001:0001d4ae       ?styleChange@QToolBar@@MAEXAAVQStyle@@@Z 1001e4ae f   qt-mt323:qt-mt323.dll
 0001:0001d4b4       ?styleChange@QWidget@@MAEXAAVQStyle@@@Z 1001e4b4 f   qt-mt323:qt-mt323.dll
 0001:0001d4ba       ?tabletEvent@QWidget@@MAEXPAVQTabletEvent@@@Z 1001e4ba f   qt-mt323:qt-mt323.dll
 0001:0001d4c0       ?takeItem@QListView@@UAEXPAVQListViewItem@@@Z 1001e4c0 f   qt-mt323:qt-mt323.dll
 0001:0001d4c6       ?takeItem@QListViewItem@@UAEXPAV1@@Z 1001e4c6 f   qt-mt323:qt-mt323.dll
 0001:0001d4cc       ?text@QListViewItem@@UBE?AVQString@@H@Z 1001e4cc f   qt-mt323:qt-mt323.dll
 0001:0001d4d2       ?timerEvent@QObject@@MAEXPAVQTimerEvent@@@Z 1001e4d2 f   qt-mt323:qt-mt323.dll
 0001:0001d4d8       ?timerEvent@QPopupMenu@@MAEXPAVQTimerEvent@@@Z 1001e4d8 f   qt-mt323:qt-mt323.dll
 0001:0001d4de       ?undock@QDockWindow@@UAEXPAVQWidget@@@Z 1001e4de f   qt-mt323:qt-mt323.dll
 0001:0001d4e4       ?undock@QDockWindow@@UAEXXZ 1001e4e4 f   qt-mt323:qt-mt323.dll
 0001:0001d4ea       ?ungetch@QFile@@UAEHH@Z    1001e4ea f   qt-mt323:qt-mt323.dll
 0001:0001d4f0       ?unsetCursor@QWidget@@UAEXXZ 1001e4f0 f   qt-mt323:qt-mt323.dll
 0001:0001d4f6       ?updateItem@QPopupMenu@@UAEXH@Z 1001e4f6 f   qt-mt323:qt-mt323.dll
 0001:0001d4fc       ?updateMask@QTabWidget@@MAEXXZ 1001e4fc f   qt-mt323:qt-mt323.dll
 0001:0001d502       ?updateMask@QWidget@@MAEXXZ 1001e502 f   qt-mt323:qt-mt323.dll
 0001:0001d508       ?viewportContextMenuEvent@QScrollView@@MAEXPAVQContextMenuEvent@@@Z 1001e508 f   qt-mt323:qt-mt323.dll
 0001:0001d50e       ?viewportDragEnterEvent@QScrollView@@MAEXPAVQDragEnterEvent@@@Z 1001e50e f   qt-mt323:qt-mt323.dll
 0001:0001d514       ?viewportDragLeaveEvent@QScrollView@@MAEXPAVQDragLeaveEvent@@@Z 1001e514 f   qt-mt323:qt-mt323.dll
 0001:0001d51a       ?viewportDragMoveEvent@QScrollView@@MAEXPAVQDragMoveEvent@@@Z 1001e51a f   qt-mt323:qt-mt323.dll
 0001:0001d520       ?viewportDropEvent@QScrollView@@MAEXPAVQDropEvent@@@Z 1001e520 f   qt-mt323:qt-mt323.dll
 0001:0001d526       ?viewportMouseDoubleClickEvent@QScrollView@@MAEXPAVQMouseEvent@@@Z 1001e526 f   qt-mt323:qt-mt323.dll
 0001:0001d52c       ?viewportMouseMoveEvent@QScrollView@@MAEXPAVQMouseEvent@@@Z 1001e52c f   qt-mt323:qt-mt323.dll
 0001:0001d532       ?viewportMousePressEvent@QScrollView@@MAEXPAVQMouseEvent@@@Z 1001e532 f   qt-mt323:qt-mt323.dll
 0001:0001d538       ?viewportMouseReleaseEvent@QScrollView@@MAEXPAVQMouseEvent@@@Z 1001e538 f   qt-mt323:qt-mt323.dll
 0001:0001d53e       ?viewportPaintEvent@QScrollView@@MAEXPAVQPaintEvent@@@Z 1001e53e f   qt-mt323:qt-mt323.dll
 0001:0001d544       ?viewportResizeEvent@QListView@@MAEXPAVQResizeEvent@@@Z 1001e544 f   qt-mt323:qt-mt323.dll
 0001:0001d54a       ?viewportWheelEvent@QScrollView@@MAEXPAVQWheelEvent@@@Z 1001e54a f   qt-mt323:qt-mt323.dll
 0001:0001d550       ?wheelEvent@QScrollView@@MAEXPAVQWheelEvent@@@Z 1001e550 f   qt-mt323:qt-mt323.dll
 0001:0001d556       ?wheelEvent@QWidget@@MAEXPAVQWheelEvent@@@Z 1001e556 f   qt-mt323:qt-mt323.dll
 0001:0001d55c       ?widget@QLayoutItem@@UAEPAVQWidget@@XZ 1001e55c f   qt-mt323:qt-mt323.dll
 0001:0001d562       ?width@QListViewItem@@UBEHABVQFontMetrics@@PBVQListView@@H@Z 1001e562 f   qt-mt323:qt-mt323.dll
 0001:0001d568       ?winEvent@QWidget@@MAE_NPAUtagMSG@@@Z 1001e568 f   qt-mt323:qt-mt323.dll
 0001:0001d56e       ?windowActivationChange@QListView@@MAEX_N@Z 1001e56e f   qt-mt323:qt-mt323.dll
 0001:0001d574       ?windowActivationChange@QWidget@@MAEX_N@Z 1001e574 f   qt-mt323:qt-mt323.dll
 0001:0001d57a       ?write@QGDict@@MBEAAVQDataStream@@AAV2@PAX@Z 1001e57a f   qt-mt323:qt-mt323.dll
 0001:0001d580       ?write@QGList@@MBEAAVQDataStream@@AAV2@PAX@Z 1001e580 f   qt-mt323:qt-mt323.dll
 0001:0001d586       ?writeBlock@QFile@@UAEJPBDK@Z 1001e586 f   qt-mt323:qt-mt323.dll
 0001:0001d58c       ?first@QSqlQuery@@UAE_NXZ  1001e58c f   qt-mt323:qt-mt323.dll
 0001:0001d592       ?value@QSqlCursor@@UBE?AVQVariant@@H@Z 1001e592 f   qt-mt323:qt-mt323.dll
 0001:0001d598       ?afterSeek@QSqlCursor@@MAEXXZ 1001e598 f   qt-mt323:qt-mt323.dll
 0001:0001d59e       ?append@QSqlCursor@@EAEXABVQSqlField@@@Z 1001e59e f   qt-mt323:qt-mt323.dll
 0001:0001d5a4       ?append@QSqlCursor@@UAEXABVQSqlFieldInfo@@@Z 1001e5a4 f   qt-mt323:qt-mt323.dll
 0001:0001d5aa       ?beforeSeek@QSqlQuery@@MAEXXZ 1001e5aa f   qt-mt323:qt-mt323.dll
 0001:0001d5b0       ?calculateField@QSqlCursor@@MAE?AVQVariant@@ABVQString@@@Z 1001e5b0 f   qt-mt323:qt-mt323.dll
 0001:0001d5b6       ?className@QTimer@@UBEPBDXZ 1001e5b6 f   qt-mt323:qt-mt323.dll
 0001:0001d5bc       ?clear@QSqlCursor@@UAEXXZ  1001e5bc f   qt-mt323:qt-mt323.dll
 0001:0001d5c2       ?clearValues@QSqlRecord@@UAEX_N@Z 1001e5c2 f   qt-mt323:qt-mt323.dll
 0001:0001d5c8       ?del@QSqlCursor@@MAEHABVQString@@_N@Z 1001e5c8 f   qt-mt323:qt-mt323.dll
 0001:0001d5ce       ?del@QSqlCursor@@UAEH_N@Z  1001e5ce f   qt-mt323:qt-mt323.dll
 0001:0001d5d4       ?editBuffer@QSqlCursor@@UAEPAVQSqlRecord@@_N@Z 1001e5d4 f   qt-mt323:qt-mt323.dll
 0001:0001d5da       ?event@QTimer@@MAE_NPAVQEvent@@@Z 1001e5da f   qt-mt323:qt-mt323.dll
 0001:0001d5e0       ?exec@QSqlCursor@@MAE_NABVQString@@@Z 1001e5e0 f   qt-mt323:qt-mt323.dll
 0001:0001d5e6       ?index@QSqlCursor@@UBE?AVQSqlIndex@@ABVQStringList@@@Z 1001e5e6 f   qt-mt323:qt-mt323.dll
 0001:0001d5ec       ?insert@QSqlCursor@@EAEXHABVQSqlField@@@Z 1001e5ec f   qt-mt323:qt-mt323.dll
 0001:0001d5f2       ?insert@QSqlCursor@@UAEH_N@Z 1001e5f2 f   qt-mt323:qt-mt323.dll
 0001:0001d5f8       ?insert@QSqlCursor@@UAEXHABVQSqlFieldInfo@@@Z 1001e5f8 f   qt-mt323:qt-mt323.dll
 0001:0001d5fe       ?last@QSqlQuery@@UAE_NXZ   1001e5fe f   qt-mt323:qt-mt323.dll
 0001:0001d604       ?metaObject@QTimer@@UBEPAVQMetaObject@@XZ 1001e604 f   qt-mt323:qt-mt323.dll
 0001:0001d60a       ?next@QSqlQuery@@UAE_NXZ   1001e60a f   qt-mt323:qt-mt323.dll
 0001:0001d610       ?prev@QSqlQuery@@UAE_NXZ   1001e610 f   qt-mt323:qt-mt323.dll
 0001:0001d616       ?primaryIndex@QSqlCursor@@UBE?AVQSqlIndex@@_N@Z 1001e616 f   qt-mt323:qt-mt323.dll
 0001:0001d61c       ?primeDelete@QSqlCursor@@UAEPAVQSqlRecord@@XZ 1001e61c f   qt-mt323:qt-mt323.dll
 0001:0001d622       ?primeInsert@QSqlCursor@@UAEPAVQSqlRecord@@XZ 1001e622 f   qt-mt323:qt-mt323.dll
 0001:0001d628       ?primeUpdate@QSqlCursor@@UAEPAVQSqlRecord@@XZ 1001e628 f   qt-mt323:qt-mt323.dll
 0001:0001d62e       ?qt_cast@QTimer@@UAEPAXPBD@Z 1001e62e f   qt-mt323:qt-mt323.dll
 0001:0001d634       ?qt_emit@QTimer@@UAE_NHPAUQUObject@@@Z 1001e634 f   qt-mt323:qt-mt323.dll
 0001:0001d63a       ?qt_invoke@QTimer@@UAE_NHPAUQUObject@@@Z 1001e63a f   qt-mt323:qt-mt323.dll
 0001:0001d640       ?qt_property@QTimer@@UAE_NHHPAVQVariant@@@Z 1001e640 f   qt-mt323:qt-mt323.dll
 0001:0001d646       ?remove@QSqlCursor@@UAEXH@Z 1001e646 f   qt-mt323:qt-mt323.dll
 0001:0001d64c       ?seek@QSqlQuery@@UAE_NH_N@Z 1001e64c f   qt-mt323:qt-mt323.dll
 0001:0001d652       ?select@QSqlCursor@@UAE_NABVQString@@ABVQSqlIndex@@@Z 1001e652 f   qt-mt323:qt-mt323.dll
 0001:0001d658       ?setCalculated@QSqlCursor@@UAEXABVQString@@_N@Z 1001e658 f   qt-mt323:qt-mt323.dll
 0001:0001d65e       ?setFilter@QSqlCursor@@UAEXABVQString@@@Z 1001e65e f   qt-mt323:qt-mt323.dll
 0001:0001d664       ?setGenerated@QSqlCursor@@UAEXABVQString@@_N@Z 1001e664 f   qt-mt323:qt-mt323.dll
 0001:0001d66a       ?setGenerated@QSqlCursor@@UAEXH_N@Z 1001e66a f   qt-mt323:qt-mt323.dll
 0001:0001d670       ?setMode@QSqlCursor@@UAEXH@Z 1001e670 f   qt-mt323:qt-mt323.dll
 0001:0001d676       ?setName@QSqlCursor@@UAEXABVQString@@_N@Z 1001e676 f   qt-mt323:qt-mt323.dll
 0001:0001d67c       ?setNull@QSqlRecord@@UAEXABVQString@@@Z 1001e67c f   qt-mt323:qt-mt323.dll
 0001:0001d682       ?setNull@QSqlRecord@@UAEXH@Z 1001e682 f   qt-mt323:qt-mt323.dll
 0001:0001d688       ?setPrimaryIndex@QSqlCursor@@UAEXABVQSqlIndex@@@Z 1001e688 f   qt-mt323:qt-mt323.dll
 0001:0001d68e       ?setSort@QSqlCursor@@UAEXABVQSqlIndex@@@Z 1001e68e f   qt-mt323:qt-mt323.dll
 0001:0001d694       ?setTrimmed@QSqlCursor@@UAEXABVQString@@_N@Z 1001e694 f   qt-mt323:qt-mt323.dll
 0001:0001d69a       ?setValue@QSqlCursor@@UAEXABVQString@@ABVQVariant@@@Z 1001e69a f   qt-mt323:qt-mt323.dll
 0001:0001d6a0       ?setValue@QSqlCursor@@UAEXHABVQVariant@@@Z 1001e6a0 f   qt-mt323:qt-mt323.dll
 0001:0001d6a6       ?toString@QSqlCursor@@MBE?AVQString@@ABV2@PAVQSqlField@@0@Z 1001e6a6 f   qt-mt323:qt-mt323.dll
 0001:0001d6ac       ?toString@QSqlCursor@@MBE?AVQString@@ABVQSqlIndex@@PAVQSqlRecord@@ABV2@22@Z 1001e6ac f   qt-mt323:qt-mt323.dll
 0001:0001d6b2       ?toString@QSqlCursor@@MBE?AVQString@@PAVQSqlRecord@@ABV2@11@Z 1001e6b2 f   qt-mt323:qt-mt323.dll
 0001:0001d6b8       ?toString@QSqlCursor@@UBE?AVQString@@ABV2@0@Z 1001e6b8 f   qt-mt323:qt-mt323.dll
 0001:0001d6be       ?toStringList@QSqlRecord@@UBE?AVQStringList@@ABVQString@@@Z 1001e6be f   qt-mt323:qt-mt323.dll
 0001:0001d6c4       ?update@QSqlCursor@@MAEHABVQString@@_N@Z 1001e6c4 f   qt-mt323:qt-mt323.dll
 0001:0001d6ca       ?update@QSqlCursor@@UAEH_N@Z 1001e6ca f   qt-mt323:qt-mt323.dll
 0001:0001d6d0       ?value@QSqlCursor@@UBE?AVQVariant@@ABVQString@@@Z 1001e6d0 f   qt-mt323:qt-mt323.dll
 0001:0001d6d6       ?accept@QDialog@@MAEXXZ    1001e6d6 f   qt-mt323:qt-mt323.dll
 0001:0001d6dc       ?alignment@QTableItem@@UBEHXZ 1001e6dc f   qt-mt323:qt-mt323.dll
 0001:0001d6e2       ?closeEvent@QDialog@@MAEXPAVQCloseEvent@@@Z 1001e6e2 f   qt-mt323:qt-mt323.dll
 0001:0001d6e8       ?contextMenuEvent@QDialog@@MAEXPAVQContextMenuEvent@@@Z 1001e6e8 f   qt-mt323:qt-mt323.dll
 0001:0001d6ee       ?createEditor@QCheckTableItem@@UBEPAVQWidget@@XZ 1001e6ee f   qt-mt323:qt-mt323.dll
 0001:0001d6f4       ?done@QDialog@@MAEXH@Z     1001e6f4 f   qt-mt323:qt-mt323.dll
 0001:0001d6fa       ?eventFilter@QDialog@@MAE_NPAVQObject@@PAVQEvent@@@Z 1001e6fa f   qt-mt323:qt-mt323.dll
 0001:0001d700       ?hide@QDialog@@UAEXXZ      1001e700 f   qt-mt323:qt-mt323.dll
 0001:0001d706       ?key@QTableItem@@UBE?AVQString@@XZ 1001e706 f   qt-mt323:qt-mt323.dll
 0001:0001d70c       ?keyPressEvent@QDialog@@MAEXPAVQKeyEvent@@@Z 1001e70c f   qt-mt323:qt-mt323.dll
 0001:0001d712       ?minimumSizeHint@QDialog@@UBE?AVQSize@@XZ 1001e712 f   qt-mt323:qt-mt323.dll
 0001:0001d718       ?move@QDialog@@UAEXHH@Z    1001e718 f   qt-mt323:qt-mt323.dll
 0001:0001d71e       ?paint@QCheckTableItem@@UAEXPAVQPainter@@ABVQColorGroup@@ABVQRect@@_N@Z 1001e71e f   qt-mt323:qt-mt323.dll
 0001:0001d724       ?pixmap@QTableItem@@UBE?AVQPixmap@@XZ 1001e724 f   qt-mt323:qt-mt323.dll
 0001:0001d72a       ?reject@QDialog@@MAEXXZ    1001e72a f   qt-mt323:qt-mt323.dll
 0001:0001d730       ?resize@QDialog@@UAEXHH@Z  1001e730 f   qt-mt323:qt-mt323.dll
 0001:0001d736       ?resizeEvent@QDialog@@MAEXPAVQResizeEvent@@@Z 1001e736 f   qt-mt323:qt-mt323.dll
 0001:0001d73c       ?rtti@QCheckTableItem@@UBEHXZ 1001e73c f   qt-mt323:qt-mt323.dll
 0001:0001d742       ?setChecked@QCheckTableItem@@UAEX_N@Z 1001e742 f   qt-mt323:qt-mt323.dll
 0001:0001d748       ?setCol@QTableItem@@UAEXH@Z 1001e748 f   qt-mt323:qt-mt323.dll
 0001:0001d74e       ?setContentFromEditor@QCheckTableItem@@UAEXPAVQWidget@@@Z 1001e74e f   qt-mt323:qt-mt323.dll
 0001:0001d754       ?setEnabled@QTableItem@@UAEX_N@Z 1001e754 f   qt-mt323:qt-mt323.dll
 0001:0001d75a       ?setGeometry@QDialog@@UAEXABVQRect@@@Z 1001e75a f   qt-mt323:qt-mt323.dll
 0001:0001d760       ?setGeometry@QDialog@@UAEXHHHH@Z 1001e760 f   qt-mt323:qt-mt323.dll
 0001:0001d766       ?setPixmap@QTableItem@@UAEXABVQPixmap@@@Z 1001e766 f   qt-mt323:qt-mt323.dll
 0001:0001d76c       ?setReplaceable@QTableItem@@UAEX_N@Z 1001e76c f   qt-mt323:qt-mt323.dll
 0001:0001d772       ?setRow@QTableItem@@UAEXH@Z 1001e772 f   qt-mt323:qt-mt323.dll
 0001:0001d778       ?setSpan@QTableItem@@UAEXHH@Z 1001e778 f   qt-mt323:qt-mt323.dll
 0001:0001d77e       ?setText@QCheckTableItem@@UAEXABVQString@@@Z 1001e77e f   qt-mt323:qt-mt323.dll
 0001:0001d784       ?setWordWrap@QTableItem@@UAEX_N@Z 1001e784 f   qt-mt323:qt-mt323.dll
 0001:0001d78a       ?show@QDialog@@UAEXXZ      1001e78a f   qt-mt323:qt-mt323.dll
 0001:0001d790       ?sizeHint@QCheckTableItem@@UBE?AVQSize@@XZ 1001e790 f   qt-mt323:qt-mt323.dll
 0001:0001d796       ?sizeHint@QDialog@@UBE?AVQSize@@XZ 1001e796 f   qt-mt323:qt-mt323.dll
 0001:0001d79c       ?text@QTableItem@@UBE?AVQString@@XZ 1001e79c f   qt-mt323:qt-mt323.dll
 0001:0001d7a2       ?addItem@QGridLayout@@UAEXPAVQLayoutItem@@@Z 1001e7a2 f   qt-mt323:qt-mt323.dll
 0001:0001d7a8       ?childEvent@QGroupBox@@MAEXPAVQChildEvent@@@Z 1001e7a8 f   qt-mt323:qt-mt323.dll
 0001:0001d7ae       ?className@QCheckBox@@UBEPBDXZ 1001e7ae f   qt-mt323:qt-mt323.dll
 0001:0001d7b4       ?className@QComboBox@@UBEPBDXZ 1001e7b4 f   qt-mt323:qt-mt323.dll
 0001:0001d7ba       ?className@QGridLayout@@UBEPBDXZ 1001e7ba f   qt-mt323:qt-mt323.dll
 0001:0001d7c0       ?className@QGroupBox@@UBEPBDXZ 1001e7c0 f   qt-mt323:qt-mt323.dll
 0001:0001d7c6       ?className@QHBoxLayout@@UBEPBDXZ 1001e7c6 f   qt-mt323:qt-mt323.dll
 0001:0001d7cc       ?className@QLabel@@UBEPBDXZ 1001e7cc f   qt-mt323:qt-mt323.dll
 0001:0001d7d2       ?className@QLineEdit@@UBEPBDXZ 1001e7d2 f   qt-mt323:qt-mt323.dll
 0001:0001d7d8       ?className@QPushButton@@UBEPBDXZ 1001e7d8 f   qt-mt323:qt-mt323.dll
 0001:0001d7de       ?className@QVBoxLayout@@UBEPBDXZ 1001e7de f   qt-mt323:qt-mt323.dll
 0001:0001d7e4       ?clear@QLineEdit@@UAEXXZ   1001e7e4 f   qt-mt323:qt-mt323.dll
 0001:0001d7ea       ?clearValidator@QLineEdit@@UAEXXZ 1001e7ea f   qt-mt323:qt-mt323.dll
 0001:0001d7f0       ?contextMenuEvent@QLineEdit@@MAEXPAVQContextMenuEvent@@@Z 1001e7f0 f   qt-mt323:qt-mt323.dll
 0001:0001d7f6       ?copy@QLineEdit@@UBEXXZ    1001e7f6 f   qt-mt323:qt-mt323.dll
 0001:0001d7fc       ?createPopupMenu@QLineEdit@@MAEPAVQPopupMenu@@XZ 1001e7fc f   qt-mt323:qt-mt323.dll
 0001:0001d802       ?cut@QLineEdit@@UAEXXZ     1001e802 f   qt-mt323:qt-mt323.dll
 0001:0001d808       ?deselect@QLineEdit@@UAEXXZ 1001e808 f   qt-mt323:qt-mt323.dll
 0001:0001d80e       ?dragEnterEvent@QLineEdit@@MAEXPAVQDragEnterEvent@@@Z 1001e80e f   qt-mt323:qt-mt323.dll
 0001:0001d814       ?dragLeaveEvent@QLineEdit@@MAEXPAVQDragLeaveEvent@@@Z 1001e814 f   qt-mt323:qt-mt323.dll
 0001:0001d81a       ?dragMoveEvent@QLineEdit@@MAEXPAVQDragMoveEvent@@@Z 1001e81a f   qt-mt323:qt-mt323.dll
 0001:0001d820       ?drawButton@QCheckBox@@MAEXPAVQPainter@@@Z 1001e820 f   qt-mt323:qt-mt323.dll
 0001:0001d826       ?drawButton@QPushButton@@MAEXPAVQPainter@@@Z 1001e826 f   qt-mt323:qt-mt323.dll
 0001:0001d82c       ?drawButtonLabel@QCheckBox@@MAEXPAVQPainter@@@Z 1001e82c f   qt-mt323:qt-mt323.dll
 0001:0001d832       ?drawButtonLabel@QPushButton@@MAEXPAVQPainter@@@Z 1001e832 f   qt-mt323:qt-mt323.dll
 0001:0001d838       ?drawContents@QLabel@@MAEXPAVQPainter@@@Z 1001e838 f   qt-mt323:qt-mt323.dll
 0001:0001d83e       ?drawContents@QLineEdit@@MAEXPAVQPainter@@@Z 1001e83e f   qt-mt323:qt-mt323.dll
 0001:0001d844       ?dropEvent@QLineEdit@@MAEXPAVQDropEvent@@@Z 1001e844 f   qt-mt323:qt-mt323.dll
 0001:0001d84a       ?enabledChange@QButton@@MAEX_N@Z 1001e84a f   qt-mt323:qt-mt323.dll
 0001:0001d850       ?event@QGroupBox@@MAE_NPAVQEvent@@@Z 1001e850 f   qt-mt323:qt-mt323.dll
 0001:0001d856       ?event@QLineEdit@@MAE_NPAVQEvent@@@Z 1001e856 f   qt-mt323:qt-mt323.dll
 0001:0001d85c       ?eventFilter@QComboBox@@UAE_NPAVQObject@@PAVQEvent@@@Z 1001e85c f   qt-mt323:qt-mt323.dll
 0001:0001d862       ?expanding@QGridLayout@@UBE?AW4ExpandData@QSizePolicy@@XZ 1001e862 f   qt-mt323:qt-mt323.dll
 0001:0001d868       ?expanding@QSpacerItem@@UBE?AW4ExpandData@QSizePolicy@@XZ 1001e868 f   qt-mt323:qt-mt323.dll
 0001:0001d86e       ?focusInEvent@QButton@@MAEXPAVQFocusEvent@@@Z 1001e86e f   qt-mt323:qt-mt323.dll
 0001:0001d874       ?focusInEvent@QComboBox@@MAEXPAVQFocusEvent@@@Z 1001e874 f   qt-mt323:qt-mt323.dll
 0001:0001d87a       ?focusInEvent@QGroupBox@@MAEXPAVQFocusEvent@@@Z 1001e87a f   qt-mt323:qt-mt323.dll
 0001:0001d880       ?focusInEvent@QLineEdit@@MAEXPAVQFocusEvent@@@Z 1001e880 f   qt-mt323:qt-mt323.dll
 0001:0001d886       ?focusInEvent@QPushButton@@MAEXPAVQFocusEvent@@@Z 1001e886 f   qt-mt323:qt-mt323.dll
 0001:0001d88c       ?focusOutEvent@QButton@@MAEXPAVQFocusEvent@@@Z 1001e88c f   qt-mt323:qt-mt323.dll
 0001:0001d892       ?focusOutEvent@QComboBox@@MAEXPAVQFocusEvent@@@Z 1001e892 f   qt-mt323:qt-mt323.dll
 0001:0001d898       ?focusOutEvent@QLineEdit@@MAEXPAVQFocusEvent@@@Z 1001e898 f   qt-mt323:qt-mt323.dll
 0001:0001d89e       ?focusOutEvent@QPushButton@@MAEXPAVQFocusEvent@@@Z 1001e89e f   qt-mt323:qt-mt323.dll
 0001:0001d8a4       ?fontChange@QGroupBox@@MAEXABVQFont@@@Z 1001e8a4 f   qt-mt323:qt-mt323.dll
 0001:0001d8aa       ?fontChange@QLabel@@MAEXABVQFont@@@Z 1001e8aa f   qt-mt323:qt-mt323.dll
 0001:0001d8b0       ?geometry@QSpacerItem@@UBE?AVQRect@@XZ 1001e8b0 f   qt-mt323:qt-mt323.dll
 0001:0001d8b6       ?hasHeightForWidth@QGridLayout@@UBE_NXZ 1001e8b6 f   qt-mt323:qt-mt323.dll
 0001:0001d8bc       ?hasHeightForWidth@QLayoutItem@@UBE_NXZ 1001e8bc f   qt-mt323:qt-mt323.dll
 0001:0001d8c2       ?heightForWidth@QGridLayout@@UBEHH@Z 1001e8c2 f   qt-mt323:qt-mt323.dll
 0001:0001d8c8       ?heightForWidth@QLabel@@UBEHH@Z 1001e8c8 f   qt-mt323:qt-mt323.dll
 0001:0001d8ce       ?heightForWidth@QLayoutItem@@UBEHH@Z 1001e8ce f   qt-mt323:qt-mt323.dll
 0001:0001d8d4       ?hitButton@QButton@@MBE_NABVQPoint@@@Z 1001e8d4 f   qt-mt323:qt-mt323.dll
 0001:0001d8da       ?hitButton@QCheckBox@@MBE_NABVQPoint@@@Z 1001e8da f   qt-mt323:qt-mt323.dll
 0001:0001d8e0       ?imComposeEvent@QLineEdit@@MAEXPAVQIMEvent@@@Z 1001e8e0 f   qt-mt323:qt-mt323.dll
 0001:0001d8e6       ?imEndEvent@QLineEdit@@MAEXPAVQIMEvent@@@Z 1001e8e6 f   qt-mt323:qt-mt323.dll
 0001:0001d8ec       ?imStartEvent@QLineEdit@@MAEXPAVQIMEvent@@@Z 1001e8ec f   qt-mt323:qt-mt323.dll
 0001:0001d8f2       ?insert@QLineEdit@@UAEXABVQString@@@Z 1001e8f2 f   qt-mt323:qt-mt323.dll
 0001:0001d8f8       ?invalidate@QGridLayout@@UAEXXZ 1001e8f8 f   qt-mt323:qt-mt323.dll
 0001:0001d8fe       ?invalidate@QLayoutItem@@UAEXXZ 1001e8fe f   qt-mt323:qt-mt323.dll
 0001:0001d904       ?isEmpty@QSpacerItem@@UBE_NXZ 1001e904 f   qt-mt323:qt-mt323.dll
 0001:0001d90a       ?iterator@QGridLayout@@UAE?AVQLayoutIterator@@XZ 1001e90a f   qt-mt323:qt-mt323.dll
 0001:0001d910       ?iterator@QLayoutItem@@UAE?AVQLayoutIterator@@XZ 1001e910 f   qt-mt323:qt-mt323.dll
 0001:0001d916       ?keyPressEvent@QButton@@MAEXPAVQKeyEvent@@@Z 1001e916 f   qt-mt323:qt-mt323.dll
 0001:0001d91c       ?keyPressEvent@QComboBox@@MAEXPAVQKeyEvent@@@Z 1001e91c f   qt-mt323:qt-mt323.dll
 0001:0001d922       ?keyPressEvent@QLineEdit@@MAEXPAVQKeyEvent@@@Z 1001e922 f   qt-mt323:qt-mt323.dll
 0001:0001d928       ?keyReleaseEvent@QButton@@MAEXPAVQKeyEvent@@@Z 1001e928 f   qt-mt323:qt-mt323.dll
 0001:0001d92e       ?layout@QLayoutItem@@UAEPAVQLayout@@XZ 1001e92e f   qt-mt323:qt-mt323.dll
 0001:0001d934       ?maximumSize@QGridLayout@@UBE?AVQSize@@XZ 1001e934 f   qt-mt323:qt-mt323.dll
 0001:0001d93a       ?maximumSize@QSpacerItem@@UBE?AVQSize@@XZ 1001e93a f   qt-mt323:qt-mt323.dll
 0001:0001d940       ?metaObject@QCheckBox@@UBEPAVQMetaObject@@XZ 1001e940 f   qt-mt323:qt-mt323.dll
 0001:0001d946       ?metaObject@QComboBox@@UBEPAVQMetaObject@@XZ 1001e946 f   qt-mt323:qt-mt323.dll
 0001:0001d94c       ?metaObject@QGridLayout@@UBEPAVQMetaObject@@XZ 1001e94c f   qt-mt323:qt-mt323.dll
 0001:0001d952       ?metaObject@QGroupBox@@UBEPAVQMetaObject@@XZ 1001e952 f   qt-mt323:qt-mt323.dll
 0001:0001d958       ?metaObject@QHBoxLayout@@UBEPAVQMetaObject@@XZ 1001e958 f   qt-mt323:qt-mt323.dll
 0001:0001d95e       ?metaObject@QLabel@@UBEPAVQMetaObject@@XZ 1001e95e f   qt-mt323:qt-mt323.dll
 0001:0001d964       ?metaObject@QLineEdit@@UBEPAVQMetaObject@@XZ 1001e964 f   qt-mt323:qt-mt323.dll
 0001:0001d96a       ?metaObject@QPushButton@@UBEPAVQMetaObject@@XZ 1001e96a f   qt-mt323:qt-mt323.dll
 0001:0001d970       ?metaObject@QVBoxLayout@@UBEPAVQMetaObject@@XZ 1001e970 f   qt-mt323:qt-mt323.dll
 0001:0001d976       ?minimumSize@QGridLayout@@UBE?AVQSize@@XZ 1001e976 f   qt-mt323:qt-mt323.dll
 0001:0001d97c       ?minimumSize@QSpacerItem@@UBE?AVQSize@@XZ 1001e97c f   qt-mt323:qt-mt323.dll
 0001:0001d982       ?minimumSizeHint@QLabel@@UBE?AVQSize@@XZ 1001e982 f   qt-mt323:qt-mt323.dll
 0001:0001d988       ?minimumSizeHint@QLineEdit@@UBE?AVQSize@@XZ 1001e988 f   qt-mt323:qt-mt323.dll
 0001:0001d98e       ?mouseDoubleClickEvent@QComboBox@@MAEXPAVQMouseEvent@@@Z 1001e98e f   qt-mt323:qt-mt323.dll
 0001:0001d994       ?mouseDoubleClickEvent@QLineEdit@@MAEXPAVQMouseEvent@@@Z 1001e994 f   qt-mt323:qt-mt323.dll
 0001:0001d99a       ?mouseMoveEvent@QButton@@MAEXPAVQMouseEvent@@@Z 1001e99a f   qt-mt323:qt-mt323.dll
 0001:0001d9a0       ?mouseMoveEvent@QComboBox@@MAEXPAVQMouseEvent@@@Z 1001e9a0 f   qt-mt323:qt-mt323.dll
 0001:0001d9a6       ?mouseMoveEvent@QLineEdit@@MAEXPAVQMouseEvent@@@Z 1001e9a6 f   qt-mt323:qt-mt323.dll
 0001:0001d9ac       ?mousePressEvent@QButton@@MAEXPAVQMouseEvent@@@Z 1001e9ac f   qt-mt323:qt-mt323.dll
 0001:0001d9b2       ?mousePressEvent@QComboBox@@MAEXPAVQMouseEvent@@@Z 1001e9b2 f   qt-mt323:qt-mt323.dll
 0001:0001d9b8       ?mousePressEvent@QLineEdit@@MAEXPAVQMouseEvent@@@Z 1001e9b8 f   qt-mt323:qt-mt323.dll
 0001:0001d9be       ?mouseReleaseEvent@QButton@@MAEXPAVQMouseEvent@@@Z 1001e9be f   qt-mt323:qt-mt323.dll
 0001:0001d9c4       ?mouseReleaseEvent@QComboBox@@MAEXPAVQMouseEvent@@@Z 1001e9c4 f   qt-mt323:qt-mt323.dll
 0001:0001d9ca       ?mouseReleaseEvent@QLineEdit@@MAEXPAVQMouseEvent@@@Z 1001e9ca f   qt-mt323:qt-mt323.dll
 0001:0001d9d0       ?move@QPushButton@@UAEXHH@Z 1001e9d0 f   qt-mt323:qt-mt323.dll
 0001:0001d9d6       ?paintEvent@QButton@@MAEXPAVQPaintEvent@@@Z 1001e9d6 f   qt-mt323:qt-mt323.dll
 0001:0001d9dc       ?paintEvent@QComboBox@@MAEXPAVQPaintEvent@@@Z 1001e9dc f   qt-mt323:qt-mt323.dll
 0001:0001d9e2       ?paintEvent@QGroupBox@@MAEXPAVQPaintEvent@@@Z 1001e9e2 f   qt-mt323:qt-mt323.dll
 0001:0001d9e8       ?paste@QLineEdit@@UAEXXZ   1001e9e8 f   qt-mt323:qt-mt323.dll
 0001:0001d9ee       ?popup@QComboBox@@UAEXXZ   1001e9ee f   qt-mt323:qt-mt323.dll
 0001:0001d9f4       ?qt_cast@QCheckBox@@UAEPAXPBD@Z 1001e9f4 f   qt-mt323:qt-mt323.dll
 0001:0001d9fa       ?qt_cast@QComboBox@@UAEPAXPBD@Z 1001e9fa f   qt-mt323:qt-mt323.dll
 0001:0001da00       ?qt_cast@QGridLayout@@UAEPAXPBD@Z 1001ea00 f   qt-mt323:qt-mt323.dll
 0001:0001da06       ?qt_cast@QGroupBox@@UAEPAXPBD@Z 1001ea06 f   qt-mt323:qt-mt323.dll
 0001:0001da0c       ?qt_cast@QHBoxLayout@@UAEPAXPBD@Z 1001ea0c f   qt-mt323:qt-mt323.dll
 0001:0001da12       ?qt_cast@QLabel@@UAEPAXPBD@Z 1001ea12 f   qt-mt323:qt-mt323.dll
 0001:0001da18       ?qt_cast@QLineEdit@@UAEPAXPBD@Z 1001ea18 f   qt-mt323:qt-mt323.dll
 0001:0001da1e       ?qt_cast@QPushButton@@UAEPAXPBD@Z 1001ea1e f   qt-mt323:qt-mt323.dll
 0001:0001da24       ?qt_cast@QVBoxLayout@@UAEPAXPBD@Z 1001ea24 f   qt-mt323:qt-mt323.dll
 0001:0001da2a       ?qt_emit@QCheckBox@@UAE_NHPAUQUObject@@@Z 1001ea2a f   qt-mt323:qt-mt323.dll
 0001:0001da30       ?qt_emit@QComboBox@@UAE_NHPAUQUObject@@@Z 1001ea30 f   qt-mt323:qt-mt323.dll
 0001:0001da36       ?qt_emit@QGridLayout@@UAE_NHPAUQUObject@@@Z 1001ea36 f   qt-mt323:qt-mt323.dll
 0001:0001da3c       ?qt_emit@QGroupBox@@UAE_NHPAUQUObject@@@Z 1001ea3c f   qt-mt323:qt-mt323.dll
 0001:0001da42       ?qt_emit@QHBoxLayout@@UAE_NHPAUQUObject@@@Z 1001ea42 f   qt-mt323:qt-mt323.dll
 0001:0001da48       ?qt_emit@QLabel@@UAE_NHPAUQUObject@@@Z 1001ea48 f   qt-mt323:qt-mt323.dll
 0001:0001da4e       ?qt_emit@QLineEdit@@UAE_NHPAUQUObject@@@Z 1001ea4e f   qt-mt323:qt-mt323.dll
 0001:0001da54       ?qt_emit@QPushButton@@UAE_NHPAUQUObject@@@Z 1001ea54 f   qt-mt323:qt-mt323.dll
 0001:0001da5a       ?qt_emit@QVBoxLayout@@UAE_NHPAUQUObject@@@Z 1001ea5a f   qt-mt323:qt-mt323.dll
 0001:0001da60       ?qt_invoke@QCheckBox@@UAE_NHPAUQUObject@@@Z 1001ea60 f   qt-mt323:qt-mt323.dll
 0001:0001da66       ?qt_invoke@QComboBox@@UAE_NHPAUQUObject@@@Z 1001ea66 f   qt-mt323:qt-mt323.dll
 0001:0001da6c       ?qt_invoke@QGridLayout@@UAE_NHPAUQUObject@@@Z 1001ea6c f   qt-mt323:qt-mt323.dll
 0001:0001da72       ?qt_invoke@QGroupBox@@UAE_NHPAUQUObject@@@Z 1001ea72 f   qt-mt323:qt-mt323.dll
 0001:0001da78       ?qt_invoke@QHBoxLayout@@UAE_NHPAUQUObject@@@Z 1001ea78 f   qt-mt323:qt-mt323.dll
 0001:0001da7e       ?qt_invoke@QLabel@@UAE_NHPAUQUObject@@@Z 1001ea7e f   qt-mt323:qt-mt323.dll
 0001:0001da84       ?qt_invoke@QLineEdit@@UAE_NHPAUQUObject@@@Z 1001ea84 f   qt-mt323:qt-mt323.dll
 0001:0001da8a       ?qt_invoke@QPushButton@@UAE_NHPAUQUObject@@@Z 1001ea8a f   qt-mt323:qt-mt323.dll
 0001:0001da90       ?qt_invoke@QVBoxLayout@@UAE_NHPAUQUObject@@@Z 1001ea90 f   qt-mt323:qt-mt323.dll
 0001:0001da96       ?qt_property@QCheckBox@@UAE_NHHPAVQVariant@@@Z 1001ea96 f   qt-mt323:qt-mt323.dll
 0001:0001da9c       ?qt_property@QComboBox@@UAE_NHHPAVQVariant@@@Z 1001ea9c f   qt-mt323:qt-mt323.dll
 0001:0001daa2       ?qt_property@QGridLayout@@UAE_NHHPAVQVariant@@@Z 1001eaa2 f   qt-mt323:qt-mt323.dll
 0001:0001daa8       ?qt_property@QGroupBox@@UAE_NHHPAVQVariant@@@Z 1001eaa8 f   qt-mt323:qt-mt323.dll
 0001:0001daae       ?qt_property@QHBoxLayout@@UAE_NHHPAVQVariant@@@Z 1001eaae f   qt-mt323:qt-mt323.dll
 0001:0001dab4       ?qt_property@QLabel@@UAE_NHHPAVQVariant@@@Z 1001eab4 f   qt-mt323:qt-mt323.dll
 0001:0001daba       ?qt_property@QLineEdit@@UAE_NHHPAVQVariant@@@Z 1001eaba f   qt-mt323:qt-mt323.dll
 0001:0001dac0       ?qt_property@QPushButton@@UAE_NHHPAVQVariant@@@Z 1001eac0 f   qt-mt323:qt-mt323.dll
 0001:0001dac6       ?qt_property@QVBoxLayout@@UAE_NHHPAVQVariant@@@Z 1001eac6 f   qt-mt323:qt-mt323.dll
 0001:0001dacc       ?redo@QLineEdit@@UAEXXZ    1001eacc f   qt-mt323:qt-mt323.dll
 0001:0001dad2       ?resize@QPushButton@@UAEXHH@Z 1001ead2 f   qt-mt323:qt-mt323.dll
 0001:0001dad8       ?resizeEvent@QCheckBox@@MAEXPAVQResizeEvent@@@Z 1001ead8 f   qt-mt323:qt-mt323.dll
 0001:0001dade       ?resizeEvent@QComboBox@@MAEXPAVQResizeEvent@@@Z 1001eade f   qt-mt323:qt-mt323.dll
 0001:0001dae4       ?resizeEvent@QGroupBox@@MAEXPAVQResizeEvent@@@Z 1001eae4 f   qt-mt323:qt-mt323.dll
 0001:0001daea       ?resizeEvent@QLabel@@MAEXPAVQResizeEvent@@@Z 1001eaea f   qt-mt323:qt-mt323.dll
 0001:0001daf0       ?resizeEvent@QLineEdit@@MAEXPAVQResizeEvent@@@Z 1001eaf0 f   qt-mt323:qt-mt323.dll
 0001:0001daf6       ?resizeEvent@QPushButton@@MAEXPAVQResizeEvent@@@Z 1001eaf6 f   qt-mt323:qt-mt323.dll
 0001:0001dafc       ?selectAll@QLineEdit@@UAEXXZ 1001eafc f   qt-mt323:qt-mt323.dll
 0001:0001db02       ?setAccel@QButton@@UAEXABVQKeySequence@@@Z 1001eb02 f   qt-mt323:qt-mt323.dll
 0001:0001db08       ?setAlignment@QGroupBox@@UAEXH@Z 1001eb08 f   qt-mt323:qt-mt323.dll
 0001:0001db0e       ?setAlignment@QLabel@@UAEXH@Z 1001eb0e f   qt-mt323:qt-mt323.dll
 0001:0001db14       ?setAlignment@QLineEdit@@UAEXH@Z 1001eb14 f   qt-mt323:qt-mt323.dll
 0001:0001db1a       ?setAutoCompletion@QComboBox@@UAEX_N@Z 1001eb1a f   qt-mt323:qt-mt323.dll
 0001:0001db20       ?setAutoDefault@QPushButton@@UAEX_N@Z 1001eb20 f   qt-mt323:qt-mt323.dll
 0001:0001db26       ?setAutoRepeat@QButton@@UAEX_N@Z 1001eb26 f   qt-mt323:qt-mt323.dll
 0001:0001db2c       ?setAutoResize@QComboBox@@UAEX_N@Z 1001eb2c f   qt-mt323:qt-mt323.dll
 0001:0001db32       ?setAutoResize@QLabel@@UAEX_N@Z 1001eb32 f   qt-mt323:qt-mt323.dll
 0001:0001db38       ?setBuddy@QLabel@@UAEXPAVQWidget@@@Z 1001eb38 f   qt-mt323:qt-mt323.dll
 0001:0001db3e       ?setColStretch@QGridLayout@@UAEXHH@Z 1001eb3e f   qt-mt323:qt-mt323.dll
 0001:0001db44       ?setColumnLayout@QGroupBox@@UAEXHW4Orientation@Qt@@@Z 1001eb44 f   qt-mt323:qt-mt323.dll
 0001:0001db4a       ?setCurrentItem@QComboBox@@UAEXH@Z 1001eb4a f   qt-mt323:qt-mt323.dll
 0001:0001db50       ?setCurrentText@QComboBox@@UAEXABVQString@@@Z 1001eb50 f   qt-mt323:qt-mt323.dll
 0001:0001db56       ?setCursorPosition@QLineEdit@@UAEXH@Z 1001eb56 f   qt-mt323:qt-mt323.dll
 0001:0001db5c       ?setDefault@QPushButton@@UAEX_N@Z 1001eb5c f   qt-mt323:qt-mt323.dll
 0001:0001db62       ?setDown@QButton@@UAEX_N@Z 1001eb62 f   qt-mt323:qt-mt323.dll
 0001:0001db68       ?setDragEnabled@QLineEdit@@UAEX_N@Z 1001eb68 f   qt-mt323:qt-mt323.dll
 0001:0001db6e       ?setEchoMode@QLineEdit@@UAEXW4EchoMode@1@@Z 1001eb6e f   qt-mt323:qt-mt323.dll
 0001:0001db74       ?setEditText@QComboBox@@UAEXABVQString@@@Z 1001eb74 f   qt-mt323:qt-mt323.dll
 0001:0001db7a       ?setEnabled@QComboBox@@UAEX_N@Z 1001eb7a f   qt-mt323:qt-mt323.dll
 0001:0001db80       ?setEnabled@QGroupBox@@UAEX_N@Z 1001eb80 f   qt-mt323:qt-mt323.dll
 0001:0001db86       ?setFont@QComboBox@@UAEXABVQFont@@@Z 1001eb86 f   qt-mt323:qt-mt323.dll
 0001:0001db8c       ?setFont@QLabel@@UAEXABVQFont@@@Z 1001eb8c f   qt-mt323:qt-mt323.dll
 0001:0001db92       ?setFont@QLineEdit@@UAEXABVQFont@@@Z 1001eb92 f   qt-mt323:qt-mt323.dll
 0001:0001db98       ?setFrame@QLineEdit@@UAEX_N@Z 1001eb98 f   qt-mt323:qt-mt323.dll
 0001:0001db9e       ?setGeometry@QGridLayout@@UAEXABVQRect@@@Z 1001eb9e f   qt-mt323:qt-mt323.dll
 0001:0001dba4       ?setGeometry@QPushButton@@UAEXABVQRect@@@Z 1001eba4 f   qt-mt323:qt-mt323.dll
 0001:0001dbaa       ?setGeometry@QPushButton@@UAEXHHHH@Z 1001ebaa f   qt-mt323:qt-mt323.dll
 0001:0001dbb0       ?setGeometry@QSpacerItem@@UAEXABVQRect@@@Z 1001ebb0 f   qt-mt323:qt-mt323.dll
 0001:0001dbb6       ?setGroup@QButton@@EAEXPAVQButtonGroup@@@Z 1001ebb6 f   qt-mt323:qt-mt323.dll
 0001:0001dbbc       ?setInsertionPolicy@QComboBox@@UAEXW4Policy@1@@Z 1001ebbc f   qt-mt323:qt-mt323.dll
 0001:0001dbc2       ?setIsMenuButton@QPushButton@@UAEX_N@Z 1001ebc2 f   qt-mt323:qt-mt323.dll
 0001:0001dbc8       ?setLineEdit@QComboBox@@UAEXPAVQLineEdit@@@Z 1001ebc8 f   qt-mt323:qt-mt323.dll
 0001:0001dbce       ?setListBox@QComboBox@@UAEXPAVQListBox@@@Z 1001ebce f   qt-mt323:qt-mt323.dll
 0001:0001dbd4       ?setMaxCount@QComboBox@@UAEXH@Z 1001ebd4 f   qt-mt323:qt-mt323.dll
 0001:0001dbda       ?setMaxLength@QLineEdit@@UAEXH@Z 1001ebda f   qt-mt323:qt-mt323.dll
 0001:0001dbe0       ?setMovie@QLabel@@UAEXABVQMovie@@@Z 1001ebe0 f   qt-mt323:qt-mt323.dll
 0001:0001dbe6       ?setNum@QLabel@@UAEXH@Z    1001ebe6 f   qt-mt323:qt-mt323.dll
 0001:0001dbec       ?setNum@QLabel@@UAEXN@Z    1001ebec f   qt-mt323:qt-mt323.dll
 0001:0001dbf2       ?setOn@QPushButton@@UAEX_N@Z 1001ebf2 f   qt-mt323:qt-mt323.dll
 0001:0001dbf8       ?setPalette@QComboBox@@UAEXABVQPalette@@@Z 1001ebf8 f   qt-mt323:qt-mt323.dll
 0001:0001dbfe       ?setPalette@QLineEdit@@UAEXABVQPalette@@@Z 1001ebfe f   qt-mt323:qt-mt323.dll
 0001:0001dc04       ?setPicture@QLabel@@UAEXABVQPicture@@@Z 1001ec04 f   qt-mt323:qt-mt323.dll
 0001:0001dc0a       ?setPixmap@QButton@@UAEXABVQPixmap@@@Z 1001ec0a f   qt-mt323:qt-mt323.dll
 0001:0001dc10       ?setPixmap@QLabel@@UAEXABVQPixmap@@@Z 1001ec10 f   qt-mt323:qt-mt323.dll
 0001:0001dc16       ?setReadOnly@QLineEdit@@UAEX_N@Z 1001ec16 f   qt-mt323:qt-mt323.dll
 0001:0001dc1c       ?setRowStretch@QGridLayout@@UAEXHH@Z 1001ec1c f   qt-mt323:qt-mt323.dll
 0001:0001dc22       ?setSelection@QLineEdit@@UAEXHH@Z 1001ec22 f   qt-mt323:qt-mt323.dll
 0001:0001dc28       ?setSizeLimit@QComboBox@@UAEXH@Z 1001ec28 f   qt-mt323:qt-mt323.dll
 0001:0001dc2e       ?setState@QButton@@MAEXW4ToggleState@1@@Z 1001ec2e f   qt-mt323:qt-mt323.dll
 0001:0001dc34       ?setText@QButton@@UAEXABVQString@@@Z 1001ec34 f   qt-mt323:qt-mt323.dll
 0001:0001dc3a       ?setText@QLabel@@UAEXABVQString@@@Z 1001ec3a f   qt-mt323:qt-mt323.dll
 0001:0001dc40       ?setText@QLineEdit@@UAEXABVQString@@@Z 1001ec40 f   qt-mt323:qt-mt323.dll
 0001:0001dc46       ?setTitle@QGroupBox@@UAEXABVQString@@@Z 1001ec46 f   qt-mt323:qt-mt323.dll
 0001:0001dc4c       ?setToggleType@QButton@@MAEXW4ToggleType@1@@Z 1001ec4c f   qt-mt323:qt-mt323.dll
 0001:0001dc52       ?setValidator@QComboBox@@UAEXPBVQValidator@@@Z 1001ec52 f   qt-mt323:qt-mt323.dll
 0001:0001dc58       ?setValidator@QLineEdit@@UAEXPBVQValidator@@@Z 1001ec58 f   qt-mt323:qt-mt323.dll
 0001:0001dc5e       ?sizeHint@QCheckBox@@UBE?AVQSize@@XZ 1001ec5e f   qt-mt323:qt-mt323.dll
 0001:0001dc64       ?sizeHint@QComboBox@@UBE?AVQSize@@XZ 1001ec64 f   qt-mt323:qt-mt323.dll
 0001:0001dc6a       ?sizeHint@QGridLayout@@UBE?AVQSize@@XZ 1001ec6a f   qt-mt323:qt-mt323.dll
 0001:0001dc70       ?sizeHint@QGroupBox@@UBE?AVQSize@@XZ 1001ec70 f   qt-mt323:qt-mt323.dll
 0001:0001dc76       ?sizeHint@QLabel@@UBE?AVQSize@@XZ 1001ec76 f   qt-mt323:qt-mt323.dll
 0001:0001dc7c       ?sizeHint@QLineEdit@@UBE?AVQSize@@XZ 1001ec7c f   qt-mt323:qt-mt323.dll
 0001:0001dc82       ?sizeHint@QPushButton@@UBE?AVQSize@@XZ 1001ec82 f   qt-mt323:qt-mt323.dll
 0001:0001dc88       ?sizeHint@QSpacerItem@@UBE?AVQSize@@XZ 1001ec88 f   qt-mt323:qt-mt323.dll
 0001:0001dc8e       ?spacerItem@QSpacerItem@@UAEPAV1@XZ 1001ec8e f   qt-mt323:qt-mt323.dll
 0001:0001dc94       ?styleChange@QComboBox@@MAEXAAVQStyle@@@Z 1001ec94 f   qt-mt323:qt-mt323.dll
 0001:0001dc9a       ?undo@QLineEdit@@UAEXXZ    1001ec9a f   qt-mt323:qt-mt323.dll
 0001:0001dca0       ?updateMask@QCheckBox@@MAEXXZ 1001eca0 f   qt-mt323:qt-mt323.dll
 0001:0001dca6       ?updateMask@QComboBox@@MAEXXZ 1001eca6 f   qt-mt323:qt-mt323.dll
 0001:0001dcac       ?updateMask@QPushButton@@MAEXXZ 1001ecac f   qt-mt323:qt-mt323.dll
 0001:0001dcb2       ?wheelEvent@QComboBox@@MAEXPAVQWheelEvent@@@Z 1001ecb2 f   qt-mt323:qt-mt323.dll
 0001:0001dcb8       ?windowActivationChange@QLineEdit@@MAEX_N@Z 1001ecb8 f   qt-mt323:qt-mt323.dll
 0001:0001dcbe       ?activateNextCell@QDataTable@@MAEXXZ 1001ecbe f   qt-mt323:qt-mt323.dll
 0001:0001dcc4       ?addColumn@QDataTable@@UAEXABVQString@@0HABVQIconSet@@@Z 1001ecc4 f   qt-mt323:qt-mt323.dll
 0001:0001dcca       ?addNumber@QDateEdit@@MAEXHH@Z 1001ecca f   qt-mt323:qt-mt323.dll
 0001:0001dcd0       ?addSelection@QTable@@UAEHABVQTableSelection@@@Z 1001ecd0 f   qt-mt323:qt-mt323.dll
 0001:0001dcd6       ?adjustColumn@QDataTable@@UAEXH@Z 1001ecd6 f   qt-mt323:qt-mt323.dll
 0001:0001dcdc       ?adjustRow@QTable@@UAEXH@Z 1001ecdc f   qt-mt323:qt-mt323.dll
 0001:0001dce2       ?beginEdit@QDataTable@@EAEPAVQWidget@@HH_N@Z 1001ece2 f   qt-mt323:qt-mt323.dll
 0001:0001dce8       ?beginInsert@QDataTable@@MAE_NXZ 1001ece8 f   qt-mt323:qt-mt323.dll
 0001:0001dcee       ?beginUpdate@QDataTable@@MAEPAVQWidget@@HH_N@Z 1001ecee f   qt-mt323:qt-mt323.dll
 0001:0001dcf4       ?cellGeometry@QTable@@UBE?AVQRect@@HH@Z 1001ecf4 f   qt-mt323:qt-mt323.dll
 0001:0001dcfa       ?cellRect@QTable@@UBE?AVQRect@@HH@Z 1001ecfa f   qt-mt323:qt-mt323.dll
 0001:0001dd00       ?cellWidget@QTable@@UBEPAVQWidget@@HH@Z 1001ed00 f   qt-mt323:qt-mt323.dll
 0001:0001dd06       ?childEvent@QSplitter@@MAEXPAVQChildEvent@@@Z 1001ed06 f   qt-mt323:qt-mt323.dll
 0001:0001dd0c       ?className@QButtonGroup@@UBEPBDXZ 1001ed0c f   qt-mt323:qt-mt323.dll
 0001:0001dd12       ?className@QDataTable@@UBEPBDXZ 1001ed12 f   qt-mt323:qt-mt323.dll
 0001:0001dd18       ?className@QDateEdit@@UBEPBDXZ 1001ed18 f   qt-mt323:qt-mt323.dll
 0001:0001dd1e       ?className@QRadioButton@@UBEPBDXZ 1001ed1e f   qt-mt323:qt-mt323.dll
 0001:0001dd24       ?className@QSpinBox@@UBEPBDXZ 1001ed24 f   qt-mt323:qt-mt323.dll
 0001:0001dd2a       ?className@QSplitter@@UBEPBDXZ 1001ed2a f   qt-mt323:qt-mt323.dll
 0001:0001dd30       ?cleanText@QSpinBox@@UBE?AVQString@@XZ 1001ed30 f   qt-mt323:qt-mt323.dll
 0001:0001dd36       ?clearCell@QDataTable@@MAEXHH@Z 1001ed36 f   qt-mt323:qt-mt323.dll
 0001:0001dd3c       ?clearCellWidget@QTable@@UAEXHH@Z 1001ed3c f   qt-mt323:qt-mt323.dll
 0001:0001dd42       ?columnAt@QTable@@UBEHH@Z  1001ed42 f   qt-mt323:qt-mt323.dll
 0001:0001dd48       ?columnClicked@QDataTable@@MAEXH@Z 1001ed48 f   qt-mt323:qt-mt323.dll
 0001:0001dd4e       ?columnIndexChanged@QTable@@MAEXHHH@Z 1001ed4e f   qt-mt323:qt-mt323.dll
 0001:0001dd54       ?columnPos@QTable@@UBEHH@Z 1001ed54 f   qt-mt323:qt-mt323.dll
 0001:0001dd5a       ?columnWidth@QTable@@UBEHH@Z 1001ed5a f   qt-mt323:qt-mt323.dll
 0001:0001dd60       ?columnWidthChanged@QTable@@MAEXH@Z 1001ed60 f   qt-mt323:qt-mt323.dll
 0001:0001dd66       ?confirmCancel@QDataTable@@MAE?AW4Confirm@QSql@@W4Op@3@@Z 1001ed66 f   qt-mt323:qt-mt323.dll
 0001:0001dd6c       ?confirmEdit@QDataTable@@MAE?AW4Confirm@QSql@@W4Op@3@@Z 1001ed6c f   qt-mt323:qt-mt323.dll
 0001:0001dd72       ?contentsContextMenuEvent@QDataTable@@MAEXPAVQContextMenuEvent@@@Z 1001ed72 f   qt-mt323:qt-mt323.dll
 0001:0001dd78       ?contentsDragEnterEvent@QTable@@MAEXPAVQDragEnterEvent@@@Z 1001ed78 f   qt-mt323:qt-mt323.dll
 0001:0001dd7e       ?contentsDragLeaveEvent@QTable@@MAEXPAVQDragLeaveEvent@@@Z 1001ed7e f   qt-mt323:qt-mt323.dll
 0001:0001dd84       ?contentsDragMoveEvent@QTable@@MAEXPAVQDragMoveEvent@@@Z 1001ed84 f   qt-mt323:qt-mt323.dll
 0001:0001dd8a       ?contentsDropEvent@QTable@@MAEXPAVQDropEvent@@@Z 1001ed8a f   qt-mt323:qt-mt323.dll
 0001:0001dd90       ?contentsMouseDoubleClickEvent@QTable@@MAEXPAVQMouseEvent@@@Z 1001ed90 f   qt-mt323:qt-mt323.dll
 0001:0001dd96       ?contentsMouseMoveEvent@QTable@@MAEXPAVQMouseEvent@@@Z 1001ed96 f   qt-mt323:qt-mt323.dll
 0001:0001dd9c       ?contentsMousePressEvent@QDataTable@@MAEXPAVQMouseEvent@@@Z 1001ed9c f   qt-mt323:qt-mt323.dll
 0001:0001dda2       ?contentsMouseReleaseEvent@QTable@@MAEXPAVQMouseEvent@@@Z 1001eda2 f   qt-mt323:qt-mt323.dll
 0001:0001dda8       ?createEditor@QDataTable@@MBEPAVQWidget@@HH_N@Z 1001eda8 f   qt-mt323:qt-mt323.dll
 0001:0001ddae       ?currentSelection@QTable@@UBEHXZ 1001edae f   qt-mt323:qt-mt323.dll
 0001:0001ddb4       ?deleteCurrent@QDataTable@@MAE_NXZ 1001edb4 f   qt-mt323:qt-mt323.dll
 0001:0001ddba       ?dragObject@QTable@@MAEPAVQDragObject@@XZ 1001edba f   qt-mt323:qt-mt323.dll
 0001:0001ddc0       ?drawButton@QRadioButton@@MAEXPAVQPainter@@@Z 1001edc0 f   qt-mt323:qt-mt323.dll
 0001:0001ddc6       ?drawButtonLabel@QRadioButton@@MAEXPAVQPainter@@@Z 1001edc6 f   qt-mt323:qt-mt323.dll
 0001:0001ddcc       ?drawContents@QDataTable@@MAEXPAVQPainter@@HHHH@Z 1001edcc f   qt-mt323:qt-mt323.dll
 0001:0001ddd2       ?drawContents@QTable@@EAEXPAVQPainter@@@Z 1001edd2 f   qt-mt323:qt-mt323.dll
 0001:0001ddd8       ?drawContentsOffset@QScrollView@@MAEXPAVQPainter@@HHHHHH@Z 1001edd8 f   qt-mt323:qt-mt323.dll
 0001:0001ddde       ?drawSplitter@QSplitter@@MAEXPAVQPainter@@HHHH@Z 1001edde f   qt-mt323:qt-mt323.dll
 0001:0001dde4       ?editCell@QTable@@UAEXHH_N@Z 1001ede4 f   qt-mt323:qt-mt323.dll
 0001:0001ddea       ?endEdit@QDataTable@@MAEXHH_N0@Z 1001edea f   qt-mt323:qt-mt323.dll
 0001:0001ddf0       ?event@QButtonGroup@@MAE_NPAVQEvent@@@Z 1001edf0 f   qt-mt323:qt-mt323.dll
 0001:0001ddf6       ?event@QDateEdit@@MAE_NPAVQEvent@@@Z 1001edf6 f   qt-mt323:qt-mt323.dll
 0001:0001ddfc       ?event@QSplitter@@MAE_NPAVQEvent@@@Z 1001edfc f   qt-mt323:qt-mt323.dll
 0001:0001de02       ?eventFilter@QDataTable@@MAE_NPAVQObject@@PAVQEvent@@@Z 1001ee02 f   qt-mt323:qt-mt323.dll
 0001:0001de08       ?eventFilter@QSpinBox@@MAE_NPAVQObject@@PAVQEvent@@@Z 1001ee08 f   qt-mt323:qt-mt323.dll
 0001:0001de0e       ?fieldAlignment@QDataTable@@MAEHPBVQSqlField@@@Z 1001ee0e f   qt-mt323:qt-mt323.dll
 0001:0001de14       ?find@QDataTable@@UAEXABVQString@@_N1@Z 1001ee14 f   qt-mt323:qt-mt323.dll
 0001:0001de1a       ?fix@QDateEdit@@MAEXXZ     1001ee1a f   qt-mt323:qt-mt323.dll
 0001:0001de20       ?focusInEvent@QTable@@MAEXPAVQFocusEvent@@@Z 1001ee20 f   qt-mt323:qt-mt323.dll
 0001:0001de26       ?focusOutEvent@QTable@@MAEXPAVQFocusEvent@@@Z 1001ee26 f   qt-mt323:qt-mt323.dll
 0001:0001de2c       ?handleError@QDataTable@@MAEXABVQSqlError@@@Z 1001ee2c f   qt-mt323:qt-mt323.dll
 0001:0001de32       ?hideColumn@QDataTable@@UAEXH@Z 1001ee32 f   qt-mt323:qt-mt323.dll
 0001:0001de38       ?hideRow@QTable@@UAEXH@Z   1001ee38 f   qt-mt323:qt-mt323.dll
 0001:0001de3e       ?hitButton@QRadioButton@@MBE_NABVQPoint@@@Z 1001ee3e f   qt-mt323:qt-mt323.dll
 0001:0001de44       ?insertColumns@QTable@@UAEXHH@Z 1001ee44 f   qt-mt323:qt-mt323.dll
 0001:0001de4a       ?insertCurrent@QDataTable@@MAE_NXZ 1001ee4a f   qt-mt323:qt-mt323.dll
 0001:0001de50       ?insertRows@QTable@@UAEXHH@Z 1001ee50 f   qt-mt323:qt-mt323.dll
 0001:0001de56       ?insertWidget@QTable@@MAEXHHPAVQWidget@@@Z 1001ee56 f   qt-mt323:qt-mt323.dll
 0001:0001de5c       ?interpretText@QSpinBox@@MAEXXZ 1001ee5c f   qt-mt323:qt-mt323.dll
 0001:0001de62       ?item@QDataTable@@MBEPAVQTableItem@@HH@Z 1001ee62 f   qt-mt323:qt-mt323.dll
 0001:0001de68       ?keyPressEvent@QDataTable@@MAEXPAVQKeyEvent@@@Z 1001ee68 f   qt-mt323:qt-mt323.dll
 0001:0001de6e       ?leaveEvent@QSpinBox@@MAEXPAVQEvent@@@Z 1001ee6e f   qt-mt323:qt-mt323.dll
 0001:0001de74       ?mapTextToValue@QSpinBox@@MAEHPA_N@Z 1001ee74 f   qt-mt323:qt-mt323.dll
 0001:0001de7a       ?mapValueToText@QSpinBox@@MAE?AVQString@@H@Z 1001ee7a f   qt-mt323:qt-mt323.dll
 0001:0001de80       ?metaObject@QButtonGroup@@UBEPAVQMetaObject@@XZ 1001ee80 f   qt-mt323:qt-mt323.dll
 0001:0001de86       ?metaObject@QDataTable@@UBEPAVQMetaObject@@XZ 1001ee86 f   qt-mt323:qt-mt323.dll
 0001:0001de8c       ?metaObject@QDateEdit@@UBEPAVQMetaObject@@XZ 1001ee8c f   qt-mt323:qt-mt323.dll
 0001:0001de92       ?metaObject@QRadioButton@@UBEPAVQMetaObject@@XZ 1001ee92 f   qt-mt323:qt-mt323.dll
 0001:0001de98       ?metaObject@QSpinBox@@UBEPAVQMetaObject@@XZ 1001ee98 f   qt-mt323:qt-mt323.dll
 0001:0001de9e       ?metaObject@QSplitter@@UBEPAVQMetaObject@@XZ 1001ee9e f   qt-mt323:qt-mt323.dll
 0001:0001dea4       ?minimumSizeHint@QDateEdit@@UBE?AVQSize@@XZ 1001eea4 f   qt-mt323:qt-mt323.dll
 0001:0001deaa       ?minimumSizeHint@QScrollView@@UBE?AVQSize@@XZ 1001eeaa f   qt-mt323:qt-mt323.dll
 0001:0001deb0       ?minimumSizeHint@QSpinBox@@UBE?AVQSize@@XZ 1001eeb0 f   qt-mt323:qt-mt323.dll
 0001:0001deb6       ?minimumSizeHint@QSplitter@@UBE?AVQSize@@XZ 1001eeb6 f   qt-mt323:qt-mt323.dll
 0001:0001debc       ?moveFocus@QButtonGroup@@UAEXH@Z 1001eebc f   qt-mt323:qt-mt323.dll
 0001:0001dec2       ?numCols@QDataTable@@UBEHXZ 1001eec2 f   qt-mt323:qt-mt323.dll
 0001:0001dec8       ?numRows@QDataTable@@UBEHXZ 1001eec8 f   qt-mt323:qt-mt323.dll
 0001:0001dece       ?outOfRange@QDateEdit@@MBE_NHHH@Z 1001eece f   qt-mt323:qt-mt323.dll
 0001:0001ded4       ?paintCell@QDataTable@@MAEXPAVQPainter@@HHABVQRect@@_NABVQColorGroup@@@Z 1001eed4 f   qt-mt323:qt-mt323.dll
 0001:0001deda       ?paintCell@QTable@@UAEXPAVQPainter@@HHABVQRect@@_N@Z 1001eeda f   qt-mt323:qt-mt323.dll
 0001:0001dee0       ?paintEmptyArea@QTable@@MAEXPAVQPainter@@HHHH@Z 1001eee0 f   qt-mt323:qt-mt323.dll
 0001:0001dee6       ?paintEvent@QTable@@MAEXPAVQPaintEvent@@@Z 1001eee6 f   qt-mt323:qt-mt323.dll
 0001:0001deec       ?paintField@QDataTable@@MAEXPAVQPainter@@PBVQSqlField@@ABVQRect@@_N@Z 1001eeec f   qt-mt323:qt-mt323.dll
 0001:0001def2       ?paintFocus@QTable@@UAEXPAVQPainter@@ABVQRect@@@Z 1001eef2 f   qt-mt323:qt-mt323.dll
 0001:0001def8       ?pixmap@QTable@@UBE?AVQPixmap@@HH@Z 1001eef8 f   qt-mt323:qt-mt323.dll
 0001:0001defe       ?prefix@QSpinBox@@UBE?AVQString@@XZ 1001eefe f   qt-mt323:qt-mt323.dll
 0001:0001df04       ?qt_cast@QButtonGroup@@UAEPAXPBD@Z 1001ef04 f   qt-mt323:qt-mt323.dll
 0001:0001df0a       ?qt_cast@QDataTable@@UAEPAXPBD@Z 1001ef0a f   qt-mt323:qt-mt323.dll
 0001:0001df10       ?qt_cast@QDateEdit@@UAEPAXPBD@Z 1001ef10 f   qt-mt323:qt-mt323.dll
 0001:0001df16       ?qt_cast@QRadioButton@@UAEPAXPBD@Z 1001ef16 f   qt-mt323:qt-mt323.dll
 0001:0001df1c       ?qt_cast@QSpinBox@@UAEPAXPBD@Z 1001ef1c f   qt-mt323:qt-mt323.dll
 0001:0001df22       ?qt_cast@QSplitter@@UAEPAXPBD@Z 1001ef22 f   qt-mt323:qt-mt323.dll
 0001:0001df28       ?qt_emit@QButtonGroup@@UAE_NHPAUQUObject@@@Z 1001ef28 f   qt-mt323:qt-mt323.dll
 0001:0001df2e       ?qt_emit@QDataTable@@UAE_NHPAUQUObject@@@Z 1001ef2e f   qt-mt323:qt-mt323.dll
 0001:0001df34       ?qt_emit@QDateEdit@@UAE_NHPAUQUObject@@@Z 1001ef34 f   qt-mt323:qt-mt323.dll
 0001:0001df3a       ?qt_emit@QRadioButton@@UAE_NHPAUQUObject@@@Z 1001ef3a f   qt-mt323:qt-mt323.dll
 0001:0001df40       ?qt_emit@QSpinBox@@UAE_NHPAUQUObject@@@Z 1001ef40 f   qt-mt323:qt-mt323.dll
 0001:0001df46       ?qt_emit@QSplitter@@UAE_NHPAUQUObject@@@Z 1001ef46 f   qt-mt323:qt-mt323.dll
 0001:0001df4c       ?qt_invoke@QButtonGroup@@UAE_NHPAUQUObject@@@Z 1001ef4c f   qt-mt323:qt-mt323.dll
 0001:0001df52       ?qt_invoke@QDataTable@@UAE_NHPAUQUObject@@@Z 1001ef52 f   qt-mt323:qt-mt323.dll
 0001:0001df58       ?qt_invoke@QDateEdit@@UAE_NHPAUQUObject@@@Z 1001ef58 f   qt-mt323:qt-mt323.dll
 0001:0001df5e       ?qt_invoke@QRadioButton@@UAE_NHPAUQUObject@@@Z 1001ef5e f   qt-mt323:qt-mt323.dll
 0001:0001df64       ?qt_invoke@QSpinBox@@UAE_NHPAUQUObject@@@Z 1001ef64 f   qt-mt323:qt-mt323.dll
 0001:0001df6a       ?qt_invoke@QSplitter@@UAE_NHPAUQUObject@@@Z 1001ef6a f   qt-mt323:qt-mt323.dll
 0001:0001df70       ?qt_property@QButtonGroup@@UAE_NHHPAVQVariant@@@Z 1001ef70 f   qt-mt323:qt-mt323.dll
 0001:0001df76       ?qt_property@QDataTable@@UAE_NHHPAVQVariant@@@Z 1001ef76 f   qt-mt323:qt-mt323.dll
 0001:0001df7c       ?qt_property@QDateEdit@@UAE_NHHPAVQVariant@@@Z 1001ef7c f   qt-mt323:qt-mt323.dll
 0001:0001df82       ?qt_property@QRadioButton@@UAE_NHHPAVQVariant@@@Z 1001ef82 f   qt-mt323:qt-mt323.dll
 0001:0001df88       ?qt_property@QSpinBox@@UAE_NHHPAVQVariant@@@Z 1001ef88 f   qt-mt323:qt-mt323.dll
 0001:0001df8e       ?qt_property@QSplitter@@UAE_NHHPAVQVariant@@@Z 1001ef8e f   qt-mt323:qt-mt323.dll
 0001:0001df94       ?rangeChange@QSpinBox@@MAEXXZ 1001ef94 f   qt-mt323:qt-mt323.dll
 0001:0001df9a       ?refresh@QDataTable@@UAEXXZ 1001ef9a f   qt-mt323:qt-mt323.dll
 0001:0001dfa0       ?removeColumn@QDataTable@@UAEXI@Z 1001efa0 f   qt-mt323:qt-mt323.dll
 0001:0001dfa6       ?removeColumn@QTable@@UAEXH@Z 1001efa6 f   qt-mt323:qt-mt323.dll
 0001:0001dfac       ?removeColumns@QTable@@UAEXABV?$QMemArray@H@@@Z 1001efac f   qt-mt323:qt-mt323.dll
 0001:0001dfb2       ?removeLastNumber@QDateEdit@@MAEXH@Z 1001efb2 f   qt-mt323:qt-mt323.dll
 0001:0001dfb8       ?removeRow@QTable@@UAEXH@Z 1001efb8 f   qt-mt323:qt-mt323.dll
 0001:0001dfbe       ?removeRows@QTable@@UAEXABV?$QMemArray@H@@@Z 1001efbe f   qt-mt323:qt-mt323.dll
 0001:0001dfc4       ?removeSelection@QTable@@UAEXABVQTableSelection@@@Z 1001efc4 f   qt-mt323:qt-mt323.dll
 0001:0001dfca       ?removeSelection@QTable@@UAEXH@Z 1001efca f   qt-mt323:qt-mt323.dll
 0001:0001dfd0       ?resizeData@QDataTable@@MAEXH@Z 1001efd0 f   qt-mt323:qt-mt323.dll
 0001:0001dfd6       ?resizeEvent@QDataTable@@MAEXPAVQResizeEvent@@@Z 1001efd6 f   qt-mt323:qt-mt323.dll
 0001:0001dfdc       ?resizeEvent@QDateEdit@@MAEXPAVQResizeEvent@@@Z 1001efdc f   qt-mt323:qt-mt323.dll
 0001:0001dfe2       ?resizeEvent@QRadioButton@@MAEXPAVQResizeEvent@@@Z 1001efe2 f   qt-mt323:qt-mt323.dll
 0001:0001dfe8       ?resizeEvent@QSpinBox@@MAEXPAVQResizeEvent@@@Z 1001efe8 f   qt-mt323:qt-mt323.dll
 0001:0001dfee       ?resizeEvent@QSplitter@@MAEXPAVQResizeEvent@@@Z 1001efee f   qt-mt323:qt-mt323.dll
 0001:0001dff4       ?rowAt@QTable@@UBEHH@Z     1001eff4 f   qt-mt323:qt-mt323.dll
 0001:0001dffa       ?rowHeight@QTable@@UBEHH@Z 1001effa f   qt-mt323:qt-mt323.dll
 0001:0001e000       ?rowHeightChanged@QTable@@MAEXH@Z 1001f000 f   qt-mt323:qt-mt323.dll
 0001:0001e006       ?rowIndexChanged@QTable@@MAEXHHH@Z 1001f006 f   qt-mt323:qt-mt323.dll
 0001:0001e00c       ?rowPos@QTable@@UBEHH@Z    1001f00c f   qt-mt323:qt-mt323.dll
 0001:0001e012       ?sectionFormattedText@QDateEdit@@MAE?AVQString@@H@Z 1001f012 f   qt-mt323:qt-mt323.dll
 0001:0001e018       ?selectAll@QSpinBox@@UAEXXZ 1001f018 f   qt-mt323:qt-mt323.dll
 0001:0001e01e       ?setAutoAdvance@QDateEdit@@UAEX_N@Z 1001f01e f   qt-mt323:qt-mt323.dll
 0001:0001e024       ?setAutoDelete@QDataTable@@UAEX_N@Z 1001f024 f   qt-mt323:qt-mt323.dll
 0001:0001e02a       ?setAutoEdit@QDataTable@@UAEX_N@Z 1001f02a f   qt-mt323:qt-mt323.dll
 0001:0001e030       ?setButton@QButtonGroup@@UAEXH@Z 1001f030 f   qt-mt323:qt-mt323.dll
 0001:0001e036       ?setButtonSymbols@QSpinBox@@UAEXW4ButtonSymbols@1@@Z 1001f036 f   qt-mt323:qt-mt323.dll
 0001:0001e03c       ?setCellContentFromEditor@QTable@@MAEXHH@Z 1001f03c f   qt-mt323:qt-mt323.dll
 0001:0001e042       ?setCellWidget@QTable@@UAEXHHPAVQWidget@@@Z 1001f042 f   qt-mt323:qt-mt323.dll
 0001:0001e048       ?setChecked@QRadioButton@@UAEX_N@Z 1001f048 f   qt-mt323:qt-mt323.dll
 0001:0001e04e       ?setColumn@QDataTable@@UAEXIABVQString@@0HABVQIconSet@@@Z 1001f04e f   qt-mt323:qt-mt323.dll
 0001:0001e054       ?setColumnMovingEnabled@QTable@@UAEX_N@Z 1001f054 f   qt-mt323:qt-mt323.dll
 0001:0001e05a       ?setColumnReadOnly@QTable@@UAEXH_N@Z 1001f05a f   qt-mt323:qt-mt323.dll
 0001:0001e060       ?setColumnStretchable@QDataTable@@UAEXH_N@Z 1001f060 f   qt-mt323:qt-mt323.dll
 0001:0001e066       ?setColumnWidth@QDataTable@@UAEXHH@Z 1001f066 f   qt-mt323:qt-mt323.dll
 0001:0001e06c       ?setConfirmCancels@QDataTable@@UAEX_N@Z 1001f06c f   qt-mt323:qt-mt323.dll
 0001:0001e072       ?setConfirmDelete@QDataTable@@UAEX_N@Z 1001f072 f   qt-mt323:qt-mt323.dll
 0001:0001e078       ?setConfirmEdits@QDataTable@@UAEX_N@Z 1001f078 f   qt-mt323:qt-mt323.dll
 0001:0001e07e       ?setConfirmInsert@QDataTable@@UAEX_N@Z 1001f07e f   qt-mt323:qt-mt323.dll
 0001:0001e084       ?setConfirmUpdate@QDataTable@@UAEX_N@Z 1001f084 f   qt-mt323:qt-mt323.dll
 0001:0001e08a       ?setContentsPos@QScrollView@@UAEXHH@Z 1001f08a f   qt-mt323:qt-mt323.dll
 0001:0001e090       ?setCurrentCell@QTable@@UAEXHH@Z 1001f090 f   qt-mt323:qt-mt323.dll
 0001:0001e096       ?setDate@QDateEdit@@UAEXABVQDate@@@Z 1001f096 f   qt-mt323:qt-mt323.dll
 0001:0001e09c       ?setDateFormat@QDataTable@@UAEXW4DateFormat@Qt@@@Z 1001f09c f   qt-mt323:qt-mt323.dll
 0001:0001e0a2       ?setDay@QDateEdit@@MAEXH@Z 1001f0a2 f   qt-mt323:qt-mt323.dll
 0001:0001e0a8       ?setDragEnabled@QTable@@UAEX_N@Z 1001f0a8 f   qt-mt323:qt-mt323.dll
 0001:0001e0ae       ?setEnabled@QSpinBox@@UAEX_N@Z 1001f0ae f   qt-mt323:qt-mt323.dll
 0001:0001e0b4       ?setEnabled@QTable@@UAEX_N@Z 1001f0b4 f   qt-mt323:qt-mt323.dll
 0001:0001e0ba       ?setExclusive@QButtonGroup@@UAEX_N@Z 1001f0ba f   qt-mt323:qt-mt323.dll
 0001:0001e0c0       ?setFalseText@QDataTable@@UAEXABVQString@@@Z 1001f0c0 f   qt-mt323:qt-mt323.dll
 0001:0001e0c6       ?setFilter@QDataTable@@UAEXABVQString@@@Z 1001f0c6 f   qt-mt323:qt-mt323.dll
 0001:0001e0cc       ?setFocusSection@QDateEdit@@MAE_NH@Z 1001f0cc f   qt-mt323:qt-mt323.dll
 0001:0001e0d2       ?setFocusStyle@QTable@@UAEXW4FocusStyle@1@@Z 1001f0d2 f   qt-mt323:qt-mt323.dll
 0001:0001e0d8       ?setItem@QDataTable@@MAEXHHPAVQTableItem@@@Z 1001f0d8 f   qt-mt323:qt-mt323.dll
 0001:0001e0de       ?setLeftMargin@QTable@@UAEXH@Z 1001f0de f   qt-mt323:qt-mt323.dll
 0001:0001e0e4       ?setMaxValue@QDateEdit@@UAEXABVQDate@@@Z 1001f0e4 f   qt-mt323:qt-mt323.dll
 0001:0001e0ea       ?setMinValue@QDateEdit@@UAEXABVQDate@@@Z 1001f0ea f   qt-mt323:qt-mt323.dll
 0001:0001e0f0       ?setMonth@QDateEdit@@MAEXH@Z 1001f0f0 f   qt-mt323:qt-mt323.dll
 0001:0001e0f6       ?setNullText@QDataTable@@UAEXABVQString@@@Z 1001f0f6 f   qt-mt323:qt-mt323.dll
 0001:0001e0fc       ?setNumCols@QDataTable@@UAEXH@Z 1001f0fc f   qt-mt323:qt-mt323.dll
 0001:0001e102       ?setNumRows@QDataTable@@UAEXH@Z 1001f102 f   qt-mt323:qt-mt323.dll
 0001:0001e108       ?setOpaqueResize@QSplitter@@UAEX_N@Z 1001f108 f   qt-mt323:qt-mt323.dll
 0001:0001e10e       ?setOrder@QDateEdit@@UAEXW4Order@1@@Z 1001f10e f   qt-mt323:qt-mt323.dll
 0001:0001e114       ?setOrientation@QSplitter@@UAEXW4Orientation@Qt@@@Z 1001f114 f   qt-mt323:qt-mt323.dll
 0001:0001e11a       ?setPixmap@QDataTable@@MAEXHHABVQPixmap@@@Z 1001f11a f   qt-mt323:qt-mt323.dll
 0001:0001e120       ?setPrefix@QSpinBox@@UAEXABVQString@@@Z 1001f120 f   qt-mt323:qt-mt323.dll
 0001:0001e126       ?setRadioButtonExclusive@QButtonGroup@@UAEX_N@Z 1001f126 f   qt-mt323:qt-mt323.dll
 0001:0001e12c       ?setRange@QDateEdit@@UAEXABVQDate@@0@Z 1001f12c f   qt-mt323:qt-mt323.dll
 0001:0001e132       ?setReadOnly@QTable@@UAEX_N@Z 1001f132 f   qt-mt323:qt-mt323.dll
 0001:0001e138       ?setResizeMode@QSplitter@@UAEXPAVQWidget@@W4ResizeMode@1@@Z 1001f138 f   qt-mt323:qt-mt323.dll
 0001:0001e13e       ?setRowHeight@QTable@@UAEXHH@Z 1001f13e f   qt-mt323:qt-mt323.dll
 0001:0001e144       ?setRowMovingEnabled@QTable@@UAEX_N@Z 1001f144 f   qt-mt323:qt-mt323.dll
 0001:0001e14a       ?setRowReadOnly@QTable@@UAEXH_N@Z 1001f14a f   qt-mt323:qt-mt323.dll
 0001:0001e150       ?setRowStretchable@QTable@@UAEXH_N@Z 1001f150 f   qt-mt323:qt-mt323.dll
 0001:0001e156       ?setRubberband@QSplitter@@MAEXH@Z 1001f156 f   qt-mt323:qt-mt323.dll
 0001:0001e15c       ?setSelectionMode@QTable@@UAEXW4SelectionMode@1@@Z 1001f15c f   qt-mt323:qt-mt323.dll
 0001:0001e162       ?setSeparator@QDateEdit@@UAEXABVQString@@@Z 1001f162 f   qt-mt323:qt-mt323.dll
 0001:0001e168       ?setShowGrid@QTable@@UAEX_N@Z 1001f168 f   qt-mt323:qt-mt323.dll
 0001:0001e16e       ?setSort@QDataTable@@UAEXABVQSqlIndex@@@Z 1001f16e f   qt-mt323:qt-mt323.dll
 0001:0001e174       ?setSort@QDataTable@@UAEXABVQStringList@@@Z 1001f174 f   qt-mt323:qt-mt323.dll
 0001:0001e17a       ?setSorting@QTable@@UAEX_N@Z 1001f17a f   qt-mt323:qt-mt323.dll
 0001:0001e180       ?setSpecialValueText@QSpinBox@@UAEXABVQString@@@Z 1001f180 f   qt-mt323:qt-mt323.dll
 0001:0001e186       ?setSqlCursor@QDataTable@@UAEXPAVQSqlCursor@@_N1@Z 1001f186 f   qt-mt323:qt-mt323.dll
 0001:0001e18c       ?setSuffix@QSpinBox@@UAEXABVQString@@@Z 1001f18c f   qt-mt323:qt-mt323.dll
 0001:0001e192       ?setText@QTable@@UAEXHHABVQString@@@Z 1001f192 f   qt-mt323:qt-mt323.dll
 0001:0001e198       ?setTopMargin@QTable@@UAEXH@Z 1001f198 f   qt-mt323:qt-mt323.dll
 0001:0001e19e       ?setTrueText@QDataTable@@UAEXABVQString@@@Z 1001f19e f   qt-mt323:qt-mt323.dll
 0001:0001e1a4       ?setValidator@QSpinBox@@UAEXPBVQValidator@@@Z 1001f1a4 f   qt-mt323:qt-mt323.dll
 0001:0001e1aa       ?setValue@QSpinBox@@UAEXH@Z 1001f1aa f   qt-mt323:qt-mt323.dll
 0001:0001e1b0       ?setWrapping@QSpinBox@@UAEX_N@Z 1001f1b0 f   qt-mt323:qt-mt323.dll
 0001:0001e1b6       ?setYear@QDateEdit@@MAEXH@Z 1001f1b6 f   qt-mt323:qt-mt323.dll
 0001:0001e1bc       ?show@QScrollView@@UAEXXZ  1001f1bc f   qt-mt323:qt-mt323.dll
 0001:0001e1c2       ?showColumn@QDataTable@@UAEXH@Z 1001f1c2 f   qt-mt323:qt-mt323.dll
 0001:0001e1c8       ?showEvent@QTable@@MAEXPAVQShowEvent@@@Z 1001f1c8 f   qt-mt323:qt-mt323.dll
 0001:0001e1ce       ?showRow@QTable@@UAEXH@Z   1001f1ce f   qt-mt323:qt-mt323.dll
 0001:0001e1d4       ?sizeHint@QDateEdit@@UBE?AVQSize@@XZ 1001f1d4 f   qt-mt323:qt-mt323.dll
 0001:0001e1da       ?sizeHint@QRadioButton@@UBE?AVQSize@@XZ 1001f1da f   qt-mt323:qt-mt323.dll
 0001:0001e1e0       ?sizeHint@QSpinBox@@UBE?AVQSize@@XZ 1001f1e0 f   qt-mt323:qt-mt323.dll
 0001:0001e1e6       ?sizeHint@QSplitter@@UBE?AVQSize@@XZ 1001f1e6 f   qt-mt323:qt-mt323.dll
 0001:0001e1ec       ?sizeHint@QTable@@UBE?AVQSize@@XZ 1001f1ec f   qt-mt323:qt-mt323.dll
 0001:0001e1f2       ?sortAscending@QDataTable@@UAEXH@Z 1001f1f2 f   qt-mt323:qt-mt323.dll
 0001:0001e1f8       ?sortColumn@QDataTable@@UAEXH_N0@Z 1001f1f8 f   qt-mt323:qt-mt323.dll
 0001:0001e1fe       ?sortDescending@QDataTable@@UAEXH@Z 1001f1fe f   qt-mt323:qt-mt323.dll
 0001:0001e204       ?startDrag@QTable@@MAEXXZ  1001f204 f   qt-mt323:qt-mt323.dll
 0001:0001e20a       ?stepChange@QRangeControl@@MAEXXZ 1001f20a f   qt-mt323:qt-mt323.dll
 0001:0001e210       ?stepDown@QDateEdit@@MAEXXZ 1001f210 f   qt-mt323:qt-mt323.dll
 0001:0001e216       ?stepDown@QSpinBox@@UAEXXZ 1001f216 f   qt-mt323:qt-mt323.dll
 0001:0001e21c       ?stepUp@QDateEdit@@MAEXXZ  1001f21c f   qt-mt323:qt-mt323.dll
 0001:0001e222       ?stepUp@QSpinBox@@UAEXXZ   1001f222 f   qt-mt323:qt-mt323.dll
 0001:0001e228       ?styleChange@QScrollView@@UAEXAAVQStyle@@@Z 1001f228 f   qt-mt323:qt-mt323.dll
 0001:0001e22e       ?styleChange@QSpinBox@@MAEXAAVQStyle@@@Z 1001f22e f   qt-mt323:qt-mt323.dll
 0001:0001e234       ?styleChange@QSplitter@@MAEXAAVQStyle@@@Z 1001f234 f   qt-mt323:qt-mt323.dll
 0001:0001e23a       ?suffix@QSpinBox@@UBE?AVQString@@XZ 1001f23a f   qt-mt323:qt-mt323.dll
 0001:0001e240       ?swapCells@QTable@@UAEXHHHH@Z 1001f240 f   qt-mt323:qt-mt323.dll
 0001:0001e246       ?swapColumns@QDataTable@@UAEXHH_N@Z 1001f246 f   qt-mt323:qt-mt323.dll
 0001:0001e24c       ?swapRows@QTable@@UAEXHH_N@Z 1001f24c f   qt-mt323:qt-mt323.dll
 0001:0001e252       ?takeItem@QDataTable@@MAEXPAVQTableItem@@@Z 1001f252 f   qt-mt323:qt-mt323.dll
 0001:0001e258       ?text@QDataTable@@UBE?AVQString@@HH@Z 1001f258 f   qt-mt323:qt-mt323.dll
 0001:0001e25e       ?timerEvent@QDateEdit@@MAEXPAVQTimerEvent@@@Z 1001f25e f   qt-mt323:qt-mt323.dll
 0001:0001e264       ?updateCurrent@QDataTable@@MAE_NXZ 1001f264 f   qt-mt323:qt-mt323.dll
 0001:0001e26a       ?updateDisplay@QSpinBox@@MAEXXZ 1001f26a f   qt-mt323:qt-mt323.dll
 0001:0001e270       ?updateMask@QRadioButton@@MAEXXZ 1001f270 f   qt-mt323:qt-mt323.dll
 0001:0001e276       ?valueChange@QSpinBox@@MAEXXZ 1001f276 f   qt-mt323:qt-mt323.dll
 0001:0001e27c       ?viewportResizeEvent@QTable@@MAEXPAVQResizeEvent@@@Z 1001f27c f   qt-mt323:qt-mt323.dll
 0001:0001e282       ?wheelEvent@QSpinBox@@MAEXPAVQWheelEvent@@@Z 1001f282 f   qt-mt323:qt-mt323.dll
 0001:0001e288       ?windowActivationChange@QTable@@MAEX_N@Z 1001f288 f   qt-mt323:qt-mt323.dll
 0001:0001e28e       ?activateNextCell@QTable@@MAEXXZ 1001f28e f   qt-mt323:qt-mt323.dll
 0001:0001e294       ?adjustColumn@QTable@@UAEXH@Z 1001f294 f   qt-mt323:qt-mt323.dll
 0001:0001e29a       ?beginEdit@QTable@@MAEPAVQWidget@@HH_N@Z 1001f29a f   qt-mt323:qt-mt323.dll
 0001:0001e2a0       ?className@QTable@@UBEPBDXZ 1001f2a0 f   qt-mt323:qt-mt323.dll
 0001:0001e2a6       ?clearCell@QTable@@UAEXHH@Z 1001f2a6 f   qt-mt323:qt-mt323.dll
 0001:0001e2ac       ?columnClicked@QTable@@MAEXH@Z 1001f2ac f   qt-mt323:qt-mt323.dll
 0001:0001e2b2       ?contentsContextMenuEvent@QTable@@MAEXPAVQContextMenuEvent@@@Z 1001f2b2 f   qt-mt323:qt-mt323.dll
 0001:0001e2b8       ?contentsMousePressEvent@QTable@@MAEXPAVQMouseEvent@@@Z 1001f2b8 f   qt-mt323:qt-mt323.dll
 0001:0001e2be       ?createEditor@QTable@@MBEPAVQWidget@@HH_N@Z 1001f2be f   qt-mt323:qt-mt323.dll
 0001:0001e2c4       ?drawContents@QTable@@MAEXPAVQPainter@@HHHH@Z 1001f2c4 f   qt-mt323:qt-mt323.dll
 0001:0001e2ca       ?endEdit@QTable@@MAEXHH_N0@Z 1001f2ca f   qt-mt323:qt-mt323.dll
 0001:0001e2d0       ?eventFilter@QTable@@UAE_NPAVQObject@@PAVQEvent@@@Z 1001f2d0 f   qt-mt323:qt-mt323.dll
 0001:0001e2d6       ?hideColumn@QTable@@UAEXH@Z 1001f2d6 f   qt-mt323:qt-mt323.dll
 0001:0001e2dc       ?item@QTable@@UBEPAVQTableItem@@HH@Z 1001f2dc f   qt-mt323:qt-mt323.dll
 0001:0001e2e2       ?keyPressEvent@QTable@@MAEXPAVQKeyEvent@@@Z 1001f2e2 f   qt-mt323:qt-mt323.dll
 0001:0001e2e8       ?metaObject@QTable@@UBEPAVQMetaObject@@XZ 1001f2e8 f   qt-mt323:qt-mt323.dll
 0001:0001e2ee       ?numCols@QTable@@UBEHXZ    1001f2ee f   qt-mt323:qt-mt323.dll
 0001:0001e2f4       ?numRows@QTable@@UBEHXZ    1001f2f4 f   qt-mt323:qt-mt323.dll
 0001:0001e2fa       ?paintCell@QTable@@UAEXPAVQPainter@@HHABVQRect@@_NABVQColorGroup@@@Z 1001f2fa f   qt-mt323:qt-mt323.dll
 0001:0001e300       ?qt_cast@QTable@@UAEPAXPBD@Z 1001f300 f   qt-mt323:qt-mt323.dll
 0001:0001e306       ?qt_emit@QTable@@UAE_NHPAUQUObject@@@Z 1001f306 f   qt-mt323:qt-mt323.dll
 0001:0001e30c       ?qt_invoke@QTable@@UAE_NHPAUQUObject@@@Z 1001f30c f   qt-mt323:qt-mt323.dll
 0001:0001e312       ?qt_property@QTable@@UAE_NHHPAVQVariant@@@Z 1001f312 f   qt-mt323:qt-mt323.dll
 0001:0001e318       ?resizeData@QTable@@MAEXH@Z 1001f318 f   qt-mt323:qt-mt323.dll
 0001:0001e31e       ?resizeEvent@QScrollView@@MAEXPAVQResizeEvent@@@Z 1001f31e f   qt-mt323:qt-mt323.dll
 0001:0001e324       ?setColumnStretchable@QTable@@UAEXH_N@Z 1001f324 f   qt-mt323:qt-mt323.dll
 0001:0001e32a       ?setColumnWidth@QTable@@UAEXHH@Z 1001f32a f   qt-mt323:qt-mt323.dll
 0001:0001e330       ?setItem@QTable@@UAEXHHPAVQTableItem@@@Z 1001f330 f   qt-mt323:qt-mt323.dll
 0001:0001e336       ?setNumCols@QTable@@UAEXH@Z 1001f336 f   qt-mt323:qt-mt323.dll
 0001:0001e33c       ?setNumRows@QTable@@UAEXH@Z 1001f33c f   qt-mt323:qt-mt323.dll
 0001:0001e342       ?setPixmap@QTable@@UAEXHHABVQPixmap@@@Z 1001f342 f   qt-mt323:qt-mt323.dll
 0001:0001e348       ?showColumn@QTable@@UAEXH@Z 1001f348 f   qt-mt323:qt-mt323.dll
 0001:0001e34e       ?sortColumn@QTable@@UAEXH_N0@Z 1001f34e f   qt-mt323:qt-mt323.dll
 0001:0001e354       ?swapColumns@QTable@@UAEXHH_N@Z 1001f354 f   qt-mt323:qt-mt323.dll
 0001:0001e35a       ?takeItem@QTable@@UAEXPAVQTableItem@@@Z 1001f35a f   qt-mt323:qt-mt323.dll
 0001:0001e360       ?text@QTable@@UBE?AVQString@@HH@Z 1001f360 f   qt-mt323:qt-mt323.dll
 0001:0001e366       ?className@CAlm_sys_select@@UBEPBDXZ 1001f366 f   alm_sys_select:alm_sys_select.dll
 0001:0001e36c       ?metaObject@CAlm_sys_select@@UBEPAVQMetaObject@@XZ 1001f36c f   alm_sys_select:alm_sys_select.dll
 0001:0001e372       ?qt_cast@CAlm_sys_select@@UAEPAXPBD@Z 1001f372 f   alm_sys_select:alm_sys_select.dll
 0001:0001e378       ?qt_emit@CAlm_sys_select@@UAE_NHPAUQUObject@@@Z 1001f378 f   alm_sys_select:alm_sys_select.dll
 0001:0001e37e       ?qt_invoke@CAlm_sys_select@@UAE_NHPAUQUObject@@@Z 1001f37e f   alm_sys_select:alm_sys_select.dll
 0001:0001e384       ?qt_property@CAlm_sys_select@@UAE_NHHPAVQVariant@@@Z 1001f384 f   alm_sys_select:alm_sys_select.dll
 0001:0001e38a       ?loadState@cfg_Settings@@SA?AVQString@@ABV2@@Z 1001f38a f   cfg_widgets001:cfg_Settings.obj
 0001:0001e41c       ?loadState@cfg_Settings@@SAXAAVQPoint@@AAVQSize@@AA_NABVQString@@@Z 1001f41c f   cfg_widgets001:cfg_Settings.obj
 0001:0001e515       ?loadState@cfg_Settings@@SAXQAVQListView@@ABVQString@@@Z 1001f515 f   cfg_widgets001:cfg_Settings.obj
 0001:0001e612       ?loadState@cfg_Settings@@SAXQAVQSplitter@@ABVQString@@@Z 1001f612 f   cfg_widgets001:cfg_Settings.obj
 0001:0001e710       ?loadState@cfg_Settings@@SAXQAVQTable@@ABVQString@@@Z 1001f710 f   cfg_widgets001:cfg_Settings.obj
 0001:0001e7fd       ?saveState@cfg_Settings@@SAXABVQPoint@@ABVQSize@@AB_NABVQString@@@Z 1001f7fd f   cfg_widgets001:cfg_Settings.obj
 0001:0001e917       ?saveState@cfg_Settings@@SAXABVQString@@0@Z 1001f917 f   cfg_widgets001:cfg_Settings.obj
 0001:0001e993       ?saveState@cfg_Settings@@SAXQBVQListView@@ABVQString@@@Z 1001f993 f   cfg_widgets001:cfg_Settings.obj
 0001:0001ea6b       ?saveState@cfg_Settings@@SAXQBVQSplitter@@ABVQString@@@Z 1001fa6b f   cfg_widgets001:cfg_Settings.obj
 0001:0001eb48       ?saveState@cfg_Settings@@SAXQBVQTable@@ABVQString@@@Z 1001fb48 f   cfg_widgets001:cfg_Settings.obj
 0001:0001ec30       ??0Document@@QAE@ABVQString@@@Z 1001fc30 f   config_alarm_utilities:Document.obj
 0001:0001ec50       ??0Document_BncsSystem@@QAE@XZ 1001fc50 f   config_alarm_utilities:Document.obj
 0001:0001ece0       ??1Document@@UAE@XZ        1001fce0 f   config_alarm_utilities:Document.obj
 0001:0001ecf0       ??1Document_BncsSystem@@UAE@XZ 1001fcf0 f   config_alarm_utilities:Document.obj
 0001:0001ed00       ??_GDocument@@UAEPAXI@Z    1001fd00 f i config_alarm_utilities:Document.obj
 0001:0001ed00       ??_EDocument@@UAEPAXI@Z    1001fd00 f i config_alarm_utilities:Document.obj
 0001:0001ed30       ??_GDocument_BncsSystem@@UAEPAXI@Z 1001fd30 f i config_alarm_utilities:Document.obj
 0001:0001ed30       ??_EDocument_BncsSystem@@UAEPAXI@Z 1001fd30 f i config_alarm_utilities:Document.obj
 0001:0001ed60       ?getMaxDevice@Document_BncsSystem@@QBEHXZ 1001fd60 f   config_alarm_utilities:Document.obj
 0001:0001ed70       ?getMaxSlot@Document_BncsSystem@@QBEHXZ 1001fd70 f   config_alarm_utilities:Document.obj
 0001:0001ed80       ?load@Document_BncsSystem@@QAE_NXZ 1001fd80 f   config_alarm_utilities:Document.obj
 0001:0001ee80       ??0FileLoad@@IAE@ABVQString@@@Z 1001fe80 f   config_alarm_utilities:Loaders.obj
 0001:0001eef0       ??0Loaders@@QAE@XZ         1001fef0 f   config_alarm_utilities:Loaders.obj
 0001:0001ef70       ??1?$QPtrList@VDirLoad@@@@UAE@XZ 1001ff70 f i config_alarm_utilities:Loaders.obj
 0001:0001efd0       ??1?$QPtrList@VFileLoad@@@@UAE@XZ 1001ffd0 f i config_alarm_utilities:Loaders.obj
 0001:0001f030       ??1FileLoad@@UAE@XZ        10020030 f   config_alarm_utilities:Loaders.obj
 0001:0001f090       ??1Loaders@@UAE@XZ         10020090 f   config_alarm_utilities:Loaders.obj
 0001:0001f140       ??_E?$QPtrList@VDirLoad@@@@UAEPAXI@Z 10020140 f i config_alarm_utilities:Loaders.obj
 0001:0001f140       ??_G?$QPtrList@VDirLoad@@@@UAEPAXI@Z 10020140 f i config_alarm_utilities:Loaders.obj
 0001:0001f1b0       ??_G?$QPtrList@VFileLoad@@@@UAEPAXI@Z 100201b0 f i config_alarm_utilities:Loaders.obj
 0001:0001f1b0       ??_E?$QPtrList@VFileLoad@@@@UAEPAXI@Z 100201b0 f i config_alarm_utilities:Loaders.obj
 0001:0001f220       ??_EFileLoad@@UAEPAXI@Z    10020220 f i config_alarm_utilities:Loaders.obj
 0001:0001f220       ??_GFileLoad@@UAEPAXI@Z    10020220 f i config_alarm_utilities:Loaders.obj
 0001:0001f250       ??_ELoaders@@UAEPAXI@Z     10020250 f i config_alarm_utilities:Loaders.obj
 0001:0001f250       ??_GLoaders@@UAEPAXI@Z     10020250 f i config_alarm_utilities:Loaders.obj
 0001:0001f280       ?append@Loaders@@QAEXPAVFileLoad@@@Z 10020280 f   config_alarm_utilities:Loaders.obj
 0001:0001f290       ?clear@?$QPtrList@VcOutputFile@@@@UAEXXZ 10020290 f i alm_db_output.obj
 0001:0001f290       ?clear@?$QPtrList@VQPopupMenu@@@@UAEXXZ 10020290 f i alm_db_output.obj
 0001:0001f290       ?clear@?$QPtrList@VDirLoad@@@@UAEXXZ 10020290 f i config_alarm_utilities:Loaders.obj
 0001:0001f290       ?clear@?$QPtrList@VFileLoad@@@@UAEXXZ 10020290 f i config_alarm_utilities:Loaders.obj
 0001:0001f290       ?clear@?$QPtrList@VcProcess@@@@UAEXXZ 10020290 f i alm_db_output.obj
 0001:0001f2a0       ?deleteItem@?$QPtrList@VDirLoad@@@@EAEXPAX@Z 100202a0 f i config_alarm_utilities:Loaders.obj
 0001:0001f2a0       ?deleteItem@?$QPtrList@VFileLoad@@@@EAEXPAX@Z 100202a0 f i config_alarm_utilities:Loaders.obj
 0001:0001f2c0       ?fileName@FileLoad@@QBE?AVQString@@XZ 100202c0 f   config_alarm_utilities:Loaders.obj
 0001:0001f2f0       ?got@FileLoad@@QBE_NXZ     100202f0 f   config_alarm_utilities:Loaders.obj
 0001:0001f300       ?lock@FileLoad@@UAEXABVQString@@@Z 10020300 f   config_alarm_utilities:Loaders.obj
 0001:0001f300       ?activate@config_plugin_base@@UAEX_N@Z 10020300 f   alm_db_output.obj
 0001:0001f300       ?reply@config_plugin_base@@UAEXPAVresponse@@@Z 10020300 f   alm_db_output.obj
 0001:0001f300       ?levelChanged@manage_temp@@QAEXH@Z 10020300 f   manage_tempimpl.obj
 0001:0001f310       ?matches@FileLoad@@QAE_NABVQString@@@Z 10020310 f   config_alarm_utilities:Loaders.obj
 0001:0001f3c0       ?request@FileLoad@@QAEXPAVISendCommand@@@Z 100203c0 f   config_alarm_utilities:Loaders.obj
 0001:0001f450       ?resetNameRead@FileLoad@@QAEXABVQString@@@Z 10020450 f   config_alarm_utilities:Loaders.obj
 0001:0001f460       ?setGot@FileLoad@@QAEXXZ   10020460 f   config_alarm_utilities:Loaders.obj
 0001:0001f466       __purecall                 10020466 f   MSVCRT:MSVCR120.dll
 0001:0001f46c       ??2@YAPAXI@Z               1002046c f   MSVCRT:MSVCR120.dll
 0001:0001f472       ??3@YAXPAX@Z               10020472 f   MSVCRT:MSVCR120.dll
 0001:0001f478       ___atonexitinit            10020478 f   MSVCRT:atonexit.obj
 0001:0001f4b4       __onexit                   100204b4 f   MSVCRT:atonexit.obj
 0001:0001f55d       _atexit                    1002055d f   MSVCRT:atonexit.obj
 0001:0001f572       _memcpy                    10020572 f   MSVCRT:MSVCR120.dll
 0001:0001f578       _strcpy                    10020578 f   MSVCRT:MSVCR120.dll
 0001:0001f57e       _strcat                    1002057e f   MSVCRT:MSVCR120.dll
 0001:0001f584       _strlen                    10020584 f   MSVCRT:MSVCR120.dll
 0001:0001f58a       @__security_check_cookie@4 1002058a f   MSVCRT:secchk.obj
 0001:0001f59a       __CxxThrowException@8      1002059a f   MSVCRT:MSVCR120.dll
 0001:0001f5a0       __EH_epilog3               100205a0 f   MSVCRT:ehprolg3.obj
 0001:0001f5b4       __EH_epilog3_GS            100205b4 f   MSVCRT:ehprolg3.obj
 0001:0001f5c3       __EH_prolog3               100205c3 f   MSVCRT:ehprolg3.obj
 0001:0001f5f6       __EH_prolog3_GS            100205f6 f   MSVCRT:ehprolg3.obj
 0001:0001f62c       __EH_prolog3_catch         1002062c f   MSVCRT:ehprolg3.obj
 0001:0001f662       ___CxxFrameHandler3        10020662 f   MSVCRT:MSVCR120.dll
 0001:0001f668       ??_Etype_info@@UAEPAXI@Z   10020668 f i MSVCRT:ti_inst.obj
 0001:0001f6c0       _strcmp                    100206c0 f   MSVCRT:MSVCR120.dll
 0001:0001f6c6       ??_L@YGXPAXIHP6EX0@Z1@Z    100206c6 f   MSVCRT:ehvecctr.obj
 0001:0001f728       ??_M@YGXPAXIHP6EX0@Z@Z     10020728 f   MSVCRT:ehvecdtr.obj
 0001:0001f797       ?__ArrayUnwind@@YGXPAXIHP6EX0@Z@Z 10020797 f   MSVCRT:ehvecdtr.obj
 0001:0001f841       __CRT_INIT@12              10020841 f   MSVCRT:crtdll.obj
 0001:0001fa38       __DllMainCRTStartup@12     10020a38 f   MSVCRT:crtdll.obj
 0001:0001fb8e       __lock                     10020b8e f   MSVCRT:MSVCR120.dll
 0001:0001fb94       __unlock                   10020b94 f   MSVCRT:MSVCR120.dll
 0001:0001fb9a       ___dllonexit               10020b9a f   MSVCRT:MSVCR120.dll
 0001:0001fba0       __SEH_prolog4              10020ba0 f   MSVCRT:sehprolg4.obj
 0001:0001fbe5       __SEH_epilog4              10020be5 f   MSVCRT:sehprolg4.obj
 0001:0001fbf9       __except_handler4          10020bf9 f   MSVCRT:chandler4gs.obj
 0001:0001fc1c       ___raise_securityfailure   10020c1c f   MSVCRT:gs_report.obj
 0001:0001fc59       ___report_gsfailure        10020c59 f   MSVCRT:gs_report.obj
 0001:0001fd54       ??1type_info@@UAE@XZ       10020d54 f   MSVCRT:MSVCR120.dll
 0001:0001fd5a       ?terminate@@YAXXZ          10020d5a f   MSVCRT:MSVCR120.dll
 0001:0001fd60       ___CppXcptFilter           10020d60 f   MSVCRT:MSVCR120.dll
 0001:0001fd66       __amsg_exit                10020d66 f   MSVCRT:MSVCR120.dll
 0001:0001fd70       __FindPESection            10020d70 f   MSVCRT:pesect.obj
 0001:0001fdc0       __IsNonwritableInCurrentImage 10020dc0 f   MSVCRT:pesect.obj
 0001:0001fe80       __ValidateImageBase        10020e80 f   MSVCRT:pesect.obj
 0001:0001feb1       ___security_init_cookie    10020eb1 f   MSVCRT:gs_support.obj
 0001:0001ff4d       _DllMain@12                10020f4d f   MSVCRT:dllmain.obj
 0001:0001ff6f       __RTC_Initialize           10020f6f f   MSVCRT:initsect.obj
 0001:0001ff8f       __RTC_Terminate            10020f8f f   MSVCRT:initsect.obj
 0001:0001ffb0       __initterm                 10020fb0 f   MSVCRT:MSVCR120.dll
 0001:0001ffb6       __initterm_e               10020fb6 f   MSVCRT:MSVCR120.dll
 0001:0001ffbc       ___clean_type_info_names   10020fbc f   MSVCRT:tncleanup.obj
 0001:0001ffc8       __except_handler4_common   10020fc8 f   MSVCRT:MSVCR120.dll
 0001:0001ffce       __crt_debugger_hook        10020fce f   MSVCRT:MSVCR120.dll
 0001:0001ffd4       ___crtUnhandledException   10020fd4 f   MSVCRT:MSVCR120.dll
 0001:0001ffda       ___crtTerminateProcess     10020fda f   MSVCRT:MSVCR120.dll
 0001:0001ffe0       ___clean_type_info_names_internal 10020fe0 f   MSVCRT:MSVCR120.dll
 0001:0001ffe6       _IsProcessorFeaturePresent@4 10020fe6 f   kernel32:KERNEL32.dll
 0002:00000000       __imp__DisableThreadLibraryCalls@4 10026000     kernel32:KERNEL32.dll
 0002:00000004       __imp__GetCurrentThreadId@0 10026004     kernel32:KERNEL32.dll
 0002:00000008       __imp__GetCurrentProcessId@0 10026008     kernel32:KERNEL32.dll
 0002:0000000c       __imp__QueryPerformanceCounter@4 1002600c     kernel32:KERNEL32.dll
 0002:00000010       __imp__IsProcessorFeaturePresent@4 10026010     kernel32:KERNEL32.dll
 0002:00000014       __imp__IsDebuggerPresent@0 10026014     kernel32:KERNEL32.dll
 0002:00000018       __imp__DecodePointer@4     10026018     kernel32:KERNEL32.dll
 0002:0000001c       __imp__EncodePointer@4     1002601c     kernel32:KERNEL32.dll
 0002:00000020       __imp__GetPrivateProfileStringA@24 10026020     kernel32:KERNEL32.dll
 0002:00000024       __imp__GetSystemTimeAsFileTime@4 10026024     kernel32:KERNEL32.dll
 0002:00000028       \177KERNEL32_NULL_THUNK_DATA 10026028     kernel32:KERNEL32.dll
 0002:0000002c       __imp_?_Xbad_alloc@std@@YAXXZ 1002602c     msvcprt:MSVCP120.dll
 0002:00000030       __imp_?_Xout_of_range@std@@YAXPBD@Z 10026030     msvcprt:MSVCP120.dll
 0002:00000034       __imp_?_Syserror_map@std@@YAPBDH@Z 10026034     msvcprt:MSVCP120.dll
 0002:00000038       __imp_?_Winerror_map@std@@YAPBDH@Z 10026038     msvcprt:MSVCP120.dll
 0002:0000003c       __imp_?_Xlength_error@std@@YAXPBD@Z 1002603c     msvcprt:MSVCP120.dll
 0002:00000040       \177MSVCP120_NULL_THUNK_DATA 10026040     msvcprt:MSVCP120.dll
 0002:00000044       __imp___initterm           10026044     MSVCRT:MSVCR120.dll
 0002:00000048       __imp___malloc_crt         10026048     MSVCRT:MSVCR120.dll
 0002:0000004c       __imp__free                1002604c     MSVCRT:MSVCR120.dll
 0002:00000050       __imp___amsg_exit          10026050     MSVCRT:MSVCR120.dll
 0002:00000054       __imp____CppXcptFilter     10026054     MSVCRT:MSVCR120.dll
 0002:00000058       __imp_?terminate@@YAXXZ    10026058     MSVCRT:MSVCR120.dll
 0002:0000005c       __imp_??1type_info@@UAE@XZ 1002605c     MSVCRT:MSVCR120.dll
 0002:00000060       __imp___onexit             10026060     MSVCRT:MSVCR120.dll
 0002:00000064       __imp____dllonexit         10026064     MSVCRT:MSVCR120.dll
 0002:00000068       __imp___calloc_crt         10026068     MSVCRT:MSVCR120.dll
 0002:0000006c       __imp___unlock             1002606c     MSVCRT:MSVCR120.dll
 0002:00000070       __imp___lock               10026070     MSVCRT:MSVCR120.dll
 0002:00000074       __imp___initterm_e         10026074     MSVCRT:MSVCR120.dll
 0002:00000078       __imp__atoi                10026078     MSVCRT:MSVCR120.dll
 0002:0000007c       __imp__strcmp              1002607c     MSVCRT:MSVCR120.dll
 0002:00000080       __imp____CxxFrameHandler3  10026080     MSVCRT:MSVCR120.dll
 0002:00000084       __imp___CxxThrowException@8 10026084     MSVCRT:MSVCR120.dll
 0002:00000088       __imp__memmove             10026088     MSVCRT:MSVCR120.dll
 0002:0000008c       __imp__strlen              1002608c     MSVCRT:MSVCR120.dll
 0002:00000090       __imp__strcat              10026090     MSVCRT:MSVCR120.dll
 0002:00000094       __imp__strcpy              10026094     MSVCRT:MSVCR120.dll
 0002:00000098       __imp__memcpy              10026098     MSVCRT:MSVCR120.dll
 0002:0000009c       __imp_??3@YAXPAX@Z         1002609c     MSVCRT:MSVCR120.dll
 0002:000000a0       __imp_??2@YAPAXI@Z         100260a0     MSVCRT:MSVCR120.dll
 0002:000000a4       __imp___purecall           100260a4     MSVCRT:MSVCR120.dll
 0002:000000a8       __imp___except_handler4_common 100260a8     MSVCRT:MSVCR120.dll
 0002:000000ac       __imp___crt_debugger_hook  100260ac     MSVCRT:MSVCR120.dll
 0002:000000b0       __imp____crtUnhandledException 100260b0     MSVCRT:MSVCR120.dll
 0002:000000b4       __imp____clean_type_info_names_internal 100260b4     MSVCRT:MSVCR120.dll
 0002:000000b8       __imp____crtTerminateProcess 100260b8     MSVCRT:MSVCR120.dll
 0002:000000bc       \177MSVCR120_NULL_THUNK_DATA 100260bc     MSVCRT:MSVCR120.dll
 0002:000000c0       __imp_?metaObject@CAlm_sys_select@@UBEPAVQMetaObject@@XZ 100260c0     alm_sys_select:alm_sys_select.dll
 0002:000000c4       __imp_?qt_property@CAlm_sys_select@@UAE_NHHPAVQVariant@@@Z 100260c4     alm_sys_select:alm_sys_select.dll
 0002:000000c8       __imp_?qt_invoke@CAlm_sys_select@@UAE_NHPAUQUObject@@@Z 100260c8     alm_sys_select:alm_sys_select.dll
 0002:000000cc       __imp_?qt_emit@CAlm_sys_select@@UAE_NHPAUQUObject@@@Z 100260cc     alm_sys_select:alm_sys_select.dll
 0002:000000d0       __imp_?qt_cast@CAlm_sys_select@@UAEPAXPBD@Z 100260d0     alm_sys_select:alm_sys_select.dll
 0002:000000d4       __imp_?getSystemName@CAlm_sys_select@@QAE?AVQString@@XZ 100260d4     alm_sys_select:alm_sys_select.dll
 0002:000000d8       __imp_?className@CAlm_sys_select@@UBEPBDXZ 100260d8     alm_sys_select:alm_sys_select.dll
 0002:000000dc       __imp_??1CAlm_sys_select@@UAE@XZ 100260dc     alm_sys_select:alm_sys_select.dll
 0002:000000e0       __imp_??0CAlm_sys_select@@QAE@PAVQWidget@@PBD@Z 100260e0     alm_sys_select:alm_sys_select.dll
 0002:000000e4       __imp_?setSystemNames@CAlm_sys_select@@QAE_NVQString@@@Z 100260e4     alm_sys_select:alm_sys_select.dll
 0002:000000e8       \177alm_sys_select_NULL_THUNK_DATA 100260e8     alm_sys_select:alm_sys_select.dll
 0002:000000ec       __imp_?fnConfig_icons@@YAPAPBDPBD@Z 100260ec     config_icons:config_icons.dll
 0002:000000f0       \177config_icons_NULL_THUNK_DATA 100260f0     config_icons:config_icons.dll
 0002:000000f4       __imp_?begin@?$QMap@VQString@@H@@QAE?AV?$QMapIterator@VQString@@H@@XZ 100260f4     qt-mt323:qt-mt323.dll
 0002:000000f8       __imp_?end@?$QMap@VQString@@H@@QAE?AV?$QMapIterator@VQString@@H@@XZ 100260f8     qt-mt323:qt-mt323.dll
 0002:000000fc       __imp_??A?$QMap@VQString@@H@@QAEAAHABVQString@@@Z 100260fc     qt-mt323:qt-mt323.dll
 0002:00000100       __imp_?clear@?$QMap@VQString@@H@@QAEXXZ 10026100     qt-mt323:qt-mt323.dll
 0002:00000104       __imp_?contains@?$QMap@VQString@@H@@QBE_NABVQString@@@Z 10026104     qt-mt323:qt-mt323.dll
 0002:00000108       __imp_?remove@?$QMap@VQString@@H@@QAEXABVQString@@@Z 10026108     qt-mt323:qt-mt323.dll
 0002:0000010c       __imp_?connect@QObject@@SA_NPBV1@PBD01@Z 1002610c     qt-mt323:qt-mt323.dll
 0002:00000110       __imp_??0QStringList@@QAE@XZ 10026110     qt-mt323:qt-mt323.dll
 0002:00000114       __imp_?split@QStringList@@SA?AV1@ABVQString@@0_N@Z 10026114     qt-mt323:qt-mt323.dll
 0002:00000118       __imp_??1QStringList@@QAE@XZ 10026118     qt-mt323:qt-mt323.dll
 0002:0000011c       __imp_??4QStringList@@QAEAAV0@ABV0@@Z 1002611c     qt-mt323:qt-mt323.dll
 0002:00000120       __imp_??0QWidget@@QAE@PAV0@PBDI@Z 10026120     qt-mt323:qt-mt323.dll
 0002:00000124       __imp_??1QWidget@@UAE@XZ   10026124     qt-mt323:qt-mt323.dll
 0002:00000128       __imp_?setName@QWidget@@UAEXPBD@Z 10026128     qt-mt323:qt-mt323.dll
 0002:0000012c       __imp_?rect@QWidget@@QBE?AVQRect@@XZ 1002612c     qt-mt323:qt-mt323.dll
 0002:00000130       __imp_?update@QWidget@@QAEXXZ 10026130     qt-mt323:qt-mt323.dll
 0002:00000134       __imp_?exec@QDialog@@QAEHXZ 10026134     qt-mt323:qt-mt323.dll
 0002:00000138       __imp_?information@QMessageBox@@SAHPAVQWidget@@ABVQString@@1111HH@Z 10026138     qt-mt323:qt-mt323.dll
 0002:0000013c       __imp_?warning@QMessageBox@@SAHPAVQWidget@@ABVQString@@1111HH@Z 1002613c     qt-mt323:qt-mt323.dll
 0002:00000140       __imp_?critical@QMessageBox@@SAHPAVQWidget@@ABVQString@@1111HH@Z 10026140     qt-mt323:qt-mt323.dll
 0002:00000144       __imp_??0QPixmap@@QAE@QAPBD@Z 10026144     qt-mt323:qt-mt323.dll
 0002:00000148       __imp_??1QPixmap@@UAE@XZ   10026148     qt-mt323:qt-mt323.dll
 0002:0000014c       __imp_??0QIconSet@@QAE@ABVQPixmap@@W4Size@0@@Z 1002614c     qt-mt323:qt-mt323.dll
 0002:00000150       __imp_??1QIconSet@@UAE@XZ  10026150     qt-mt323:qt-mt323.dll
 0002:00000154       __imp_??0QKeySequence@@QAE@H@Z 10026154     qt-mt323:qt-mt323.dll
 0002:00000158       __imp_??0QAction@@QAE@ABVQString@@ABVQIconSet@@0VQKeySequence@@PAVQObject@@PBD_N@Z 10026158     qt-mt323:qt-mt323.dll
 0002:0000015c       __imp_??1QAction@@UAE@XZ   1002615c     qt-mt323:qt-mt323.dll
 0002:00000160       __imp_??0QDockWindow@@QAE@W4Place@0@PAVQWidget@@PBDI@Z 10026160     qt-mt323:qt-mt323.dll
 0002:00000164       __imp_??1QDockWindow@@UAE@XZ 10026164     qt-mt323:qt-mt323.dll
 0002:00000168       __imp_??1?$QPtrList@VQDockWindow@@@@UAE@XZ 10026168     qt-mt323:qt-mt323.dll
 0002:0000016c       __imp_??0QToolBar@@QAE@PAVQMainWindow@@PBD@Z 1002616c     qt-mt323:qt-mt323.dll
 0002:00000170       __imp_??1QToolBar@@UAE@XZ  10026170     qt-mt323:qt-mt323.dll
 0002:00000174       __imp_?currentItem@QComboBox@@QBEHXZ 10026174     qt-mt323:qt-mt323.dll
 0002:00000178       __imp_?currentText@QComboBox@@QBE?AVQString@@XZ 10026178     qt-mt323:qt-mt323.dll
 0002:0000017c       __imp_?text@QLineEdit@@QBE?AVQString@@XZ 1002617c     qt-mt323:qt-mt323.dll
 0002:00000180       __imp_?text@QSpinBox@@QBE?AVQString@@XZ 10026180     qt-mt323:qt-mt323.dll
 0002:00000184       __imp_?minValue@QSpinBox@@QBEHXZ 10026184     qt-mt323:qt-mt323.dll
 0002:00000188       __imp_?value@QSpinBox@@QBEHXZ 10026188     qt-mt323:qt-mt323.dll
 0002:0000018c       __imp_??0QListViewItem@@QAE@PAVQListView@@VQString@@1111111@Z 1002618c     qt-mt323:qt-mt323.dll
 0002:00000190       __imp_??1QListViewItem@@UAE@XZ 10026190     qt-mt323:qt-mt323.dll
 0002:00000194       __imp_?setVisible@QListViewItem@@QAEX_N@Z 10026194     qt-mt323:qt-mt323.dll
 0002:00000198       __imp_??0QListView@@QAE@PAVQWidget@@PBDI@Z 10026198     qt-mt323:qt-mt323.dll
 0002:0000019c       __imp_??1QListView@@UAE@XZ 1002619c     qt-mt323:qt-mt323.dll
 0002:000001a0       __imp_?ensureItemVisible@QListView@@QAEXPBVQListViewItem@@@Z 100261a0     qt-mt323:qt-mt323.dll
 0002:000001a4       __imp_?selectedItem@QListView@@QBEPAVQListViewItem@@XZ 100261a4     qt-mt323:qt-mt323.dll
 0002:000001a8       __imp_?currentItem@QListView@@QBEPAVQListViewItem@@XZ 100261a8     qt-mt323:qt-mt323.dll
 0002:000001ac       __imp_?firstChild@QListView@@QBEPAVQListViewItem@@XZ 100261ac     qt-mt323:qt-mt323.dll
 0002:000001b0       __imp_?findItem@QListView@@QBEPAVQListViewItem@@ABVQString@@HI@Z 100261b0     qt-mt323:qt-mt323.dll
 0002:000001b4       __imp_??0QListViewItemIterator@@QAE@XZ 100261b4     qt-mt323:qt-mt323.dll
 0002:000001b8       __imp_??0QListViewItemIterator@@QAE@PAVQListView@@@Z 100261b8     qt-mt323:qt-mt323.dll
 0002:000001bc       __imp_??4QListViewItemIterator@@QAEAAV0@ABV0@@Z 100261bc     qt-mt323:qt-mt323.dll
 0002:000001c0       __imp_??1QListViewItemIterator@@QAE@XZ 100261c0     qt-mt323:qt-mt323.dll
 0002:000001c4       __imp_??EQListViewItemIterator@@QAE?BV0@H@Z 100261c4     qt-mt323:qt-mt323.dll
 0002:000001c8       __imp_?current@QListViewItemIterator@@QBEPAVQListViewItem@@XZ 100261c8     qt-mt323:qt-mt323.dll
 0002:000001cc       __imp_??0QFile@@QAE@ABVQString@@@Z 100261cc     qt-mt323:qt-mt323.dll
 0002:000001d0       __imp_??1QFile@@UAE@XZ     100261d0     qt-mt323:qt-mt323.dll
 0002:000001d4       __imp_?exists@QFile@@QBE_NXZ 100261d4     qt-mt323:qt-mt323.dll
 0002:000001d8       __imp_?remove@QFile@@QAE_NXZ 100261d8     qt-mt323:qt-mt323.dll
 0002:000001dc       __imp_?open@QFile@@UAE_NH@Z 100261dc     qt-mt323:qt-mt323.dll
 0002:000001e0       __imp_?close@QFile@@UAEXXZ 100261e0     qt-mt323:qt-mt323.dll
 0002:000001e4       __imp_??8QDateTime@@QBE_NABV0@@Z 100261e4     qt-mt323:qt-mt323.dll
 0002:000001e8       __imp_??9QDateTime@@QBE_NABV0@@Z 100261e8     qt-mt323:qt-mt323.dll
 0002:000001ec       __imp_??0QFileInfo@@QAE@XZ 100261ec     qt-mt323:qt-mt323.dll
 0002:000001f0       __imp_??0QFileInfo@@QAE@ABVQString@@@Z 100261f0     qt-mt323:qt-mt323.dll
 0002:000001f4       __imp_??1QFileInfo@@QAE@XZ 100261f4     qt-mt323:qt-mt323.dll
 0002:000001f8       __imp_?setFile@QFileInfo@@QAEXABVQString@@@Z 100261f8     qt-mt323:qt-mt323.dll
 0002:000001fc       __imp_?exists@QFileInfo@@QBE_NXZ 100261fc     qt-mt323:qt-mt323.dll
 0002:00000200       __imp_?isFile@QFileInfo@@QBE_NXZ 10026200     qt-mt323:qt-mt323.dll
 0002:00000204       __imp_?lastModified@QFileInfo@@QBE?AVQDateTime@@XZ 10026204     qt-mt323:qt-mt323.dll
 0002:00000208       __imp_??0QTabWidget@@QAE@PAVQWidget@@PBDI@Z 10026208     qt-mt323:qt-mt323.dll
 0002:0000020c       __imp_??1QTabWidget@@UAE@XZ 1002620c     qt-mt323:qt-mt323.dll
 0002:00000210       __imp_?currentPage@QTabWidget@@QBEPAVQWidget@@XZ 10026210     qt-mt323:qt-mt323.dll
 0002:00000214       __imp_?setCurrentPage@QTabWidget@@QAEXH@Z 10026214     qt-mt323:qt-mt323.dll
 0002:00000218       __imp_??0QDir@@QAE@XZ      10026218     qt-mt323:qt-mt323.dll
 0002:0000021c       __imp_??0QDir@@QAE@ABVQString@@0HH@Z 1002621c     qt-mt323:qt-mt323.dll
 0002:00000220       __imp_??1QDir@@UAE@XZ      10026220     qt-mt323:qt-mt323.dll
 0002:00000224       __imp_?setPath@QDir@@UAEXABVQString@@@Z 10026224     qt-mt323:qt-mt323.dll
 0002:00000228       __imp_?entryList@QDir@@UBE?AVQStringList@@HH@Z 10026228     qt-mt323:qt-mt323.dll
 0002:0000022c       __imp_?mkdir@QDir@@UBE_NABVQString@@_N@Z 1002622c     qt-mt323:qt-mt323.dll
 0002:00000230       __imp_?exists@QDir@@UBE_NXZ 10026230     qt-mt323:qt-mt323.dll
 0002:00000234       __imp_?add@QLayout@@QAEXPAVQWidget@@@Z 10026234     qt-mt323:qt-mt323.dll
 0002:00000238       __imp_??0QBoxLayout@@QAE@PAVQWidget@@W4Direction@0@HHPBD@Z 10026238     qt-mt323:qt-mt323.dll
 0002:0000023c       __imp_??1QBoxLayout@@UAE@XZ 1002623c     qt-mt323:qt-mt323.dll
 0002:00000240       __imp_?text@QClipboard@@QBE?AVQString@@XZ 10026240     qt-mt323:qt-mt323.dll
 0002:00000244       __imp_?setText@QClipboard@@QAEXABVQString@@@Z 10026244     qt-mt323:qt-mt323.dll
 0002:00000248       __imp_??0QGDict@@IAE@IW4KeyType@0@_N1@Z 10026248     qt-mt323:qt-mt323.dll
 0002:0000024c       __imp_??1QGDict@@MAE@XZ    1002624c     qt-mt323:qt-mt323.dll
 0002:00000250       __imp_?clear@QGDict@@MAEXXZ 10026250     qt-mt323:qt-mt323.dll
 0002:00000254       __imp_?clipboard@QApplication@@SAPAVQClipboard@@XZ 10026254     qt-mt323:qt-mt323.dll
 0002:00000258       __imp_??0QRegExp@@QAE@ABVQString@@_N1@Z 10026258     qt-mt323:qt-mt323.dll
 0002:0000025c       __imp_??1QRegExp@@QAE@XZ   1002625c     qt-mt323:qt-mt323.dll
 0002:00000260       __imp_?setCaseSensitive@QRegExp@@QAEX_N@Z 10026260     qt-mt323:qt-mt323.dll
 0002:00000264       __imp_?search@QRegExp@@QBEHABVQString@@H@Z 10026264     qt-mt323:qt-mt323.dll
 0002:00000268       __imp_??0QGuardedPtrPrivate@@QAE@PAVQObject@@@Z 10026268     qt-mt323:qt-mt323.dll
 0002:0000026c       __imp_??1QGuardedPtrPrivate@@UAE@XZ 1002626c     qt-mt323:qt-mt323.dll
 0002:00000270       __imp_?reconnect@QGuardedPtrPrivate@@QAEXPAVQObject@@@Z 10026270     qt-mt323:qt-mt323.dll
 0002:00000274       __imp_?isChecked@QCheckTableItem@@QBE_NXZ 10026274     qt-mt323:qt-mt323.dll
 0002:00000278       __imp_??0QPopupMenu@@QAE@PAVQWidget@@PBD@Z 10026278     qt-mt323:qt-mt323.dll
 0002:0000027c       __imp_??1QPopupMenu@@UAE@XZ 1002627c     qt-mt323:qt-mt323.dll
 0002:00000280       __imp_?exec@QPopupMenu@@QAEHABVQPoint@@H@Z 10026280     qt-mt323:qt-mt323.dll
 0002:00000284       __imp_?acceptDrop@QListViewItem@@UBE_NPBVQMimeSource@@@Z 10026284     qt-mt323:qt-mt323.dll
 0002:00000288       __imp_?activate@QListViewItem@@MAEXXZ 10026288     qt-mt323:qt-mt323.dll
 0002:0000028c       __imp_?activateItemAt@QPopupMenu@@UAEXH@Z 1002628c     qt-mt323:qt-mt323.dll
 0002:00000290       __imp_?addChild@QScrollView@@UAEXPAVQWidget@@HH@Z 10026290     qt-mt323:qt-mt323.dll
 0002:00000294       __imp_?addColumn@QListView@@UAEHABVQIconSet@@ABVQString@@H@Z 10026294     qt-mt323:qt-mt323.dll
 0002:00000298       __imp_?addColumn@QListView@@UAEHABVQString@@H@Z 10026298     qt-mt323:qt-mt323.dll
 0002:0000029c       __imp_?addItem@QBoxLayout@@UAEXPAVQLayoutItem@@@Z 1002629c     qt-mt323:qt-mt323.dll
 0002:000002a0       __imp_?addTab@QTabWidget@@UAEXPAVQWidget@@ABVQIconSet@@ABVQString@@@Z 100262a0     qt-mt323:qt-mt323.dll
 0002:000002a4       __imp_?addTab@QTabWidget@@UAEXPAVQWidget@@ABVQString@@@Z 100262a4     qt-mt323:qt-mt323.dll
 0002:000002a8       __imp_?addTab@QTabWidget@@UAEXPAVQWidget@@PAVQTab@@@Z 100262a8     qt-mt323:qt-mt323.dll
 0002:000002ac       __imp_?addTo@QAction@@UAE_NPAVQWidget@@@Z 100262ac     qt-mt323:qt-mt323.dll
 0002:000002b0       __imp_?addedTo@QAction@@MAEXHPAVQPopupMenu@@@Z 100262b0     qt-mt323:qt-mt323.dll
 0002:000002b4       __imp_?addedTo@QAction@@MAEXPAVQWidget@@0@Z 100262b4     qt-mt323:qt-mt323.dll
 0002:000002b8       __imp_?adjustSize@QWidget@@UAEXXZ 100262b8     qt-mt323:qt-mt323.dll
 0002:000002bc       __imp_?at@QFile@@UAE_NK@Z  100262bc     qt-mt323:qt-mt323.dll
 0002:000002c0       __imp_?at@QFile@@UBEKXZ    100262c0     qt-mt323:qt-mt323.dll
 0002:000002c4       __imp_?atEnd@QFile@@UBE_NXZ 100262c4     qt-mt323:qt-mt323.dll
 0002:000002c8       __imp_?cancelRename@QListViewItem@@MAEXH@Z 100262c8     qt-mt323:qt-mt323.dll
 0002:000002cc       __imp_?checkConnectArgs@QObject@@MAE_NPBDPBV1@0@Z 100262cc     qt-mt323:qt-mt323.dll
 0002:000002d0       __imp_?childEvent@QLayout@@MAEXPAVQChildEvent@@@Z 100262d0     qt-mt323:qt-mt323.dll
 0002:000002d4       __imp_?childEvent@QObject@@MAEXPAVQChildEvent@@@Z 100262d4     qt-mt323:qt-mt323.dll
 0002:000002d8       __imp_?className@QAction@@UBEPBDXZ 100262d8     qt-mt323:qt-mt323.dll
 0002:000002dc       __imp_?className@QBoxLayout@@UBEPBDXZ 100262dc     qt-mt323:qt-mt323.dll
 0002:000002e0       __imp_?className@QDockWindow@@UBEPBDXZ 100262e0     qt-mt323:qt-mt323.dll
 0002:000002e4       __imp_?className@QGuardedPtrPrivate@@UBEPBDXZ 100262e4     qt-mt323:qt-mt323.dll
 0002:000002e8       __imp_?className@QListView@@UBEPBDXZ 100262e8     qt-mt323:qt-mt323.dll
 0002:000002ec       __imp_?className@QPopupMenu@@UBEPBDXZ 100262ec     qt-mt323:qt-mt323.dll
 0002:000002f0       __imp_?className@QTabWidget@@UBEPBDXZ 100262f0     qt-mt323:qt-mt323.dll
 0002:000002f4       __imp_?className@QToolBar@@UBEPBDXZ 100262f4     qt-mt323:qt-mt323.dll
 0002:000002f8       __imp_?className@QWidget@@UBEPBDXZ 100262f8     qt-mt323:qt-mt323.dll
 0002:000002fc       __imp_?clear@?$QPtrList@VQDockWindow@@@@UAEXXZ 100262fc     qt-mt323:qt-mt323.dll
 0002:00000300       __imp_?clear@QListView@@UAEXXZ 10026300     qt-mt323:qt-mt323.dll
 0002:00000304       __imp_?clear@QToolBar@@UAEXXZ 10026304     qt-mt323:qt-mt323.dll
 0002:00000308       __imp_?clearSelection@QListView@@UAEXXZ 10026308     qt-mt323:qt-mt323.dll
 0002:0000030c       __imp_?close@QWidget@@UAE_N_N@Z 1002630c     qt-mt323:qt-mt323.dll
 0002:00000310       __imp_?closeEvent@QPopupMenu@@MAEXPAVQCloseEvent@@@Z 10026310     qt-mt323:qt-mt323.dll
 0002:00000314       __imp_?closeEvent@QWidget@@MAEXPAVQCloseEvent@@@Z 10026314     qt-mt323:qt-mt323.dll
 0002:00000318       __imp_?cmd@QPaintDevice@@MAE_NHPAVQPainter@@PATQPDevCmdParam@@@Z 10026318     qt-mt323:qt-mt323.dll
 0002:0000031c       __imp_?compare@QListViewItem@@UBEHPAV1@H_N@Z 1002631c     qt-mt323:qt-mt323.dll
 0002:00000320       __imp_?compareItems@QGList@@MAEHPAX0@Z 10026320     qt-mt323:qt-mt323.dll
 0002:00000324       __imp_?connectNotify@QObject@@MAEXPBD@Z 10026324     qt-mt323:qt-mt323.dll
 0002:00000328       __imp_?contentsContextMenuEvent@QListView@@MAEXPAVQContextMenuEvent@@@Z 10026328     qt-mt323:qt-mt323.dll
 0002:0000032c       __imp_?contentsDragEnterEvent@QListView@@MAEXPAVQDragEnterEvent@@@Z 1002632c     qt-mt323:qt-mt323.dll
 0002:00000330       __imp_?contentsDragLeaveEvent@QListView@@MAEXPAVQDragLeaveEvent@@@Z 10026330     qt-mt323:qt-mt323.dll
 0002:00000334       __imp_?contentsDragMoveEvent@QListView@@MAEXPAVQDragMoveEvent@@@Z 10026334     qt-mt323:qt-mt323.dll
 0002:00000338       __imp_?contentsDropEvent@QListView@@MAEXPAVQDropEvent@@@Z 10026338     qt-mt323:qt-mt323.dll
 0002:0000033c       __imp_?contentsMouseDoubleClickEvent@QListView@@MAEXPAVQMouseEvent@@@Z 1002633c     qt-mt323:qt-mt323.dll
 0002:00000340       __imp_?contentsMouseMoveEvent@QListView@@MAEXPAVQMouseEvent@@@Z 10026340     qt-mt323:qt-mt323.dll
 0002:00000344       __imp_?contentsMousePressEvent@QListView@@MAEXPAVQMouseEvent@@@Z 10026344     qt-mt323:qt-mt323.dll
 0002:00000348       __imp_?contentsMouseReleaseEvent@QListView@@MAEXPAVQMouseEvent@@@Z 10026348     qt-mt323:qt-mt323.dll
 0002:0000034c       __imp_?contentsWheelEvent@QScrollView@@MAEXPAVQWheelEvent@@@Z 1002634c     qt-mt323:qt-mt323.dll
 0002:00000350       __imp_?contextMenuEvent@QDockWindow@@MAEXPAVQContextMenuEvent@@@Z 10026350     qt-mt323:qt-mt323.dll
 0002:00000354       __imp_?contextMenuEvent@QScrollView@@MAEXPAVQContextMenuEvent@@@Z 10026354     qt-mt323:qt-mt323.dll
 0002:00000358       __imp_?contextMenuEvent@QWidget@@MAEXPAVQContextMenuEvent@@@Z 10026358     qt-mt323:qt-mt323.dll
 0002:0000035c       __imp_?count@?$QPtrList@VQDockWindow@@@@UBEIXZ 1002635c     qt-mt323:qt-mt323.dll
 0002:00000360       __imp_?create@QWidget@@MAEXPAUHWND__@@_N1@Z 10026360     qt-mt323:qt-mt323.dll
 0002:00000364       __imp_?customEvent@QObject@@MAEXPAVQCustomEvent@@@Z 10026364     qt-mt323:qt-mt323.dll
 0002:00000368       __imp_?customWhatsThis@QPopupMenu@@UBE_NXZ 10026368     qt-mt323:qt-mt323.dll
 0002:0000036c       __imp_?customWhatsThis@QWidget@@UBE_NXZ 1002636c     qt-mt323:qt-mt323.dll
 0002:00000370       __imp_?deleteItem@?$QPtrList@VQDockWindow@@@@EAEXPAX@Z 10026370     qt-mt323:qt-mt323.dll
 0002:00000374       __imp_?destroy@QWidget@@MAEX_N0@Z 10026374     qt-mt323:qt-mt323.dll
 0002:00000378       __imp_?disconnectNotify@QObject@@MAEXPBD@Z 10026378     qt-mt323:qt-mt323.dll
 0002:0000037c       __imp_?dock@QDockWindow@@UAEXXZ 1002637c     qt-mt323:qt-mt323.dll
 0002:00000380       __imp_?dragEnterEvent@QWidget@@MAEXPAVQDragEnterEvent@@@Z 10026380     qt-mt323:qt-mt323.dll
 0002:00000384       __imp_?dragEntered@QListViewItem@@MAEXXZ 10026384     qt-mt323:qt-mt323.dll
 0002:00000388       __imp_?dragLeaveEvent@QWidget@@MAEXPAVQDragLeaveEvent@@@Z 10026388     qt-mt323:qt-mt323.dll
 0002:0000038c       __imp_?dragLeft@QListViewItem@@MAEXXZ 1002638c     qt-mt323:qt-mt323.dll
 0002:00000390       __imp_?dragMoveEvent@QWidget@@MAEXPAVQDragMoveEvent@@@Z 10026390     qt-mt323:qt-mt323.dll
 0002:00000394       __imp_?dragObject@QListView@@MAEPAVQDragObject@@XZ 10026394     qt-mt323:qt-mt323.dll
 0002:00000398       __imp_?drawContents@QDockWindow@@MAEXPAVQPainter@@@Z 10026398     qt-mt323:qt-mt323.dll
 0002:0000039c       __imp_?drawContents@QFrame@@MAEXPAVQPainter@@@Z 1002639c     qt-mt323:qt-mt323.dll
 0002:000003a0       __imp_?drawContents@QPopupMenu@@MAEXPAVQPainter@@@Z 100263a0     qt-mt323:qt-mt323.dll
 0002:000003a4       __imp_?drawContents@QScrollView@@EAEXPAVQPainter@@@Z 100263a4     qt-mt323:qt-mt323.dll
 0002:000003a8       __imp_?drawContents@QScrollView@@MAEXPAVQPainter@@HHHH@Z 100263a8     qt-mt323:qt-mt323.dll
 0002:000003ac       __imp_?drawContentsOffset@QListView@@MAEXPAVQPainter@@HHHHHH@Z 100263ac     qt-mt323:qt-mt323.dll
 0002:000003b0       __imp_?drawFrame@QDockWindow@@MAEXPAVQPainter@@@Z 100263b0     qt-mt323:qt-mt323.dll
 0002:000003b4       __imp_?drawFrame@QFrame@@MAEXPAVQPainter@@@Z 100263b4     qt-mt323:qt-mt323.dll
 0002:000003b8       __imp_?dropEvent@QWidget@@MAEXPAVQDropEvent@@@Z 100263b8     qt-mt323:qt-mt323.dll
 0002:000003bc       __imp_?dropped@QListViewItem@@MAEXPAVQDropEvent@@@Z 100263bc     qt-mt323:qt-mt323.dll
 0002:000003c0       __imp_?enabledChange@QPopupMenu@@MAEX_N@Z 100263c0     qt-mt323:qt-mt323.dll
 0002:000003c4       __imp_?enabledChange@QWidget@@MAEX_N@Z 100263c4     qt-mt323:qt-mt323.dll
 0002:000003c8       __imp_?enforceSortOrder@QListViewItem@@MBEXXZ 100263c8     qt-mt323:qt-mt323.dll
 0002:000003cc       __imp_?enterEvent@QWidget@@MAEXPAVQEvent@@@Z 100263cc     qt-mt323:qt-mt323.dll
 0002:000003d0       __imp_?event@QDockWindow@@MAE_NPAVQEvent@@@Z 100263d0     qt-mt323:qt-mt323.dll
 0002:000003d4       __imp_?event@QObject@@UAE_NPAVQEvent@@@Z 100263d4     qt-mt323:qt-mt323.dll
 0002:000003d8       __imp_?event@QToolBar@@UAE_NPAVQEvent@@@Z 100263d8     qt-mt323:qt-mt323.dll
 0002:000003dc       __imp_?event@QWidget@@MAE_NPAVQEvent@@@Z 100263dc     qt-mt323:qt-mt323.dll
 0002:000003e0       __imp_?eventFilter@QDockWindow@@UAE_NPAVQObject@@PAVQEvent@@@Z 100263e0     qt-mt323:qt-mt323.dll
 0002:000003e4       __imp_?eventFilter@QLayout@@MAE_NPAVQObject@@PAVQEvent@@@Z 100263e4     qt-mt323:qt-mt323.dll
 0002:000003e8       __imp_?eventFilter@QListView@@UAE_NPAVQObject@@PAVQEvent@@@Z 100263e8     qt-mt323:qt-mt323.dll
 0002:000003ec       __imp_?eventFilter@QObject@@UAE_NPAV1@PAVQEvent@@@Z 100263ec     qt-mt323:qt-mt323.dll
 0002:000003f0       __imp_?eventFilter@QTabWidget@@MAE_NPAVQObject@@PAVQEvent@@@Z 100263f0     qt-mt323:qt-mt323.dll
 0002:000003f4       __imp_?expanding@QBoxLayout@@UBE?AW4ExpandData@QSizePolicy@@XZ 100263f4     qt-mt323:qt-mt323.dll
 0002:000003f8       __imp_?flush@QFile@@UAEXXZ 100263f8     qt-mt323:qt-mt323.dll
 0002:000003fc       __imp_?focusInEvent@QListView@@MAEXPAVQFocusEvent@@@Z 100263fc     qt-mt323:qt-mt323.dll
 0002:00000400       __imp_?focusInEvent@QPopupMenu@@MAEXPAVQFocusEvent@@@Z 10026400     qt-mt323:qt-mt323.dll
 0002:00000404       __imp_?focusInEvent@QWidget@@MAEXPAVQFocusEvent@@@Z 10026404     qt-mt323:qt-mt323.dll
 0002:00000408       __imp_?focusNextPrevChild@QPopupMenu@@MAE_N_N@Z 10026408     qt-mt323:qt-mt323.dll
 0002:0000040c       __imp_?focusNextPrevChild@QScrollView@@MAE_N_N@Z 1002640c     qt-mt323:qt-mt323.dll
 0002:00000410       __imp_?focusNextPrevChild@QWidget@@MAE_N_N@Z 10026410     qt-mt323:qt-mt323.dll
 0002:00000414       __imp_?focusOutEvent@QListView@@MAEXPAVQFocusEvent@@@Z 10026414     qt-mt323:qt-mt323.dll
 0002:00000418       __imp_?focusOutEvent@QPopupMenu@@MAEXPAVQFocusEvent@@@Z 10026418     qt-mt323:qt-mt323.dll
 0002:0000041c       __imp_?focusOutEvent@QWidget@@MAEXPAVQFocusEvent@@@Z 1002641c     qt-mt323:qt-mt323.dll
 0002:00000420       __imp_?fontChange@QScrollView@@MAEXABVQFont@@@Z 10026420     qt-mt323:qt-mt323.dll
 0002:00000424       __imp_?fontChange@QWidget@@MAEXABVQFont@@@Z 10026424     qt-mt323:qt-mt323.dll
 0002:00000428       __imp_?fontInf@QPaintDevice@@MBEHPAVQFont@@H@Z 10026428     qt-mt323:qt-mt323.dll
 0002:0000042c       __imp_?fontMet@QPaintDevice@@MBEHPAVQFont@@HPBDH@Z 1002642c     qt-mt323:qt-mt323.dll
 0002:00000430       __imp_?frameChanged@QFrame@@MAEXXZ 10026430     qt-mt323:qt-mt323.dll
 0002:00000434       __imp_?frameChanged@QHBox@@MAEXXZ 10026434     qt-mt323:qt-mt323.dll
 0002:00000438       __imp_?frameChanged@QPopupMenu@@EAEXXZ 10026438     qt-mt323:qt-mt323.dll
 0002:0000043c       __imp_?frameChanged@QScrollView@@MAEXXZ 1002643c     qt-mt323:qt-mt323.dll
 0002:00000440       __imp_?geometry@QLayout@@UBE?AVQRect@@XZ 10026440     qt-mt323:qt-mt323.dll
 0002:00000444       __imp_?getch@QFile@@UAEHXZ 10026444     qt-mt323:qt-mt323.dll
 0002:00000448       __imp_?handle@QPaintDevice@@UBEPAUHDC__@@XZ 10026448     qt-mt323:qt-mt323.dll
 0002:0000044c       __imp_?hasHeightForWidth@QBoxLayout@@UBE_NXZ 1002644c     qt-mt323:qt-mt323.dll
 0002:00000450       __imp_?heightForWidth@QBoxLayout@@UBEHH@Z 10026450     qt-mt323:qt-mt323.dll
 0002:00000454       __imp_?heightForWidth@QWidget@@UBEHH@Z 10026454     qt-mt323:qt-mt323.dll
 0002:00000458       __imp_?hide@QPopupMenu@@UAEXXZ 10026458     qt-mt323:qt-mt323.dll
 0002:0000045c       __imp_?hide@QToolBar@@UAEXXZ 1002645c     qt-mt323:qt-mt323.dll
 0002:00000460       __imp_?hide@QWidget@@UAEXXZ 10026460     qt-mt323:qt-mt323.dll
 0002:00000464       __imp_?hideEvent@QDockWindow@@MAEXPAVQHideEvent@@@Z 10026464     qt-mt323:qt-mt323.dll
 0002:00000468       __imp_?hideEvent@QWidget@@MAEXPAVQHideEvent@@@Z 10026468     qt-mt323:qt-mt323.dll
 0002:0000046c       __imp_?imComposeEvent@QWidget@@MAEXPAVQIMEvent@@@Z 1002646c     qt-mt323:qt-mt323.dll
 0002:00000470       __imp_?imEndEvent@QWidget@@MAEXPAVQIMEvent@@@Z 10026470     qt-mt323:qt-mt323.dll
 0002:00000474       __imp_?imStartEvent@QWidget@@MAEXPAVQIMEvent@@@Z 10026474     qt-mt323:qt-mt323.dll
 0002:00000478       __imp_?insertChild@QObject@@UAEXPAV1@@Z 10026478     qt-mt323:qt-mt323.dll
 0002:0000047c       __imp_?insertItem@QListView@@UAEXPAVQListViewItem@@@Z 1002647c     qt-mt323:qt-mt323.dll
 0002:00000480       __imp_?insertItem@QListViewItem@@UAEXPAV1@@Z 10026480     qt-mt323:qt-mt323.dll
 0002:00000484       __imp_?insertTab@QTabWidget@@UAEXPAVQWidget@@ABVQIconSet@@ABVQString@@H@Z 10026484     qt-mt323:qt-mt323.dll
 0002:00000488       __imp_?insertTab@QTabWidget@@UAEXPAVQWidget@@ABVQString@@H@Z 10026488     qt-mt323:qt-mt323.dll
 0002:0000048c       __imp_?insertTab@QTabWidget@@UAEXPAVQWidget@@PAVQTab@@H@Z 1002648c     qt-mt323:qt-mt323.dll
 0002:00000490       __imp_?invalidate@QBoxLayout@@UAEXXZ 10026490     qt-mt323:qt-mt323.dll
 0002:00000494       __imp_?invalidateHeight@QListViewItem@@UAEXXZ 10026494     qt-mt323:qt-mt323.dll
 0002:00000498       __imp_?invertSelection@QListView@@UAEXXZ 10026498     qt-mt323:qt-mt323.dll
 0002:0000049c       __imp_?isEmpty@QLayout@@UBE_NXZ 1002649c     qt-mt323:qt-mt323.dll
 0002:000004a0       __imp_?iterator@QBoxLayout@@UAE?AVQLayoutIterator@@XZ 100264a0     qt-mt323:qt-mt323.dll
 0002:000004a4       __imp_?key@QListViewItem@@UBE?AVQString@@H_N@Z 100264a4     qt-mt323:qt-mt323.dll
 0002:000004a8       __imp_?keyPressEvent@QListView@@MAEXPAVQKeyEvent@@@Z 100264a8     qt-mt323:qt-mt323.dll
 0002:000004ac       __imp_?keyPressEvent@QPopupMenu@@MAEXPAVQKeyEvent@@@Z 100264ac     qt-mt323:qt-mt323.dll
 0002:000004b0       __imp_?keyPressEvent@QWidget@@MAEXPAVQKeyEvent@@@Z 100264b0     qt-mt323:qt-mt323.dll
 0002:000004b4       __imp_?keyReleaseEvent@QWidget@@MAEXPAVQKeyEvent@@@Z 100264b4     qt-mt323:qt-mt323.dll
 0002:000004b8       __imp_?layout@QLayout@@UAEPAV1@XZ 100264b8     qt-mt323:qt-mt323.dll
 0002:000004bc       __imp_?leaveEvent@QPopupMenu@@MAEXPAVQEvent@@@Z 100264bc     qt-mt323:qt-mt323.dll
 0002:000004c0       __imp_?leaveEvent@QWidget@@MAEXPAVQEvent@@@Z 100264c0     qt-mt323:qt-mt323.dll
 0002:000004c4       __imp_?maximumSize@QBoxLayout@@UBE?AVQSize@@XZ 100264c4     qt-mt323:qt-mt323.dll
 0002:000004c8       __imp_?menuContentsChanged@QPopupMenu@@EAEXXZ 100264c8     qt-mt323:qt-mt323.dll
 0002:000004cc       __imp_?menuDelPopup@QPopupMenu@@EAEXPAV1@@Z 100264cc     qt-mt323:qt-mt323.dll
 0002:000004d0       __imp_?menuInsPopup@QPopupMenu@@EAEXPAV1@@Z 100264d0     qt-mt323:qt-mt323.dll
 0002:000004d4       __imp_?menuStateChanged@QPopupMenu@@EAEXXZ 100264d4     qt-mt323:qt-mt323.dll
 0002:000004d8       __imp_?metaObject@QAction@@UBEPAVQMetaObject@@XZ 100264d8     qt-mt323:qt-mt323.dll
 0002:000004dc       __imp_?metaObject@QBoxLayout@@UBEPAVQMetaObject@@XZ 100264dc     qt-mt323:qt-mt323.dll
 0002:000004e0       __imp_?metaObject@QDockWindow@@UBEPAVQMetaObject@@XZ 100264e0     qt-mt323:qt-mt323.dll
 0002:000004e4       __imp_?metaObject@QGuardedPtrPrivate@@UBEPAVQMetaObject@@XZ 100264e4     qt-mt323:qt-mt323.dll
 0002:000004e8       __imp_?metaObject@QListView@@UBEPAVQMetaObject@@XZ 100264e8     qt-mt323:qt-mt323.dll
 0002:000004ec       __imp_?metaObject@QPopupMenu@@UBEPAVQMetaObject@@XZ 100264ec     qt-mt323:qt-mt323.dll
 0002:000004f0       __imp_?metaObject@QTabWidget@@UBEPAVQMetaObject@@XZ 100264f0     qt-mt323:qt-mt323.dll
 0002:000004f4       __imp_?metaObject@QToolBar@@UBEPAVQMetaObject@@XZ 100264f4     qt-mt323:qt-mt323.dll
 0002:000004f8       __imp_?metaObject@QWidget@@UBEPAVQMetaObject@@XZ 100264f8     qt-mt323:qt-mt323.dll
 0002:000004fc       __imp_?metric@QWidget@@MBEHH@Z 100264fc     qt-mt323:qt-mt323.dll
 0002:00000500       __imp_?minimumSize@QBoxLayout@@UBE?AVQSize@@XZ 10026500     qt-mt323:qt-mt323.dll
 0002:00000504       __imp_?minimumSizeHint@QDockWindow@@UBE?AVQSize@@XZ 10026504     qt-mt323:qt-mt323.dll
 0002:00000508       __imp_?minimumSizeHint@QListView@@UBE?AVQSize@@XZ 10026508     qt-mt323:qt-mt323.dll
 0002:0000050c       __imp_?minimumSizeHint@QTabWidget@@UBE?AVQSize@@XZ 1002650c     qt-mt323:qt-mt323.dll
 0002:00000510       __imp_?minimumSizeHint@QToolBar@@UBE?AVQSize@@XZ 10026510     qt-mt323:qt-mt323.dll
 0002:00000514       __imp_?minimumSizeHint@QWidget@@UBE?AVQSize@@XZ 10026514     qt-mt323:qt-mt323.dll
 0002:00000518       __imp_?mouseDoubleClickEvent@QScrollView@@MAEXPAVQMouseEvent@@@Z 10026518     qt-mt323:qt-mt323.dll
 0002:0000051c       __imp_?mouseDoubleClickEvent@QWidget@@MAEXPAVQMouseEvent@@@Z 1002651c     qt-mt323:qt-mt323.dll
 0002:00000520       __imp_?mouseMoveEvent@QPopupMenu@@MAEXPAVQMouseEvent@@@Z 10026520     qt-mt323:qt-mt323.dll
 0002:00000524       __imp_?mouseMoveEvent@QScrollView@@MAEXPAVQMouseEvent@@@Z 10026524     qt-mt323:qt-mt323.dll
 0002:00000528       __imp_?mouseMoveEvent@QWidget@@MAEXPAVQMouseEvent@@@Z 10026528     qt-mt323:qt-mt323.dll
 0002:0000052c       __imp_?mousePressEvent@QPopupMenu@@MAEXPAVQMouseEvent@@@Z 1002652c     qt-mt323:qt-mt323.dll
 0002:00000530       __imp_?mousePressEvent@QScrollView@@MAEXPAVQMouseEvent@@@Z 10026530     qt-mt323:qt-mt323.dll
 0002:00000534       __imp_?mousePressEvent@QWidget@@MAEXPAVQMouseEvent@@@Z 10026534     qt-mt323:qt-mt323.dll
 0002:00000538       __imp_?mouseReleaseEvent@QPopupMenu@@MAEXPAVQMouseEvent@@@Z 10026538     qt-mt323:qt-mt323.dll
 0002:0000053c       __imp_?mouseReleaseEvent@QScrollView@@MAEXPAVQMouseEvent@@@Z 1002653c     qt-mt323:qt-mt323.dll
 0002:00000540       __imp_?mouseReleaseEvent@QWidget@@MAEXPAVQMouseEvent@@@Z 10026540     qt-mt323:qt-mt323.dll
 0002:00000544       __imp_?move@QWidget@@UAEXHH@Z 10026544     qt-mt323:qt-mt323.dll
 0002:00000548       __imp_?moveChild@QScrollView@@UAEXPAVQWidget@@HH@Z 10026548     qt-mt323:qt-mt323.dll
 0002:0000054c       __imp_?moveEvent@QWidget@@MAEXPAVQMoveEvent@@@Z 1002654c     qt-mt323:qt-mt323.dll
 0002:00000550       __imp_?newItem@QPtrCollection@@MAEPAXPAX@Z 10026550     qt-mt323:qt-mt323.dll
 0002:00000554       __imp_?okRename@QListViewItem@@MAEXH@Z 10026554     qt-mt323:qt-mt323.dll
 0002:00000558       __imp_?paintBranches@QListViewItem@@UAEXPAVQPainter@@ABVQColorGroup@@HHH@Z 10026558     qt-mt323:qt-mt323.dll
 0002:0000055c       __imp_?paintCell@QListViewItem@@UAEXPAVQPainter@@ABVQColorGroup@@HHH@Z 1002655c     qt-mt323:qt-mt323.dll
 0002:00000560       __imp_?paintEmptyArea@QListView@@MAEXPAVQPainter@@ABVQRect@@@Z 10026560     qt-mt323:qt-mt323.dll
 0002:00000564       __imp_?paintEvent@QFrame@@MAEXPAVQPaintEvent@@@Z 10026564     qt-mt323:qt-mt323.dll
 0002:00000568       __imp_?paintEvent@QPopupMenu@@MAEXPAVQPaintEvent@@@Z 10026568     qt-mt323:qt-mt323.dll
 0002:0000056c       __imp_?paintEvent@QWidget@@MAEXPAVQPaintEvent@@@Z 1002656c     qt-mt323:qt-mt323.dll
 0002:00000570       __imp_?paintFocus@QListViewItem@@UAEXPAVQPainter@@ABVQColorGroup@@ABVQRect@@@Z 10026570     qt-mt323:qt-mt323.dll
 0002:00000574       __imp_?paletteChange@QWidget@@MAEXABVQPalette@@@Z 10026574     qt-mt323:qt-mt323.dll
 0002:00000578       __imp_?pixmap@QListViewItem@@UBEPBVQPixmap@@H@Z 10026578     qt-mt323:qt-mt323.dll
 0002:0000057c       __imp_?polish@QWidget@@UAEXXZ 1002657c     qt-mt323:qt-mt323.dll
 0002:00000580       __imp_?property@QObject@@UBE?AVQVariant@@PBD@Z 10026580     qt-mt323:qt-mt323.dll
 0002:00000584       __imp_?putch@QFile@@UAEHH@Z 10026584     qt-mt323:qt-mt323.dll
 0002:00000588       __imp_?qt_cast@QAction@@UAEPAXPBD@Z 10026588     qt-mt323:qt-mt323.dll
 0002:0000058c       __imp_?qt_cast@QBoxLayout@@UAEPAXPBD@Z 1002658c     qt-mt323:qt-mt323.dll
 0002:00000590       __imp_?qt_cast@QDockWindow@@UAEPAXPBD@Z 10026590     qt-mt323:qt-mt323.dll
 0002:00000594       __imp_?qt_cast@QGuardedPtrPrivate@@UAEPAXPBD@Z 10026594     qt-mt323:qt-mt323.dll
 0002:00000598       __imp_?qt_cast@QListView@@UAEPAXPBD@Z 10026598     qt-mt323:qt-mt323.dll
 0002:0000059c       __imp_?qt_cast@QPopupMenu@@UAEPAXPBD@Z 1002659c     qt-mt323:qt-mt323.dll
 0002:000005a0       __imp_?qt_cast@QTabWidget@@UAEPAXPBD@Z 100265a0     qt-mt323:qt-mt323.dll
 0002:000005a4       __imp_?qt_cast@QToolBar@@UAEPAXPBD@Z 100265a4     qt-mt323:qt-mt323.dll
 0002:000005a8       __imp_?qt_cast@QWidget@@UAEPAXPBD@Z 100265a8     qt-mt323:qt-mt323.dll
 0002:000005ac       __imp_?qt_emit@QAction@@UAE_NHPAUQUObject@@@Z 100265ac     qt-mt323:qt-mt323.dll
 0002:000005b0       __imp_?qt_emit@QBoxLayout@@UAE_NHPAUQUObject@@@Z 100265b0     qt-mt323:qt-mt323.dll
 0002:000005b4       __imp_?qt_emit@QDockWindow@@UAE_NHPAUQUObject@@@Z 100265b4     qt-mt323:qt-mt323.dll
 0002:000005b8       __imp_?qt_emit@QGuardedPtrPrivate@@UAE_NHPAUQUObject@@@Z 100265b8     qt-mt323:qt-mt323.dll
 0002:000005bc       __imp_?qt_emit@QListView@@UAE_NHPAUQUObject@@@Z 100265bc     qt-mt323:qt-mt323.dll
 0002:000005c0       __imp_?qt_emit@QPopupMenu@@UAE_NHPAUQUObject@@@Z 100265c0     qt-mt323:qt-mt323.dll
 0002:000005c4       __imp_?qt_emit@QTabWidget@@UAE_NHPAUQUObject@@@Z 100265c4     qt-mt323:qt-mt323.dll
 0002:000005c8       __imp_?qt_emit@QToolBar@@UAE_NHPAUQUObject@@@Z 100265c8     qt-mt323:qt-mt323.dll
 0002:000005cc       __imp_?qt_emit@QWidget@@UAE_NHPAUQUObject@@@Z 100265cc     qt-mt323:qt-mt323.dll
 0002:000005d0       __imp_?qt_invoke@QAction@@UAE_NHPAUQUObject@@@Z 100265d0     qt-mt323:qt-mt323.dll
 0002:000005d4       __imp_?qt_invoke@QBoxLayout@@UAE_NHPAUQUObject@@@Z 100265d4     qt-mt323:qt-mt323.dll
 0002:000005d8       __imp_?qt_invoke@QDockWindow@@UAE_NHPAUQUObject@@@Z 100265d8     qt-mt323:qt-mt323.dll
 0002:000005dc       __imp_?qt_invoke@QGuardedPtrPrivate@@UAE_NHPAUQUObject@@@Z 100265dc     qt-mt323:qt-mt323.dll
 0002:000005e0       __imp_?qt_invoke@QListView@@UAE_NHPAUQUObject@@@Z 100265e0     qt-mt323:qt-mt323.dll
 0002:000005e4       __imp_?qt_invoke@QPopupMenu@@UAE_NHPAUQUObject@@@Z 100265e4     qt-mt323:qt-mt323.dll
 0002:000005e8       __imp_?qt_invoke@QTabWidget@@UAE_NHPAUQUObject@@@Z 100265e8     qt-mt323:qt-mt323.dll
 0002:000005ec       __imp_?qt_invoke@QToolBar@@UAE_NHPAUQUObject@@@Z 100265ec     qt-mt323:qt-mt323.dll
 0002:000005f0       __imp_?qt_invoke@QWidget@@UAE_NHPAUQUObject@@@Z 100265f0     qt-mt323:qt-mt323.dll
 0002:000005f4       __imp_?qt_property@QAction@@UAE_NHHPAVQVariant@@@Z 100265f4     qt-mt323:qt-mt323.dll
 0002:000005f8       __imp_?qt_property@QBoxLayout@@UAE_NHHPAVQVariant@@@Z 100265f8     qt-mt323:qt-mt323.dll
 0002:000005fc       __imp_?qt_property@QDockWindow@@UAE_NHHPAVQVariant@@@Z 100265fc     qt-mt323:qt-mt323.dll
 0002:00000600       __imp_?qt_property@QGuardedPtrPrivate@@UAE_NHHPAVQVariant@@@Z 10026600     qt-mt323:qt-mt323.dll
 0002:00000604       __imp_?qt_property@QListView@@UAE_NHHPAVQVariant@@@Z 10026604     qt-mt323:qt-mt323.dll
 0002:00000608       __imp_?qt_property@QPopupMenu@@UAE_NHHPAVQVariant@@@Z 10026608     qt-mt323:qt-mt323.dll
 0002:0000060c       __imp_?qt_property@QTabWidget@@UAE_NHHPAVQVariant@@@Z 1002660c     qt-mt323:qt-mt323.dll
 0002:00000610       __imp_?qt_property@QToolBar@@UAE_NHHPAVQVariant@@@Z 10026610     qt-mt323:qt-mt323.dll
 0002:00000614       __imp_?qt_property@QWidget@@UAE_NHHPAVQVariant@@@Z 10026614     qt-mt323:qt-mt323.dll
 0002:00000618       __imp_?read@QGDict@@MAEAAVQDataStream@@AAV2@AAPAX@Z 10026618     qt-mt323:qt-mt323.dll
 0002:0000061c       __imp_?read@QGList@@MAEAAVQDataStream@@AAV2@AAPAX@Z 1002661c     qt-mt323:qt-mt323.dll
 0002:00000620       __imp_?readAll@QIODevice@@UAE?AV?$QMemArray@D@@XZ 10026620     qt-mt323:qt-mt323.dll
 0002:00000624       __imp_?readBlock@QFile@@UAEJPADK@Z 10026624     qt-mt323:qt-mt323.dll
 0002:00000628       __imp_?readLine@QFile@@UAEJPADK@Z 10026628     qt-mt323:qt-mt323.dll
 0002:0000062c       __imp_?removeChild@QObject@@UAEXPAV1@@Z 1002662c     qt-mt323:qt-mt323.dll
 0002:00000630       __imp_?removeChild@QScrollView@@UAEXPAVQObject@@@Z 10026630     qt-mt323:qt-mt323.dll
 0002:00000634       __imp_?removeColumn@QListView@@UAEXH@Z 10026634     qt-mt323:qt-mt323.dll
 0002:00000638       __imp_?removeFrom@QAction@@UAE_NPAVQWidget@@@Z 10026638     qt-mt323:qt-mt323.dll
 0002:0000063c       __imp_?removeItem@QListView@@UAEXPAVQListViewItem@@@Z 1002663c     qt-mt323:qt-mt323.dll
 0002:00000640       __imp_?removeItem@QListViewItem@@UAEXPAV1@@Z 10026640     qt-mt323:qt-mt323.dll
 0002:00000644       __imp_?removePage@QTabWidget@@UAEXPAVQWidget@@@Z 10026644     qt-mt323:qt-mt323.dll
 0002:00000648       __imp_?reparent@QWidget@@UAEXPAV1@IABVQPoint@@_N@Z 10026648     qt-mt323:qt-mt323.dll
 0002:0000064c       __imp_?resize@QScrollView@@UAEXHH@Z 1002664c     qt-mt323:qt-mt323.dll
 0002:00000650       __imp_?resize@QWidget@@UAEXHH@Z 10026650     qt-mt323:qt-mt323.dll
 0002:00000654       __imp_?resizeContents@QScrollView@@UAEXHH@Z 10026654     qt-mt323:qt-mt323.dll
 0002:00000658       __imp_?resizeEvent@QDockWindow@@MAEXPAVQResizeEvent@@@Z 10026658     qt-mt323:qt-mt323.dll
 0002:0000065c       __imp_?resizeEvent@QFrame@@MAEXPAVQResizeEvent@@@Z 1002665c     qt-mt323:qt-mt323.dll
 0002:00000660       __imp_?resizeEvent@QListView@@MAEXPAVQResizeEvent@@@Z 10026660     qt-mt323:qt-mt323.dll
 0002:00000664       __imp_?resizeEvent@QTabWidget@@MAEXPAVQResizeEvent@@@Z 10026664     qt-mt323:qt-mt323.dll
 0002:00000668       __imp_?resizeEvent@QToolBar@@MAEXPAVQResizeEvent@@@Z 10026668     qt-mt323:qt-mt323.dll
 0002:0000066c       __imp_?resizeEvent@QWidget@@MAEXPAVQResizeEvent@@@Z 1002666c     qt-mt323:qt-mt323.dll
 0002:00000670       __imp_?resolution@QPaintDevice@@UBEHXZ 10026670     qt-mt323:qt-mt323.dll
 0002:00000674       __imp_?rtti@QListViewItem@@UBEHXZ 10026674     qt-mt323:qt-mt323.dll
 0002:00000678       __imp_?selectAll@QListView@@UAEX_N@Z 10026678     qt-mt323:qt-mt323.dll
 0002:0000067c       __imp_?setAccel@QAction@@UAEXABVQKeySequence@@@Z 1002667c     qt-mt323:qt-mt323.dll
 0002:00000680       __imp_?setAcceptDrops@QWidget@@UAEX_N@Z 10026680     qt-mt323:qt-mt323.dll
 0002:00000684       __imp_?setActiveItem@QPopupMenu@@UAEXH@Z 10026684     qt-mt323:qt-mt323.dll
 0002:00000688       __imp_?setActiveWindow@QWidget@@UAEXXZ 10026688     qt-mt323:qt-mt323.dll
 0002:0000068c       __imp_?setAlignment@QLayoutItem@@UAEXH@Z 1002668c     qt-mt323:qt-mt323.dll
 0002:00000690       __imp_?setAllColumnsShowFocus@QListView@@UAEX_N@Z 10026690     qt-mt323:qt-mt323.dll
 0002:00000694       __imp_?setAutoAdd@QLayout@@UAEX_N@Z 10026694     qt-mt323:qt-mt323.dll
 0002:00000698       __imp_?setAutoMask@QWidget@@UAEX_N@Z 10026698     qt-mt323:qt-mt323.dll
 0002:0000069c       __imp_?setBackgroundColor@QWidget@@UAEXABVQColor@@@Z 1002669c     qt-mt323:qt-mt323.dll
 0002:000006a0       __imp_?setBackgroundMode@QWidget@@UAEXW4BackgroundMode@Qt@@@Z 100266a0     qt-mt323:qt-mt323.dll
 0002:000006a4       __imp_?setBackgroundOrigin@QWidget@@UAEXW4BackgroundOrigin@1@@Z 100266a4     qt-mt323:qt-mt323.dll
 0002:000006a8       __imp_?setBackgroundPixmap@QWidget@@UAEXABVQPixmap@@@Z 100266a8     qt-mt323:qt-mt323.dll
 0002:000006ac       __imp_?setCaption@QDockWindow@@UAEXABVQString@@@Z 100266ac     qt-mt323:qt-mt323.dll
 0002:000006b0       __imp_?setCaption@QWidget@@UAEXABVQString@@@Z 100266b0     qt-mt323:qt-mt323.dll
 0002:000006b4       __imp_?setCheckable@QPopupMenu@@UAEX_N@Z 100266b4     qt-mt323:qt-mt323.dll
 0002:000006b8       __imp_?setCloseMode@QDockWindow@@UAEXH@Z 100266b8     qt-mt323:qt-mt323.dll
 0002:000006bc       __imp_?setColumnAlignment@QListView@@UAEXHH@Z 100266bc     qt-mt323:qt-mt323.dll
 0002:000006c0       __imp_?setColumnText@QListView@@UAEXHABVQIconSet@@ABVQString@@@Z 100266c0     qt-mt323:qt-mt323.dll
 0002:000006c4       __imp_?setColumnText@QListView@@UAEXHABVQString@@@Z 100266c4     qt-mt323:qt-mt323.dll
 0002:000006c8       __imp_?setColumnWidth@QListView@@UAEXHH@Z 100266c8     qt-mt323:qt-mt323.dll
 0002:000006cc       __imp_?setColumnWidthMode@QListView@@UAEXHW4WidthMode@1@@Z 100266cc     qt-mt323:qt-mt323.dll
 0002:000006d0       __imp_?setContentsPos@QListView@@UAEXHH@Z 100266d0     qt-mt323:qt-mt323.dll
 0002:000006d4       __imp_?setCornerWidget@QScrollView@@UAEXPAVQWidget@@@Z 100266d4     qt-mt323:qt-mt323.dll
 0002:000006d8       __imp_?setCurrentItem@QListView@@UAEXPAVQListViewItem@@@Z 100266d8     qt-mt323:qt-mt323.dll
 0002:000006dc       __imp_?setCursor@QWidget@@UAEXABVQCursor@@@Z 100266dc     qt-mt323:qt-mt323.dll
 0002:000006e0       __imp_?setDefaultRenameAction@QListView@@UAEXW4RenameAction@1@@Z 100266e0     qt-mt323:qt-mt323.dll
 0002:000006e4       __imp_?setDragAutoScroll@QScrollView@@UAEX_N@Z 100266e4     qt-mt323:qt-mt323.dll
 0002:000006e8       __imp_?setDragEnabled@QListViewItem@@UAEX_N@Z 100266e8     qt-mt323:qt-mt323.dll
 0002:000006ec       __imp_?setDropEnabled@QListViewItem@@UAEX_N@Z 100266ec     qt-mt323:qt-mt323.dll
 0002:000006f0       __imp_?setEnabled@QAction@@UAEX_N@Z 100266f0     qt-mt323:qt-mt323.dll
 0002:000006f4       __imp_?setEnabled@QListViewItem@@UAEX_N@Z 100266f4     qt-mt323:qt-mt323.dll
 0002:000006f8       __imp_?setEnabled@QScrollView@@UAEX_N@Z 100266f8     qt-mt323:qt-mt323.dll
 0002:000006fc       __imp_?setEnabled@QWidget@@UAEX_N@Z 100266fc     qt-mt323:qt-mt323.dll
 0002:00000700       __imp_?setEraseColor@QWidget@@UAEXABVQColor@@@Z 10026700     qt-mt323:qt-mt323.dll
 0002:00000704       __imp_?setErasePixmap@QWidget@@UAEXABVQPixmap@@@Z 10026704     qt-mt323:qt-mt323.dll
 0002:00000708       __imp_?setExpandable@QListViewItem@@UAEX_N@Z 10026708     qt-mt323:qt-mt323.dll
 0002:0000070c       __imp_?setFirstItemActive@QPopupMenu@@EAEXXZ 1002670c     qt-mt323:qt-mt323.dll
 0002:00000710       __imp_?setFixedExtentHeight@QDockWindow@@UAEXH@Z 10026710     qt-mt323:qt-mt323.dll
 0002:00000714       __imp_?setFixedExtentWidth@QDockWindow@@UAEXH@Z 10026714     qt-mt323:qt-mt323.dll
 0002:00000718       __imp_?setFocus@QWidget@@UAEXXZ 10026718     qt-mt323:qt-mt323.dll
 0002:0000071c       __imp_?setFocusPolicy@QWidget@@UAEXW4FocusPolicy@1@@Z 1002671c     qt-mt323:qt-mt323.dll
 0002:00000720       __imp_?setFocusProxy@QWidget@@UAEXPAV1@@Z 10026720     qt-mt323:qt-mt323.dll
 0002:00000724       __imp_?setFont@QListView@@UAEXABVQFont@@@Z 10026724     qt-mt323:qt-mt323.dll
 0002:00000728       __imp_?setFont@QPopupMenu@@UAEXABVQFont@@@Z 10026728     qt-mt323:qt-mt323.dll
 0002:0000072c       __imp_?setFont@QWidget@@UAEXABVQFont@@@Z 1002672c     qt-mt323:qt-mt323.dll
 0002:00000730       __imp_?setFrameRect@QFrame@@UAEXABVQRect@@@Z 10026730     qt-mt323:qt-mt323.dll
 0002:00000734       __imp_?setFrameStyle@QFrame@@UAEXH@Z 10026734     qt-mt323:qt-mt323.dll
 0002:00000738       __imp_?setGeometry@QBoxLayout@@UAEXABVQRect@@@Z 10026738     qt-mt323:qt-mt323.dll
 0002:0000073c       __imp_?setGeometry@QWidget@@UAEXABVQRect@@@Z 1002673c     qt-mt323:qt-mt323.dll
 0002:00000740       __imp_?setGeometry@QWidget@@UAEXHHHH@Z 10026740     qt-mt323:qt-mt323.dll
 0002:00000744       __imp_?setHBarGeometry@QScrollView@@MAEXAAVQScrollBar@@HHHH@Z 10026744     qt-mt323:qt-mt323.dll
 0002:00000748       __imp_?setHScrollBarMode@QScrollView@@UAEXW4ScrollBarMode@1@@Z 10026748     qt-mt323:qt-mt323.dll
 0002:0000074c       __imp_?setHeight@QListViewItem@@MAEXH@Z 1002674c     qt-mt323:qt-mt323.dll
 0002:00000750       __imp_?setHorizontallyStretchable@QDockWindow@@UAEX_N@Z 10026750     qt-mt323:qt-mt323.dll
 0002:00000754       __imp_?setIcon@QWidget@@UAEXABVQPixmap@@@Z 10026754     qt-mt323:qt-mt323.dll
 0002:00000758       __imp_?setIconSet@QAction@@UAEXABVQIconSet@@@Z 10026758     qt-mt323:qt-mt323.dll
 0002:0000075c       __imp_?setIconText@QWidget@@UAEXABVQString@@@Z 1002675c     qt-mt323:qt-mt323.dll
 0002:00000760       __imp_?setId@QMenuData@@UAEXHH@Z 10026760     qt-mt323:qt-mt323.dll
 0002:00000764       __imp_?setItemMargin@QListView@@UAEXH@Z 10026764     qt-mt323:qt-mt323.dll
 0002:00000768       __imp_?setKeyCompression@QWidget@@MAEX_N@Z 10026768     qt-mt323:qt-mt323.dll
 0002:0000076c       __imp_?setLabel@QToolBar@@UAEXABVQString@@@Z 1002676c     qt-mt323:qt-mt323.dll
 0002:00000770       __imp_?setLineWidth@QFrame@@UAEXH@Z 10026770     qt-mt323:qt-mt323.dll
 0002:00000774       __imp_?setMargin@QFrame@@UAEXH@Z 10026774     qt-mt323:qt-mt323.dll
 0002:00000778       __imp_?setMargin@QLayout@@UAEXH@Z 10026778     qt-mt323:qt-mt323.dll
 0002:0000077c       __imp_?setMargins@QScrollView@@MAEXHHHH@Z 1002677c     qt-mt323:qt-mt323.dll
 0002:00000780       __imp_?setMask@QWidget@@UAEXABVQBitmap@@@Z 10026780     qt-mt323:qt-mt323.dll
 0002:00000784       __imp_?setMask@QWidget@@UAEXABVQRegion@@@Z 10026784     qt-mt323:qt-mt323.dll
 0002:00000788       __imp_?setMaximumSize@QWidget@@UAEXHH@Z 10026788     qt-mt323:qt-mt323.dll
 0002:0000078c       __imp_?setMenuBar@QLayout@@UAEXPAVQMenuBar@@@Z 1002678c     qt-mt323:qt-mt323.dll
 0002:00000790       __imp_?setMenuText@QAction@@UAEXABVQString@@@Z 10026790     qt-mt323:qt-mt323.dll
 0002:00000794       __imp_?setMicroFocusHint@QWidget@@MAEXHHHH_NPAVQFont@@@Z 10026794     qt-mt323:qt-mt323.dll
 0002:00000798       __imp_?setMidLineWidth@QFrame@@UAEXH@Z 10026798     qt-mt323:qt-mt323.dll
 0002:0000079c       __imp_?setMinimumSize@QToolBar@@UAEXHH@Z 1002679c     qt-mt323:qt-mt323.dll
 0002:000007a0       __imp_?setMinimumSize@QWidget@@UAEXHH@Z 100267a0     qt-mt323:qt-mt323.dll
 0002:000007a4       __imp_?setMouseTracking@QWidget@@UAEX_N@Z 100267a4     qt-mt323:qt-mt323.dll
 0002:000007a8       __imp_?setMovingEnabled@QDockWindow@@UAEX_N@Z 100267a8     qt-mt323:qt-mt323.dll
 0002:000007ac       __imp_?setMultiLinesEnabled@QListViewItem@@UAEX_N@Z 100267ac     qt-mt323:qt-mt323.dll
 0002:000007b0       __imp_?setMultiSelection@QListView@@UAEX_N@Z 100267b0     qt-mt323:qt-mt323.dll
 0002:000007b4       __imp_?setName@QObject@@UAEXPBD@Z 100267b4     qt-mt323:qt-mt323.dll
 0002:000007b8       __imp_?setNewLine@QDockWindow@@UAEX_N@Z 100267b8     qt-mt323:qt-mt323.dll
 0002:000007bc       __imp_?setOffset@QDockWindow@@UAEXH@Z 100267bc     qt-mt323:qt-mt323.dll
 0002:000007c0       __imp_?setOn@QAction@@UAEX_N@Z 100267c0     qt-mt323:qt-mt323.dll
 0002:000007c4       __imp_?setOpaqueMoving@QDockWindow@@UAEX_N@Z 100267c4     qt-mt323:qt-mt323.dll
 0002:000007c8       __imp_?setOpen@QListView@@UAEXPAVQListViewItem@@_N@Z 100267c8     qt-mt323:qt-mt323.dll
 0002:000007cc       __imp_?setOpen@QListViewItem@@UAEX_N@Z 100267cc     qt-mt323:qt-mt323.dll
 0002:000007d0       __imp_?setOrientation@QDockWindow@@UAEXW4Orientation@Qt@@@Z 100267d0     qt-mt323:qt-mt323.dll
 0002:000007d4       __imp_?setOrientation@QToolBar@@UAEXW4Orientation@Qt@@@Z 100267d4     qt-mt323:qt-mt323.dll
 0002:000007d8       __imp_?setPalette@QListView@@UAEXABVQPalette@@@Z 100267d8     qt-mt323:qt-mt323.dll
 0002:000007dc       __imp_?setPalette@QWidget@@UAEXABVQPalette@@@Z 100267dc     qt-mt323:qt-mt323.dll
 0002:000007e0       __imp_?setPaletteBackgroundColor@QWidget@@UAEXABVQColor@@@Z 100267e0     qt-mt323:qt-mt323.dll
 0002:000007e4       __imp_?setPaletteBackgroundPixmap@QWidget@@UAEXABVQPixmap@@@Z 100267e4     qt-mt323:qt-mt323.dll
 0002:000007e8       __imp_?setPixmap@QListViewItem@@UAEXHABVQPixmap@@@Z 100267e8     qt-mt323:qt-mt323.dll
 0002:000007ec       __imp_?setProperty@QObject@@UAE_NPBDABVQVariant@@@Z 100267ec     qt-mt323:qt-mt323.dll
 0002:000007f0       __imp_?setRenameEnabled@QListViewItem@@UAEXH_N@Z 100267f0     qt-mt323:qt-mt323.dll
 0002:000007f4       __imp_?setResizeEnabled@QDockWindow@@UAEX_N@Z 100267f4     qt-mt323:qt-mt323.dll
 0002:000007f8       __imp_?setResizeMode@QListView@@UAEXW4ResizeMode@1@@Z 100267f8     qt-mt323:qt-mt323.dll
 0002:000007fc       __imp_?setResizePolicy@QScrollView@@UAEXW4ResizePolicy@1@@Z 100267fc     qt-mt323:qt-mt323.dll
 0002:00000800       __imp_?setResolution@QPaintDevice@@UAEXH@Z 10026800     qt-mt323:qt-mt323.dll
 0002:00000804       __imp_?setRootIsDecorated@QListView@@UAEX_N@Z 10026804     qt-mt323:qt-mt323.dll
 0002:00000808       __imp_?setSelectable@QListViewItem@@UAEX_N@Z 10026808     qt-mt323:qt-mt323.dll
 0002:0000080c       __imp_?setSelected@QListView@@UAEXPAVQListViewItem@@_N@Z 1002680c     qt-mt323:qt-mt323.dll
 0002:00000810       __imp_?setSelected@QListViewItem@@UAEX_N@Z 10026810     qt-mt323:qt-mt323.dll
 0002:00000814       __imp_?setShowSortIndicator@QListView@@UAEX_N@Z 10026814     qt-mt323:qt-mt323.dll
 0002:00000818       __imp_?setShowToolTips@QListView@@UAEX_N@Z 10026818     qt-mt323:qt-mt323.dll
 0002:0000081c       __imp_?setSizeIncrement@QWidget@@UAEXHH@Z 1002681c     qt-mt323:qt-mt323.dll
 0002:00000820       __imp_?setSizePolicy@QWidget@@UAEXVQSizePolicy@@@Z 10026820     qt-mt323:qt-mt323.dll
 0002:00000824       __imp_?setSorting@QListView@@UAEXH_N@Z 10026824     qt-mt323:qt-mt323.dll
 0002:00000828       __imp_?setSpacing@QLayout@@UAEXH@Z 10026828     qt-mt323:qt-mt323.dll
 0002:0000082c       __imp_?setStatusTip@QAction@@UAEXABVQString@@@Z 1002682c     qt-mt323:qt-mt323.dll
 0002:00000830       __imp_?setStretchableWidget@QToolBar@@UAEXPAVQWidget@@@Z 10026830     qt-mt323:qt-mt323.dll
 0002:00000834       __imp_?setText@QAction@@UAEXABVQString@@@Z 10026834     qt-mt323:qt-mt323.dll
 0002:00000838       __imp_?setText@QListViewItem@@UAEXHABVQString@@@Z 10026838     qt-mt323:qt-mt323.dll
 0002:0000083c       __imp_?setToggleAction@QAction@@UAEX_N@Z 1002683c     qt-mt323:qt-mt323.dll
 0002:00000840       __imp_?setToolTip@QAction@@UAEXABVQString@@@Z 10026840     qt-mt323:qt-mt323.dll
 0002:00000844       __imp_?setTreeStepSize@QListView@@UAEXH@Z 10026844     qt-mt323:qt-mt323.dll
 0002:00000848       __imp_?setUpdatesEnabled@QWidget@@UAEX_N@Z 10026848     qt-mt323:qt-mt323.dll
 0002:0000084c       __imp_?setVBarGeometry@QScrollView@@MAEXAAVQScrollBar@@HHHH@Z 1002684c     qt-mt323:qt-mt323.dll
 0002:00000850       __imp_?setVScrollBarMode@QScrollView@@UAEXW4ScrollBarMode@1@@Z 10026850     qt-mt323:qt-mt323.dll
 0002:00000854       __imp_?setVerticallyStretchable@QDockWindow@@UAEX_N@Z 10026854     qt-mt323:qt-mt323.dll
 0002:00000858       __imp_?setWFlags@QWidget@@MAEXI@Z 10026858     qt-mt323:qt-mt323.dll
 0002:0000085c       __imp_?setWState@QWidget@@MAEXI@Z 1002685c     qt-mt323:qt-mt323.dll
 0002:00000860       __imp_?setWhatsThis@QAction@@UAEXABVQString@@@Z 10026860     qt-mt323:qt-mt323.dll
 0002:00000864       __imp_?setWidget@QDockWindow@@UAEXPAVQWidget@@@Z 10026864     qt-mt323:qt-mt323.dll
 0002:00000868       __imp_?setup@QListViewItem@@UAEXXZ 10026868     qt-mt323:qt-mt323.dll
 0002:0000086c       __imp_?show@QListView@@UAEXXZ 1002686c     qt-mt323:qt-mt323.dll
 0002:00000870       __imp_?show@QPopupMenu@@UAEXXZ 10026870     qt-mt323:qt-mt323.dll
 0002:00000874       __imp_?show@QToolBar@@UAEXXZ 10026874     qt-mt323:qt-mt323.dll
 0002:00000878       __imp_?show@QWidget@@UAEXXZ 10026878     qt-mt323:qt-mt323.dll
 0002:0000087c       __imp_?showEvent@QDockWindow@@MAEXPAVQShowEvent@@@Z 1002687c     qt-mt323:qt-mt323.dll
 0002:00000880       __imp_?showEvent@QListView@@MAEXPAVQShowEvent@@@Z 10026880     qt-mt323:qt-mt323.dll
 0002:00000884       __imp_?showEvent@QTabWidget@@MAEXPAVQShowEvent@@@Z 10026884     qt-mt323:qt-mt323.dll
 0002:00000888       __imp_?showEvent@QWidget@@MAEXPAVQShowEvent@@@Z 10026888     qt-mt323:qt-mt323.dll
 0002:0000088c       __imp_?showMaximized@QWidget@@UAEXXZ 1002688c     qt-mt323:qt-mt323.dll
 0002:00000890       __imp_?showMinimized@QWidget@@UAEXXZ 10026890     qt-mt323:qt-mt323.dll
 0002:00000894       __imp_?showNormal@QWidget@@UAEXXZ 10026894     qt-mt323:qt-mt323.dll
 0002:00000898       __imp_?showPage@QTabWidget@@UAEXPAVQWidget@@@Z 10026898     qt-mt323:qt-mt323.dll
 0002:0000089c       __imp_?size@QFile@@UBEKXZ  1002689c     qt-mt323:qt-mt323.dll
 0002:000008a0       __imp_?sizeHint@QBoxLayout@@UBE?AVQSize@@XZ 100268a0     qt-mt323:qt-mt323.dll
 0002:000008a4       __imp_?sizeHint@QDockWindow@@UBE?AVQSize@@XZ 100268a4     qt-mt323:qt-mt323.dll
 0002:000008a8       __imp_?sizeHint@QHBox@@UBE?AVQSize@@XZ 100268a8     qt-mt323:qt-mt323.dll
 0002:000008ac       __imp_?sizeHint@QListView@@UBE?AVQSize@@XZ 100268ac     qt-mt323:qt-mt323.dll
 0002:000008b0       __imp_?sizeHint@QPopupMenu@@UBE?AVQSize@@XZ 100268b0     qt-mt323:qt-mt323.dll
 0002:000008b4       __imp_?sizeHint@QTabWidget@@UBE?AVQSize@@XZ 100268b4     qt-mt323:qt-mt323.dll
 0002:000008b8       __imp_?sizeHint@QWidget@@UBE?AVQSize@@XZ 100268b8     qt-mt323:qt-mt323.dll
 0002:000008bc       __imp_?sizePolicy@QWidget@@UBE?AVQSizePolicy@@XZ 100268bc     qt-mt323:qt-mt323.dll
 0002:000008c0       __imp_?sort@QListView@@UAEXXZ 100268c0     qt-mt323:qt-mt323.dll
 0002:000008c4       __imp_?sort@QListViewItem@@UAEXXZ 100268c4     qt-mt323:qt-mt323.dll
 0002:000008c8       __imp_?sortChildItems@QListViewItem@@UAEXH_N@Z 100268c8     qt-mt323:qt-mt323.dll
 0002:000008cc       __imp_?spacerItem@QLayoutItem@@UAEPAVQSpacerItem@@XZ 100268cc     qt-mt323:qt-mt323.dll
 0002:000008d0       __imp_?startDrag@QListView@@MAEXXZ 100268d0     qt-mt323:qt-mt323.dll
 0002:000008d4       __imp_?startRename@QListViewItem@@UAEXH@Z 100268d4     qt-mt323:qt-mt323.dll
 0002:000008d8       __imp_?styleChange@QFrame@@MAEXAAVQStyle@@@Z 100268d8     qt-mt323:qt-mt323.dll
 0002:000008dc       __imp_?styleChange@QListView@@MAEXAAVQStyle@@@Z 100268dc     qt-mt323:qt-mt323.dll
 0002:000008e0       __imp_?styleChange@QPopupMenu@@MAEXAAVQStyle@@@Z 100268e0     qt-mt323:qt-mt323.dll
 0002:000008e4       __imp_?styleChange@QTabWidget@@MAEXAAVQStyle@@@Z 100268e4     qt-mt323:qt-mt323.dll
 0002:000008e8       __imp_?styleChange@QToolBar@@MAEXAAVQStyle@@@Z 100268e8     qt-mt323:qt-mt323.dll
 0002:000008ec       __imp_?styleChange@QWidget@@MAEXAAVQStyle@@@Z 100268ec     qt-mt323:qt-mt323.dll
 0002:000008f0       __imp_?tabletEvent@QWidget@@MAEXPAVQTabletEvent@@@Z 100268f0     qt-mt323:qt-mt323.dll
 0002:000008f4       __imp_?takeItem@QListView@@UAEXPAVQListViewItem@@@Z 100268f4     qt-mt323:qt-mt323.dll
 0002:000008f8       __imp_?takeItem@QListViewItem@@UAEXPAV1@@Z 100268f8     qt-mt323:qt-mt323.dll
 0002:000008fc       __imp_?text@QListViewItem@@UBE?AVQString@@H@Z 100268fc     qt-mt323:qt-mt323.dll
 0002:00000900       __imp_?timerEvent@QObject@@MAEXPAVQTimerEvent@@@Z 10026900     qt-mt323:qt-mt323.dll
 0002:00000904       __imp_?timerEvent@QPopupMenu@@MAEXPAVQTimerEvent@@@Z 10026904     qt-mt323:qt-mt323.dll
 0002:00000908       __imp_?undock@QDockWindow@@UAEXPAVQWidget@@@Z 10026908     qt-mt323:qt-mt323.dll
 0002:0000090c       __imp_?undock@QDockWindow@@UAEXXZ 1002690c     qt-mt323:qt-mt323.dll
 0002:00000910       __imp_?ungetch@QFile@@UAEHH@Z 10026910     qt-mt323:qt-mt323.dll
 0002:00000914       __imp_?unsetCursor@QWidget@@UAEXXZ 10026914     qt-mt323:qt-mt323.dll
 0002:00000918       __imp_?updateItem@QPopupMenu@@UAEXH@Z 10026918     qt-mt323:qt-mt323.dll
 0002:0000091c       __imp_?updateMask@QTabWidget@@MAEXXZ 1002691c     qt-mt323:qt-mt323.dll
 0002:00000920       __imp_?updateMask@QWidget@@MAEXXZ 10026920     qt-mt323:qt-mt323.dll
 0002:00000924       __imp_?viewportContextMenuEvent@QScrollView@@MAEXPAVQContextMenuEvent@@@Z 10026924     qt-mt323:qt-mt323.dll
 0002:00000928       __imp_?viewportDragEnterEvent@QScrollView@@MAEXPAVQDragEnterEvent@@@Z 10026928     qt-mt323:qt-mt323.dll
 0002:0000092c       __imp_?viewportDragLeaveEvent@QScrollView@@MAEXPAVQDragLeaveEvent@@@Z 1002692c     qt-mt323:qt-mt323.dll
 0002:00000930       __imp_?viewportDragMoveEvent@QScrollView@@MAEXPAVQDragMoveEvent@@@Z 10026930     qt-mt323:qt-mt323.dll
 0002:00000934       __imp_?viewportDropEvent@QScrollView@@MAEXPAVQDropEvent@@@Z 10026934     qt-mt323:qt-mt323.dll
 0002:00000938       __imp_?viewportMouseDoubleClickEvent@QScrollView@@MAEXPAVQMouseEvent@@@Z 10026938     qt-mt323:qt-mt323.dll
 0002:0000093c       __imp_?viewportMouseMoveEvent@QScrollView@@MAEXPAVQMouseEvent@@@Z 1002693c     qt-mt323:qt-mt323.dll
 0002:00000940       __imp_?viewportMousePressEvent@QScrollView@@MAEXPAVQMouseEvent@@@Z 10026940     qt-mt323:qt-mt323.dll
 0002:00000944       __imp_?viewportMouseReleaseEvent@QScrollView@@MAEXPAVQMouseEvent@@@Z 10026944     qt-mt323:qt-mt323.dll
 0002:00000948       __imp_?viewportPaintEvent@QScrollView@@MAEXPAVQPaintEvent@@@Z 10026948     qt-mt323:qt-mt323.dll
 0002:0000094c       __imp_?viewportResizeEvent@QListView@@MAEXPAVQResizeEvent@@@Z 1002694c     qt-mt323:qt-mt323.dll
 0002:00000950       __imp_?viewportWheelEvent@QScrollView@@MAEXPAVQWheelEvent@@@Z 10026950     qt-mt323:qt-mt323.dll
 0002:00000954       __imp_?wheelEvent@QScrollView@@MAEXPAVQWheelEvent@@@Z 10026954     qt-mt323:qt-mt323.dll
 0002:00000958       __imp_?wheelEvent@QWidget@@MAEXPAVQWheelEvent@@@Z 10026958     qt-mt323:qt-mt323.dll
 0002:0000095c       __imp_?widget@QLayoutItem@@UAEPAVQWidget@@XZ 1002695c     qt-mt323:qt-mt323.dll
 0002:00000960       __imp_?width@QListViewItem@@UBEHABVQFontMetrics@@PBVQListView@@H@Z 10026960     qt-mt323:qt-mt323.dll
 0002:00000964       __imp_?winEvent@QWidget@@MAE_NPAUtagMSG@@@Z 10026964     qt-mt323:qt-mt323.dll
 0002:00000968       __imp_?windowActivationChange@QListView@@MAEX_N@Z 10026968     qt-mt323:qt-mt323.dll
 0002:0000096c       __imp_?windowActivationChange@QWidget@@MAEX_N@Z 1002696c     qt-mt323:qt-mt323.dll
 0002:00000970       __imp_?write@QGDict@@MBEAAVQDataStream@@AAV2@PAX@Z 10026970     qt-mt323:qt-mt323.dll
 0002:00000974       __imp_?write@QGList@@MBEAAVQDataStream@@AAV2@PAX@Z 10026974     qt-mt323:qt-mt323.dll
 0002:00000978       __imp_?writeBlock@QFile@@UAEJPBDK@Z 10026978     qt-mt323:qt-mt323.dll
 0002:0000097c       __imp_?null@QString@@2V1@A 1002697c     qt-mt323:qt-mt323.dll
 0002:00000980       __imp_??_7?$QPtrList@VQDockWindow@@@@6B@ 10026980     qt-mt323:qt-mt323.dll
 0002:00000984       __imp_??1QSqlError@@UAE@XZ 10026984     qt-mt323:qt-mt323.dll
 0002:00000988       __imp_?driverText@QSqlError@@QBE?AVQString@@XZ 10026988     qt-mt323:qt-mt323.dll
 0002:0000098c       __imp_?databaseText@QSqlError@@QBE?AVQString@@XZ 1002698c     qt-mt323:qt-mt323.dll
 0002:00000990       __imp_?type@QSqlError@@QBEHXZ 10026990     qt-mt323:qt-mt323.dll
 0002:00000994       __imp_?number@QSqlError@@QBEHXZ 10026994     qt-mt323:qt-mt323.dll
 0002:00000998       __imp_?text@QSqlError@@QBE?AVQString@@XZ 10026998     qt-mt323:qt-mt323.dll
 0002:0000099c       __imp_?open@QSqlDatabase@@QAE_NXZ 1002699c     qt-mt323:qt-mt323.dll
 0002:000009a0       __imp_?close@QSqlDatabase@@QAEXXZ 100269a0     qt-mt323:qt-mt323.dll
 0002:000009a4       __imp_?isOpen@QSqlDatabase@@QBE_NXZ 100269a4     qt-mt323:qt-mt323.dll
 0002:000009a8       __imp_?lastError@QSqlDatabase@@QBE?AVQSqlError@@XZ 100269a8     qt-mt323:qt-mt323.dll
 0002:000009ac       __imp_?port@QSqlDatabase@@QBEHXZ 100269ac     qt-mt323:qt-mt323.dll
 0002:000009b0       __imp_?addDatabase@QSqlDatabase@@SAPAV1@ABVQString@@0@Z 100269b0     qt-mt323:qt-mt323.dll
 0002:000009b4       __imp_?database@QSqlDatabase@@SAPAV1@ABVQString@@_N@Z 100269b4     qt-mt323:qt-mt323.dll
 0002:000009b8       __imp_??0QThread@@QAE@XZ   100269b8     qt-mt323:qt-mt323.dll
 0002:000009bc       __imp_??1QThread@@UAE@XZ   100269bc     qt-mt323:qt-mt323.dll
 0002:000009c0       __imp_??1QVariant@@QAE@XZ  100269c0     qt-mt323:qt-mt323.dll
 0002:000009c4       __imp_??0QVariant@@QAE@ABVQString@@@Z 100269c4     qt-mt323:qt-mt323.dll
 0002:000009c8       __imp_?toString@QVariant@@QBE?BVQString@@XZ 100269c8     qt-mt323:qt-mt323.dll
 0002:000009cc       __imp_??6?$QValueList@VQString@@@@QAEAAV0@ABVQString@@@Z 100269cc     qt-mt323:qt-mt323.dll
 0002:000009d0       __imp_??A?$QValueList@VQString@@@@QBEABVQString@@I@Z 100269d0     qt-mt323:qt-mt323.dll
 0002:000009d4       __imp_?findIndex@?$QValueList@VQString@@@@QBEHABVQString@@@Z 100269d4     qt-mt323:qt-mt323.dll
 0002:000009d8       __imp_?split@QStringList@@SA?AV1@ABVQChar@@ABVQString@@_N@Z 100269d8     qt-mt323:qt-mt323.dll
 0002:000009dc       __imp_?join@QStringList@@QBE?AVQString@@ABV2@@Z 100269dc     qt-mt323:qt-mt323.dll
 0002:000009e0       __imp_?name@QObject@@QBEPBDXZ 100269e0     qt-mt323:qt-mt323.dll
 0002:000009e4       __imp_?hasFocus@QWidget@@QBE_NXZ 100269e4     qt-mt323:qt-mt323.dll
 0002:000009e8       __imp_?setSelectionMode@QListView@@QAEXW4SelectionMode@1@@Z 100269e8     qt-mt323:qt-mt323.dll
 0002:000009ec       __imp_?insertStringList@QComboBox@@QAEXABVQStringList@@H@Z 100269ec     qt-mt323:qt-mt323.dll
 0002:000009f0       __imp_?insertItem@QComboBox@@QAEXABVQString@@H@Z 100269f0     qt-mt323:qt-mt323.dll
 0002:000009f4       __imp_?clear@QComboBox@@QAEXXZ 100269f4     qt-mt323:qt-mt323.dll
 0002:000009f8       __imp_?clearEdit@QComboBox@@QAEXXZ 100269f8     qt-mt323:qt-mt323.dll
 0002:000009fc       __imp_?setMaxValue@QSpinBox@@QAEXH@Z 100269fc     qt-mt323:qt-mt323.dll
 0002:00000a00       __imp_??0QSqlQuery@@QAE@ABVQString@@PAVQSqlDatabase@@@Z 10026a00     qt-mt323:qt-mt323.dll
 0002:00000a04       __imp_??1QSqlQuery@@UAE@XZ 10026a04     qt-mt323:qt-mt323.dll
 0002:00000a08       __imp_?isActive@QSqlQuery@@QBE_NXZ 10026a08     qt-mt323:qt-mt323.dll
 0002:00000a0c       __imp_?lastQuery@QSqlQuery@@QBE?AVQString@@XZ 10026a0c     qt-mt323:qt-mt323.dll
 0002:00000a10       __imp_?numRowsAffected@QSqlQuery@@QBEHXZ 10026a10     qt-mt323:qt-mt323.dll
 0002:00000a14       __imp_?exec@QSqlQuery@@UAE_NABVQString@@@Z 10026a14     qt-mt323:qt-mt323.dll
 0002:00000a18       __imp_?value@QSqlQuery@@UBE?AVQVariant@@H@Z 10026a18     qt-mt323:qt-mt323.dll
 0002:00000a1c       __imp_?first@QSqlQuery@@UAE_NXZ 10026a1c     qt-mt323:qt-mt323.dll
 0002:00000a20       __imp_?tables@QSqlDatabase@@QBE?AVQStringList@@XZ 10026a20     qt-mt323:qt-mt323.dll
 0002:00000a24       __imp_?drivers@QSqlDatabase@@SA?AVQStringList@@XZ 10026a24     qt-mt323:qt-mt323.dll
 0002:00000a28       __imp_??0QSqlCursor@@QAE@ABVQString@@_NPAVQSqlDatabase@@@Z 10026a28     qt-mt323:qt-mt323.dll
 0002:00000a2c       __imp_??1QSqlCursor@@UAE@XZ 10026a2c     qt-mt323:qt-mt323.dll
 0002:00000a30       __imp_?value@QSqlCursor@@UBE?AVQVariant@@H@Z 10026a30     qt-mt323:qt-mt323.dll
 0002:00000a34       __imp_?select@QSqlCursor@@QAE_NXZ 10026a34     qt-mt323:qt-mt323.dll
 0002:00000a38       __imp_?numSelections@QTable@@QBEHXZ 10026a38     qt-mt323:qt-mt323.dll
 0002:00000a3c       __imp_?selection@QTable@@QBE?AVQTableSelection@@H@Z 10026a3c     qt-mt323:qt-mt323.dll
 0002:00000a40       __imp_?selectCells@QTable@@QAEXHHHH@Z 10026a40     qt-mt323:qt-mt323.dll
 0002:00000a44       __imp_?sqlCursor@QDataTable@@QBEPAVQSqlCursor@@XZ 10026a44     qt-mt323:qt-mt323.dll
 0002:00000a48       __imp_?refresh@QDataTable@@QAEXW4Refresh@1@@Z 10026a48     qt-mt323:qt-mt323.dll
 0002:00000a4c       __imp_??0QTimer@@QAE@PAVQObject@@PBD@Z 10026a4c     qt-mt323:qt-mt323.dll
 0002:00000a50       __imp_??1QTimer@@UAE@XZ    10026a50     qt-mt323:qt-mt323.dll
 0002:00000a54       __imp_?start@QTimer@@QAEHH_N@Z 10026a54     qt-mt323:qt-mt323.dll
 0002:00000a58       __imp_?stop@QTimer@@QAEXXZ 10026a58     qt-mt323:qt-mt323.dll
 0002:00000a5c       __imp_?toString@QDate@@QBE?AVQString@@ABV2@@Z 10026a5c     qt-mt323:qt-mt323.dll
 0002:00000a60       __imp_?currentDate@QDate@@SA?AV1@XZ 10026a60     qt-mt323:qt-mt323.dll
 0002:00000a64       __imp_?date@QDateEdit@@QBE?AVQDate@@XZ 10026a64     qt-mt323:qt-mt323.dll
 0002:00000a68       __imp_??0QAction@@QAE@ABVQString@@0VQKeySequence@@PAVQObject@@PBD_N@Z 10026a68     qt-mt323:qt-mt323.dll
 0002:00000a6c       __imp_?page@QTabWidget@@QBEPAVQWidget@@H@Z 10026a6c     qt-mt323:qt-mt323.dll
 0002:00000a70       __imp_?start@QThread@@QAEXXZ 10026a70     qt-mt323:qt-mt323.dll
 0002:00000a74       __imp_?running@QThread@@QBE_NXZ 10026a74     qt-mt323:qt-mt323.dll
 0002:00000a78       __imp_?afterSeek@QSqlCursor@@MAEXXZ 10026a78     qt-mt323:qt-mt323.dll
 0002:00000a7c       __imp_?append@QSqlCursor@@EAEXABVQSqlField@@@Z 10026a7c     qt-mt323:qt-mt323.dll
 0002:00000a80       __imp_?append@QSqlCursor@@UAEXABVQSqlFieldInfo@@@Z 10026a80     qt-mt323:qt-mt323.dll
 0002:00000a84       __imp_?beforeSeek@QSqlQuery@@MAEXXZ 10026a84     qt-mt323:qt-mt323.dll
 0002:00000a88       __imp_?calculateField@QSqlCursor@@MAE?AVQVariant@@ABVQString@@@Z 10026a88     qt-mt323:qt-mt323.dll
 0002:00000a8c       __imp_?className@QTimer@@UBEPBDXZ 10026a8c     qt-mt323:qt-mt323.dll
 0002:00000a90       __imp_?clear@QSqlCursor@@UAEXXZ 10026a90     qt-mt323:qt-mt323.dll
 0002:00000a94       __imp_?clearValues@QSqlRecord@@UAEX_N@Z 10026a94     qt-mt323:qt-mt323.dll
 0002:00000a98       __imp_?del@QSqlCursor@@MAEHABVQString@@_N@Z 10026a98     qt-mt323:qt-mt323.dll
 0002:00000a9c       __imp_?del@QSqlCursor@@UAEH_N@Z 10026a9c     qt-mt323:qt-mt323.dll
 0002:00000aa0       __imp_?editBuffer@QSqlCursor@@UAEPAVQSqlRecord@@_N@Z 10026aa0     qt-mt323:qt-mt323.dll
 0002:00000aa4       __imp_?event@QTimer@@MAE_NPAVQEvent@@@Z 10026aa4     qt-mt323:qt-mt323.dll
 0002:00000aa8       __imp_?exec@QSqlCursor@@MAE_NABVQString@@@Z 10026aa8     qt-mt323:qt-mt323.dll
 0002:00000aac       __imp_?index@QSqlCursor@@UBE?AVQSqlIndex@@ABVQStringList@@@Z 10026aac     qt-mt323:qt-mt323.dll
 0002:00000ab0       __imp_?insert@QSqlCursor@@EAEXHABVQSqlField@@@Z 10026ab0     qt-mt323:qt-mt323.dll
 0002:00000ab4       __imp_?insert@QSqlCursor@@UAEH_N@Z 10026ab4     qt-mt323:qt-mt323.dll
 0002:00000ab8       __imp_?insert@QSqlCursor@@UAEXHABVQSqlFieldInfo@@@Z 10026ab8     qt-mt323:qt-mt323.dll
 0002:00000abc       __imp_?last@QSqlQuery@@UAE_NXZ 10026abc     qt-mt323:qt-mt323.dll
 0002:00000ac0       __imp_?metaObject@QTimer@@UBEPAVQMetaObject@@XZ 10026ac0     qt-mt323:qt-mt323.dll
 0002:00000ac4       __imp_?next@QSqlQuery@@UAE_NXZ 10026ac4     qt-mt323:qt-mt323.dll
 0002:00000ac8       __imp_?prev@QSqlQuery@@UAE_NXZ 10026ac8     qt-mt323:qt-mt323.dll
 0002:00000acc       __imp_?primaryIndex@QSqlCursor@@UBE?AVQSqlIndex@@_N@Z 10026acc     qt-mt323:qt-mt323.dll
 0002:00000ad0       __imp_?primeDelete@QSqlCursor@@UAEPAVQSqlRecord@@XZ 10026ad0     qt-mt323:qt-mt323.dll
 0002:00000ad4       __imp_?primeInsert@QSqlCursor@@UAEPAVQSqlRecord@@XZ 10026ad4     qt-mt323:qt-mt323.dll
 0002:00000ad8       __imp_?primeUpdate@QSqlCursor@@UAEPAVQSqlRecord@@XZ 10026ad8     qt-mt323:qt-mt323.dll
 0002:00000adc       __imp_?qt_cast@QTimer@@UAEPAXPBD@Z 10026adc     qt-mt323:qt-mt323.dll
 0002:00000ae0       __imp_?qt_emit@QTimer@@UAE_NHPAUQUObject@@@Z 10026ae0     qt-mt323:qt-mt323.dll
 0002:00000ae4       __imp_?qt_invoke@QTimer@@UAE_NHPAUQUObject@@@Z 10026ae4     qt-mt323:qt-mt323.dll
 0002:00000ae8       __imp_?qt_property@QTimer@@UAE_NHHPAVQVariant@@@Z 10026ae8     qt-mt323:qt-mt323.dll
 0002:00000aec       __imp_?remove@QSqlCursor@@UAEXH@Z 10026aec     qt-mt323:qt-mt323.dll
 0002:00000af0       __imp_?seek@QSqlQuery@@UAE_NH_N@Z 10026af0     qt-mt323:qt-mt323.dll
 0002:00000af4       __imp_?select@QSqlCursor@@UAE_NABVQString@@ABVQSqlIndex@@@Z 10026af4     qt-mt323:qt-mt323.dll
 0002:00000af8       __imp_?setCalculated@QSqlCursor@@UAEXABVQString@@_N@Z 10026af8     qt-mt323:qt-mt323.dll
 0002:00000afc       __imp_?setFilter@QSqlCursor@@UAEXABVQString@@@Z 10026afc     qt-mt323:qt-mt323.dll
 0002:00000b00       __imp_?setGenerated@QSqlCursor@@UAEXABVQString@@_N@Z 10026b00     qt-mt323:qt-mt323.dll
 0002:00000b04       __imp_?setGenerated@QSqlCursor@@UAEXH_N@Z 10026b04     qt-mt323:qt-mt323.dll
 0002:00000b08       __imp_?setMode@QSqlCursor@@UAEXH@Z 10026b08     qt-mt323:qt-mt323.dll
 0002:00000b0c       __imp_?setName@QSqlCursor@@UAEXABVQString@@_N@Z 10026b0c     qt-mt323:qt-mt323.dll
 0002:00000b10       __imp_?setNull@QSqlRecord@@UAEXABVQString@@@Z 10026b10     qt-mt323:qt-mt323.dll
 0002:00000b14       __imp_?setNull@QSqlRecord@@UAEXH@Z 10026b14     qt-mt323:qt-mt323.dll
 0002:00000b18       __imp_??1?$QMap@VQString@@H@@QAE@XZ 10026b18     qt-mt323:qt-mt323.dll
 0002:00000b1c       __imp_?atEnd@QTextStream@@QBE_NXZ 10026b1c     qt-mt323:qt-mt323.dll
 0002:00000b20       __imp_?setTrimmed@QSqlCursor@@UAEXABVQString@@_N@Z 10026b20     qt-mt323:qt-mt323.dll
 0002:00000b24       __imp_?setValue@QSqlCursor@@UAEXABVQString@@ABVQVariant@@@Z 10026b24     qt-mt323:qt-mt323.dll
 0002:00000b28       __imp_?setValue@QSqlCursor@@UAEXHABVQVariant@@@Z 10026b28     qt-mt323:qt-mt323.dll
 0002:00000b2c       __imp_?toString@QSqlCursor@@MBE?AVQString@@ABV2@PAVQSqlField@@0@Z 10026b2c     qt-mt323:qt-mt323.dll
 0002:00000b30       __imp_?toString@QSqlCursor@@MBE?AVQString@@ABVQSqlIndex@@PAVQSqlRecord@@ABV2@22@Z 10026b30     qt-mt323:qt-mt323.dll
 0002:00000b34       __imp_?toString@QSqlCursor@@MBE?AVQString@@PAVQSqlRecord@@ABV2@11@Z 10026b34     qt-mt323:qt-mt323.dll
 0002:00000b38       __imp_?toString@QSqlCursor@@UBE?AVQString@@ABV2@0@Z 10026b38     qt-mt323:qt-mt323.dll
 0002:00000b3c       __imp_?toStringList@QSqlRecord@@UBE?AVQStringList@@ABVQString@@@Z 10026b3c     qt-mt323:qt-mt323.dll
 0002:00000b40       __imp_?update@QSqlCursor@@MAEHABVQString@@_N@Z 10026b40     qt-mt323:qt-mt323.dll
 0002:00000b44       __imp_?update@QSqlCursor@@UAEH_N@Z 10026b44     qt-mt323:qt-mt323.dll
 0002:00000b48       __imp_?value@QSqlCursor@@UBE?AVQVariant@@ABVQString@@@Z 10026b48     qt-mt323:qt-mt323.dll
 0002:00000b4c       __imp_?left@QString@@QBE?AV1@I@Z 10026b4c     qt-mt323:qt-mt323.dll
 0002:00000b50       __imp_?setNum@QString@@QAEAAV1@_JH@Z 10026b50     qt-mt323:qt-mt323.dll
 0002:00000b54       __imp_?disconnect@QObject@@SA_NPBV1@PBD01@Z 10026b54     qt-mt323:qt-mt323.dll
 0002:00000b58       __imp_?pos@QWidget@@QBE?AVQPoint@@XZ 10026b58     qt-mt323:qt-mt323.dll
 0002:00000b5c       __imp_?isMaximized@QWidget@@QBE_NXZ 10026b5c     qt-mt323:qt-mt323.dll
 0002:00000b60       __imp_?childCount@QListView@@QBEHXZ 10026b60     qt-mt323:qt-mt323.dll
 0002:00000b64       __imp_??1QTableItem@@UAE@XZ 10026b64     qt-mt323:qt-mt323.dll
 0002:00000b68       __imp_??0QCheckTableItem@@QAE@PAVQTable@@ABVQString@@@Z 10026b68     qt-mt323:qt-mt323.dll
 0002:00000b6c       __imp_?isRowSelected@QTable@@QBE_NH_N@Z 10026b6c     qt-mt323:qt-mt323.dll
 0002:00000b70       __imp_?move@QDialog@@QAEXABVQPoint@@@Z 10026b70     qt-mt323:qt-mt323.dll
 0002:00000b74       __imp_?resize@QDialog@@QAEXABVQSize@@@Z 10026b74     qt-mt323:qt-mt323.dll
 0002:00000b78       __imp_?accept@QDialog@@MAEXXZ 10026b78     qt-mt323:qt-mt323.dll
 0002:00000b7c       __imp_?alignment@QTableItem@@UBEHXZ 10026b7c     qt-mt323:qt-mt323.dll
 0002:00000b80       __imp_?closeEvent@QDialog@@MAEXPAVQCloseEvent@@@Z 10026b80     qt-mt323:qt-mt323.dll
 0002:00000b84       __imp_?contextMenuEvent@QDialog@@MAEXPAVQContextMenuEvent@@@Z 10026b84     qt-mt323:qt-mt323.dll
 0002:00000b88       __imp_?createEditor@QCheckTableItem@@UBEPAVQWidget@@XZ 10026b88     qt-mt323:qt-mt323.dll
 0002:00000b8c       __imp_?done@QDialog@@MAEXH@Z 10026b8c     qt-mt323:qt-mt323.dll
 0002:00000b90       __imp_?eventFilter@QDialog@@MAE_NPAVQObject@@PAVQEvent@@@Z 10026b90     qt-mt323:qt-mt323.dll
 0002:00000b94       __imp_?hide@QDialog@@UAEXXZ 10026b94     qt-mt323:qt-mt323.dll
 0002:00000b98       __imp_?key@QTableItem@@UBE?AVQString@@XZ 10026b98     qt-mt323:qt-mt323.dll
 0002:00000b9c       __imp_?keyPressEvent@QDialog@@MAEXPAVQKeyEvent@@@Z 10026b9c     qt-mt323:qt-mt323.dll
 0002:00000ba0       __imp_?minimumSizeHint@QDialog@@UBE?AVQSize@@XZ 10026ba0     qt-mt323:qt-mt323.dll
 0002:00000ba4       __imp_?move@QDialog@@UAEXHH@Z 10026ba4     qt-mt323:qt-mt323.dll
 0002:00000ba8       __imp_?paint@QCheckTableItem@@UAEXPAVQPainter@@ABVQColorGroup@@ABVQRect@@_N@Z 10026ba8     qt-mt323:qt-mt323.dll
 0002:00000bac       __imp_?pixmap@QTableItem@@UBE?AVQPixmap@@XZ 10026bac     qt-mt323:qt-mt323.dll
 0002:00000bb0       __imp_?reject@QDialog@@MAEXXZ 10026bb0     qt-mt323:qt-mt323.dll
 0002:00000bb4       __imp_?resize@QDialog@@UAEXHH@Z 10026bb4     qt-mt323:qt-mt323.dll
 0002:00000bb8       __imp_?resizeEvent@QDialog@@MAEXPAVQResizeEvent@@@Z 10026bb8     qt-mt323:qt-mt323.dll
 0002:00000bbc       __imp_?rtti@QCheckTableItem@@UBEHXZ 10026bbc     qt-mt323:qt-mt323.dll
 0002:00000bc0       __imp_?setChecked@QCheckTableItem@@UAEX_N@Z 10026bc0     qt-mt323:qt-mt323.dll
 0002:00000bc4       __imp_?setCol@QTableItem@@UAEXH@Z 10026bc4     qt-mt323:qt-mt323.dll
 0002:00000bc8       __imp_??0QString@@QAE@ABV0@@Z 10026bc8     qt-mt323:qt-mt323.dll
 0002:00000bcc       __imp_?setEnabled@QTableItem@@UAEX_N@Z 10026bcc     qt-mt323:qt-mt323.dll
 0002:00000bd0       __imp_?setGeometry@QDialog@@UAEXABVQRect@@@Z 10026bd0     qt-mt323:qt-mt323.dll
 0002:00000bd4       __imp_?setGeometry@QDialog@@UAEXHHHH@Z 10026bd4     qt-mt323:qt-mt323.dll
 0002:00000bd8       __imp_?setPixmap@QTableItem@@UAEXABVQPixmap@@@Z 10026bd8     qt-mt323:qt-mt323.dll
 0002:00000bdc       __imp_?setReplaceable@QTableItem@@UAEX_N@Z 10026bdc     qt-mt323:qt-mt323.dll
 0002:00000be0       __imp_?setRow@QTableItem@@UAEXH@Z 10026be0     qt-mt323:qt-mt323.dll
 0002:00000be4       __imp_?setSpan@QTableItem@@UAEXHH@Z 10026be4     qt-mt323:qt-mt323.dll
 0002:00000be8       __imp_?setText@QCheckTableItem@@UAEXABVQString@@@Z 10026be8     qt-mt323:qt-mt323.dll
 0002:00000bec       __imp_?setWordWrap@QTableItem@@UAEX_N@Z 10026bec     qt-mt323:qt-mt323.dll
 0002:00000bf0       __imp_?show@QDialog@@UAEXXZ 10026bf0     qt-mt323:qt-mt323.dll
 0002:00000bf4       __imp_?sizeHint@QCheckTableItem@@UBE?AVQSize@@XZ 10026bf4     qt-mt323:qt-mt323.dll
 0002:00000bf8       __imp_?sizeHint@QDialog@@UBE?AVQSize@@XZ 10026bf8     qt-mt323:qt-mt323.dll
 0002:00000bfc       __imp_?text@QTableItem@@UBE?AVQString@@XZ 10026bfc     qt-mt323:qt-mt323.dll
 0002:00000c00       __imp_?qstrcmp@@YAHPBD0@Z  10026c00     qt-mt323:qt-mt323.dll
 0002:00000c04       __imp_?fromLatin1@QString@@SA?AV1@PBDH@Z 10026c04     qt-mt323:qt-mt323.dll
 0002:00000c08       __imp_?qt_cast@QDialog@@UAEPAXPBD@Z 10026c08     qt-mt323:qt-mt323.dll
 0002:00000c0c       __imp_?qt_invoke@QDialog@@UAE_NHPAUQUObject@@@Z 10026c0c     qt-mt323:qt-mt323.dll
 0002:00000c10       __imp_?qt_emit@QDialog@@UAE_NHPAUQUObject@@@Z 10026c10     qt-mt323:qt-mt323.dll
 0002:00000c14       __imp_?qt_property@QDialog@@UAE_NHHPAVQVariant@@@Z 10026c14     qt-mt323:qt-mt323.dll
 0002:00000c18       __imp_?staticMetaObject@QDialog@@SAPAVQMetaObject@@XZ 10026c18     qt-mt323:qt-mt323.dll
 0002:00000c1c       __imp_?new_metaobject@QMetaObject@@SAPAV1@PBDPAV1@QBUQMetaData@@H2HQBVQMetaProperty@@HQBUQMetaEnum@@HQBUQClassInfo@@H@Z 10026c1c     qt-mt323:qt-mt323.dll
 0002:00000c20       __imp_??0QMetaObjectCleanUp@@QAE@PBDP6APAVQMetaObject@@XZ@Z 10026c20     qt-mt323:qt-mt323.dll
 0002:00000c24       __imp_??1QMetaObjectCleanUp@@QAE@XZ 10026c24     qt-mt323:qt-mt323.dll
 0002:00000c28       __imp_?setMetaObject@QMetaObjectCleanUp@@QAEXAAPAVQMetaObject@@@Z 10026c28     qt-mt323:qt-mt323.dll
 0002:00000c2c       __imp_?translate@QApplication@@QBE?AVQString@@PBD00W4Encoding@1@@Z 10026c2c     qt-mt323:qt-mt323.dll
 0002:00000c30       __imp_?qApp@@3PAVQApplication@@A 10026c30     qt-mt323:qt-mt323.dll
 0002:00000c34       __imp_?setTabOrder@QWidget@@SAXPAV1@0@Z 10026c34     qt-mt323:qt-mt323.dll
 0002:00000c38       __imp_??0QDialog@@QAE@PAVQWidget@@PBD_NI@Z 10026c38     qt-mt323:qt-mt323.dll
 0002:00000c3c       __imp_??1QDialog@@UAE@XZ   10026c3c     qt-mt323:qt-mt323.dll
 0002:00000c40       __imp_?setSizeGripEnabled@QDialog@@QAEX_N@Z 10026c40     qt-mt323:qt-mt323.dll
 0002:00000c44       __imp_??0QKeySequence@@QAE@ABVQString@@@Z 10026c44     qt-mt323:qt-mt323.dll
 0002:00000c48       __imp_??1QKeySequence@@QAE@XZ 10026c48     qt-mt323:qt-mt323.dll
 0002:00000c4c       __imp_??1QButton@@UAE@XZ   10026c4c     qt-mt323:qt-mt323.dll
 0002:00000c50       __imp_??0QPushButton@@QAE@PAVQWidget@@PBD@Z 10026c50     qt-mt323:qt-mt323.dll
 0002:00000c54       __imp_??1QPushButton@@UAE@XZ 10026c54     qt-mt323:qt-mt323.dll
 0002:00000c58       __imp_?setFrameShape@QFrame@@QAEXW4Shape@1@@Z 10026c58     qt-mt323:qt-mt323.dll
 0002:00000c5c       __imp_?setFrameShadow@QFrame@@QAEXW4Shadow@1@@Z 10026c5c     qt-mt323:qt-mt323.dll
 0002:00000c60       __imp_??0QGroupBox@@QAE@PAVQWidget@@PBD@Z 10026c60     qt-mt323:qt-mt323.dll
 0002:00000c64       __imp_??1QGroupBox@@UAE@XZ 10026c64     qt-mt323:qt-mt323.dll
 0002:00000c68       __imp_??0QLabel@@QAE@PAVQWidget@@PBDI@Z 10026c68     qt-mt323:qt-mt323.dll
 0002:00000c6c       __imp_??1QLabel@@UAE@XZ    10026c6c     qt-mt323:qt-mt323.dll
 0002:00000c70       __imp_??0QLineEdit@@QAE@PAVQWidget@@PBD@Z 10026c70     qt-mt323:qt-mt323.dll
 0002:00000c74       __imp_??1QLineEdit@@UAE@XZ 10026c74     qt-mt323:qt-mt323.dll
 0002:00000c78       __imp_??0QComboBox@@QAE@_NPAVQWidget@@PBD@Z 10026c78     qt-mt323:qt-mt323.dll
 0002:00000c7c       __imp_??1QComboBox@@UAE@XZ 10026c7c     qt-mt323:qt-mt323.dll
 0002:00000c80       __imp_??0QCheckBox@@QAE@PAVQWidget@@PBD@Z 10026c80     qt-mt323:qt-mt323.dll
 0002:00000c84       __imp_??1QLayoutItem@@UAE@XZ 10026c84     qt-mt323:qt-mt323.dll
 0002:00000c88       __imp_??0QSpacerItem@@QAE@HHW4SizeType@QSizePolicy@@0@Z 10026c88     qt-mt323:qt-mt323.dll
 0002:00000c8c       __imp_?setResizeMode@QLayout@@QAEXW4ResizeMode@1@@Z 10026c8c     qt-mt323:qt-mt323.dll
 0002:00000c90       __imp_??0QGridLayout@@QAE@PAVQLayout@@HHHPBD@Z 10026c90     qt-mt323:qt-mt323.dll
 0002:00000c94       __imp_??1QGridLayout@@UAE@XZ 10026c94     qt-mt323:qt-mt323.dll
 0002:00000c98       __imp_?addItem@QGridLayout@@QAEXPAVQLayoutItem@@HH@Z 10026c98     qt-mt323:qt-mt323.dll
 0002:00000c9c       __imp_?addWidget@QGridLayout@@QAEXPAVQWidget@@HHH@Z 10026c9c     qt-mt323:qt-mt323.dll
 0002:00000ca0       __imp_?addMultiCellWidget@QGridLayout@@QAEXPAVQWidget@@HHHHH@Z 10026ca0     qt-mt323:qt-mt323.dll
 0002:00000ca4       __imp_?addWidget@QBoxLayout@@QAEXPAVQWidget@@HH@Z 10026ca4     qt-mt323:qt-mt323.dll
 0002:00000ca8       __imp_?addLayout@QBoxLayout@@QAEXPAVQLayout@@H@Z 10026ca8     qt-mt323:qt-mt323.dll
 0002:00000cac       __imp_??0QHBoxLayout@@QAE@PAVQWidget@@HHPBD@Z 10026cac     qt-mt323:qt-mt323.dll
 0002:00000cb0       __imp_??1QHBoxLayout@@UAE@XZ 10026cb0     qt-mt323:qt-mt323.dll
 0002:00000cb4       __imp_??0QVBoxLayout@@QAE@PAVQWidget@@HHPBD@Z 10026cb4     qt-mt323:qt-mt323.dll
 0002:00000cb8       __imp_??1QVBoxLayout@@UAE@XZ 10026cb8     qt-mt323:qt-mt323.dll
 0002:00000cbc       __imp_?addItem@QGridLayout@@UAEXPAVQLayoutItem@@@Z 10026cbc     qt-mt323:qt-mt323.dll
 0002:00000cc0       __imp_?childEvent@QGroupBox@@MAEXPAVQChildEvent@@@Z 10026cc0     qt-mt323:qt-mt323.dll
 0002:00000cc4       __imp_?className@QCheckBox@@UBEPBDXZ 10026cc4     qt-mt323:qt-mt323.dll
 0002:00000cc8       __imp_?className@QComboBox@@UBEPBDXZ 10026cc8     qt-mt323:qt-mt323.dll
 0002:00000ccc       __imp_?className@QGridLayout@@UBEPBDXZ 10026ccc     qt-mt323:qt-mt323.dll
 0002:00000cd0       __imp_?className@QGroupBox@@UBEPBDXZ 10026cd0     qt-mt323:qt-mt323.dll
 0002:00000cd4       __imp_?className@QHBoxLayout@@UBEPBDXZ 10026cd4     qt-mt323:qt-mt323.dll
 0002:00000cd8       __imp_?className@QLabel@@UBEPBDXZ 10026cd8     qt-mt323:qt-mt323.dll
 0002:00000cdc       __imp_?className@QLineEdit@@UBEPBDXZ 10026cdc     qt-mt323:qt-mt323.dll
 0002:00000ce0       __imp_?className@QPushButton@@UBEPBDXZ 10026ce0     qt-mt323:qt-mt323.dll
 0002:00000ce4       __imp_?className@QVBoxLayout@@UBEPBDXZ 10026ce4     qt-mt323:qt-mt323.dll
 0002:00000ce8       __imp_?clear@QLineEdit@@UAEXXZ 10026ce8     qt-mt323:qt-mt323.dll
 0002:00000cec       __imp_?clearValidator@QLineEdit@@UAEXXZ 10026cec     qt-mt323:qt-mt323.dll
 0002:00000cf0       __imp_?contextMenuEvent@QLineEdit@@MAEXPAVQContextMenuEvent@@@Z 10026cf0     qt-mt323:qt-mt323.dll
 0002:00000cf4       __imp_?copy@QLineEdit@@UBEXXZ 10026cf4     qt-mt323:qt-mt323.dll
 0002:00000cf8       __imp_?createPopupMenu@QLineEdit@@MAEPAVQPopupMenu@@XZ 10026cf8     qt-mt323:qt-mt323.dll
 0002:00000cfc       __imp_?cut@QLineEdit@@UAEXXZ 10026cfc     qt-mt323:qt-mt323.dll
 0002:00000d00       __imp_?deselect@QLineEdit@@UAEXXZ 10026d00     qt-mt323:qt-mt323.dll
 0002:00000d04       __imp_?dragEnterEvent@QLineEdit@@MAEXPAVQDragEnterEvent@@@Z 10026d04     qt-mt323:qt-mt323.dll
 0002:00000d08       __imp_?dragLeaveEvent@QLineEdit@@MAEXPAVQDragLeaveEvent@@@Z 10026d08     qt-mt323:qt-mt323.dll
 0002:00000d0c       __imp_?dragMoveEvent@QLineEdit@@MAEXPAVQDragMoveEvent@@@Z 10026d0c     qt-mt323:qt-mt323.dll
 0002:00000d10       __imp_?drawButton@QCheckBox@@MAEXPAVQPainter@@@Z 10026d10     qt-mt323:qt-mt323.dll
 0002:00000d14       __imp_?drawButton@QPushButton@@MAEXPAVQPainter@@@Z 10026d14     qt-mt323:qt-mt323.dll
 0002:00000d18       __imp_?drawButtonLabel@QCheckBox@@MAEXPAVQPainter@@@Z 10026d18     qt-mt323:qt-mt323.dll
 0002:00000d1c       __imp_?drawButtonLabel@QPushButton@@MAEXPAVQPainter@@@Z 10026d1c     qt-mt323:qt-mt323.dll
 0002:00000d20       __imp_?drawContents@QLabel@@MAEXPAVQPainter@@@Z 10026d20     qt-mt323:qt-mt323.dll
 0002:00000d24       __imp_?drawContents@QLineEdit@@MAEXPAVQPainter@@@Z 10026d24     qt-mt323:qt-mt323.dll
 0002:00000d28       __imp_?dropEvent@QLineEdit@@MAEXPAVQDropEvent@@@Z 10026d28     qt-mt323:qt-mt323.dll
 0002:00000d2c       __imp_?enabledChange@QButton@@MAEX_N@Z 10026d2c     qt-mt323:qt-mt323.dll
 0002:00000d30       __imp_?event@QGroupBox@@MAE_NPAVQEvent@@@Z 10026d30     qt-mt323:qt-mt323.dll
 0002:00000d34       __imp_?event@QLineEdit@@MAE_NPAVQEvent@@@Z 10026d34     qt-mt323:qt-mt323.dll
 0002:00000d38       __imp_?eventFilter@QComboBox@@UAE_NPAVQObject@@PAVQEvent@@@Z 10026d38     qt-mt323:qt-mt323.dll
 0002:00000d3c       __imp_?expanding@QGridLayout@@UBE?AW4ExpandData@QSizePolicy@@XZ 10026d3c     qt-mt323:qt-mt323.dll
 0002:00000d40       __imp_?expanding@QSpacerItem@@UBE?AW4ExpandData@QSizePolicy@@XZ 10026d40     qt-mt323:qt-mt323.dll
 0002:00000d44       __imp_?focusInEvent@QButton@@MAEXPAVQFocusEvent@@@Z 10026d44     qt-mt323:qt-mt323.dll
 0002:00000d48       __imp_?focusInEvent@QComboBox@@MAEXPAVQFocusEvent@@@Z 10026d48     qt-mt323:qt-mt323.dll
 0002:00000d4c       __imp_?focusInEvent@QGroupBox@@MAEXPAVQFocusEvent@@@Z 10026d4c     qt-mt323:qt-mt323.dll
 0002:00000d50       __imp_?focusInEvent@QLineEdit@@MAEXPAVQFocusEvent@@@Z 10026d50     qt-mt323:qt-mt323.dll
 0002:00000d54       __imp_?focusInEvent@QPushButton@@MAEXPAVQFocusEvent@@@Z 10026d54     qt-mt323:qt-mt323.dll
 0002:00000d58       __imp_?focusOutEvent@QButton@@MAEXPAVQFocusEvent@@@Z 10026d58     qt-mt323:qt-mt323.dll
 0002:00000d5c       __imp_?focusOutEvent@QComboBox@@MAEXPAVQFocusEvent@@@Z 10026d5c     qt-mt323:qt-mt323.dll
 0002:00000d60       __imp_?focusOutEvent@QLineEdit@@MAEXPAVQFocusEvent@@@Z 10026d60     qt-mt323:qt-mt323.dll
 0002:00000d64       __imp_?focusOutEvent@QPushButton@@MAEXPAVQFocusEvent@@@Z 10026d64     qt-mt323:qt-mt323.dll
 0002:00000d68       __imp_?fontChange@QGroupBox@@MAEXABVQFont@@@Z 10026d68     qt-mt323:qt-mt323.dll
 0002:00000d6c       __imp_?fontChange@QLabel@@MAEXABVQFont@@@Z 10026d6c     qt-mt323:qt-mt323.dll
 0002:00000d70       __imp_?geometry@QSpacerItem@@UBE?AVQRect@@XZ 10026d70     qt-mt323:qt-mt323.dll
 0002:00000d74       __imp_?hasHeightForWidth@QGridLayout@@UBE_NXZ 10026d74     qt-mt323:qt-mt323.dll
 0002:00000d78       __imp_?hasHeightForWidth@QLayoutItem@@UBE_NXZ 10026d78     qt-mt323:qt-mt323.dll
 0002:00000d7c       __imp_?heightForWidth@QGridLayout@@UBEHH@Z 10026d7c     qt-mt323:qt-mt323.dll
 0002:00000d80       __imp_?heightForWidth@QLabel@@UBEHH@Z 10026d80     qt-mt323:qt-mt323.dll
 0002:00000d84       __imp_?heightForWidth@QLayoutItem@@UBEHH@Z 10026d84     qt-mt323:qt-mt323.dll
 0002:00000d88       __imp_?hitButton@QButton@@MBE_NABVQPoint@@@Z 10026d88     qt-mt323:qt-mt323.dll
 0002:00000d8c       __imp_?hitButton@QCheckBox@@MBE_NABVQPoint@@@Z 10026d8c     qt-mt323:qt-mt323.dll
 0002:00000d90       __imp_?imComposeEvent@QLineEdit@@MAEXPAVQIMEvent@@@Z 10026d90     qt-mt323:qt-mt323.dll
 0002:00000d94       __imp_?imEndEvent@QLineEdit@@MAEXPAVQIMEvent@@@Z 10026d94     qt-mt323:qt-mt323.dll
 0002:00000d98       __imp_?imStartEvent@QLineEdit@@MAEXPAVQIMEvent@@@Z 10026d98     qt-mt323:qt-mt323.dll
 0002:00000d9c       __imp_?insert@QLineEdit@@UAEXABVQString@@@Z 10026d9c     qt-mt323:qt-mt323.dll
 0002:00000da0       __imp_?invalidate@QGridLayout@@UAEXXZ 10026da0     qt-mt323:qt-mt323.dll
 0002:00000da4       __imp_?invalidate@QLayoutItem@@UAEXXZ 10026da4     qt-mt323:qt-mt323.dll
 0002:00000da8       __imp_?isEmpty@QSpacerItem@@UBE_NXZ 10026da8     qt-mt323:qt-mt323.dll
 0002:00000dac       __imp_?iterator@QGridLayout@@UAE?AVQLayoutIterator@@XZ 10026dac     qt-mt323:qt-mt323.dll
 0002:00000db0       __imp_?iterator@QLayoutItem@@UAE?AVQLayoutIterator@@XZ 10026db0     qt-mt323:qt-mt323.dll
 0002:00000db4       __imp_?keyPressEvent@QButton@@MAEXPAVQKeyEvent@@@Z 10026db4     qt-mt323:qt-mt323.dll
 0002:00000db8       __imp_?keyPressEvent@QComboBox@@MAEXPAVQKeyEvent@@@Z 10026db8     qt-mt323:qt-mt323.dll
 0002:00000dbc       __imp_?keyPressEvent@QLineEdit@@MAEXPAVQKeyEvent@@@Z 10026dbc     qt-mt323:qt-mt323.dll
 0002:00000dc0       __imp_?keyReleaseEvent@QButton@@MAEXPAVQKeyEvent@@@Z 10026dc0     qt-mt323:qt-mt323.dll
 0002:00000dc4       __imp_?layout@QLayoutItem@@UAEPAVQLayout@@XZ 10026dc4     qt-mt323:qt-mt323.dll
 0002:00000dc8       __imp_?maximumSize@QGridLayout@@UBE?AVQSize@@XZ 10026dc8     qt-mt323:qt-mt323.dll
 0002:00000dcc       __imp_?maximumSize@QSpacerItem@@UBE?AVQSize@@XZ 10026dcc     qt-mt323:qt-mt323.dll
 0002:00000dd0       __imp_?metaObject@QCheckBox@@UBEPAVQMetaObject@@XZ 10026dd0     qt-mt323:qt-mt323.dll
 0002:00000dd4       __imp_?metaObject@QComboBox@@UBEPAVQMetaObject@@XZ 10026dd4     qt-mt323:qt-mt323.dll
 0002:00000dd8       __imp_?metaObject@QGridLayout@@UBEPAVQMetaObject@@XZ 10026dd8     qt-mt323:qt-mt323.dll
 0002:00000ddc       __imp_?metaObject@QGroupBox@@UBEPAVQMetaObject@@XZ 10026ddc     qt-mt323:qt-mt323.dll
 0002:00000de0       __imp_?metaObject@QHBoxLayout@@UBEPAVQMetaObject@@XZ 10026de0     qt-mt323:qt-mt323.dll
 0002:00000de4       __imp_?metaObject@QLabel@@UBEPAVQMetaObject@@XZ 10026de4     qt-mt323:qt-mt323.dll
 0002:00000de8       __imp_?metaObject@QLineEdit@@UBEPAVQMetaObject@@XZ 10026de8     qt-mt323:qt-mt323.dll
 0002:00000dec       __imp_?metaObject@QPushButton@@UBEPAVQMetaObject@@XZ 10026dec     qt-mt323:qt-mt323.dll
 0002:00000df0       __imp_?metaObject@QVBoxLayout@@UBEPAVQMetaObject@@XZ 10026df0     qt-mt323:qt-mt323.dll
 0002:00000df4       __imp_?minimumSize@QGridLayout@@UBE?AVQSize@@XZ 10026df4     qt-mt323:qt-mt323.dll
 0002:00000df8       __imp_?minimumSize@QSpacerItem@@UBE?AVQSize@@XZ 10026df8     qt-mt323:qt-mt323.dll
 0002:00000dfc       __imp_?minimumSizeHint@QLabel@@UBE?AVQSize@@XZ 10026dfc     qt-mt323:qt-mt323.dll
 0002:00000e00       __imp_?minimumSizeHint@QLineEdit@@UBE?AVQSize@@XZ 10026e00     qt-mt323:qt-mt323.dll
 0002:00000e04       __imp_?mouseDoubleClickEvent@QComboBox@@MAEXPAVQMouseEvent@@@Z 10026e04     qt-mt323:qt-mt323.dll
 0002:00000e08       __imp_?mouseDoubleClickEvent@QLineEdit@@MAEXPAVQMouseEvent@@@Z 10026e08     qt-mt323:qt-mt323.dll
 0002:00000e0c       __imp_?mouseMoveEvent@QButton@@MAEXPAVQMouseEvent@@@Z 10026e0c     qt-mt323:qt-mt323.dll
 0002:00000e10       __imp_?mouseMoveEvent@QComboBox@@MAEXPAVQMouseEvent@@@Z 10026e10     qt-mt323:qt-mt323.dll
 0002:00000e14       __imp_?mouseMoveEvent@QLineEdit@@MAEXPAVQMouseEvent@@@Z 10026e14     qt-mt323:qt-mt323.dll
 0002:00000e18       __imp_?mousePressEvent@QButton@@MAEXPAVQMouseEvent@@@Z 10026e18     qt-mt323:qt-mt323.dll
 0002:00000e1c       __imp_?mousePressEvent@QComboBox@@MAEXPAVQMouseEvent@@@Z 10026e1c     qt-mt323:qt-mt323.dll
 0002:00000e20       __imp_?mousePressEvent@QLineEdit@@MAEXPAVQMouseEvent@@@Z 10026e20     qt-mt323:qt-mt323.dll
 0002:00000e24       __imp_?mouseReleaseEvent@QButton@@MAEXPAVQMouseEvent@@@Z 10026e24     qt-mt323:qt-mt323.dll
 0002:00000e28       __imp_?mouseReleaseEvent@QComboBox@@MAEXPAVQMouseEvent@@@Z 10026e28     qt-mt323:qt-mt323.dll
 0002:00000e2c       __imp_?mouseReleaseEvent@QLineEdit@@MAEXPAVQMouseEvent@@@Z 10026e2c     qt-mt323:qt-mt323.dll
 0002:00000e30       __imp_?move@QPushButton@@UAEXHH@Z 10026e30     qt-mt323:qt-mt323.dll
 0002:00000e34       __imp_?paintEvent@QButton@@MAEXPAVQPaintEvent@@@Z 10026e34     qt-mt323:qt-mt323.dll
 0002:00000e38       __imp_?paintEvent@QComboBox@@MAEXPAVQPaintEvent@@@Z 10026e38     qt-mt323:qt-mt323.dll
 0002:00000e3c       __imp_?paintEvent@QGroupBox@@MAEXPAVQPaintEvent@@@Z 10026e3c     qt-mt323:qt-mt323.dll
 0002:00000e40       __imp_?paste@QLineEdit@@UAEXXZ 10026e40     qt-mt323:qt-mt323.dll
 0002:00000e44       __imp_?popup@QComboBox@@UAEXXZ 10026e44     qt-mt323:qt-mt323.dll
 0002:00000e48       __imp_?qt_cast@QCheckBox@@UAEPAXPBD@Z 10026e48     qt-mt323:qt-mt323.dll
 0002:00000e4c       __imp_?qt_cast@QComboBox@@UAEPAXPBD@Z 10026e4c     qt-mt323:qt-mt323.dll
 0002:00000e50       __imp_?qt_cast@QGridLayout@@UAEPAXPBD@Z 10026e50     qt-mt323:qt-mt323.dll
 0002:00000e54       __imp_?qt_cast@QGroupBox@@UAEPAXPBD@Z 10026e54     qt-mt323:qt-mt323.dll
 0002:00000e58       __imp_?qt_cast@QHBoxLayout@@UAEPAXPBD@Z 10026e58     qt-mt323:qt-mt323.dll
 0002:00000e5c       __imp_?qt_cast@QLabel@@UAEPAXPBD@Z 10026e5c     qt-mt323:qt-mt323.dll
 0002:00000e60       __imp_?qt_cast@QLineEdit@@UAEPAXPBD@Z 10026e60     qt-mt323:qt-mt323.dll
 0002:00000e64       __imp_?qt_cast@QPushButton@@UAEPAXPBD@Z 10026e64     qt-mt323:qt-mt323.dll
 0002:00000e68       __imp_?qt_cast@QVBoxLayout@@UAEPAXPBD@Z 10026e68     qt-mt323:qt-mt323.dll
 0002:00000e6c       __imp_?qt_emit@QCheckBox@@UAE_NHPAUQUObject@@@Z 10026e6c     qt-mt323:qt-mt323.dll
 0002:00000e70       __imp_?qt_emit@QComboBox@@UAE_NHPAUQUObject@@@Z 10026e70     qt-mt323:qt-mt323.dll
 0002:00000e74       __imp_?qt_emit@QGridLayout@@UAE_NHPAUQUObject@@@Z 10026e74     qt-mt323:qt-mt323.dll
 0002:00000e78       __imp_?qt_emit@QGroupBox@@UAE_NHPAUQUObject@@@Z 10026e78     qt-mt323:qt-mt323.dll
 0002:00000e7c       __imp_?qt_emit@QHBoxLayout@@UAE_NHPAUQUObject@@@Z 10026e7c     qt-mt323:qt-mt323.dll
 0002:00000e80       __imp_?qt_emit@QLabel@@UAE_NHPAUQUObject@@@Z 10026e80     qt-mt323:qt-mt323.dll
 0002:00000e84       __imp_?qt_emit@QLineEdit@@UAE_NHPAUQUObject@@@Z 10026e84     qt-mt323:qt-mt323.dll
 0002:00000e88       __imp_?qt_emit@QPushButton@@UAE_NHPAUQUObject@@@Z 10026e88     qt-mt323:qt-mt323.dll
 0002:00000e8c       __imp_?qt_emit@QVBoxLayout@@UAE_NHPAUQUObject@@@Z 10026e8c     qt-mt323:qt-mt323.dll
 0002:00000e90       __imp_?qt_invoke@QCheckBox@@UAE_NHPAUQUObject@@@Z 10026e90     qt-mt323:qt-mt323.dll
 0002:00000e94       __imp_?qt_invoke@QComboBox@@UAE_NHPAUQUObject@@@Z 10026e94     qt-mt323:qt-mt323.dll
 0002:00000e98       __imp_?qt_invoke@QGridLayout@@UAE_NHPAUQUObject@@@Z 10026e98     qt-mt323:qt-mt323.dll
 0002:00000e9c       __imp_?qt_invoke@QGroupBox@@UAE_NHPAUQUObject@@@Z 10026e9c     qt-mt323:qt-mt323.dll
 0002:00000ea0       __imp_?qt_invoke@QHBoxLayout@@UAE_NHPAUQUObject@@@Z 10026ea0     qt-mt323:qt-mt323.dll
 0002:00000ea4       __imp_?qt_invoke@QLabel@@UAE_NHPAUQUObject@@@Z 10026ea4     qt-mt323:qt-mt323.dll
 0002:00000ea8       __imp_?qt_invoke@QLineEdit@@UAE_NHPAUQUObject@@@Z 10026ea8     qt-mt323:qt-mt323.dll
 0002:00000eac       __imp_?qt_invoke@QPushButton@@UAE_NHPAUQUObject@@@Z 10026eac     qt-mt323:qt-mt323.dll
 0002:00000eb0       __imp_?qt_invoke@QVBoxLayout@@UAE_NHPAUQUObject@@@Z 10026eb0     qt-mt323:qt-mt323.dll
 0002:00000eb4       __imp_?qt_property@QCheckBox@@UAE_NHHPAVQVariant@@@Z 10026eb4     qt-mt323:qt-mt323.dll
 0002:00000eb8       __imp_?qt_property@QComboBox@@UAE_NHHPAVQVariant@@@Z 10026eb8     qt-mt323:qt-mt323.dll
 0002:00000ebc       __imp_?qt_property@QGridLayout@@UAE_NHHPAVQVariant@@@Z 10026ebc     qt-mt323:qt-mt323.dll
 0002:00000ec0       __imp_?qt_property@QGroupBox@@UAE_NHHPAVQVariant@@@Z 10026ec0     qt-mt323:qt-mt323.dll
 0002:00000ec4       __imp_?qt_property@QHBoxLayout@@UAE_NHHPAVQVariant@@@Z 10026ec4     qt-mt323:qt-mt323.dll
 0002:00000ec8       __imp_?qt_property@QLabel@@UAE_NHHPAVQVariant@@@Z 10026ec8     qt-mt323:qt-mt323.dll
 0002:00000ecc       __imp_?qt_property@QLineEdit@@UAE_NHHPAVQVariant@@@Z 10026ecc     qt-mt323:qt-mt323.dll
 0002:00000ed0       __imp_?qt_property@QPushButton@@UAE_NHHPAVQVariant@@@Z 10026ed0     qt-mt323:qt-mt323.dll
 0002:00000ed4       __imp_?qt_property@QVBoxLayout@@UAE_NHHPAVQVariant@@@Z 10026ed4     qt-mt323:qt-mt323.dll
 0002:00000ed8       __imp_?redo@QLineEdit@@UAEXXZ 10026ed8     qt-mt323:qt-mt323.dll
 0002:00000edc       __imp_?resize@QPushButton@@UAEXHH@Z 10026edc     qt-mt323:qt-mt323.dll
 0002:00000ee0       __imp_?resizeEvent@QCheckBox@@MAEXPAVQResizeEvent@@@Z 10026ee0     qt-mt323:qt-mt323.dll
 0002:00000ee4       __imp_?resizeEvent@QComboBox@@MAEXPAVQResizeEvent@@@Z 10026ee4     qt-mt323:qt-mt323.dll
 0002:00000ee8       __imp_?resizeEvent@QGroupBox@@MAEXPAVQResizeEvent@@@Z 10026ee8     qt-mt323:qt-mt323.dll
 0002:00000eec       __imp_?resizeEvent@QLabel@@MAEXPAVQResizeEvent@@@Z 10026eec     qt-mt323:qt-mt323.dll
 0002:00000ef0       __imp_?resizeEvent@QLineEdit@@MAEXPAVQResizeEvent@@@Z 10026ef0     qt-mt323:qt-mt323.dll
 0002:00000ef4       __imp_?resizeEvent@QPushButton@@MAEXPAVQResizeEvent@@@Z 10026ef4     qt-mt323:qt-mt323.dll
 0002:00000ef8       __imp_?selectAll@QLineEdit@@UAEXXZ 10026ef8     qt-mt323:qt-mt323.dll
 0002:00000efc       __imp_?setAccel@QButton@@UAEXABVQKeySequence@@@Z 10026efc     qt-mt323:qt-mt323.dll
 0002:00000f00       __imp_?setAlignment@QGroupBox@@UAEXH@Z 10026f00     qt-mt323:qt-mt323.dll
 0002:00000f04       __imp_?setAlignment@QLabel@@UAEXH@Z 10026f04     qt-mt323:qt-mt323.dll
 0002:00000f08       __imp_?setAlignment@QLineEdit@@UAEXH@Z 10026f08     qt-mt323:qt-mt323.dll
 0002:00000f0c       __imp_?setAutoCompletion@QComboBox@@UAEX_N@Z 10026f0c     qt-mt323:qt-mt323.dll
 0002:00000f10       __imp_?setAutoDefault@QPushButton@@UAEX_N@Z 10026f10     qt-mt323:qt-mt323.dll
 0002:00000f14       __imp_?setAutoRepeat@QButton@@UAEX_N@Z 10026f14     qt-mt323:qt-mt323.dll
 0002:00000f18       __imp_?setAutoResize@QComboBox@@UAEX_N@Z 10026f18     qt-mt323:qt-mt323.dll
 0002:00000f1c       __imp_?setAutoResize@QLabel@@UAEX_N@Z 10026f1c     qt-mt323:qt-mt323.dll
 0002:00000f20       __imp_?setBuddy@QLabel@@UAEXPAVQWidget@@@Z 10026f20     qt-mt323:qt-mt323.dll
 0002:00000f24       __imp_?setColStretch@QGridLayout@@UAEXHH@Z 10026f24     qt-mt323:qt-mt323.dll
 0002:00000f28       __imp_?setColumnLayout@QGroupBox@@UAEXHW4Orientation@Qt@@@Z 10026f28     qt-mt323:qt-mt323.dll
 0002:00000f2c       __imp_?setCurrentItem@QComboBox@@UAEXH@Z 10026f2c     qt-mt323:qt-mt323.dll
 0002:00000f30       __imp_?setCurrentText@QComboBox@@UAEXABVQString@@@Z 10026f30     qt-mt323:qt-mt323.dll
 0002:00000f34       __imp_?setCursorPosition@QLineEdit@@UAEXH@Z 10026f34     qt-mt323:qt-mt323.dll
 0002:00000f38       __imp_?setDefault@QPushButton@@UAEX_N@Z 10026f38     qt-mt323:qt-mt323.dll
 0002:00000f3c       __imp_?setDown@QButton@@UAEX_N@Z 10026f3c     qt-mt323:qt-mt323.dll
 0002:00000f40       __imp_?setDragEnabled@QLineEdit@@UAEX_N@Z 10026f40     qt-mt323:qt-mt323.dll
 0002:00000f44       __imp_?setEchoMode@QLineEdit@@UAEXW4EchoMode@1@@Z 10026f44     qt-mt323:qt-mt323.dll
 0002:00000f48       __imp_?setEditText@QComboBox@@UAEXABVQString@@@Z 10026f48     qt-mt323:qt-mt323.dll
 0002:00000f4c       __imp_?setEnabled@QComboBox@@UAEX_N@Z 10026f4c     qt-mt323:qt-mt323.dll
 0002:00000f50       __imp_?setEnabled@QGroupBox@@UAEX_N@Z 10026f50     qt-mt323:qt-mt323.dll
 0002:00000f54       __imp_?setFont@QComboBox@@UAEXABVQFont@@@Z 10026f54     qt-mt323:qt-mt323.dll
 0002:00000f58       __imp_?setFont@QLabel@@UAEXABVQFont@@@Z 10026f58     qt-mt323:qt-mt323.dll
 0002:00000f5c       __imp_?setFont@QLineEdit@@UAEXABVQFont@@@Z 10026f5c     qt-mt323:qt-mt323.dll
 0002:00000f60       __imp_?setFrame@QLineEdit@@UAEX_N@Z 10026f60     qt-mt323:qt-mt323.dll
 0002:00000f64       __imp_?setGeometry@QGridLayout@@UAEXABVQRect@@@Z 10026f64     qt-mt323:qt-mt323.dll
 0002:00000f68       __imp_?setGeometry@QPushButton@@UAEXABVQRect@@@Z 10026f68     qt-mt323:qt-mt323.dll
 0002:00000f6c       __imp_?setGeometry@QPushButton@@UAEXHHHH@Z 10026f6c     qt-mt323:qt-mt323.dll
 0002:00000f70       __imp_?setGeometry@QSpacerItem@@UAEXABVQRect@@@Z 10026f70     qt-mt323:qt-mt323.dll
 0002:00000f74       __imp_?setGroup@QButton@@EAEXPAVQButtonGroup@@@Z 10026f74     qt-mt323:qt-mt323.dll
 0002:00000f78       __imp_?setInsertionPolicy@QComboBox@@UAEXW4Policy@1@@Z 10026f78     qt-mt323:qt-mt323.dll
 0002:00000f7c       __imp_?setIsMenuButton@QPushButton@@UAEX_N@Z 10026f7c     qt-mt323:qt-mt323.dll
 0002:00000f80       __imp_?setLineEdit@QComboBox@@UAEXPAVQLineEdit@@@Z 10026f80     qt-mt323:qt-mt323.dll
 0002:00000f84       __imp_?setListBox@QComboBox@@UAEXPAVQListBox@@@Z 10026f84     qt-mt323:qt-mt323.dll
 0002:00000f88       __imp_?setMaxCount@QComboBox@@UAEXH@Z 10026f88     qt-mt323:qt-mt323.dll
 0002:00000f8c       __imp_?setMaxLength@QLineEdit@@UAEXH@Z 10026f8c     qt-mt323:qt-mt323.dll
 0002:00000f90       __imp_?setMovie@QLabel@@UAEXABVQMovie@@@Z 10026f90     qt-mt323:qt-mt323.dll
 0002:00000f94       __imp_?setNum@QLabel@@UAEXH@Z 10026f94     qt-mt323:qt-mt323.dll
 0002:00000f98       __imp_?setNum@QLabel@@UAEXN@Z 10026f98     qt-mt323:qt-mt323.dll
 0002:00000f9c       __imp_?setOn@QPushButton@@UAEX_N@Z 10026f9c     qt-mt323:qt-mt323.dll
 0002:00000fa0       __imp_?setPalette@QComboBox@@UAEXABVQPalette@@@Z 10026fa0     qt-mt323:qt-mt323.dll
 0002:00000fa4       __imp_?setPalette@QLineEdit@@UAEXABVQPalette@@@Z 10026fa4     qt-mt323:qt-mt323.dll
 0002:00000fa8       __imp_?setPicture@QLabel@@UAEXABVQPicture@@@Z 10026fa8     qt-mt323:qt-mt323.dll
 0002:00000fac       __imp_?setPixmap@QButton@@UAEXABVQPixmap@@@Z 10026fac     qt-mt323:qt-mt323.dll
 0002:00000fb0       __imp_?setPixmap@QLabel@@UAEXABVQPixmap@@@Z 10026fb0     qt-mt323:qt-mt323.dll
 0002:00000fb4       __imp_?setReadOnly@QLineEdit@@UAEX_N@Z 10026fb4     qt-mt323:qt-mt323.dll
 0002:00000fb8       __imp_?setRowStretch@QGridLayout@@UAEXHH@Z 10026fb8     qt-mt323:qt-mt323.dll
 0002:00000fbc       __imp_?setSelection@QLineEdit@@UAEXHH@Z 10026fbc     qt-mt323:qt-mt323.dll
 0002:00000fc0       __imp_?setSizeLimit@QComboBox@@UAEXH@Z 10026fc0     qt-mt323:qt-mt323.dll
 0002:00000fc4       __imp_?setState@QButton@@MAEXW4ToggleState@1@@Z 10026fc4     qt-mt323:qt-mt323.dll
 0002:00000fc8       __imp_?setText@QButton@@UAEXABVQString@@@Z 10026fc8     qt-mt323:qt-mt323.dll
 0002:00000fcc       __imp_?setText@QLabel@@UAEXABVQString@@@Z 10026fcc     qt-mt323:qt-mt323.dll
 0002:00000fd0       __imp_?setText@QLineEdit@@UAEXABVQString@@@Z 10026fd0     qt-mt323:qt-mt323.dll
 0002:00000fd4       __imp_?setTitle@QGroupBox@@UAEXABVQString@@@Z 10026fd4     qt-mt323:qt-mt323.dll
 0002:00000fd8       __imp_?setToggleType@QButton@@MAEXW4ToggleType@1@@Z 10026fd8     qt-mt323:qt-mt323.dll
 0002:00000fdc       __imp_?setValidator@QComboBox@@UAEXPBVQValidator@@@Z 10026fdc     qt-mt323:qt-mt323.dll
 0002:00000fe0       __imp_?setValidator@QLineEdit@@UAEXPBVQValidator@@@Z 10026fe0     qt-mt323:qt-mt323.dll
 0002:00000fe4       __imp_?sizeHint@QCheckBox@@UBE?AVQSize@@XZ 10026fe4     qt-mt323:qt-mt323.dll
 0002:00000fe8       __imp_?sizeHint@QComboBox@@UBE?AVQSize@@XZ 10026fe8     qt-mt323:qt-mt323.dll
 0002:00000fec       __imp_?sizeHint@QGridLayout@@UBE?AVQSize@@XZ 10026fec     qt-mt323:qt-mt323.dll
 0002:00000ff0       __imp_?sizeHint@QGroupBox@@UBE?AVQSize@@XZ 10026ff0     qt-mt323:qt-mt323.dll
 0002:00000ff4       __imp_?sizeHint@QLabel@@UBE?AVQSize@@XZ 10026ff4     qt-mt323:qt-mt323.dll
 0002:00000ff8       __imp_?sizeHint@QLineEdit@@UBE?AVQSize@@XZ 10026ff8     qt-mt323:qt-mt323.dll
 0002:00000ffc       __imp_?sizeHint@QPushButton@@UBE?AVQSize@@XZ 10026ffc     qt-mt323:qt-mt323.dll
 0002:00001000       __imp_?sizeHint@QSpacerItem@@UBE?AVQSize@@XZ 10027000     qt-mt323:qt-mt323.dll
 0002:00001004       __imp_?spacerItem@QSpacerItem@@UAEPAV1@XZ 10027004     qt-mt323:qt-mt323.dll
 0002:00001008       __imp_?styleChange@QComboBox@@MAEXAAVQStyle@@@Z 10027008     qt-mt323:qt-mt323.dll
 0002:0000100c       __imp_?undo@QLineEdit@@UAEXXZ 1002700c     qt-mt323:qt-mt323.dll
 0002:00001010       __imp_?updateMask@QCheckBox@@MAEXXZ 10027010     qt-mt323:qt-mt323.dll
 0002:00001014       __imp_?updateMask@QComboBox@@MAEXXZ 10027014     qt-mt323:qt-mt323.dll
 0002:00001018       __imp_?updateMask@QPushButton@@MAEXXZ 10027018     qt-mt323:qt-mt323.dll
 0002:0000101c       __imp_?wheelEvent@QComboBox@@MAEXPAVQWheelEvent@@@Z 1002701c     qt-mt323:qt-mt323.dll
 0002:00001020       __imp_?windowActivationChange@QLineEdit@@MAEX_N@Z 10027020     qt-mt323:qt-mt323.dll
 0002:00001024       __imp_??1QFont@@QAE@XZ     10027024     qt-mt323:qt-mt323.dll
 0002:00001028       __imp_?setMinimumSize@QWidget@@QAEXABVQSize@@@Z 10027028     qt-mt323:qt-mt323.dll
 0002:0000102c       __imp_?setMaximumSize@QWidget@@QAEXABVQSize@@@Z 1002702c     qt-mt323:qt-mt323.dll
 0002:00001030       __imp_?font@QWidget@@QBE?AVQFont@@XZ 10027030     qt-mt323:qt-mt323.dll
 0002:00001034       __imp_?resize@QWidget@@QAEXABVQSize@@@Z 10027034     qt-mt323:qt-mt323.dll
 0002:00001038       __imp_?changeTab@QTabWidget@@QAEXPAVQWidget@@ABVQString@@@Z 10027038     qt-mt323:qt-mt323.dll
 0002:0000103c       __imp_?setDuplicatesEnabled@QComboBox@@QAEX_N@Z 1002703c     qt-mt323:qt-mt323.dll
 0002:00001040       __imp_?setEditable@QComboBox@@QAEX_N@Z 10027040     qt-mt323:qt-mt323.dll
 0002:00001044       __imp_??0QSpinBox@@QAE@PAVQWidget@@PBD@Z 10027044     qt-mt323:qt-mt323.dll
 0002:00001048       __imp_??1QSpinBox@@UAE@XZ  10027048     qt-mt323:qt-mt323.dll
 0002:0000104c       __imp_?setMinValue@QSpinBox@@QAEXH@Z 1002704c     qt-mt323:qt-mt323.dll
 0002:00001050       __imp_??0QButtonGroup@@QAE@PAVQWidget@@PBD@Z 10027050     qt-mt323:qt-mt323.dll
 0002:00001054       __imp_??1QButtonGroup@@UAE@XZ 10027054     qt-mt323:qt-mt323.dll
 0002:00001058       __imp_??0QSplitter@@QAE@PAVQWidget@@PBD@Z 10027058     qt-mt323:qt-mt323.dll
 0002:0000105c       __imp_??1QSplitter@@UAE@XZ 1002705c     qt-mt323:qt-mt323.dll
 0002:00001060       __imp_?header@QListView@@QBEPAVQHeader@@XZ 10027060     qt-mt323:qt-mt323.dll
 0002:00001064       __imp_??0QRadioButton@@QAE@PAVQWidget@@PBD@Z 10027064     qt-mt323:qt-mt323.dll
 0002:00001068       __imp_??0QDateEdit@@QAE@PAVQWidget@@PBD@Z 10027068     qt-mt323:qt-mt323.dll
 0002:0000106c       __imp_??1QDateEdit@@UAE@XZ 1002706c     qt-mt323:qt-mt323.dll
 0002:00001070       __imp_??0QDataTable@@QAE@PAVQWidget@@PBD@Z 10027070     qt-mt323:qt-mt323.dll
 0002:00001074       __imp_??1QDataTable@@UAE@XZ 10027074     qt-mt323:qt-mt323.dll
 0002:00001078       __imp_??0QGridLayout@@QAE@PAVQWidget@@HHHHPBD@Z 10027078     qt-mt323:qt-mt323.dll
 0002:0000107c       __imp_?addMultiCell@QGridLayout@@QAEXPAVQLayoutItem@@HHHHH@Z 1002707c     qt-mt323:qt-mt323.dll
 0002:00001080       __imp_?addLayout@QGridLayout@@QAEXPAVQLayout@@HH@Z 10027080     qt-mt323:qt-mt323.dll
 0002:00001084       __imp_?addMultiCellLayout@QGridLayout@@QAEXPAVQLayout@@HHHHH@Z 10027084     qt-mt323:qt-mt323.dll
 0002:00001088       __imp_??0QHBoxLayout@@QAE@PAVQLayout@@HPBD@Z 10027088     qt-mt323:qt-mt323.dll
 0002:0000108c       __imp_??0QVBoxLayout@@QAE@PAVQLayout@@HPBD@Z 1002708c     qt-mt323:qt-mt323.dll
 0002:00001090       __imp_?activateNextCell@QDataTable@@MAEXXZ 10027090     qt-mt323:qt-mt323.dll
 0002:00001094       __imp_?addColumn@QDataTable@@UAEXABVQString@@0HABVQIconSet@@@Z 10027094     qt-mt323:qt-mt323.dll
 0002:00001098       __imp_?addNumber@QDateEdit@@MAEXHH@Z 10027098     qt-mt323:qt-mt323.dll
 0002:0000109c       __imp_?addSelection@QTable@@UAEHABVQTableSelection@@@Z 1002709c     qt-mt323:qt-mt323.dll
 0002:000010a0       __imp_?adjustColumn@QDataTable@@UAEXH@Z 100270a0     qt-mt323:qt-mt323.dll
 0002:000010a4       __imp_?adjustRow@QTable@@UAEXH@Z 100270a4     qt-mt323:qt-mt323.dll
 0002:000010a8       __imp_?beginEdit@QDataTable@@EAEPAVQWidget@@HH_N@Z 100270a8     qt-mt323:qt-mt323.dll
 0002:000010ac       __imp_?beginInsert@QDataTable@@MAE_NXZ 100270ac     qt-mt323:qt-mt323.dll
 0002:000010b0       __imp_?beginUpdate@QDataTable@@MAEPAVQWidget@@HH_N@Z 100270b0     qt-mt323:qt-mt323.dll
 0002:000010b4       __imp_?cellGeometry@QTable@@UBE?AVQRect@@HH@Z 100270b4     qt-mt323:qt-mt323.dll
 0002:000010b8       __imp_?cellRect@QTable@@UBE?AVQRect@@HH@Z 100270b8     qt-mt323:qt-mt323.dll
 0002:000010bc       __imp_?cellWidget@QTable@@UBEPAVQWidget@@HH@Z 100270bc     qt-mt323:qt-mt323.dll
 0002:000010c0       __imp_?childEvent@QSplitter@@MAEXPAVQChildEvent@@@Z 100270c0     qt-mt323:qt-mt323.dll
 0002:000010c4       __imp_?className@QButtonGroup@@UBEPBDXZ 100270c4     qt-mt323:qt-mt323.dll
 0002:000010c8       __imp_?className@QDataTable@@UBEPBDXZ 100270c8     qt-mt323:qt-mt323.dll
 0002:000010cc       __imp_?className@QDateEdit@@UBEPBDXZ 100270cc     qt-mt323:qt-mt323.dll
 0002:000010d0       __imp_?className@QRadioButton@@UBEPBDXZ 100270d0     qt-mt323:qt-mt323.dll
 0002:000010d4       __imp_?className@QSpinBox@@UBEPBDXZ 100270d4     qt-mt323:qt-mt323.dll
 0002:000010d8       __imp_?className@QSplitter@@UBEPBDXZ 100270d8     qt-mt323:qt-mt323.dll
 0002:000010dc       __imp_?cleanText@QSpinBox@@UBE?AVQString@@XZ 100270dc     qt-mt323:qt-mt323.dll
 0002:000010e0       __imp_?clearCell@QDataTable@@MAEXHH@Z 100270e0     qt-mt323:qt-mt323.dll
 0002:000010e4       __imp_?clearCellWidget@QTable@@UAEXHH@Z 100270e4     qt-mt323:qt-mt323.dll
 0002:000010e8       __imp_?columnAt@QTable@@UBEHH@Z 100270e8     qt-mt323:qt-mt323.dll
 0002:000010ec       __imp_?columnClicked@QDataTable@@MAEXH@Z 100270ec     qt-mt323:qt-mt323.dll
 0002:000010f0       __imp_?columnIndexChanged@QTable@@MAEXHHH@Z 100270f0     qt-mt323:qt-mt323.dll
 0002:000010f4       __imp_?columnPos@QTable@@UBEHH@Z 100270f4     qt-mt323:qt-mt323.dll
 0002:000010f8       __imp_?columnWidth@QTable@@UBEHH@Z 100270f8     qt-mt323:qt-mt323.dll
 0002:000010fc       __imp_?columnWidthChanged@QTable@@MAEXH@Z 100270fc     qt-mt323:qt-mt323.dll
 0002:00001100       __imp_?confirmCancel@QDataTable@@MAE?AW4Confirm@QSql@@W4Op@3@@Z 10027100     qt-mt323:qt-mt323.dll
 0002:00001104       __imp_?confirmEdit@QDataTable@@MAE?AW4Confirm@QSql@@W4Op@3@@Z 10027104     qt-mt323:qt-mt323.dll
 0002:00001108       __imp_?contentsContextMenuEvent@QDataTable@@MAEXPAVQContextMenuEvent@@@Z 10027108     qt-mt323:qt-mt323.dll
 0002:0000110c       __imp_?contentsDragEnterEvent@QTable@@MAEXPAVQDragEnterEvent@@@Z 1002710c     qt-mt323:qt-mt323.dll
 0002:00001110       __imp_?contentsDragLeaveEvent@QTable@@MAEXPAVQDragLeaveEvent@@@Z 10027110     qt-mt323:qt-mt323.dll
 0002:00001114       __imp_?contentsDragMoveEvent@QTable@@MAEXPAVQDragMoveEvent@@@Z 10027114     qt-mt323:qt-mt323.dll
 0002:00001118       __imp_?contentsDropEvent@QTable@@MAEXPAVQDropEvent@@@Z 10027118     qt-mt323:qt-mt323.dll
 0002:0000111c       __imp_?contentsMouseDoubleClickEvent@QTable@@MAEXPAVQMouseEvent@@@Z 1002711c     qt-mt323:qt-mt323.dll
 0002:00001120       __imp_?contentsMouseMoveEvent@QTable@@MAEXPAVQMouseEvent@@@Z 10027120     qt-mt323:qt-mt323.dll
 0002:00001124       __imp_?contentsMousePressEvent@QDataTable@@MAEXPAVQMouseEvent@@@Z 10027124     qt-mt323:qt-mt323.dll
 0002:00001128       __imp_?contentsMouseReleaseEvent@QTable@@MAEXPAVQMouseEvent@@@Z 10027128     qt-mt323:qt-mt323.dll
 0002:0000112c       __imp_?createEditor@QDataTable@@MBEPAVQWidget@@HH_N@Z 1002712c     qt-mt323:qt-mt323.dll
 0002:00001130       __imp_?currentSelection@QTable@@UBEHXZ 10027130     qt-mt323:qt-mt323.dll
 0002:00001134       __imp_?deleteCurrent@QDataTable@@MAE_NXZ 10027134     qt-mt323:qt-mt323.dll
 0002:00001138       __imp_?dragObject@QTable@@MAEPAVQDragObject@@XZ 10027138     qt-mt323:qt-mt323.dll
 0002:0000113c       __imp_?drawButton@QRadioButton@@MAEXPAVQPainter@@@Z 1002713c     qt-mt323:qt-mt323.dll
 0002:00001140       __imp_?drawButtonLabel@QRadioButton@@MAEXPAVQPainter@@@Z 10027140     qt-mt323:qt-mt323.dll
 0002:00001144       __imp_?drawContents@QDataTable@@MAEXPAVQPainter@@HHHH@Z 10027144     qt-mt323:qt-mt323.dll
 0002:00001148       __imp_?drawContents@QTable@@EAEXPAVQPainter@@@Z 10027148     qt-mt323:qt-mt323.dll
 0002:0000114c       __imp_?drawContentsOffset@QScrollView@@MAEXPAVQPainter@@HHHHHH@Z 1002714c     qt-mt323:qt-mt323.dll
 0002:00001150       __imp_?drawSplitter@QSplitter@@MAEXPAVQPainter@@HHHH@Z 10027150     qt-mt323:qt-mt323.dll
 0002:00001154       __imp_?editCell@QTable@@UAEXHH_N@Z 10027154     qt-mt323:qt-mt323.dll
 0002:00001158       __imp_?endEdit@QDataTable@@MAEXHH_N0@Z 10027158     qt-mt323:qt-mt323.dll
 0002:0000115c       __imp_?event@QButtonGroup@@MAE_NPAVQEvent@@@Z 1002715c     qt-mt323:qt-mt323.dll
 0002:00001160       __imp_?event@QDateEdit@@MAE_NPAVQEvent@@@Z 10027160     qt-mt323:qt-mt323.dll
 0002:00001164       __imp_?event@QSplitter@@MAE_NPAVQEvent@@@Z 10027164     qt-mt323:qt-mt323.dll
 0002:00001168       __imp_?eventFilter@QDataTable@@MAE_NPAVQObject@@PAVQEvent@@@Z 10027168     qt-mt323:qt-mt323.dll
 0002:0000116c       __imp_?eventFilter@QSpinBox@@MAE_NPAVQObject@@PAVQEvent@@@Z 1002716c     qt-mt323:qt-mt323.dll
 0002:00001170       __imp_?fieldAlignment@QDataTable@@MAEHPBVQSqlField@@@Z 10027170     qt-mt323:qt-mt323.dll
 0002:00001174       __imp_?find@QDataTable@@UAEXABVQString@@_N1@Z 10027174     qt-mt323:qt-mt323.dll
 0002:00001178       __imp_?fix@QDateEdit@@MAEXXZ 10027178     qt-mt323:qt-mt323.dll
 0002:0000117c       __imp_?focusInEvent@QTable@@MAEXPAVQFocusEvent@@@Z 1002717c     qt-mt323:qt-mt323.dll
 0002:00001180       __imp_?focusOutEvent@QTable@@MAEXPAVQFocusEvent@@@Z 10027180     qt-mt323:qt-mt323.dll
 0002:00001184       __imp_?handleError@QDataTable@@MAEXABVQSqlError@@@Z 10027184     qt-mt323:qt-mt323.dll
 0002:00001188       __imp_?hideColumn@QDataTable@@UAEXH@Z 10027188     qt-mt323:qt-mt323.dll
 0002:0000118c       __imp_?hideRow@QTable@@UAEXH@Z 1002718c     qt-mt323:qt-mt323.dll
 0002:00001190       __imp_?hitButton@QRadioButton@@MBE_NABVQPoint@@@Z 10027190     qt-mt323:qt-mt323.dll
 0002:00001194       __imp_?insertColumns@QTable@@UAEXHH@Z 10027194     qt-mt323:qt-mt323.dll
 0002:00001198       __imp_?insertCurrent@QDataTable@@MAE_NXZ 10027198     qt-mt323:qt-mt323.dll
 0002:0000119c       __imp_?insertRows@QTable@@UAEXHH@Z 1002719c     qt-mt323:qt-mt323.dll
 0002:000011a0       __imp_?insertWidget@QTable@@MAEXHHPAVQWidget@@@Z 100271a0     qt-mt323:qt-mt323.dll
 0002:000011a4       __imp_?interpretText@QSpinBox@@MAEXXZ 100271a4     qt-mt323:qt-mt323.dll
 0002:000011a8       __imp_?item@QDataTable@@MBEPAVQTableItem@@HH@Z 100271a8     qt-mt323:qt-mt323.dll
 0002:000011ac       __imp_?keyPressEvent@QDataTable@@MAEXPAVQKeyEvent@@@Z 100271ac     qt-mt323:qt-mt323.dll
 0002:000011b0       __imp_?leaveEvent@QSpinBox@@MAEXPAVQEvent@@@Z 100271b0     qt-mt323:qt-mt323.dll
 0002:000011b4       __imp_?mapTextToValue@QSpinBox@@MAEHPA_N@Z 100271b4     qt-mt323:qt-mt323.dll
 0002:000011b8       __imp_?mapValueToText@QSpinBox@@MAE?AVQString@@H@Z 100271b8     qt-mt323:qt-mt323.dll
 0002:000011bc       __imp_?metaObject@QButtonGroup@@UBEPAVQMetaObject@@XZ 100271bc     qt-mt323:qt-mt323.dll
 0002:000011c0       __imp_?metaObject@QDataTable@@UBEPAVQMetaObject@@XZ 100271c0     qt-mt323:qt-mt323.dll
 0002:000011c4       __imp_?metaObject@QDateEdit@@UBEPAVQMetaObject@@XZ 100271c4     qt-mt323:qt-mt323.dll
 0002:000011c8       __imp_?metaObject@QRadioButton@@UBEPAVQMetaObject@@XZ 100271c8     qt-mt323:qt-mt323.dll
 0002:000011cc       __imp_?metaObject@QSpinBox@@UBEPAVQMetaObject@@XZ 100271cc     qt-mt323:qt-mt323.dll
 0002:000011d0       __imp_?metaObject@QSplitter@@UBEPAVQMetaObject@@XZ 100271d0     qt-mt323:qt-mt323.dll
 0002:000011d4       __imp_?minimumSizeHint@QDateEdit@@UBE?AVQSize@@XZ 100271d4     qt-mt323:qt-mt323.dll
 0002:000011d8       __imp_?minimumSizeHint@QScrollView@@UBE?AVQSize@@XZ 100271d8     qt-mt323:qt-mt323.dll
 0002:000011dc       __imp_?minimumSizeHint@QSpinBox@@UBE?AVQSize@@XZ 100271dc     qt-mt323:qt-mt323.dll
 0002:000011e0       __imp_?minimumSizeHint@QSplitter@@UBE?AVQSize@@XZ 100271e0     qt-mt323:qt-mt323.dll
 0002:000011e4       __imp_?moveFocus@QButtonGroup@@UAEXH@Z 100271e4     qt-mt323:qt-mt323.dll
 0002:000011e8       __imp_?numCols@QDataTable@@UBEHXZ 100271e8     qt-mt323:qt-mt323.dll
 0002:000011ec       __imp_?numRows@QDataTable@@UBEHXZ 100271ec     qt-mt323:qt-mt323.dll
 0002:000011f0       __imp_?outOfRange@QDateEdit@@MBE_NHHH@Z 100271f0     qt-mt323:qt-mt323.dll
 0002:000011f4       __imp_?paintCell@QDataTable@@MAEXPAVQPainter@@HHABVQRect@@_NABVQColorGroup@@@Z 100271f4     qt-mt323:qt-mt323.dll
 0002:000011f8       __imp_?paintCell@QTable@@UAEXPAVQPainter@@HHABVQRect@@_N@Z 100271f8     qt-mt323:qt-mt323.dll
 0002:000011fc       __imp_?paintEmptyArea@QTable@@MAEXPAVQPainter@@HHHH@Z 100271fc     qt-mt323:qt-mt323.dll
 0002:00001200       __imp_?paintEvent@QTable@@MAEXPAVQPaintEvent@@@Z 10027200     qt-mt323:qt-mt323.dll
 0002:00001204       __imp_?paintField@QDataTable@@MAEXPAVQPainter@@PBVQSqlField@@ABVQRect@@_N@Z 10027204     qt-mt323:qt-mt323.dll
 0002:00001208       __imp_?paintFocus@QTable@@UAEXPAVQPainter@@ABVQRect@@@Z 10027208     qt-mt323:qt-mt323.dll
 0002:0000120c       __imp_?pixmap@QTable@@UBE?AVQPixmap@@HH@Z 1002720c     qt-mt323:qt-mt323.dll
 0002:00001210       __imp_?prefix@QSpinBox@@UBE?AVQString@@XZ 10027210     qt-mt323:qt-mt323.dll
 0002:00001214       __imp_?qt_cast@QButtonGroup@@UAEPAXPBD@Z 10027214     qt-mt323:qt-mt323.dll
 0002:00001218       __imp_?qt_cast@QDataTable@@UAEPAXPBD@Z 10027218     qt-mt323:qt-mt323.dll
 0002:0000121c       __imp_?qt_cast@QDateEdit@@UAEPAXPBD@Z 1002721c     qt-mt323:qt-mt323.dll
 0002:00001220       __imp_?qt_cast@QRadioButton@@UAEPAXPBD@Z 10027220     qt-mt323:qt-mt323.dll
 0002:00001224       __imp_?qt_cast@QSpinBox@@UAEPAXPBD@Z 10027224     qt-mt323:qt-mt323.dll
 0002:00001228       __imp_?qt_cast@QSplitter@@UAEPAXPBD@Z 10027228     qt-mt323:qt-mt323.dll
 0002:0000122c       __imp_?qt_emit@QButtonGroup@@UAE_NHPAUQUObject@@@Z 1002722c     qt-mt323:qt-mt323.dll
 0002:00001230       __imp_?qt_emit@QDataTable@@UAE_NHPAUQUObject@@@Z 10027230     qt-mt323:qt-mt323.dll
 0002:00001234       __imp_?qt_emit@QDateEdit@@UAE_NHPAUQUObject@@@Z 10027234     qt-mt323:qt-mt323.dll
 0002:00001238       __imp_?qt_emit@QRadioButton@@UAE_NHPAUQUObject@@@Z 10027238     qt-mt323:qt-mt323.dll
 0002:0000123c       __imp_?qt_emit@QSpinBox@@UAE_NHPAUQUObject@@@Z 1002723c     qt-mt323:qt-mt323.dll
 0002:00001240       __imp_?qt_emit@QSplitter@@UAE_NHPAUQUObject@@@Z 10027240     qt-mt323:qt-mt323.dll
 0002:00001244       __imp_?qt_invoke@QButtonGroup@@UAE_NHPAUQUObject@@@Z 10027244     qt-mt323:qt-mt323.dll
 0002:00001248       __imp_?qt_invoke@QDataTable@@UAE_NHPAUQUObject@@@Z 10027248     qt-mt323:qt-mt323.dll
 0002:0000124c       __imp_?qt_invoke@QDateEdit@@UAE_NHPAUQUObject@@@Z 1002724c     qt-mt323:qt-mt323.dll
 0002:00001250       __imp_?qt_invoke@QRadioButton@@UAE_NHPAUQUObject@@@Z 10027250     qt-mt323:qt-mt323.dll
 0002:00001254       __imp_?qt_invoke@QSpinBox@@UAE_NHPAUQUObject@@@Z 10027254     qt-mt323:qt-mt323.dll
 0002:00001258       __imp_?qt_invoke@QSplitter@@UAE_NHPAUQUObject@@@Z 10027258     qt-mt323:qt-mt323.dll
 0002:0000125c       __imp_?qt_property@QButtonGroup@@UAE_NHHPAVQVariant@@@Z 1002725c     qt-mt323:qt-mt323.dll
 0002:00001260       __imp_?qt_property@QDataTable@@UAE_NHHPAVQVariant@@@Z 10027260     qt-mt323:qt-mt323.dll
 0002:00001264       __imp_?qt_property@QDateEdit@@UAE_NHHPAVQVariant@@@Z 10027264     qt-mt323:qt-mt323.dll
 0002:00001268       __imp_?qt_property@QRadioButton@@UAE_NHHPAVQVariant@@@Z 10027268     qt-mt323:qt-mt323.dll
 0002:0000126c       __imp_?qt_property@QSpinBox@@UAE_NHHPAVQVariant@@@Z 1002726c     qt-mt323:qt-mt323.dll
 0002:00001270       __imp_?qt_property@QSplitter@@UAE_NHHPAVQVariant@@@Z 10027270     qt-mt323:qt-mt323.dll
 0002:00001274       __imp_?rangeChange@QSpinBox@@MAEXXZ 10027274     qt-mt323:qt-mt323.dll
 0002:00001278       __imp_?refresh@QDataTable@@UAEXXZ 10027278     qt-mt323:qt-mt323.dll
 0002:0000127c       __imp_?removeColumn@QDataTable@@UAEXI@Z 1002727c     qt-mt323:qt-mt323.dll
 0002:00001280       __imp_?removeColumn@QTable@@UAEXH@Z 10027280     qt-mt323:qt-mt323.dll
 0002:00001284       __imp_?removeColumns@QTable@@UAEXABV?$QMemArray@H@@@Z 10027284     qt-mt323:qt-mt323.dll
 0002:00001288       __imp_?removeLastNumber@QDateEdit@@MAEXH@Z 10027288     qt-mt323:qt-mt323.dll
 0002:0000128c       __imp_?removeRow@QTable@@UAEXH@Z 1002728c     qt-mt323:qt-mt323.dll
 0002:00001290       __imp_?removeRows@QTable@@UAEXABV?$QMemArray@H@@@Z 10027290     qt-mt323:qt-mt323.dll
 0002:00001294       __imp_?removeSelection@QTable@@UAEXABVQTableSelection@@@Z 10027294     qt-mt323:qt-mt323.dll
 0002:00001298       __imp_?removeSelection@QTable@@UAEXH@Z 10027298     qt-mt323:qt-mt323.dll
 0002:0000129c       __imp_?resizeData@QDataTable@@MAEXH@Z 1002729c     qt-mt323:qt-mt323.dll
 0002:000012a0       __imp_?resizeEvent@QDataTable@@MAEXPAVQResizeEvent@@@Z 100272a0     qt-mt323:qt-mt323.dll
 0002:000012a4       __imp_?resizeEvent@QDateEdit@@MAEXPAVQResizeEvent@@@Z 100272a4     qt-mt323:qt-mt323.dll
 0002:000012a8       __imp_?resizeEvent@QRadioButton@@MAEXPAVQResizeEvent@@@Z 100272a8     qt-mt323:qt-mt323.dll
 0002:000012ac       __imp_?resizeEvent@QSpinBox@@MAEXPAVQResizeEvent@@@Z 100272ac     qt-mt323:qt-mt323.dll
 0002:000012b0       __imp_?resizeEvent@QSplitter@@MAEXPAVQResizeEvent@@@Z 100272b0     qt-mt323:qt-mt323.dll
 0002:000012b4       __imp_?rowAt@QTable@@UBEHH@Z 100272b4     qt-mt323:qt-mt323.dll
 0002:000012b8       __imp_?rowHeight@QTable@@UBEHH@Z 100272b8     qt-mt323:qt-mt323.dll
 0002:000012bc       __imp_?rowHeightChanged@QTable@@MAEXH@Z 100272bc     qt-mt323:qt-mt323.dll
 0002:000012c0       __imp_?rowIndexChanged@QTable@@MAEXHHH@Z 100272c0     qt-mt323:qt-mt323.dll
 0002:000012c4       __imp_?rowPos@QTable@@UBEHH@Z 100272c4     qt-mt323:qt-mt323.dll
 0002:000012c8       __imp_?sectionFormattedText@QDateEdit@@MAE?AVQString@@H@Z 100272c8     qt-mt323:qt-mt323.dll
 0002:000012cc       __imp_?selectAll@QSpinBox@@UAEXXZ 100272cc     qt-mt323:qt-mt323.dll
 0002:000012d0       __imp_?setAutoAdvance@QDateEdit@@UAEX_N@Z 100272d0     qt-mt323:qt-mt323.dll
 0002:000012d4       __imp_?setAutoDelete@QDataTable@@UAEX_N@Z 100272d4     qt-mt323:qt-mt323.dll
 0002:000012d8       __imp_?setAutoEdit@QDataTable@@UAEX_N@Z 100272d8     qt-mt323:qt-mt323.dll
 0002:000012dc       __imp_?setButton@QButtonGroup@@UAEXH@Z 100272dc     qt-mt323:qt-mt323.dll
 0002:000012e0       __imp_?setButtonSymbols@QSpinBox@@UAEXW4ButtonSymbols@1@@Z 100272e0     qt-mt323:qt-mt323.dll
 0002:000012e4       __imp_?setCellContentFromEditor@QTable@@MAEXHH@Z 100272e4     qt-mt323:qt-mt323.dll
 0002:000012e8       __imp_?setCellWidget@QTable@@UAEXHHPAVQWidget@@@Z 100272e8     qt-mt323:qt-mt323.dll
 0002:000012ec       __imp_?setChecked@QRadioButton@@UAEX_N@Z 100272ec     qt-mt323:qt-mt323.dll
 0002:000012f0       __imp_?setColumn@QDataTable@@UAEXIABVQString@@0HABVQIconSet@@@Z 100272f0     qt-mt323:qt-mt323.dll
 0002:000012f4       __imp_?setColumnMovingEnabled@QTable@@UAEX_N@Z 100272f4     qt-mt323:qt-mt323.dll
 0002:000012f8       __imp_?setColumnReadOnly@QTable@@UAEXH_N@Z 100272f8     qt-mt323:qt-mt323.dll
 0002:000012fc       __imp_?setColumnStretchable@QDataTable@@UAEXH_N@Z 100272fc     qt-mt323:qt-mt323.dll
 0002:00001300       __imp_?setColumnWidth@QDataTable@@UAEXHH@Z 10027300     qt-mt323:qt-mt323.dll
 0002:00001304       __imp_?setConfirmCancels@QDataTable@@UAEX_N@Z 10027304     qt-mt323:qt-mt323.dll
 0002:00001308       __imp_?setConfirmDelete@QDataTable@@UAEX_N@Z 10027308     qt-mt323:qt-mt323.dll
 0002:0000130c       __imp_?setConfirmEdits@QDataTable@@UAEX_N@Z 1002730c     qt-mt323:qt-mt323.dll
 0002:00001310       __imp_?setConfirmInsert@QDataTable@@UAEX_N@Z 10027310     qt-mt323:qt-mt323.dll
 0002:00001314       __imp_?setConfirmUpdate@QDataTable@@UAEX_N@Z 10027314     qt-mt323:qt-mt323.dll
 0002:00001318       __imp_?setContentsPos@QScrollView@@UAEXHH@Z 10027318     qt-mt323:qt-mt323.dll
 0002:0000131c       __imp_?setCurrentCell@QTable@@UAEXHH@Z 1002731c     qt-mt323:qt-mt323.dll
 0002:00001320       __imp_?setDate@QDateEdit@@UAEXABVQDate@@@Z 10027320     qt-mt323:qt-mt323.dll
 0002:00001324       __imp_?setDateFormat@QDataTable@@UAEXW4DateFormat@Qt@@@Z 10027324     qt-mt323:qt-mt323.dll
 0002:00001328       __imp_?setDay@QDateEdit@@MAEXH@Z 10027328     qt-mt323:qt-mt323.dll
 0002:0000132c       __imp_?setDragEnabled@QTable@@UAEX_N@Z 1002732c     qt-mt323:qt-mt323.dll
 0002:00001330       __imp_?setEnabled@QSpinBox@@UAEX_N@Z 10027330     qt-mt323:qt-mt323.dll
 0002:00001334       __imp_?setEnabled@QTable@@UAEX_N@Z 10027334     qt-mt323:qt-mt323.dll
 0002:00001338       __imp_?setExclusive@QButtonGroup@@UAEX_N@Z 10027338     qt-mt323:qt-mt323.dll
 0002:0000133c       __imp_?setFalseText@QDataTable@@UAEXABVQString@@@Z 1002733c     qt-mt323:qt-mt323.dll
 0002:00001340       __imp_?setFilter@QDataTable@@UAEXABVQString@@@Z 10027340     qt-mt323:qt-mt323.dll
 0002:00001344       __imp_?setFocusSection@QDateEdit@@MAE_NH@Z 10027344     qt-mt323:qt-mt323.dll
 0002:00001348       __imp_?setFocusStyle@QTable@@UAEXW4FocusStyle@1@@Z 10027348     qt-mt323:qt-mt323.dll
 0002:0000134c       __imp_?setItem@QDataTable@@MAEXHHPAVQTableItem@@@Z 1002734c     qt-mt323:qt-mt323.dll
 0002:00001350       __imp_?setLeftMargin@QTable@@UAEXH@Z 10027350     qt-mt323:qt-mt323.dll
 0002:00001354       __imp_?setMaxValue@QDateEdit@@UAEXABVQDate@@@Z 10027354     qt-mt323:qt-mt323.dll
 0002:00001358       __imp_?setMinValue@QDateEdit@@UAEXABVQDate@@@Z 10027358     qt-mt323:qt-mt323.dll
 0002:0000135c       __imp_?setMonth@QDateEdit@@MAEXH@Z 1002735c     qt-mt323:qt-mt323.dll
 0002:00001360       __imp_?setNullText@QDataTable@@UAEXABVQString@@@Z 10027360     qt-mt323:qt-mt323.dll
 0002:00001364       __imp_?setNumCols@QDataTable@@UAEXH@Z 10027364     qt-mt323:qt-mt323.dll
 0002:00001368       __imp_?setNumRows@QDataTable@@UAEXH@Z 10027368     qt-mt323:qt-mt323.dll
 0002:0000136c       __imp_?setOpaqueResize@QSplitter@@UAEX_N@Z 1002736c     qt-mt323:qt-mt323.dll
 0002:00001370       __imp_?setOrder@QDateEdit@@UAEXW4Order@1@@Z 10027370     qt-mt323:qt-mt323.dll
 0002:00001374       __imp_?setOrientation@QSplitter@@UAEXW4Orientation@Qt@@@Z 10027374     qt-mt323:qt-mt323.dll
 0002:00001378       __imp_?setPixmap@QDataTable@@MAEXHHABVQPixmap@@@Z 10027378     qt-mt323:qt-mt323.dll
 0002:0000137c       __imp_?setPrefix@QSpinBox@@UAEXABVQString@@@Z 1002737c     qt-mt323:qt-mt323.dll
 0002:00001380       __imp_?setRadioButtonExclusive@QButtonGroup@@UAEX_N@Z 10027380     qt-mt323:qt-mt323.dll
 0002:00001384       __imp_?setRange@QDateEdit@@UAEXABVQDate@@0@Z 10027384     qt-mt323:qt-mt323.dll
 0002:00001388       __imp_?setReadOnly@QTable@@UAEX_N@Z 10027388     qt-mt323:qt-mt323.dll
 0002:0000138c       __imp_?setResizeMode@QSplitter@@UAEXPAVQWidget@@W4ResizeMode@1@@Z 1002738c     qt-mt323:qt-mt323.dll
 0002:00001390       __imp_?setRowHeight@QTable@@UAEXHH@Z 10027390     qt-mt323:qt-mt323.dll
 0002:00001394       __imp_?setRowMovingEnabled@QTable@@UAEX_N@Z 10027394     qt-mt323:qt-mt323.dll
 0002:00001398       __imp_?setRowReadOnly@QTable@@UAEXH_N@Z 10027398     qt-mt323:qt-mt323.dll
 0002:0000139c       __imp_?setRowStretchable@QTable@@UAEXH_N@Z 1002739c     qt-mt323:qt-mt323.dll
 0002:000013a0       __imp_?setRubberband@QSplitter@@MAEXH@Z 100273a0     qt-mt323:qt-mt323.dll
 0002:000013a4       __imp_?setSelectionMode@QTable@@UAEXW4SelectionMode@1@@Z 100273a4     qt-mt323:qt-mt323.dll
 0002:000013a8       __imp_?setSeparator@QDateEdit@@UAEXABVQString@@@Z 100273a8     qt-mt323:qt-mt323.dll
 0002:000013ac       __imp_?setShowGrid@QTable@@UAEX_N@Z 100273ac     qt-mt323:qt-mt323.dll
 0002:000013b0       __imp_?setSort@QDataTable@@UAEXABVQSqlIndex@@@Z 100273b0     qt-mt323:qt-mt323.dll
 0002:000013b4       __imp_?setSort@QDataTable@@UAEXABVQStringList@@@Z 100273b4     qt-mt323:qt-mt323.dll
 0002:000013b8       __imp_?setSorting@QTable@@UAEX_N@Z 100273b8     qt-mt323:qt-mt323.dll
 0002:000013bc       __imp_?setSpecialValueText@QSpinBox@@UAEXABVQString@@@Z 100273bc     qt-mt323:qt-mt323.dll
 0002:000013c0       __imp_?setSqlCursor@QDataTable@@UAEXPAVQSqlCursor@@_N1@Z 100273c0     qt-mt323:qt-mt323.dll
 0002:000013c4       __imp_?setSuffix@QSpinBox@@UAEXABVQString@@@Z 100273c4     qt-mt323:qt-mt323.dll
 0002:000013c8       __imp_?setText@QTable@@UAEXHHABVQString@@@Z 100273c8     qt-mt323:qt-mt323.dll
 0002:000013cc       __imp_?setTopMargin@QTable@@UAEXH@Z 100273cc     qt-mt323:qt-mt323.dll
 0002:000013d0       __imp_?setTrueText@QDataTable@@UAEXABVQString@@@Z 100273d0     qt-mt323:qt-mt323.dll
 0002:000013d4       __imp_?setValidator@QSpinBox@@UAEXPBVQValidator@@@Z 100273d4     qt-mt323:qt-mt323.dll
 0002:000013d8       __imp_?setValue@QSpinBox@@UAEXH@Z 100273d8     qt-mt323:qt-mt323.dll
 0002:000013dc       __imp_?setWrapping@QSpinBox@@UAEX_N@Z 100273dc     qt-mt323:qt-mt323.dll
 0002:000013e0       __imp_?setYear@QDateEdit@@MAEXH@Z 100273e0     qt-mt323:qt-mt323.dll
 0002:000013e4       __imp_?show@QScrollView@@UAEXXZ 100273e4     qt-mt323:qt-mt323.dll
 0002:000013e8       __imp_?showColumn@QDataTable@@UAEXH@Z 100273e8     qt-mt323:qt-mt323.dll
 0002:000013ec       __imp_?showEvent@QTable@@MAEXPAVQShowEvent@@@Z 100273ec     qt-mt323:qt-mt323.dll
 0002:000013f0       __imp_?showRow@QTable@@UAEXH@Z 100273f0     qt-mt323:qt-mt323.dll
 0002:000013f4       __imp_?sizeHint@QDateEdit@@UBE?AVQSize@@XZ 100273f4     qt-mt323:qt-mt323.dll
 0002:000013f8       __imp_?sizeHint@QRadioButton@@UBE?AVQSize@@XZ 100273f8     qt-mt323:qt-mt323.dll
 0002:000013fc       __imp_?sizeHint@QSpinBox@@UBE?AVQSize@@XZ 100273fc     qt-mt323:qt-mt323.dll
 0002:00001400       __imp_?sizeHint@QSplitter@@UBE?AVQSize@@XZ 10027400     qt-mt323:qt-mt323.dll
 0002:00001404       __imp_?sizeHint@QTable@@UBE?AVQSize@@XZ 10027404     qt-mt323:qt-mt323.dll
 0002:00001408       __imp_?sortAscending@QDataTable@@UAEXH@Z 10027408     qt-mt323:qt-mt323.dll
 0002:0000140c       __imp_?sortColumn@QDataTable@@UAEXH_N0@Z 1002740c     qt-mt323:qt-mt323.dll
 0002:00001410       __imp_?sortDescending@QDataTable@@UAEXH@Z 10027410     qt-mt323:qt-mt323.dll
 0002:00001414       __imp_?startDrag@QTable@@MAEXXZ 10027414     qt-mt323:qt-mt323.dll
 0002:00001418       __imp_?stepChange@QRangeControl@@MAEXXZ 10027418     qt-mt323:qt-mt323.dll
 0002:0000141c       __imp_?stepDown@QDateEdit@@MAEXXZ 1002741c     qt-mt323:qt-mt323.dll
 0002:00001420       __imp_?stepDown@QSpinBox@@UAEXXZ 10027420     qt-mt323:qt-mt323.dll
 0002:00001424       __imp_?stepUp@QDateEdit@@MAEXXZ 10027424     qt-mt323:qt-mt323.dll
 0002:00001428       __imp_?stepUp@QSpinBox@@UAEXXZ 10027428     qt-mt323:qt-mt323.dll
 0002:0000142c       __imp_?styleChange@QScrollView@@UAEXAAVQStyle@@@Z 1002742c     qt-mt323:qt-mt323.dll
 0002:00001430       __imp_?styleChange@QSpinBox@@MAEXAAVQStyle@@@Z 10027430     qt-mt323:qt-mt323.dll
 0002:00001434       __imp_?styleChange@QSplitter@@MAEXAAVQStyle@@@Z 10027434     qt-mt323:qt-mt323.dll
 0002:00001438       __imp_?suffix@QSpinBox@@UBE?AVQString@@XZ 10027438     qt-mt323:qt-mt323.dll
 0002:0000143c       __imp_?swapCells@QTable@@UAEXHHHH@Z 1002743c     qt-mt323:qt-mt323.dll
 0002:00001440       __imp_?swapColumns@QDataTable@@UAEXHH_N@Z 10027440     qt-mt323:qt-mt323.dll
 0002:00001444       __imp_?swapRows@QTable@@UAEXHH_N@Z 10027444     qt-mt323:qt-mt323.dll
 0002:00001448       __imp_?takeItem@QDataTable@@MAEXPAVQTableItem@@@Z 10027448     qt-mt323:qt-mt323.dll
 0002:0000144c       __imp_?text@QDataTable@@UBE?AVQString@@HH@Z 1002744c     qt-mt323:qt-mt323.dll
 0002:00001450       __imp_?timerEvent@QDateEdit@@MAEXPAVQTimerEvent@@@Z 10027450     qt-mt323:qt-mt323.dll
 0002:00001454       __imp_?updateCurrent@QDataTable@@MAE_NXZ 10027454     qt-mt323:qt-mt323.dll
 0002:00001458       __imp_?updateDisplay@QSpinBox@@MAEXXZ 10027458     qt-mt323:qt-mt323.dll
 0002:0000145c       __imp_?updateMask@QRadioButton@@MAEXXZ 1002745c     qt-mt323:qt-mt323.dll
 0002:00001460       __imp_?valueChange@QSpinBox@@MAEXXZ 10027460     qt-mt323:qt-mt323.dll
 0002:00001464       __imp_?viewportResizeEvent@QTable@@MAEXPAVQResizeEvent@@@Z 10027464     qt-mt323:qt-mt323.dll
 0002:00001468       __imp_?wheelEvent@QSpinBox@@MAEXPAVQWheelEvent@@@Z 10027468     qt-mt323:qt-mt323.dll
 0002:0000146c       __imp_?windowActivationChange@QTable@@MAEX_N@Z 1002746c     qt-mt323:qt-mt323.dll
 0002:00001470       __imp_??0QTable@@QAE@PAVQWidget@@PBD@Z 10027470     qt-mt323:qt-mt323.dll
 0002:00001474       __imp_??1QTable@@UAE@XZ    10027474     qt-mt323:qt-mt323.dll
 0002:00001478       __imp_?horizontalHeader@QTable@@QBEPAVQHeader@@XZ 10027478     qt-mt323:qt-mt323.dll
 0002:0000147c       __imp_?activateNextCell@QTable@@MAEXXZ 1002747c     qt-mt323:qt-mt323.dll
 0002:00001480       __imp_?adjustColumn@QTable@@UAEXH@Z 10027480     qt-mt323:qt-mt323.dll
 0002:00001484       __imp_?beginEdit@QTable@@MAEPAVQWidget@@HH_N@Z 10027484     qt-mt323:qt-mt323.dll
 0002:00001488       __imp_?className@QTable@@UBEPBDXZ 10027488     qt-mt323:qt-mt323.dll
 0002:0000148c       __imp_?clearCell@QTable@@UAEXHH@Z 1002748c     qt-mt323:qt-mt323.dll
 0002:00001490       __imp_?columnClicked@QTable@@MAEXH@Z 10027490     qt-mt323:qt-mt323.dll
 0002:00001494       __imp_?contentsContextMenuEvent@QTable@@MAEXPAVQContextMenuEvent@@@Z 10027494     qt-mt323:qt-mt323.dll
 0002:00001498       __imp_?contentsMousePressEvent@QTable@@MAEXPAVQMouseEvent@@@Z 10027498     qt-mt323:qt-mt323.dll
 0002:0000149c       __imp_?createEditor@QTable@@MBEPAVQWidget@@HH_N@Z 1002749c     qt-mt323:qt-mt323.dll
 0002:000014a0       __imp_?drawContents@QTable@@MAEXPAVQPainter@@HHHH@Z 100274a0     qt-mt323:qt-mt323.dll
 0002:000014a4       __imp_?endEdit@QTable@@MAEXHH_N0@Z 100274a4     qt-mt323:qt-mt323.dll
 0002:000014a8       __imp_?eventFilter@QTable@@UAE_NPAVQObject@@PAVQEvent@@@Z 100274a8     qt-mt323:qt-mt323.dll
 0002:000014ac       __imp_?hideColumn@QTable@@UAEXH@Z 100274ac     qt-mt323:qt-mt323.dll
 0002:000014b0       __imp_?item@QTable@@UBEPAVQTableItem@@HH@Z 100274b0     qt-mt323:qt-mt323.dll
 0002:000014b4       __imp_?keyPressEvent@QTable@@MAEXPAVQKeyEvent@@@Z 100274b4     qt-mt323:qt-mt323.dll
 0002:000014b8       __imp_?metaObject@QTable@@UBEPAVQMetaObject@@XZ 100274b8     qt-mt323:qt-mt323.dll
 0002:000014bc       __imp_?numCols@QTable@@UBEHXZ 100274bc     qt-mt323:qt-mt323.dll
 0002:000014c0       __imp_?numRows@QTable@@UBEHXZ 100274c0     qt-mt323:qt-mt323.dll
 0002:000014c4       __imp_?paintCell@QTable@@UAEXPAVQPainter@@HHABVQRect@@_NABVQColorGroup@@@Z 100274c4     qt-mt323:qt-mt323.dll
 0002:000014c8       __imp_?qt_cast@QTable@@UAEPAXPBD@Z 100274c8     qt-mt323:qt-mt323.dll
 0002:000014cc       __imp_?qt_emit@QTable@@UAE_NHPAUQUObject@@@Z 100274cc     qt-mt323:qt-mt323.dll
 0002:000014d0       __imp_?qt_invoke@QTable@@UAE_NHPAUQUObject@@@Z 100274d0     qt-mt323:qt-mt323.dll
 0002:000014d4       __imp_?qt_property@QTable@@UAE_NHHPAVQVariant@@@Z 100274d4     qt-mt323:qt-mt323.dll
 0002:000014d8       __imp_?resizeData@QTable@@MAEXH@Z 100274d8     qt-mt323:qt-mt323.dll
 0002:000014dc       __imp_?resizeEvent@QScrollView@@MAEXPAVQResizeEvent@@@Z 100274dc     qt-mt323:qt-mt323.dll
 0002:000014e0       __imp_?setColumnStretchable@QTable@@UAEXH_N@Z 100274e0     qt-mt323:qt-mt323.dll
 0002:000014e4       __imp_?setColumnWidth@QTable@@UAEXHH@Z 100274e4     qt-mt323:qt-mt323.dll
 0002:000014e8       __imp_?setItem@QTable@@UAEXHHPAVQTableItem@@@Z 100274e8     qt-mt323:qt-mt323.dll
 0002:000014ec       __imp_?setNumCols@QTable@@UAEXH@Z 100274ec     qt-mt323:qt-mt323.dll
 0002:000014f0       __imp_?setNumRows@QTable@@UAEXH@Z 100274f0     qt-mt323:qt-mt323.dll
 0002:000014f4       __imp_?setPixmap@QTable@@UAEXHHABVQPixmap@@@Z 100274f4     qt-mt323:qt-mt323.dll
 0002:000014f8       __imp_?showColumn@QTable@@UAEXH@Z 100274f8     qt-mt323:qt-mt323.dll
 0002:000014fc       __imp_?sortColumn@QTable@@UAEXH_N0@Z 100274fc     qt-mt323:qt-mt323.dll
 0002:00001500       __imp_?swapColumns@QTable@@UAEXHH_N@Z 10027500     qt-mt323:qt-mt323.dll
 0002:00001504       __imp_?takeItem@QTable@@UAEXPAVQTableItem@@@Z 10027504     qt-mt323:qt-mt323.dll
 0002:00001508       __imp_?text@QTable@@UBE?AVQString@@HH@Z 10027508     qt-mt323:qt-mt323.dll
 0002:0000150c       __imp_?receivers@QObject@@IBEPAVQConnectionList@@H@Z 1002750c     qt-mt323:qt-mt323.dll
 0002:00001510       __imp_?activate_signal@QObject@@IAEXPAVQConnectionList@@PAUQUObject@@@Z 10027510     qt-mt323:qt-mt323.dll
 0002:00001514       __imp_?staticMetaObject@QWidget@@SAPAVQMetaObject@@XZ 10027514     qt-mt323:qt-mt323.dll
 0002:00001518       __imp_??0QUObject@@QAE@XZ  10027518     qt-mt323:qt-mt323.dll
 0002:0000151c       __imp_??1QUObject@@QAE@XZ  1002751c     qt-mt323:qt-mt323.dll
 0002:00001520       __imp_?set@QUType_QString@@QAEXPAUQUObject@@ABVQString@@@Z 10027520     qt-mt323:qt-mt323.dll
 0002:00001524       __imp_?static_QUType_ptr@@3UQUType_ptr@@A 10027524     qt-mt323:qt-mt323.dll
 0002:00001528       __imp_?static_QUType_bool@@3UQUType_bool@@A 10027528     qt-mt323:qt-mt323.dll
 0002:0000152c       __imp_?static_QUType_int@@3UQUType_int@@A 1002752c     qt-mt323:qt-mt323.dll
 0002:00001530       __imp_?static_QUType_QString@@3UQUType_QString@@A 10027530     qt-mt323:qt-mt323.dll
 0002:00001534       __imp_?static_QUType_varptr@@3UQUType_varptr@@A 10027534     qt-mt323:qt-mt323.dll
 0002:00001538       __imp_?activate_signal@QObject@@IAEXH@Z 10027538     qt-mt323:qt-mt323.dll
 0002:0000153c       __imp_??0?$QMap@VQString@@H@@QAE@XZ 1002753c     qt-mt323:qt-mt323.dll
 0002:00001540       __imp_?rebalance@QMapPrivateBase@@QAEXPAUQMapNodeBase@@AAPAU2@@Z 10027540     qt-mt323:qt-mt323.dll
 0002:00001544       __imp_?detachInternal@?$QValueList@VQString@@@@AAEXXZ 10027544     qt-mt323:qt-mt323.dll
 0002:00001548       __imp_?contains@?$QValueList@VQString@@@@QBEIABVQString@@@Z 10027548     qt-mt323:qt-mt323.dll
 0002:0000154c       __imp_??A?$QValueList@VQString@@@@QAEAAVQString@@I@Z 1002754c     qt-mt323:qt-mt323.dll
 0002:00001550       __imp_?append@?$QValueList@VQString@@@@QAE?AV?$QValueListIterator@VQString@@@@ABVQString@@@Z 10027550     qt-mt323:qt-mt323.dll
 0002:00001554       __imp_?clear@?$QValueList@VQString@@@@QAEXXZ 10027554     qt-mt323:qt-mt323.dll
 0002:00001558       __imp_?begin@?$QValueList@VQString@@@@QAE?AV?$QValueListIterator@VQString@@@@XZ 10027558     qt-mt323:qt-mt323.dll
 0002:0000155c       __imp_?readLine@QTextStream@@QAE?AVQString@@XZ 1002755c     qt-mt323:qt-mt323.dll
 0002:00001560       __imp_??6QTextStream@@QAEAAV0@ABVQString@@@Z 10027560     qt-mt323:qt-mt323.dll
 0002:00001564       __imp_??6QTextStream@@QAEAAV0@PBD@Z 10027564     qt-mt323:qt-mt323.dll
 0002:00001568       __imp_?setPrimaryIndex@QSqlCursor@@UAEXABVQSqlIndex@@@Z 10027568     qt-mt323:qt-mt323.dll
 0002:0000156c       __imp_??6QTextStream@@QAEAAV0@H@Z 1002756c     qt-mt323:qt-mt323.dll
 0002:00001570       __imp_??0QString@@QAE@XZ   10027570     qt-mt323:qt-mt323.dll
 0002:00001574       __imp_?next@QGList@@IAEPAXXZ 10027574     qt-mt323:qt-mt323.dll
 0002:00001578       __imp_??1QTextStream@@UAE@XZ 10027578     qt-mt323:qt-mt323.dll
 0002:0000157c       __imp_??0QTextStream@@QAE@PAVQIODevice@@@Z 1002757c     qt-mt323:qt-mt323.dll
 0002:00001580       __imp_?reset@QIODevice@@QAE_NXZ 10027580     qt-mt323:qt-mt323.dll
 0002:00001584       __imp_??H@YA?BVQString@@PBDABV0@@Z 10027584     qt-mt323:qt-mt323.dll
 0002:00001588       __imp_??H@YA?BVQString@@ABV0@PBD@Z 10027588     qt-mt323:qt-mt323.dll
 0002:0000158c       __imp_??H@YA?BVQString@@ABV0@0@Z 1002758c     qt-mt323:qt-mt323.dll
 0002:00001590       __imp_??8@YA_NABVQString@@PBD@Z 10027590     qt-mt323:qt-mt323.dll
 0002:00001594       __imp_??9@YA_NABVQString@@PBD@Z 10027594     qt-mt323:qt-mt323.dll
 0002:00001598       __imp_??8@YA_NABVQString@@0@Z 10027598     qt-mt323:qt-mt323.dll
 0002:0000159c       __imp_??M@YA_NABVQString@@0@Z 1002759c     qt-mt323:qt-mt323.dll
 0002:000015a0       __imp_??9@YA_NABVQString@@0@Z 100275a0     qt-mt323:qt-mt323.dll
 0002:000015a4       __imp_?setLength@QString@@QAEXI@Z 100275a4     qt-mt323:qt-mt323.dll
 0002:000015a8       __imp_?endsWith@QString@@QBE_NABV1@@Z 100275a8     qt-mt323:qt-mt323.dll
 0002:000015ac       __imp_?startsWith@QString@@QBE_NABV1@@Z 100275ac     qt-mt323:qt-mt323.dll
 0002:000015b0       __imp_?latin1@QString@@QBEPBDXZ 100275b0     qt-mt323:qt-mt323.dll
 0002:000015b4       __imp_?ascii@QString@@QBEPBDXZ 100275b4     qt-mt323:qt-mt323.dll
 0002:000015b8       __imp_??YQString@@QAEAAV0@PBD@Z 100275b8     qt-mt323:qt-mt323.dll
 0002:000015bc       __imp_??YQString@@QAEAAV0@ABV0@@Z 100275bc     qt-mt323:qt-mt323.dll
 0002:000015c0       __imp_?number@QString@@SA?AV1@HH@Z 100275c0     qt-mt323:qt-mt323.dll
 0002:000015c4       __imp_?toInt@QString@@QBEHPA_NH@Z 100275c4     qt-mt323:qt-mt323.dll
 0002:000015c8       __imp_?replace@QString@@QAEAAV1@ABV1@0@Z 100275c8     qt-mt323:qt-mt323.dll
 0002:000015cc       __imp_?remove@QString@@QAEAAV1@ABV1@_N@Z 100275cc     qt-mt323:qt-mt323.dll
 0002:000015d0       __imp_?remove@QString@@QAEAAV1@ABV1@@Z 100275d0     qt-mt323:qt-mt323.dll
 0002:000015d4       __imp_?remove@QString@@QAEAAV1@II@Z 100275d4     qt-mt323:qt-mt323.dll
 0002:000015d8       __imp_?insert@QString@@QAEAAV1@IABV1@@Z 100275d8     qt-mt323:qt-mt323.dll
 0002:000015dc       __imp_?stripWhiteSpace@QString@@QBE?AV1@XZ 100275dc     qt-mt323:qt-mt323.dll
 0002:000015e0       __imp_?right@QString@@QBE?AV1@I@Z 100275e0     qt-mt323:qt-mt323.dll
 0002:000015e4       __imp_?section@QString@@QBE?AV1@PBDHHH@Z 100275e4     qt-mt323:qt-mt323.dll
 0002:000015e8       __imp_?contains@QString@@QBEHABVQRegExp@@@Z 100275e8     qt-mt323:qt-mt323.dll
 0002:000015ec       __imp_?contains@QString@@QBEHABV1@_N@Z 100275ec     qt-mt323:qt-mt323.dll
 0002:000015f0       __imp_?contains@QString@@QBEHPBD_N@Z 100275f0     qt-mt323:qt-mt323.dll
 0002:000015f4       __imp_?sprintf@QString@@QAAAAV1@PBDZZ 100275f4     qt-mt323:qt-mt323.dll
 0002:000015f8       __imp_?arg@QString@@QBE?AV1@ABV1@H@Z 100275f8     qt-mt323:qt-mt323.dll
 0002:000015fc       __imp_?arg@QString@@QBE?AV1@HHH@Z 100275fc     qt-mt323:qt-mt323.dll
 0002:00001600       __imp_??4QString@@QAEAAV0@PBD@Z 10027600     qt-mt323:qt-mt323.dll
 0002:00001604       __imp_??4QString@@QAEAAV0@ABV0@@Z 10027604     qt-mt323:qt-mt323.dll
 0002:00001608       __imp_??1QString@@QAE@XZ   10027608     qt-mt323:qt-mt323.dll
 0002:0000160c       __imp_?setSort@QSqlCursor@@UAEXABVQSqlIndex@@@Z 1002760c     qt-mt323:qt-mt323.dll
 0002:00001610       __imp_??0QString@@QAE@PBD@Z 10027610     qt-mt323:qt-mt323.dll
 0002:00001614       __imp_??0?$QValueList@H@@QAE@XZ 10027614     qt-mt323:qt-mt323.dll
 0002:00001618       __imp_??1?$QValueList@H@@QAE@XZ 10027618     qt-mt323:qt-mt323.dll
 0002:0000161c       __imp_?begin@?$QValueList@H@@QAE?AV?$QValueListIterator@H@@XZ 1002761c     qt-mt323:qt-mt323.dll
 0002:00001620       __imp_?append@?$QValueList@H@@QAE?AV?$QValueListIterator@H@@ABH@Z 10027620     qt-mt323:qt-mt323.dll
 0002:00001624       __imp_?detachInternal@?$QValueList@H@@AAEXXZ 10027624     qt-mt323:qt-mt323.dll
 0002:00001628       __imp_??0QSettings@@QAE@W4Format@0@@Z 10027628     qt-mt323:qt-mt323.dll
 0002:0000162c       __imp_??1QSettings@@QAE@XZ 1002762c     qt-mt323:qt-mt323.dll
 0002:00001630       __imp_?writeEntry@QSettings@@QAE_NABVQString@@0@Z 10027630     qt-mt323:qt-mt323.dll
 0002:00001634       __imp_?readEntry@QSettings@@QAE?AVQString@@ABV2@0PA_N@Z 10027634     qt-mt323:qt-mt323.dll
 0002:00001638       __imp_?sizes@QSplitter@@QBE?AV?$QValueList@H@@XZ 10027638     qt-mt323:qt-mt323.dll
 0002:0000163c       __imp_?setSizes@QSplitter@@QAEXV?$QValueList@H@@@Z 1002763c     qt-mt323:qt-mt323.dll
 0002:00001640       __imp_?columnWidth@QListView@@QBEHH@Z 10027640     qt-mt323:qt-mt323.dll
 0002:00001644       __imp_?columns@QListView@@QBEHXZ 10027644     qt-mt323:qt-mt323.dll
 0002:00001648       __imp_?deleteSelf@QStringData@@QAEXXZ 10027648     qt-mt323:qt-mt323.dll
 0002:0000164c       __imp_?lower@QString@@QBE?AV1@XZ 1002764c     qt-mt323:qt-mt323.dll
 0002:00001650       __imp_?makeSharedNull@QString@@CAPAUQStringData@@XZ 10027650     qt-mt323:qt-mt323.dll
 0002:00001654       __imp_?shared_null@QString@@0PAUQStringData@@A 10027654     qt-mt323:qt-mt323.dll
 0002:00001658       __imp_?first@QGList@@IAEPAXXZ 10027658     qt-mt323:qt-mt323.dll
 0002:0000165c       __imp_?clear@QGList@@MAEXXZ 1002765c     qt-mt323:qt-mt323.dll
 0002:00001660       __imp_?remove@QGList@@IAE_NPAX@Z 10027660     qt-mt323:qt-mt323.dll
 0002:00001664       __imp_?append@QGList@@IAEXPAX@Z 10027664     qt-mt323:qt-mt323.dll
 0002:00001668       __imp_??1QGList@@MAE@XZ    10027668     qt-mt323:qt-mt323.dll
 0002:0000166c       __imp_??0QGList@@IAE@XZ    1002766c     qt-mt323:qt-mt323.dll
 0002:00001670       __imp_?setContentFromEditor@QCheckTableItem@@UAEXPAVQWidget@@@Z 10027670     qt-mt323:qt-mt323.dll
 0002:00001674       __imp_?qDebug@@YAXPBDZZ    10027674     qt-mt323:qt-mt323.dll
 0002:00001678       \177qt-mt323_NULL_THUNK_DATA 10027678     qt-mt323:qt-mt323.dll
 0002:0000167c       ___xc_a                    1002767c     MSVCRT:cinitexe.obj
 0002:000016ac       ___xc_z                    100276ac     MSVCRT:cinitexe.obj
 0002:000016b0       ___xi_a                    100276b0     MSVCRT:cinitexe.obj
 0002:000016bc       ___xi_z                    100276bc     MSVCRT:cinitexe.obj
 0002:000016c4       ??_SQWidget@@6BQObject@@@  100276c4     alm_db_output.obj
 0002:00001878       ??_SQWidget@@6BQPaintDevice@@@ 10027878     alm_db_output.obj
 0002:00001898       ??_C@_02GIPFHKNO@OK?$AA@   10027898     alm_db_output.obj
 0002:000018a4       ??_SQAction@@6B@           100278a4     alm_db_output.obj
 0002:00001934       ??_SQDockWindow@@6BQObject@@@ 10027934     alm_db_output.obj
 0002:00001b44       ??_SQDockWindow@@6BQPaintDevice@@@ 10027b44     alm_db_output.obj
 0002:00001b6c       ??_SQToolBar@@6BQObject@@@ 10027b6c     alm_db_output.obj
 0002:00001d88       ??_SQToolBar@@6BQPaintDevice@@@ 10027d88     alm_db_output.obj
 0002:00001dac       ??_SQListViewItem@@6B@     10027dac     alm_db_output.obj
 0002:00001e4c       ??_SQListView@@6BQObject@@@ 10027e4c     alm_db_output.obj
 0002:00002130       ??_SQListView@@6BQPaintDevice@@@ 10028130     alm_db_output.obj
 0002:00002154       ??_SQFile@@6B@             10028154     alm_db_output.obj
 0002:00002194       ??_SQTabWidget@@6BQObject@@@ 10028194     alm_db_output.obj
 0002:00002368       ??_SQTabWidget@@6BQPaintDevice@@@ 10028368     alm_db_output.obj
 0002:0000238c       ??_SQBoxLayout@@6BQObject@@@ 1002838c     alm_db_output.obj
 0002:000023f4       ??_SQBoxLayout@@6BQLayoutItem@@@ 100283f4     alm_db_output.obj
 0002:00002434       ??_C@_00CNPNBAHC@?$AA@     10028434     alm_db_output.obj
 0002:0000243c       ??_7error_category@std@@6B@ 1002843c     alm_db_output.obj
 0002:00002458       ??_7_Generic_error_category@std@@6B@ 10028458     alm_db_output.obj
 0002:00002470       ??_C@_07DCLBNMLN@generic?$AA@ 10028470     alm_db_output.obj
 0002:00002478       ??_C@_0O@BFJCFAAK@unknown?5error?$AA@ 10028478     alm_db_output.obj
 0002:0000248c       ??_7_Iostream_error_category@std@@6B@ 1002848c     alm_db_output.obj
 0002:000024a4       ??_C@_08LLGCOLLL@iostream?$AA@ 100284a4     alm_db_output.obj
 0002:000024b0       ??_C@_0BG@PADBLCHM@iostream?5stream?5error?$AA@ 100284b0     alm_db_output.obj
 0002:000024cc       ??_7_System_error_category@std@@6B@ 100284cc     alm_db_output.obj
 0002:000024e4       ??_C@_06FHFOAHML@system?$AA@ 100284e4     alm_db_output.obj
 0002:000024f4       ??_SCAlm_sys_select@@6BQObject@@@ 100284f4     alm_db_output.obj
 0002:000026c8       ??_SCAlm_sys_select@@6BQPaintDevice@@@ 100286c8     alm_db_output.obj
 0002:000026ec       ??_SQGuardedPtrPrivate@@6B@ 100286ec     alm_db_output.obj
 0002:00002740       ??_7QDockWindowList@@6B@   10028740     alm_db_output.obj
 0002:00002764       ??_SQPopupMenu@@6BQObject@@@ 10028764     alm_db_output.obj
 0002:00002944       ??_SQPopupMenu@@6BQPaintDevice@@@ 10028944     alm_db_output.obj
 0002:00002968       ??_SQPopupMenu@@6B@        10028968     alm_db_output.obj
 0002:0000298c       ??_7?$QPtrList@VQPopupMenu@@@@6B@ 1002898c     alm_db_output.obj
 0002:000029b0       ??_7QPopupMenuList@@6B@    100289b0     alm_db_output.obj
 0002:000029d4       ??_7IGetDocuments@@6B@     100289d4     alm_db_output.obj
 0002:000029f0       ??_7ISendCommand@@6B@      100289f0     alm_db_output.obj
 0002:000029f8       ??_7config_plugin_base@@6BQObject@@@ 100289f8     alm_db_output.obj
 0002:00002bd0       ??_7config_plugin_base@@6BQPaintDevice@@@ 10028bd0     alm_db_output.obj
 0002:00002bf0       ??_C@_0EB@GNDACMDJ@?$CC?5?9?5the?5author?5should?5have?5defin@ 10028bf0     alm_db_output.obj
 0002:00002c34       ??_C@_0CH@BDPDPLDP@This?5is?5the?5default?5?$CCAbout?$CC?5text@ 10028c34     alm_db_output.obj
 0002:00002c60       ??_7FileLoad_BncsSystem@alm_db_output@@6B@ 10028c60     alm_db_output.obj
 0002:00002c70       ??_7?$QDict@VQAction@@@@6B@ 10028c70     alm_db_output.obj
 0002:00002c90       ??_7?$QPtrList@VcOutputFile@@@@6B@ 10028c90     alm_db_output.obj
 0002:00002cb4       ??_7alm_db_output@@6BQObject@@@ 10028cb4     alm_db_output.obj
 0002:00002e8c       ??_7alm_db_output@@6BQPaintDevice@@@ 10028e8c     alm_db_output.obj
 0002:00002eb0       ??_7alm_db_output@@6BIGetDocuments@@@ 10028eb0     alm_db_output.obj
 0002:00002ecc       ??_7alm_db_output@@6BISendCommand@@@ 10028ecc     alm_db_output.obj
 0002:00002ed0       ??_C@_08DFEIFMHK@?1browser?$AA@ 10028ed0     alm_db_output.obj
 0002:00002edc       ??_C@_0BG@LMBECLGB@Alarm?5Outputs?5modules?$AA@ 10028edc     alm_db_output.obj
 0002:00002ef4       ??_C@_04FABLJDN@Name?$AA@  10028ef4     alm_db_output.obj
 0002:00002efc       ??_C@_0M@KOGPIGII@Config?5File?$AA@ 10028efc     alm_db_output.obj
 0002:00002f08       ??_C@_08KJDMPFAO@FileList?$AA@ 10028f08     alm_db_output.obj
 0002:00002f14       ??_C@_0BO@BFLDMNNG@Home?1Alarms?1Outputs?1Database?1?$AA@ 10028f14     alm_db_output.obj
 0002:00002f34       ??_C@_0BB@KOMMNKDC@?$CGDatabase?5Output?$AA@ 10028f34     alm_db_output.obj
 0002:00002f48       ??_C@_0O@FCCLFDMG@?1Database?5I?1F?$AA@ 10028f48     alm_db_output.obj
 0002:00002f58       ??_C@_03CLCAEGCJ@new?$AA@  10028f58     alm_db_output.obj
 0002:00002f5c       ??_C@_0M@OKPFFIMJ@?$CGNew?5Db?5I?1F?$AA@ 10028f5c     alm_db_output.obj
 0002:00002f68       ??_C@_07EJAINBEK@filenew?$AA@ 10028f68     alm_db_output.obj
 0002:00002f70       ??_C@_0L@NKLFBFC@New?5Db?5I?1F?$AA@ 10028f70     alm_db_output.obj
 0002:00002f7c       ??_C@_0P@CBINDBNH@1menuNewFile?$CI?$CJ?$AA@ 10028f7c     alm_db_output.obj
 0002:00002f8c       ??_C@_0N@KCMOKDBB@2activated?$CI?$CJ?$AA@ 10028f8c     alm_db_output.obj
 0002:00002f9c       ??_C@_06FOBLBEIN@delete?$AA@ 10028f9c     alm_db_output.obj
 0002:00002fa4       ??_C@_0P@JCLGLBKJ@?$CGDelete?5Db?5I?1F?$AA@ 10028fa4     alm_db_output.obj
 0002:00002fb4       ??_C@_0L@BPDPNFLB@filedelete?$AA@ 10028fb4     alm_db_output.obj
 0002:00002fc0       ??_C@_0O@DOOBCBOF@Delete?5Db?5I?1F?$AA@ 10028fc0     alm_db_output.obj
 0002:00002fd0       ??_C@_0BC@FIBCFKLP@1menuDeleteFile?$CI?$CJ?$AA@ 10028fd0     alm_db_output.obj
 0002:00002fe4       ??_C@_09KHIKJOBP@duplicate?$AA@ 10028fe4     alm_db_output.obj
 0002:00002ff0       ??_C@_0N@HDGJJGDN@?$CGCopy?5Db?5I?1F?$AA@ 10028ff0     alm_db_output.obj
 0002:00003000       ??_C@_0BB@NNGNCLAP@Duplicate?5Output?$AA@ 10029000     alm_db_output.obj
 0002:00003014       ??_C@_0BF@LDLOGHID@1menuDuplicateFile?$CI?$CJ?$AA@ 10029014     alm_db_output.obj
 0002:0000302c       ??_C@_06LMEAOBLB@rename?$AA@ 1002902c     alm_db_output.obj
 0002:00003034       ??_C@_0P@ILJPIBEM@?$CGRename?5Db?5I?1F?$AA@ 10029034     alm_db_output.obj
 0002:00003044       ??_C@_0O@CHMIBBAA@Rename?5Db?5I?1F?$AA@ 10029044     alm_db_output.obj
 0002:00003054       ??_C@_0O@DALNGBDG@1menuRename?$CI?$CJ?$AA@ 10029054     alm_db_output.obj
 0002:00003064       ??_C@_0DL@BGNECHKO@1fileListContextMenu?$CIQListViewIt@ 10029064     alm_db_output.obj
 0002:000030a0       ??_C@_0DL@JIJPNNOD@2contextMenuRequested?$CIQListViewI@ 100290a0     alm_db_output.obj
 0002:000030dc       ??_C@_0BN@PALMGDOM@1selectFile?$CIQListViewItem?5?$CK?$CJ?$AA@ 100290dc     alm_db_output.obj
 0002:000030fc       ??_C@_0CC@LCOLGNI@2selectionChanged?$CIQListViewItem?$CK@ 100290fc     alm_db_output.obj
 0002:00003120       ??_C@_0DE@NNBCFON@1renameModule?$CIQListViewItem?$CK?0?5in@ 10029120     alm_db_output.obj
 0002:00003154       ??_C@_0DD@FNLKOMHF@2itemRenamed?$CIQListViewItem?$CK?0?5int@ 10029154     alm_db_output.obj
 0002:00003188       ??_C@_0BP@KFJPMMLE@1selectSystem?$CIconst?5QString?5?$CG?$CJ?$AA@ 10029188     alm_db_output.obj
 0002:000031a8       ??_C@_0BN@DDAIKEMB@2sysChanged?$CIconst?5QString?5?$CG?$CJ?$AA@ 100291a8     alm_db_output.obj
 0002:000031c8       ??_C@_0N@LMCHKLFE@1markDirty?$CI?$CJ?$AA@ 100291c8     alm_db_output.obj
 0002:000031d8       ??_C@_0BA@LHBDKNBL@2itemsChanged?$CI?$CJ?$AA@ 100291d8     alm_db_output.obj
 0002:000031e8       ??_C@_0BF@HDMKHFLG@1editSelectedProcs?$CI?$CJ?$AA@ 100291e8     alm_db_output.obj
 0002:00003200       ??_C@_0L@OELOHDKG@2clicked?$CI?$CJ?$AA@ 10029200     alm_db_output.obj
 0002:0000320c       ??_C@_0BD@POIAIBAF@1templateProcess?$CI?$CJ?$AA@ 1002920c     alm_db_output.obj
 0002:00003220       ??_C@_0BB@PMPKEMJD@1procSelection?$CI?$CJ?$AA@ 10029220     alm_db_output.obj
 0002:00003234       ??_C@_0P@GLIODLHI@2dataChanged?$CI?$CJ?$AA@ 10029234     alm_db_output.obj
 0002:00003244       ??_C@_0BE@BLJBKCLJ@2selectionChanged?$CI?$CJ?$AA@ 10029244     alm_db_output.obj
 0002:00003258       ??_C@_0P@JECNNCNO@1EditProcess?$CI?$CJ?$AA@ 10029258     alm_db_output.obj
 0002:00003268       ??_C@_0BD@JHFHEMLD@1copyToClipBoard?$CI?$CJ?$AA@ 10029268     alm_db_output.obj
 0002:0000327c       ??_C@_0BB@JEGMINHG@1pasteAllProcs?$CI?$CJ?$AA@ 1002927c     alm_db_output.obj
 0002:00003290       ??_C@_0BG@JNPCOJCF@1pasteSelectedProcs?$CI?$CJ?$AA@ 10029290     alm_db_output.obj
 0002:000032a8       ??_C@_0BA@MAJNLODJ@1filterChange?$CI?$CJ?$AA@ 100292a8     alm_db_output.obj
 0002:000032b8       ??_C@_0BO@JONBIMPD@2textChanged?$CIconst?5QString?5?$CG?$CJ?$AA@ 100292b8     alm_db_output.obj
 0002:000032d8       ??_C@_0BA@HAKGEOGG@2activated?$CIint?$CJ?$AA@ 100292d8     alm_db_output.obj
 0002:000032e8       ??_C@_0BL@GMAFMKJD@alm_db_output?5constructed?4?$AA@ 100292e8     alm_db_output.obj
 0002:00003304       ??_C@_06BNCCALCL@unlock?$AA@ 10029304     alm_db_output.obj
 0002:0000330c       ??_C@_08HNIAHLMM@download?$AA@ 1002930c     alm_db_output.obj
 0002:00003318       ??_C@_0BD@DDFIPJEJ@File?5downloaded?5?9?5?$AA@ 10029318     alm_db_output.obj
 0002:0000332c       ??_C@_04MKMCLCOO@lock?$AA@ 1002932c     alm_db_output.obj
 0002:00003334       ??_C@_06KAOCKAGB@upload?$AA@ 10029334     alm_db_output.obj
 0002:0000333c       ??_C@_03DAPAKLGM@dir?$AA@  1002933c     alm_db_output.obj
 0002:00003340       ??_C@_07MPPKIBJA@Error?3?6?$AA@ 10029340     alm_db_output.obj
 0002:00003348       ??_C@_05NAOIJFC@Error?$AA@ 10029348     alm_db_output.obj
 0002:00003350       ??_C@_0BB@GABCCOJN@Unknown?5response?$AA@ 10029350     alm_db_output.obj
 0002:00003364       ??_C@_08JBEPPOLH@?1outputs?$AA@ 10029364     alm_db_output.obj
 0002:00003370       ??_C@_01KMDKNFGN@?1?$AA@   10029370     alm_db_output.obj
 0002:00003374       ??_C@_0O@MIFBLPDN@config?1alarms?$AA@ 10029374     alm_db_output.obj
 0002:00003384       ??_C@_07BOAKCNCF@al_out_?$AA@ 10029384     alm_db_output.obj
 0002:0000338c       ??_C@_04IFJILJI@?4cfg?$AA@ 1002938c     alm_db_output.obj
 0002:00003394       ??_C@_0L@FGNBINDG@ConfigTool?$AA@ 10029394     alm_db_output.obj
 0002:000033a0       ??_C@_06JIODDOFH@System?$AA@ 100293a0     alm_db_output.obj
 0002:000033a8       ??_C@_0N@LEBPCLIG@proc_def?4cfg?$AA@ 100293a8     alm_db_output.obj
 0002:000033b8       ??_C@_0M@FNMDGLGJ@Got?5file?5?9?5?$AA@ 100293b8     alm_db_output.obj
 0002:000033c4       ??_C@_0L@GBLJJCHL@File?5is?5?$CFs?$AA@ 100293c4     alm_db_output.obj
 0002:000033d0       ??_C@_03GJCOJFLC@?4?6?6?$AA@ 100293d0     alm_db_output.obj
 0002:000033d4       ??_C@_0BM@CGOIHJMM@Could?5not?5Create?5directory?6?$AA@ 100293d4     alm_db_output.obj
 0002:000033f0       ??_C@_0BB@IMCDCEGC@Alarms?1Processes?$AA@ 100293f0     alm_db_output.obj
 0002:00003404       ??_C@_0CC@OAGIAEAC@?6File?5will?5be?5available?5read?5onl@ 10029404     alm_db_output.obj
 0002:00003428       ??_C@_03NLJIHOMM@?5?9?5?$AA@ 10029428     alm_db_output.obj
 0002:0000342c       ??_C@_06JGFHLLHI@Lock?3?5?$AA@ 1002942c     alm_db_output.obj
 0002:00003434       ??_C@_04LADJNOK@Lock?$AA@  10029434     alm_db_output.obj
 0002:0000343c       ??_C@_05CCAMFJOL@clean?$AA@ 1002943c     alm_db_output.obj
 0002:00003444       ??_C@_0CO@DMDPGOMC@Being?5asked?5to?5navigate?5to?5?$CFs?5wi@ 10029444     alm_db_output.obj
 0002:00003474       ??_C@_01ICJEACDI@?$DL?$AA@ 10029474     alm_db_output.obj
 0002:00003478       ??_C@_02PEIOPPKO@?2S?$AA@  10029478     alm_db_output.obj
 0002:0000347c       ??_C@_0BC@PDAHGCDI@Process?5not?5found?$AA@ 1002947c     alm_db_output.obj
 0002:00003490       ??_C@_09OLBIFBJN@Process?3?5?$AA@ 10029490     alm_db_output.obj
 0002:0000349c       ??_C@_07MNGBFJEN@Process?$AA@ 1002949c     alm_db_output.obj
 0002:000034a4       ??_C@_0P@DBCHBMCI@File?5not?5found?$AA@ 100294a4     alm_db_output.obj
 0002:000034b4       ??_C@_06IGPBOHMJ@File?3?5?$AA@ 100294b4     alm_db_output.obj
 0002:000034bc       ??_C@_04PBAHLACE@File?$AA@ 100294bc     alm_db_output.obj
 0002:000034c4       ??_C@_0CE@LKBINMEK@Db?5Out?3?9?5ACTIVATE?5ME?5?9?5reload?5fi@ 100294c4     alm_db_output.obj
 0002:000034e8       ??_C@_0DO@EOJCMIED@Db?5Out?3?9?5ACTIVATE?5NOT?5ME?5?9?5save?5@ 100294e8     alm_db_output.obj
 0002:00003528       ??_C@_0BM@FNNNONDJ@Db?5Out?3?9?5Activate?5finished?4?$AA@ 10029528     alm_db_output.obj
 0002:00003544       ??_C@_0BF@LGJHIGH@alm_db_output?3?3apply?$AA@ 10029544     alm_db_output.obj
 0002:0000355c       ??_C@_0O@JFGJGFB@syncDirUpload?$AA@ 1002955c     alm_db_output.obj
 0002:0000356c       ??_C@_0CB@CAKMLGGF@alm_db_output?3?3loadProcesses?$CI?$CJ?3?5@ 1002956c     alm_db_output.obj
 0002:00003590       ??_C@_0BC@CGAJBIJG@File?5not?5valid?5?9?5?$AA@ 10029590     alm_db_output.obj
 0002:000035a4       ??_C@_01OHGJGJJP@?$FL?$AA@ 100295a4     alm_db_output.obj
 0002:000035a8       ??_C@_01LBDDMOBJ@?$FN?$AA@ 100295a8     alm_db_output.obj
 0002:000035ac       ??_C@_05MBDCODDP@Group?$AA@ 100295ac     alm_db_output.obj
 0002:000035b4       ??_C@_01NEMOKFLO@?$DN?$AA@ 100295b4     alm_db_output.obj
 0002:000035b8       ??_C@_0CO@HIEKFOCL@alm_db_output?3?3selectFile?$CIQListV@ 100295b8     alm_db_output.obj
 0002:000035e8       ??_C@_0O@DHFAHCBE@No?5file?5found?$AA@ 100295e8     alm_db_output.obj
 0002:000035f8       ??_C@_0BM@BFLMOKII@alm_db_output?3?3loadFile?$CI?$CJ?3?5?$AA@ 100295f8     alm_db_output.obj
 0002:00003614       ??_C@_0CA@HHJMCMFL@?$DMh1?$DOAlarms?5Database?5Output?$DM?1h1?$DO?$AA@ 10029614     alm_db_output.obj
 0002:00003634       ??_C@_0BO@KHKJPMKP@config?1system?1bncs_system?4ini?$AA@ 10029634     alm_db_output.obj
 0002:00003654       ??_C@_09OOGHBKNF@?$FLSystem?$FN?6?$AA@ 10029654     alm_db_output.obj
 0002:00003660       ??_C@_01EEMJAFIK@?6?$AA@   10029660     alm_db_output.obj
 0002:00003664       ??_C@_07GKKGDMMG@dbHost?$DN?$AA@ 10029664     alm_db_output.obj
 0002:0000366c       ??_C@_0M@MCEEBFLD@dbDatabase?$DN?$AA@ 1002966c     alm_db_output.obj
 0002:00003678       ??_C@_07BABCDPB@dbUser?$DN?$AA@ 10029678     alm_db_output.obj
 0002:00003680       ??_C@_0M@EDNAJAME@dbPassword?$DN?$AA@ 10029680     alm_db_output.obj
 0002:0000368c       ??_C@_09IMACPPI@dbDriver?$DN?$AA@ 1002968c     alm_db_output.obj
 0002:00003698       ??_C@_07DNJPNLFF@dbPort?$DN?$AA@ 10029698     alm_db_output.obj
 0002:000036a0       ??_C@_08BDNJMODK@dbHost2?$DN?$AA@ 100296a0     alm_db_output.obj
 0002:000036ac       ??_C@_0N@DDBOKJKA@dbDatabase2?$DN?$AA@ 100296ac     alm_db_output.obj
 0002:000036bc       ??_C@_08KLAPMMCK@dbUser2?$DN?$AA@ 100296bc     alm_db_output.obj
 0002:000036c8       ??_C@_0N@PNPONJLK@dbPassword2?$DN?$AA@ 100296c8     alm_db_output.obj
 0002:000036d8       ??_C@_0L@NCNKLFIC@dbDriver2?$DN?$AA@ 100296d8     alm_db_output.obj
 0002:000036e4       ??_C@_08HKIIDFCD@dbPort2?$DN?$AA@ 100296e4     alm_db_output.obj
 0002:000036f0       ??_C@_0BB@FEEDOMDB@bncs_log_driver?$DN?$AA@ 100296f0     alm_db_output.obj
 0002:00003704       ??_C@_0M@KFAEAMKK@ConfigTool?$DN?$AA@ 10029704     alm_db_output.obj
 0002:00003710       ??_C@_0L@OAOLEFHA@AlmSystem?$DN?$AA@ 10029710     alm_db_output.obj
 0002:0000371c       ??_C@_0BF@CNMAFCJA@Module?$DNalm_db_output?$AA@ 1002971c     alm_db_output.obj
 0002:00003734       ??_C@_02BIKLEMDE@db?$AA@   10029734     alm_db_output.obj
 0002:00003738       ??_C@_05DCIFAFBG@Name?$DN?$AA@ 10029738     alm_db_output.obj
 0002:00003740       ??_C@_02JODFHDIE@?$FN?6?$AA@ 10029740     alm_db_output.obj
 0002:00003744       ??_C@_03LOLECBH@OK?$DN?$AA@ 10029744     alm_db_output.obj
 0002:00003748       ??_C@_05FOGFCLKD@Fail?$DN?$AA@ 10029748     alm_db_output.obj
 0002:00003750       ??_C@_04FLLHENIJ@Ack?$DN?$AA@ 10029750     alm_db_output.obj
 0002:00003758       ??_C@_07COEACMOP@Ignore?$DN?$AA@ 10029758     alm_db_output.obj
 0002:00003760       ??_C@_08JKDGPNPJ@Unknown?$DN?$AA@ 10029760     alm_db_output.obj
 0002:0000376c       ??_C@_08CLNKCCFE@Latched?$DN?$AA@ 1002976c     alm_db_output.obj
 0002:00003778       ??_C@_07KKLKGNLL@Device?$DN?$AA@ 10029778     alm_db_output.obj
 0002:00003780       ??_C@_0L@MGLCCEAJ@UserGroup?$DN?$AA@ 10029780     alm_db_output.obj
 0002:0000378c       ??_C@_06OIEOMJMB@Level?$DN?$AA@ 1002978c     alm_db_output.obj
 0002:00003794       ??_C@_01GEODFPGF@?8?$AA@   10029794     alm_db_output.obj
 0002:00003798       ??_C@_0DE@PIGJJLIF@alm_db_output?3?3selectProcess?5?9?5c@ 10029798     alm_db_output.obj
 0002:000037cc       ??_C@_0BI@MDFPOOBO@New?5name?5already?5exist?4?$AA@ 100297cc     alm_db_output.obj
 0002:000037e4       ??_C@_0BA@PBLBBHIA@Database?5editor?$AA@ 100297e4     alm_db_output.obj
 0002:000037f4       ??_C@_05OEOKGKGJ@?$DM?1h1?$DO?$AA@ 100297f4     alm_db_output.obj
 0002:000037fc       ??_C@_0BO@IDKEIIA@?$DMh1?$DOAlarms?5Database?5Output?5?9?5?$AA@ 100297fc     alm_db_output.obj
 0002:0000381c       ??_C@_0BH@LOOPHGAH@Home?1Alarms?1Processes?0?$AA@ 1002981c     alm_db_output.obj
 0002:00003834       ??_C@_08NCKPMOJE@navigate?$AA@ 10029834     alm_db_output.obj
 0002:00003840       ??_C@_0CE@POGKJFEJ@Failed?5to?5remove?5the?5file?5from?5l@ 10029840     alm_db_output.obj
 0002:00003864       ??_C@_09EHIIFBLM@?1outputs?1?$AA@ 10029864     alm_db_output.obj
 0002:00003870       ??_C@_0BG@KMKMBJP@?$FOal_out_?$CI?2d?$HL4?$HN?$CJ?2?4cfg$?$AA@ 10029870     alm_db_output.obj
 0002:00003888       ??_C@_06NHPJKFDC@Module?$AA@ 10029888     alm_db_output.obj
 0002:00003890       ??_C@_04OCCELDNI@?$CF04d?$AA@ 10029890     alm_db_output.obj
 0002:00003898       ??_C@_0O@GMPFIJO@Copy?5?$CF1?5of?5?$CF2?$AA@ 10029898     alm_db_output.obj
 0002:000038a8       ??_C@_05CFEJGMAI@dirty?$AA@ 100298a8     alm_db_output.obj
 0002:000038b0       ??_C@_0DG@KMJPGEOM@?$DMnobr?$DO?$DMh3?$DOAlarm?5System?5Database?5@ 100298b0     alm_db_output.obj
 0002:000038e8       ??_C@_0CN@IJPOCBJI@?$DMp?$DOWritten?5by?5Mark?5Baldry?0?5Richa@ 100298e8     alm_db_output.obj
 0002:00003918       ??_C@_08NJGCOHDN@Process?7?$AA@ 10029918     alm_db_output.obj
 0002:00003924       ??_C@_07BBJAJOEM@Device?7?$AA@ 10029924     alm_db_output.obj
 0002:0000392c       ??_C@_06GHGFKEJH@Group?7?$AA@ 1002992c     alm_db_output.obj
 0002:00003934       ??_C@_0N@OFOHJIAB@Level?5?$CI0?95?$CJ?7?$AA@ 10029934     alm_db_output.obj
 0002:00003944       ??_C@_03IIIMPHAA@Ok?7?$AA@ 10029944     alm_db_output.obj
 0002:00003948       ??_C@_05OFEPNIFE@Fail?7?$AA@ 10029948     alm_db_output.obj
 0002:00003950       ??_C@_05FLJNCKKJ@Ack?4?7?$AA@ 10029950     alm_db_output.obj
 0002:00003958       ??_C@_07JFGKNPBI@Ignore?7?$AA@ 10029958     alm_db_output.obj
 0002:00003960       ??_C@_08JAPANBKD@Latched?7?$AA@ 10029960     alm_db_output.obj
 0002:0000396c       ??_C@_08CBBMAOAO@Unknown?7?$AA@ 1002996c     alm_db_output.obj
 0002:00003978       ??_C@_01GPOEFGEJ@?7?$AA@   10029978     alm_db_output.obj
 0002:0000397c       ??_C@_06EOHEHIAA@dbHost?$AA@ 1002997c     alm_db_output.obj
 0002:00003984       ??_C@_0L@MLICFIKN@dbDatabase?$AA@ 10029984     alm_db_output.obj
 0002:00003990       ??_C@_06ICDKLLFA@dbUser?$AA@ 10029990     alm_db_output.obj
 0002:00003998       ??_C@_0L@OBBBOCHJ@dbPassword?$AA@ 10029998     alm_db_output.obj
 0002:000039a4       ??_C@_08PFHKJJFM@dbDriver?$AA@ 100299a4     alm_db_output.obj
 0002:000039b0       ??_C@_06BPCGMOHE@dbPort?$AA@ 100299b0     alm_db_output.obj
 0002:000039b8       ??_C@_07ONDOCAAJ@dbHost2?$AA@ 100299b8     alm_db_output.obj
 0002:000039c0       ??_C@_0M@EFNMAJHM@dbDatabase2?$AA@ 100299c0     alm_db_output.obj
 0002:000039cc       ??_C@_07IGJJDPDO@dbUser2?$AA@ 100299cc     alm_db_output.obj
 0002:000039d4       ??_C@_0M@MEEIIMAL@dbPassword2?$AA@ 100299d4     alm_db_output.obj
 0002:000039e0       ??_C@_09IPFIDDDH@dbDriver2?$AA@ 100299e0     alm_db_output.obj
 0002:000039ec       ??_C@_07LKAHMHJK@dbPort2?$AA@ 100299ec     alm_db_output.obj
 0002:000039f4       ??_C@_0BA@MFNDFEOH@bncs_log_driver?$AA@ 100299f4     alm_db_output.obj
 0002:00003a04       ??_C@_04ODLKOBGJ@Fail?$AA@ 10029a04     alm_db_output.obj
 0002:00003a0c       ??_C@_03DBILNIKO@Ack?$AA@  10029a0c     alm_db_output.obj
 0002:00003a10       ??_C@_06KMEJCCGM@Ignore?$AA@ 10029a10     alm_db_output.obj
 0002:00003a18       ??_C@_07NBCGADJA@Unknown?$AA@ 10029a18     alm_db_output.obj
 0002:00003a20       ??_C@_07DGBAIKKL@Latched?$AA@ 10029a20     alm_db_output.obj
 0002:00003a28       ??_C@_06OIEJKIHP@Device?$AA@ 10029a28     alm_db_output.obj
 0002:00003a30       ??_C@_09OGJFPHCL@UserGroup?$AA@ 10029a30     alm_db_output.obj
 0002:00003a3c       ??_C@_05KOHFLOFG@Level?$AA@ 10029a3c     alm_db_output.obj
 0002:00003a44       ??_C@_0N@LJNCPLAD@downloadFile?$AA@ 10029a44     alm_db_output.obj
 0002:00003a54       ??_C@_0M@IKGKPMGN@checkoutDir?$AA@ 10029a54     alm_db_output.obj
 0002:00003a60       ??_C@_08EKDELGFG@?$CFalt_id?$CF?$AA@ 10029a60     alm_db_output.obj
 0002:00003a6c       ??_C@_02PIGFKFFE@?$CF1?$AA@ 10029a6c     alm_db_output.obj
 0002:00003a74       ??_7?$QPtrList@VcProcess@@@@6B@ 10029a74     alm_db_output.obj
 0002:00003a94       ??_C@_01IDAFKMJL@_?$AA@    10029a94     alm_db_output.obj
 0002:00003a98       ??_C@_07JLEKEEPN@?$CGCancel?$AA@ 10029a98     alm_db_output.obj
 0002:00003aa0       ??_C@_09OMIPBCDE@?$CGSelected?$AA@ 10029aa0     alm_db_output.obj
 0002:00003aac       ??_C@_04NMHBPLPB@?$CGAll?$AA@ 10029aac     alm_db_output.obj
 0002:00003ab4       ??_C@_0CN@PBGAEEEL@Do?5you?5want?5to?5Paste?5All?5procs?5o@ 10029ab4     alm_db_output.obj
 0002:00003ae4       ??_C@_0BH@NILMKAJ@Alarms?5Database?5Output?$AA@ 10029ae4     alm_db_output.obj
 0002:00003afc       ??_C@_0BA@JFNIOLAK@string?5too?5long?$AA@ 10029afc     alm_db_output.obj
 0002:00003b0c       ??_C@_0BI@CFPLBAOH@invalid?5string?5position?$AA@ 10029b0c     alm_db_output.obj
 0002:00003b28       ??_7cOutputFile@@6B@       10029b28     cOutputFile.obj
 0002:00003b30       ??_7cProcess@@6B@          10029b30     cProcess.obj
 0002:00003b38       ??_7dbConnection@@6B@      10029b38     DBCONNECTION.obj
 0002:00003b40       ??_C@_08HDBDMMBI@Database?$AA@ 10029b40     DBCONNECTION.obj
 0002:00003b4c       ??_C@_0M@MIMLKFFE@?5to?5driver?5?$AA@ 10029b4c     DBCONNECTION.obj
 0002:00003b58       ??_C@_0BB@BALJNGMD@Adding?5database?5?$AA@ 10029b58     DBCONNECTION.obj
 0002:00003b6c       ??_C@_0P@NNKAJFFA@Open?5database?5?$AA@ 10029b6c     DBCONNECTION.obj
 0002:00003b7c       ??_C@_0BB@LBGJGNLJ@Opened?5database?4?$AA@ 10029b7c     DBCONNECTION.obj
 0002:00003b90       ??_C@_0BB@CPOKEADH@Opened?5database?5?$AA@ 10029b90     DBCONNECTION.obj
 0002:00003ba4       ??_C@_0BJ@IOAKHLHF@Failed?5to?5open?5database?4?$AA@ 10029ba4     DBCONNECTION.obj
 0002:00003bc0       ??_C@_0BJ@BAIJFGPL@Failed?5to?5open?5database?5?$AA@ 10029bc0     DBCONNECTION.obj
 0002:00003bdc       ??_C@_09CGEJCEMB@?5to?5start?$AA@ 10029bdc     DBCONNECTION.obj
 0002:00003be8       ??_C@_0BF@PGFMEGFF@Can?8t?5find?5database?5?$AA@ 10029be8     DBCONNECTION.obj
 0002:00003c00       ??_C@_0O@NPFKCNOE@Unknown?5Error?$AA@ 10029c00     DBCONNECTION.obj
 0002:00003c10       ??_C@_0N@KJKAAMLA@No?5SQL?5error?$AA@ 10029c10     DBCONNECTION.obj
 0002:00003c20       ??_C@_0BF@IJMCAOFE@SQL?5Connection?5error?$AA@ 10029c20     DBCONNECTION.obj
 0002:00003c38       ??_C@_0BH@PHCPCCHG@SQL?5Statement?5error?5?9?5?$AA@ 10029c38     DBCONNECTION.obj
 0002:00003c50       ??_C@_0BG@EONPGLNH@SQL?5Transaction?5error?$AA@ 10029c50     DBCONNECTION.obj
 0002:00003c68       ??_C@_0BA@LICLPFOB@SQL?5other?5error?$AA@ 10029c68     DBCONNECTION.obj
 0002:00003c78       ??_C@_01CLKCMJKC@?5?$AA@   10029c78     DBCONNECTION.obj
 0002:00003c7c       ??_C@_0BJ@IIAAECEJ@sql?5error?5?9?5db?5text?5?5?3?5?8?$AA@ 10029c7c     DBCONNECTION.obj
 0002:00003c98       ??_C@_0BJ@KIFGMMLN@sql?5error?5?9?5drv?5text?5?3?5?8?$AA@ 10029c98     DBCONNECTION.obj
 0002:00003cb4       ??_C@_0BI@EHBJIBNO@sql?5error?5?9?5number?5?5?5?3?5?$AA@ 10029cb4     DBCONNECTION.obj
 0002:00003ccc       ??_C@_0BI@MEKKAFMI@sql?5error?5?9?5text?5?5?5?5?5?3?5?$AA@ 10029ccc     DBCONNECTION.obj
 0002:00003ce8       ??_7dialog@@6BQObject@@@   10029ce8     dialogimpl.obj
 0002:00003ea0       ??_7dialog@@6BQPaintDevice@@@ 10029ea0     dialogimpl.obj
 0002:00003ec4       ??_SQSqlCursor@@6BQSqlRecord@@@ 10029ec4     dialogimpl.obj
 0002:00003f6c       ??_SQSqlCursor@@6BQSqlQuery@@@ 10029f6c     dialogimpl.obj
 0002:00003f9c       ??_SQTimer@@6B@            10029f9c     dialogimpl.obj
 0002:00003fec       ??_C@_07BMAFLFHF@?$DMspace?$DO?$AA@ 10029fec     dialogimpl.obj
 0002:00003ff4       ??_C@_0P@CLNKHPBJ@?$DMunderscore?$DO?5_?$AA@ 10029ff4     dialogimpl.obj
 0002:00004004       ??_C@_0L@EKJJPBII@?$DMhyphen?$DO?5?9?$AA@ 1002a004     dialogimpl.obj
 0002:00004010       ??_C@_08LAIGBKAI@ProcList?$AA@ 1002a010     dialogimpl.obj
 0002:0000401c       ??_C@_08CGIOBMAK@Splitter?$AA@ 1002a01c     dialogimpl.obj
 0002:00004028       ??_C@_08DOGFHPBI@Defaults?$AA@ 1002a028     dialogimpl.obj
 0002:00004034       ??_C@_04LOAJBDKD@true?$AA@ 1002a034     dialogimpl.obj
 0002:0000403c       ??_C@_04DBLCCBDK@?$DMsp?$DO?$AA@ 1002a03c     dialogimpl.obj
 0002:00004044       ??_C@_01JOAMLHOP@?9?$AA@   1002a044     dialogimpl.obj
 0002:00004048       ??_C@_0CC@FFCBGHP@1dbDriverChanged?$CIconst?5QString?5?$CG@ 1002a048     dialogimpl.obj
 0002:0000406c       ??_C@_0CK@ICLJGFE@1dbDriverChanged_reserve?$CIconst?5Q@ 1002a06c     dialogimpl.obj
 0002:00004098       ??_C@_0BJ@NENOIPPG@1showingWidget?$CIQWidget?$CK?$CJ?$AA@ 1002a098     dialogimpl.obj
 0002:000040b4       ??_C@_0BK@EHJILHMI@2currentChanged?$CIQWidget?$CK?$CJ?$AA@ 1002a0b4     dialogimpl.obj
 0002:000040d0       ??_C@_0BD@PMMLDDED@1levelChanged?$CIint?$CJ?$AA@ 1002a0d0     dialogimpl.obj
 0002:000040e4       ??_C@_0BH@DKNLIPIJ@1setGroupDefaultText?$CI?$CJ?$AA@ 1002a0e4     dialogimpl.obj
 0002:000040fc       ??_C@_0M@LPGBGFJN@2clicked?5?$CI?$CJ?$AA@ 1002a0fc     dialogimpl.obj
 0002:00004108       ??_C@_0BF@GHNKFJB@1setAllDefaultText?$CI?$CJ?$AA@ 1002a108     dialogimpl.obj
 0002:00004120       ??_C@_0BA@CDBFBPLP@1clearAllText?$CI?$CJ?$AA@ 1002a120     dialogimpl.obj
 0002:00004130       ??_C@_0BE@NDKJMENJ@1setOkDefaultText?$CI?$CJ?$AA@ 1002a130     dialogimpl.obj
 0002:00004144       ??_C@_0BG@ELLLMMNB@1setFailDefaultText?$CI?$CJ?$AA@ 1002a144     dialogimpl.obj
 0002:0000415c       ??_C@_0BF@BDJGMNLB@1setAckDefaultText?$CI?$CJ?$AA@ 1002a15c     dialogimpl.obj
 0002:00004174       ??_C@_0BI@NOOPLJND@1setIgnoreDefaultText?$CI?$CJ?$AA@ 1002a174     dialogimpl.obj
 0002:0000418c       ??_C@_0BJ@MDBNFDJM@1setUnknownDefaultText?$CI?$CJ?$AA@ 1002a18c     dialogimpl.obj
 0002:000041a8       ??_C@_0BJ@MLCCMDDG@1setLatchedDefaultText?$CI?$CJ?$AA@ 1002a1a8     dialogimpl.obj
 0002:000041c4       ??_C@_0BB@KHGEEKPN@1resetDefaults?$CI?$CJ?$AA@ 1002a1c4     dialogimpl.obj
 0002:000041d8       ??_C@_0BF@GKGFDPMP@1createNewLogTable?$CI?$CJ?$AA@ 1002a1d8     dialogimpl.obj
 0002:000041f0       ??_C@_0BA@KJNINGJK@1clearAllLogs?$CI?$CJ?$AA@ 1002a1f0     dialogimpl.obj
 0002:00004200       ??_C@_0BD@CIGHDOD@1clearLogsBefore?$CI?$CJ?$AA@ 1002a200     dialogimpl.obj
 0002:00004214       ??_C@_0BG@NJGDEPPJ@1createNewProcTable?$CI?$CJ?$AA@ 1002a214     dialogimpl.obj
 0002:0000422c       ??_C@_0BF@FFHKPALO@1clearAllProcesses?$CI?$CJ?$AA@ 1002a22c     dialogimpl.obj
 0002:00004244       ??_C@_0BI@GDCBGJN@1clearProcessesBefore?$CI?$CJ?$AA@ 1002a244     dialogimpl.obj
 0002:0000425c       ??_C@_0BB@GJIPNBEI@1fillDataTable?$CI?$CJ?$AA@ 1002a25c     dialogimpl.obj
 0002:00004270       ??_C@_0BM@EIICMPGC@2activated?$CIconst?5QString?5?$CG?$CJ?$AA@ 1002a270     dialogimpl.obj
 0002:0000428c       ??_C@_0BI@LEMDACFG@1fillDataTableEdit?$CIint?$CJ?$AA@ 1002a28c     dialogimpl.obj
 0002:000042a4       ??_C@_0BJ@IBBAKJEM@1fillDataTableTools?$CIint?$CJ?$AA@ 1002a2a4     dialogimpl.obj
 0002:000042c0       ??_C@_0BO@FHLKKLPM@1itemChanged?$CIconst?5QString?5?$CG?$CJ?$AA@ 1002a2c0     dialogimpl.obj
 0002:000042e0       ??_C@_0BC@ELMOLHPA@1itemChanged?$CIint?$CJ?$AA@ 1002a2e0     dialogimpl.obj
 0002:000042f4       ??_C@_0BD@OIBDOPAP@2valueChanged?$CIint?$CJ?$AA@ 1002a2f4     dialogimpl.obj
 0002:00004308       ??_C@_0BP@NEBIFMCI@2valueChanged?$CIconst?5QString?5?$CG?$CJ?$AA@ 1002a308     dialogimpl.obj
 0002:00004328       ??_C@_0BA@CILBMLGP@1dbToolUpdate?$CI?$CJ?$AA@ 1002a328     dialogimpl.obj
 0002:00004338       ??_C@_0L@CHKJBFLD@2timeout?$CI?$CJ?$AA@ 1002a338     dialogimpl.obj
 0002:00004344       ??_C@_0P@HLKPKBAK@1dbEditStart?$CI?$CJ?$AA@ 1002a344     dialogimpl.obj
 0002:00004354       ??_C@_05NDLFFNHM@paste?$AA@ 1002a354     dialogimpl.obj
 0002:0000435c       ??_C@_06FENKCKDB@?$CGPaste?$AA@ 1002a35c     dialogimpl.obj
 0002:00004364       ??_C@_05NEBJFIEK@Paste?$AA@ 1002a364     dialogimpl.obj
 0002:0000436c       ??_C@_0N@DJHCJEAJ@1pasteData?$CI?$CJ?$AA@ 1002a36c     dialogimpl.obj
 0002:0000437c       ??_C@_04COAGEIMF@copy?$AA@ 1002a37c     dialogimpl.obj
 0002:00004384       ??_C@_05EJNCNHFE@?$CGCopy?$AA@ 1002a384     dialogimpl.obj
 0002:0000438c       ??_C@_04OPMHGHMB@Copy?$AA@ 1002a38c     dialogimpl.obj
 0002:00004394       ??_C@_0M@CPPMHGBO@1copyData?$CI?$CJ?$AA@ 1002a394     dialogimpl.obj
 0002:000043a0       ??_C@_0BA@CHFPLOFG@1pasteOptions?$CI?$CJ?$AA@ 1002a3a0     dialogimpl.obj
 0002:000043b0       ??_C@_01MIFGBAGJ@?$CL?$AA@ 1002a3b0     dialogimpl.obj
 0002:000043b4       ??_C@_05LAPONLG@false?$AA@ 1002a3b4     dialogimpl.obj
 0002:000043bc       ??_C@_01IHBHIGKO@?0?$AA@   1002a3bc     dialogimpl.obj
 0002:000043c0       ??_C@_0BL@FHDOIDCO@?$CF1?0?$CF2?0?$CF3?0?$CF4?0?$CF5?0?$CF6?0?$CF7?0?$CF8?0?$CF9?$AA@ 1002a3c0     dialogimpl.obj
 0002:000043dc       ??_C@_04DKFIAMBL@Ack?4?$AA@ 1002a3dc     dialogimpl.obj
 0002:000043e4       ??_C@_07EFDJMKPC@Ignored?$AA@ 1002a3e4     dialogimpl.obj
 0002:000043ec       ??_C@_07HILCIGEC@dbTools?$AA@ 1002a3ec     dialogimpl.obj
 0002:000043f4       ??_C@_06HAFEBNBG@dbEdit?$AA@ 1002a3f4     dialogimpl.obj
 0002:000043fc       ??_C@_0CE@DPLNHNEH@dbToolsStart?4?5no?5connection?4?5sta@ 1002a3fc     dialogimpl.obj
 0002:00004420       ??_C@_0BN@GLODCJKF@dbToolsStart?4?5no?5connection?4?$AA@ 1002a420     dialogimpl.obj
 0002:00004440       ??_C@_0L@NPJJHNMF@Connecting?$AA@ 1002a440     dialogimpl.obj
 0002:0000444c       ??_C@_05HOPBAMFM@?9?5?9?5?9?$AA@ 1002a44c     dialogimpl.obj
 0002:00004454       ??_C@_0BL@KEDIJCFF@dbToolsEnd?4?5stop?5timer?4?5?$CFx?$AA@ 1002a454     dialogimpl.obj
 0002:00004470       ??_C@_0CE@PNNCIDFF@dbToolUpdate?4?5no?5connection?4?5sta@ 1002a470     dialogimpl.obj
 0002:00004494       ??_C@_0CE@CPGIAIDF@SELECT?5COUNT?$CI?$CK?$CJ?5FROM?5historical_@ 1002a494     dialogimpl.obj
 0002:000044b8       ??_C@_07DJMIGIHO@Invalid?$AA@ 1002a4b8     dialogimpl.obj
 0002:000044c0       ??_C@_0CC@GEMFKHMF@SELECT?5COUNT?$CI?$CK?$CJ?5FROM?5process_dat@ 1002a4c0     dialogimpl.obj
 0002:000044e4       ??_C@_07IMOFFCAA@QMYSQL3?$AA@ 1002a4e4     dialogimpl.obj
 0002:000044ec       ??_C@_02LJALELK@?$CJ?$DL?$AA@ 1002a4ec     dialogimpl.obj
 0002:000044f0       ??_C@_0BP@EPDKCFKE@?5PRIMARY?5KEY?5?5?$CI?$GAindex_number?$GA?$CJ?$AA@ 1002a4f0     dialogimpl.obj
 0002:00004510       ??_C@_0CH@BFICMLMJ@?5?$GAprocess_id?$GA?5varchar?$CI100?$CJ?5defau@ 1002a510     dialogimpl.obj
 0002:00004538       ??_C@_0CG@PBPMDECA@?5?$GAusergroup?$GA?5varchar?$CI100?$CJ?5defaul@ 1002a538     dialogimpl.obj
 0002:00004560       ??_C@_0BN@HLHKIJBD@?5?$GAstate?$GA?5int?$CI1?$CJ?5default?5?80?8?0?$AA@ 1002a560     dialogimpl.obj
 0002:00004580       ??_C@_0BN@ILNFCHIL@?5?$GAlevel?$GA?5int?$CI1?$CJ?5default?5?80?8?0?$AA@ 1002a580     dialogimpl.obj
 0002:000045a0       ??_C@_0CB@KBGKKGMN@?5?$GAtext?$GA?5varchar?$CI100?$CJ?5default?5?8?8?0@ 1002a5a0     dialogimpl.obj
 0002:000045c4       ??_C@_0CJ@ODHKNBJD@?5?$GAdevice_name?$GA?5varchar?$CI100?$CJ?5defa@ 1002a5c4     dialogimpl.obj
 0002:000045f0       ??_C@_0CF@BOIKBOND@?5?$GAmSec?$GA?5int?$CI3?$CJ?5NOT?5NULL?5default?5@ 1002a5f0     dialogimpl.obj
 0002:00004618       ??_C@_0DO@DILKHBFL@?5?$GAdate_time?$GA?5datetime?5NOT?5NULL?5d@ 1002a618     dialogimpl.obj
 0002:00004658       ??_C@_0DJ@CGKOIPFK@?5?$GAindex_number?$GA?5int?$CI8?$CJ?5unsigned?5@ 1002a658     dialogimpl.obj
 0002:00004694       ??_C@_0CA@GIENLFGJ@CREATE?5TABLE?5?$GAhistorical_log?$GA?5?$CI?$AA@ 1002a694     dialogimpl.obj
 0002:000046b4       ??_C@_06DOGECKN@QODBC3?$AA@ 1002a6b4     dialogimpl.obj
 0002:000046bc       ??_C@_0BN@BPDMGBBE@?5PRIMARY?5KEY?5?5?$CIindex_number?$CJ?$AA@ 1002a6bc     dialogimpl.obj
 0002:000046dc       ??_C@_0CF@NCKMOOOJ@?5process_id?5varchar?$CI100?$CJ?5default@ 1002a6dc     dialogimpl.obj
 0002:00004704       ??_C@_0CE@EENIINKF@?5usergroup?5varchar?$CI100?$CJ?5default?5@ 1002a704     dialogimpl.obj
 0002:00004728       ??_C@_0BI@HGCPIEK@?5state?5int?5default?5?80?8?0?$AA@ 1002a728     dialogimpl.obj
 0002:00004740       ??_C@_0BI@LHCOBCAF@?5level?5int?5default?5?80?8?0?$AA@ 1002a740     dialogimpl.obj
 0002:00004758       ??_C@_0BP@CLGKLBOB@?5text?5varchar?$CI100?$CJ?5default?5?8?8?0?$AA@ 1002a758     dialogimpl.obj
 0002:00004778       ??_C@_0CH@LEPGNFHL@?5device_name?5varchar?$CI100?$CJ?5defaul@ 1002a778     dialogimpl.obj
 0002:000047a0       ??_C@_0CA@DNDAJOFD@?5mSec?5int?5NOT?5NULL?5default?5?80?8?0?$AA@ 1002a7a0     dialogimpl.obj
 0002:000047c0       ??_C@_0DM@ODKCMKJG@?5date_time?5datetime?5NOT?5NULL?5def@ 1002a7c0     dialogimpl.obj
 0002:000047fc       ??_C@_0CL@OKMKMNJG@?5index_number?5INT?5NOT?5NULL?5?5IDEN@ 1002a7fc     dialogimpl.obj
 0002:00004828       ??_C@_0BP@JGECIFIE@CREATE?5TABLE?5historical_log?5?5?$CI?$AA@ 1002a828     dialogimpl.obj
 0002:00004848       ??_C@_0BL@INDDHLHE@?5PRIMARY?5KEY?5?5?$CIprocess_id?$CJ?$AA@ 1002a848     dialogimpl.obj
 0002:00004864       ??_C@_0CA@BHDNCAJJ@?5current_level?5int?5default?5?80?8?0?$AA@ 1002a864     dialogimpl.obj
 0002:00004884       ??_C@_0CG@DFCOEMCB@?5device_name?5varchar?$CI100?$CJ?5defaul@ 1002a884     dialogimpl.obj
 0002:000048ac       ??_C@_0CH@CAJLPPFI@?5current_text?5varchar?$CI100?$CJ?5defau@ 1002a8ac     dialogimpl.obj
 0002:000048d4       ??_C@_0CA@KHHBMKNG@?5current_state?5int?5default?5?80?8?0?$AA@ 1002a8d4     dialogimpl.obj
 0002:000048f4       ??_C@_0DM@IHHEOGEC@?5date_time?5datetime?5NOT?5NULL?5def@ 1002a8f4     dialogimpl.obj
 0002:00004930       ??_C@_0CP@MOEPHHLM@?5process_id?5varchar?$CI100?$CJ?5NOT?5NUL@ 1002a930     dialogimpl.obj
 0002:00004960       ??_C@_0BM@IIONCEGL@CREATE?5TABLE?5process_data?5?$CI?$AA@ 1002a960     dialogimpl.obj
 0002:0000497c       ??_C@_0BL@PAKCCOCB@DELETE?5FROM?5historical_log?$AA@ 1002a97c     dialogimpl.obj
 0002:00004998       ??_C@_0CO@CKLBODJF@DELETE?5FROM?5historical_log?5WHERE@ 1002a998     dialogimpl.obj
 0002:000049c8       ??_C@_0L@FFIMBEKI@yyyy?9MM?9dd?$AA@ 1002a9c8     dialogimpl.obj
 0002:000049d4       ??_C@_0L@JCGGBBH@?500?300?300?8?$AA@ 1002a9d4     dialogimpl.obj
 0002:000049e0       ??_C@_0BJ@KHFOFEKL@DELETE?5FROM?5process_data?$AA@ 1002a9e0     dialogimpl.obj
 0002:000049fc       ??_C@_0CM@GINICMKN@DELETE?5FROM?5process_data?5WHERE?5d@ 1002a9fc     dialogimpl.obj
 0002:00004a28       ??_C@_0O@ODFBCHC@No?5Connection?$AA@ 1002aa28     dialogimpl.obj
 0002:00004a38       ??_C@_09NJLBODLJ@Connected?$AA@ 1002aa38     dialogimpl.obj
 0002:00004a44       ??_C@_0BN@LFCCLANH@dialog?3?3dbStartConnect?$CI?$CJ?4?5?$CFx?$AA@ 1002aa44     dialogimpl.obj
 0002:00004a64       ??_C@_0CD@PEABEOEH@dbEditStart?4?5no?5connection?4?5star@ 1002aa64     dialogimpl.obj
 0002:00004a88       ??_C@_0BM@EEKOFAB@dbEditStart?4?5no?5connection?4?$AA@ 1002aa88     dialogimpl.obj
 0002:00004aa4       ??_C@_0O@IIKJJNKF@No?5connection?$AA@ 1002aaa4     dialogimpl.obj
 0002:00004ab4       ??_C@_03MDIDAHKD@?$CGNo?$AA@ 1002aab4     dialogimpl.obj
 0002:00004ab8       ??_C@_04ILFHLBJA@?$CGYes?$AA@ 1002aab8     dialogimpl.obj
 0002:00004ac0       ??_C@_0EG@JCAEPHHD@Selected?5Area?5does?5not?5match?4?6Do@ 1002aac0     dialogimpl.obj
 0002:00004b08       ??_C@_0BB@LNOIOJNO@Database?5Edtitor?$AA@ 1002ab08     dialogimpl.obj
 0002:00004b1c       ??_C@_0BA@NKFGFPDM@No?5record?5found?$AA@ 1002ab1c     dialogimpl.obj
 0002:00004b30       ??_C@_0FE@LMLMPEGJ@Unable?5to?5update?5all?5records?4?6Ch@ 1002ab30     dialogimpl.obj
 0002:00004b8c       ??_SQCheckTableItem@@6B@   1002ab8c     manage_tempimpl.obj
 0002:00004bdc       ??_7manage_temp@@6BQObject@@@ 1002abdc     manage_tempimpl.obj
 0002:00004da0       ??_7manage_temp@@6BQPaintDevice@@@ 1002ada0     manage_tempimpl.obj
 0002:00004dc0       ??_C@_0BP@DNDFBBBF@1prefixChanged?$CIconst?5QString?$CG?$CJ?$AA@ 1002adc0     manage_tempimpl.obj
 0002:00004de0       ??_C@_0BN@HELOKIBG@2textChanged?$CIconst?5QString?$CG?$CJ?$AA@ 1002ade0     manage_tempimpl.obj
 0002:00004e00       ??_C@_0BP@DGHGKHCM@1selectProcess?$CIQListViewItem?$CK?$CJ?$AA@ 1002ae00     manage_tempimpl.obj
 0002:00004e20       ??_C@_0CA@PAGEECMI@2currentChanged?$CIQListViewItem?$CK?$CJ?$AA@ 1002ae20     manage_tempimpl.obj
 0002:00004e40       ??_C@_0BL@LFHECKMJ@1setAllParamsDefaultText?$CI?$CJ?$AA@ 1002ae40     manage_tempimpl.obj
 0002:00004e5c       ??_C@_0BG@DENAFDFL@1clearAllParamsText?$CI?$CJ?$AA@ 1002ae5c     manage_tempimpl.obj
 0002:00004e74       ??_C@_0BI@MKIDFDJM@1setDeviceDefaultText?$CI?$CJ?$AA@ 1002ae74     manage_tempimpl.obj
 0002:00004e8c       ??_C@_0BH@MOPGFHEM@1setLevelDefaultText?$CI?$CJ?$AA@ 1002ae8c     manage_tempimpl.obj
 0002:00004ea4       ??_C@_0BB@POOMLMGO@2activated?5?$CIint?$CJ?$AA@ 1002aea4     manage_tempimpl.obj
 0002:00004eb8       ??_C@_0BG@NIEHCODN@1selectAllInstances?$CI?$CJ?$AA@ 1002aeb8     manage_tempimpl.obj
 0002:00004ed0       ??_C@_0BI@OLFMPPCA@1deselectAllInstances?$CI?$CJ?$AA@ 1002aed0     manage_tempimpl.obj
 0002:00004ee8       ??_C@_0BL@JEPDDKNC@1selectSelectedInstances?$CI?$CJ?$AA@ 1002aee8     manage_tempimpl.obj
 0002:00004f04       ??_C@_0BN@HGHDJOLM@1deselectSelectedInstances?$CI?$CJ?$AA@ 1002af04     manage_tempimpl.obj
 0002:00004f24       ??_C@_07EHMCOPMF@PosSize?$AA@ 1002af24     manage_tempimpl.obj
 0002:00004f2c       ??_C@_0CO@NCPOMDBI@Home?1Alarms?1Outputs?1Database?1Man@ 1002af2c     manage_tempimpl.obj
 0002:00004f5c       ??_C@_09LALMMIOK@ListSlots?$AA@ 1002af5c     manage_tempimpl.obj
 0002:00004f68       ??_C@_0O@LNDMEONL@TableInstance?$AA@ 1002af68     manage_tempimpl.obj
 0002:00004f78       ??_C@_0CD@BFHHIOMP@manage_temp?3?3prefixChanged?5to?5?8?$CF@ 1002af78     manage_tempimpl.obj
 0002:00004f9c       ??_C@_0DM@GKECHOCK@check?5proc?5list?5for?5param?5?8?$CFs?8?4?5@ 1002af9c     manage_tempimpl.obj
 0002:00004fd8       ??_C@_0DC@INOGGAPN@proc?5map?5doesn?8t?5contain?5?8?$CFs?8?4?5F@ 1002afd8     manage_tempimpl.obj
 0002:0000500c       ??_C@_0CH@JLKPDKOJ@add?5to?5available?5indexes?4?5prefix@ 1002b00c     manage_tempimpl.obj
 0002:00005034       ??_C@_08KLEPBNHL@Selected?$AA@ 1002b034     manage_tempimpl.obj
 0002:00005040       ??_C@_0P@PJIGAHMH@1itemChanged?$CI?$CJ?$AA@ 1002b040     manage_tempimpl.obj
 0002:00005050       ??_C@_0BP@DPPANLBE@2textChanged?5?$CIconst?5QString?5?$CG?$CJ?$AA@ 1002b050     manage_tempimpl.obj
 0002:00005070       ??_C@_0BM@LNAMPNMP@manage_temp?3?3setProcess?5?9?5?8?$AA@ 1002b070     manage_tempimpl.obj
 0002:0000508c       ??_C@_0BA@GLGEMNPK@setDefaultsBase?$AA@ 1002b08c     moc_setdefaults.obj
 0002:000050a8       ??_C@_0P@DMEOIADN@languageChange?$AA@ 1002b0a8     moc_setdefaults.obj
 0002:000050c4       ??_C@_0BB@PFEIHPGD@languageChange?$CI?$CJ?$AA@ 1002b0c4     moc_setdefaults.obj
 0002:000050d8       ??_C@_0M@COEMOBEF@setDefaults?$AA@ 1002b0d8     moc_setdefaultsimpl.obj
 0002:000050e4       ??_C@_0CD@BFGBAEB@?5?5?5?514?5?5?5?514?5?5?5?5?5?5?5?54?5?5?5?5?5?5?5?5?5?5?5@ 1002b0e4     plugindesc.obj
 0002:00005108       ??_C@_0M@EKMPMHDK@?4?5c?5?$CD040404?$AA@ 1002b108     plugindesc.obj
 0002:00005114       ??_C@_0M@NBLJLJNN@?$CD?5c?5?$CD808304?$AA@ 1002b114     plugindesc.obj
 0002:00005120       ??_C@_0M@EAFJJBBG@a?5c?5?$CDbfc2bf?$AA@ 1002b120     plugindesc.obj
 0002:0000512c       ??_C@_08PBKCALNO@b?5c?5None?$AA@ 1002b12c     plugindesc.obj
 0002:00005138       ??_C@_0P@HFKAALMG@?4?4?4?4?4?4?4?4?4?4?4?4?4?4?$AA@ 1002b138     plugindesc.obj
 0002:00005148       ??_C@_0P@LGBCEGMD@?4?$CD?4aaaaaaaa?4a?4?$AA@ 1002b148     plugindesc.obj
 0002:00005158       ??_C@_0P@MNNEIMDO@?4?$CD?4aaaaaaaa?4?4?4?$AA@ 1002b158     plugindesc.obj
 0002:00005168       ??_C@_0P@MFAMBPGN@?4?$CD?4aaaaaaaa?4?$CD?4?$AA@ 1002b168     plugindesc.obj
 0002:00005178       ??_C@_0P@HPMEFAGN@?4?$CD?$CD?4?4?4?4?4?4?4?4?$CD?$CD?4?$AA@ 1002b178     plugindesc.obj
 0002:00005188       ??_C@_0P@JAJCNDBN@?4?$CD?$CD?$CD?$CD?$CD?$CD?$CD?$CD?$CD?$CD?$CD?$CD?4?$AA@ 1002b188     plugindesc.obj
 0002:00005198       ??_C@_0P@INKOIILA@?4?$CD?$CD?4?4?4?4?4?4?4?4?4?$CD?4?$AA@ 1002b198     plugindesc.obj
 0002:000051a8       ??_C@_0P@KJADPPJB@?4?$CD?$CD?4?4?4?4?4?4aa?4?$CD?4?$AA@ 1002b1a8     plugindesc.obj
 0002:000051b8       ??_C@_0P@PKKONJFP@b?4?4?4?4?4?4?4?4?4?4?4?4?4?$AA@ 1002b1b8     plugindesc.obj
 0002:000051cc       ??_7config_plugin_desc_base@@6B@ 1002b1cc     plugindesc.obj
 0002:000051e0       ??_7plugindesc@@6B@        1002b1e0     plugindesc.obj
 0002:000051f0       ??_C@_0BN@MCDBKCAE@Home?1Alarms?1Outputs?1Database?$AA@ 1002b1f0     plugindesc.obj
 0002:00005214       ??_7processList@@6B@       1002b214     processList.obj
 0002:0000521c       ??_7setDefaultsBase@@6BQObject@@@ 1002b21c     setdefaults.obj
 0002:000053e0       ??_7setDefaultsBase@@6BQPaintDevice@@@ 1002b3e0     setdefaults.obj
 0002:00005404       ??_SQPushButton@@6BQObject@@@ 1002b404     setdefaults.obj
 0002:000055f4       ??_SQPushButton@@6BQPaintDevice@@@ 1002b5f4     setdefaults.obj
 0002:0000561c       ??_SQGroupBox@@6BQObject@@@ 1002b61c     setdefaults.obj
 0002:000057fc       ??_SQGroupBox@@6BQPaintDevice@@@ 1002b7fc     setdefaults.obj
 0002:00005824       ??_SQLabel@@6BQObject@@@   1002b824     setdefaults.obj
 0002:00005a1c       ??_SQLabel@@6BQPaintDevice@@@ 1002ba1c     setdefaults.obj
 0002:00005a44       ??_SQLineEdit@@6BQObject@@@ 1002ba44     setdefaults.obj
 0002:00005c6c       ??_SQLineEdit@@6BQPaintDevice@@@ 1002bc6c     setdefaults.obj
 0002:00005c94       ??_SQComboBox@@6BQObject@@@ 1002bc94     setdefaults.obj
 0002:00005e78       ??_SQComboBox@@6BQPaintDevice@@@ 1002be78     setdefaults.obj
 0002:00005e9c       ??_SQCheckBox@@6BQObject@@@ 1002be9c     setdefaults.obj
 0002:0000607c       ??_SQCheckBox@@6BQPaintDevice@@@ 1002c07c     setdefaults.obj
 0002:000060a4       ??_SQSpacerItem@@6B@       1002c0a4     setdefaults.obj
 0002:000060ec       ??_SQGridLayout@@6BQObject@@@ 1002c0ec     setdefaults.obj
 0002:0000615c       ??_SQGridLayout@@6BQLayoutItem@@@ 1002c15c     setdefaults.obj
 0002:000061a4       ??_SQHBoxLayout@@6BQObject@@@ 1002c1a4     setdefaults.obj
 0002:0000620c       ??_SQHBoxLayout@@6BQLayoutItem@@@ 1002c20c     setdefaults.obj
 0002:00006254       ??_SQVBoxLayout@@6BQObject@@@ 1002c254     setdefaults.obj
 0002:000062bc       ??_SQVBoxLayout@@6BQLayoutItem@@@ 1002c2bc     setdefaults.obj
 0002:000062fc       ??_C@_0BG@JLKHOCNA@setDefaultsBaseLayout?$AA@ 1002c2fc     setdefaults.obj
 0002:00006314       ??_C@_0M@INIPOPME@deviceGroup?$AA@ 1002c314     setdefaults.obj
 0002:00006320       ??_C@_0N@LBCDIEML@textLabel3_6?$AA@ 1002c320     setdefaults.obj
 0002:00006330       ??_C@_0P@MHCJFCDE@textLabel3_2_2?$AA@ 1002c330     setdefaults.obj
 0002:00006340       ??_C@_0P@HPJFDFFB@textLabel3_3_2?$AA@ 1002c340     setdefaults.obj
 0002:00006350       ??_C@_0L@MFMDFGPD@deviceEdit?$AA@ 1002c350     setdefaults.obj
 0002:0000635c       ??_C@_09GFKANILJ@groupEdit?$AA@ 1002c35c     setdefaults.obj
 0002:00006368       ??_C@_0L@FMAIGIGP@levelCombo?$AA@ 1002c368     setdefaults.obj
 0002:00006374       ??_C@_0P@BNBJGKGA@checkSetDevice?$AA@ 1002c374     setdefaults.obj
 0002:00006384       ??_C@_0BB@DBEIABFI@checkClearDevice?$AA@ 1002c384     setdefaults.obj
 0002:00006398       ??_C@_0BA@BGMBBING@checkClearGroup?$AA@ 1002c398     setdefaults.obj
 0002:000063a8       ??_C@_0O@JODEKLGI@checkSetGroup?$AA@ 1002c3a8     setdefaults.obj
 0002:000063b8       ??_C@_0BA@HJIGEFLP@checkClearLevel?$AA@ 1002c3b8     setdefaults.obj
 0002:000063c8       ??_C@_0O@PBHDPGAB@checkSetLevel?$AA@ 1002c3c8     setdefaults.obj
 0002:000063d8       ??_C@_0N@JHNILLN@logTextGroup?$AA@ 1002c3d8     setdefaults.obj
 0002:000063e8       ??_C@_0N@MMFEHAIO@textLabel3_3?$AA@ 1002c3e8     setdefaults.obj
 0002:000063f8       ??_C@_0L@JMAFEMDM@checkSetOk?$AA@ 1002c3f8     setdefaults.obj
 0002:00006404       ??_C@_0P@FJBJOAHD@checkSetIgnore?$AA@ 1002c404     setdefaults.obj
 0002:00006414       ??_C@_0N@IDBFOGEJ@textLabel3_4?$AA@ 1002c414     setdefaults.obj
 0002:00006424       ??_C@_0BA@EGOOJCEC@checkClearLatch?$AA@ 1002c424     setdefaults.obj
 0002:00006434       ??_C@_0BC@HEPFLHFC@checkClearUnknown?$AA@ 1002c434     setdefaults.obj
 0002:00006448       ??_C@_0N@OAHKLOFA@checkSetFail?$AA@ 1002c448     setdefaults.obj
 0002:00006458       ??_C@_0O@MOBLCBPM@checkSetLatch?$AA@ 1002c458     setdefaults.obj
 0002:00006468       ??_C@_0N@NFEPEBMP@textLabel3_2?$AA@ 1002c468     setdefaults.obj
 0002:00006478       ??_C@_0N@JKAONHAI@textLabel3_5?$AA@ 1002c478     setdefaults.obj
 0002:00006488       ??_C@_0BB@HFEIILEL@checkClearIgnore?$AA@ 1002c488     setdefaults.obj
 0002:0000649c       ??_C@_0N@KIDILFIK@textLabel3_7?$AA@ 1002c49c     setdefaults.obj
 0002:000064ac       ??_C@_0M@EHDGONCM@checkSetAck?$AA@ 1002c4ac     setdefaults.obj
 0002:000064b8       ??_C@_0O@MMJHEPDG@checkClearAck?$AA@ 1002c4b8     setdefaults.obj
 0002:000064c8       ??_C@_0P@BNJDOGII@checkClearFail?$AA@ 1002c4c8     setdefaults.obj
 0002:000064d8       ??_C@_0BA@FMNLFOKH@checkSetUnknown?$AA@ 1002c4d8     setdefaults.obj
 0002:000064e8       ??_C@_07IOCLMCHC@ackText?$AA@ 1002c4e8     setdefaults.obj
 0002:000064f0       ??_C@_0L@OCKEKFEN@ignoreText?$AA@ 1002c4f0     setdefaults.obj
 0002:000064fc       ??_C@_08JLAMJOGN@failText?$AA@ 1002c4fc     setdefaults.obj
 0002:00006508       ??_C@_0M@DLFLLHEC@latchedText?$AA@ 1002c508     setdefaults.obj
 0002:00006514       ??_C@_0M@EFOHAOED@unknownText?$AA@ 1002c514     setdefaults.obj
 0002:00006520       ??_C@_09NOOIEFAK@failText2?$AA@ 1002c520     setdefaults.obj
 0002:0000652c       ??_C@_0N@HFJJCPHK@latchedText2?$AA@ 1002c52c     setdefaults.obj
 0002:0000653c       ??_C@_08FDPFGPKD@ackText2?$AA@ 1002c53c     setdefaults.obj
 0002:00006548       ??_C@_0N@COAKDFF@unknownText2?$AA@ 1002c548     setdefaults.obj
 0002:00006558       ??_C@_0M@OFPPMNPJ@ignoreText2?$AA@ 1002c558     setdefaults.obj
 0002:00006564       ??_C@_0N@CPKAKJEF@textLabel3_8?$AA@ 1002c564     setdefaults.obj
 0002:00006574       ??_C@_06KNIEAIDE@okText?$AA@ 1002c574     setdefaults.obj
 0002:0000657c       ??_C@_07MMGJCEMM@okText2?$AA@ 1002c57c     setdefaults.obj
 0002:00006584       ??_C@_0L@JEIDOJGL@textLabel3?$AA@ 1002c584     setdefaults.obj
 0002:00006590       ??_C@_0N@IDBPLMGG@checkClearOk?$AA@ 1002c590     setdefaults.obj
 0002:000065a0       ??_C@_0L@FMBOONKA@checkAltId?$AA@ 1002c5a0     setdefaults.obj
 0002:000065ac       ??_C@_08GNEFAENG@layout15?$AA@ 1002c5ac     setdefaults.obj
 0002:000065b8       ??_C@_08DKBDHOFF@buttonOk?$AA@ 1002c5b8     setdefaults.obj
 0002:000065c4       ??_C@_0N@OLKBNHFJ@buttonCancel?$AA@ 1002c5c4     setdefaults.obj
 0002:000065d4       ??_C@_09DMINLBG@1accept?$CI?$CJ?$AA@ 1002c5d4     setdefaults.obj
 0002:000065e0       ??_C@_09OCDCAEKE@1reject?$CI?$CJ?$AA@ 1002c5e0     setdefaults.obj
 0002:000065ec       ??_C@_0BD@PLBAHKNL@1setDisabled?$CIbool?$CJ?$AA@ 1002c5ec     setdefaults.obj
 0002:00006600       ??_C@_0P@POCECEMJ@2toggled?$CIbool?$CJ?$AA@ 1002c600     setdefaults.obj
 0002:00006610       ??_C@_0BC@DLEJKFKG@1setEnabled?$CIbool?$CJ?$AA@ 1002c610     setdefaults.obj
 0002:00006624       ??_C@_0BH@JCNFIBJO@Set?5Selected?5Processes?$AA@ 1002c624     setdefaults.obj
 0002:0000663c       ??_C@_0P@PAHPFFKL@Device?5Details?$AA@ 1002c63c     setdefaults.obj
 0002:0000664c       ??_C@_03CEMDFJG@Set?$AA@   1002c64c     setdefaults.obj
 0002:00006650       ??_C@_05MDNHABIA@Clear?$AA@ 1002c650     setdefaults.obj
 0002:00006658       ??_C@_0M@LDMCKHDB@Text?5to?5Log?$AA@ 1002c658     setdefaults.obj
 0002:00006664       ??_C@_05ILNFHAJH@?5ack?4?$AA@ 1002c664     setdefaults.obj
 0002:0000666c       ??_C@_07GCMMHJLB@?5ignore?$AA@ 1002c66c     setdefaults.obj
 0002:00006674       ??_C@_05FCDHJNOF@?5fail?$AA@ 1002c674     setdefaults.obj
 0002:0000667c       ??_C@_08MOLMKBJJ@?5latched?$AA@ 1002c67c     setdefaults.obj
 0002:00006688       ??_C@_08CJIKCIKC@?5unknown?$AA@ 1002c688     setdefaults.obj
 0002:00006694       ??_C@_0BK@JECLKGBH@?4?4?4?5?$CL?5Process?5Name?5?$CL?5?4?4?4?4?$AA@ 1002c694     setdefaults.obj
 0002:000066b0       ??_C@_03BGMCNDOO@?5OK?$AA@ 1002c6b0     setdefaults.obj
 0002:000066b4       ??_C@_02PNHBFOHM@Ok?$AA@   1002c6b4     setdefaults.obj
 0002:000066b8       ??_C@_0BC@NLHOIKDG@Use?5device?5Alt_Id?$AA@ 1002c6b8     setdefaults.obj
 0002:000066cc       ??_C@_03DDKJIMDC@?$CGOK?$AA@ 1002c6cc     setdefaults.obj
 0002:000066d0       ??_C@_05HBFPNANJ@Alt?$CLO?$AA@ 1002c6d0     setdefaults.obj
 0002:000066d8       ??_C@_05NNOKJPNF@Alt?$CLC?$AA@ 1002c6d8     setdefaults.obj
 0002:000066e4       ??_7setDefaults@@6BQObject@@@ 1002c6e4     setdefaultsimpl.obj
 0002:000068a8       ??_7setDefaults@@6BQPaintDevice@@@ 1002c8a8     setdefaultsimpl.obj
 0002:000068c8       ??_C@_07PGIDBGNN@Not?5set?$AA@ 1002c8c8     setdefaultsimpl.obj
 0002:000068d0       ??_C@_0BA@MIGPEEKI@1?5?9?5Information?$AA@ 1002c8d0     setdefaultsimpl.obj
 0002:000068e0       ??_C@_0BC@GHPAKMAA@2?5?9?5Minor?5Warning?$AA@ 1002c8e0     setdefaultsimpl.obj
 0002:000068f4       ??_C@_0BC@NBKHPCPD@3?5?9?5Major?5Warning?$AA@ 1002c8f4     setdefaultsimpl.obj
 0002:00006908       ??_C@_0BA@DFLHBHF@4?5?9?5Minor?5Alarm?$AA@ 1002c908     setdefaultsimpl.obj
 0002:00006918       ??_C@_0BA@BOBLKBNL@5?5?9?5Major?5Alarm?$AA@ 1002c918     setdefaultsimpl.obj
 0002:0000692c       ??_7dialogBase@@6BQObject@@@ 1002c92c     dialog.obj
 0002:00006ae4       ??_7dialogBase@@6BQPaintDevice@@@ 1002cae4     dialog.obj
 0002:00006b0c       ??_SQSpinBox@@6BQObject@@@ 1002cb0c     dialog.obj
 0002:00006d04       ??_SQSpinBox@@6BQPaintDevice@@@ 1002cd04     dialog.obj
 0002:00006d28       ??_SQSpinBox@@6B@          1002cd28     dialog.obj
 0002:00006d3c       ??_SQButtonGroup@@6BQObject@@@ 1002cd3c     dialog.obj
 0002:00006f2c       ??_SQButtonGroup@@6BQPaintDevice@@@ 1002cf2c     dialog.obj
 0002:00006f54       ??_SQSplitter@@6BQObject@@@ 1002cf54     dialog.obj
 0002:0000713c       ??_SQSplitter@@6BQPaintDevice@@@ 1002d13c     dialog.obj
 0002:00007164       ??_SQRadioButton@@6BQObject@@@ 1002d164     dialog.obj
 0002:00007348       ??_SQRadioButton@@6BQPaintDevice@@@ 1002d348     dialog.obj
 0002:0000736c       ??_SQDateEdit@@6BQObject@@@ 1002d36c     dialog.obj
 0002:00007568       ??_SQDateEdit@@6BQPaintDevice@@@ 1002d568     dialog.obj
 0002:0000758c       ??_SQDataTable@@6BQObject@@@ 1002d58c     dialog.obj
 0002:000079ac       ??_SQDataTable@@6BQPaintDevice@@@ 1002d9ac     dialog.obj
 0002:000079cc       ??_C@_0L@BCEAHFEK@dialogBase?$AA@ 1002d9cc     dialog.obj
 0002:000079d8       ??_C@_0BB@NFKKNJMG@dialogBaseLayout?$AA@ 1002d9d8     dialog.obj
 0002:000079ec       ??_C@_08JLKJJNLG@topLabel?$AA@ 1002d9ec     dialog.obj
 0002:000079f8       ??_C@_09DMIEKCOP@tabWidget?$AA@ 1002d9f8     dialog.obj
 0002:00007a04       ??_C@_0N@EFMDMCJD@systemLayout?$AA@ 1002da04     dialog.obj
 0002:00007a14       ??_C@_08MFHNDHGI@layout79?$AA@ 1002da14     dialog.obj
 0002:00007a20       ??_C@_08NMGGAGCJ@layout78?$AA@ 1002da20     dialog.obj
 0002:00007a2c       ??_C@_09MGDBFGCJ@groupBox7?$AA@ 1002da2c     dialog.obj
 0002:00007a38       ??_C@_0N@CJBMCOMC@textLabel1_4?$AA@ 1002da38     dialog.obj
 0002:00007a48       ??_C@_0N@HPEGIJEE@textLabel1_2?$AA@ 1002da48     dialog.obj
 0002:00007a58       ??_C@_0N@GGFNLIAF@textLabel1_3?$AA@ 1002da58     dialog.obj
 0002:00007a68       ??_C@_0P@DCFNJEFK@textLabel1_3_2?$AA@ 1002da68     dialog.obj
 0002:00007a78       ??_C@_0BB@DNKGONCC@textLabel1_3_2_2?$AA@ 1002da78     dialog.obj
 0002:00007a8c       ??_C@_08NLHBPEGP@password?$AA@ 1002da8c     dialog.obj
 0002:00007a98       ??_C@_08ODGEKKOL@username?$AA@ 1002da98     dialog.obj
 0002:00007aa4       ??_C@_08PBOCEOLL@database?$AA@ 1002daa4     dialog.obj
 0002:00007ab0       ??_C@_08IGGJEOEE@hostName?$AA@ 1002dab0     dialog.obj
 0002:00007abc       ??_C@_06NCODBMHO@driver?$AA@ 1002dabc     dialog.obj
 0002:00007ac4       ??_C@_0N@JMDNNJBI@m_pqSpinPort?$AA@ 1002dac4     dialog.obj
 0002:00007ad4       ??_C@_0N@DAAHBPID@textLabel1_5?$AA@ 1002dad4     dialog.obj
 0002:00007ae4       ??_C@_0M@EMNOJAOH@groupBox7_2?$AA@ 1002dae4     dialog.obj
 0002:00007af0       ??_C@_0P@BHDGMLIG@textLabel1_5_2?$AA@ 1002daf0     dialog.obj
 0002:00007b00       ??_C@_0P@KPIKKMOD@textLabel1_4_2?$AA@ 1002db00     dialog.obj
 0002:00007b10       ??_C@_0P@CLEGKFBL@textLabel1_3_3?$AA@ 1002db10     dialog.obj
 0002:00007b20       ??_C@_0BB@CELNNMGD@textLabel1_3_2_3?$AA@ 1002db20     dialog.obj
 0002:00007b34       ??_C@_0BD@PDJJNILP@textLabel1_3_2_2_2?$AA@ 1002db34     dialog.obj
 0002:00007b48       ??_C@_0BB@GIBFCDLM@password_reserve?$AA@ 1002db48     dialog.obj
 0002:00007b5c       ??_C@_0BB@OMEFKBJ@username_reserve?$AA@ 1002db5c     dialog.obj
 0002:00007b70       ??_C@_0BB@GHAKMGNO@hostName_reserve?$AA@ 1002db70     dialog.obj
 0002:00007b84       ??_C@_0P@LFPFCPEA@driver_reserve?$AA@ 1002db84     dialog.obj
 0002:00007b94       ??_C@_0BF@PCKDKNCH@m_pqSpinPort_reserve?$AA@ 1002db94     dialog.obj
 0002:00007bac       ??_C@_0P@IKOBPDDP@textLabel1_2_2?$AA@ 1002dbac     dialog.obj
 0002:00007bbc       ??_C@_0BB@HOMEBIPM@database_reserve?$AA@ 1002dbbc     dialog.obj
 0002:00007bd0       ??_C@_0N@MHEGOAAO@buttonGroup1?$AA@ 1002dbd0     dialog.obj
 0002:00007be0       ??_C@_0BD@OKICOJPO@textLabel1_3_2_2_3?$AA@ 1002dbe0     dialog.obj
 0002:00007bf4       ??_C@_0L@GLBCHLFI@bncsDriver?$AA@ 1002dbf4     dialog.obj
 0002:00007c00       ??_C@_05OLMLFICL@procs?$AA@ 1002dc00     dialog.obj
 0002:00007c08       ??_C@_0M@KPBOJHOJ@procsLayout?$AA@ 1002dc08     dialog.obj
 0002:00007c14       ??_C@_0N@IICKINDC@splProcesses?$AA@ 1002dc14     dialog.obj
 0002:00007c24       ??_C@_08CCAEJCBB@layout12?$AA@ 1002dc24     dialog.obj
 0002:00007c30       ??_C@_08JCJMBNC@layout11?$AA@ 1002dc30     dialog.obj
 0002:00007c3c       ??_C@_07GIKHDDO@layout9?$AA@ 1002dc3c     dialog.obj
 0002:00007c44       ??_C@_08NCMFJPMO@lbFilter?$AA@ 1002dc44     dialog.obj
 0002:00007c50       ??_C@_0L@FGIHNJBP@editFilter?$AA@ 1002dc50     dialog.obj
 0002:00007c5c       ??_C@_08BADCPAJD@layout10?$AA@ 1002dc5c     dialog.obj
 0002:00007c68       ??_C@_0O@HLGEBCAL@lbLevelFilter?$AA@ 1002dc68     dialog.obj
 0002:00007c78       ??_C@_0O@CNPAKGPN@cbLevelFilter?$AA@ 1002dc78     dialog.obj
 0002:00007c88       ??_C@_0M@DHKELJGL@procListBox?$AA@ 1002dc88     dialog.obj
 0002:00007c94       ??_C@_08DLBPKDFA@layout13?$AA@ 1002dc94     dialog.obj
 0002:00007ca0       ??_C@_0BA@BECJNAOP@setGroupDefault?$AA@ 1002dca0     dialog.obj
 0002:00007cb0       ??_C@_0N@OAOBBDPN@setOkDefault?$AA@ 1002dcb0     dialog.obj
 0002:00007cc0       ??_C@_0P@MMEGHOIO@setFailDefault?$AA@ 1002dcc0     dialog.obj
 0002:00007cd0       ??_C@_0O@CHCDGGLC@setAckDefault?$AA@ 1002dcd0     dialog.obj
 0002:00007ce0       ??_C@_0BB@OMLHCPAN@setIgnoreDefault?$AA@ 1002dce0     dialog.obj
 0002:00007cf4       ??_C@_0P@FKPOGKIN@textLabel3_5_2?$AA@ 1002dcf4     dialog.obj
 0002:00007d04       ??_C@_0BC@IMEICLO@setLatchedDefault?$AA@ 1002dd04     dialog.obj
 0002:00007d18       ??_C@_0BC@PONGACKB@setUnknownDefault?$AA@ 1002dd18     dialog.obj
 0002:00007d2c       ??_C@_0O@LCEJFAPG@setAllDefault?$AA@ 1002dd2c     dialog.obj
 0002:00007d3c       ??_C@_08MJEFMGGB@clearAll?$AA@ 1002dd3c     dialog.obj
 0002:00007d48       ??_C@_0L@MHEIMOIA@layout12_2?$AA@ 1002dd48     dialog.obj
 0002:00007d54       ??_C@_0L@NFPNGBGO@layout11_2?$AA@ 1002dd54     dialog.obj
 0002:00007d60       ??_C@_0P@EIMJINCC@templateButton?$AA@ 1002dd60     dialog.obj
 0002:00007d70       ??_C@_0BE@PIGJEMHB@m_qPushEditSelected?$AA@ 1002dd70     dialog.obj
 0002:00007d84       ??_C@_0L@OGJPOLGL@copyButton?$AA@ 1002dd84     dialog.obj
 0002:00007d90       ??_C@_0P@KKLJDAFI@pasteAllButton?$AA@ 1002dd90     dialog.obj
 0002:00007da0       ??_C@_0BF@MFGFKLBD@pasteSelectionButton?$AA@ 1002dda0     dialog.obj
 0002:00007db8       ??_C@_09CIDKMNDE@navToProc?$AA@ 1002ddb8     dialog.obj
 0002:00007dc4       ??_C@_07MNNHCJEA@TabPage?$AA@ 1002ddc4     dialog.obj
 0002:00007dcc       ??_C@_0O@CPJAHDHK@TabPageLayout?$AA@ 1002ddcc     dialog.obj
 0002:00007ddc       ??_C@_0N@OMGLLDMN@buttonGroup2?$AA@ 1002dddc     dialog.obj
 0002:00007dec       ??_C@_08HGBIILMO@layout24?$AA@ 1002ddec     dialog.obj
 0002:00007df8       ??_C@_08FPHDGGFE@layout17?$AA@ 1002ddf8     dialog.obj
 0002:00007e04       ??_C@_0L@LNIHPBPJ@radioAltId?$AA@ 1002de04     dialog.obj
 0002:00007e10       ??_C@_0L@HHOPOAEP@separator0?$AA@ 1002de10     dialog.obj
 0002:00007e1c       ??_C@_0L@KGLFILOJ@textLabel1?$AA@ 1002de1c     dialog.obj
 0002:00007e28       ??_C@_08CAECCMEI@layout22?$AA@ 1002de28     dialog.obj
 0002:00007e34       ??_C@_0BB@IFBKIKEH@textLabel1_3_3_2?$AA@ 1002de34     dialog.obj
 0002:00007e48       ??_C@_0BD@DIMFALBK@textLabel1_3_3_2_2?$AA@ 1002de48     dialog.obj
 0002:00007e5c       ??_C@_08LGPHPIL@layout21?$AA@ 1002de5c     dialog.obj
 0002:00007e68       ??_C@_0L@GOPENBAO@separator1?$AA@ 1002de68     dialog.obj
 0002:00007e74       ??_C@_0L@EFNJICMN@separator2?$AA@ 1002de74     dialog.obj
 0002:00007e80       ??_C@_0L@KFIDOLIM@layout24_2?$AA@ 1002de80     dialog.obj
 0002:00007e8c       ??_C@_0O@NDPMKACE@radioNotAltId?$AA@ 1002de8c     dialog.obj
 0002:00007e9c       ??_C@_0O@BJJFHGAH@groupDefaults?$AA@ 1002de9c     dialog.obj
 0002:00007eac       ??_C@_0P@EDOFFLMM@textLabel3_5_3?$AA@ 1002deac     dialog.obj
 0002:00007ebc       ??_C@_0P@GGIOAEBA@textLabel3_3_3?$AA@ 1002debc     dialog.obj
 0002:00007ecc       ??_C@_0P@OCECANOI@textLabel3_4_2?$AA@ 1002decc     dialog.obj
 0002:00007edc       ??_C@_0P@NODCGDHF@textLabel3_2_3?$AA@ 1002dedc     dialog.obj
 0002:00007eec       ??_C@_0BB@KJNKAJEC@textLabel3_5_2_2?$AA@ 1002deec     dialog.obj
 0002:00007f00       ??_C@_08PEKBABCL@btnReset?$AA@ 1002df00     dialog.obj
 0002:00007f0c       ??_C@_0L@LJBNGEBG@ackDefault?$AA@ 1002df0c     dialog.obj
 0002:00007f18       ??_C@_0O@MBJBKFAG@ignoreDefault?$AA@ 1002df18     dialog.obj
 0002:00007f28       ??_C@_0M@BNGDCHHN@failDefault?$AA@ 1002df28     dialog.obj
 0002:00007f34       ??_C@_0P@GJCJPNKD@unknownDefault?$AA@ 1002df34     dialog.obj
 0002:00007f44       ??_C@_0P@JPDLHNLM@latchedDefault?$AA@ 1002df44     dialog.obj
 0002:00007f54       ??_C@_09LKHGBEPK@okDefault?$AA@ 1002df54     dialog.obj
 0002:00007f60       ??_C@_0BD@PHGMAIIC@textLabel3_3_2_2_2?$AA@ 1002df60     dialog.obj
 0002:00007f74       ??_C@_0BC@HACLIJBH@levelComboDefault?$AA@ 1002df74     dialog.obj
 0002:00007f88       ??_C@_0O@FPECOBPM@dbToolsLayout?$AA@ 1002df88     dialog.obj
 0002:00007f98       ??_C@_06KMCIPFID@dbProc?$AA@ 1002df98     dialog.obj
 0002:00007fa0       ??_C@_09EAKJIPAF@procCount?$AA@ 1002dfa0     dialog.obj
 0002:00007fac       ??_C@_0BA@FPDCILMK@createProcTable?$AA@ 1002dfac     dialog.obj
 0002:00007fbc       ??_C@_0N@NNFDLGC@clearProcAll?$AA@ 1002dfbc     dialog.obj
 0002:00007fcc       ??_C@_0BA@PBLFEBFN@clearProcBefore?$AA@ 1002dfcc     dialog.obj
 0002:00007fdc       ??_C@_08JBCFMOBA@procDate?$AA@ 1002dfdc     dialog.obj
 0002:00007fe8       ??_C@_05IGFPKBMF@dbLog?$AA@ 1002dfe8     dialog.obj
 0002:00007ff0       ??_C@_08CDCOMLLF@logCount?$AA@ 1002dff0     dialog.obj
 0002:00007ffc       ??_C@_0P@CNCJLFFI@createLogTable?$AA@ 1002dffc     dialog.obj
 0002:0000800c       ??_C@_0M@OJLNGPMB@clearLogAll?$AA@ 1002e00c     dialog.obj
 0002:00008018       ??_C@_0P@LHDFNDLK@clearLogBefore?$AA@ 1002e018     dialog.obj
 0002:00008028       ??_C@_07BAANKHAN@logDate?$AA@ 1002e028     dialog.obj
 0002:00008030       ??_C@_09PEAHDEKL@groupBox5?$AA@ 1002e030     dialog.obj
 0002:0000803c       ??_C@_08BOBOMJHK@dbStatus?$AA@ 1002e03c     dialog.obj
 0002:00008048       ??_C@_0BH@OIJBBILA@m_pqComboDatabaseTools?$AA@ 1002e048     dialog.obj
 0002:00008060       ??_C@_07JIAJFOLA@layout7?$AA@ 1002e060     dialog.obj
 0002:00008068       ??_C@_0L@NLMCHPKM@textLabel4?$AA@ 1002e068     dialog.obj
 0002:00008074       ??_C@_0N@JDIMPCEA@dbEditLayout?$AA@ 1002e074     dialog.obj
 0002:00008084       ??_C@_0L@PAJGDOLC@layout17_2?$AA@ 1002e084     dialog.obj
 0002:00008090       ??_C@_0L@KLIJIBPJ@groupBox12?$AA@ 1002e090     dialog.obj
 0002:0000809c       ??_C@_0BG@OMNHHOBJ@m_pqComboDatabaseEdit?$AA@ 1002e09c     dialog.obj
 0002:000080b4       ??_C@_0M@OGNHFIGM@groupBox5_2?$AA@ 1002e0b4     dialog.obj
 0002:000080c0       ??_C@_09FNLONCJK@dbStatus2?$AA@ 1002e0c0     dialog.obj
 0002:000080cc       ??_C@_0O@CGGICGEG@groupBox5_2_2?$AA@ 1002e0cc     dialog.obj
 0002:000080dc       ??_C@_0L@DKCNKABO@tableCombo?$AA@ 1002e0dc     dialog.obj
 0002:000080e8       ??_C@_0BA@FJMBALID@m_pqPushRefresh?$AA@ 1002e0e8     dialog.obj
 0002:000080f8       ??_C@_0N@EIJIHJHG@textLabel4_2?$AA@ 1002e0f8     dialog.obj
 0002:00008108       ??_C@_09HBJPPIGN@dataTable?$AA@ 1002e108     dialog.obj
 0002:00008114       ??_C@_06IOAEHBNO@dialog?$AA@ 1002e114     dialog.obj
 0002:0000811c       ??_C@_0BP@OFCIDEEL@?$DMh1?$DOAlarm?5Database?5Output?$DM?1h1?$DO?$AA@ 1002e11c     dialog.obj
 0002:0000813c       ??_C@_0BL@CKGGFCJK@Database?5Connection?5?9?5Main?$AA@ 1002e13c     dialog.obj
 0002:00008158       ??_C@_04CPPPJGME@Host?$AA@ 1002e158     dialog.obj
 0002:00008160       ??_C@_09FCOKPOKB@User?5Name?$AA@ 1002e160     dialog.obj
 0002:0000816c       ??_C@_08FJIAHGMM@Password?$AA@ 1002e16c     dialog.obj
 0002:00008178       ??_C@_04HOKNCALA@Port?$AA@ 1002e178     dialog.obj
 0002:00008180       ??_C@_07DLHCIBDH@default?$AA@ 1002e180     dialog.obj
 0002:00008188       ??_C@_06BNFOCFOC@Driver?$AA@ 1002e188     dialog.obj
 0002:00008190       ??_C@_0BO@NBFBDCNI@Database?5Connection?5?9?5Reserve?$AA@ 1002e190     dialog.obj
 0002:000081b0       ??_C@_0FI@EFABCMCI@?$DMp?5align?$DN?$CCleft?$CC?$DOLeave?5all?5these?5@ 1002e1b0     dialog.obj
 0002:00008208       ??_C@_0M@GEKFIEDD@BNCS?5Driver?$AA@ 1002e208     dialog.obj
 0002:00008214       ??_C@_0L@NGHPBBJO@Log?5Driver?$AA@ 1002e214     dialog.obj
 0002:00008220       ??_C@_06IBDJIBGI@Filter?$AA@ 1002e220     dialog.obj
 0002:00008228       ??_C@_0N@OGJPGMLO@Level?5Filter?$AA@ 1002e228     dialog.obj
 0002:00008238       ??_C@_0N@PJBOIAE@Not?5filtered?$AA@ 1002e238     dialog.obj
 0002:00008248       ??_C@_07MCAEODGB@Default?$AA@ 1002e248     dialog.obj
 0002:00008250       ??_C@_0BD@LOPDFLOH@Set?5all?5to?5Default?$AA@ 1002e250     dialog.obj
 0002:00008264       ??_C@_09EKGDBKGN@Clear?5All?$AA@ 1002e264     dialog.obj
 0002:00008270       ??_C@_0O@FDJFBAFB@Edit?5Template?$AA@ 1002e270     dialog.obj
 0002:00008280       ??_C@_0O@CDPACNHO@Edit?5Selected?$AA@ 1002e280     dialog.obj
 0002:00008290       ??_C@_0BC@NOIFPMEL@Copy?5to?5Clipboard?$AA@ 1002e290     dialog.obj
 0002:000082a4       ??_C@_09OGFEHODH@Paste?5All?$AA@ 1002e2a4     dialog.obj
 0002:000082b0       ??_C@_0BG@GMDKPAML@?5?5?5Paste?5Selection?5?5?5?$AA@ 1002e2b0     dialog.obj
 0002:000082c8       ??_C@_0N@HKALLKJF@Edit?5Process?$AA@ 1002e2c8     dialog.obj
 0002:000082d8       ??_C@_09BNGODGIH@Processes?$AA@ 1002e2d8     dialog.obj
 0002:000082e4       ??_C@_06PEPCFMNJ@Format?$AA@ 1002e2e4     dialog.obj
 0002:000082ec       ??_C@_0M@DDFIGBGP@?$DMparameter?$DO?$AA@ 1002e2ec     dialog.obj
 0002:000082f8       ??_C@_07EKFKJIEF@?$DMstate?$DO?$AA@ 1002e2f8     dialog.obj
 0002:00008300       ??_C@_0N@LLNLILCB@?$DMdevicename?$DO?$AA@ 1002e300     dialog.obj
 0002:00008310       ??_C@_0O@HEMOKBB@Text?5Defaults?$AA@ 1002e310     dialog.obj
 0002:00008320       ??_C@_05CCGMLFNG@Reset?$AA@ 1002e320     dialog.obj
 0002:00008328       ??_C@_0N@CHHMCFHH@Process?5Data?$AA@ 1002e328     dialog.obj
 0002:00008338       ??_C@_0L@PHKNIMLH@Create?5New?$AA@ 1002e338     dialog.obj
 0002:00008344       ??_C@_0BE@CEGPOEJJ@Clear?5All?5Processes?$AA@ 1002e344     dialog.obj
 0002:00008358       ??_C@_0BH@MJPGGCHJ@Clear?5Processes?5Before?$AA@ 1002e358     dialog.obj
 0002:00008370       ??_C@_0P@JLFAAHDK@Historical?5Log?$AA@ 1002e370     dialog.obj
 0002:00008380       ??_C@_0P@KOGBHGEK@Clear?5All?5Logs?$AA@ 1002e380     dialog.obj
 0002:00008390       ??_C@_0BC@GKPDPGHF@Clear?5Logs?5Before?$AA@ 1002e390     dialog.obj
 0002:000083a4       ??_C@_06PGDKHFME@Status?$AA@ 1002e3a4     dialog.obj
 0002:000083ac       ??_C@_0BG@KCPPGAEF@Primary?1Main?5Database?$AA@ 1002e3ac     dialog.obj
 0002:000083c4       ??_C@_0BL@POFOHFFC@Secondary?1Reserve?5Database?$AA@ 1002e3c4     dialog.obj
 0002:000083e0       ??_C@_0FB@DCKJMLJH@?$DMfont?5color?$DN?$CC?$CDff0000?$CC?5size?$DN?$CC?$CL4?$CC?$DO@ 1002e3e0     dialog.obj
 0002:00008434       ??_C@_0P@LCCBMHJB@Database?5Tools?$AA@ 1002e434     dialog.obj
 0002:00008444       ??_C@_05LFBINIGO@Table?$AA@ 1002e444     dialog.obj
 0002:0000844c       ??_C@_07POIENIBA@Refresh?$AA@ 1002e44c     dialog.obj
 0002:00008458       ??_C@_0EM@ONNHLHKB@?$DMfont?5color?$DN?$CC?$CDff0000?$CC?5size?$DN?$CC?$CL4?$CC?$DO@ 1002e458     dialog.obj
 0002:000084a4       ??_C@_0O@FJNHEEOH@Database?5Edit?$AA@ 1002e4a4     dialog.obj
 0002:000084b8       ??_7manage_tempBase@@6BQObject@@@ 1002e4b8     manage_temp.obj
 0002:0000867c       ??_7manage_tempBase@@6BQPaintDevice@@@ 1002e67c     manage_temp.obj
 0002:000086a4       ??_SQTable@@6BQObject@@@   1002e6a4     manage_temp.obj
 0002:00008a44       ??_SQTable@@6BQPaintDevice@@@ 1002ea44     manage_temp.obj
 0002:00008a64       ??_C@_0BA@ECGMJAHD@manage_tempBase?$AA@ 1002ea64     manage_temp.obj
 0002:00008a74       ??_C@_0BG@JALDPJDK@manage_tempBaseLayout?$AA@ 1002ea74     manage_temp.obj
 0002:00008a8c       ??_C@_03CEDILPBK@tab?$AA@  1002ea8c     manage_temp.obj
 0002:00008a90       ??_C@_09PEOMDABK@tabLayout?$AA@ 1002ea90     manage_temp.obj
 0002:00008a9c       ??_C@_09GABCAMHI@splManage?$AA@ 1002ea9c     manage_temp.obj
 0002:00008aa8       ??_C@_07BPJBECHP@layout8?$AA@ 1002eaa8     manage_temp.obj
 0002:00008ab0       ??_C@_07LDCEANHD@layout4?$AA@ 1002eab0     manage_temp.obj
 0002:00008ab8       ??_C@_0L@DPGNGODI@editPrefix?$AA@ 1002eab8     manage_temp.obj
 0002:00008ac4       ??_C@_09PPOBMLDK@listSlots?$AA@ 1002eac4     manage_temp.obj
 0002:00008ad0       ??_C@_09HPDNJEFH@Parameter?$AA@ 1002ead0     manage_temp.obj
 0002:00008adc       ??_C@_07IBBCGPPB@layout6?$AA@ 1002eadc     manage_temp.obj
 0002:00008ae4       ??_C@_0BE@FMGEBHEF@setAllParamsDefault?$AA@ 1002eae4     manage_temp.obj
 0002:00008af8       ??_C@_0P@DDKBKAID@clearAllParams?$AA@ 1002eaf8     manage_temp.obj
 0002:00008b08       ??_C@_0BB@HPIDOKFP@textLabel3_3_2_2?$AA@ 1002eb08     manage_temp.obj
 0002:00008b1c       ??_C@_0BB@LENPDJPK@textLabel3_2_2_2?$AA@ 1002eb1c     manage_temp.obj
 0002:00008b30       ??_C@_0BA@DDIBKBPM@setLevelDefault?$AA@ 1002eb30     manage_temp.obj
 0002:00008b40       ??_C@_0BB@BBNMFBIK@setDeviceDefault?$AA@ 1002eb40     manage_temp.obj
 0002:00008b54       ??_C@_09JNHIMIKJ@groupText?$AA@ 1002eb54     manage_temp.obj
 0002:00008b60       ??_C@_0L@DNBLEGOD@deviceText?$AA@ 1002eb60     manage_temp.obj
 0002:00008b6c       ??_C@_05GBGDENAC@tab_2?$AA@ 1002eb6c     manage_temp.obj
 0002:00008b74       ??_C@_0M@BMGEADGH@tabLayout_2?$AA@ 1002eb74     manage_temp.obj
 0002:00008b80       ??_C@_0O@HAFIDGAD@tableInstance?$AA@ 1002eb80     manage_temp.obj
 0002:00008b90       ??_C@_07DOAOMMKG@Enabled?$AA@ 1002eb90     manage_temp.obj
 0002:00008b98       ??_C@_09LKOFGHOI@layout8_2?$AA@ 1002eb98     manage_temp.obj
 0002:00008ba4       ??_C@_0BA@PMLLJDGK@btnNoneSelected?$AA@ 1002eba4     manage_temp.obj
 0002:00008bb4       ??_C@_0P@ENCIAPGO@btnAllSelected?$AA@ 1002ebb4     manage_temp.obj
 0002:00008bc4       ??_C@_07PMIPGFPH@btnNone?$AA@ 1002ebc4     manage_temp.obj
 0002:00008bcc       ??_C@_06GDCGNCAB@btnAll?$AA@ 1002ebcc     manage_temp.obj
 0002:00008bd4       ??_C@_09FKDKBANL@layout6_2?$AA@ 1002ebd4     manage_temp.obj
 0002:00008be0       ??_C@_0BB@GBAJKNMD@Manage?5Templates?$AA@ 1002ebe0     manage_temp.obj
 0002:00008bf4       ??_C@_0BE@MBBKLJIA@Prefix?5for?5Template?$AA@ 1002ebf4     manage_temp.obj
 0002:00008c08       ??_C@_0BD@BEKFCONC@For?5each?5parameter?$AA@ 1002ec08     manage_temp.obj
 0002:00008c1c       ??_C@_0CH@PBGEALM@Set?5all?5to?5Default?5for?5each?5para@ 1002ec1c     manage_temp.obj
 0002:00008c44       ??_C@_0BO@HKDGKKGJ@Clear?5all?5for?5each?5parameters?$AA@ 1002ec44     manage_temp.obj
 0002:00008c64       ??_C@_09OKFBLFFD@Clear?5all?$AA@ 1002ec64     manage_temp.obj
 0002:00008c70       ??_C@_0O@PIILMNHI@Configuration?$AA@ 1002ec70     manage_temp.obj
 0002:00008c80       ??_C@_0BC@HALKMNOP@Deselect?5Selected?$AA@ 1002ec80     manage_temp.obj
 0002:00008c94       ??_C@_0BA@NKELCOGO@Select?5Selected?$AA@ 1002ec94     manage_temp.obj
 0002:00008ca4       ??_C@_0N@PBNGBON@Deselect?5All?$AA@ 1002eca4     manage_temp.obj
 0002:00008cb4       ??_C@_0L@CALHPJHB@Select?5All?$AA@ 1002ecb4     manage_temp.obj
 0002:00008cc0       ??_C@_07MEEAAPDA@Devices?$AA@ 1002ecc0     manage_temp.obj
 0002:00008cc8       ??_C@_0BA@PFMNDNMK@Create?5?$CGOutputs?$AA@ 1002ecc8     manage_temp.obj
 0002:00008cd8       ??_C@_0O@IIOOHDCA@alm_db_output?$AA@ 1002ecd8     moc_alm_db_output.obj
 0002:00008cf4       ??_C@_05JLNEMJLN@dummy?$AA@ 1002ecf4     moc_alm_db_output.obj
 0002:00008d08       ??_C@_0BD@IODKAMCM@pasteSelectedProcs?$AA@ 1002ed08     moc_alm_db_output.obj
 0002:00008d1c       ??_C@_0O@PKECGKLD@bOnlySelected?$AA@ 1002ed1c     moc_alm_db_output.obj
 0002:00008d44       ??_C@_0O@JNEOAMIH@pasteAllProcs?$AA@ 1002ed44     moc_alm_db_output.obj
 0002:00008d60       ??_C@_0N@EKEEEBKO@pasteOptions?$AA@ 1002ed60     moc_alm_db_output.obj
 0002:00008d7c       ??_C@_0BA@FOLOKBKN@copyToClipBoard?$AA@ 1002ed7c     moc_alm_db_output.obj
 0002:00008d98       ??_C@_0BC@GFHIKBGI@editSelectedProcs?$AA@ 1002ed98     moc_alm_db_output.obj
 0002:00008db8       ??_C@_09HIGIDEDO@markDirty?$AA@ 1002edb8     moc_alm_db_output.obj
 0002:00008dd0       ??_C@_0P@CNFJKBJI@menuDeleteFile?$AA@ 1002edd0     moc_alm_db_output.obj
 0002:00008dec       ??_C@_0BC@HKAEEBBP@menuDuplicateFile?$AA@ 1002edec     moc_alm_db_output.obj
 0002:00008e0c       ??_C@_0L@FJIJGHHG@menuRename?$AA@ 1002ee0c     moc_alm_db_output.obj
 0002:00008e24       ??_C@_0M@FNCKOKHH@menuNewFile?$AA@ 1002ee24     moc_alm_db_output.obj
 0002:00008e3c       ??_C@_0M@BLOGNIHC@EditProcess?$AA@ 1002ee3c     moc_alm_db_output.obj
 0002:00008e48       ??_C@_04NHONDGDE@item?$AA@ 1002ee48     moc_alm_db_output.obj
 0002:00008e50       ??_C@_0O@LAFKAPIP@QListViewItem?$AA@ 1002ee50     moc_alm_db_output.obj
 0002:00008e60       ??_C@_03HNOLNALI@col?$AA@  1002ee60     moc_alm_db_output.obj
 0002:00008e64       ??_C@_04CIMGMMMG@text?$AA@ 1002ee64     moc_alm_db_output.obj
 0002:00008e78       ??_C@_0N@CGBIPEEF@renameModule?$AA@ 1002ee78     moc_alm_db_output.obj
 0002:00008e94       ??_C@_0L@EBNMIND@selectFile?$AA@ 1002ee94     moc_alm_db_output.obj
 0002:00008ea0       ??_C@_03PCBNCGFH@pos?$AA@  1002eea0     moc_alm_db_output.obj
 0002:00008ea4       ??_C@_01CAKFMAIO@?$AO?$AA@ 1002eea4     moc_alm_db_output.obj
 0002:00008eb4       ??_C@_0BE@EOPNNNEB@fileListContextMenu?$AA@ 1002eeb4     moc_alm_db_output.obj
 0002:00008ed4       ??_C@_0O@OLIHJJKC@procSelection?$AA@ 1002eed4     moc_alm_db_output.obj
 0002:00008ef0       ??_C@_05KAEIDCAL@apply?$AA@ 1002eef0     moc_alm_db_output.obj
 0002:00008ef8       ??_C@_07ECHCKIDD@sSystem?$AA@ 1002eef8     moc_alm_db_output.obj
 0002:00008f0c       ??_C@_0N@JNMAEFDJ@selectSystem?$AA@ 1002ef0c     moc_alm_db_output.obj
 0002:00008f28       ??_C@_0N@NHGOHCF@filterChange?$AA@ 1002ef28     moc_alm_db_output.obj
 0002:00008f44       ??_C@_0BA@OKJBMDAJ@templateProcess?$AA@ 1002ef44     moc_alm_db_output.obj
 0002:00009054       ??_C@_07MBMLLJIG@dummy?$CI?$CJ?$AA@ 1002f054     moc_alm_db_output.obj
 0002:0000905c       ??_C@_0BF@ECJPCBAM@pasteSelectedProcs?$CI?$CJ?$AA@ 1002f05c     moc_alm_db_output.obj
 0002:00009074       ??_C@_0BJ@FGBHFMP@pasteSelectedProcs?$CIbool?$CJ?$AA@ 1002f074     moc_alm_db_output.obj
 0002:00009090       ??_C@_0BA@PGMFHFK@pasteAllProcs?$CI?$CJ?$AA@ 1002f090     moc_alm_db_output.obj
 0002:000090a0       ??_C@_0P@EDEHCCJG@pasteOptions?$CI?$CJ?$AA@ 1002f0a0     moc_alm_db_output.obj
 0002:000090b0       ??_C@_0BC@MIGAIHNH@copyToClipBoard?$CI?$CJ?$AA@ 1002f0b0     moc_alm_db_output.obj
 0002:000090c4       ??_C@_0BE@HOONJPBK@editSelectedProcs?$CI?$CJ?$AA@ 1002f0c4     moc_alm_db_output.obj
 0002:000090d8       ??_C@_0M@BCGJBPBD@markDirty?$CI?$CJ?$AA@ 1002f0d8     moc_alm_db_output.obj
 0002:000090e4       ??_C@_0BB@GKFBDGIG@menuDeleteFile?$CI?$CJ?$AA@ 1002f0e4     moc_alm_db_output.obj
 0002:000090f8       ??_C@_0BE@LOJJINCP@menuDuplicateFile?$CI?$CJ?$AA@ 1002f0f8     moc_alm_db_output.obj
 0002:0000910c       ??_C@_0N@NIKLPLLB@menuRename?$CI?$CJ?$AA@ 1002f10c     moc_alm_db_output.obj
 0002:0000911c       ??_C@_0O@FCLJDBMO@menuNewFile?$CI?$CJ?$AA@ 1002f11c     moc_alm_db_output.obj
 0002:0000912c       ??_C@_0O@OHBJNCMH@EditProcess?$CI?$CJ?$AA@ 1002f12c     moc_alm_db_output.obj
 0002:0000913c       ??_C@_0DA@KLJABHB@renameModule?$CIQListViewItem?$CK?0int?0@ 1002f13c     moc_alm_db_output.obj
 0002:0000916c       ??_C@_0BL@GBKHEMNO@selectFile?$CIQListViewItem?$CK?$CJ?$AA@ 1002f16c     moc_alm_db_output.obj
 0002:00009188       ??_C@_0DG@IBBHMLFJ@fileListContextMenu?$CIQListViewIte@ 1002f188     moc_alm_db_output.obj
 0002:000091c0       ??_C@_0BA@GHPKJGLP@procSelection?$CI?$CJ?$AA@ 1002f1c0     moc_alm_db_output.obj
 0002:000091d0       ??_C@_07FJDLKALA@apply?$CI?$CJ?$AA@ 1002f1d0     moc_alm_db_output.obj
 0002:000091d8       ??_C@_0BN@PCNKHLKL@selectSystem?$CIconst?5QString?$CG?$CJ?$AA@ 1002f1d8     moc_alm_db_output.obj
 0002:000091f8       ??_C@_0P@KEIFCCPJ@filterChange?$CI?$CJ?$AA@ 1002f1f8     moc_alm_db_output.obj
 0002:00009208       ??_C@_0BC@KBLHEKGB@templateProcess?$CI?$CJ?$AA@ 1002f208     moc_alm_db_output.obj
 0002:00009228       ??_C@_07KMMNMMFF@command?$AA@ 1002f228     moc_alm_db_output.obj
 0002:0000923c       ??_C@_0BJ@FEFNJDLM@command?$CIQString?0QString?$CJ?$AA@ 1002f23c     moc_alm_db_output.obj
 0002:00009258       ??_C@_0O@GCELBMFI@IGetDocuments?$AA@ 1002f258     moc_alm_db_output.obj
 0002:00009268       ??_C@_0N@KBDCPKEG@ISendCommand?$AA@ 1002f268     moc_alm_db_output.obj
 0002:00009284       ??_C@_06JGCGFIEG@polish?$AA@ 1002f284     moc_dialog.obj
 0002:000092b0       ??_C@_08LBILCPNA@polish?$CI?$CJ?$AA@ 1002f2b0     moc_dialog.obj
 0002:000092d4       ??_C@_0M@PGFFFNDC@itemChanged?$AA@ 1002f2d4     moc_dialogimpl.obj
 0002:000092e0       ??_C@_06ICGJLFIM@string?$AA@ 1002f2e0     moc_dialogimpl.obj
 0002:000092f4       ??_C@_06DJHIOBEC@iValue?$AA@ 1002f2f4     moc_dialogimpl.obj
 0002:00009308       ??_C@_07MHMPLDIG@sDriver?$AA@ 1002f308     moc_dialogimpl.obj
 0002:0000931c       ??_C@_0BA@MPFLGADO@dbDriverChanged?$AA@ 1002f31c     moc_dialogimpl.obj
 0002:00009338       ??_C@_0BI@NJEJJFNJ@dbDriverChanged_reserve?$AA@ 1002f338     moc_dialogimpl.obj
 0002:00009350       ??_C@_06JMPFMJLN@iLevel?$AA@ 1002f350     moc_dialogimpl.obj
 0002:00009364       ??_C@_0N@FMKAFOHJ@levelChanged?$AA@ 1002f364     moc_dialogimpl.obj
 0002:00009380       ??_C@_08LEGBJMIA@copyData?$AA@ 1002f380     moc_dialogimpl.obj
 0002:00009398       ??_C@_09MCBCIPNB@pasteData?$AA@ 1002f398     moc_dialogimpl.obj
 0002:000093b0       ??_C@_0M@BAKNLOAG@dbEditStart?$AA@ 1002f3b0     moc_dialogimpl.obj
 0002:000093c8       ??_C@_0O@IGBMNLFD@fillDataTable?$AA@ 1002f3c8     moc_dialogimpl.obj
 0002:000093d8       ??_C@_06GPFGCBFO@iIndex?$AA@ 1002f3d8     moc_dialogimpl.obj
 0002:000093ec       ??_C@_0BC@JCMKPKOF@fillDataTableEdit?$AA@ 1002f3ec     moc_dialogimpl.obj
 0002:0000940c       ??_C@_0BD@FMOELLAD@fillDataTableTools?$AA@ 1002f40c     moc_dialogimpl.obj
 0002:0000942c       ??_C@_0BC@NGBOGPPL@clearAllProcesses?$AA@ 1002f42c     moc_dialogimpl.obj
 0002:0000944c       ??_C@_0BA@EAGKIODK@clearLogsBefore?$AA@ 1002f44c     moc_dialogimpl.obj
 0002:00009468       ??_C@_0N@MOMCBOEN@clearAllLogs?$AA@ 1002f468     moc_dialogimpl.obj
 0002:00009484       ??_C@_0BF@PHBLPLOJ@clearProcessesBefore?$AA@ 1002f484     moc_dialogimpl.obj
 0002:000094a8       ??_C@_0BC@BFPOJGJF@createNewLogTable?$AA@ 1002f4a8     moc_dialogimpl.obj
 0002:000094c8       ??_C@_0BD@LKNPOCOE@createNewProcTable?$AA@ 1002f4c8     moc_dialogimpl.obj
 0002:000094e8       ??_C@_0N@MICICEKM@dbToolUpdate?$AA@ 1002f4e8     moc_dialogimpl.obj
 0002:000094f8       ??_C@_04FBGDBCCI@widg?$AA@ 1002f4f8     moc_dialogimpl.obj
 0002:00009500       ??_C@_07FNEPBGL@QWidget?$AA@ 1002f500     moc_dialogimpl.obj
 0002:00009514       ??_C@_0O@EJNFDBH@showingWidget?$AA@ 1002f514     moc_dialogimpl.obj
 0002:00009530       ??_C@_0BC@BLLPKKAH@setAllDefaultText?$AA@ 1002f530     moc_dialogimpl.obj
 0002:00009550       ??_C@_0N@KJNEFAOA@clearAllText?$AA@ 1002f550     moc_dialogimpl.obj
 0002:0000956c       ??_C@_0BB@FNNJBIKG@setOkDefaultText?$AA@ 1002f56c     moc_dialogimpl.obj
 0002:0000958c       ??_C@_0BD@LHMCAJGK@setFailDefaultText?$AA@ 1002f58c     moc_dialogimpl.obj
 0002:000095ac       ??_C@_0BC@DAFIBIKJ@setAckDefaultText?$AA@ 1002f5ac     moc_dialogimpl.obj
 0002:000095cc       ??_C@_0BF@BDJJKEAM@setIgnoreDefaultText?$AA@ 1002f5cc     moc_dialogimpl.obj
 0002:000095f0       ??_C@_0BG@KLOOPMKM@setUnknownDefaultText?$AA@ 1002f5f0     moc_dialogimpl.obj
 0002:00009614       ??_C@_0BG@GOILIHBP@setLatchedDefaultText?$AA@ 1002f614     moc_dialogimpl.obj
 0002:00009638       ??_C@_0BE@INNDMEOI@setGroupDefaultText?$AA@ 1002f638     moc_dialogimpl.obj
 0002:00009658       ??_C@_0O@JMPPEAEI@resetDefaults?$AA@ 1002f658     moc_dialogimpl.obj
 0002:00009674       ??_C@_0BE@FDCIHIHG@setBncsSystemValues?$AA@ 1002f674     moc_dialogimpl.obj
 0002:00009808       ??_C@_0O@IKLCAHNO@itemChanged?$CI?$CJ?$AA@ 1002f808     moc_dialogimpl.obj
 0002:00009818       ??_C@_0BM@KLLCNLMA@itemChanged?$CIconst?5QString?$CG?$CJ?$AA@ 1002f818     moc_dialogimpl.obj
 0002:00009834       ??_C@_0BB@HJINNLMJ@itemChanged?$CIint?$CJ?$AA@ 1002f834     moc_dialogimpl.obj
 0002:00009848       ??_C@_0CA@HHEOGJJC@dbDriverChanged?$CIconst?5QString?$CG?$CJ?$AA@ 1002f848     moc_dialogimpl.obj
 0002:00009868       ??_C@_0CI@HGJOEMO@dbDriverChanged_reserve?$CIconst?5QS@ 1002f868     moc_dialogimpl.obj
 0002:00009890       ??_C@_0BC@KDPMPICH@levelChanged?$CIint?$CJ?$AA@ 1002f890     moc_dialogimpl.obj
 0002:000098a4       ??_C@_0L@LACCHLPG@copyData?$CI?$CJ?$AA@ 1002f8a4     moc_dialogimpl.obj
 0002:000098b0       ??_C@_0M@JHDMCAEO@pasteData?$CI?$CJ?$AA@ 1002f8b0     moc_dialogimpl.obj
 0002:000098bc       ??_C@_0O@IJLKBBD@dbEditStart?$CI?$CJ?$AA@ 1002f8bc     moc_dialogimpl.obj
 0002:000098cc       ??_C@_0BA@PCIPALGE@fillDataTable?$CI?$CJ?$AA@ 1002f8cc     moc_dialogimpl.obj
 0002:000098dc       ??_C@_0BH@GFDKAIFC@fillDataTableEdit?$CIint?$CJ?$AA@ 1002f8dc     moc_dialogimpl.obj
 0002:000098f4       ??_C@_0BI@IGKMJEFP@fillDataTableTools?$CIint?$CJ?$AA@ 1002f8f4     moc_dialogimpl.obj
 0002:0000990c       ??_C@_0BE@FIFNBKBC@clearAllProcesses?$CI?$CJ?$AA@ 1002f90c     moc_dialogimpl.obj
 0002:00009920       ??_C@_0BC@FNLBLIIH@clearLogsBefore?$CI?$CJ?$AA@ 1002f920     moc_dialogimpl.obj
 0002:00009934       ??_C@_0P@MNMAEKFK@clearAllLogs?$CI?$CJ?$AA@ 1002f934     moc_dialogimpl.obj
 0002:00009944       ??_C@_0BH@NHMLBMJJ@clearProcessesBefore?$CI?$CJ?$AA@ 1002f944     moc_dialogimpl.obj
 0002:0000995c       ??_C@_0BE@GHECNFGD@createNewLogTable?$CI?$CJ?$AA@ 1002f95c     moc_dialogimpl.obj
 0002:00009970       ??_C@_0BF@GAOIHNA@createNewProcTable?$CI?$CJ?$AA@ 1002f970     moc_dialogimpl.obj
 0002:00009988       ??_C@_0P@EMKJFHKP@dbToolUpdate?$CI?$CJ?$AA@ 1002f988     moc_dialogimpl.obj
 0002:00009998       ??_C@_0BI@NDGCLCOF@showingWidget?$CIQWidget?$CK?$CJ?$AA@ 1002f998     moc_dialogimpl.obj
 0002:000099b0       ??_C@_0BE@LFKEPDN@setAllDefaultText?$CI?$CJ?$AA@ 1002f9b0     moc_dialogimpl.obj
 0002:000099c4       ??_C@_0P@EHANIDHP@clearAllText?$CI?$CJ?$AA@ 1002f9c4     moc_dialogimpl.obj
 0002:000099d4       ??_C@_0BD@JJCJFGFD@setOkDefaultText?$CI?$CJ?$AA@ 1002f9d4     moc_dialogimpl.obj
 0002:000099e8       ??_C@_0BF@JENGAEPI@setFailDefaultText?$CI?$CJ?$AA@ 1002f9e8     moc_dialogimpl.obj
 0002:00009a00       ??_C@_0BE@BOLBCHBN@setAckDefaultText?$CI?$CJ?$AA@ 1002fa00     moc_dialogimpl.obj
 0002:00009a14       ??_C@_0BH@PBGLDNH@setIgnoreDefaultText?$CI?$CJ?$AA@ 1002fa14     moc_dialogimpl.obj
 0002:00009a2c       ??_C@_0BI@MEKBGOIP@setUnknownDefaultText?$CI?$CJ?$AA@ 1002fa2c     moc_dialogimpl.obj
 0002:00009a44       ??_C@_0BI@MMJOPOCF@setLatchedDefaultText?$CI?$CJ?$AA@ 1002fa44     moc_dialogimpl.obj
 0002:00009a5c       ??_C@_0BG@HILGHKCN@setGroupDefaultText?$CI?$CJ?$AA@ 1002fa5c     moc_dialogimpl.obj
 0002:00009a74       ??_C@_0BA@DMGEJANB@resetDefaults?$CI?$CJ?$AA@ 1002fa74     moc_dialogimpl.obj
 0002:00009a84       ??_C@_0BG@FFKDPMOF@setBncsSystemValues?$CI?$CJ?$AA@ 1002fa84     moc_dialogimpl.obj
 0002:00009aa8       ??_C@_0N@IBIICDGH@itemsChanged?$AA@ 1002faa8     moc_dialogimpl.obj
 0002:00009ac4       ??_C@_0P@PKMDIFCJ@itemsChanged?$CI?$CJ?$AA@ 1002fac4     moc_dialogimpl.obj
 0002:00009aec       ??_C@_0M@LGFJKMND@manage_temp?$AA@ 1002faec     moc_manage_tempimpl.obj
 0002:00009b04       ??_C@_05BDFBMKBD@sText?$AA@ 1002fb04     moc_manage_tempimpl.obj
 0002:00009b18       ??_C@_0O@GDAHEPCL@prefixChanged?$AA@ 1002fb18     moc_manage_tempimpl.obj
 0002:00009b34       ??_C@_0O@GHGODGGJ@selectProcess?$AA@ 1002fb34     moc_manage_tempimpl.obj
 0002:00009b5c       ??_C@_0BI@GDFEFKG@setAllParamsDefaultText?$AA@ 1002fb5c     moc_manage_tempimpl.obj
 0002:00009b80       ??_C@_0BD@POICEDCL@clearAllParamsText?$AA@ 1002fb80     moc_manage_tempimpl.obj
 0002:00009bb8       ??_C@_0BF@HIHNFDBJ@setDeviceDefaultText?$AA@ 1002fbb8     moc_manage_tempimpl.obj
 0002:00009c30       ??_C@_0BE@FJJILNHE@setLevelDefaultText?$AA@ 1002fc30     moc_manage_tempimpl.obj
 0002:00009c5c       ??_C@_0BD@KFHHNDDN@selectAllInstances?$AA@ 1002fc5c     moc_manage_tempimpl.obj
 0002:00009c7c       ??_C@_0BF@ELCFJDEJ@deselectAllInstances?$AA@ 1002fc7c     moc_manage_tempimpl.obj
 0002:00009ca0       ??_C@_0BI@OBIGJEML@selectSelectedInstances?$AA@ 1002fca0     moc_manage_tempimpl.obj
 0002:00009cc4       ??_C@_0BK@NJAFKOEF@deselectSelectedInstances?$AA@ 1002fcc4     moc_manage_tempimpl.obj
 0002:00009de8       ??_C@_0BO@LDCNPKLA@prefixChanged?$CIconst?5QString?$CG?$CJ?$AA@ 1002fde8     moc_manage_tempimpl.obj
 0002:00009e08       ??_C@_0BO@LIGOEMIJ@selectProcess?$CIQListViewItem?$CK?$CJ?$AA@ 1002fe08     moc_manage_tempimpl.obj
 0002:00009e28       ??_C@_0BK@IMPDCAPG@setAllParamsDefaultText?$CI?$CJ?$AA@ 1002fe28     moc_manage_tempimpl.obj
 0002:00009e44       ??_C@_0BF@OLLNJLHC@clearAllParamsText?$CI?$CJ?$AA@ 1002fe44     moc_manage_tempimpl.obj
 0002:00009e5c       ??_C@_0BH@BLHKFJJI@setDeviceDefaultText?$CI?$CJ?$AA@ 1002fe5c     moc_manage_tempimpl.obj
 0002:00009e74       ??_C@_0BG@IMJLKCOI@setLevelDefaultText?$CI?$CJ?$AA@ 1002fe74     moc_manage_tempimpl.obj
 0002:00009e8c       ??_C@_0BF@HCKOGBE@selectAllInstances?$CI?$CJ?$AA@ 1002fe8c     moc_manage_tempimpl.obj
 0002:00009ea4       ??_C@_0BH@DKKFPFCE@deselectAllInstances?$CI?$CJ?$AA@ 1002fea4     moc_manage_tempimpl.obj
 0002:00009ebc       ??_C@_0BK@KNHEDAON@selectSelectedInstances?$CI?$CJ?$AA@ 1002febc     moc_manage_tempimpl.obj
 0002:00009ed8       ??_C@_0BM@MOHIGEBJ@deselectSelectedInstances?$CI?$CJ?$AA@ 1002fed8     moc_manage_tempimpl.obj
 0002:00009ef4       ??_C@_0BI@GGLIKMPP@CC_ConfigEdit?1Controls?1?$AA@ 1002fef4     cfg_widgets001:cfg_Settings.obj
 0002:00009f0c       ??_C@_03MMIELDNM@?0?$CF1?$AA@ 1002ff0c     cfg_widgets001:cfg_Settings.obj
 0002:00009f10       ??_C@_03FFMPJLOG@?$CF1?0?$AA@ 1002ff10     cfg_widgets001:cfg_Settings.obj
 0002:00009f14       ??_C@_0P@JHCMIKMI@?$CF1?0?$CF2?0?$CF3?0?$CF4?0?$CF5?$AA@ 1002ff14     cfg_widgets001:cfg_Settings.obj
 0002:00009f28       ??_7Document@@6B@          1002ff28     config_alarm_utilities:Document.obj
 0002:00009f30       ??_7Document_BncsSystem@@6B@ 1002ff30     config_alarm_utilities:Document.obj
 0002:00009f34       ??_C@_08FKACIMPB@?1config?1?$AA@ 1002ff34     config_alarm_utilities:Document.obj
 0002:00009f40       ??_C@_0BH@EEDFIBDB@system?1bncs_system?4ini?$AA@ 1002ff40     config_alarm_utilities:Document.obj
 0002:00009f58       ??_C@_02PGHGPEOM@?91?$AA@  1002ff58     config_alarm_utilities:Document.obj
 0002:00009f5c       ??_C@_0BD@FPEGEEKL@DeviceInfodriverId?$AA@ 1002ff5c     config_alarm_utilities:Document.obj
 0002:00009f70       ??_C@_0CA@EAAGFFNA@Failed?5to?5read?5Device?5Status?5ID?$AA@ 1002ff70     config_alarm_utilities:Document.obj
 0002:00009f94       ??_7FileLoad@@6B@          1002ff94     config_alarm_utilities:Loaders.obj
 0002:00009fa4       ??_7?$QPtrList@VFileLoad@@@@6B@ 1002ffa4     config_alarm_utilities:Loaders.obj
 0002:00009fc8       ??_7?$QPtrList@VDirLoad@@@@6B@ 1002ffc8     config_alarm_utilities:Loaders.obj
 0002:00009fec       ??_7Loaders@@6B@           1002ffec     config_alarm_utilities:Loaders.obj
 0002:00009ff4       ??_7type_info@@6B@         1002fff4     MSVCRT:ti_inst.obj
 0002:00009ff8       __pRawDllMain              1002fff8     MSVCRT:crtdll.obj
 0002:00009ff8       __pDefaultRawDllMain       1002fff8     MSVCRT:crtdll.obj
 0002:0000a008       __load_config_used         10030008     MSVCRT:loadcfg.obj
 0002:0000a050       ??_R1A@?0A@EA@QGList@@8    10030050     alm_db_output.obj
 0002:0000a06c       ??_R3QGList@@8             1003006c     alm_db_output.obj
 0002:0000a07c       ??_R2QGList@@8             1003007c     alm_db_output.obj
 0002:0000a088       ??_R1A@?0A@EA@QPtrCollection@@8 10030088     alm_db_output.obj
 0002:0000a0a4       ??_R3QPtrCollection@@8     100300a4     alm_db_output.obj
 0002:0000a0b4       ??_R2QPtrCollection@@8     100300b4     alm_db_output.obj
 0002:0000a0bc       ??_R4QWidget@@6BQObject@@@ 100300bc     alm_db_output.obj
 0002:0000a0d0       ??_R3QWidget@@8            100300d0     alm_db_output.obj
 0002:0000a0e0       ??_R2QWidget@@8            100300e0     alm_db_output.obj
 0002:0000a0f4       ??_R1A@?0A@EA@QWidget@@8   100300f4     alm_db_output.obj
 0002:0000a110       ??_R1A@?0A@EA@QObject@@8   10030110     alm_db_output.obj
 0002:0000a12c       ??_R3QObject@@8            1003012c     alm_db_output.obj
 0002:0000a13c       ??_R2QObject@@8            1003013c     alm_db_output.obj
 0002:0000a148       ??_R13?0A@EA@Qt@@8         10030148     alm_db_output.obj
 0002:0000a164       ??_R3Qt@@8                 10030164     alm_db_output.obj
 0002:0000a174       ??_R2Qt@@8                 10030174     alm_db_output.obj
 0002:0000a17c       ??_R1A@?0A@EA@Qt@@8        1003017c     alm_db_output.obj
 0002:0000a198       ??_R1CI@?0A@EA@QPaintDevice@@8 10030198     alm_db_output.obj
 0002:0000a1b4       ??_R3QPaintDevice@@8       100301b4     alm_db_output.obj
 0002:0000a1c4       ??_R2QPaintDevice@@8       100301c4     alm_db_output.obj
 0002:0000a1cc       ??_R1A@?0A@EA@QPaintDevice@@8 100301cc     alm_db_output.obj
 0002:0000a1e8       ??_R4QWidget@@6BQPaintDevice@@@ 100301e8     alm_db_output.obj
 0002:0000a1fc       ??_R3QShared@@8            100301fc     alm_db_output.obj
 0002:0000a20c       ??_R2QShared@@8            1003020c     alm_db_output.obj
 0002:0000a214       ??_R1A@?0A@EA@QShared@@8   10030214     alm_db_output.obj
 0002:0000a230       ??_R4QPopupMenu@@6BQObject@@@ 10030230     alm_db_output.obj
 0002:0000a244       ??_R3QPopupMenu@@8         10030244     alm_db_output.obj
 0002:0000a254       ??_R2QPopupMenu@@8         10030254     alm_db_output.obj
 0002:0000a274       ??_R1A@?0A@EA@QPopupMenu@@8 10030274     alm_db_output.obj
 0002:0000a290       ??_R1A@?0A@EA@QFrame@@8    10030290     alm_db_output.obj
 0002:0000a2ac       ??_R3QFrame@@8             100302ac     alm_db_output.obj
 0002:0000a2bc       ??_R2QFrame@@8             100302bc     alm_db_output.obj
 0002:0000a2d4       ??_R1IM@?0A@EA@QMenuData@@8 100302d4     alm_db_output.obj
 0002:0000a2f0       ??_R3QMenuData@@8          100302f0     alm_db_output.obj
 0002:0000a300       ??_R2QMenuData@@8          10030300     alm_db_output.obj
 0002:0000a308       ??_R1A@?0A@EA@QMenuData@@8 10030308     alm_db_output.obj
 0002:0000a324       ??_R4QPopupMenu@@6BQPaintDevice@@@ 10030324     alm_db_output.obj
 0002:0000a338       ??_R4QPopupMenu@@6B@       10030338     alm_db_output.obj
 0002:0000a34c       ??_R4QAction@@6B@          1003034c     alm_db_output.obj
 0002:0000a360       ??_R3QAction@@8            10030360     alm_db_output.obj
 0002:0000a370       ??_R2QAction@@8            10030370     alm_db_output.obj
 0002:0000a380       ??_R1A@?0A@EA@QAction@@8   10030380     alm_db_output.obj
 0002:0000a39c       ??_R4QBoxLayout@@6BQObject@@@ 1003039c     alm_db_output.obj
 0002:0000a3b0       ??_R3QBoxLayout@@8         100303b0     alm_db_output.obj
 0002:0000a3c0       ??_R2QBoxLayout@@8         100303c0     alm_db_output.obj
 0002:0000a3d8       ??_R1A@?0A@EA@QBoxLayout@@8 100303d8     alm_db_output.obj
 0002:0000a3f4       ??_R1A@?0A@EA@QLayout@@8   100303f4     alm_db_output.obj
 0002:0000a410       ??_R3QLayout@@8            10030410     alm_db_output.obj
 0002:0000a420       ??_R2QLayout@@8            10030420     alm_db_output.obj
 0002:0000a434       ??_R1CI@?0A@EA@QLayoutItem@@8 10030434     alm_db_output.obj
 0002:0000a450       ??_R3QLayoutItem@@8        10030450     alm_db_output.obj
 0002:0000a460       ??_R2QLayoutItem@@8        10030460     alm_db_output.obj
 0002:0000a468       ??_R1A@?0A@EA@QLayoutItem@@8 10030468     alm_db_output.obj
 0002:0000a484       ??_R4QBoxLayout@@6BQLayoutItem@@@ 10030484     alm_db_output.obj
 0002:0000a498       ??_R4QToolBar@@6BQObject@@@ 10030498     alm_db_output.obj
 0002:0000a4ac       ??_R3QToolBar@@8           100304ac     alm_db_output.obj
 0002:0000a4bc       ??_R2QToolBar@@8           100304bc     alm_db_output.obj
 0002:0000a4dc       ??_R1A@?0A@EA@QToolBar@@8  100304dc     alm_db_output.obj
 0002:0000a4f8       ??_R1A@?0A@EA@QDockWindow@@8 100304f8     alm_db_output.obj
 0002:0000a514       ??_R3QDockWindow@@8        10030514     alm_db_output.obj
 0002:0000a524       ??_R2QDockWindow@@8        10030524     alm_db_output.obj
 0002:0000a540       ??_R4QToolBar@@6BQPaintDevice@@@ 10030540     alm_db_output.obj
 0002:0000a554       ??_R4QDockWindow@@6BQObject@@@ 10030554     alm_db_output.obj
 0002:0000a568       ??_R4QDockWindow@@6BQPaintDevice@@@ 10030568     alm_db_output.obj
 0002:0000a57c       ??_R4QListView@@6BQObject@@@ 1003057c     alm_db_output.obj
 0002:0000a590       ??_R3QListView@@8          10030590     alm_db_output.obj
 0002:0000a5a0       ??_R2QListView@@8          100305a0     alm_db_output.obj
 0002:0000a5c0       ??_R1A@?0A@EA@QListView@@8 100305c0     alm_db_output.obj
 0002:0000a5dc       ??_R1A@?0A@EA@QScrollView@@8 100305dc     alm_db_output.obj
 0002:0000a5f8       ??_R3QScrollView@@8        100305f8     alm_db_output.obj
 0002:0000a608       ??_R2QScrollView@@8        10030608     alm_db_output.obj
 0002:0000a624       ??_R4QListView@@6BQPaintDevice@@@ 10030624     alm_db_output.obj
 0002:0000a638       ??_R4QListViewItem@@6B@    10030638     alm_db_output.obj
 0002:0000a64c       ??_R3QListViewItem@@8      1003064c     alm_db_output.obj
 0002:0000a65c       ??_R2QListViewItem@@8      1003065c     alm_db_output.obj
 0002:0000a668       ??_R1A@?0A@EA@QListViewItem@@8 10030668     alm_db_output.obj
 0002:0000a684       ??_R4QFile@@6B@            10030684     alm_db_output.obj
 0002:0000a698       ??_R3QFile@@8              10030698     alm_db_output.obj
 0002:0000a6a8       ??_R2QFile@@8              100306a8     alm_db_output.obj
 0002:0000a6b4       ??_R1A@?0A@EA@QFile@@8     100306b4     alm_db_output.obj
 0002:0000a6d0       ??_R1A@?0A@EA@QIODevice@@8 100306d0     alm_db_output.obj
 0002:0000a6ec       ??_R3QIODevice@@8          100306ec     alm_db_output.obj
 0002:0000a6fc       ??_R2QIODevice@@8          100306fc     alm_db_output.obj
 0002:0000a704       ??_R4QTabWidget@@6BQObject@@@ 10030704     alm_db_output.obj
 0002:0000a718       ??_R3QTabWidget@@8         10030718     alm_db_output.obj
 0002:0000a728       ??_R2QTabWidget@@8         10030728     alm_db_output.obj
 0002:0000a740       ??_R1A@?0A@EA@QTabWidget@@8 10030740     alm_db_output.obj
 0002:0000a75c       ??_R4QTabWidget@@6BQPaintDevice@@@ 1003075c     alm_db_output.obj
 0002:0000a770       ??_R1A@?0A@EA@QGDict@@8    10030770     alm_db_output.obj
 0002:0000a78c       ??_R3QGDict@@8             1003078c     alm_db_output.obj
 0002:0000a79c       ??_R2QGDict@@8             1003079c     alm_db_output.obj
 0002:0000a7a8       ??_R4error_category@std@@6B@ 100307a8     alm_db_output.obj
 0002:0000a7bc       ??_R3error_category@std@@8 100307bc     alm_db_output.obj
 0002:0000a7cc       ??_R2error_category@std@@8 100307cc     alm_db_output.obj
 0002:0000a7d4       ??_R1A@?0A@EA@error_category@std@@8 100307d4     alm_db_output.obj
 0002:0000a7f0       ??_R4_Generic_error_category@std@@6B@ 100307f0     alm_db_output.obj
 0002:0000a804       ??_R3_Generic_error_category@std@@8 10030804     alm_db_output.obj
 0002:0000a814       ??_R2_Generic_error_category@std@@8 10030814     alm_db_output.obj
 0002:0000a820       ??_R1A@?0A@EA@_Generic_error_category@std@@8 10030820     alm_db_output.obj
 0002:0000a83c       ??_R4_Iostream_error_category@std@@6B@ 1003083c     alm_db_output.obj
 0002:0000a850       ??_R3_Iostream_error_category@std@@8 10030850     alm_db_output.obj
 0002:0000a860       ??_R2_Iostream_error_category@std@@8 10030860     alm_db_output.obj
 0002:0000a870       ??_R1A@?0A@EA@_Iostream_error_category@std@@8 10030870     alm_db_output.obj
 0002:0000a88c       ??_R4_System_error_category@std@@6B@ 1003088c     alm_db_output.obj
 0002:0000a8a0       ??_R3_System_error_category@std@@8 100308a0     alm_db_output.obj
 0002:0000a8b0       ??_R2_System_error_category@std@@8 100308b0     alm_db_output.obj
 0002:0000a8c0       ??_R1A@?0A@EA@_System_error_category@std@@8 100308c0     alm_db_output.obj
 0002:0000a8dc       ??_R4CAlm_sys_select@@6BQObject@@@ 100308dc     alm_db_output.obj
 0002:0000a8f0       ??_R3CAlm_sys_select@@8    100308f0     alm_db_output.obj
 0002:0000a900       ??_R2CAlm_sys_select@@8    10030900     alm_db_output.obj
 0002:0000a924       ??_R1A@?0A@EA@CAlm_sys_select@@8 10030924     alm_db_output.obj
 0002:0000a940       ??_R1A@?0A@EA@QVBox@@8     10030940     alm_db_output.obj
 0002:0000a95c       ??_R3QVBox@@8              1003095c     alm_db_output.obj
 0002:0000a96c       ??_R2QVBox@@8              1003096c     alm_db_output.obj
 0002:0000a98c       ??_R1A@?0A@EA@QHBox@@8     1003098c     alm_db_output.obj
 0002:0000a9a8       ??_R3QHBox@@8              100309a8     alm_db_output.obj
 0002:0000a9b8       ??_R2QHBox@@8              100309b8     alm_db_output.obj
 0002:0000a9d4       ??_R4CAlm_sys_select@@6BQPaintDevice@@@ 100309d4     alm_db_output.obj
 0002:0000a9e8       ??_R4QGuardedPtrPrivate@@6B@ 100309e8     alm_db_output.obj
 0002:0000a9fc       ??_R3QGuardedPtrPrivate@@8 100309fc     alm_db_output.obj
 0002:0000aa0c       ??_R2QGuardedPtrPrivate@@8 10030a0c     alm_db_output.obj
 0002:0000aa20       ??_R1A@?0A@EA@QGuardedPtrPrivate@@8 10030a20     alm_db_output.obj
 0002:0000aa3c       ??_R1CI@?0A@EA@QShared@@8  10030a3c     alm_db_output.obj
 0002:0000aa58       ??_R4QDockWindowList@@6B@  10030a58     alm_db_output.obj
 0002:0000aa6c       ??_R3QDockWindowList@@8    10030a6c     alm_db_output.obj
 0002:0000aa7c       ??_R2QDockWindowList@@8    10030a7c     alm_db_output.obj
 0002:0000aa90       ??_R1A@?0A@EA@QDockWindowList@@8 10030a90     alm_db_output.obj
 0002:0000aaac       ??_R1A@?0A@EA@?$QPtrList@VQDockWindow@@@@8 10030aac     alm_db_output.obj
 0002:0000aac8       ??_R3?$QPtrList@VQDockWindow@@@@8 10030ac8     alm_db_output.obj
 0002:0000aad8       ??_R2?$QPtrList@VQDockWindow@@@@8 10030ad8     alm_db_output.obj
 0002:0000aae8       ??_R4QPopupMenuList@@6B@   10030ae8     alm_db_output.obj
 0002:0000aafc       ??_R3QPopupMenuList@@8     10030afc     alm_db_output.obj
 0002:0000ab0c       ??_R2QPopupMenuList@@8     10030b0c     alm_db_output.obj
 0002:0000ab20       ??_R1A@?0A@EA@QPopupMenuList@@8 10030b20     alm_db_output.obj
 0002:0000ab3c       ??_R1A@?0A@EA@?$QPtrList@VQPopupMenu@@@@8 10030b3c     alm_db_output.obj
 0002:0000ab58       ??_R3?$QPtrList@VQPopupMenu@@@@8 10030b58     alm_db_output.obj
 0002:0000ab68       ??_R2?$QPtrList@VQPopupMenu@@@@8 10030b68     alm_db_output.obj
 0002:0000ab78       ??_R4?$QPtrList@VQPopupMenu@@@@6B@ 10030b78     alm_db_output.obj
 0002:0000ab8c       ??_R4IGetDocuments@@6B@    10030b8c     alm_db_output.obj
 0002:0000aba0       ??_R3IGetDocuments@@8      10030ba0     alm_db_output.obj
 0002:0000abb0       ??_R2IGetDocuments@@8      10030bb0     alm_db_output.obj
 0002:0000abb8       ??_R1A@?0A@EA@IGetDocuments@@8 10030bb8     alm_db_output.obj
 0002:0000abd4       ??_R4ISendCommand@@6B@     10030bd4     alm_db_output.obj
 0002:0000abe8       ??_R3ISendCommand@@8       10030be8     alm_db_output.obj
 0002:0000abf8       ??_R2ISendCommand@@8       10030bf8     alm_db_output.obj
 0002:0000ac00       ??_R1A@?0A@EA@ISendCommand@@8 10030c00     alm_db_output.obj
 0002:0000ac1c       ??_R4config_plugin_base@@6BQObject@@@ 10030c1c     alm_db_output.obj
 0002:0000ac30       ??_R3config_plugin_base@@8 10030c30     alm_db_output.obj
 0002:0000ac40       ??_R2config_plugin_base@@8 10030c40     alm_db_output.obj
 0002:0000ac58       ??_R1A@?0A@EA@config_plugin_base@@8 10030c58     alm_db_output.obj
 0002:0000ac74       ??_R4config_plugin_base@@6BQPaintDevice@@@ 10030c74     alm_db_output.obj
 0002:0000ac88       ??_R4alm_db_output@@6BQObject@@@ 10030c88     alm_db_output.obj
 0002:0000ac9c       ??_R3alm_db_output@@8      10030c9c     alm_db_output.obj
 0002:0000acac       ??_R2alm_db_output@@8      10030cac     alm_db_output.obj
 0002:0000acd0       ??_R1A@?0A@EA@alm_db_output@@8 10030cd0     alm_db_output.obj
 0002:0000acec       ??_R1HI@?0A@EA@IGetDocuments@@8 10030cec     alm_db_output.obj
 0002:0000ad08       ??_R1HM@?0A@EA@ISendCommand@@8 10030d08     alm_db_output.obj
 0002:0000ad24       ??_R4alm_db_output@@6BQPaintDevice@@@ 10030d24     alm_db_output.obj
 0002:0000ad38       ??_R4alm_db_output@@6BIGetDocuments@@@ 10030d38     alm_db_output.obj
 0002:0000ad4c       ??_R4alm_db_output@@6BISendCommand@@@ 10030d4c     alm_db_output.obj
 0002:0000ad60       ??_R4FileLoad_BncsSystem@alm_db_output@@6B@ 10030d60     alm_db_output.obj
 0002:0000ad74       ??_R3FileLoad_BncsSystem@alm_db_output@@8 10030d74     alm_db_output.obj
 0002:0000ad84       ??_R2FileLoad_BncsSystem@alm_db_output@@8 10030d84     alm_db_output.obj
 0002:0000ad90       ??_R1A@?0A@EA@FileLoad_BncsSystem@alm_db_output@@8 10030d90     alm_db_output.obj
 0002:0000adac       ??_R1A@?0A@EA@FileLoad@@8  10030dac     alm_db_output.obj
 0002:0000adc8       ??_R3FileLoad@@8           10030dc8     alm_db_output.obj
 0002:0000add8       ??_R2FileLoad@@8           10030dd8     alm_db_output.obj
 0002:0000ade0       ??_R4?$QDict@VQAction@@@@6B@ 10030de0     alm_db_output.obj
 0002:0000adf4       ??_R3?$QDict@VQAction@@@@8 10030df4     alm_db_output.obj
 0002:0000ae04       ??_R2?$QDict@VQAction@@@@8 10030e04     alm_db_output.obj
 0002:0000ae14       ??_R1A@?0A@EA@?$QDict@VQAction@@@@8 10030e14     alm_db_output.obj
 0002:0000ae30       ??_R4?$QPtrList@VcOutputFile@@@@6B@ 10030e30     alm_db_output.obj
 0002:0000ae44       ??_R3?$QPtrList@VcOutputFile@@@@8 10030e44     alm_db_output.obj
 0002:0000ae54       ??_R2?$QPtrList@VcOutputFile@@@@8 10030e54     alm_db_output.obj
 0002:0000ae64       ??_R1A@?0A@EA@?$QPtrList@VcOutputFile@@@@8 10030e64     alm_db_output.obj
 0002:0000ae80       ??_R4?$QPtrList@VcProcess@@@@6B@ 10030e80     alm_db_output.obj
 0002:0000ae94       ??_R3?$QPtrList@VcProcess@@@@8 10030e94     alm_db_output.obj
 0002:0000aea4       ??_R2?$QPtrList@VcProcess@@@@8 10030ea4     alm_db_output.obj
 0002:0000aeb4       ??_R1A@?0A@EA@?$QPtrList@VcProcess@@@@8 10030eb4     alm_db_output.obj
 0002:0000aed0       ??_R4cOutputFile@@6B@      10030ed0     cOutputFile.obj
 0002:0000aee4       ??_R3cOutputFile@@8        10030ee4     cOutputFile.obj
 0002:0000aef4       ??_R2cOutputFile@@8        10030ef4     cOutputFile.obj
 0002:0000aefc       ??_R1A@?0A@EA@cOutputFile@@8 10030efc     cOutputFile.obj
 0002:0000af18       ??_R4cProcess@@6B@         10030f18     cProcess.obj
 0002:0000af2c       ??_R3cProcess@@8           10030f2c     cProcess.obj
 0002:0000af3c       ??_R2cProcess@@8           10030f3c     cProcess.obj
 0002:0000af44       ??_R1A@?0A@EA@cProcess@@8  10030f44     cProcess.obj
 0002:0000af60       ??_R4dbConnection@@6B@     10030f60     DBCONNECTION.obj
 0002:0000af74       ??_R3dbConnection@@8       10030f74     DBCONNECTION.obj
 0002:0000af84       ??_R2dbConnection@@8       10030f84     DBCONNECTION.obj
 0002:0000af94       ??_R1A@?0A@EA@dbConnection@@8 10030f94     DBCONNECTION.obj
 0002:0000afb0       ??_R1A@?0A@EA@QThread@@8   10030fb0     DBCONNECTION.obj
 0002:0000afcc       ??_R3QThread@@8            10030fcc     DBCONNECTION.obj
 0002:0000afdc       ??_R2QThread@@8            10030fdc     DBCONNECTION.obj
 0002:0000afe8       ??_R4QTimer@@6B@           10030fe8     dialogimpl.obj
 0002:0000affc       ??_R3QTimer@@8             10030ffc     dialogimpl.obj
 0002:0000b00c       ??_R2QTimer@@8             1003100c     dialogimpl.obj
 0002:0000b01c       ??_R1A@?0A@EA@QTimer@@8    1003101c     dialogimpl.obj
 0002:0000b038       ??_R4dialog@@6BQObject@@@  10031038     dialogimpl.obj
 0002:0000b04c       ??_R3dialog@@8             1003104c     dialogimpl.obj
 0002:0000b05c       ??_R2dialog@@8             1003105c     dialogimpl.obj
 0002:0000b078       ??_R1A@?0A@EA@dialog@@8    10031078     dialogimpl.obj
 0002:0000b094       ??_R1A@?0A@EA@dialogBase@@8 10031094     dialogimpl.obj
 0002:0000b0b0       ??_R3dialogBase@@8         100310b0     dialogimpl.obj
 0002:0000b0c0       ??_R2dialogBase@@8         100310c0     dialogimpl.obj
 0002:0000b0d8       ??_R4dialog@@6BQPaintDevice@@@ 100310d8     dialogimpl.obj
 0002:0000b0ec       ??_R4QSqlCursor@@6BQSqlRecord@@@ 100310ec     dialogimpl.obj
 0002:0000b100       ??_R3QSqlCursor@@8         10031100     dialogimpl.obj
 0002:0000b110       ??_R2QSqlCursor@@8         10031110     dialogimpl.obj
 0002:0000b120       ??_R1A@?0A@EA@QSqlCursor@@8 10031120     dialogimpl.obj
 0002:0000b13c       ??_R1A@?0A@EA@QSqlRecord@@8 1003113c     dialogimpl.obj
 0002:0000b158       ??_R3QSqlRecord@@8         10031158     dialogimpl.obj
 0002:0000b168       ??_R2QSqlRecord@@8         10031168     dialogimpl.obj
 0002:0000b170       ??_R17?0A@EA@QSqlQuery@@8  10031170     dialogimpl.obj
 0002:0000b18c       ??_R3QSqlQuery@@8          1003118c     dialogimpl.obj
 0002:0000b19c       ??_R2QSqlQuery@@8          1003119c     dialogimpl.obj
 0002:0000b1a4       ??_R1A@?0A@EA@QSqlQuery@@8 100311a4     dialogimpl.obj
 0002:0000b1c0       ??_R4QSqlCursor@@6BQSqlQuery@@@ 100311c0     dialogimpl.obj
 0002:0000b1d4       ??_R4QCheckTableItem@@6B@  100311d4     manage_tempimpl.obj
 0002:0000b1e8       ??_R3QCheckTableItem@@8    100311e8     manage_tempimpl.obj
 0002:0000b1f8       ??_R2QCheckTableItem@@8    100311f8     manage_tempimpl.obj
 0002:0000b208       ??_R1A@?0A@EA@QCheckTableItem@@8 10031208     manage_tempimpl.obj
 0002:0000b224       ??_R1A@?0A@EA@QTableItem@@8 10031224     manage_tempimpl.obj
 0002:0000b240       ??_R3QTableItem@@8         10031240     manage_tempimpl.obj
 0002:0000b250       ??_R2QTableItem@@8         10031250     manage_tempimpl.obj
 0002:0000b25c       ??_R4manage_temp@@6BQObject@@@ 1003125c     manage_tempimpl.obj
 0002:0000b270       ??_R3manage_temp@@8        10031270     manage_tempimpl.obj
 0002:0000b280       ??_R2manage_temp@@8        10031280     manage_tempimpl.obj
 0002:0000b2a0       ??_R1A@?0A@EA@manage_temp@@8 100312a0     manage_tempimpl.obj
 0002:0000b2bc       ??_R1A@?0A@EA@manage_tempBase@@8 100312bc     manage_tempimpl.obj
 0002:0000b2d8       ??_R3manage_tempBase@@8    100312d8     manage_tempimpl.obj
 0002:0000b2e8       ??_R2manage_tempBase@@8    100312e8     manage_tempimpl.obj
 0002:0000b304       ??_R1A@?0A@EA@QDialog@@8   10031304     manage_tempimpl.obj
 0002:0000b320       ??_R3QDialog@@8            10031320     manage_tempimpl.obj
 0002:0000b330       ??_R2QDialog@@8            10031330     manage_tempimpl.obj
 0002:0000b348       ??_R4manage_temp@@6BQPaintDevice@@@ 10031348     manage_tempimpl.obj
 0002:0000b35c       ??_R4config_plugin_desc_base@@6B@ 1003135c     plugindesc.obj
 0002:0000b370       ??_R3config_plugin_desc_base@@8 10031370     plugindesc.obj
 0002:0000b380       ??_R2config_plugin_desc_base@@8 10031380     plugindesc.obj
 0002:0000b388       ??_R1A@?0A@EA@config_plugin_desc_base@@8 10031388     plugindesc.obj
 0002:0000b3a4       ??_R4plugindesc@@6B@       100313a4     plugindesc.obj
 0002:0000b3b8       ??_R3plugindesc@@8         100313b8     plugindesc.obj
 0002:0000b3c8       ??_R2plugindesc@@8         100313c8     plugindesc.obj
 0002:0000b3d4       ??_R1A@?0A@EA@plugindesc@@8 100313d4     plugindesc.obj
 0002:0000b3f0       ??_R4processList@@6B@      100313f0     processList.obj
 0002:0000b404       ??_R3processList@@8        10031404     processList.obj
 0002:0000b414       ??_R2processList@@8        10031414     processList.obj
 0002:0000b41c       ??_R1A@?0A@EA@processList@@8 1003141c     processList.obj
 0002:0000b438       ??_R4QPushButton@@6BQObject@@@ 10031438     setdefaults.obj
 0002:0000b44c       ??_R3QPushButton@@8        1003144c     setdefaults.obj
 0002:0000b45c       ??_R2QPushButton@@8        1003145c     setdefaults.obj
 0002:0000b478       ??_R1A@?0A@EA@QPushButton@@8 10031478     setdefaults.obj
 0002:0000b494       ??_R1A@?0A@EA@QButton@@8   10031494     setdefaults.obj
 0002:0000b4b0       ??_R3QButton@@8            100314b0     setdefaults.obj
 0002:0000b4c0       ??_R2QButton@@8            100314c0     setdefaults.obj
 0002:0000b4d8       ??_R4QPushButton@@6BQPaintDevice@@@ 100314d8     setdefaults.obj
 0002:0000b4ec       ??_R4QVBoxLayout@@6BQObject@@@ 100314ec     setdefaults.obj
 0002:0000b500       ??_R3QVBoxLayout@@8        10031500     setdefaults.obj
 0002:0000b510       ??_R2QVBoxLayout@@8        10031510     setdefaults.obj
 0002:0000b52c       ??_R1A@?0A@EA@QVBoxLayout@@8 1003152c     setdefaults.obj
 0002:0000b548       ??_R4QVBoxLayout@@6BQLayoutItem@@@ 10031548     setdefaults.obj
 0002:0000b55c       ??_R4QHBoxLayout@@6BQObject@@@ 1003155c     setdefaults.obj
 0002:0000b570       ??_R3QHBoxLayout@@8        10031570     setdefaults.obj
 0002:0000b580       ??_R2QHBoxLayout@@8        10031580     setdefaults.obj
 0002:0000b59c       ??_R1A@?0A@EA@QHBoxLayout@@8 1003159c     setdefaults.obj
 0002:0000b5b8       ??_R4QHBoxLayout@@6BQLayoutItem@@@ 100315b8     setdefaults.obj
 0002:0000b5cc       ??_R4QGridLayout@@6BQObject@@@ 100315cc     setdefaults.obj
 0002:0000b5e0       ??_R3QGridLayout@@8        100315e0     setdefaults.obj
 0002:0000b5f0       ??_R2QGridLayout@@8        100315f0     setdefaults.obj
 0002:0000b608       ??_R1A@?0A@EA@QGridLayout@@8 10031608     setdefaults.obj
 0002:0000b624       ??_R4QGridLayout@@6BQLayoutItem@@@ 10031624     setdefaults.obj
 0002:0000b638       ??_R4QGroupBox@@6BQObject@@@ 10031638     setdefaults.obj
 0002:0000b64c       ??_R3QGroupBox@@8          1003164c     setdefaults.obj
 0002:0000b65c       ??_R2QGroupBox@@8          1003165c     setdefaults.obj
 0002:0000b678       ??_R1A@?0A@EA@QGroupBox@@8 10031678     setdefaults.obj
 0002:0000b694       ??_R4QGroupBox@@6BQPaintDevice@@@ 10031694     setdefaults.obj
 0002:0000b6a8       ??_R4QLabel@@6BQObject@@@  100316a8     setdefaults.obj
 0002:0000b6bc       ??_R3QLabel@@8             100316bc     setdefaults.obj
 0002:0000b6cc       ??_R2QLabel@@8             100316cc     setdefaults.obj
 0002:0000b6e8       ??_R1A@?0A@EA@QLabel@@8    100316e8     setdefaults.obj
 0002:0000b704       ??_R4QLabel@@6BQPaintDevice@@@ 10031704     setdefaults.obj
 0002:0000b718       ??_R4QLineEdit@@6BQObject@@@ 10031718     setdefaults.obj
 0002:0000b72c       ??_R3QLineEdit@@8          1003172c     setdefaults.obj
 0002:0000b73c       ??_R2QLineEdit@@8          1003173c     setdefaults.obj
 0002:0000b758       ??_R1A@?0A@EA@QLineEdit@@8 10031758     setdefaults.obj
 0002:0000b774       ??_R4QLineEdit@@6BQPaintDevice@@@ 10031774     setdefaults.obj
 0002:0000b788       ??_R4QComboBox@@6BQObject@@@ 10031788     setdefaults.obj
 0002:0000b79c       ??_R3QComboBox@@8          1003179c     setdefaults.obj
 0002:0000b7ac       ??_R2QComboBox@@8          100317ac     setdefaults.obj
 0002:0000b7c4       ??_R1A@?0A@EA@QComboBox@@8 100317c4     setdefaults.obj
 0002:0000b7e0       ??_R4QComboBox@@6BQPaintDevice@@@ 100317e0     setdefaults.obj
 0002:0000b7f4       ??_R4QCheckBox@@6BQObject@@@ 100317f4     setdefaults.obj
 0002:0000b808       ??_R3QCheckBox@@8          10031808     setdefaults.obj
 0002:0000b818       ??_R2QCheckBox@@8          10031818     setdefaults.obj
 0002:0000b834       ??_R1A@?0A@EA@QCheckBox@@8 10031834     setdefaults.obj
 0002:0000b850       ??_R4QCheckBox@@6BQPaintDevice@@@ 10031850     setdefaults.obj
 0002:0000b864       ??_R4setDefaultsBase@@6BQObject@@@ 10031864     setdefaults.obj
 0002:0000b878       ??_R3setDefaultsBase@@8    10031878     setdefaults.obj
 0002:0000b888       ??_R2setDefaultsBase@@8    10031888     setdefaults.obj
 0002:0000b8a4       ??_R1A@?0A@EA@setDefaultsBase@@8 100318a4     setdefaults.obj
 0002:0000b8c0       ??_R4setDefaultsBase@@6BQPaintDevice@@@ 100318c0     setdefaults.obj
 0002:0000b8d4       ??_R4QSpacerItem@@6B@      100318d4     setdefaults.obj
 0002:0000b8e8       ??_R3QSpacerItem@@8        100318e8     setdefaults.obj
 0002:0000b8f8       ??_R2QSpacerItem@@8        100318f8     setdefaults.obj
 0002:0000b904       ??_R1A@?0A@EA@QSpacerItem@@8 10031904     setdefaults.obj
 0002:0000b920       ??_R4setDefaults@@6BQObject@@@ 10031920     setdefaultsimpl.obj
 0002:0000b934       ??_R3setDefaults@@8        10031934     setdefaultsimpl.obj
 0002:0000b944       ??_R2setDefaults@@8        10031944     setdefaultsimpl.obj
 0002:0000b964       ??_R1A@?0A@EA@setDefaults@@8 10031964     setdefaultsimpl.obj
 0002:0000b980       ??_R4setDefaults@@6BQPaintDevice@@@ 10031980     setdefaultsimpl.obj
 0002:0000b994       ??_R4QSpinBox@@6BQObject@@@ 10031994     dialog.obj
 0002:0000b9a8       ??_R3QSpinBox@@8           100319a8     dialog.obj
 0002:0000b9b8       ??_R2QSpinBox@@8           100319b8     dialog.obj
 0002:0000b9d4       ??_R1A@?0A@EA@QSpinBox@@8  100319d4     dialog.obj
 0002:0000b9f0       ??_R1GM@?0A@EA@QRangeControl@@8 100319f0     dialog.obj
 0002:0000ba0c       ??_R3QRangeControl@@8      10031a0c     dialog.obj
 0002:0000ba1c       ??_R2QRangeControl@@8      10031a1c     dialog.obj
 0002:0000ba24       ??_R1A@?0A@EA@QRangeControl@@8 10031a24     dialog.obj
 0002:0000ba40       ??_R4QSpinBox@@6BQPaintDevice@@@ 10031a40     dialog.obj
 0002:0000ba54       ??_R4QSpinBox@@6B@         10031a54     dialog.obj
 0002:0000ba68       ??_R4QButtonGroup@@6BQObject@@@ 10031a68     dialog.obj
 0002:0000ba7c       ??_R3QButtonGroup@@8       10031a7c     dialog.obj
 0002:0000ba8c       ??_R2QButtonGroup@@8       10031a8c     dialog.obj
 0002:0000baac       ??_R1A@?0A@EA@QButtonGroup@@8 10031aac     dialog.obj
 0002:0000bac8       ??_R4QButtonGroup@@6BQPaintDevice@@@ 10031ac8     dialog.obj
 0002:0000badc       ??_R4QSplitter@@6BQObject@@@ 10031adc     dialog.obj
 0002:0000baf0       ??_R3QSplitter@@8          10031af0     dialog.obj
 0002:0000bb00       ??_R2QSplitter@@8          10031b00     dialog.obj
 0002:0000bb1c       ??_R1A@?0A@EA@QSplitter@@8 10031b1c     dialog.obj
 0002:0000bb38       ??_R4QSplitter@@6BQPaintDevice@@@ 10031b38     dialog.obj
 0002:0000bb4c       ??_R4QRadioButton@@6BQObject@@@ 10031b4c     dialog.obj
 0002:0000bb60       ??_R3QRadioButton@@8       10031b60     dialog.obj
 0002:0000bb70       ??_R2QRadioButton@@8       10031b70     dialog.obj
 0002:0000bb8c       ??_R1A@?0A@EA@QRadioButton@@8 10031b8c     dialog.obj
 0002:0000bba8       ??_R4QRadioButton@@6BQPaintDevice@@@ 10031ba8     dialog.obj
 0002:0000bbbc       ??_R4QDateEdit@@6BQObject@@@ 10031bbc     dialog.obj
 0002:0000bbd0       ??_R3QDateEdit@@8          10031bd0     dialog.obj
 0002:0000bbe0       ??_R2QDateEdit@@8          10031be0     dialog.obj
 0002:0000bbfc       ??_R1A@?0A@EA@QDateEdit@@8 10031bfc     dialog.obj
 0002:0000bc18       ??_R1A@?0A@EA@QDateTimeEditBase@@8 10031c18     dialog.obj
 0002:0000bc34       ??_R3QDateTimeEditBase@@8  10031c34     dialog.obj
 0002:0000bc44       ??_R2QDateTimeEditBase@@8  10031c44     dialog.obj
 0002:0000bc5c       ??_R4QDateEdit@@6BQPaintDevice@@@ 10031c5c     dialog.obj
 0002:0000bc70       ??_R4QDataTable@@6BQObject@@@ 10031c70     dialog.obj
 0002:0000bc84       ??_R3QDataTable@@8         10031c84     dialog.obj
 0002:0000bc94       ??_R2QDataTable@@8         10031c94     dialog.obj
 0002:0000bcb8       ??_R1A@?0A@EA@QDataTable@@8 10031cb8     dialog.obj
 0002:0000bcd4       ??_R1A@?0A@EA@QTable@@8    10031cd4     dialog.obj
 0002:0000bcf0       ??_R3QTable@@8             10031cf0     dialog.obj
 0002:0000bd00       ??_R2QTable@@8             10031d00     dialog.obj
 0002:0000bd20       ??_R4QDataTable@@6BQPaintDevice@@@ 10031d20     dialog.obj
 0002:0000bd34       ??_R4dialogBase@@6BQObject@@@ 10031d34     dialog.obj
 0002:0000bd48       ??_R4dialogBase@@6BQPaintDevice@@@ 10031d48     dialog.obj
 0002:0000bd5c       ??_R4QTable@@6BQObject@@@  10031d5c     manage_temp.obj
 0002:0000bd70       ??_R4QTable@@6BQPaintDevice@@@ 10031d70     manage_temp.obj
 0002:0000bd84       ??_R4manage_tempBase@@6BQObject@@@ 10031d84     manage_temp.obj
 0002:0000bd98       ??_R4manage_tempBase@@6BQPaintDevice@@@ 10031d98     manage_temp.obj
 0002:0000bdac       ??_R4Document@@6B@         10031dac     config_alarm_utilities:Document.obj
 0002:0000bdc0       ??_R3Document@@8           10031dc0     config_alarm_utilities:Document.obj
 0002:0000bdd0       ??_R2Document@@8           10031dd0     config_alarm_utilities:Document.obj
 0002:0000bdd8       ??_R1A@?0A@EA@Document@@8  10031dd8     config_alarm_utilities:Document.obj
 0002:0000bdf4       ??_R4Document_BncsSystem@@6B@ 10031df4     config_alarm_utilities:Document.obj
 0002:0000be08       ??_R3Document_BncsSystem@@8 10031e08     config_alarm_utilities:Document.obj
 0002:0000be18       ??_R2Document_BncsSystem@@8 10031e18     config_alarm_utilities:Document.obj
 0002:0000be24       ??_R1A@?0A@EA@Document_BncsSystem@@8 10031e24     config_alarm_utilities:Document.obj
 0002:0000be40       ??_R1A@?0A@EN@Document@@8  10031e40     config_alarm_utilities:Document.obj
 0002:0000be5c       ??_R4FileLoad@@6B@         10031e5c     config_alarm_utilities:Loaders.obj
 0002:0000be70       ??_R4Loaders@@6B@          10031e70     config_alarm_utilities:Loaders.obj
 0002:0000be84       ??_R3Loaders@@8            10031e84     config_alarm_utilities:Loaders.obj
 0002:0000be94       ??_R2Loaders@@8            10031e94     config_alarm_utilities:Loaders.obj
 0002:0000be9c       ??_R1A@?0A@EA@Loaders@@8   10031e9c     config_alarm_utilities:Loaders.obj
 0002:0000beb8       ??_R4?$QPtrList@VFileLoad@@@@6B@ 10031eb8     config_alarm_utilities:Loaders.obj
 0002:0000becc       ??_R3?$QPtrList@VFileLoad@@@@8 10031ecc     config_alarm_utilities:Loaders.obj
 0002:0000bedc       ??_R2?$QPtrList@VFileLoad@@@@8 10031edc     config_alarm_utilities:Loaders.obj
 0002:0000beec       ??_R1A@?0A@EA@?$QPtrList@VFileLoad@@@@8 10031eec     config_alarm_utilities:Loaders.obj
 0002:0000bf08       ??_R4?$QPtrList@VDirLoad@@@@6B@ 10031f08     config_alarm_utilities:Loaders.obj
 0002:0000bf1c       ??_R3?$QPtrList@VDirLoad@@@@8 10031f1c     config_alarm_utilities:Loaders.obj
 0002:0000bf2c       ??_R2?$QPtrList@VDirLoad@@@@8 10031f2c     config_alarm_utilities:Loaders.obj
 0002:0000bf3c       ??_R1A@?0A@EA@?$QPtrList@VDirLoad@@@@8 10031f3c     config_alarm_utilities:Loaders.obj
 0002:0000bf58       ??_R4type_info@@6B@        10031f58     MSVCRT:ti_inst.obj
 0002:0000bf6c       ??_R3type_info@@8          10031f6c     MSVCRT:ti_inst.obj
 0002:0000bf7c       ??_R2type_info@@8          10031f7c     MSVCRT:ti_inst.obj
 0002:0000bf84       ??_R1A@?0A@EA@type_info@@8 10031f84     MSVCRT:ti_inst.obj
 0002:0000bfa0       ___rtc_iaa                 10031fa0     MSVCRT:initsect.obj
 0002:0000bfa4       ___rtc_izz                 10031fa4     MSVCRT:initsect.obj
 0002:0000bfa8       ___rtc_taa                 10031fa8     MSVCRT:initsect.obj
 0002:0000bfac       ___rtc_tzz                 10031fac     MSVCRT:initsect.obj
 0002:00010858       __IMPORT_DESCRIPTOR_qt-mt323 10036858     qt-mt323:qt-mt323.dll
 0002:0001086c       __IMPORT_DESCRIPTOR_alm_sys_select 1003686c     alm_sys_select:alm_sys_select.dll
 0002:00010880       __IMPORT_DESCRIPTOR_config_icons 10036880     config_icons:config_icons.dll
 0002:00010894       __IMPORT_DESCRIPTOR_KERNEL32 10036894     kernel32:KERNEL32.dll
 0002:000108a8       __IMPORT_DESCRIPTOR_MSVCP120 100368a8     msvcprt:MSVCP120.dll
 0002:000108bc       __IMPORT_DESCRIPTOR_MSVCR120 100368bc     MSVCRT:MSVCR120.dll
 0002:000108d0       __NULL_IMPORT_DESCRIPTOR   100368d0     qt-mt323:qt-mt323.dll
 0003:00000000       ?_Generic_object@?$_Error_objects@H@std@@2V_Generic_error_category@2@A 10047000     alm_db_output.obj
 0003:00000004       ?_Iostream_object@?$_Error_objects@H@std@@2V_Iostream_error_category@2@A 10047004     alm_db_output.obj
 0003:00000008       ?_System_object@?$_Error_objects@H@std@@2V_System_error_category@2@A 10047008     alm_db_output.obj
 0003:00000180       ___security_cookie         10047180     MSVCRT:gs_cookie.obj
 0003:00000184       ___security_cookie_complement 10047184     MSVCRT:gs_cookie.obj
 0003:00000190       ___native_dllmain_reason   10047190     MSVCRT:natstart.obj
 0003:00000194       ??_R0?AVQGList@@@8         10047194     alm_db_output.obj
 0003:000001ac       ??_R0?AVQPtrCollection@@@8 100471ac     alm_db_output.obj
 0003:000001cc       ??_R0?AVQWidget@@@8        100471cc     alm_db_output.obj
 0003:000001e4       ??_R0?AVQObject@@@8        100471e4     alm_db_output.obj
 0003:000001fc       ??_R0?AVQt@@@8             100471fc     alm_db_output.obj
 0003:00000210       ??_R0?AVQPaintDevice@@@8   10047210     alm_db_output.obj
 0003:0000022c       ??_R0?AUQShared@@@8        1004722c     alm_db_output.obj
 0003:00000244       ??_R0?AVQPopupMenu@@@8     10047244     alm_db_output.obj
 0003:00000260       ??_R0?AVQFrame@@@8         10047260     alm_db_output.obj
 0003:00000278       ??_R0?AVQMenuData@@@8      10047278     alm_db_output.obj
 0003:00000290       ??_R0?AVQAction@@@8        10047290     alm_db_output.obj
 0003:000002a8       ??_R0?AVQBoxLayout@@@8     100472a8     alm_db_output.obj
 0003:000002c4       ??_R0?AVQLayout@@@8        100472c4     alm_db_output.obj
 0003:000002dc       ??_R0?AVQLayoutItem@@@8    100472dc     alm_db_output.obj
 0003:000002f8       ??_R0?AVQToolBar@@@8       100472f8     alm_db_output.obj
 0003:00000310       ??_R0?AVQDockWindow@@@8    10047310     alm_db_output.obj
 0003:0000032c       ??_R0?AVQListView@@@8      1004732c     alm_db_output.obj
 0003:00000344       ??_R0?AVQScrollView@@@8    10047344     alm_db_output.obj
 0003:00000360       ??_R0?AVQListViewItem@@@8  10047360     alm_db_output.obj
 0003:0000037c       ??_R0?AVQFile@@@8          1004737c     alm_db_output.obj
 0003:00000390       ??_R0?AVQIODevice@@@8      10047390     alm_db_output.obj
 0003:000003a8       ??_R0?AVQTabWidget@@@8     100473a8     alm_db_output.obj
 0003:000003c4       ??_R0?AVQGDict@@@8         100473c4     alm_db_output.obj
 0003:000003dc       ??_R0?AVerror_category@std@@@8 100473dc     alm_db_output.obj
 0003:00000400       ??_R0?AV_Generic_error_category@std@@@8 10047400     alm_db_output.obj
 0003:0000042c       ??_R0?AV_Iostream_error_category@std@@@8 1004742c     alm_db_output.obj
 0003:00000458       ??_R0?AV_System_error_category@std@@@8 10047458     alm_db_output.obj
 0003:00000484       ??_R0?AVCAlm_sys_select@@@8 10047484     alm_db_output.obj
 0003:000004a4       ??_R0?AVQVBox@@@8          100474a4     alm_db_output.obj
 0003:000004b8       ??_R0?AVQHBox@@@8          100474b8     alm_db_output.obj
 0003:000004cc       ??_R0?AVQGuardedPtrPrivate@@@8 100474cc     alm_db_output.obj
 0003:000004f0       ??_R0?AVQDockWindowList@@@8 100474f0     alm_db_output.obj
 0003:00000510       ??_R0?AV?$QPtrList@VQDockWindow@@@@@8 10047510     alm_db_output.obj
 0003:00000538       ??_R0?AVQPopupMenuList@@@8 10047538     alm_db_output.obj
 0003:00000558       ??_R0?AV?$QPtrList@VQPopupMenu@@@@@8 10047558     alm_db_output.obj
 0003:00000580       ??_R0?AVIGetDocuments@@@8  10047580     alm_db_output.obj
 0003:0000059c       ??_R0?AVISendCommand@@@8   1004759c     alm_db_output.obj
 0003:000005b8       ??_R0?AVconfig_plugin_base@@@8 100475b8     alm_db_output.obj
 0003:000005dc       ??_R0?AValm_db_output@@@8  100475dc     alm_db_output.obj
 0003:000005f8       ??_R0?AVFileLoad_BncsSystem@alm_db_output@@@8 100475f8     alm_db_output.obj
 0003:00000628       ??_R0?AVFileLoad@@@8       10047628     alm_db_output.obj
 0003:00000640       ??_R0?AV?$QDict@VQAction@@@@@8 10047640     alm_db_output.obj
 0003:00000664       ??_R0?AV?$QPtrList@VcOutputFile@@@@@8 10047664     alm_db_output.obj
 0003:0000068c       ??_R0?AV?$QPtrList@VcProcess@@@@@8 1004768c     alm_db_output.obj
 0003:000006b4       ??_R0?AVcOutputFile@@@8    100476b4     cOutputFile.obj
 0003:000006d0       ??_R0?AVcProcess@@@8       100476d0     cProcess.obj
 0003:000006e8       ??_R0?AVdbConnection@@@8   100476e8     DBCONNECTION.obj
 0003:00000704       ??_R0?AVQThread@@@8        10047704     DBCONNECTION.obj
 0003:0000071c       ??_R0?AVQTimer@@@8         1004771c     dialogimpl.obj
 0003:00000734       ??_R0?AVdialog@@@8         10047734     dialogimpl.obj
 0003:0000074c       ??_R0?AVdialogBase@@@8     1004774c     dialogimpl.obj
 0003:00000768       ??_R0?AVQSqlCursor@@@8     10047768     dialogimpl.obj
 0003:00000784       ??_R0?AVQSqlRecord@@@8     10047784     dialogimpl.obj
 0003:000007a0       ??_R0?AVQSqlQuery@@@8      100477a0     dialogimpl.obj
 0003:000007b8       ??_R0?AVQCheckTableItem@@@8 100477b8     manage_tempimpl.obj
 0003:000007d8       ??_R0?AVQTableItem@@@8     100477d8     manage_tempimpl.obj
 0003:000007f4       ??_R0?AVmanage_temp@@@8    100477f4     manage_tempimpl.obj
 0003:00000810       ??_R0?AVmanage_tempBase@@@8 10047810     manage_tempimpl.obj
 0003:00000830       ??_R0?AVQDialog@@@8        10047830     manage_tempimpl.obj
 0003:00000848       ??_R0?AVconfig_plugin_desc_base@@@8 10047848     plugindesc.obj
 0003:00000870       ??_R0?AVplugindesc@@@8     10047870     plugindesc.obj
 0003:0000088c       ??_R0?AVprocessList@@@8    1004788c     processList.obj
 0003:000008a8       ??_R0?AVQPushButton@@@8    100478a8     setdefaults.obj
 0003:000008c4       ??_R0?AVQButton@@@8        100478c4     setdefaults.obj
 0003:000008dc       ??_R0?AVQVBoxLayout@@@8    100478dc     setdefaults.obj
 0003:000008f8       ??_R0?AVQHBoxLayout@@@8    100478f8     setdefaults.obj
 0003:00000914       ??_R0?AVQGridLayout@@@8    10047914     setdefaults.obj
 0003:00000930       ??_R0?AVQGroupBox@@@8      10047930     setdefaults.obj
 0003:00000948       ??_R0?AVQLabel@@@8         10047948     setdefaults.obj
 0003:00000960       ??_R0?AVQLineEdit@@@8      10047960     setdefaults.obj
 0003:00000978       ??_R0?AVQComboBox@@@8      10047978     setdefaults.obj
 0003:00000990       ??_R0?AVQCheckBox@@@8      10047990     setdefaults.obj
 0003:000009a8       ??_R0?AVsetDefaultsBase@@@8 100479a8     setdefaults.obj
 0003:000009c8       ??_R0?AVQSpacerItem@@@8    100479c8     setdefaults.obj
 0003:000009e4       ??_R0?AVsetDefaults@@@8    100479e4     setdefaultsimpl.obj
 0003:00000a00       ??_R0?AVQSpinBox@@@8       10047a00     dialog.obj
 0003:00000a18       ??_R0?AVQRangeControl@@@8  10047a18     dialog.obj
 0003:00000a34       ??_R0?AVQButtonGroup@@@8   10047a34     dialog.obj
 0003:00000a50       ??_R0?AVQSplitter@@@8      10047a50     dialog.obj
 0003:00000a68       ??_R0?AVQRadioButton@@@8   10047a68     dialog.obj
 0003:00000a84       ??_R0?AVQDateEdit@@@8      10047a84     dialog.obj
 0003:00000a9c       ??_R0?AVQDateTimeEditBase@@@8 10047a9c     dialog.obj
 0003:00000abc       ??_R0?AVQDataTable@@@8     10047abc     dialog.obj
 0003:00000ad8       ??_R0?AVQTable@@@8         10047ad8     dialog.obj
 0003:00000af0       ??_R0?AVDocument@@@8       10047af0     config_alarm_utilities:Document.obj
 0003:00000b08       ??_R0?AVDocument_BncsSystem@@@8 10047b08     config_alarm_utilities:Document.obj
 0003:00000b2c       ??_R0?AVLoaders@@@8        10047b2c     config_alarm_utilities:Loaders.obj
 0003:00000b44       ??_R0?AV?$QPtrList@VFileLoad@@@@@8 10047b44     config_alarm_utilities:Loaders.obj
 0003:00000b6c       ??_R0?AV?$QPtrList@VDirLoad@@@@@8 10047b6c     config_alarm_utilities:Loaders.obj
 0003:00000b90       ??_R0?AVtype_info@@@8      10047b90     MSVCRT:ti_inst.obj
 0003:00000bac       ?id@?$num_put@DV?$back_insert_iterator@V?$basic_string@DU?$char_traits@D@std@@V?$allocator@D@2@@std@@@std@@@std@@2V0locale@2@A 10047bac     alm_db_output.obj
 0003:00000bb0       ?id@?$num_put@_WV?$back_insert_iterator@V?$basic_string@_WU?$char_traits@_W@std@@V?$allocator@_W@2@@std@@@std@@@std@@2V0locale@2@A 10047bb0     alm_db_output.obj
 0003:00000bbc       ?metaObj@setDefaultsBase@@0PAVQMetaObject@@A 10047bbc     moc_setdefaults.obj
 0003:00000bc4       ?metaObj@setDefaults@@0PAVQMetaObject@@A 10047bc4     moc_setdefaultsimpl.obj
 0003:00000bcc       ?metaObj@alm_db_output@@0PAVQMetaObject@@A 10047bcc     moc_alm_db_output.obj
 0003:00000c08       ?metaObj@dialogBase@@0PAVQMetaObject@@A 10047c08     moc_dialog.obj
 0003:00000c10       ?metaObj@dialog@@0PAVQMetaObject@@A 10047c10     moc_dialogimpl.obj
 0003:00000c1c       ?metaObj@manage_tempBase@@0PAVQMetaObject@@A 10047c1c     moc_manage_temp.obj
 0003:00000c24       ?metaObj@manage_temp@@0PAVQMetaObject@@A 10047c24     moc_manage_tempimpl.obj
 0003:00000c40       ?sm_sSystemFolder@Document@@1VQString@@A 10047c40     config_alarm_utilities:Document.obj
 0003:00000f68       ?__type_info_root_node@@3U__type_info_node@@A 10047f68     MSVCRT:tncleanup.obj
 0003:00000f70       ___native_startup_lock     10047f70     <common>
 0003:00000f74       ___native_startup_state    10047f74     <common>
 0003:00000f78       ___dyn_tls_init_callback   10047f78     <common>
 0003:00000f7c       ___onexitend               10047f7c     <common>
 0003:00000f80       ___onexitbegin             10047f80     <common>

 entry point at        0001:0001fa38

 Static symbols

 0001:00000000       ??__E?_Generic_object@?$_Error_objects@H@std@@2V_Generic_error_category@2@A@@YAXXZ 10001000 f   alm_db_output.obj
 0001:0000000c       ??__E?_Iostream_object@?$_Error_objects@H@std@@2V_Iostream_error_category@2@A@@YAXXZ 1000100c f   alm_db_output.obj
 0001:00000018       ??__E?_System_object@?$_Error_objects@H@std@@2V_System_error_category@2@A@@YAXXZ 10001018 f   alm_db_output.obj
 0001:00000024       ??__EcleanUp_setDefaultsBase@@YAXXZ 10001024 f   moc_setdefaults.obj
 0001:00000045       ??__EcleanUp_setDefaults@@YAXXZ 10001045 f   moc_setdefaultsimpl.obj
 0001:00000066       ??__EcleanUp_alm_db_output@@YAXXZ 10001066 f   moc_alm_db_output.obj
 0001:00000087       ??__EcleanUp_dialogBase@@YAXXZ 10001087 f   moc_dialog.obj
 0001:000000a8       ??__EcleanUp_dialog@@YAXXZ 100010a8 f   moc_dialogimpl.obj
 0001:000000c9       ??__EcleanUp_manage_tempBase@@YAXXZ 100010c9 f   moc_manage_temp.obj
 0001:000000ea       ??__EcleanUp_manage_temp@@YAXXZ 100010ea f   moc_manage_tempimpl.obj
 0001:00000110       ??__E?sm_sSystemFolder@Document@@1VQString@@A@@YAXXZ 10001110 f   config_alarm_utilities:Document.obj
 0001:00001bf1       __catch$?_Copy@?$basic_string@DU?$char_traits@D@std@@V?$allocator@D@2@@std@@QAEXII@Z$0 10002bf1 f i alm_db_output.obj
 0001:00001c70       __catch$?_Copy@?$basic_string@DU?$char_traits@D@std@@V?$allocator@D@2@@std@@QAEXII@Z$1 10002c70 f i alm_db_output.obj
 0001:0001bfd0       $LN51                      1001cfd0     moc_alm_db_output.obj
 0001:0001c580       $LN66                      1001d580     moc_dialogimpl.obj
 0001:0001c9d5       $LN39                      1001d9d5     moc_manage_tempimpl.obj
 0001:0001f7f5       _pre_c_init                100207f5 f   MSVCRT:crtdll.obj
 0001:0001fa5b       ___DllMainCRTStartup       10020a5b f   MSVCRT:crtdll.obj
 0001:0001fba0       $$000000                   10020ba0     MSVCRT:sehprolg4.obj
 0001:0001fff0       __unwindfunclet$??0?$QMapNode@VQString@@PAVcProcess@@@@QAE@ABVQString@@@Z$0 10020ff0 f   alm_db_output.obj
 0001:0001fff0       __unwindfunclet$??0?$QMapNode@VQString@@PAVcProcess@@@@QAE@ABU0@@Z$0 10020ff0 f   alm_db_output.obj
 0001:0001fffc       __ehhandler$??0?$QMapNode@VQString@@PAVcProcess@@@@QAE@ABVQString@@@Z 10020ffc f   alm_db_output.obj
 0001:0001fffc       __ehhandler$??0?$QMapNode@VQString@@PAVcProcess@@@@QAE@ABU0@@Z 10020ffc f   alm_db_output.obj
 0001:00020017       __unwindfunclet$??0FileLoad_BncsSystem@alm_db_output@@QAE@PAV1@@Z$0 10021017 f   alm_db_output.obj
 0001:00020020       __unwindfunclet$??0FileLoad_BncsSystem@alm_db_output@@QAE@PAV1@@Z$1 10021020 f   alm_db_output.obj
 0001:00020028       __unwindfunclet$??0FileLoad_BncsSystem@alm_db_output@@QAE@PAV1@@Z$2 10021028 f   alm_db_output.obj
 0001:00020032       __ehhandler$??0FileLoad_BncsSystem@alm_db_output@@QAE@PAV1@@Z 10021032 f   alm_db_output.obj
 0001:0002004d       __unwindfunclet$??0alm_db_output@@QAE@ABVQString@@00@Z$0 1002104d f   alm_db_output.obj
 0001:00020055       __unwindfunclet$??0alm_db_output@@QAE@ABVQString@@00@Z$1 10021055 f   alm_db_output.obj
 0001:00020064       __unwindfunclet$??0alm_db_output@@QAE@ABVQString@@00@Z$2 10021064 f   alm_db_output.obj
 0001:00020073       __unwindfunclet$??0alm_db_output@@QAE@ABVQString@@00@Z$3 10021073 f   alm_db_output.obj
 0001:00020082       __unwindfunclet$??0alm_db_output@@QAE@ABVQString@@00@Z$4 10021082 f   alm_db_output.obj
 0001:00020091       __unwindfunclet$??0alm_db_output@@QAE@ABVQString@@00@Z$5 10021091 f   alm_db_output.obj
 0001:000200a0       __unwindfunclet$??0alm_db_output@@QAE@ABVQString@@00@Z$6 100210a0 f   alm_db_output.obj
 0001:000200af       __unwindfunclet$??0alm_db_output@@QAE@ABVQString@@00@Z$7 100210af f   alm_db_output.obj
 0001:000200bd       __unwindfunclet$??0alm_db_output@@QAE@ABVQString@@00@Z$8 100210bd f   alm_db_output.obj
 0001:000200cb       __unwindfunclet$??0alm_db_output@@QAE@ABVQString@@00@Z$9 100210cb f   alm_db_output.obj
 0001:000200d9       __unwindfunclet$??0alm_db_output@@QAE@ABVQString@@00@Z$10 100210d9 f   alm_db_output.obj
 0001:000200e7       __unwindfunclet$??0alm_db_output@@QAE@ABVQString@@00@Z$11 100210e7 f   alm_db_output.obj
 0001:000200f5       __unwindfunclet$??0alm_db_output@@QAE@ABVQString@@00@Z$12 100210f5 f   alm_db_output.obj
 0001:00020103       __unwindfunclet$??0alm_db_output@@QAE@ABVQString@@00@Z$13 10021103 f   alm_db_output.obj
 0001:0002010d       __unwindfunclet$??0alm_db_output@@QAE@ABVQString@@00@Z$14 1002110d f   alm_db_output.obj
 0001:00020117       __unwindfunclet$??0alm_db_output@@QAE@ABVQString@@00@Z$15 10021117 f   alm_db_output.obj
 0001:00020121       __unwindfunclet$??0alm_db_output@@QAE@ABVQString@@00@Z$16 10021121 f   alm_db_output.obj
 0001:0002012b       __unwindfunclet$??0alm_db_output@@QAE@ABVQString@@00@Z$17 1002112b f   alm_db_output.obj
 0001:00020134       __unwindfunclet$??0alm_db_output@@QAE@ABVQString@@00@Z$18 10021134 f   alm_db_output.obj
 0001:0002013e       __unwindfunclet$??0alm_db_output@@QAE@ABVQString@@00@Z$19 1002113e f   alm_db_output.obj
 0001:00020148       __unwindfunclet$??0alm_db_output@@QAE@ABVQString@@00@Z$20 10021148 f   alm_db_output.obj
 0001:00020151       __unwindfunclet$??0alm_db_output@@QAE@ABVQString@@00@Z$21 10021151 f   alm_db_output.obj
 0001:0002015b       __unwindfunclet$??0alm_db_output@@QAE@ABVQString@@00@Z$22 1002115b f   alm_db_output.obj
 0001:00020165       __unwindfunclet$??0alm_db_output@@QAE@ABVQString@@00@Z$23 10021165 f   alm_db_output.obj
 0001:0002016f       __unwindfunclet$??0alm_db_output@@QAE@ABVQString@@00@Z$24 1002116f f   alm_db_output.obj
 0001:00020178       __unwindfunclet$??0alm_db_output@@QAE@ABVQString@@00@Z$25 10021178 f   alm_db_output.obj
 0001:00020181       __unwindfunclet$??0alm_db_output@@QAE@ABVQString@@00@Z$26 10021181 f   alm_db_output.obj
 0001:0002018a       __unwindfunclet$??0alm_db_output@@QAE@ABVQString@@00@Z$27 1002118a f   alm_db_output.obj
 0001:00020193       __unwindfunclet$??0alm_db_output@@QAE@ABVQString@@00@Z$28 10021193 f   alm_db_output.obj
 0001:0002019d       __unwindfunclet$??0alm_db_output@@QAE@ABVQString@@00@Z$29 1002119d f   alm_db_output.obj
 0001:000201a7       __unwindfunclet$??0alm_db_output@@QAE@ABVQString@@00@Z$30 100211a7 f   alm_db_output.obj
 0001:000201b0       __unwindfunclet$??0alm_db_output@@QAE@ABVQString@@00@Z$31 100211b0 f   alm_db_output.obj
 0001:000201ba       __unwindfunclet$??0alm_db_output@@QAE@ABVQString@@00@Z$32 100211ba f   alm_db_output.obj
 0001:000201d4       __unwindfunclet$??0alm_db_output@@QAE@ABVQString@@00@Z$33 100211d4 f   alm_db_output.obj
 0001:000201ee       __unwindfunclet$??0alm_db_output@@QAE@ABVQString@@00@Z$34 100211ee f   alm_db_output.obj
 0001:00020208       __unwindfunclet$??0alm_db_output@@QAE@ABVQString@@00@Z$35 10021208 f   alm_db_output.obj
 0001:00020222       __unwindfunclet$??0alm_db_output@@QAE@ABVQString@@00@Z$37 10021222 f   alm_db_output.obj
 0001:0002022c       __unwindfunclet$??0alm_db_output@@QAE@ABVQString@@00@Z$38 1002122c f   alm_db_output.obj
 0001:00020246       __unwindfunclet$??0alm_db_output@@QAE@ABVQString@@00@Z$39 10021246 f   alm_db_output.obj
 0001:00020260       __unwindfunclet$??0alm_db_output@@QAE@ABVQString@@00@Z$40 10021260 f   alm_db_output.obj
 0001:0002027a       __unwindfunclet$??0alm_db_output@@QAE@ABVQString@@00@Z$41 1002127a f   alm_db_output.obj
 0001:00020299       __unwindfunclet$??0alm_db_output@@QAE@ABVQString@@00@Z$43 10021299 f   alm_db_output.obj
 0001:000202a3       __unwindfunclet$??0alm_db_output@@QAE@ABVQString@@00@Z$44 100212a3 f   alm_db_output.obj
 0001:000202c2       __unwindfunclet$??0alm_db_output@@QAE@ABVQString@@00@Z$45 100212c2 f   alm_db_output.obj
 0001:000202e1       __unwindfunclet$??0alm_db_output@@QAE@ABVQString@@00@Z$46 100212e1 f   alm_db_output.obj
 0001:00020300       __unwindfunclet$??0alm_db_output@@QAE@ABVQString@@00@Z$47 10021300 f   alm_db_output.obj
 0001:0002031f       __unwindfunclet$??0alm_db_output@@QAE@ABVQString@@00@Z$49 1002131f f   alm_db_output.obj
 0001:00020329       __unwindfunclet$??0alm_db_output@@QAE@ABVQString@@00@Z$50 10021329 f   alm_db_output.obj
 0001:00020348       __unwindfunclet$??0alm_db_output@@QAE@ABVQString@@00@Z$51 10021348 f   alm_db_output.obj
 0001:00020367       __unwindfunclet$??0alm_db_output@@QAE@ABVQString@@00@Z$52 10021367 f   alm_db_output.obj
 0001:00020386       __unwindfunclet$??0alm_db_output@@QAE@ABVQString@@00@Z$53 10021386 f   alm_db_output.obj
 0001:000203a5       __ehhandler$??0alm_db_output@@QAE@ABVQString@@00@Z 100213a5 f   alm_db_output.obj
 0001:000203c0       __unwindfunclet$??0config_plugin_base@@QAE@ABVQString@@00@Z$0 100213c0 f   alm_db_output.obj
 0001:000203c9       __unwindfunclet$??0config_plugin_base@@QAE@ABVQString@@00@Z$1 100213c9 f   alm_db_output.obj
 0001:000203d5       __unwindfunclet$??0config_plugin_base@@QAE@ABVQString@@00@Z$2 100213d5 f   alm_db_output.obj
 0001:000203e1       __unwindfunclet$??0config_plugin_base@@QAE@ABVQString@@00@Z$3 100213e1 f   alm_db_output.obj
 0001:000203ed       __ehhandler$??0config_plugin_base@@QAE@ABVQString@@00@Z 100213ed f   alm_db_output.obj
 0001:00020408       __unwindfunclet$??1?$QDict@VQAction@@@@UAE@XZ$0 10021408 f   alm_db_output.obj
 0001:00020411       __ehhandler$??1?$QDict@VQAction@@@@UAE@XZ 10021411 f   alm_db_output.obj
 0001:0002042c       __unwindfunclet$??1?$QPtrList@VcProcess@@@@UAE@XZ$0 1002142c f   alm_db_output.obj
 0001:0002042c       __unwindfunclet$??1?$QPtrList@VQPopupMenu@@@@UAE@XZ$0 1002142c f   alm_db_output.obj
 0001:0002042c       __unwindfunclet$??1?$QPtrList@VcOutputFile@@@@UAE@XZ$0 1002142c f   alm_db_output.obj
 0001:00020435       __ehhandler$??1?$QPtrList@VcProcess@@@@UAE@XZ 10021435 f   alm_db_output.obj
 0001:00020435       __ehhandler$??1?$QPtrList@VcOutputFile@@@@UAE@XZ 10021435 f   alm_db_output.obj
 0001:00020435       __ehhandler$??1?$QPtrList@VQPopupMenu@@@@UAE@XZ 10021435 f   alm_db_output.obj
 0001:00020450       __unwindfunclet$??1FileLoad_BncsSystem@alm_db_output@@UAE@XZ$0 10021450 f   alm_db_output.obj
 0001:00020458       __ehhandler$??1FileLoad_BncsSystem@alm_db_output@@UAE@XZ 10021458 f   alm_db_output.obj
 0001:00020473       __unwindfunclet$??1QDockWindowList@@UAE@XZ$0 10021473 f   alm_db_output.obj
 0001:0002047c       __unwindfunclet$??1QDockWindowList@@UAE@XZ$1 1002147c f   alm_db_output.obj
 0001:00020485       __ehhandler$??1QDockWindowList@@UAE@XZ 10021485 f   alm_db_output.obj
 0001:000204a0       __unwindfunclet$??1QPopupMenuList@@UAE@XZ$0 100214a0 f   alm_db_output.obj
 0001:000204a8       __ehhandler$??1QPopupMenuList@@UAE@XZ 100214a8 f   alm_db_output.obj
 0001:000204c3       __unwindfunclet$??1alm_db_output@@UAE@XZ$0 100214c3 f   alm_db_output.obj
 0001:000204cb       __unwindfunclet$??1alm_db_output@@UAE@XZ$1 100214cb f   alm_db_output.obj
 0001:000204da       __unwindfunclet$??1alm_db_output@@UAE@XZ$2 100214da f   alm_db_output.obj
 0001:000204e9       __unwindfunclet$??1alm_db_output@@UAE@XZ$3 100214e9 f   alm_db_output.obj
 0001:000204f8       __unwindfunclet$??1alm_db_output@@UAE@XZ$4 100214f8 f   alm_db_output.obj
 0001:00020507       __unwindfunclet$??1alm_db_output@@UAE@XZ$5 10021507 f   alm_db_output.obj
 0001:00020516       __unwindfunclet$??1alm_db_output@@UAE@XZ$6 10021516 f   alm_db_output.obj
 0001:00020525       __unwindfunclet$??1alm_db_output@@UAE@XZ$7 10021525 f   alm_db_output.obj
 0001:00020533       __unwindfunclet$??1alm_db_output@@UAE@XZ$8 10021533 f   alm_db_output.obj
 0001:00020541       __unwindfunclet$??1alm_db_output@@UAE@XZ$9 10021541 f   alm_db_output.obj
 0001:0002054f       __unwindfunclet$??1alm_db_output@@UAE@XZ$10 1002154f f   alm_db_output.obj
 0001:0002055d       __unwindfunclet$??1alm_db_output@@UAE@XZ$11 1002155d f   alm_db_output.obj
 0001:0002056b       __unwindfunclet$??1alm_db_output@@UAE@XZ$12 1002156b f   alm_db_output.obj
 0001:00020579       __unwindfunclet$??1alm_db_output@@UAE@XZ$13 10021579 f   alm_db_output.obj
 0001:00020582       __unwindfunclet$??1alm_db_output@@UAE@XZ$14 10021582 f   alm_db_output.obj
 0001:0002058b       __ehhandler$??1alm_db_output@@UAE@XZ 1002158b f   alm_db_output.obj
 0001:000205a6       __unwindfunclet$??1config_plugin_base@@UAE@XZ$0 100215a6 f   alm_db_output.obj
 0001:000205af       __unwindfunclet$??1config_plugin_base@@UAE@XZ$1 100215af f   alm_db_output.obj
 0001:000205bb       __unwindfunclet$??1config_plugin_base@@UAE@XZ$2 100215bb f   alm_db_output.obj
 0001:000205c7       __ehhandler$??1config_plugin_base@@UAE@XZ 100215c7 f   alm_db_output.obj
 0001:000205e2       __unwindfunclet$?AllocateCfgFileName@alm_db_output@@AAEXAAVQString@@0AAH@Z$0 100215e2 f   alm_db_output.obj
 0001:000205eb       __unwindfunclet$?AllocateCfgFileName@alm_db_output@@AAEXAAVQString@@0AAH@Z$1 100215eb f   alm_db_output.obj
 0001:000205f4       __unwindfunclet$?AllocateCfgFileName@alm_db_output@@AAEXAAVQString@@0AAH@Z$2 100215f4 f   alm_db_output.obj
 0001:000205fd       __unwindfunclet$?AllocateCfgFileName@alm_db_output@@AAEXAAVQString@@0AAH@Z$3 100215fd f   alm_db_output.obj
 0001:00020606       __unwindfunclet$?AllocateCfgFileName@alm_db_output@@AAEXAAVQString@@0AAH@Z$4 10021606 f   alm_db_output.obj
 0001:0002060f       __unwindfunclet$?AllocateCfgFileName@alm_db_output@@AAEXAAVQString@@0AAH@Z$5 1002160f f   alm_db_output.obj
 0001:00020618       __unwindfunclet$?AllocateCfgFileName@alm_db_output@@AAEXAAVQString@@0AAH@Z$6 10021618 f   alm_db_output.obj
 0001:00020621       __unwindfunclet$?AllocateCfgFileName@alm_db_output@@AAEXAAVQString@@0AAH@Z$7 10021621 f   alm_db_output.obj
 0001:0002062a       __unwindfunclet$?AllocateCfgFileName@alm_db_output@@AAEXAAVQString@@0AAH@Z$8 1002162a f   alm_db_output.obj
 0001:00020633       __ehhandler$?AllocateCfgFileName@alm_db_output@@AAEXAAVQString@@0AAH@Z 10021633 f   alm_db_output.obj
 0001:0002064e       __unwindfunclet$?markDirty@alm_db_output@@AAEXXZ$0 1002164e f   alm_db_output.obj
 0001:0002064e       __unwindfunclet$?apply@alm_db_output@@EAEXXZ$0 1002164e f   alm_db_output.obj
 0001:0002064e       __unwindfunclet$?EditProcess@alm_db_output@@AAEXXZ$0 1002164e f   alm_db_output.obj
 0001:00020657       __ehhandler$?EditProcess@alm_db_output@@AAEXXZ 10021657 f   alm_db_output.obj
 0001:00020657       __ehhandler$?markDirty@alm_db_output@@AAEXXZ 10021657 f   alm_db_output.obj
 0001:00020657       __ehhandler$?apply@alm_db_output@@EAEXXZ 10021657 f   alm_db_output.obj
 0001:00020672       __ehhandler$?_Copy@?$basic_string@DU?$char_traits@D@std@@V?$allocator@D@2@@std@@QAEXII@Z 10021672 f   alm_db_output.obj
 0001:0002068d       __unwindfunclet$?about@alm_db_output@@UAE?AVQString@@XZ$0 1002168d f   alm_db_output.obj
 0001:000206a7       __ehhandler$?about@alm_db_output@@UAE?AVQString@@XZ 100216a7 f   alm_db_output.obj
 0001:000206c2       __unwindfunclet$?about@config_plugin_base@@UAE?AVQString@@XZ$0 100216c2 f   alm_db_output.obj
 0001:000206cb       __unwindfunclet$?about@config_plugin_base@@UAE?AVQString@@XZ$1 100216cb f   alm_db_output.obj
 0001:000206e5       __ehhandler$?about@config_plugin_base@@UAE?AVQString@@XZ 100216e5 f   alm_db_output.obj
 0001:00020700       __unwindfunclet$?activate@alm_db_output@@UAEX_N@Z$0 10021700 f   alm_db_output.obj
 0001:00020709       __unwindfunclet$?activate@alm_db_output@@UAEX_N@Z$3 10021709 f   alm_db_output.obj
 0001:00020712       __unwindfunclet$?activate@alm_db_output@@UAEX_N@Z$4 10021712 f   alm_db_output.obj
 0001:0002071c       __ehhandler$?activate@alm_db_output@@UAEX_N@Z 1002171c f   alm_db_output.obj
 0001:00020737       __unwindfunclet$?addProcSetting@alm_db_output@@AAEXPAVcProcess@@ABVQString@@@Z$0 10021737 f   alm_db_output.obj
 0001:00020740       __unwindfunclet$?addProcSetting@alm_db_output@@AAEXPAVcProcess@@ABVQString@@@Z$1 10021740 f   alm_db_output.obj
 0001:00020749       __ehhandler$?addProcSetting@alm_db_output@@AAEXPAVcProcess@@ABVQString@@@Z 10021749 f   alm_db_output.obj
 0001:00020764       __unwindfunclet$?allocateSystemName@alm_db_output@@AAEXAAVQString@@@Z$0 10021764 f   alm_db_output.obj
 0001:0002076d       __unwindfunclet$?allocateSystemName@alm_db_output@@AAEXAAVQString@@@Z$1 1002176d f   alm_db_output.obj
 0001:00020776       __unwindfunclet$?allocateSystemName@alm_db_output@@AAEXAAVQString@@@Z$2 10021776 f   alm_db_output.obj
 0001:0002077f       __ehhandler$?allocateSystemName@alm_db_output@@AAEXAAVQString@@@Z 1002177f f   alm_db_output.obj
 0001:0002079a       __unwindfunclet$?closeEvent@alm_db_output@@UAEXPAVQCloseEvent@@@Z$0 1002179a f   alm_db_output.obj
 0001:000207a3       __ehhandler$?closeEvent@alm_db_output@@UAEXPAVQCloseEvent@@@Z 100217a3 f   alm_db_output.obj
 0001:000207be       __unwindfunclet$?copy@?$QMapPrivate@VQString@@PAVcProcess@@@@QAEPAU?$QMapNode@VQString@@PAVcProcess@@@@PAU2@@Z$0 100217be f   alm_db_output.obj
 0001:000207be       __unwindfunclet$??0?$QMapPrivate@VQString@@PAVcProcess@@@@QAE@PBV0@@Z$0 100217be f   alm_db_output.obj
 0001:000207c8       __ehhandler$?copy@?$QMapPrivate@VQString@@PAVcProcess@@@@QAEPAU?$QMapNode@VQString@@PAVcProcess@@@@PAU2@@Z 100217c8 f   alm_db_output.obj
 0001:000207c8       __ehhandler$??0?$QMapPrivate@VQString@@PAVcProcess@@@@QAE@PBV0@@Z 100217c8 f   alm_db_output.obj
 0001:000207e3       __unwindfunclet$?copyToClipBoard@alm_db_output@@AAEXXZ$0 100217e3 f   alm_db_output.obj
 0001:000207ec       __unwindfunclet$?copyToClipBoard@alm_db_output@@AAEXXZ$1 100217ec f   alm_db_output.obj
 0001:000207f5       __unwindfunclet$?copyToClipBoard@alm_db_output@@AAEXXZ$2 100217f5 f   alm_db_output.obj
 0001:000207fe       __unwindfunclet$?copyToClipBoard@alm_db_output@@AAEXXZ$3 100217fe f   alm_db_output.obj
 0001:00020807       __unwindfunclet$?copyToClipBoard@alm_db_output@@AAEXXZ$4 10021807 f   alm_db_output.obj
 0001:00020810       __unwindfunclet$?copyToClipBoard@alm_db_output@@AAEXXZ$5 10021810 f   alm_db_output.obj
 0001:00020819       __unwindfunclet$?copyToClipBoard@alm_db_output@@AAEXXZ$6 10021819 f   alm_db_output.obj
 0001:00020822       __unwindfunclet$?copyToClipBoard@alm_db_output@@AAEXXZ$7 10021822 f   alm_db_output.obj
 0001:0002082b       __unwindfunclet$?copyToClipBoard@alm_db_output@@AAEXXZ$8 1002182b f   alm_db_output.obj
 0001:00020834       __unwindfunclet$?copyToClipBoard@alm_db_output@@AAEXXZ$9 10021834 f   alm_db_output.obj
 0001:0002083d       __unwindfunclet$?copyToClipBoard@alm_db_output@@AAEXXZ$10 1002183d f   alm_db_output.obj
 0001:00020846       __unwindfunclet$?copyToClipBoard@alm_db_output@@AAEXXZ$11 10021846 f   alm_db_output.obj
 0001:0002084f       __unwindfunclet$?copyToClipBoard@alm_db_output@@AAEXXZ$12 1002184f f   alm_db_output.obj
 0001:00020858       __ehhandler$?copyToClipBoard@alm_db_output@@AAEXXZ 10021858 f   alm_db_output.obj
 0001:00020873       __unwindfunclet$?decodeSystem@alm_db_output@@AAEXABVQString@@@Z$0 10021873 f   alm_db_output.obj
 0001:0002087c       __unwindfunclet$?decodeSystem@alm_db_output@@AAEXABVQString@@@Z$1 1002187c f   alm_db_output.obj
 0001:00020885       __unwindfunclet$?decodeSystem@alm_db_output@@AAEXABVQString@@@Z$2 10021885 f   alm_db_output.obj
 0001:0002088e       __unwindfunclet$?decodeSystem@alm_db_output@@AAEXABVQString@@@Z$3 1002188e f   alm_db_output.obj
 0001:00020897       __unwindfunclet$?decodeSystem@alm_db_output@@AAEXABVQString@@@Z$4 10021897 f   alm_db_output.obj
 0001:000208a0       __unwindfunclet$?decodeSystem@alm_db_output@@AAEXABVQString@@@Z$5 100218a0 f   alm_db_output.obj
 0001:000208a9       __unwindfunclet$?decodeSystem@alm_db_output@@AAEXABVQString@@@Z$6 100218a9 f   alm_db_output.obj
 0001:000208b2       __ehhandler$?decodeSystem@alm_db_output@@AAEXABVQString@@@Z 100218b2 f   alm_db_output.obj
 0001:000208cd       __unwindfunclet$?doDone@alm_db_output@@AAEXPAVresponse@@@Z$0 100218cd f   alm_db_output.obj
 0001:000208d6       __unwindfunclet$?doDone@alm_db_output@@AAEXPAVresponse@@@Z$1 100218d6 f   alm_db_output.obj
 0001:000208df       __unwindfunclet$?doDone@alm_db_output@@AAEXPAVresponse@@@Z$2 100218df f   alm_db_output.obj
 0001:000208e8       __unwindfunclet$?doDone@alm_db_output@@AAEXPAVresponse@@@Z$3 100218e8 f   alm_db_output.obj
 0001:000208f1       __unwindfunclet$?doDone@alm_db_output@@AAEXPAVresponse@@@Z$4 100218f1 f   alm_db_output.obj
 0001:000208fa       __unwindfunclet$?doDone@alm_db_output@@AAEXPAVresponse@@@Z$5 100218fa f   alm_db_output.obj
 0001:00020903       __unwindfunclet$?doDone@alm_db_output@@AAEXPAVresponse@@@Z$6 10021903 f   alm_db_output.obj
 0001:0002090c       __unwindfunclet$?doDone@alm_db_output@@AAEXPAVresponse@@@Z$7 1002190c f   alm_db_output.obj
 0001:00020915       __unwindfunclet$?doDone@alm_db_output@@AAEXPAVresponse@@@Z$8 10021915 f   alm_db_output.obj
 0001:0002091e       __unwindfunclet$?doDone@alm_db_output@@AAEXPAVresponse@@@Z$9 1002191e f   alm_db_output.obj
 0001:00020927       __unwindfunclet$?doDone@alm_db_output@@AAEXPAVresponse@@@Z$10 10021927 f   alm_db_output.obj
 0001:00020930       __unwindfunclet$?doDone@alm_db_output@@AAEXPAVresponse@@@Z$11 10021930 f   alm_db_output.obj
 0001:00020939       __unwindfunclet$?doDone@alm_db_output@@AAEXPAVresponse@@@Z$12 10021939 f   alm_db_output.obj
 0001:00020942       __unwindfunclet$?doDone@alm_db_output@@AAEXPAVresponse@@@Z$13 10021942 f   alm_db_output.obj
 0001:0002094b       __unwindfunclet$?doDone@alm_db_output@@AAEXPAVresponse@@@Z$14 1002194b f   alm_db_output.obj
 0001:00020954       __unwindfunclet$?doDone@alm_db_output@@AAEXPAVresponse@@@Z$15 10021954 f   alm_db_output.obj
 0001:0002095d       __unwindfunclet$?doDone@alm_db_output@@AAEXPAVresponse@@@Z$16 1002195d f   alm_db_output.obj
 0001:00020966       __unwindfunclet$?doDone@alm_db_output@@AAEXPAVresponse@@@Z$17 10021966 f   alm_db_output.obj
 0001:0002096f       __unwindfunclet$?doDone@alm_db_output@@AAEXPAVresponse@@@Z$18 1002196f f   alm_db_output.obj
 0001:00020978       __unwindfunclet$?doDone@alm_db_output@@AAEXPAVresponse@@@Z$19 10021978 f   alm_db_output.obj
 0001:00020981       __unwindfunclet$?doDone@alm_db_output@@AAEXPAVresponse@@@Z$20 10021981 f   alm_db_output.obj
 0001:0002098a       __unwindfunclet$?doDone@alm_db_output@@AAEXPAVresponse@@@Z$21 1002198a f   alm_db_output.obj
 0001:00020993       __unwindfunclet$?doDone@alm_db_output@@AAEXPAVresponse@@@Z$22 10021993 f   alm_db_output.obj
 0001:0002099c       __unwindfunclet$?doDone@alm_db_output@@AAEXPAVresponse@@@Z$23 1002199c f   alm_db_output.obj
 0001:000209a5       __ehhandler$?doDone@alm_db_output@@AAEXPAVresponse@@@Z 100219a5 f   alm_db_output.obj
 0001:000209c0       __unwindfunclet$?doDownload@alm_db_output@@AAEXPAVresponse@@@Z$0 100219c0 f   alm_db_output.obj
 0001:000209c9       __unwindfunclet$?doDownload@alm_db_output@@AAEXPAVresponse@@@Z$1 100219c9 f   alm_db_output.obj
 0001:000209d2       __ehhandler$?doDownload@alm_db_output@@AAEXPAVresponse@@@Z 100219d2 f   alm_db_output.obj
 0001:000209ed       __unwindfunclet$?doDownloadRead@alm_db_output@@AAEXPAVresponse@@@Z$0 100219ed f   alm_db_output.obj
 0001:000209f9       __unwindfunclet$?doDownloadRead@alm_db_output@@AAEXPAVresponse@@@Z$1 100219f9 f   alm_db_output.obj
 0001:00020a05       __unwindfunclet$?doDownloadRead@alm_db_output@@AAEXPAVresponse@@@Z$2 10021a05 f   alm_db_output.obj
 0001:00020a11       __unwindfunclet$?doDownloadRead@alm_db_output@@AAEXPAVresponse@@@Z$3 10021a11 f   alm_db_output.obj
 0001:00020a1d       __unwindfunclet$?doDownloadRead@alm_db_output@@AAEXPAVresponse@@@Z$4 10021a1d f   alm_db_output.obj
 0001:00020a29       __unwindfunclet$?doDownloadRead@alm_db_output@@AAEXPAVresponse@@@Z$5 10021a29 f   alm_db_output.obj
 0001:00020a35       __unwindfunclet$?doDownloadRead@alm_db_output@@AAEXPAVresponse@@@Z$6 10021a35 f   alm_db_output.obj
 0001:00020a41       __unwindfunclet$?doDownloadRead@alm_db_output@@AAEXPAVresponse@@@Z$7 10021a41 f   alm_db_output.obj
 0001:00020a4d       __unwindfunclet$?doDownloadRead@alm_db_output@@AAEXPAVresponse@@@Z$8 10021a4d f   alm_db_output.obj
 0001:00020a59       __unwindfunclet$?doDownloadRead@alm_db_output@@AAEXPAVresponse@@@Z$9 10021a59 f   alm_db_output.obj
 0001:00020a65       __unwindfunclet$?doDownloadRead@alm_db_output@@AAEXPAVresponse@@@Z$10 10021a65 f   alm_db_output.obj
 0001:00020a88       __unwindfunclet$?doDownloadRead@alm_db_output@@AAEXPAVresponse@@@Z$11 10021a88 f   alm_db_output.obj
 0001:00020aab       __unwindfunclet$?doDownloadRead@alm_db_output@@AAEXPAVresponse@@@Z$12 10021aab f   alm_db_output.obj
 0001:00020ab7       __unwindfunclet$?doDownloadRead@alm_db_output@@AAEXPAVresponse@@@Z$13 10021ab7 f   alm_db_output.obj
 0001:00020ac3       __unwindfunclet$?doDownloadRead@alm_db_output@@AAEXPAVresponse@@@Z$14 10021ac3 f   alm_db_output.obj
 0001:00020acf       __unwindfunclet$?doDownloadRead@alm_db_output@@AAEXPAVresponse@@@Z$15 10021acf f   alm_db_output.obj
 0001:00020adc       __unwindfunclet$?doDownloadRead@alm_db_output@@AAEXPAVresponse@@@Z$16 10021adc f   alm_db_output.obj
 0001:00020ae8       __unwindfunclet$?doDownloadRead@alm_db_output@@AAEXPAVresponse@@@Z$17 10021ae8 f   alm_db_output.obj
 0001:00020af5       __unwindfunclet$?doDownloadRead@alm_db_output@@AAEXPAVresponse@@@Z$18 10021af5 f   alm_db_output.obj
 0001:00020b01       __unwindfunclet$?doDownloadRead@alm_db_output@@AAEXPAVresponse@@@Z$19 10021b01 f   alm_db_output.obj
 0001:00020b0d       __unwindfunclet$?doDownloadRead@alm_db_output@@AAEXPAVresponse@@@Z$20 10021b0d f   alm_db_output.obj
 0001:00020b19       __unwindfunclet$?doDownloadRead@alm_db_output@@AAEXPAVresponse@@@Z$21 10021b19 f   alm_db_output.obj
 0001:00020b25       __unwindfunclet$?doDownloadRead@alm_db_output@@AAEXPAVresponse@@@Z$22 10021b25 f   alm_db_output.obj
 0001:00020b31       __unwindfunclet$?doDownloadRead@alm_db_output@@AAEXPAVresponse@@@Z$23 10021b31 f   alm_db_output.obj
 0001:00020b3d       __unwindfunclet$?doDownloadRead@alm_db_output@@AAEXPAVresponse@@@Z$24 10021b3d f   alm_db_output.obj
 0001:00020b49       __unwindfunclet$?doDownloadRead@alm_db_output@@AAEXPAVresponse@@@Z$26 10021b49 f   alm_db_output.obj
 0001:00020b55       __unwindfunclet$?doDownloadRead@alm_db_output@@AAEXPAVresponse@@@Z$27 10021b55 f   alm_db_output.obj
 0001:00020b61       __unwindfunclet$?doDownloadRead@alm_db_output@@AAEXPAVresponse@@@Z$28 10021b61 f   alm_db_output.obj
 0001:00020b6d       __unwindfunclet$?doDownloadRead@alm_db_output@@AAEXPAVresponse@@@Z$29 10021b6d f   alm_db_output.obj
 0001:00020b79       __unwindfunclet$?doDownloadRead@alm_db_output@@AAEXPAVresponse@@@Z$30 10021b79 f   alm_db_output.obj
 0001:00020b85       __unwindfunclet$?doDownloadRead@alm_db_output@@AAEXPAVresponse@@@Z$31 10021b85 f   alm_db_output.obj
 0001:00020b91       __unwindfunclet$?doDownloadRead@alm_db_output@@AAEXPAVresponse@@@Z$32 10021b91 f   alm_db_output.obj
 0001:00020b9d       __unwindfunclet$?doDownloadRead@alm_db_output@@AAEXPAVresponse@@@Z$33 10021b9d f   alm_db_output.obj
 0001:00020ba9       __ehhandler$?doDownloadRead@alm_db_output@@AAEXPAVresponse@@@Z 10021ba9 f   alm_db_output.obj
 0001:00020bd1       __unwindfunclet$?doLock@alm_db_output@@AAEXPAVresponse@@@Z$0 10021bd1 f   alm_db_output.obj
 0001:00020bda       __unwindfunclet$?doLock@alm_db_output@@AAEXPAVresponse@@@Z$1 10021bda f   alm_db_output.obj
 0001:00020be3       __unwindfunclet$?doLock@alm_db_output@@AAEXPAVresponse@@@Z$2 10021be3 f   alm_db_output.obj
 0001:00020bec       __unwindfunclet$?doLock@alm_db_output@@AAEXPAVresponse@@@Z$3 10021bec f   alm_db_output.obj
 0001:00020bf5       __unwindfunclet$?doLock@alm_db_output@@AAEXPAVresponse@@@Z$4 10021bf5 f   alm_db_output.obj
 0001:00020bfe       __unwindfunclet$?doLock@alm_db_output@@AAEXPAVresponse@@@Z$5 10021bfe f   alm_db_output.obj
 0001:00020c07       __unwindfunclet$?doLock@alm_db_output@@AAEXPAVresponse@@@Z$6 10021c07 f   alm_db_output.obj
 0001:00020c10       __unwindfunclet$?doLock@alm_db_output@@AAEXPAVresponse@@@Z$7 10021c10 f   alm_db_output.obj
 0001:00020c19       __unwindfunclet$?doLock@alm_db_output@@AAEXPAVresponse@@@Z$8 10021c19 f   alm_db_output.obj
 0001:00020c22       __unwindfunclet$?doLock@alm_db_output@@AAEXPAVresponse@@@Z$9 10021c22 f   alm_db_output.obj
 0001:00020c2b       __unwindfunclet$?doLock@alm_db_output@@AAEXPAVresponse@@@Z$10 10021c2b f   alm_db_output.obj
 0001:00020c34       __unwindfunclet$?doLock@alm_db_output@@AAEXPAVresponse@@@Z$11 10021c34 f   alm_db_output.obj
 0001:00020c3d       __unwindfunclet$?doLock@alm_db_output@@AAEXPAVresponse@@@Z$12 10021c3d f   alm_db_output.obj
 0001:00020c46       __unwindfunclet$?doLock@alm_db_output@@AAEXPAVresponse@@@Z$13 10021c46 f   alm_db_output.obj
 0001:00020c4f       __unwindfunclet$?doLock@alm_db_output@@AAEXPAVresponse@@@Z$14 10021c4f f   alm_db_output.obj
 0001:00020c58       __unwindfunclet$?doLock@alm_db_output@@AAEXPAVresponse@@@Z$15 10021c58 f   alm_db_output.obj
 0001:00020c61       __unwindfunclet$?doLock@alm_db_output@@AAEXPAVresponse@@@Z$16 10021c61 f   alm_db_output.obj
 0001:00020c6a       __unwindfunclet$?doLock@alm_db_output@@AAEXPAVresponse@@@Z$17 10021c6a f   alm_db_output.obj
 0001:00020c73       __unwindfunclet$?doLock@alm_db_output@@AAEXPAVresponse@@@Z$18 10021c73 f   alm_db_output.obj
 0001:00020c7c       __unwindfunclet$?doLock@alm_db_output@@AAEXPAVresponse@@@Z$19 10021c7c f   alm_db_output.obj
 0001:00020c85       __unwindfunclet$?doLock@alm_db_output@@AAEXPAVresponse@@@Z$20 10021c85 f   alm_db_output.obj
 0001:00020c8e       __ehhandler$?doLock@alm_db_output@@AAEXPAVresponse@@@Z 10021c8e f   alm_db_output.obj
 0001:00020ca9       __unwindfunclet$?doUpload@alm_db_output@@AAEXPAVresponse@@@Z$0 10021ca9 f   alm_db_output.obj
 0001:00020cb2       __ehhandler$?doUpload@alm_db_output@@AAEXPAVresponse@@@Z 10021cb2 f   alm_db_output.obj
 0001:00020ccd       __unwindfunclet$?editSelectedProcs@alm_db_output@@AAEXXZ$0 10021ccd f   alm_db_output.obj
 0001:00020cd7       __unwindfunclet$?editSelectedProcs@alm_db_output@@AAEXXZ$1 10021cd7 f   alm_db_output.obj
 0001:00020ce0       __unwindfunclet$?editSelectedProcs@alm_db_output@@AAEXXZ$2 10021ce0 f   alm_db_output.obj
 0001:00020ce9       __unwindfunclet$?editSelectedProcs@alm_db_output@@AAEXXZ$3 10021ce9 f   alm_db_output.obj
 0001:00020cf2       __unwindfunclet$?editSelectedProcs@alm_db_output@@AAEXXZ$4 10021cf2 f   alm_db_output.obj
 0001:00020cfb       __unwindfunclet$?editSelectedProcs@alm_db_output@@AAEXXZ$5 10021cfb f   alm_db_output.obj
 0001:00020d04       __unwindfunclet$?editSelectedProcs@alm_db_output@@AAEXXZ$6 10021d04 f   alm_db_output.obj
 0001:00020d0d       __unwindfunclet$?editSelectedProcs@alm_db_output@@AAEXXZ$7 10021d0d f   alm_db_output.obj
 0001:00020d16       __unwindfunclet$?editSelectedProcs@alm_db_output@@AAEXXZ$8 10021d16 f   alm_db_output.obj
 0001:00020d1f       __unwindfunclet$?editSelectedProcs@alm_db_output@@AAEXXZ$9 10021d1f f   alm_db_output.obj
 0001:00020d28       __unwindfunclet$?editSelectedProcs@alm_db_output@@AAEXXZ$10 10021d28 f   alm_db_output.obj
 0001:00020d31       __unwindfunclet$?editSelectedProcs@alm_db_output@@AAEXXZ$11 10021d31 f   alm_db_output.obj
 0001:00020d3a       __unwindfunclet$?editSelectedProcs@alm_db_output@@AAEXXZ$12 10021d3a f   alm_db_output.obj
 0001:00020d43       __unwindfunclet$?editSelectedProcs@alm_db_output@@AAEXXZ$13 10021d43 f   alm_db_output.obj
 0001:00020d4c       __unwindfunclet$?editSelectedProcs@alm_db_output@@AAEXXZ$14 10021d4c f   alm_db_output.obj
 0001:00020d55       __unwindfunclet$?editSelectedProcs@alm_db_output@@AAEXXZ$15 10021d55 f   alm_db_output.obj
 0001:00020d5e       __unwindfunclet$?editSelectedProcs@alm_db_output@@AAEXXZ$16 10021d5e f   alm_db_output.obj
 0001:00020d67       __unwindfunclet$?editSelectedProcs@alm_db_output@@AAEXXZ$17 10021d67 f   alm_db_output.obj
 0001:00020d70       __unwindfunclet$?editSelectedProcs@alm_db_output@@AAEXXZ$18 10021d70 f   alm_db_output.obj
 0001:00020d79       __unwindfunclet$?editSelectedProcs@alm_db_output@@AAEXXZ$19 10021d79 f   alm_db_output.obj
 0001:00020d82       __unwindfunclet$?editSelectedProcs@alm_db_output@@AAEXXZ$20 10021d82 f   alm_db_output.obj
 0001:00020d8b       __unwindfunclet$?editSelectedProcs@alm_db_output@@AAEXXZ$21 10021d8b f   alm_db_output.obj
 0001:00020d94       __unwindfunclet$?editSelectedProcs@alm_db_output@@AAEXXZ$22 10021d94 f   alm_db_output.obj
 0001:00020d9d       __unwindfunclet$?editSelectedProcs@alm_db_output@@AAEXXZ$23 10021d9d f   alm_db_output.obj
 0001:00020da6       __unwindfunclet$?editSelectedProcs@alm_db_output@@AAEXXZ$24 10021da6 f   alm_db_output.obj
 0001:00020daf       __unwindfunclet$?editSelectedProcs@alm_db_output@@AAEXXZ$25 10021daf f   alm_db_output.obj
 0001:00020db8       __unwindfunclet$?editSelectedProcs@alm_db_output@@AAEXXZ$26 10021db8 f   alm_db_output.obj
 0001:00020dc1       __unwindfunclet$?editSelectedProcs@alm_db_output@@AAEXXZ$27 10021dc1 f   alm_db_output.obj
 0001:00020dca       __unwindfunclet$?editSelectedProcs@alm_db_output@@AAEXXZ$28 10021dca f   alm_db_output.obj
 0001:00020dd3       __unwindfunclet$?editSelectedProcs@alm_db_output@@AAEXXZ$29 10021dd3 f   alm_db_output.obj
 0001:00020ddc       __unwindfunclet$?editSelectedProcs@alm_db_output@@AAEXXZ$30 10021ddc f   alm_db_output.obj
 0001:00020de5       __unwindfunclet$?editSelectedProcs@alm_db_output@@AAEXXZ$31 10021de5 f   alm_db_output.obj
 0001:00020dee       __unwindfunclet$?editSelectedProcs@alm_db_output@@AAEXXZ$32 10021dee f   alm_db_output.obj
 0001:00020dfa       __unwindfunclet$?editSelectedProcs@alm_db_output@@AAEXXZ$34 10021dfa f   alm_db_output.obj
 0001:00020e06       __unwindfunclet$?editSelectedProcs@alm_db_output@@AAEXXZ$35 10021e06 f   alm_db_output.obj
 0001:00020e12       __unwindfunclet$?editSelectedProcs@alm_db_output@@AAEXXZ$37 10021e12 f   alm_db_output.obj
 0001:00020e1b       __unwindfunclet$?editSelectedProcs@alm_db_output@@AAEXXZ$38 10021e1b f   alm_db_output.obj
 0001:00020e27       __unwindfunclet$?editSelectedProcs@alm_db_output@@AAEXXZ$40 10021e27 f   alm_db_output.obj
 0001:00020e33       __unwindfunclet$?editSelectedProcs@alm_db_output@@AAEXXZ$41 10021e33 f   alm_db_output.obj
 0001:00020e3c       __unwindfunclet$?editSelectedProcs@alm_db_output@@AAEXXZ$43 10021e3c f   alm_db_output.obj
 0001:00020e45       __unwindfunclet$?editSelectedProcs@alm_db_output@@AAEXXZ$44 10021e45 f   alm_db_output.obj
 0001:00020e51       __unwindfunclet$?editSelectedProcs@alm_db_output@@AAEXXZ$46 10021e51 f   alm_db_output.obj
 0001:00020e5d       __unwindfunclet$?editSelectedProcs@alm_db_output@@AAEXXZ$47 10021e5d f   alm_db_output.obj
 0001:00020e66       __unwindfunclet$?editSelectedProcs@alm_db_output@@AAEXXZ$49 10021e66 f   alm_db_output.obj
 0001:00020e72       __ehhandler$?editSelectedProcs@alm_db_output@@AAEXXZ 10021e72 f   alm_db_output.obj
 0001:00020e90       __unwindfunclet$?filterChange@alm_db_output@@AAEXXZ$0 10021e90 f   alm_db_output.obj
 0001:00020e99       __unwindfunclet$?filterChange@alm_db_output@@AAEXXZ$1 10021e99 f   alm_db_output.obj
 0001:00020ea2       __unwindfunclet$?filterChange@alm_db_output@@AAEXXZ$3 10021ea2 f   alm_db_output.obj
 0001:00020eab       __unwindfunclet$?filterChange@alm_db_output@@AAEXXZ$4 10021eab f   alm_db_output.obj
 0001:00020eb4       __unwindfunclet$?filterChange@alm_db_output@@AAEXXZ$5 10021eb4 f   alm_db_output.obj
 0001:00020ebd       __ehhandler$?filterChange@alm_db_output@@AAEXXZ 10021ebd f   alm_db_output.obj
 0001:00020ed8       __unwindfunclet$?loadFile@alm_db_output@@AAE_NABVQString@@@Z$0 10021ed8 f   alm_db_output.obj
 0001:00020ee1       __unwindfunclet$?loadFile@alm_db_output@@AAE_NABVQString@@@Z$1 10021ee1 f   alm_db_output.obj
 0001:00020eea       __unwindfunclet$?loadFile@alm_db_output@@AAE_NABVQString@@@Z$2 10021eea f   alm_db_output.obj
 0001:00020ef6       __unwindfunclet$?loadFile@alm_db_output@@AAE_NABVQString@@@Z$3 10021ef6 f   alm_db_output.obj
 0001:00020eff       __unwindfunclet$?loadFile@alm_db_output@@AAE_NABVQString@@@Z$4 10021eff f   alm_db_output.obj
 0001:00020f08       __unwindfunclet$?loadFile@alm_db_output@@AAE_NABVQString@@@Z$5 10021f08 f   alm_db_output.obj
 0001:00020f11       __unwindfunclet$?loadFile@alm_db_output@@AAE_NABVQString@@@Z$6 10021f11 f   alm_db_output.obj
 0001:00020f1a       __unwindfunclet$?loadFile@alm_db_output@@AAE_NABVQString@@@Z$7 10021f1a f   alm_db_output.obj
 0001:00020f23       __unwindfunclet$?loadFile@alm_db_output@@AAE_NABVQString@@@Z$8 10021f23 f   alm_db_output.obj
 0001:00020f2c       __unwindfunclet$?loadFile@alm_db_output@@AAE_NABVQString@@@Z$9 10021f2c f   alm_db_output.obj
 0001:00020f35       __unwindfunclet$?loadFile@alm_db_output@@AAE_NABVQString@@@Z$10 10021f35 f   alm_db_output.obj
 0001:00020f3e       __unwindfunclet$?loadFile@alm_db_output@@AAE_NABVQString@@@Z$11 10021f3e f   alm_db_output.obj
 0001:00020f47       __unwindfunclet$?loadFile@alm_db_output@@AAE_NABVQString@@@Z$12 10021f47 f   alm_db_output.obj
 0001:00020f50       __unwindfunclet$?loadFile@alm_db_output@@AAE_NABVQString@@@Z$13 10021f50 f   alm_db_output.obj
 0001:00020f59       __unwindfunclet$?loadFile@alm_db_output@@AAE_NABVQString@@@Z$14 10021f59 f   alm_db_output.obj
 0001:00020f62       __unwindfunclet$?loadFile@alm_db_output@@AAE_NABVQString@@@Z$15 10021f62 f   alm_db_output.obj
 0001:00020f6b       __unwindfunclet$?loadFile@alm_db_output@@AAE_NABVQString@@@Z$16 10021f6b f   alm_db_output.obj
 0001:00020f74       __unwindfunclet$?loadFile@alm_db_output@@AAE_NABVQString@@@Z$17 10021f74 f   alm_db_output.obj
 0001:00020f7d       __unwindfunclet$?loadFile@alm_db_output@@AAE_NABVQString@@@Z$18 10021f7d f   alm_db_output.obj
 0001:00020f86       __unwindfunclet$?loadFile@alm_db_output@@AAE_NABVQString@@@Z$19 10021f86 f   alm_db_output.obj
 0001:00020f8f       __unwindfunclet$?loadFile@alm_db_output@@AAE_NABVQString@@@Z$20 10021f8f f   alm_db_output.obj
 0001:00020f98       __unwindfunclet$?loadFile@alm_db_output@@AAE_NABVQString@@@Z$21 10021f98 f   alm_db_output.obj
 0001:00020fa1       __unwindfunclet$?loadFile@alm_db_output@@AAE_NABVQString@@@Z$22 10021fa1 f   alm_db_output.obj
 0001:00020fbb       __unwindfunclet$?loadFile@alm_db_output@@AAE_NABVQString@@@Z$23 10021fbb f   alm_db_output.obj
 0001:00020fd5       __unwindfunclet$?loadFile@alm_db_output@@AAE_NABVQString@@@Z$24 10021fd5 f   alm_db_output.obj
 0001:00020fdf       __unwindfunclet$?loadFile@alm_db_output@@AAE_NABVQString@@@Z$26 10021fdf f   alm_db_output.obj
 0001:00020fe9       __unwindfunclet$?loadFile@alm_db_output@@AAE_NABVQString@@@Z$28 10021fe9 f   alm_db_output.obj
 0001:00020ff3       __ehhandler$?loadFile@alm_db_output@@AAE_NABVQString@@@Z 10021ff3 f   alm_db_output.obj
 0001:00021011       __unwindfunclet$?loadProcesses@alm_db_output@@AAE_NABVQString@@@Z$0 10022011 f   alm_db_output.obj
 0001:0002101a       __unwindfunclet$?loadProcesses@alm_db_output@@AAE_NABVQString@@@Z$1 1002201a f   alm_db_output.obj
 0001:00021023       __unwindfunclet$?loadProcesses@alm_db_output@@AAE_NABVQString@@@Z$2 10022023 f   alm_db_output.obj
 0001:0002102c       __unwindfunclet$?loadProcesses@alm_db_output@@AAE_NABVQString@@@Z$3 1002202c f   alm_db_output.obj
 0001:00021035       __unwindfunclet$?loadProcesses@alm_db_output@@AAE_NABVQString@@@Z$4 10022035 f   alm_db_output.obj
 0001:00021041       __unwindfunclet$?loadProcesses@alm_db_output@@AAE_NABVQString@@@Z$5 10022041 f   alm_db_output.obj
 0001:0002104d       __unwindfunclet$?loadProcesses@alm_db_output@@AAE_NABVQString@@@Z$6 1002204d f   alm_db_output.obj
 0001:00021056       __unwindfunclet$?loadProcesses@alm_db_output@@AAE_NABVQString@@@Z$7 10022056 f   alm_db_output.obj
 0001:0002105f       __unwindfunclet$?loadProcesses@alm_db_output@@AAE_NABVQString@@@Z$8 1002205f f   alm_db_output.obj
 0001:00021068       __unwindfunclet$?loadProcesses@alm_db_output@@AAE_NABVQString@@@Z$9 10022068 f   alm_db_output.obj
 0001:00021071       __unwindfunclet$?loadProcesses@alm_db_output@@AAE_NABVQString@@@Z$10 10022071 f   alm_db_output.obj
 0001:0002107a       __unwindfunclet$?loadProcesses@alm_db_output@@AAE_NABVQString@@@Z$11 1002207a f   alm_db_output.obj
 0001:00021094       __unwindfunclet$?loadProcesses@alm_db_output@@AAE_NABVQString@@@Z$12 10022094 f   alm_db_output.obj
 0001:000210ae       __unwindfunclet$?loadProcesses@alm_db_output@@AAE_NABVQString@@@Z$13 100220ae f   alm_db_output.obj
 0001:000210b8       __unwindfunclet$?loadProcesses@alm_db_output@@AAE_NABVQString@@@Z$14 100220b8 f   alm_db_output.obj
 0001:000210c1       __unwindfunclet$?loadProcesses@alm_db_output@@AAE_NABVQString@@@Z$15 100220c1 f   alm_db_output.obj
 0001:000210ca       __unwindfunclet$?loadProcesses@alm_db_output@@AAE_NABVQString@@@Z$16 100220ca f   alm_db_output.obj
 0001:000210d3       __unwindfunclet$?loadProcesses@alm_db_output@@AAE_NABVQString@@@Z$17 100220d3 f   alm_db_output.obj
 0001:000210dc       __unwindfunclet$?loadProcesses@alm_db_output@@AAE_NABVQString@@@Z$18 100220dc f   alm_db_output.obj
 0001:000210e5       __unwindfunclet$?loadProcesses@alm_db_output@@AAE_NABVQString@@@Z$19 100220e5 f   alm_db_output.obj
 0001:000210ee       __unwindfunclet$?loadProcesses@alm_db_output@@AAE_NABVQString@@@Z$20 100220ee f   alm_db_output.obj
 0001:000210f7       __unwindfunclet$?loadProcesses@alm_db_output@@AAE_NABVQString@@@Z$22 100220f7 f   alm_db_output.obj
 0001:00021100       __unwindfunclet$?loadProcesses@alm_db_output@@AAE_NABVQString@@@Z$23 10022100 f   alm_db_output.obj
 0001:00021109       __unwindfunclet$?loadProcesses@alm_db_output@@AAE_NABVQString@@@Z$24 10022109 f   alm_db_output.obj
 0001:00021113       __unwindfunclet$?loadProcesses@alm_db_output@@AAE_NABVQString@@@Z$25 10022113 f   alm_db_output.obj
 0001:0002111c       __unwindfunclet$?loadProcesses@alm_db_output@@AAE_NABVQString@@@Z$26 1002211c f   alm_db_output.obj
 0001:00021125       __unwindfunclet$?loadProcesses@alm_db_output@@AAE_NABVQString@@@Z$27 10022125 f   alm_db_output.obj
 0001:0002112e       __unwindfunclet$?loadProcesses@alm_db_output@@AAE_NABVQString@@@Z$28 1002212e f   alm_db_output.obj
 0001:00021137       __unwindfunclet$?loadProcesses@alm_db_output@@AAE_NABVQString@@@Z$29 10022137 f   alm_db_output.obj
 0001:00021140       __unwindfunclet$?loadProcesses@alm_db_output@@AAE_NABVQString@@@Z$30 10022140 f   alm_db_output.obj
 0001:00021149       __unwindfunclet$?loadProcesses@alm_db_output@@AAE_NABVQString@@@Z$31 10022149 f   alm_db_output.obj
 0001:00021152       __ehhandler$?loadProcesses@alm_db_output@@AAE_NABVQString@@@Z 10022152 f   alm_db_output.obj
 0001:00021170       __unwindfunclet$?menuDeleteFile@alm_db_output@@AAEXXZ$0 10022170 f   alm_db_output.obj
 0001:0002117c       __unwindfunclet$?menuDeleteFile@alm_db_output@@AAEXXZ$1 1002217c f   alm_db_output.obj
 0001:00021188       __ehhandler$?menuDeleteFile@alm_db_output@@AAEXXZ 10022188 f   alm_db_output.obj
 0001:000211b0       __unwindfunclet$?menuDuplicateFile@alm_db_output@@AAEXXZ$0 100221b0 f   alm_db_output.obj
 0001:000211ba       __unwindfunclet$?menuDuplicateFile@alm_db_output@@AAEXXZ$1 100221ba f   alm_db_output.obj
 0001:000211c3       __unwindfunclet$?menuDuplicateFile@alm_db_output@@AAEXXZ$2 100221c3 f   alm_db_output.obj
 0001:000211cc       __unwindfunclet$?menuDuplicateFile@alm_db_output@@AAEXXZ$3 100221cc f   alm_db_output.obj
 0001:000211d5       __unwindfunclet$?menuDuplicateFile@alm_db_output@@AAEXXZ$4 100221d5 f   alm_db_output.obj
 0001:000211de       __unwindfunclet$?menuDuplicateFile@alm_db_output@@AAEXXZ$5 100221de f   alm_db_output.obj
 0001:000211e8       __unwindfunclet$?menuDuplicateFile@alm_db_output@@AAEXXZ$6 100221e8 f   alm_db_output.obj
 0001:000211f1       __unwindfunclet$?menuDuplicateFile@alm_db_output@@AAEXXZ$7 100221f1 f   alm_db_output.obj
 0001:000211fa       __unwindfunclet$?menuDuplicateFile@alm_db_output@@AAEXXZ$8 100221fa f   alm_db_output.obj
 0001:00021203       __unwindfunclet$?menuDuplicateFile@alm_db_output@@AAEXXZ$9 10022203 f   alm_db_output.obj
 0001:0002120c       __unwindfunclet$?menuDuplicateFile@alm_db_output@@AAEXXZ$10 1002220c f   alm_db_output.obj
 0001:00021215       __unwindfunclet$?menuDuplicateFile@alm_db_output@@AAEXXZ$11 10022215 f   alm_db_output.obj
 0001:0002121e       __unwindfunclet$?menuDuplicateFile@alm_db_output@@AAEXXZ$12 1002221e f   alm_db_output.obj
 0001:00021227       __ehhandler$?menuDuplicateFile@alm_db_output@@AAEXXZ 10022227 f   alm_db_output.obj
 0001:00021242       __unwindfunclet$?menus@alm_db_output@@UAE?AVQPopupMenuList@@XZ$0 10022242 f   alm_db_output.obj
 0001:0002125b       __ehhandler$?menus@alm_db_output@@UAE?AVQPopupMenuList@@XZ 1002225b f   alm_db_output.obj
 0001:00021276       __unwindfunclet$?navigate@alm_db_output@@UAEXABVQString@@0@Z$0 10022276 f   alm_db_output.obj
 0001:0002127f       __unwindfunclet$?navigate@alm_db_output@@UAEXABVQString@@0@Z$1 1002227f f   alm_db_output.obj
 0001:00021288       __unwindfunclet$?navigate@alm_db_output@@UAEXABVQString@@0@Z$2 10022288 f   alm_db_output.obj
 0001:00021291       __unwindfunclet$?navigate@alm_db_output@@UAEXABVQString@@0@Z$3 10022291 f   alm_db_output.obj
 0001:0002129a       __unwindfunclet$?navigate@alm_db_output@@UAEXABVQString@@0@Z$4 1002229a f   alm_db_output.obj
 0001:000212a3       __unwindfunclet$?navigate@alm_db_output@@UAEXABVQString@@0@Z$5 100222a3 f   alm_db_output.obj
 0001:000212ac       __unwindfunclet$?navigate@alm_db_output@@UAEXABVQString@@0@Z$6 100222ac f   alm_db_output.obj
 0001:000212c6       __unwindfunclet$?navigate@alm_db_output@@UAEXABVQString@@0@Z$7 100222c6 f   alm_db_output.obj
 0001:000212e0       __unwindfunclet$?navigate@alm_db_output@@UAEXABVQString@@0@Z$8 100222e0 f   alm_db_output.obj
 0001:000212e9       __unwindfunclet$?navigate@alm_db_output@@UAEXABVQString@@0@Z$9 100222e9 f   alm_db_output.obj
 0001:000212f2       __unwindfunclet$?navigate@alm_db_output@@UAEXABVQString@@0@Z$10 100222f2 f   alm_db_output.obj
 0001:000212fb       __unwindfunclet$?navigate@alm_db_output@@UAEXABVQString@@0@Z$11 100222fb f   alm_db_output.obj
 0001:00021304       __unwindfunclet$?navigate@alm_db_output@@UAEXABVQString@@0@Z$12 10022304 f   alm_db_output.obj
 0001:0002130d       __unwindfunclet$?navigate@alm_db_output@@UAEXABVQString@@0@Z$13 1002230d f   alm_db_output.obj
 0001:00021316       __unwindfunclet$?navigate@alm_db_output@@UAEXABVQString@@0@Z$14 10022316 f   alm_db_output.obj
 0001:0002131f       __unwindfunclet$?navigate@alm_db_output@@UAEXABVQString@@0@Z$15 1002231f f   alm_db_output.obj
 0001:00021328       __ehhandler$?navigate@alm_db_output@@UAEXABVQString@@0@Z 10022328 f   alm_db_output.obj
 0001:00021343       __unwindfunclet$?newFile@alm_db_output@@AAEXABVQString@@@Z$0 10022343 f   alm_db_output.obj
 0001:0002134c       __unwindfunclet$?newFile@alm_db_output@@AAEXABVQString@@@Z$1 1002234c f   alm_db_output.obj
 0001:00021355       __unwindfunclet$?newFile@alm_db_output@@AAEXABVQString@@@Z$2 10022355 f   alm_db_output.obj
 0001:0002135f       __unwindfunclet$?newFile@alm_db_output@@AAEXABVQString@@@Z$3 1002235f f   alm_db_output.obj
 0001:00021368       __unwindfunclet$?newFile@alm_db_output@@AAEXABVQString@@@Z$4 10022368 f   alm_db_output.obj
 0001:00021372       __unwindfunclet$?newFile@alm_db_output@@AAEXABVQString@@@Z$5 10022372 f   alm_db_output.obj
 0001:0002137b       __unwindfunclet$?newFile@alm_db_output@@AAEXABVQString@@@Z$6 1002237b f   alm_db_output.obj
 0001:00021384       __unwindfunclet$?newFile@alm_db_output@@AAEXABVQString@@@Z$7 10022384 f   alm_db_output.obj
 0001:0002138d       __unwindfunclet$?newFile@alm_db_output@@AAEXABVQString@@@Z$8 1002238d f   alm_db_output.obj
 0001:00021396       __unwindfunclet$?newFile@alm_db_output@@AAEXABVQString@@@Z$9 10022396 f   alm_db_output.obj
 0001:0002139f       __unwindfunclet$?newFile@alm_db_output@@AAEXABVQString@@@Z$10 1002239f f   alm_db_output.obj
 0001:000213a8       __unwindfunclet$?newFile@alm_db_output@@AAEXABVQString@@@Z$11 100223a8 f   alm_db_output.obj
 0001:000213b1       __unwindfunclet$?newFile@alm_db_output@@AAEXABVQString@@@Z$13 100223b1 f   alm_db_output.obj
 0001:000213bb       __unwindfunclet$?newFile@alm_db_output@@AAEXABVQString@@@Z$14 100223bb f   alm_db_output.obj
 0001:000213d5       __unwindfunclet$?newFile@alm_db_output@@AAEXABVQString@@@Z$15 100223d5 f   alm_db_output.obj
 0001:000213ef       __unwindfunclet$?newFile@alm_db_output@@AAEXABVQString@@@Z$16 100223ef f   alm_db_output.obj
 0001:000213f8       __ehhandler$?newFile@alm_db_output@@AAEXABVQString@@@Z 100223f8 f   alm_db_output.obj
 0001:00021413       __unwindfunclet$?pasteOptions@alm_db_output@@AAEXXZ$0 10022413 f   alm_db_output.obj
 0001:0002141c       __unwindfunclet$?pasteOptions@alm_db_output@@AAEXXZ$1 1002241c f   alm_db_output.obj
 0001:00021425       __unwindfunclet$?pasteOptions@alm_db_output@@AAEXXZ$2 10022425 f   alm_db_output.obj
 0001:0002142e       __unwindfunclet$?pasteOptions@alm_db_output@@AAEXXZ$3 1002242e f   alm_db_output.obj
 0001:00021437       __unwindfunclet$?pasteOptions@alm_db_output@@AAEXXZ$4 10022437 f   alm_db_output.obj
 0001:00021440       __ehhandler$?pasteOptions@alm_db_output@@AAEXXZ 10022440 f   alm_db_output.obj
 0001:0002145b       __unwindfunclet$?pasteSelectedProcs@alm_db_output@@AAEX_N@Z$0 1002245b f   alm_db_output.obj
 0001:00021464       __unwindfunclet$?pasteSelectedProcs@alm_db_output@@AAEX_N@Z$1 10022464 f   alm_db_output.obj
 0001:0002146d       __unwindfunclet$?pasteSelectedProcs@alm_db_output@@AAEX_N@Z$2 1002246d f   alm_db_output.obj
 0001:00021476       __unwindfunclet$?pasteSelectedProcs@alm_db_output@@AAEX_N@Z$3 10022476 f   alm_db_output.obj
 0001:0002147f       __unwindfunclet$?pasteSelectedProcs@alm_db_output@@AAEX_N@Z$4 1002247f f   alm_db_output.obj
 0001:00021488       __unwindfunclet$?pasteSelectedProcs@alm_db_output@@AAEX_N@Z$5 10022488 f   alm_db_output.obj
 0001:00021491       __unwindfunclet$?pasteSelectedProcs@alm_db_output@@AAEX_N@Z$6 10022491 f   alm_db_output.obj
 0001:0002149a       __unwindfunclet$?pasteSelectedProcs@alm_db_output@@AAEX_N@Z$7 1002249a f   alm_db_output.obj
 0001:000214a3       __unwindfunclet$?pasteSelectedProcs@alm_db_output@@AAEX_N@Z$8 100224a3 f   alm_db_output.obj
 0001:000214ac       __unwindfunclet$?pasteSelectedProcs@alm_db_output@@AAEX_N@Z$9 100224ac f   alm_db_output.obj
 0001:000214b5       __unwindfunclet$?pasteSelectedProcs@alm_db_output@@AAEX_N@Z$10 100224b5 f   alm_db_output.obj
 0001:000214be       __unwindfunclet$?pasteSelectedProcs@alm_db_output@@AAEX_N@Z$11 100224be f   alm_db_output.obj
 0001:000214c7       __unwindfunclet$?pasteSelectedProcs@alm_db_output@@AAEX_N@Z$12 100224c7 f   alm_db_output.obj
 0001:000214d0       __unwindfunclet$?pasteSelectedProcs@alm_db_output@@AAEX_N@Z$13 100224d0 f   alm_db_output.obj
 0001:000214d9       __unwindfunclet$?pasteSelectedProcs@alm_db_output@@AAEX_N@Z$14 100224d9 f   alm_db_output.obj
 0001:000214e2       __unwindfunclet$?pasteSelectedProcs@alm_db_output@@AAEX_N@Z$15 100224e2 f   alm_db_output.obj
 0001:000214eb       __unwindfunclet$?pasteSelectedProcs@alm_db_output@@AAEX_N@Z$16 100224eb f   alm_db_output.obj
 0001:000214f4       __unwindfunclet$?pasteSelectedProcs@alm_db_output@@AAEX_N@Z$17 100224f4 f   alm_db_output.obj
 0001:000214fd       __ehhandler$?pasteSelectedProcs@alm_db_output@@AAEX_N@Z 100224fd f   alm_db_output.obj
 0001:00021518       __unwindfunclet$?renameModule@alm_db_output@@AAEXPAVQListViewItem@@HABVQString@@@Z$0 10022518 f   alm_db_output.obj
 0001:00021521       __unwindfunclet$?renameModule@alm_db_output@@AAEXPAVQListViewItem@@HABVQString@@@Z$1 10022521 f   alm_db_output.obj
 0001:0002152a       __unwindfunclet$?renameModule@alm_db_output@@AAEXPAVQListViewItem@@HABVQString@@@Z$2 1002252a f   alm_db_output.obj
 0001:00021533       __unwindfunclet$?renameModule@alm_db_output@@AAEXPAVQListViewItem@@HABVQString@@@Z$3 10022533 f   alm_db_output.obj
 0001:0002153c       __unwindfunclet$?renameModule@alm_db_output@@AAEXPAVQListViewItem@@HABVQString@@@Z$4 1002253c f   alm_db_output.obj
 0001:00021545       __ehhandler$?renameModule@alm_db_output@@AAEXPAVQListViewItem@@HABVQString@@@Z 10022545 f   alm_db_output.obj
 0001:00021560       __unwindfunclet$?reply@alm_db_output@@UAEXPAVresponse@@@Z$0 10022560 f   alm_db_output.obj
 0001:00021569       __ehhandler$?reply@alm_db_output@@UAEXPAVresponse@@@Z 10022569 f   alm_db_output.obj
 0001:00021584       __unwindfunclet$?saveFile@alm_db_output@@AAE_NPAVcOutputFile@@@Z$0 10022584 f   alm_db_output.obj
 0001:0002158d       __unwindfunclet$?saveFile@alm_db_output@@AAE_NPAVcOutputFile@@@Z$1 1002258d f   alm_db_output.obj
 0001:00021596       __unwindfunclet$?saveFile@alm_db_output@@AAE_NPAVcOutputFile@@@Z$2 10022596 f   alm_db_output.obj
 0001:0002159f       __unwindfunclet$?saveFile@alm_db_output@@AAE_NPAVcOutputFile@@@Z$3 1002259f f   alm_db_output.obj
 0001:000215ab       __unwindfunclet$?saveFile@alm_db_output@@AAE_NPAVcOutputFile@@@Z$4 100225ab f   alm_db_output.obj
 0001:000215b4       __unwindfunclet$?saveFile@alm_db_output@@AAE_NPAVcOutputFile@@@Z$5 100225b4 f   alm_db_output.obj
 0001:000215bd       __unwindfunclet$?saveFile@alm_db_output@@AAE_NPAVcOutputFile@@@Z$6 100225bd f   alm_db_output.obj
 0001:000215c6       __unwindfunclet$?saveFile@alm_db_output@@AAE_NPAVcOutputFile@@@Z$7 100225c6 f   alm_db_output.obj
 0001:000215cf       __unwindfunclet$?saveFile@alm_db_output@@AAE_NPAVcOutputFile@@@Z$8 100225cf f   alm_db_output.obj
 0001:000215d8       __unwindfunclet$?saveFile@alm_db_output@@AAE_NPAVcOutputFile@@@Z$9 100225d8 f   alm_db_output.obj
 0001:000215e1       __unwindfunclet$?saveFile@alm_db_output@@AAE_NPAVcOutputFile@@@Z$10 100225e1 f   alm_db_output.obj
 0001:000215ea       __unwindfunclet$?saveFile@alm_db_output@@AAE_NPAVcOutputFile@@@Z$11 100225ea f   alm_db_output.obj
 0001:000215f3       __unwindfunclet$?saveFile@alm_db_output@@AAE_NPAVcOutputFile@@@Z$12 100225f3 f   alm_db_output.obj
 0001:000215fc       __unwindfunclet$?saveFile@alm_db_output@@AAE_NPAVcOutputFile@@@Z$13 100225fc f   alm_db_output.obj
 0001:00021605       __unwindfunclet$?saveFile@alm_db_output@@AAE_NPAVcOutputFile@@@Z$14 10022605 f   alm_db_output.obj
 0001:0002160e       __unwindfunclet$?saveFile@alm_db_output@@AAE_NPAVcOutputFile@@@Z$15 1002260e f   alm_db_output.obj
 0001:00021617       __unwindfunclet$?saveFile@alm_db_output@@AAE_NPAVcOutputFile@@@Z$16 10022617 f   alm_db_output.obj
 0001:00021620       __unwindfunclet$?saveFile@alm_db_output@@AAE_NPAVcOutputFile@@@Z$17 10022620 f   alm_db_output.obj
 0001:00021629       __unwindfunclet$?saveFile@alm_db_output@@AAE_NPAVcOutputFile@@@Z$18 10022629 f   alm_db_output.obj
 0001:00021632       __unwindfunclet$?saveFile@alm_db_output@@AAE_NPAVcOutputFile@@@Z$19 10022632 f   alm_db_output.obj
 0001:0002163b       __unwindfunclet$?saveFile@alm_db_output@@AAE_NPAVcOutputFile@@@Z$20 1002263b f   alm_db_output.obj
 0001:00021644       __unwindfunclet$?saveFile@alm_db_output@@AAE_NPAVcOutputFile@@@Z$21 10022644 f   alm_db_output.obj
 0001:0002164d       __unwindfunclet$?saveFile@alm_db_output@@AAE_NPAVcOutputFile@@@Z$22 1002264d f   alm_db_output.obj
 0001:00021656       __unwindfunclet$?saveFile@alm_db_output@@AAE_NPAVcOutputFile@@@Z$23 10022656 f   alm_db_output.obj
 0001:0002165f       __unwindfunclet$?saveFile@alm_db_output@@AAE_NPAVcOutputFile@@@Z$24 1002265f f   alm_db_output.obj
 0001:00021668       __unwindfunclet$?saveFile@alm_db_output@@AAE_NPAVcOutputFile@@@Z$25 10022668 f   alm_db_output.obj
 0001:00021671       __unwindfunclet$?saveFile@alm_db_output@@AAE_NPAVcOutputFile@@@Z$26 10022671 f   alm_db_output.obj
 0001:0002167a       __unwindfunclet$?saveFile@alm_db_output@@AAE_NPAVcOutputFile@@@Z$27 1002267a f   alm_db_output.obj
 0001:00021683       __unwindfunclet$?saveFile@alm_db_output@@AAE_NPAVcOutputFile@@@Z$28 10022683 f   alm_db_output.obj
 0001:0002168c       __unwindfunclet$?saveFile@alm_db_output@@AAE_NPAVcOutputFile@@@Z$29 1002268c f   alm_db_output.obj
 0001:00021695       __unwindfunclet$?saveFile@alm_db_output@@AAE_NPAVcOutputFile@@@Z$30 10022695 f   alm_db_output.obj
 0001:0002169e       __unwindfunclet$?saveFile@alm_db_output@@AAE_NPAVcOutputFile@@@Z$31 1002269e f   alm_db_output.obj
 0001:000216a7       __unwindfunclet$?saveFile@alm_db_output@@AAE_NPAVcOutputFile@@@Z$32 100226a7 f   alm_db_output.obj
 0001:000216b0       __unwindfunclet$?saveFile@alm_db_output@@AAE_NPAVcOutputFile@@@Z$33 100226b0 f   alm_db_output.obj
 0001:000216b9       __unwindfunclet$?saveFile@alm_db_output@@AAE_NPAVcOutputFile@@@Z$34 100226b9 f   alm_db_output.obj
 0001:000216c2       __unwindfunclet$?saveFile@alm_db_output@@AAE_NPAVcOutputFile@@@Z$35 100226c2 f   alm_db_output.obj
 0001:000216cb       __unwindfunclet$?saveFile@alm_db_output@@AAE_NPAVcOutputFile@@@Z$36 100226cb f   alm_db_output.obj
 0001:000216d4       __unwindfunclet$?saveFile@alm_db_output@@AAE_NPAVcOutputFile@@@Z$37 100226d4 f   alm_db_output.obj
 0001:000216dd       __unwindfunclet$?saveFile@alm_db_output@@AAE_NPAVcOutputFile@@@Z$38 100226dd f   alm_db_output.obj
 0001:000216e6       __unwindfunclet$?saveFile@alm_db_output@@AAE_NPAVcOutputFile@@@Z$39 100226e6 f   alm_db_output.obj
 0001:000216ef       __unwindfunclet$?saveFile@alm_db_output@@AAE_NPAVcOutputFile@@@Z$40 100226ef f   alm_db_output.obj
 0001:000216f8       __unwindfunclet$?saveFile@alm_db_output@@AAE_NPAVcOutputFile@@@Z$41 100226f8 f   alm_db_output.obj
 0001:00021701       __unwindfunclet$?saveFile@alm_db_output@@AAE_NPAVcOutputFile@@@Z$42 10022701 f   alm_db_output.obj
 0001:0002170a       __unwindfunclet$?saveFile@alm_db_output@@AAE_NPAVcOutputFile@@@Z$43 1002270a f   alm_db_output.obj
 0001:00021713       __unwindfunclet$?saveFile@alm_db_output@@AAE_NPAVcOutputFile@@@Z$44 10022713 f   alm_db_output.obj
 0001:0002171c       __unwindfunclet$?saveFile@alm_db_output@@AAE_NPAVcOutputFile@@@Z$45 1002271c f   alm_db_output.obj
 0001:00021725       __unwindfunclet$?saveFile@alm_db_output@@AAE_NPAVcOutputFile@@@Z$46 10022725 f   alm_db_output.obj
 0001:0002172e       __unwindfunclet$?saveFile@alm_db_output@@AAE_NPAVcOutputFile@@@Z$47 1002272e f   alm_db_output.obj
 0001:00021737       __unwindfunclet$?saveFile@alm_db_output@@AAE_NPAVcOutputFile@@@Z$48 10022737 f   alm_db_output.obj
 0001:00021740       __unwindfunclet$?saveFile@alm_db_output@@AAE_NPAVcOutputFile@@@Z$49 10022740 f   alm_db_output.obj
 0001:00021749       __unwindfunclet$?saveFile@alm_db_output@@AAE_NPAVcOutputFile@@@Z$50 10022749 f   alm_db_output.obj
 0001:00021752       __unwindfunclet$?saveFile@alm_db_output@@AAE_NPAVcOutputFile@@@Z$51 10022752 f   alm_db_output.obj
 0001:0002175b       __unwindfunclet$?saveFile@alm_db_output@@AAE_NPAVcOutputFile@@@Z$52 1002275b f   alm_db_output.obj
 0001:00021767       __unwindfunclet$?saveFile@alm_db_output@@AAE_NPAVcOutputFile@@@Z$53 10022767 f   alm_db_output.obj
 0001:00021770       __unwindfunclet$?saveFile@alm_db_output@@AAE_NPAVcOutputFile@@@Z$54 10022770 f   alm_db_output.obj
 0001:00021779       __unwindfunclet$?saveFile@alm_db_output@@AAE_NPAVcOutputFile@@@Z$55 10022779 f   alm_db_output.obj
 0001:00021785       __unwindfunclet$?saveFile@alm_db_output@@AAE_NPAVcOutputFile@@@Z$56 10022785 f   alm_db_output.obj
 0001:0002178e       __unwindfunclet$?saveFile@alm_db_output@@AAE_NPAVcOutputFile@@@Z$57 1002278e f   alm_db_output.obj
 0001:0002179a       __unwindfunclet$?saveFile@alm_db_output@@AAE_NPAVcOutputFile@@@Z$58 1002279a f   alm_db_output.obj
 0001:000217a3       __unwindfunclet$?saveFile@alm_db_output@@AAE_NPAVcOutputFile@@@Z$59 100227a3 f   alm_db_output.obj
 0001:000217af       __unwindfunclet$?saveFile@alm_db_output@@AAE_NPAVcOutputFile@@@Z$60 100227af f   alm_db_output.obj
 0001:000217b8       __unwindfunclet$?saveFile@alm_db_output@@AAE_NPAVcOutputFile@@@Z$61 100227b8 f   alm_db_output.obj
 0001:000217c4       __unwindfunclet$?saveFile@alm_db_output@@AAE_NPAVcOutputFile@@@Z$62 100227c4 f   alm_db_output.obj
 0001:000217cd       __unwindfunclet$?saveFile@alm_db_output@@AAE_NPAVcOutputFile@@@Z$63 100227cd f   alm_db_output.obj
 0001:000217d9       __unwindfunclet$?saveFile@alm_db_output@@AAE_NPAVcOutputFile@@@Z$64 100227d9 f   alm_db_output.obj
 0001:000217e2       __unwindfunclet$?saveFile@alm_db_output@@AAE_NPAVcOutputFile@@@Z$65 100227e2 f   alm_db_output.obj
 0001:000217eb       __unwindfunclet$?saveFile@alm_db_output@@AAE_NPAVcOutputFile@@@Z$66 100227eb f   alm_db_output.obj
 0001:000217f4       __unwindfunclet$?saveFile@alm_db_output@@AAE_NPAVcOutputFile@@@Z$67 100227f4 f   alm_db_output.obj
 0001:000217fd       __unwindfunclet$?saveFile@alm_db_output@@AAE_NPAVcOutputFile@@@Z$68 100227fd f   alm_db_output.obj
 0001:00021806       __unwindfunclet$?saveFile@alm_db_output@@AAE_NPAVcOutputFile@@@Z$69 10022806 f   alm_db_output.obj
 0001:0002180f       __unwindfunclet$?saveFile@alm_db_output@@AAE_NPAVcOutputFile@@@Z$70 1002280f f   alm_db_output.obj
 0001:00021818       __unwindfunclet$?saveFile@alm_db_output@@AAE_NPAVcOutputFile@@@Z$71 10022818 f   alm_db_output.obj
 0001:00021824       __ehhandler$?saveFile@alm_db_output@@AAE_NPAVcOutputFile@@@Z 10022824 f   alm_db_output.obj
 0001:00021842       __unwindfunclet$?selectFile@alm_db_output@@AAEXPAVQListViewItem@@@Z$0 10022842 f   alm_db_output.obj
 0001:0002184b       __unwindfunclet$?selectFile@alm_db_output@@AAEXPAVQListViewItem@@@Z$1 1002284b f   alm_db_output.obj
 0001:00021854       __unwindfunclet$?selectFile@alm_db_output@@AAEXPAVQListViewItem@@@Z$2 10022854 f   alm_db_output.obj
 0001:0002185d       __unwindfunclet$?selectFile@alm_db_output@@AAEXPAVQListViewItem@@@Z$3 1002285d f   alm_db_output.obj
 0001:00021866       __unwindfunclet$?selectFile@alm_db_output@@AAEXPAVQListViewItem@@@Z$4 10022866 f   alm_db_output.obj
 0001:0002186f       __unwindfunclet$?selectFile@alm_db_output@@AAEXPAVQListViewItem@@@Z$5 1002286f f   alm_db_output.obj
 0001:00021878       __unwindfunclet$?selectFile@alm_db_output@@AAEXPAVQListViewItem@@@Z$6 10022878 f   alm_db_output.obj
 0001:00021881       __unwindfunclet$?selectFile@alm_db_output@@AAEXPAVQListViewItem@@@Z$7 10022881 f   alm_db_output.obj
 0001:0002188a       __ehhandler$?selectFile@alm_db_output@@AAEXPAVQListViewItem@@@Z 1002288a f   alm_db_output.obj
 0001:000218a5       __unwindfunclet$?selectProcess@alm_db_output@@AAEXABVQString@@@Z$0 100228a5 f   alm_db_output.obj
 0001:000218ae       __unwindfunclet$?selectProcess@alm_db_output@@AAEXABVQString@@@Z$1 100228ae f   alm_db_output.obj
 0001:000218b7       __ehhandler$?selectProcess@alm_db_output@@AAEXABVQString@@@Z 100228b7 f   alm_db_output.obj
 0001:000218d2       __unwindfunclet$?selectSystem@alm_db_output@@AAEXABVQString@@@Z$0 100228d2 f   alm_db_output.obj
 0001:000218db       __unwindfunclet$?selectSystem@alm_db_output@@AAEXABVQString@@@Z$1 100228db f   alm_db_output.obj
 0001:000218e4       __unwindfunclet$?selectSystem@alm_db_output@@AAEXABVQString@@@Z$2 100228e4 f   alm_db_output.obj
 0001:000218ed       __unwindfunclet$?selectSystem@alm_db_output@@AAEXABVQString@@@Z$3 100228ed f   alm_db_output.obj
 0001:000218f6       __unwindfunclet$?selectSystem@alm_db_output@@AAEXABVQString@@@Z$4 100228f6 f   alm_db_output.obj
 0001:000218ff       __unwindfunclet$?selectSystem@alm_db_output@@AAEXABVQString@@@Z$5 100228ff f   alm_db_output.obj
 0001:00021908       __unwindfunclet$?selectSystem@alm_db_output@@AAEXABVQString@@@Z$6 10022908 f   alm_db_output.obj
 0001:00021911       __unwindfunclet$?selectSystem@alm_db_output@@AAEXABVQString@@@Z$7 10022911 f   alm_db_output.obj
 0001:0002191a       __unwindfunclet$?selectSystem@alm_db_output@@AAEXABVQString@@@Z$8 1002291a f   alm_db_output.obj
 0001:00021923       __unwindfunclet$?selectSystem@alm_db_output@@AAEXABVQString@@@Z$9 10022923 f   alm_db_output.obj
 0001:0002192c       __unwindfunclet$?selectSystem@alm_db_output@@AAEXABVQString@@@Z$11 1002292c f   alm_db_output.obj
 0001:00021935       __unwindfunclet$?selectSystem@alm_db_output@@AAEXABVQString@@@Z$12 10022935 f   alm_db_output.obj
 0001:0002193e       __unwindfunclet$?selectSystem@alm_db_output@@AAEXABVQString@@@Z$13 1002293e f   alm_db_output.obj
 0001:00021947       __unwindfunclet$?selectSystem@alm_db_output@@AAEXABVQString@@@Z$14 10022947 f   alm_db_output.obj
 0001:00021950       __unwindfunclet$?selectSystem@alm_db_output@@AAEXABVQString@@@Z$15 10022950 f   alm_db_output.obj
 0001:00021959       __unwindfunclet$?selectSystem@alm_db_output@@AAEXABVQString@@@Z$16 10022959 f   alm_db_output.obj
 0001:00021962       __unwindfunclet$?selectSystem@alm_db_output@@AAEXABVQString@@@Z$17 10022962 f   alm_db_output.obj
 0001:0002196b       __unwindfunclet$?selectSystem@alm_db_output@@AAEXABVQString@@@Z$18 1002296b f   alm_db_output.obj
 0001:00021974       __unwindfunclet$?selectSystem@alm_db_output@@AAEXABVQString@@@Z$19 10022974 f   alm_db_output.obj
 0001:0002197d       __unwindfunclet$?selectSystem@alm_db_output@@AAEXABVQString@@@Z$20 1002297d f   alm_db_output.obj
 0001:00021986       __unwindfunclet$?selectSystem@alm_db_output@@AAEXABVQString@@@Z$21 10022986 f   alm_db_output.obj
 0001:0002198f       __unwindfunclet$?selectSystem@alm_db_output@@AAEXABVQString@@@Z$22 1002298f f   alm_db_output.obj
 0001:00021998       __unwindfunclet$?selectSystem@alm_db_output@@AAEXABVQString@@@Z$23 10022998 f   alm_db_output.obj
 0001:000219a1       __unwindfunclet$?selectSystem@alm_db_output@@AAEXABVQString@@@Z$24 100229a1 f   alm_db_output.obj
 0001:000219aa       __ehhandler$?selectSystem@alm_db_output@@AAEXABVQString@@@Z 100229aa f   alm_db_output.obj
 0001:000219c5       __unwindfunclet$?sendCommand@alm_db_output@@UAEXABVQString@@0@Z$0 100229c5 f   alm_db_output.obj
 0001:000219ce       __ehhandler$?sendCommand@alm_db_output@@UAEXABVQString@@0@Z 100229ce f   alm_db_output.obj
 0001:000219e9       __unwindfunclet$?templateProcess@alm_db_output@@AAEXXZ$0 100229e9 f   alm_db_output.obj
 0001:000219f2       __unwindfunclet$?templateProcess@alm_db_output@@AAEXXZ$1 100229f2 f   alm_db_output.obj
 0001:000219fd       __unwindfunclet$?templateProcess@alm_db_output@@AAEXXZ$2 100229fd f   alm_db_output.obj
 0001:00021a06       __unwindfunclet$?templateProcess@alm_db_output@@AAEXXZ$3 10022a06 f   alm_db_output.obj
 0001:00021a0f       __unwindfunclet$?templateProcess@alm_db_output@@AAEXXZ$4 10022a0f f   alm_db_output.obj
 0001:00021a19       __unwindfunclet$?templateProcess@alm_db_output@@AAEXXZ$5 10022a19 f   alm_db_output.obj
 0001:00021a22       __unwindfunclet$?templateProcess@alm_db_output@@AAEXXZ$6 10022a22 f   alm_db_output.obj
 0001:00021a2b       __unwindfunclet$?templateProcess@alm_db_output@@AAEXXZ$8 10022a2b f   alm_db_output.obj
 0001:00021a34       __unwindfunclet$?templateProcess@alm_db_output@@AAEXXZ$9 10022a34 f   alm_db_output.obj
 0001:00021a3d       __unwindfunclet$?templateProcess@alm_db_output@@AAEXXZ$10 10022a3d f   alm_db_output.obj
 0001:00021a46       __unwindfunclet$?templateProcess@alm_db_output@@AAEXXZ$11 10022a46 f   alm_db_output.obj
 0001:00021a4f       __unwindfunclet$?templateProcess@alm_db_output@@AAEXXZ$13 10022a4f f   alm_db_output.obj
 0001:00021a58       __unwindfunclet$?templateProcess@alm_db_output@@AAEXXZ$14 10022a58 f   alm_db_output.obj
 0001:00021a61       __unwindfunclet$?templateProcess@alm_db_output@@AAEXXZ$15 10022a61 f   alm_db_output.obj
 0001:00021a6a       __unwindfunclet$?templateProcess@alm_db_output@@AAEXXZ$16 10022a6a f   alm_db_output.obj
 0001:00021a73       __unwindfunclet$?templateProcess@alm_db_output@@AAEXXZ$18 10022a73 f   alm_db_output.obj
 0001:00021a7c       __unwindfunclet$?templateProcess@alm_db_output@@AAEXXZ$19 10022a7c f   alm_db_output.obj
 0001:00021a85       __unwindfunclet$?templateProcess@alm_db_output@@AAEXXZ$20 10022a85 f   alm_db_output.obj
 0001:00021a8e       __unwindfunclet$?templateProcess@alm_db_output@@AAEXXZ$21 10022a8e f   alm_db_output.obj
 0001:00021a97       __unwindfunclet$?templateProcess@alm_db_output@@AAEXXZ$22 10022a97 f   alm_db_output.obj
 0001:00021aa0       __unwindfunclet$?templateProcess@alm_db_output@@AAEXXZ$23 10022aa0 f   alm_db_output.obj
 0001:00021aa9       __unwindfunclet$?templateProcess@alm_db_output@@AAEXXZ$24 10022aa9 f   alm_db_output.obj
 0001:00021ab2       __unwindfunclet$?templateProcess@alm_db_output@@AAEXXZ$25 10022ab2 f   alm_db_output.obj
 0001:00021abb       __unwindfunclet$?templateProcess@alm_db_output@@AAEXXZ$26 10022abb f   alm_db_output.obj
 0001:00021ac4       __unwindfunclet$?templateProcess@alm_db_output@@AAEXXZ$27 10022ac4 f   alm_db_output.obj
 0001:00021acd       __unwindfunclet$?templateProcess@alm_db_output@@AAEXXZ$28 10022acd f   alm_db_output.obj
 0001:00021ad6       __unwindfunclet$?templateProcess@alm_db_output@@AAEXXZ$29 10022ad6 f   alm_db_output.obj
 0001:00021adf       __unwindfunclet$?templateProcess@alm_db_output@@AAEXXZ$30 10022adf f   alm_db_output.obj
 0001:00021ae8       __ehhandler$?templateProcess@alm_db_output@@AAEXXZ 10022ae8 f   alm_db_output.obj
 0001:00021b06       __unwindfunclet$?toolbars@alm_db_output@@UAE?AVQDockWindowList@@XZ$0 10022b06 f   alm_db_output.obj
 0001:00021b1f       __ehhandler$?toolbars@alm_db_output@@UAE?AVQDockWindowList@@XZ 10022b1f f   alm_db_output.obj
 0001:00021b3a       __unwindfunclet$?updateFileList@alm_db_output@@AAEXXZ$0 10022b3a f   alm_db_output.obj
 0001:00021b46       __unwindfunclet$?updateFileList@alm_db_output@@AAEXXZ$1 10022b46 f   alm_db_output.obj
 0001:00021b52       __unwindfunclet$?updateFileList@alm_db_output@@AAEXXZ$2 10022b52 f   alm_db_output.obj
 0001:00021b5e       __unwindfunclet$?updateFileList@alm_db_output@@AAEXXZ$3 10022b5e f   alm_db_output.obj
 0001:00021b6a       __unwindfunclet$?updateFileList@alm_db_output@@AAEXXZ$4 10022b6a f   alm_db_output.obj
 0001:00021b76       __unwindfunclet$?updateFileList@alm_db_output@@AAEXXZ$5 10022b76 f   alm_db_output.obj
 0001:00021b82       __unwindfunclet$?updateFileList@alm_db_output@@AAEXXZ$6 10022b82 f   alm_db_output.obj
 0001:00021b8e       __unwindfunclet$?updateFileList@alm_db_output@@AAEXXZ$7 10022b8e f   alm_db_output.obj
 0001:00021b99       __unwindfunclet$?updateFileList@alm_db_output@@AAEXXZ$8 10022b99 f   alm_db_output.obj
 0001:00021ba5       __unwindfunclet$?updateFileList@alm_db_output@@AAEXXZ$9 10022ba5 f   alm_db_output.obj
 0001:00021bb1       __unwindfunclet$?updateFileList@alm_db_output@@AAEXXZ$10 10022bb1 f   alm_db_output.obj
 0001:00021bbd       __unwindfunclet$?updateFileList@alm_db_output@@AAEXXZ$11 10022bbd f   alm_db_output.obj
 0001:00021bc9       __unwindfunclet$?updateFileList@alm_db_output@@AAEXXZ$12 10022bc9 f   alm_db_output.obj
 0001:00021bd5       __unwindfunclet$?updateFileList@alm_db_output@@AAEXXZ$13 10022bd5 f   alm_db_output.obj
 0001:00021be1       __unwindfunclet$?updateFileList@alm_db_output@@AAEXXZ$14 10022be1 f   alm_db_output.obj
 0001:00021bed       __unwindfunclet$?updateFileList@alm_db_output@@AAEXXZ$15 10022bed f   alm_db_output.obj
 0001:00021bf9       __unwindfunclet$?updateFileList@alm_db_output@@AAEXXZ$16 10022bf9 f   alm_db_output.obj
 0001:00021c05       __unwindfunclet$?updateFileList@alm_db_output@@AAEXXZ$17 10022c05 f   alm_db_output.obj
 0001:00021c11       __unwindfunclet$?updateFileList@alm_db_output@@AAEXXZ$18 10022c11 f   alm_db_output.obj
 0001:00021c1d       __unwindfunclet$?updateFileList@alm_db_output@@AAEXXZ$19 10022c1d f   alm_db_output.obj
 0001:00021c29       __unwindfunclet$?updateFileList@alm_db_output@@AAEXXZ$20 10022c29 f   alm_db_output.obj
 0001:00021c35       __unwindfunclet$?updateFileList@alm_db_output@@AAEXXZ$21 10022c35 f   alm_db_output.obj
 0001:00021c41       __unwindfunclet$?updateFileList@alm_db_output@@AAEXXZ$22 10022c41 f   alm_db_output.obj
 0001:00021c4d       __unwindfunclet$?updateFileList@alm_db_output@@AAEXXZ$23 10022c4d f   alm_db_output.obj
 0001:00021c59       __unwindfunclet$?updateFileList@alm_db_output@@AAEXXZ$24 10022c59 f   alm_db_output.obj
 0001:00021c65       __unwindfunclet$?updateFileList@alm_db_output@@AAEXXZ$25 10022c65 f   alm_db_output.obj
 0001:00021c71       __unwindfunclet$?updateFileList@alm_db_output@@AAEXXZ$26 10022c71 f   alm_db_output.obj
 0001:00021c7d       __unwindfunclet$?updateFileList@alm_db_output@@AAEXXZ$27 10022c7d f   alm_db_output.obj
 0001:00021c89       __unwindfunclet$?updateFileList@alm_db_output@@AAEXXZ$28 10022c89 f   alm_db_output.obj
 0001:00021c95       __unwindfunclet$?updateFileList@alm_db_output@@AAEXXZ$29 10022c95 f   alm_db_output.obj
 0001:00021ca2       __unwindfunclet$?updateFileList@alm_db_output@@AAEXXZ$30 10022ca2 f   alm_db_output.obj
 0001:00021cae       __unwindfunclet$?updateFileList@alm_db_output@@AAEXXZ$31 10022cae f   alm_db_output.obj
 0001:00021cba       __unwindfunclet$?updateFileList@alm_db_output@@AAEXXZ$32 10022cba f   alm_db_output.obj
 0001:00021cc6       __unwindfunclet$?updateFileList@alm_db_output@@AAEXXZ$33 10022cc6 f   alm_db_output.obj
 0001:00021cd2       __unwindfunclet$?updateFileList@alm_db_output@@AAEXXZ$34 10022cd2 f   alm_db_output.obj
 0001:00021cde       __unwindfunclet$?updateFileList@alm_db_output@@AAEXXZ$35 10022cde f   alm_db_output.obj
 0001:00021cea       __unwindfunclet$?updateFileList@alm_db_output@@AAEXXZ$36 10022cea f   alm_db_output.obj
 0001:00021cf6       __unwindfunclet$?updateFileList@alm_db_output@@AAEXXZ$38 10022cf6 f   alm_db_output.obj
 0001:00021d02       __unwindfunclet$?updateFileList@alm_db_output@@AAEXXZ$39 10022d02 f   alm_db_output.obj
 0001:00021d0e       __unwindfunclet$?updateFileList@alm_db_output@@AAEXXZ$40 10022d0e f   alm_db_output.obj
 0001:00021d1a       __unwindfunclet$?updateFileList@alm_db_output@@AAEXXZ$41 10022d1a f   alm_db_output.obj
 0001:00021d27       __unwindfunclet$?updateFileList@alm_db_output@@AAEXXZ$42 10022d27 f   alm_db_output.obj
 0001:00021d33       __unwindfunclet$?updateFileList@alm_db_output@@AAEXXZ$43 10022d33 f   alm_db_output.obj
 0001:00021d3f       __unwindfunclet$?updateFileList@alm_db_output@@AAEXXZ$44 10022d3f f   alm_db_output.obj
 0001:00021d4b       __unwindfunclet$?updateFileList@alm_db_output@@AAEXXZ$45 10022d4b f   alm_db_output.obj
 0001:00021d57       __unwindfunclet$?updateFileList@alm_db_output@@AAEXXZ$46 10022d57 f   alm_db_output.obj
 0001:00021d63       __unwindfunclet$?updateFileList@alm_db_output@@AAEXXZ$47 10022d63 f   alm_db_output.obj
 0001:00021d6f       __unwindfunclet$?updateFileList@alm_db_output@@AAEXXZ$48 10022d6f f   alm_db_output.obj
 0001:00021d7c       __unwindfunclet$?updateFileList@alm_db_output@@AAEXXZ$49 10022d7c f   alm_db_output.obj
 0001:00021d88       __unwindfunclet$?updateFileList@alm_db_output@@AAEXXZ$50 10022d88 f   alm_db_output.obj
 0001:00021d94       __unwindfunclet$?updateFileList@alm_db_output@@AAEXXZ$51 10022d94 f   alm_db_output.obj
 0001:00021da0       __unwindfunclet$?updateFileList@alm_db_output@@AAEXXZ$52 10022da0 f   alm_db_output.obj
 0001:00021dac       __unwindfunclet$?updateFileList@alm_db_output@@AAEXXZ$53 10022dac f   alm_db_output.obj
 0001:00021db8       __unwindfunclet$?updateFileList@alm_db_output@@AAEXXZ$54 10022db8 f   alm_db_output.obj
 0001:00021dc4       __unwindfunclet$?updateFileList@alm_db_output@@AAEXXZ$55 10022dc4 f   alm_db_output.obj
 0001:00021dd0       __ehhandler$?updateFileList@alm_db_output@@AAEXXZ 10022dd0 f   alm_db_output.obj
 0001:00021df8       __unwindfunclet$?updateList@alm_db_output@@AAEXXZ$0 10022df8 f   alm_db_output.obj
 0001:00021e01       __unwindfunclet$?updateList@alm_db_output@@AAEXXZ$1 10022e01 f   alm_db_output.obj
 0001:00021e0a       __unwindfunclet$?updateList@alm_db_output@@AAEXXZ$3 10022e0a f   alm_db_output.obj
 0001:00021e13       __unwindfunclet$?updateList@alm_db_output@@AAEXXZ$4 10022e13 f   alm_db_output.obj
 0001:00021e1c       __unwindfunclet$?updateList@alm_db_output@@AAEXXZ$5 10022e1c f   alm_db_output.obj
 0001:00021e25       __ehhandler$?updateList@alm_db_output@@AAEXXZ 10022e25 f   alm_db_output.obj
 0001:00021e40       __unwindfunclet$?useAltId@alm_db_output@@AAE?AVQString@@V2@ABV2@_N@Z$0 10022e40 f   alm_db_output.obj
 0001:00021e49       __unwindfunclet$?useAltId@alm_db_output@@AAE?AVQString@@V2@ABV2@_N@Z$1 10022e49 f   alm_db_output.obj
 0001:00021e63       __unwindfunclet$?useAltId@alm_db_output@@AAE?AVQString@@V2@ABV2@_N@Z$2 10022e63 f   alm_db_output.obj
 0001:00021e6c       __ehhandler$?useAltId@alm_db_output@@AAE?AVQString@@V2@ABV2@_N@Z 10022e6c f   alm_db_output.obj
 0001:00021e87       __unwindfunclet$??1cOutputFile@@UAE@XZ$0 10022e87 f   cOutputFile.obj
 0001:00021e87       __unwindfunclet$??0cOutputFile@@QAE@XZ$0 10022e87 f   cOutputFile.obj
 0001:00021e93       __unwindfunclet$??0cOutputFile@@QAE@XZ$1 10022e93 f   cOutputFile.obj
 0001:00021e93       __unwindfunclet$??1cOutputFile@@UAE@XZ$1 10022e93 f   cOutputFile.obj
 0001:00021e9f       __ehhandler$??0cOutputFile@@QAE@XZ 10022e9f f   cOutputFile.obj
 0001:00021e9f       __ehhandler$??1cOutputFile@@UAE@XZ 10022e9f f   cOutputFile.obj
 0001:00021eba       __unwindfunclet$??0cProcess@@QAE@VQString@@@Z$0 10022eba f   cProcess.obj
 0001:00021ec3       __unwindfunclet$??0cProcess@@QAE@VQString@@@Z$1 10022ec3 f   cProcess.obj
 0001:00021ecf       __unwindfunclet$??0cProcess@@QAE@VQString@@@Z$2 10022ecf f   cProcess.obj
 0001:00021edb       __unwindfunclet$??0cProcess@@QAE@VQString@@@Z$3 10022edb f   cProcess.obj
 0001:00021ee7       __unwindfunclet$??0cProcess@@QAE@VQString@@@Z$4 10022ee7 f   cProcess.obj
 0001:00021ef3       __unwindfunclet$??0cProcess@@QAE@VQString@@@Z$5 10022ef3 f   cProcess.obj
 0001:00021eff       __unwindfunclet$??0cProcess@@QAE@VQString@@@Z$6 10022eff f   cProcess.obj
 0001:00021f0b       __unwindfunclet$??0cProcess@@QAE@VQString@@@Z$7 10022f0b f   cProcess.obj
 0001:00021f17       __unwindfunclet$??0cProcess@@QAE@VQString@@@Z$8 10022f17 f   cProcess.obj
 0001:00021f23       __unwindfunclet$??0cProcess@@QAE@VQString@@@Z$9 10022f23 f   cProcess.obj
 0001:00021f2f       __ehhandler$??0cProcess@@QAE@VQString@@@Z 10022f2f f   cProcess.obj
 0001:00021f4a       __unwindfunclet$??1cProcess@@UAE@XZ$0 10022f4a f   cProcess.obj
 0001:00021f56       __unwindfunclet$??1cProcess@@UAE@XZ$1 10022f56 f   cProcess.obj
 0001:00021f62       __unwindfunclet$??1cProcess@@UAE@XZ$2 10022f62 f   cProcess.obj
 0001:00021f6e       __unwindfunclet$??1cProcess@@UAE@XZ$3 10022f6e f   cProcess.obj
 0001:00021f7a       __unwindfunclet$??1cProcess@@UAE@XZ$4 10022f7a f   cProcess.obj
 0001:00021f86       __unwindfunclet$??1cProcess@@UAE@XZ$5 10022f86 f   cProcess.obj
 0001:00021f92       __unwindfunclet$??1cProcess@@UAE@XZ$6 10022f92 f   cProcess.obj
 0001:00021f9e       __unwindfunclet$??1cProcess@@UAE@XZ$7 10022f9e f   cProcess.obj
 0001:00021faa       __ehhandler$??1cProcess@@UAE@XZ 10022faa f   cProcess.obj
 0001:00021fc5       __unwindfunclet$??0dbConnection@@QAE@XZ$0 10022fc5 f   DBCONNECTION.obj
 0001:00021fce       __unwindfunclet$??0dbConnection@@QAE@XZ$1 10022fce f   DBCONNECTION.obj
 0001:00021fda       __unwindfunclet$??0dbConnection@@QAE@XZ$2 10022fda f   DBCONNECTION.obj
 0001:00021fe6       __unwindfunclet$??0dbConnection@@QAE@XZ$3 10022fe6 f   DBCONNECTION.obj
 0001:00021ff2       __unwindfunclet$??0dbConnection@@QAE@XZ$4 10022ff2 f   DBCONNECTION.obj
 0001:00021ffe       __unwindfunclet$??0dbConnection@@QAE@XZ$5 10022ffe f   DBCONNECTION.obj
 0001:0002200a       __unwindfunclet$??0dbConnection@@QAE@XZ$6 1002300a f   DBCONNECTION.obj
 0001:00022016       __unwindfunclet$??0dbConnection@@QAE@XZ$7 10023016 f   DBCONNECTION.obj
 0001:00022022       __unwindfunclet$??0dbConnection@@QAE@XZ$8 10023022 f   DBCONNECTION.obj
 0001:0002202b       __unwindfunclet$??0dbConnection@@QAE@XZ$9 1002302b f   DBCONNECTION.obj
 0001:00022034       __ehhandler$??0dbConnection@@QAE@XZ 10023034 f   DBCONNECTION.obj
 0001:0002204f       __unwindfunclet$??1dbConnection@@UAE@XZ$0 1002304f f   DBCONNECTION.obj
 0001:00022058       __unwindfunclet$??1dbConnection@@UAE@XZ$1 10023058 f   DBCONNECTION.obj
 0001:00022064       __unwindfunclet$??1dbConnection@@UAE@XZ$2 10023064 f   DBCONNECTION.obj
 0001:00022070       __unwindfunclet$??1dbConnection@@UAE@XZ$3 10023070 f   DBCONNECTION.obj
 0001:0002207c       __unwindfunclet$??1dbConnection@@UAE@XZ$4 1002307c f   DBCONNECTION.obj
 0001:00022088       __unwindfunclet$??1dbConnection@@UAE@XZ$5 10023088 f   DBCONNECTION.obj
 0001:00022094       __unwindfunclet$??1dbConnection@@UAE@XZ$6 10023094 f   DBCONNECTION.obj
 0001:000220a0       __ehhandler$??1dbConnection@@UAE@XZ 100230a0 f   DBCONNECTION.obj
 0001:000220bb       __unwindfunclet$?lastError@dbConnection@@QAE?AVQString@@XZ$0 100230bb f   DBCONNECTION.obj
 0001:000220d5       __unwindfunclet$?lastError@dbConnection@@QAE?AVQString@@XZ$1 100230d5 f   DBCONNECTION.obj
 0001:000220de       __unwindfunclet$?lastError@dbConnection@@QAE?AVQString@@XZ$2 100230de f   DBCONNECTION.obj
 0001:000220e7       __unwindfunclet$?lastError@dbConnection@@QAE?AVQString@@XZ$3 100230e7 f   DBCONNECTION.obj
 0001:000220f0       __unwindfunclet$?lastError@dbConnection@@QAE?AVQString@@XZ$4 100230f0 f   DBCONNECTION.obj
 0001:000220f9       __unwindfunclet$?lastError@dbConnection@@QAE?AVQString@@XZ$5 100230f9 f   DBCONNECTION.obj
 0001:00022102       __unwindfunclet$?lastError@dbConnection@@QAE?AVQString@@XZ$6 10023102 f   DBCONNECTION.obj
 0001:0002210b       __unwindfunclet$?lastError@dbConnection@@QAE?AVQString@@XZ$7 1002310b f   DBCONNECTION.obj
 0001:00022114       __unwindfunclet$?lastError@dbConnection@@QAE?AVQString@@XZ$8 10023114 f   DBCONNECTION.obj
 0001:0002211d       __unwindfunclet$?lastError@dbConnection@@QAE?AVQString@@XZ$9 1002311d f   DBCONNECTION.obj
 0001:00022126       __unwindfunclet$?lastError@dbConnection@@QAE?AVQString@@XZ$10 10023126 f   DBCONNECTION.obj
 0001:0002212f       __unwindfunclet$?lastError@dbConnection@@QAE?AVQString@@XZ$11 1002312f f   DBCONNECTION.obj
 0001:00022138       __unwindfunclet$?lastError@dbConnection@@QAE?AVQString@@XZ$12 10023138 f   DBCONNECTION.obj
 0001:00022141       __unwindfunclet$?lastError@dbConnection@@QAE?AVQString@@XZ$13 10023141 f   DBCONNECTION.obj
 0001:0002214a       __unwindfunclet$?lastError@dbConnection@@QAE?AVQString@@XZ$14 1002314a f   DBCONNECTION.obj
 0001:00022153       __ehhandler$?lastError@dbConnection@@QAE?AVQString@@XZ 10023153 f   DBCONNECTION.obj
 0001:0002216e       __unwindfunclet$?run@dbConnection@@UAEXXZ$0 1002316e f   DBCONNECTION.obj
 0001:00022177       __unwindfunclet$?run@dbConnection@@UAEXXZ$1 10023177 f   DBCONNECTION.obj
 0001:00022180       __unwindfunclet$?run@dbConnection@@UAEXXZ$2 10023180 f   DBCONNECTION.obj
 0001:00022189       __unwindfunclet$?run@dbConnection@@UAEXXZ$3 10023189 f   DBCONNECTION.obj
 0001:00022192       __unwindfunclet$?run@dbConnection@@UAEXXZ$4 10023192 f   DBCONNECTION.obj
 0001:0002219b       __unwindfunclet$?run@dbConnection@@UAEXXZ$5 1002319b f   DBCONNECTION.obj
 0001:000221a4       __unwindfunclet$?run@dbConnection@@UAEXXZ$6 100231a4 f   DBCONNECTION.obj
 0001:000221ad       __unwindfunclet$?run@dbConnection@@UAEXXZ$7 100231ad f   DBCONNECTION.obj
 0001:000221b6       __unwindfunclet$?run@dbConnection@@UAEXXZ$8 100231b6 f   DBCONNECTION.obj
 0001:000221bf       __unwindfunclet$?run@dbConnection@@UAEXXZ$9 100231bf f   DBCONNECTION.obj
 0001:000221c8       __unwindfunclet$?run@dbConnection@@UAEXXZ$10 100231c8 f   DBCONNECTION.obj
 0001:000221d1       __ehhandler$?run@dbConnection@@UAEXXZ 100231d1 f   DBCONNECTION.obj
 0001:000221ec       __unwindfunclet$??0dialog@@QAE@PAVIGetDocuments@@PAVQWidget@@PBDI@Z$0 100231ec f   dialogimpl.obj
 0001:000221f4       __unwindfunclet$??0dialog@@QAE@PAVIGetDocuments@@PAVQWidget@@PBDI@Z$1 100231f4 f   dialogimpl.obj
 0001:000221fd       __unwindfunclet$??0dialog@@QAE@PAVIGetDocuments@@PAVQWidget@@PBDI@Z$2 100231fd f   dialogimpl.obj
 0001:00022206       __unwindfunclet$??0dialog@@QAE@PAVIGetDocuments@@PAVQWidget@@PBDI@Z$3 10023206 f   dialogimpl.obj
 0001:0002220f       __unwindfunclet$??0dialog@@QAE@PAVIGetDocuments@@PAVQWidget@@PBDI@Z$4 1002320f f   dialogimpl.obj
 0001:00022218       __unwindfunclet$??0dialog@@QAE@PAVIGetDocuments@@PAVQWidget@@PBDI@Z$5 10023218 f   dialogimpl.obj
 0001:00022221       __unwindfunclet$??0dialog@@QAE@PAVIGetDocuments@@PAVQWidget@@PBDI@Z$6 10023221 f   dialogimpl.obj
 0001:0002222a       __unwindfunclet$??0dialog@@QAE@PAVIGetDocuments@@PAVQWidget@@PBDI@Z$7 1002322a f   dialogimpl.obj
 0001:00022233       __unwindfunclet$??0dialog@@QAE@PAVIGetDocuments@@PAVQWidget@@PBDI@Z$8 10023233 f   dialogimpl.obj
 0001:0002223c       __unwindfunclet$??0dialog@@QAE@PAVIGetDocuments@@PAVQWidget@@PBDI@Z$9 1002323c f   dialogimpl.obj
 0001:00022245       __unwindfunclet$??0dialog@@QAE@PAVIGetDocuments@@PAVQWidget@@PBDI@Z$10 10023245 f   dialogimpl.obj
 0001:0002224e       __unwindfunclet$??0dialog@@QAE@PAVIGetDocuments@@PAVQWidget@@PBDI@Z$11 1002324e f   dialogimpl.obj
 0001:00022257       __unwindfunclet$??0dialog@@QAE@PAVIGetDocuments@@PAVQWidget@@PBDI@Z$12 10023257 f   dialogimpl.obj
 0001:00022260       __unwindfunclet$??0dialog@@QAE@PAVIGetDocuments@@PAVQWidget@@PBDI@Z$13 10023260 f   dialogimpl.obj
 0001:00022269       __unwindfunclet$??0dialog@@QAE@PAVIGetDocuments@@PAVQWidget@@PBDI@Z$14 10023269 f   dialogimpl.obj
 0001:00022272       __unwindfunclet$??0dialog@@QAE@PAVIGetDocuments@@PAVQWidget@@PBDI@Z$15 10023272 f   dialogimpl.obj
 0001:0002227b       __unwindfunclet$??0dialog@@QAE@PAVIGetDocuments@@PAVQWidget@@PBDI@Z$16 1002327b f   dialogimpl.obj
 0001:00022284       __unwindfunclet$??0dialog@@QAE@PAVIGetDocuments@@PAVQWidget@@PBDI@Z$17 10023284 f   dialogimpl.obj
 0001:0002228d       __unwindfunclet$??0dialog@@QAE@PAVIGetDocuments@@PAVQWidget@@PBDI@Z$18 1002328d f   dialogimpl.obj
 0001:00022296       __unwindfunclet$??0dialog@@QAE@PAVIGetDocuments@@PAVQWidget@@PBDI@Z$19 10023296 f   dialogimpl.obj
 0001:0002229f       __unwindfunclet$??0dialog@@QAE@PAVIGetDocuments@@PAVQWidget@@PBDI@Z$20 1002329f f   dialogimpl.obj
 0001:000222a9       __unwindfunclet$??0dialog@@QAE@PAVIGetDocuments@@PAVQWidget@@PBDI@Z$21 100232a9 f   dialogimpl.obj
 0001:000222b3       __unwindfunclet$??0dialog@@QAE@PAVIGetDocuments@@PAVQWidget@@PBDI@Z$22 100232b3 f   dialogimpl.obj
 0001:000222bd       __unwindfunclet$??0dialog@@QAE@PAVIGetDocuments@@PAVQWidget@@PBDI@Z$23 100232bd f   dialogimpl.obj
 0001:000222d7       __unwindfunclet$??0dialog@@QAE@PAVIGetDocuments@@PAVQWidget@@PBDI@Z$24 100232d7 f   dialogimpl.obj
 0001:000222f1       __unwindfunclet$??0dialog@@QAE@PAVIGetDocuments@@PAVQWidget@@PBDI@Z$26 100232f1 f   dialogimpl.obj
 0001:000222fb       __unwindfunclet$??0dialog@@QAE@PAVIGetDocuments@@PAVQWidget@@PBDI@Z$27 100232fb f   dialogimpl.obj
 0001:00022315       __unwindfunclet$??0dialog@@QAE@PAVIGetDocuments@@PAVQWidget@@PBDI@Z$28 10023315 f   dialogimpl.obj
 0001:0002232f       __unwindfunclet$??0dialog@@QAE@PAVIGetDocuments@@PAVQWidget@@PBDI@Z$30 1002332f f   dialogimpl.obj
 0001:00022339       __unwindfunclet$??0dialog@@QAE@PAVIGetDocuments@@PAVQWidget@@PBDI@Z$31 10023339 f   dialogimpl.obj
 0001:00022353       __unwindfunclet$??0dialog@@QAE@PAVIGetDocuments@@PAVQWidget@@PBDI@Z$32 10023353 f   dialogimpl.obj
 0001:0002236d       __unwindfunclet$??0dialog@@QAE@PAVIGetDocuments@@PAVQWidget@@PBDI@Z$33 1002336d f   dialogimpl.obj
 0001:00022387       __unwindfunclet$??0dialog@@QAE@PAVIGetDocuments@@PAVQWidget@@PBDI@Z$34 10023387 f   dialogimpl.obj
 0001:000223a6       __unwindfunclet$??0dialog@@QAE@PAVIGetDocuments@@PAVQWidget@@PBDI@Z$36 100233a6 f   dialogimpl.obj
 0001:000223b0       __unwindfunclet$??0dialog@@QAE@PAVIGetDocuments@@PAVQWidget@@PBDI@Z$37 100233b0 f   dialogimpl.obj
 0001:000223cf       __unwindfunclet$??0dialog@@QAE@PAVIGetDocuments@@PAVQWidget@@PBDI@Z$38 100233cf f   dialogimpl.obj
 0001:000223ee       __unwindfunclet$??0dialog@@QAE@PAVIGetDocuments@@PAVQWidget@@PBDI@Z$39 100233ee f   dialogimpl.obj
 0001:0002240d       __unwindfunclet$??0dialog@@QAE@PAVIGetDocuments@@PAVQWidget@@PBDI@Z$40 1002340d f   dialogimpl.obj
 0001:0002242c       __ehhandler$??0dialog@@QAE@PAVIGetDocuments@@PAVQWidget@@PBDI@Z 1002342c f   dialogimpl.obj
 0001:00022447       __unwindfunclet$??1dialog@@UAE@XZ$0 10023447 f   dialogimpl.obj
 0001:0002244f       __unwindfunclet$??1dialog@@UAE@XZ$1 1002344f f   dialogimpl.obj
 0001:00022458       __unwindfunclet$??1dialog@@UAE@XZ$2 10023458 f   dialogimpl.obj
 0001:00022461       __unwindfunclet$??1dialog@@UAE@XZ$3 10023461 f   dialogimpl.obj
 0001:0002246a       __unwindfunclet$??1dialog@@UAE@XZ$4 1002346a f   dialogimpl.obj
 0001:00022473       __unwindfunclet$??1dialog@@UAE@XZ$5 10023473 f   dialogimpl.obj
 0001:0002247c       __unwindfunclet$??1dialog@@UAE@XZ$6 1002347c f   dialogimpl.obj
 0001:00022485       __unwindfunclet$??1dialog@@UAE@XZ$7 10023485 f   dialogimpl.obj
 0001:0002248e       __unwindfunclet$??1dialog@@UAE@XZ$8 1002348e f   dialogimpl.obj
 0001:00022497       __unwindfunclet$??1dialog@@UAE@XZ$9 10023497 f   dialogimpl.obj
 0001:000224a0       __unwindfunclet$??1dialog@@UAE@XZ$10 100234a0 f   dialogimpl.obj
 0001:000224a9       __unwindfunclet$??1dialog@@UAE@XZ$11 100234a9 f   dialogimpl.obj
 0001:000224b2       __unwindfunclet$??1dialog@@UAE@XZ$12 100234b2 f   dialogimpl.obj
 0001:000224bb       __unwindfunclet$??1dialog@@UAE@XZ$13 100234bb f   dialogimpl.obj
 0001:000224c4       __unwindfunclet$??1dialog@@UAE@XZ$14 100234c4 f   dialogimpl.obj
 0001:000224cd       __unwindfunclet$??1dialog@@UAE@XZ$15 100234cd f   dialogimpl.obj
 0001:000224d6       __unwindfunclet$??1dialog@@UAE@XZ$16 100234d6 f   dialogimpl.obj
 0001:000224df       __unwindfunclet$??1dialog@@UAE@XZ$17 100234df f   dialogimpl.obj
 0001:000224e8       __unwindfunclet$??1dialog@@UAE@XZ$18 100234e8 f   dialogimpl.obj
 0001:000224f1       __unwindfunclet$??1dialog@@UAE@XZ$19 100234f1 f   dialogimpl.obj
 0001:000224fa       __unwindfunclet$??1dialog@@UAE@XZ$20 100234fa f   dialogimpl.obj
 0001:00022503       __unwindfunclet$??1dialog@@UAE@XZ$21 10023503 f   dialogimpl.obj
 0001:0002250c       __unwindfunclet$??1dialog@@UAE@XZ$22 1002350c f   dialogimpl.obj
 0001:00022515       __unwindfunclet$??1dialog@@UAE@XZ$23 10023515 f   dialogimpl.obj
 0001:0002251e       __unwindfunclet$??1dialog@@UAE@XZ$24 1002351e f   dialogimpl.obj
 0001:00022527       __unwindfunclet$??1dialog@@UAE@XZ$25 10023527 f   dialogimpl.obj
 0001:00022530       __unwindfunclet$??1dialog@@UAE@XZ$26 10023530 f   dialogimpl.obj
 0001:00022539       __unwindfunclet$??1dialog@@UAE@XZ$27 10023539 f   dialogimpl.obj
 0001:00022542       __unwindfunclet$??1dialog@@UAE@XZ$28 10023542 f   dialogimpl.obj
 0001:0002254b       __unwindfunclet$??1dialog@@UAE@XZ$29 1002354b f   dialogimpl.obj
 0001:00022554       __unwindfunclet$??1dialog@@UAE@XZ$30 10023554 f   dialogimpl.obj
 0001:0002255d       __unwindfunclet$??1dialog@@UAE@XZ$31 1002355d f   dialogimpl.obj
 0001:00022566       __unwindfunclet$??1dialog@@UAE@XZ$32 10023566 f   dialogimpl.obj
 0001:0002256f       __unwindfunclet$??1dialog@@UAE@XZ$33 1002356f f   dialogimpl.obj
 0001:00022578       __unwindfunclet$??1dialog@@UAE@XZ$34 10023578 f   dialogimpl.obj
 0001:00022581       __unwindfunclet$??1dialog@@UAE@XZ$35 10023581 f   dialogimpl.obj
 0001:0002258a       __unwindfunclet$??1dialog@@UAE@XZ$36 1002358a f   dialogimpl.obj
 0001:00022593       __unwindfunclet$??1dialog@@UAE@XZ$37 10023593 f   dialogimpl.obj
 0001:0002259c       __unwindfunclet$??1dialog@@UAE@XZ$38 1002359c f   dialogimpl.obj
 0001:000225a5       __unwindfunclet$??1dialog@@UAE@XZ$39 100235a5 f   dialogimpl.obj
 0001:000225ae       __unwindfunclet$??1dialog@@UAE@XZ$40 100235ae f   dialogimpl.obj
 0001:000225b7       __unwindfunclet$??1dialog@@UAE@XZ$41 100235b7 f   dialogimpl.obj
 0001:000225c0       __ehhandler$??1dialog@@UAE@XZ 100235c0 f   dialogimpl.obj
 0001:000225db       __unwindfunclet$?clearAllProcesses@dialog@@QAEXXZ$0 100235db f   dialogimpl.obj
 0001:000225db       __unwindfunclet$?clearAllLogs@dialog@@QAEXXZ$0 100235db f   dialogimpl.obj
 0001:000225e4       __unwindfunclet$?clearAllLogs@dialog@@QAEXXZ$1 100235e4 f   dialogimpl.obj
 0001:000225e4       __unwindfunclet$?clearAllProcesses@dialog@@QAEXXZ$1 100235e4 f   dialogimpl.obj
 0001:000225ed       __unwindfunclet$?clearAllProcesses@dialog@@QAEXXZ$2 100235ed f   dialogimpl.obj
 0001:000225ed       __unwindfunclet$?clearAllLogs@dialog@@QAEXXZ$2 100235ed f   dialogimpl.obj
 0001:000225f6       __ehhandler$?clearAllLogs@dialog@@QAEXXZ 100235f6 f   dialogimpl.obj
 0001:000225f6       __ehhandler$?clearAllProcesses@dialog@@QAEXXZ 100235f6 f   dialogimpl.obj
 0001:00022611       __unwindfunclet$?clearAllText@dialog@@QAEXXZ$0 10023611 f   dialogimpl.obj
 0001:0002261a       __unwindfunclet$?clearAllText@dialog@@QAEXXZ$1 1002361a f   dialogimpl.obj
 0001:00022623       __unwindfunclet$?clearAllText@dialog@@QAEXXZ$2 10023623 f   dialogimpl.obj
 0001:0002262c       __unwindfunclet$?clearAllText@dialog@@QAEXXZ$3 1002362c f   dialogimpl.obj
 0001:00022635       __unwindfunclet$?clearAllText@dialog@@QAEXXZ$4 10023635 f   dialogimpl.obj
 0001:0002263e       __unwindfunclet$?clearAllText@dialog@@QAEXXZ$5 1002363e f   dialogimpl.obj
 0001:00022647       __unwindfunclet$?clearAllText@dialog@@QAEXXZ$6 10023647 f   dialogimpl.obj
 0001:00022650       __ehhandler$?clearAllText@dialog@@QAEXXZ 10023650 f   dialogimpl.obj
 0001:0002266b       __unwindfunclet$?clearProcessesBefore@dialog@@QAEXXZ$0 1002366b f   dialogimpl.obj
 0001:0002266b       __unwindfunclet$?clearLogsBefore@dialog@@QAEXXZ$0 1002366b f   dialogimpl.obj
 0001:00022674       __unwindfunclet$?clearLogsBefore@dialog@@QAEXXZ$1 10023674 f   dialogimpl.obj
 0001:00022674       __unwindfunclet$?clearProcessesBefore@dialog@@QAEXXZ$1 10023674 f   dialogimpl.obj
 0001:0002267d       __unwindfunclet$?clearProcessesBefore@dialog@@QAEXXZ$2 1002367d f   dialogimpl.obj
 0001:0002267d       __unwindfunclet$?clearLogsBefore@dialog@@QAEXXZ$2 1002367d f   dialogimpl.obj
 0001:00022686       __unwindfunclet$?clearLogsBefore@dialog@@QAEXXZ$3 10023686 f   dialogimpl.obj
 0001:00022686       __unwindfunclet$?clearProcessesBefore@dialog@@QAEXXZ$3 10023686 f   dialogimpl.obj
 0001:0002268f       __unwindfunclet$?clearLogsBefore@dialog@@QAEXXZ$4 1002368f f   dialogimpl.obj
 0001:0002268f       __unwindfunclet$?clearProcessesBefore@dialog@@QAEXXZ$4 1002368f f   dialogimpl.obj
 0001:00022698       __ehhandler$?clearLogsBefore@dialog@@QAEXXZ 10023698 f   dialogimpl.obj
 0001:00022698       __ehhandler$?clearProcessesBefore@dialog@@QAEXXZ 10023698 f   dialogimpl.obj
 0001:000226b3       __unwindfunclet$?connectDb@dialog@@AAEPAVQSqlDatabase@@XZ$0 100236b3 f   dialogimpl.obj
 0001:000226bc       __unwindfunclet$?connectDb@dialog@@AAEPAVQSqlDatabase@@XZ$1 100236bc f   dialogimpl.obj
 0001:000226c5       __unwindfunclet$?connectDb@dialog@@AAEPAVQSqlDatabase@@XZ$2 100236c5 f   dialogimpl.obj
 0001:000226ce       __unwindfunclet$?connectDb@dialog@@AAEPAVQSqlDatabase@@XZ$3 100236ce f   dialogimpl.obj
 0001:000226d7       __ehhandler$?connectDb@dialog@@AAEPAVQSqlDatabase@@XZ 100236d7 f   dialogimpl.obj
 0001:000226f2       __unwindfunclet$?copyData@dialog@@QAEXXZ$0 100236f2 f   dialogimpl.obj
 0001:000226fb       __unwindfunclet$?copyData@dialog@@QAEXXZ$1 100236fb f   dialogimpl.obj
 0001:00022704       __unwindfunclet$?copyData@dialog@@QAEXXZ$2 10023704 f   dialogimpl.obj
 0001:0002270d       __ehhandler$?copyData@dialog@@QAEXXZ 1002370d f   dialogimpl.obj
 0001:00022728       __unwindfunclet$?createNewLogTable@dialog@@QAEXXZ$0 10023728 f   dialogimpl.obj
 0001:00022731       __unwindfunclet$?createNewLogTable@dialog@@QAEXXZ$1 10023731 f   dialogimpl.obj
 0001:0002273a       __unwindfunclet$?createNewLogTable@dialog@@QAEXXZ$2 1002373a f   dialogimpl.obj
 0001:00022743       __unwindfunclet$?createNewLogTable@dialog@@QAEXXZ$3 10023743 f   dialogimpl.obj
 0001:0002274c       __unwindfunclet$?createNewLogTable@dialog@@QAEXXZ$4 1002374c f   dialogimpl.obj
 0001:00022755       __unwindfunclet$?createNewLogTable@dialog@@QAEXXZ$5 10023755 f   dialogimpl.obj
 0001:0002275e       __unwindfunclet$?createNewLogTable@dialog@@QAEXXZ$6 1002375e f   dialogimpl.obj
 0001:00022767       __unwindfunclet$?createNewLogTable@dialog@@QAEXXZ$7 10023767 f   dialogimpl.obj
 0001:00022770       __unwindfunclet$?createNewLogTable@dialog@@QAEXXZ$8 10023770 f   dialogimpl.obj
 0001:00022779       __unwindfunclet$?createNewLogTable@dialog@@QAEXXZ$9 10023779 f   dialogimpl.obj
 0001:00022782       __unwindfunclet$?createNewLogTable@dialog@@QAEXXZ$10 10023782 f   dialogimpl.obj
 0001:0002278b       __unwindfunclet$?createNewLogTable@dialog@@QAEXXZ$11 1002378b f   dialogimpl.obj
 0001:00022794       __unwindfunclet$?createNewLogTable@dialog@@QAEXXZ$12 10023794 f   dialogimpl.obj
 0001:0002279d       __unwindfunclet$?createNewLogTable@dialog@@QAEXXZ$13 1002379d f   dialogimpl.obj
 0001:000227a6       __unwindfunclet$?createNewLogTable@dialog@@QAEXXZ$14 100237a6 f   dialogimpl.obj
 0001:000227af       __unwindfunclet$?createNewLogTable@dialog@@QAEXXZ$15 100237af f   dialogimpl.obj
 0001:000227b8       __unwindfunclet$?createNewLogTable@dialog@@QAEXXZ$16 100237b8 f   dialogimpl.obj
 0001:000227c1       __unwindfunclet$?createNewLogTable@dialog@@QAEXXZ$17 100237c1 f   dialogimpl.obj
 0001:000227ca       __unwindfunclet$?createNewLogTable@dialog@@QAEXXZ$18 100237ca f   dialogimpl.obj
 0001:000227d3       __unwindfunclet$?createNewLogTable@dialog@@QAEXXZ$19 100237d3 f   dialogimpl.obj
 0001:000227dc       __unwindfunclet$?createNewLogTable@dialog@@QAEXXZ$20 100237dc f   dialogimpl.obj
 0001:000227e5       __unwindfunclet$?createNewLogTable@dialog@@QAEXXZ$21 100237e5 f   dialogimpl.obj
 0001:000227ee       __unwindfunclet$?createNewLogTable@dialog@@QAEXXZ$22 100237ee f   dialogimpl.obj
 0001:000227f7       __unwindfunclet$?createNewLogTable@dialog@@QAEXXZ$23 100237f7 f   dialogimpl.obj
 0001:00022800       __unwindfunclet$?createNewLogTable@dialog@@QAEXXZ$24 10023800 f   dialogimpl.obj
 0001:00022809       __unwindfunclet$?createNewLogTable@dialog@@QAEXXZ$25 10023809 f   dialogimpl.obj
 0001:00022812       __unwindfunclet$?createNewLogTable@dialog@@QAEXXZ$26 10023812 f   dialogimpl.obj
 0001:0002281b       __ehhandler$?createNewLogTable@dialog@@QAEXXZ 1002381b f   dialogimpl.obj
 0001:00022836       __unwindfunclet$?createNewProcTable@dialog@@QAEXXZ$0 10023836 f   dialogimpl.obj
 0001:0002283f       __unwindfunclet$?createNewProcTable@dialog@@QAEXXZ$1 1002383f f   dialogimpl.obj
 0001:00022848       __unwindfunclet$?createNewProcTable@dialog@@QAEXXZ$2 10023848 f   dialogimpl.obj
 0001:00022851       __unwindfunclet$?createNewProcTable@dialog@@QAEXXZ$3 10023851 f   dialogimpl.obj
 0001:0002285a       __unwindfunclet$?createNewProcTable@dialog@@QAEXXZ$4 1002385a f   dialogimpl.obj
 0001:00022863       __unwindfunclet$?createNewProcTable@dialog@@QAEXXZ$5 10023863 f   dialogimpl.obj
 0001:0002286c       __unwindfunclet$?createNewProcTable@dialog@@QAEXXZ$6 1002386c f   dialogimpl.obj
 0001:00022875       __unwindfunclet$?createNewProcTable@dialog@@QAEXXZ$7 10023875 f   dialogimpl.obj
 0001:0002287e       __unwindfunclet$?createNewProcTable@dialog@@QAEXXZ$8 1002387e f   dialogimpl.obj
 0001:00022887       __unwindfunclet$?createNewProcTable@dialog@@QAEXXZ$9 10023887 f   dialogimpl.obj
 0001:00022890       __unwindfunclet$?createNewProcTable@dialog@@QAEXXZ$10 10023890 f   dialogimpl.obj
 0001:00022899       __unwindfunclet$?createNewProcTable@dialog@@QAEXXZ$11 10023899 f   dialogimpl.obj
 0001:000228a2       __unwindfunclet$?createNewProcTable@dialog@@QAEXXZ$12 100238a2 f   dialogimpl.obj
 0001:000228ab       __unwindfunclet$?createNewProcTable@dialog@@QAEXXZ$13 100238ab f   dialogimpl.obj
 0001:000228b4       __unwindfunclet$?createNewProcTable@dialog@@QAEXXZ$14 100238b4 f   dialogimpl.obj
 0001:000228bd       __unwindfunclet$?createNewProcTable@dialog@@QAEXXZ$15 100238bd f   dialogimpl.obj
 0001:000228c6       __unwindfunclet$?createNewProcTable@dialog@@QAEXXZ$16 100238c6 f   dialogimpl.obj
 0001:000228cf       __unwindfunclet$?createNewProcTable@dialog@@QAEXXZ$17 100238cf f   dialogimpl.obj
 0001:000228d8       __unwindfunclet$?createNewProcTable@dialog@@QAEXXZ$18 100238d8 f   dialogimpl.obj
 0001:000228e1       __unwindfunclet$?createNewProcTable@dialog@@QAEXXZ$19 100238e1 f   dialogimpl.obj
 0001:000228ea       __unwindfunclet$?createNewProcTable@dialog@@QAEXXZ$20 100238ea f   dialogimpl.obj
 0001:000228f3       __unwindfunclet$?createNewProcTable@dialog@@QAEXXZ$21 100238f3 f   dialogimpl.obj
 0001:000228fc       __unwindfunclet$?createNewProcTable@dialog@@QAEXXZ$22 100238fc f   dialogimpl.obj
 0001:00022905       __unwindfunclet$?createNewProcTable@dialog@@QAEXXZ$23 10023905 f   dialogimpl.obj
 0001:0002290e       __unwindfunclet$?createNewProcTable@dialog@@QAEXXZ$24 1002390e f   dialogimpl.obj
 0001:00022917       __ehhandler$?createNewProcTable@dialog@@QAEXXZ 10023917 f   dialogimpl.obj
 0001:00022932       __unwindfunclet$?dbDriverChanged@dialog@@QAEXABVQString@@@Z$0 10023932 f   dialogimpl.obj
 0001:00022932       __unwindfunclet$?dbDriverChanged_reserve@dialog@@QAEXABVQString@@@Z$0 10023932 f   dialogimpl.obj
 0001:0002293b       __unwindfunclet$?dbDriverChanged@dialog@@QAEXABVQString@@@Z$1 1002393b f   dialogimpl.obj
 0001:0002293b       __unwindfunclet$?dbDriverChanged_reserve@dialog@@QAEXABVQString@@@Z$1 1002393b f   dialogimpl.obj
 0001:00022944       __ehhandler$?dbDriverChanged_reserve@dialog@@QAEXABVQString@@@Z 10023944 f   dialogimpl.obj
 0001:00022944       __ehhandler$?dbDriverChanged@dialog@@QAEXABVQString@@@Z 10023944 f   dialogimpl.obj
 0001:0002295f       __unwindfunclet$?dbEditStart@dialog@@QAEXXZ$0 1002395f f   dialogimpl.obj
 0001:00022968       __unwindfunclet$?dbEditStart@dialog@@QAEXXZ$1 10023968 f   dialogimpl.obj
 0001:00022971       __unwindfunclet$?dbEditStart@dialog@@QAEXXZ$2 10023971 f   dialogimpl.obj
 0001:0002297a       __unwindfunclet$?dbEditStart@dialog@@QAEXXZ$3 1002397a f   dialogimpl.obj
 0001:00022983       __unwindfunclet$?dbEditStart@dialog@@QAEXXZ$4 10023983 f   dialogimpl.obj
 0001:0002298c       __ehhandler$?dbEditStart@dialog@@QAEXXZ 1002398c f   dialogimpl.obj
 0001:000229a7       __unwindfunclet$?dbStartConnect@dialog@@AAEXXZ$0 100239a7 f   dialogimpl.obj
 0001:000229b1       __unwindfunclet$?dbStartConnect@dialog@@AAEXXZ$1 100239b1 f   dialogimpl.obj
 0001:000229ba       __unwindfunclet$?dbStartConnect@dialog@@AAEXXZ$2 100239ba f   dialogimpl.obj
 0001:000229c3       __unwindfunclet$?dbStartConnect@dialog@@AAEXXZ$3 100239c3 f   dialogimpl.obj
 0001:000229cc       __unwindfunclet$?dbStartConnect@dialog@@AAEXXZ$4 100239cc f   dialogimpl.obj
 0001:000229d5       __unwindfunclet$?dbStartConnect@dialog@@AAEXXZ$5 100239d5 f   dialogimpl.obj
 0001:000229de       __unwindfunclet$?dbStartConnect@dialog@@AAEXXZ$6 100239de f   dialogimpl.obj
 0001:000229e7       __unwindfunclet$?dbStartConnect@dialog@@AAEXXZ$7 100239e7 f   dialogimpl.obj
 0001:000229f0       __unwindfunclet$?dbStartConnect@dialog@@AAEXXZ$8 100239f0 f   dialogimpl.obj
 0001:000229f9       __unwindfunclet$?dbStartConnect@dialog@@AAEXXZ$9 100239f9 f   dialogimpl.obj
 0001:00022a02       __unwindfunclet$?dbStartConnect@dialog@@AAEXXZ$10 10023a02 f   dialogimpl.obj
 0001:00022a0b       __unwindfunclet$?dbStartConnect@dialog@@AAEXXZ$11 10023a0b f   dialogimpl.obj
 0001:00022a14       __unwindfunclet$?dbStartConnect@dialog@@AAEXXZ$12 10023a14 f   dialogimpl.obj
 0001:00022a1d       __ehhandler$?dbStartConnect@dialog@@AAEXXZ 10023a1d f   dialogimpl.obj
 0001:00022a38       __unwindfunclet$?dbToolUpdate@dialog@@QAEXXZ$0 10023a38 f   dialogimpl.obj
 0001:00022a41       __unwindfunclet$?dbToolUpdate@dialog@@QAEXXZ$1 10023a41 f   dialogimpl.obj
 0001:00022a4a       __unwindfunclet$?dbToolUpdate@dialog@@QAEXXZ$2 10023a4a f   dialogimpl.obj
 0001:00022a53       __unwindfunclet$?dbToolUpdate@dialog@@QAEXXZ$3 10023a53 f   dialogimpl.obj
 0001:00022a5c       __unwindfunclet$?dbToolUpdate@dialog@@QAEXXZ$4 10023a5c f   dialogimpl.obj
 0001:00022a65       __unwindfunclet$?dbToolUpdate@dialog@@QAEXXZ$5 10023a65 f   dialogimpl.obj
 0001:00022a6e       __unwindfunclet$?dbToolUpdate@dialog@@QAEXXZ$6 10023a6e f   dialogimpl.obj
 0001:00022a77       __unwindfunclet$?dbToolUpdate@dialog@@QAEXXZ$7 10023a77 f   dialogimpl.obj
 0001:00022a80       __unwindfunclet$?dbToolUpdate@dialog@@QAEXXZ$8 10023a80 f   dialogimpl.obj
 0001:00022a89       __unwindfunclet$?dbToolUpdate@dialog@@QAEXXZ$9 10023a89 f   dialogimpl.obj
 0001:00022a92       __unwindfunclet$?dbToolUpdate@dialog@@QAEXXZ$10 10023a92 f   dialogimpl.obj
 0001:00022a9b       __unwindfunclet$?dbToolUpdate@dialog@@QAEXXZ$11 10023a9b f   dialogimpl.obj
 0001:00022aa4       __unwindfunclet$?dbToolUpdate@dialog@@QAEXXZ$12 10023aa4 f   dialogimpl.obj
 0001:00022aad       __ehhandler$?dbToolUpdate@dialog@@QAEXXZ 10023aad f   dialogimpl.obj
 0001:00022ac8       __unwindfunclet$?dbToolsStart@dialog@@QAEXXZ$0 10023ac8 f   dialogimpl.obj
 0001:00022ad1       __unwindfunclet$?dbToolsStart@dialog@@QAEXXZ$1 10023ad1 f   dialogimpl.obj
 0001:00022ada       __unwindfunclet$?dbToolsStart@dialog@@QAEXXZ$2 10023ada f   dialogimpl.obj
 0001:00022ae3       __ehhandler$?dbToolsStart@dialog@@QAEXXZ 10023ae3 f   dialogimpl.obj
 0001:00022afe       __unwindfunclet$?defaultText@dialog@@AAE?AVQString@@W4AlarmStates@Alarms@@@Z$0 10023afe f   dialogimpl.obj
 0001:00022b18       __unwindfunclet$?defaultText@dialog@@AAE?AVQString@@W4AlarmStates@Alarms@@@Z$1 10023b18 f   dialogimpl.obj
 0001:00022b32       __unwindfunclet$?defaultText@dialog@@AAE?AVQString@@W4AlarmStates@Alarms@@@Z$2 10023b32 f   dialogimpl.obj
 0001:00022b3b       __unwindfunclet$?defaultText@dialog@@AAE?AVQString@@W4AlarmStates@Alarms@@@Z$3 10023b3b f   dialogimpl.obj
 0001:00022b44       __unwindfunclet$?defaultText@dialog@@AAE?AVQString@@W4AlarmStates@Alarms@@@Z$4 10023b44 f   dialogimpl.obj
 0001:00022b4d       __unwindfunclet$?defaultText@dialog@@AAE?AVQString@@W4AlarmStates@Alarms@@@Z$10 10023b4d f   dialogimpl.obj
 0001:00022b56       __unwindfunclet$?defaultText@dialog@@AAE?AVQString@@W4AlarmStates@Alarms@@@Z$9 10023b56 f   dialogimpl.obj
 0001:00022b5f       __unwindfunclet$?defaultText@dialog@@AAE?AVQString@@W4AlarmStates@Alarms@@@Z$8 10023b5f f   dialogimpl.obj
 0001:00022b68       __unwindfunclet$?defaultText@dialog@@AAE?AVQString@@W4AlarmStates@Alarms@@@Z$7 10023b68 f   dialogimpl.obj
 0001:00022b71       __unwindfunclet$?defaultText@dialog@@AAE?AVQString@@W4AlarmStates@Alarms@@@Z$6 10023b71 f   dialogimpl.obj
 0001:00022b7a       __unwindfunclet$?defaultText@dialog@@AAE?AVQString@@W4AlarmStates@Alarms@@@Z$5 10023b7a f   dialogimpl.obj
 0001:00022b83       __unwindfunclet$?defaultText@dialog@@AAE?AVQString@@W4AlarmStates@Alarms@@@Z$11 10023b83 f   dialogimpl.obj
 0001:00022b8c       __unwindfunclet$?defaultText@dialog@@AAE?AVQString@@W4AlarmStates@Alarms@@@Z$13 10023b8c f   dialogimpl.obj
 0001:00022ba6       __ehhandler$?defaultText@dialog@@AAE?AVQString@@W4AlarmStates@Alarms@@@Z 10023ba6 f   dialogimpl.obj
 0001:00022bc1       __unwindfunclet$?fillDataTable@dialog@@QAEXXZ$0 10023bc1 f   dialogimpl.obj
 0001:00022bca       __unwindfunclet$?fillDataTable@dialog@@QAEXXZ$1 10023bca f   dialogimpl.obj
 0001:00022bd4       __ehhandler$?fillDataTable@dialog@@QAEXXZ 10023bd4 f   dialogimpl.obj
 0001:00022bef       __unwindfunclet$?getSep@dialog@@QAE?AVQString@@H@Z$0 10023bef f   dialogimpl.obj
 0001:00022c09       __unwindfunclet$?getSep@dialog@@QAE?AVQString@@H@Z$1 10023c09 f   dialogimpl.obj
 0001:00022c12       __unwindfunclet$?getSep@dialog@@QAE?AVQString@@H@Z$2 10023c12 f   dialogimpl.obj
 0001:00022c1b       __unwindfunclet$?getSep@dialog@@QAE?AVQString@@H@Z$3 10023c1b f   dialogimpl.obj
 0001:00022c24       __unwindfunclet$?getSep@dialog@@QAE?AVQString@@H@Z$4 10023c24 f   dialogimpl.obj
 0001:00022c2d       __unwindfunclet$?getSep@dialog@@QAE?AVQString@@H@Z$5 10023c2d f   dialogimpl.obj
 0001:00022c36       __ehhandler$?getSep@dialog@@QAE?AVQString@@H@Z 10023c36 f   dialogimpl.obj
 0001:00022c51       __unwindfunclet$?itemChanged@dialog@@QAEXABVQString@@@Z$0 10023c51 f   dialogimpl.obj
 0001:00022c5a       __unwindfunclet$?itemChanged@dialog@@QAEXABVQString@@@Z$1 10023c5a f   dialogimpl.obj
 0001:00022c63       __unwindfunclet$?itemChanged@dialog@@QAEXABVQString@@@Z$2 10023c63 f   dialogimpl.obj
 0001:00022c6c       __unwindfunclet$?itemChanged@dialog@@QAEXABVQString@@@Z$3 10023c6c f   dialogimpl.obj
 0001:00022c75       __unwindfunclet$?itemChanged@dialog@@QAEXABVQString@@@Z$4 10023c75 f   dialogimpl.obj
 0001:00022c7e       __unwindfunclet$?itemChanged@dialog@@QAEXABVQString@@@Z$5 10023c7e f   dialogimpl.obj
 0001:00022c87       __unwindfunclet$?itemChanged@dialog@@QAEXABVQString@@@Z$6 10023c87 f   dialogimpl.obj
 0001:00022c90       __unwindfunclet$?itemChanged@dialog@@QAEXABVQString@@@Z$7 10023c90 f   dialogimpl.obj
 0001:00022c99       __ehhandler$?itemChanged@dialog@@QAEXABVQString@@@Z 10023c99 f   dialogimpl.obj
 0001:00022cb4       __unwindfunclet$?pasteData@dialog@@QAEXXZ$0 10023cb4 f   dialogimpl.obj
 0001:00022cbd       __unwindfunclet$?pasteData@dialog@@QAEXXZ$1 10023cbd f   dialogimpl.obj
 0001:00022cc6       __unwindfunclet$?pasteData@dialog@@QAEXXZ$2 10023cc6 f   dialogimpl.obj
 0001:00022ccf       __unwindfunclet$?pasteData@dialog@@QAEXXZ$3 10023ccf f   dialogimpl.obj
 0001:00022cd8       __unwindfunclet$?pasteData@dialog@@QAEXXZ$4 10023cd8 f   dialogimpl.obj
 0001:00022ce1       __unwindfunclet$?pasteData@dialog@@QAEXXZ$5 10023ce1 f   dialogimpl.obj
 0001:00022cea       __unwindfunclet$?pasteData@dialog@@QAEXXZ$6 10023cea f   dialogimpl.obj
 0001:00022cf3       __unwindfunclet$?pasteData@dialog@@QAEXXZ$7 10023cf3 f   dialogimpl.obj
 0001:00022cfc       __unwindfunclet$?pasteData@dialog@@QAEXXZ$8 10023cfc f   dialogimpl.obj
 0001:00022d05       __unwindfunclet$?pasteData@dialog@@QAEXXZ$9 10023d05 f   dialogimpl.obj
 0001:00022d0e       __unwindfunclet$?pasteData@dialog@@QAEXXZ$10 10023d0e f   dialogimpl.obj
 0001:00022d17       __unwindfunclet$?pasteData@dialog@@QAEXXZ$11 10023d17 f   dialogimpl.obj
 0001:00022d20       __unwindfunclet$?pasteData@dialog@@QAEXXZ$12 10023d20 f   dialogimpl.obj
 0001:00022d29       __unwindfunclet$?pasteData@dialog@@QAEXXZ$13 10023d29 f   dialogimpl.obj
 0001:00022d32       __unwindfunclet$?pasteData@dialog@@QAEXXZ$14 10023d32 f   dialogimpl.obj
 0001:00022d3b       __ehhandler$?pasteData@dialog@@QAEXXZ 10023d3b f   dialogimpl.obj
 0001:00022d56       __unwindfunclet$?saveProcess@dialog@@QAE_NPAVcProcess@@@Z$0 10023d56 f   dialogimpl.obj
 0001:00022d5f       __unwindfunclet$?saveProcess@dialog@@QAE_NPAVcProcess@@@Z$1 10023d5f f   dialogimpl.obj
 0001:00022d68       __unwindfunclet$?saveProcess@dialog@@QAE_NPAVcProcess@@@Z$2 10023d68 f   dialogimpl.obj
 0001:00022d71       __unwindfunclet$?saveProcess@dialog@@QAE_NPAVcProcess@@@Z$3 10023d71 f   dialogimpl.obj
 0001:00022d7a       __unwindfunclet$?saveProcess@dialog@@QAE_NPAVcProcess@@@Z$4 10023d7a f   dialogimpl.obj
 0001:00022d83       __unwindfunclet$?saveProcess@dialog@@QAE_NPAVcProcess@@@Z$5 10023d83 f   dialogimpl.obj
 0001:00022d8c       __unwindfunclet$?saveProcess@dialog@@QAE_NPAVcProcess@@@Z$6 10023d8c f   dialogimpl.obj
 0001:00022d95       __unwindfunclet$?saveProcess@dialog@@QAE_NPAVcProcess@@@Z$7 10023d95 f   dialogimpl.obj
 0001:00022d9e       __ehhandler$?saveProcess@dialog@@QAE_NPAVcProcess@@@Z 10023d9e f   dialogimpl.obj
 0001:00022db9       __unwindfunclet$?setOkDefaultText@dialog@@QAEXXZ$0 10023db9 f   dialogimpl.obj
 0001:00022db9       __unwindfunclet$?setLatchedDefaultText@dialog@@QAEXXZ$0 10023db9 f   dialogimpl.obj
 0001:00022db9       __unwindfunclet$?setFailDefaultText@dialog@@QAEXXZ$0 10023db9 f   dialogimpl.obj
 0001:00022db9       __unwindfunclet$?setIgnoreDefaultText@dialog@@QAEXXZ$0 10023db9 f   dialogimpl.obj
 0001:00022db9       __unwindfunclet$?setAckDefaultText@dialog@@QAEXXZ$0 10023db9 f   dialogimpl.obj
 0001:00022db9       __unwindfunclet$?setUnknownDefaultText@dialog@@QAEXXZ$0 10023db9 f   dialogimpl.obj
 0001:00022dc2       __unwindfunclet$?setIgnoreDefaultText@dialog@@QAEXXZ$1 10023dc2 f   dialogimpl.obj
 0001:00022dc2       __unwindfunclet$?setOkDefaultText@dialog@@QAEXXZ$1 10023dc2 f   dialogimpl.obj
 0001:00022dc2       __unwindfunclet$?setLatchedDefaultText@dialog@@QAEXXZ$1 10023dc2 f   dialogimpl.obj
 0001:00022dc2       __unwindfunclet$?setUnknownDefaultText@dialog@@QAEXXZ$1 10023dc2 f   dialogimpl.obj
 0001:00022dc2       __unwindfunclet$?setFailDefaultText@dialog@@QAEXXZ$1 10023dc2 f   dialogimpl.obj
 0001:00022dc2       __unwindfunclet$?setAckDefaultText@dialog@@QAEXXZ$1 10023dc2 f   dialogimpl.obj
 0001:00022dcb       __ehhandler$?setLatchedDefaultText@dialog@@QAEXXZ 10023dcb f   dialogimpl.obj
 0001:00022dcb       __ehhandler$?setFailDefaultText@dialog@@QAEXXZ 10023dcb f   dialogimpl.obj
 0001:00022dcb       __ehhandler$?setOkDefaultText@dialog@@QAEXXZ 10023dcb f   dialogimpl.obj
 0001:00022dcb       __ehhandler$?setIgnoreDefaultText@dialog@@QAEXXZ 10023dcb f   dialogimpl.obj
 0001:00022dcb       __ehhandler$?setUnknownDefaultText@dialog@@QAEXXZ 10023dcb f   dialogimpl.obj
 0001:00022dcb       __ehhandler$?setAckDefaultText@dialog@@QAEXXZ 10023dcb f   dialogimpl.obj
 0001:00022de6       __unwindfunclet$?setAllDefaultText@dialog@@QAEXXZ$0 10023de6 f   dialogimpl.obj
 0001:00022def       __unwindfunclet$?setAllDefaultText@dialog@@QAEXXZ$1 10023def f   dialogimpl.obj
 0001:00022df8       __unwindfunclet$?setAllDefaultText@dialog@@QAEXXZ$2 10023df8 f   dialogimpl.obj
 0001:00022e01       __unwindfunclet$?setAllDefaultText@dialog@@QAEXXZ$3 10023e01 f   dialogimpl.obj
 0001:00022e0a       __unwindfunclet$?setAllDefaultText@dialog@@QAEXXZ$4 10023e0a f   dialogimpl.obj
 0001:00022e13       __unwindfunclet$?setAllDefaultText@dialog@@QAEXXZ$5 10023e13 f   dialogimpl.obj
 0001:00022e1c       __unwindfunclet$?setAllDefaultText@dialog@@QAEXXZ$6 10023e1c f   dialogimpl.obj
 0001:00022e25       __ehhandler$?setAllDefaultText@dialog@@QAEXXZ 10023e25 f   dialogimpl.obj
 0001:00022e40       __unwindfunclet$?procSelection@alm_db_output@@AAEXXZ$0 10023e40 f   dialogimpl.obj
 0001:00022e40       __unwindfunclet$?setGroupDefaultText@dialog@@QAEXXZ$0 10023e40 f   dialogimpl.obj
 0001:00022e49       __unwindfunclet$?setGroupDefaultText@dialog@@QAEXXZ$1 10023e49 f   dialogimpl.obj
 0001:00022e49       __unwindfunclet$?procSelection@alm_db_output@@AAEXXZ$1 10023e49 f   dialogimpl.obj
 0001:00022e52       __ehhandler$?procSelection@alm_db_output@@AAEXXZ 10023e52 f   dialogimpl.obj
 0001:00022e52       __ehhandler$?setGroupDefaultText@dialog@@QAEXXZ 10023e52 f   dialogimpl.obj
 0001:00022e6d       __unwindfunclet$?useAltId@dialog@@AAE?AVQString@@V2@0_N@Z$0 10023e6d f   dialogimpl.obj
 0001:00022e76       __unwindfunclet$?useAltId@dialog@@AAE?AVQString@@V2@0_N@Z$1 10023e76 f   dialogimpl.obj
 0001:00022e7f       __unwindfunclet$?useAltId@dialog@@AAE?AVQString@@V2@0_N@Z$2 10023e7f f   dialogimpl.obj
 0001:00022e99       __unwindfunclet$?useAltId@dialog@@AAE?AVQString@@V2@0_N@Z$3 10023e99 f   dialogimpl.obj
 0001:00022ea2       __unwindfunclet$?useAltId@dialog@@AAE?AVQString@@V2@0_N@Z$4 10023ea2 f   dialogimpl.obj
 0001:00022eab       __unwindfunclet$?useAltId@dialog@@AAE?AVQString@@V2@0_N@Z$5 10023eab f   dialogimpl.obj
 0001:00022eb4       __ehhandler$?useAltId@dialog@@AAE?AVQString@@V2@0_N@Z 10023eb4 f   dialogimpl.obj
 0001:00022ecf       __unwindfunclet$??0manage_temp@@QAE@QAV?$QMap@VQString@@PAVcProcess@@@@PAVdialog@@@Z$0 10023ecf f   manage_tempimpl.obj
 0001:00022ed7       __unwindfunclet$??0manage_temp@@QAE@QAV?$QMap@VQString@@PAVcProcess@@@@PAVdialog@@@Z$1 10023ed7 f   manage_tempimpl.obj
 0001:00022ee6       __unwindfunclet$??0manage_temp@@QAE@QAV?$QMap@VQString@@PAVcProcess@@@@PAVdialog@@@Z$2 10023ee6 f   manage_tempimpl.obj
 0001:00022ef5       __unwindfunclet$??0manage_temp@@QAE@QAV?$QMap@VQString@@PAVcProcess@@@@PAVdialog@@@Z$3 10023ef5 f   manage_tempimpl.obj
 0001:00022efe       __unwindfunclet$??0manage_temp@@QAE@QAV?$QMap@VQString@@PAVcProcess@@@@PAVdialog@@@Z$4 10023efe f   manage_tempimpl.obj
 0001:00022f07       __unwindfunclet$??0manage_temp@@QAE@QAV?$QMap@VQString@@PAVcProcess@@@@PAVdialog@@@Z$5 10023f07 f   manage_tempimpl.obj
 0001:00022f10       __unwindfunclet$??0manage_temp@@QAE@QAV?$QMap@VQString@@PAVcProcess@@@@PAVdialog@@@Z$6 10023f10 f   manage_tempimpl.obj
 0001:00022f19       __unwindfunclet$??0manage_temp@@QAE@QAV?$QMap@VQString@@PAVcProcess@@@@PAVdialog@@@Z$7 10023f19 f   manage_tempimpl.obj
 0001:00022f22       __unwindfunclet$??0manage_temp@@QAE@QAV?$QMap@VQString@@PAVcProcess@@@@PAVdialog@@@Z$8 10023f22 f   manage_tempimpl.obj
 0001:00022f2b       __unwindfunclet$??0manage_temp@@QAE@QAV?$QMap@VQString@@PAVcProcess@@@@PAVdialog@@@Z$9 10023f2b f   manage_tempimpl.obj
 0001:00022f34       __unwindfunclet$??0manage_temp@@QAE@QAV?$QMap@VQString@@PAVcProcess@@@@PAVdialog@@@Z$10 10023f34 f   manage_tempimpl.obj
 0001:00022f3d       __ehhandler$??0manage_temp@@QAE@QAV?$QMap@VQString@@PAVcProcess@@@@PAVdialog@@@Z 10023f3d f   manage_tempimpl.obj
 0001:00022f58       __unwindfunclet$??1manage_temp@@UAE@XZ$0 10023f58 f   manage_tempimpl.obj
 0001:00022f60       __unwindfunclet$??1manage_temp@@UAE@XZ$1 10023f60 f   manage_tempimpl.obj
 0001:00022f6f       __unwindfunclet$??1manage_temp@@UAE@XZ$2 10023f6f f   manage_tempimpl.obj
 0001:00022f7e       __unwindfunclet$??1manage_temp@@UAE@XZ$3 10023f7e f   manage_tempimpl.obj
 0001:00022f87       __unwindfunclet$??1manage_temp@@UAE@XZ$4 10023f87 f   manage_tempimpl.obj
 0001:00022f90       __unwindfunclet$??1manage_temp@@UAE@XZ$5 10023f90 f   manage_tempimpl.obj
 0001:00022f99       __unwindfunclet$??1manage_temp@@UAE@XZ$6 10023f99 f   manage_tempimpl.obj
 0001:00022fa2       __unwindfunclet$??1manage_temp@@UAE@XZ$7 10023fa2 f   manage_tempimpl.obj
 0001:00022fab       __unwindfunclet$??1manage_temp@@UAE@XZ$8 10023fab f   manage_tempimpl.obj
 0001:00022fb4       __unwindfunclet$??1manage_temp@@UAE@XZ$9 10023fb4 f   manage_tempimpl.obj
 0001:00022fbd       __unwindfunclet$??1manage_temp@@UAE@XZ$10 10023fbd f   manage_tempimpl.obj
 0001:00022fc6       __ehhandler$??1manage_temp@@UAE@XZ 10023fc6 f   manage_tempimpl.obj
 0001:00022fe1       __unwindfunclet$?clearAllParamsText@manage_temp@@QAEXXZ$0 10023fe1 f   manage_tempimpl.obj
 0001:00022fe1       __unwindfunclet$?setAllParamsDefaultText@manage_temp@@QAEXXZ$0 10023fe1 f   manage_tempimpl.obj
 0001:00022fea       __unwindfunclet$?setAllParamsDefaultText@manage_temp@@QAEXXZ$1 10023fea f   manage_tempimpl.obj
 0001:00022fea       __unwindfunclet$?clearAllParamsText@manage_temp@@QAEXXZ$1 10023fea f   manage_tempimpl.obj
 0001:00022ff3       __ehhandler$?setAllParamsDefaultText@manage_temp@@QAEXXZ 10023ff3 f   manage_tempimpl.obj
 0001:00022ff3       __ehhandler$?clearAllParamsText@manage_temp@@QAEXXZ 10023ff3 f   manage_tempimpl.obj
 0001:0002300e       __unwindfunclet$?clearAllText@manage_temp@@QAEXXZ$0 1002400e f   manage_tempimpl.obj
 0001:00023017       __unwindfunclet$?clearAllText@manage_temp@@QAEXXZ$1 10024017 f   manage_tempimpl.obj
 0001:00023020       __unwindfunclet$?clearAllText@manage_temp@@QAEXXZ$2 10024020 f   manage_tempimpl.obj
 0001:00023029       __unwindfunclet$?clearAllText@manage_temp@@QAEXXZ$3 10024029 f   manage_tempimpl.obj
 0001:00023032       __unwindfunclet$?clearAllText@manage_temp@@QAEXXZ$4 10024032 f   manage_tempimpl.obj
 0001:0002303b       __unwindfunclet$?clearAllText@manage_temp@@QAEXXZ$5 1002403b f   manage_tempimpl.obj
 0001:00023044       __unwindfunclet$?clearAllText@manage_temp@@QAEXXZ$6 10024044 f   manage_tempimpl.obj
 0001:0002304d       __unwindfunclet$?clearAllText@manage_temp@@QAEXXZ$7 1002404d f   manage_tempimpl.obj
 0001:00023056       __ehhandler$?clearAllText@manage_temp@@QAEXXZ 10024056 f   manage_tempimpl.obj
 0001:00023071       __unwindfunclet$?defaultText@manage_temp@@AAE?AVQString@@W4AlarmStates@Alarms@@@Z$0 10024071 f   manage_tempimpl.obj
 0001:0002307a       __unwindfunclet$?defaultText@manage_temp@@AAE?AVQString@@W4AlarmStates@Alarms@@@Z$1 1002407a f   manage_tempimpl.obj
 0001:00023083       __unwindfunclet$?defaultText@manage_temp@@AAE?AVQString@@W4AlarmStates@Alarms@@@Z$2 10024083 f   manage_tempimpl.obj
 0001:0002308c       __unwindfunclet$?defaultText@manage_temp@@AAE?AVQString@@W4AlarmStates@Alarms@@@Z$3 1002408c f   manage_tempimpl.obj
 0001:00023095       __unwindfunclet$?defaultText@manage_temp@@AAE?AVQString@@W4AlarmStates@Alarms@@@Z$4 10024095 f   manage_tempimpl.obj
 0001:0002309e       __unwindfunclet$?defaultText@manage_temp@@AAE?AVQString@@W4AlarmStates@Alarms@@@Z$5 1002409e f   manage_tempimpl.obj
 0001:000230a7       __unwindfunclet$?defaultText@manage_temp@@AAE?AVQString@@W4AlarmStates@Alarms@@@Z$6 100240a7 f   manage_tempimpl.obj
 0001:000230b0       __unwindfunclet$?defaultText@manage_temp@@AAE?AVQString@@W4AlarmStates@Alarms@@@Z$7 100240b0 f   manage_tempimpl.obj
 0001:000230b9       __unwindfunclet$?defaultText@manage_temp@@AAE?AVQString@@W4AlarmStates@Alarms@@@Z$8 100240b9 f   manage_tempimpl.obj
 0001:000230c2       __unwindfunclet$?defaultText@manage_temp@@AAE?AVQString@@W4AlarmStates@Alarms@@@Z$9 100240c2 f   manage_tempimpl.obj
 0001:000230cb       __unwindfunclet$?defaultText@manage_temp@@AAE?AVQString@@W4AlarmStates@Alarms@@@Z$10 100240cb f   manage_tempimpl.obj
 0001:000230d4       __unwindfunclet$?defaultText@manage_temp@@AAE?AVQString@@W4AlarmStates@Alarms@@@Z$11 100240d4 f   manage_tempimpl.obj
 0001:000230dd       __unwindfunclet$?defaultText@manage_temp@@AAE?AVQString@@W4AlarmStates@Alarms@@@Z$17 100240dd f   manage_tempimpl.obj
 0001:000230e6       __unwindfunclet$?defaultText@manage_temp@@AAE?AVQString@@W4AlarmStates@Alarms@@@Z$16 100240e6 f   manage_tempimpl.obj
 0001:000230ef       __unwindfunclet$?defaultText@manage_temp@@AAE?AVQString@@W4AlarmStates@Alarms@@@Z$15 100240ef f   manage_tempimpl.obj
 0001:000230f8       __unwindfunclet$?defaultText@manage_temp@@AAE?AVQString@@W4AlarmStates@Alarms@@@Z$14 100240f8 f   manage_tempimpl.obj
 0001:00023101       __unwindfunclet$?defaultText@manage_temp@@AAE?AVQString@@W4AlarmStates@Alarms@@@Z$13 10024101 f   manage_tempimpl.obj
 0001:0002310a       __unwindfunclet$?defaultText@manage_temp@@AAE?AVQString@@W4AlarmStates@Alarms@@@Z$12 1002410a f   manage_tempimpl.obj
 0001:00023113       __unwindfunclet$?defaultText@manage_temp@@AAE?AVQString@@W4AlarmStates@Alarms@@@Z$18 10024113 f   manage_tempimpl.obj
 0001:0002312d       __ehhandler$?defaultText@manage_temp@@AAE?AVQString@@W4AlarmStates@Alarms@@@Z 1002412d f   manage_tempimpl.obj
 0001:00023148       __unwindfunclet$?itemChanged@manage_temp@@QAEXXZ$0 10024148 f   manage_tempimpl.obj
 0001:00023151       __unwindfunclet$?itemChanged@manage_temp@@QAEXXZ$1 10024151 f   manage_tempimpl.obj
 0001:0002315a       __unwindfunclet$?itemChanged@manage_temp@@QAEXXZ$2 1002415a f   manage_tempimpl.obj
 0001:00023163       __unwindfunclet$?itemChanged@manage_temp@@QAEXXZ$3 10024163 f   manage_tempimpl.obj
 0001:0002316c       __unwindfunclet$?itemChanged@manage_temp@@QAEXXZ$4 1002416c f   manage_tempimpl.obj
 0001:00023175       __unwindfunclet$?itemChanged@manage_temp@@QAEXXZ$5 10024175 f   manage_tempimpl.obj
 0001:0002317e       __unwindfunclet$?itemChanged@manage_temp@@QAEXXZ$6 1002417e f   manage_tempimpl.obj
 0001:00023187       __unwindfunclet$?itemChanged@manage_temp@@QAEXXZ$7 10024187 f   manage_tempimpl.obj
 0001:00023190       __unwindfunclet$?itemChanged@manage_temp@@QAEXXZ$8 10024190 f   manage_tempimpl.obj
 0001:00023199       __ehhandler$?itemChanged@manage_temp@@QAEXXZ 10024199 f   manage_tempimpl.obj
 0001:000231b4       __unwindfunclet$?prefixChanged@manage_temp@@QAEXABVQString@@@Z$0 100241b4 f   manage_tempimpl.obj
 0001:000231bd       __unwindfunclet$?prefixChanged@manage_temp@@QAEXABVQString@@@Z$1 100241bd f   manage_tempimpl.obj
 0001:000231c6       __unwindfunclet$?prefixChanged@manage_temp@@QAEXABVQString@@@Z$2 100241c6 f   manage_tempimpl.obj
 0001:000231d0       __unwindfunclet$?prefixChanged@manage_temp@@QAEXABVQString@@@Z$3 100241d0 f   manage_tempimpl.obj
 0001:000231d9       __unwindfunclet$?prefixChanged@manage_temp@@QAEXABVQString@@@Z$4 100241d9 f   manage_tempimpl.obj
 0001:000231e2       __unwindfunclet$?prefixChanged@manage_temp@@QAEXABVQString@@@Z$5 100241e2 f   manage_tempimpl.obj
 0001:000231eb       __unwindfunclet$?prefixChanged@manage_temp@@QAEXABVQString@@@Z$6 100241eb f   manage_tempimpl.obj
 0001:000231f4       __unwindfunclet$?prefixChanged@manage_temp@@QAEXABVQString@@@Z$7 100241f4 f   manage_tempimpl.obj
 0001:000231fd       __unwindfunclet$?prefixChanged@manage_temp@@QAEXABVQString@@@Z$8 100241fd f   manage_tempimpl.obj
 0001:00023206       __unwindfunclet$?prefixChanged@manage_temp@@QAEXABVQString@@@Z$9 10024206 f   manage_tempimpl.obj
 0001:0002320f       __unwindfunclet$?prefixChanged@manage_temp@@QAEXABVQString@@@Z$11 1002420f f   manage_tempimpl.obj
 0001:00023218       __unwindfunclet$?prefixChanged@manage_temp@@QAEXABVQString@@@Z$12 10024218 f   manage_tempimpl.obj
 0001:00023221       __unwindfunclet$?prefixChanged@manage_temp@@QAEXABVQString@@@Z$13 10024221 f   manage_tempimpl.obj
 0001:0002322a       __unwindfunclet$?prefixChanged@manage_temp@@QAEXABVQString@@@Z$14 1002422a f   manage_tempimpl.obj
 0001:00023233       __unwindfunclet$?prefixChanged@manage_temp@@QAEXABVQString@@@Z$15 10024233 f   manage_tempimpl.obj
 0001:0002323c       __unwindfunclet$?prefixChanged@manage_temp@@QAEXABVQString@@@Z$17 1002423c f   manage_tempimpl.obj
 0001:00023245       __unwindfunclet$?prefixChanged@manage_temp@@QAEXABVQString@@@Z$18 10024245 f   manage_tempimpl.obj
 0001:0002324e       __unwindfunclet$?prefixChanged@manage_temp@@QAEXABVQString@@@Z$19 1002424e f   manage_tempimpl.obj
 0001:00023257       __unwindfunclet$?prefixChanged@manage_temp@@QAEXABVQString@@@Z$20 10024257 f   manage_tempimpl.obj
 0001:00023261       __unwindfunclet$?prefixChanged@manage_temp@@QAEXABVQString@@@Z$21 10024261 f   manage_tempimpl.obj
 0001:0002327b       __ehhandler$?prefixChanged@manage_temp@@QAEXABVQString@@@Z 1002427b f   manage_tempimpl.obj
 0001:00023296       __unwindfunclet$?selectProcess@manage_temp@@QAEXPAVQListViewItem@@@Z$0 10024296 f   manage_tempimpl.obj
 0001:0002329f       __unwindfunclet$?selectProcess@manage_temp@@QAEXPAVQListViewItem@@@Z$1 1002429f f   manage_tempimpl.obj
 0001:000232a8       __unwindfunclet$?selectProcess@manage_temp@@QAEXPAVQListViewItem@@@Z$2 100242a8 f   manage_tempimpl.obj
 0001:000232b1       __unwindfunclet$?selectProcess@manage_temp@@QAEXPAVQListViewItem@@@Z$3 100242b1 f   manage_tempimpl.obj
 0001:000232ba       __unwindfunclet$?selectProcess@manage_temp@@QAEXPAVQListViewItem@@@Z$4 100242ba f   manage_tempimpl.obj
 0001:000232c3       __unwindfunclet$?selectProcess@manage_temp@@QAEXPAVQListViewItem@@@Z$5 100242c3 f   manage_tempimpl.obj
 0001:000232cc       __unwindfunclet$?selectProcess@manage_temp@@QAEXPAVQListViewItem@@@Z$6 100242cc f   manage_tempimpl.obj
 0001:000232d5       __unwindfunclet$?selectProcess@manage_temp@@QAEXPAVQListViewItem@@@Z$7 100242d5 f   manage_tempimpl.obj
 0001:000232de       __unwindfunclet$?selectProcess@manage_temp@@QAEXPAVQListViewItem@@@Z$8 100242de f   manage_tempimpl.obj
 0001:000232e7       __ehhandler$?selectProcess@manage_temp@@QAEXPAVQListViewItem@@@Z 100242e7 f   manage_tempimpl.obj
 0001:00023302       __unwindfunclet$?resetDefaults@dialog@@QAEXXZ$0 10024302 f   manage_tempimpl.obj
 0001:00023302       __unwindfunclet$?setAllDefaultText@manage_temp@@QAEXXZ$0 10024302 f   manage_tempimpl.obj
 0001:0002330b       __unwindfunclet$?setAllDefaultText@manage_temp@@QAEXXZ$1 1002430b f   manage_tempimpl.obj
 0001:0002330b       __unwindfunclet$?resetDefaults@dialog@@QAEXXZ$1 1002430b f   manage_tempimpl.obj
 0001:00023314       __unwindfunclet$?setAllDefaultText@manage_temp@@QAEXXZ$2 10024314 f   manage_tempimpl.obj
 0001:00023314       __unwindfunclet$?resetDefaults@dialog@@QAEXXZ$2 10024314 f   manage_tempimpl.obj
 0001:0002331d       __unwindfunclet$?resetDefaults@dialog@@QAEXXZ$3 1002431d f   manage_tempimpl.obj
 0001:0002331d       __unwindfunclet$?setAllDefaultText@manage_temp@@QAEXXZ$3 1002431d f   manage_tempimpl.obj
 0001:00023326       __unwindfunclet$?resetDefaults@dialog@@QAEXXZ$4 10024326 f   manage_tempimpl.obj
 0001:00023326       __unwindfunclet$?setAllDefaultText@manage_temp@@QAEXXZ$4 10024326 f   manage_tempimpl.obj
 0001:0002332f       __unwindfunclet$?setAllDefaultText@manage_temp@@QAEXXZ$5 1002432f f   manage_tempimpl.obj
 0001:0002332f       __unwindfunclet$?resetDefaults@dialog@@QAEXXZ$5 1002432f f   manage_tempimpl.obj
 0001:00023338       __ehhandler$?setAllDefaultText@manage_temp@@QAEXXZ 10024338 f   manage_tempimpl.obj
 0001:00023338       __ehhandler$?resetDefaults@dialog@@QAEXXZ 10024338 f   manage_tempimpl.obj
 0001:00023353       __unwindfunclet$?levelChanged@dialog@@QAEXH@Z$0 10024353 f   manage_tempimpl.obj
 0001:00023353       __unwindfunclet$?setDefaultGroup@manage_temp@@QAEXVQString@@@Z$0 10024353 f   manage_tempimpl.obj
 0001:0002335c       __ehhandler$?levelChanged@dialog@@QAEXH@Z 1002435c f   manage_tempimpl.obj
 0001:0002335c       __ehhandler$?setDefaultGroup@manage_temp@@QAEXVQString@@@Z 1002435c f   manage_tempimpl.obj
 0001:00023377       __unwindfunclet$?setDeviceDefaultText@manage_temp@@QAEXXZ$0 10024377 f   manage_tempimpl.obj
 0001:00023380       __unwindfunclet$?setDeviceDefaultText@manage_temp@@QAEXXZ$1 10024380 f   manage_tempimpl.obj
 0001:00023389       __ehhandler$?setDeviceDefaultText@manage_temp@@QAEXXZ 10024389 f   manage_tempimpl.obj
 0001:000233a4       __unwindfunclet$?setProcess@manage_temp@@AAEXPAVQListViewItem@@@Z$0 100243a4 f   manage_tempimpl.obj
 0001:000233ad       __unwindfunclet$?setProcess@manage_temp@@AAEXPAVQListViewItem@@@Z$1 100243ad f   manage_tempimpl.obj
 0001:000233b6       __unwindfunclet$?setProcess@manage_temp@@AAEXPAVQListViewItem@@@Z$2 100243b6 f   manage_tempimpl.obj
 0001:000233bf       __unwindfunclet$?setProcess@manage_temp@@AAEXPAVQListViewItem@@@Z$3 100243bf f   manage_tempimpl.obj
 0001:000233c8       __unwindfunclet$?setProcess@manage_temp@@AAEXPAVQListViewItem@@@Z$4 100243c8 f   manage_tempimpl.obj
 0001:000233d1       __ehhandler$?setProcess@manage_temp@@AAEXPAVQListViewItem@@@Z 100243d1 f   manage_tempimpl.obj
 0001:000233ec       __unwindfunclet$??4?$QGuardedPtr@VQPopupMenu@@@@QAEAAV0@PAVQPopupMenu@@@Z$0 100243ec f   plugindesc.obj
 0001:000233ec       __unwindfunclet$??4?$QGuardedPtr@VQDockWindow@@@@QAEAAV0@PAVQDockWindow@@@Z$0 100243ec f   plugindesc.obj
 0001:000233ec       __unwindfunclet$??0?$QMap@VQString@@PAVcProcess@@@@QAE@XZ$0 100243ec f   plugindesc.obj
 0001:000233ec       __unwindfunclet$??0?$QGuardedPtr@VQPopupMenu@@@@QAE@XZ$0 100243ec f   plugindesc.obj
 0001:000233ec       __unwindfunclet$?insert@?$QMapPrivate@VQString@@PAVcProcess@@@@QAE?AV?$QMapIterator@VQString@@PAVcProcess@@@@PAUQMapNodeBase@@0ABVQString@@@Z$0 100243ec f   plugindesc.obj
 0001:000233ec       __unwindfunclet$??0?$QMapPrivate@VQString@@PAVcProcess@@@@QAE@XZ$0 100243ec f   plugindesc.obj
 0001:000233ec       __unwindfunclet$?detachInternal@?$QMap@VQString@@PAVcProcess@@@@AAEXXZ$0 100243ec f   plugindesc.obj
 0001:000233ec       __unwindfunclet$?create@plugindesc@@UAEPAVconfig_plugin_base@@ABVQString@@00@Z$0 100243ec f   plugindesc.obj
 0001:000233ec       __unwindfunclet$?clear@?$QMap@VQString@@PAVcProcess@@@@QAEXXZ$0 100243ec f   plugindesc.obj
 0001:000233ec       __unwindfunclet$??0?$QGuardedPtr@VQDockWindow@@@@QAE@XZ$0 100243ec f   plugindesc.obj
 0001:000233f6       __ehhandler$??0?$QMap@VQString@@PAVcProcess@@@@QAE@XZ 100243f6 f   plugindesc.obj
 0001:000233f6       __ehhandler$??0?$QGuardedPtr@VQDockWindow@@@@QAE@XZ 100243f6 f   plugindesc.obj
 0001:000233f6       __ehhandler$??0?$QMapPrivate@VQString@@PAVcProcess@@@@QAE@XZ 100243f6 f   plugindesc.obj
 0001:000233f6       __ehhandler$??4?$QGuardedPtr@VQDockWindow@@@@QAEAAV0@PAVQDockWindow@@@Z 100243f6 f   plugindesc.obj
 0001:000233f6       __ehhandler$??4?$QGuardedPtr@VQPopupMenu@@@@QAEAAV0@PAVQPopupMenu@@@Z 100243f6 f   plugindesc.obj
 0001:000233f6       __ehhandler$??0?$QGuardedPtr@VQPopupMenu@@@@QAE@XZ 100243f6 f   plugindesc.obj
 0001:000233f6       __ehhandler$?insert@?$QMapPrivate@VQString@@PAVcProcess@@@@QAE?AV?$QMapIterator@VQString@@PAVcProcess@@@@PAUQMapNodeBase@@0ABVQString@@@Z 100243f6 f   plugindesc.obj
 0001:000233f6       __ehhandler$?create@plugindesc@@UAEPAVconfig_plugin_base@@ABVQString@@00@Z 100243f6 f   plugindesc.obj
 0001:000233f6       __ehhandler$?clear@?$QMap@VQString@@PAVcProcess@@@@QAEXXZ 100243f6 f   plugindesc.obj
 0001:000233f6       __ehhandler$?detachInternal@?$QMap@VQString@@PAVcProcess@@@@AAEXXZ 100243f6 f   plugindesc.obj
 0001:00023411       __unwindfunclet$?keys@plugindesc@@UAE?AVQStringList@@ABVQString@@0@Z$0 10024411 f   plugindesc.obj
 0001:0002342b       __unwindfunclet$?keys@plugindesc@@UAE?AVQStringList@@ABVQString@@0@Z$1 1002442b f   plugindesc.obj
 0001:00023434       __ehhandler$?keys@plugindesc@@UAE?AVQStringList@@ABVQString@@0@Z 10024434 f   plugindesc.obj
 0001:0002344f       __unwindfunclet$??0setDefaultsBase@@QAE@PAVQWidget@@PBD_NI@Z$0 1002444f f   setdefaults.obj
 0001:00023458       __unwindfunclet$??0setDefaultsBase@@QAE@PAVQWidget@@PBD_NI@Z$1 10024458 f   setdefaults.obj
 0001:00023462       __unwindfunclet$??0setDefaultsBase@@QAE@PAVQWidget@@PBD_NI@Z$2 10024462 f   setdefaults.obj
 0001:0002346c       __unwindfunclet$??0setDefaultsBase@@QAE@PAVQWidget@@PBD_NI@Z$3 1002446c f   setdefaults.obj
 0001:00023476       __unwindfunclet$??0setDefaultsBase@@QAE@PAVQWidget@@PBD_NI@Z$4 10024476 f   setdefaults.obj
 0001:00023480       __unwindfunclet$??0setDefaultsBase@@QAE@PAVQWidget@@PBD_NI@Z$5 10024480 f   setdefaults.obj
 0001:0002348a       __unwindfunclet$??0setDefaultsBase@@QAE@PAVQWidget@@PBD_NI@Z$6 1002448a f   setdefaults.obj
 0001:00023494       __unwindfunclet$??0setDefaultsBase@@QAE@PAVQWidget@@PBD_NI@Z$7 10024494 f   setdefaults.obj
 0001:0002349e       __unwindfunclet$??0setDefaultsBase@@QAE@PAVQWidget@@PBD_NI@Z$8 1002449e f   setdefaults.obj
 0001:000234a8       __unwindfunclet$??0setDefaultsBase@@QAE@PAVQWidget@@PBD_NI@Z$9 100244a8 f   setdefaults.obj
 0001:000234b2       __unwindfunclet$??0setDefaultsBase@@QAE@PAVQWidget@@PBD_NI@Z$10 100244b2 f   setdefaults.obj
 0001:000234bc       __unwindfunclet$??0setDefaultsBase@@QAE@PAVQWidget@@PBD_NI@Z$11 100244bc f   setdefaults.obj
 0001:000234c6       __unwindfunclet$??0setDefaultsBase@@QAE@PAVQWidget@@PBD_NI@Z$12 100244c6 f   setdefaults.obj
 0001:000234d0       __unwindfunclet$??0setDefaultsBase@@QAE@PAVQWidget@@PBD_NI@Z$13 100244d0 f   setdefaults.obj
 0001:000234da       __unwindfunclet$??0setDefaultsBase@@QAE@PAVQWidget@@PBD_NI@Z$14 100244da f   setdefaults.obj
 0001:000234e4       __unwindfunclet$??0setDefaultsBase@@QAE@PAVQWidget@@PBD_NI@Z$15 100244e4 f   setdefaults.obj
 0001:000234ee       __unwindfunclet$??0setDefaultsBase@@QAE@PAVQWidget@@PBD_NI@Z$16 100244ee f   setdefaults.obj
 0001:000234f8       __unwindfunclet$??0setDefaultsBase@@QAE@PAVQWidget@@PBD_NI@Z$17 100244f8 f   setdefaults.obj
 0001:00023502       __unwindfunclet$??0setDefaultsBase@@QAE@PAVQWidget@@PBD_NI@Z$18 10024502 f   setdefaults.obj
 0001:0002350c       __unwindfunclet$??0setDefaultsBase@@QAE@PAVQWidget@@PBD_NI@Z$19 1002450c f   setdefaults.obj
 0001:00023516       __unwindfunclet$??0setDefaultsBase@@QAE@PAVQWidget@@PBD_NI@Z$20 10024516 f   setdefaults.obj
 0001:00023520       __unwindfunclet$??0setDefaultsBase@@QAE@PAVQWidget@@PBD_NI@Z$21 10024520 f   setdefaults.obj
 0001:0002352a       __unwindfunclet$??0setDefaultsBase@@QAE@PAVQWidget@@PBD_NI@Z$22 1002452a f   setdefaults.obj
 0001:00023534       __unwindfunclet$??0setDefaultsBase@@QAE@PAVQWidget@@PBD_NI@Z$23 10024534 f   setdefaults.obj
 0001:0002353e       __unwindfunclet$??0setDefaultsBase@@QAE@PAVQWidget@@PBD_NI@Z$24 1002453e f   setdefaults.obj
 0001:00023548       __unwindfunclet$??0setDefaultsBase@@QAE@PAVQWidget@@PBD_NI@Z$25 10024548 f   setdefaults.obj
 0001:00023552       __unwindfunclet$??0setDefaultsBase@@QAE@PAVQWidget@@PBD_NI@Z$26 10024552 f   setdefaults.obj
 0001:0002355c       __unwindfunclet$??0setDefaultsBase@@QAE@PAVQWidget@@PBD_NI@Z$27 1002455c f   setdefaults.obj
 0001:00023566       __unwindfunclet$??0setDefaultsBase@@QAE@PAVQWidget@@PBD_NI@Z$28 10024566 f   setdefaults.obj
 0001:00023570       __unwindfunclet$??0setDefaultsBase@@QAE@PAVQWidget@@PBD_NI@Z$29 10024570 f   setdefaults.obj
 0001:0002357a       __unwindfunclet$??0setDefaultsBase@@QAE@PAVQWidget@@PBD_NI@Z$30 1002457a f   setdefaults.obj
 0001:00023584       __unwindfunclet$??0setDefaultsBase@@QAE@PAVQWidget@@PBD_NI@Z$31 10024584 f   setdefaults.obj
 0001:0002358e       __unwindfunclet$??0setDefaultsBase@@QAE@PAVQWidget@@PBD_NI@Z$32 1002458e f   setdefaults.obj
 0001:00023598       __unwindfunclet$??0setDefaultsBase@@QAE@PAVQWidget@@PBD_NI@Z$33 10024598 f   setdefaults.obj
 0001:000235a2       __unwindfunclet$??0setDefaultsBase@@QAE@PAVQWidget@@PBD_NI@Z$34 100245a2 f   setdefaults.obj
 0001:000235ac       __unwindfunclet$??0setDefaultsBase@@QAE@PAVQWidget@@PBD_NI@Z$35 100245ac f   setdefaults.obj
 0001:000235b6       __unwindfunclet$??0setDefaultsBase@@QAE@PAVQWidget@@PBD_NI@Z$36 100245b6 f   setdefaults.obj
 0001:000235c0       __unwindfunclet$??0setDefaultsBase@@QAE@PAVQWidget@@PBD_NI@Z$37 100245c0 f   setdefaults.obj
 0001:000235ca       __unwindfunclet$??0setDefaultsBase@@QAE@PAVQWidget@@PBD_NI@Z$38 100245ca f   setdefaults.obj
 0001:000235d4       __unwindfunclet$??0setDefaultsBase@@QAE@PAVQWidget@@PBD_NI@Z$39 100245d4 f   setdefaults.obj
 0001:000235de       __unwindfunclet$??0setDefaultsBase@@QAE@PAVQWidget@@PBD_NI@Z$40 100245de f   setdefaults.obj
 0001:000235e8       __unwindfunclet$??0setDefaultsBase@@QAE@PAVQWidget@@PBD_NI@Z$41 100245e8 f   setdefaults.obj
 0001:000235f2       __unwindfunclet$??0setDefaultsBase@@QAE@PAVQWidget@@PBD_NI@Z$42 100245f2 f   setdefaults.obj
 0001:000235fc       __unwindfunclet$??0setDefaultsBase@@QAE@PAVQWidget@@PBD_NI@Z$43 100245fc f   setdefaults.obj
 0001:00023606       __unwindfunclet$??0setDefaultsBase@@QAE@PAVQWidget@@PBD_NI@Z$44 10024606 f   setdefaults.obj
 0001:00023610       __unwindfunclet$??0setDefaultsBase@@QAE@PAVQWidget@@PBD_NI@Z$45 10024610 f   setdefaults.obj
 0001:0002361a       __unwindfunclet$??0setDefaultsBase@@QAE@PAVQWidget@@PBD_NI@Z$46 1002461a f   setdefaults.obj
 0001:00023624       __unwindfunclet$??0setDefaultsBase@@QAE@PAVQWidget@@PBD_NI@Z$47 10024624 f   setdefaults.obj
 0001:0002362e       __unwindfunclet$??0setDefaultsBase@@QAE@PAVQWidget@@PBD_NI@Z$48 1002462e f   setdefaults.obj
 0001:00023638       __unwindfunclet$??0setDefaultsBase@@QAE@PAVQWidget@@PBD_NI@Z$49 10024638 f   setdefaults.obj
 0001:00023642       __unwindfunclet$??0setDefaultsBase@@QAE@PAVQWidget@@PBD_NI@Z$50 10024642 f   setdefaults.obj
 0001:0002364c       __unwindfunclet$??0setDefaultsBase@@QAE@PAVQWidget@@PBD_NI@Z$51 1002464c f   setdefaults.obj
 0001:00023656       __unwindfunclet$??0setDefaultsBase@@QAE@PAVQWidget@@PBD_NI@Z$52 10024656 f   setdefaults.obj
 0001:00023660       __unwindfunclet$??0setDefaultsBase@@QAE@PAVQWidget@@PBD_NI@Z$53 10024660 f   setdefaults.obj
 0001:0002366a       __unwindfunclet$??0setDefaultsBase@@QAE@PAVQWidget@@PBD_NI@Z$54 1002466a f   setdefaults.obj
 0001:00023674       __unwindfunclet$??0setDefaultsBase@@QAE@PAVQWidget@@PBD_NI@Z$55 10024674 f   setdefaults.obj
 0001:0002367e       __ehhandler$??0setDefaultsBase@@QAE@PAVQWidget@@PBD_NI@Z 1002467e f   setdefaults.obj
 0001:00023699       __unwindfunclet$?languageChange@setDefaultsBase@@MAEXXZ$0 10024699 f   setdefaults.obj
 0001:000236a2       __unwindfunclet$?languageChange@setDefaultsBase@@MAEXXZ$1 100246a2 f   setdefaults.obj
 0001:000236ab       __unwindfunclet$?languageChange@setDefaultsBase@@MAEXXZ$2 100246ab f   setdefaults.obj
 0001:000236b4       __unwindfunclet$?languageChange@setDefaultsBase@@MAEXXZ$3 100246b4 f   setdefaults.obj
 0001:000236bd       __unwindfunclet$?languageChange@setDefaultsBase@@MAEXXZ$4 100246bd f   setdefaults.obj
 0001:000236c6       __unwindfunclet$?languageChange@setDefaultsBase@@MAEXXZ$5 100246c6 f   setdefaults.obj
 0001:000236cf       __unwindfunclet$?languageChange@setDefaultsBase@@MAEXXZ$6 100246cf f   setdefaults.obj
 0001:000236d8       __unwindfunclet$?languageChange@setDefaultsBase@@MAEXXZ$7 100246d8 f   setdefaults.obj
 0001:000236e1       __unwindfunclet$?languageChange@setDefaultsBase@@MAEXXZ$8 100246e1 f   setdefaults.obj
 0001:000236ea       __unwindfunclet$?languageChange@setDefaultsBase@@MAEXXZ$9 100246ea f   setdefaults.obj
 0001:000236f3       __unwindfunclet$?languageChange@setDefaultsBase@@MAEXXZ$10 100246f3 f   setdefaults.obj
 0001:000236fc       __unwindfunclet$?languageChange@setDefaultsBase@@MAEXXZ$11 100246fc f   setdefaults.obj
 0001:00023705       __unwindfunclet$?languageChange@setDefaultsBase@@MAEXXZ$12 10024705 f   setdefaults.obj
 0001:0002370e       __unwindfunclet$?languageChange@setDefaultsBase@@MAEXXZ$13 1002470e f   setdefaults.obj
 0001:00023717       __unwindfunclet$?languageChange@setDefaultsBase@@MAEXXZ$14 10024717 f   setdefaults.obj
 0001:00023720       __unwindfunclet$?languageChange@setDefaultsBase@@MAEXXZ$15 10024720 f   setdefaults.obj
 0001:00023729       __unwindfunclet$?languageChange@setDefaultsBase@@MAEXXZ$16 10024729 f   setdefaults.obj
 0001:00023732       __unwindfunclet$?languageChange@setDefaultsBase@@MAEXXZ$17 10024732 f   setdefaults.obj
 0001:0002373b       __unwindfunclet$?languageChange@setDefaultsBase@@MAEXXZ$18 1002473b f   setdefaults.obj
 0001:00023744       __unwindfunclet$?languageChange@setDefaultsBase@@MAEXXZ$19 10024744 f   setdefaults.obj
 0001:0002374d       __unwindfunclet$?languageChange@setDefaultsBase@@MAEXXZ$20 1002474d f   setdefaults.obj
 0001:00023756       __unwindfunclet$?languageChange@setDefaultsBase@@MAEXXZ$21 10024756 f   setdefaults.obj
 0001:0002375f       __unwindfunclet$?languageChange@setDefaultsBase@@MAEXXZ$22 1002475f f   setdefaults.obj
 0001:00023768       __unwindfunclet$?languageChange@setDefaultsBase@@MAEXXZ$23 10024768 f   setdefaults.obj
 0001:00023771       __unwindfunclet$?languageChange@setDefaultsBase@@MAEXXZ$24 10024771 f   setdefaults.obj
 0001:0002377a       __unwindfunclet$?languageChange@setDefaultsBase@@MAEXXZ$25 1002477a f   setdefaults.obj
 0001:00023783       __unwindfunclet$?languageChange@setDefaultsBase@@MAEXXZ$26 10024783 f   setdefaults.obj
 0001:0002378c       __unwindfunclet$?languageChange@setDefaultsBase@@MAEXXZ$27 1002478c f   setdefaults.obj
 0001:00023795       __unwindfunclet$?languageChange@setDefaultsBase@@MAEXXZ$28 10024795 f   setdefaults.obj
 0001:0002379e       __unwindfunclet$?languageChange@setDefaultsBase@@MAEXXZ$29 1002479e f   setdefaults.obj
 0001:000237a7       __unwindfunclet$?languageChange@setDefaultsBase@@MAEXXZ$30 100247a7 f   setdefaults.obj
 0001:000237b0       __unwindfunclet$?languageChange@setDefaultsBase@@MAEXXZ$31 100247b0 f   setdefaults.obj
 0001:000237b9       __unwindfunclet$?languageChange@setDefaultsBase@@MAEXXZ$32 100247b9 f   setdefaults.obj
 0001:000237c2       __unwindfunclet$?languageChange@setDefaultsBase@@MAEXXZ$33 100247c2 f   setdefaults.obj
 0001:000237cb       __unwindfunclet$?languageChange@setDefaultsBase@@MAEXXZ$34 100247cb f   setdefaults.obj
 0001:000237d4       __unwindfunclet$?languageChange@setDefaultsBase@@MAEXXZ$35 100247d4 f   setdefaults.obj
 0001:000237dd       __unwindfunclet$?languageChange@setDefaultsBase@@MAEXXZ$36 100247dd f   setdefaults.obj
 0001:000237e6       __unwindfunclet$?languageChange@setDefaultsBase@@MAEXXZ$37 100247e6 f   setdefaults.obj
 0001:000237ef       __unwindfunclet$?languageChange@setDefaultsBase@@MAEXXZ$38 100247ef f   setdefaults.obj
 0001:000237f8       __unwindfunclet$?languageChange@setDefaultsBase@@MAEXXZ$39 100247f8 f   setdefaults.obj
 0001:00023801       __unwindfunclet$?languageChange@setDefaultsBase@@MAEXXZ$40 10024801 f   setdefaults.obj
 0001:0002380a       __unwindfunclet$?languageChange@setDefaultsBase@@MAEXXZ$41 1002480a f   setdefaults.obj
 0001:00023813       __unwindfunclet$?languageChange@setDefaultsBase@@MAEXXZ$42 10024813 f   setdefaults.obj
 0001:0002381c       __unwindfunclet$?languageChange@setDefaultsBase@@MAEXXZ$43 1002481c f   setdefaults.obj
 0001:00023825       __ehhandler$?languageChange@setDefaultsBase@@MAEXXZ 10024825 f   setdefaults.obj
 0001:00023840       __unwindfunclet$??0setDefaults@@QAE@PAVQWidget@@PBD_NI@Z$0 10024840 f   setdefaultsimpl.obj
 0001:00023848       __unwindfunclet$??0setDefaults@@QAE@PAVQWidget@@PBD_NI@Z$1 10024848 f   setdefaultsimpl.obj
 0001:00023851       __unwindfunclet$??0setDefaults@@QAE@PAVQWidget@@PBD_NI@Z$2 10024851 f   setdefaultsimpl.obj
 0001:0002385a       __unwindfunclet$??0setDefaults@@QAE@PAVQWidget@@PBD_NI@Z$3 1002485a f   setdefaultsimpl.obj
 0001:00023863       __unwindfunclet$??0setDefaults@@QAE@PAVQWidget@@PBD_NI@Z$4 10024863 f   setdefaultsimpl.obj
 0001:0002386c       __unwindfunclet$??0setDefaults@@QAE@PAVQWidget@@PBD_NI@Z$5 1002486c f   setdefaultsimpl.obj
 0001:00023875       __unwindfunclet$??0setDefaults@@QAE@PAVQWidget@@PBD_NI@Z$6 10024875 f   setdefaultsimpl.obj
 0001:0002387e       __ehhandler$??0setDefaults@@QAE@PAVQWidget@@PBD_NI@Z 1002487e f   setdefaultsimpl.obj
 0001:00023899       __unwindfunclet$??0dialogBase@@QAE@PAVQWidget@@PBDI@Z$0 10024899 f   dialog.obj
 0001:000238a2       __unwindfunclet$??0dialogBase@@QAE@PAVQWidget@@PBDI@Z$1 100248a2 f   dialog.obj
 0001:000238ac       __unwindfunclet$??0dialogBase@@QAE@PAVQWidget@@PBDI@Z$2 100248ac f   dialog.obj
 0001:000238b6       __unwindfunclet$??0dialogBase@@QAE@PAVQWidget@@PBDI@Z$3 100248b6 f   dialog.obj
 0001:000238c0       __unwindfunclet$??0dialogBase@@QAE@PAVQWidget@@PBDI@Z$4 100248c0 f   dialog.obj
 0001:000238ca       __unwindfunclet$??0dialogBase@@QAE@PAVQWidget@@PBDI@Z$5 100248ca f   dialog.obj
 0001:000238d4       __unwindfunclet$??0dialogBase@@QAE@PAVQWidget@@PBDI@Z$6 100248d4 f   dialog.obj
 0001:000238de       __unwindfunclet$??0dialogBase@@QAE@PAVQWidget@@PBDI@Z$7 100248de f   dialog.obj
 0001:000238e8       __unwindfunclet$??0dialogBase@@QAE@PAVQWidget@@PBDI@Z$8 100248e8 f   dialog.obj
 0001:000238f2       __unwindfunclet$??0dialogBase@@QAE@PAVQWidget@@PBDI@Z$9 100248f2 f   dialog.obj
 0001:000238fc       __unwindfunclet$??0dialogBase@@QAE@PAVQWidget@@PBDI@Z$10 100248fc f   dialog.obj
 0001:00023906       __unwindfunclet$??0dialogBase@@QAE@PAVQWidget@@PBDI@Z$11 10024906 f   dialog.obj
 0001:00023910       __unwindfunclet$??0dialogBase@@QAE@PAVQWidget@@PBDI@Z$12 10024910 f   dialog.obj
 0001:0002391a       __unwindfunclet$??0dialogBase@@QAE@PAVQWidget@@PBDI@Z$13 1002491a f   dialog.obj
 0001:00023924       __unwindfunclet$??0dialogBase@@QAE@PAVQWidget@@PBDI@Z$14 10024924 f   dialog.obj
 0001:0002392e       __unwindfunclet$??0dialogBase@@QAE@PAVQWidget@@PBDI@Z$15 1002492e f   dialog.obj
 0001:00023938       __unwindfunclet$??0dialogBase@@QAE@PAVQWidget@@PBDI@Z$16 10024938 f   dialog.obj
 0001:00023942       __unwindfunclet$??0dialogBase@@QAE@PAVQWidget@@PBDI@Z$17 10024942 f   dialog.obj
 0001:0002394c       __unwindfunclet$??0dialogBase@@QAE@PAVQWidget@@PBDI@Z$18 1002494c f   dialog.obj
 0001:00023956       __unwindfunclet$??0dialogBase@@QAE@PAVQWidget@@PBDI@Z$19 10024956 f   dialog.obj
 0001:00023960       __unwindfunclet$??0dialogBase@@QAE@PAVQWidget@@PBDI@Z$20 10024960 f   dialog.obj
 0001:0002396a       __unwindfunclet$??0dialogBase@@QAE@PAVQWidget@@PBDI@Z$21 1002496a f   dialog.obj
 0001:00023974       __unwindfunclet$??0dialogBase@@QAE@PAVQWidget@@PBDI@Z$22 10024974 f   dialog.obj
 0001:0002397e       __unwindfunclet$??0dialogBase@@QAE@PAVQWidget@@PBDI@Z$23 1002497e f   dialog.obj
 0001:00023988       __unwindfunclet$??0dialogBase@@QAE@PAVQWidget@@PBDI@Z$24 10024988 f   dialog.obj
 0001:00023992       __unwindfunclet$??0dialogBase@@QAE@PAVQWidget@@PBDI@Z$25 10024992 f   dialog.obj
 0001:0002399c       __unwindfunclet$??0dialogBase@@QAE@PAVQWidget@@PBDI@Z$26 1002499c f   dialog.obj
 0001:000239a6       __unwindfunclet$??0dialogBase@@QAE@PAVQWidget@@PBDI@Z$27 100249a6 f   dialog.obj
 0001:000239b0       __unwindfunclet$??0dialogBase@@QAE@PAVQWidget@@PBDI@Z$28 100249b0 f   dialog.obj
 0001:000239ba       __unwindfunclet$??0dialogBase@@QAE@PAVQWidget@@PBDI@Z$29 100249ba f   dialog.obj
 0001:000239c4       __unwindfunclet$??0dialogBase@@QAE@PAVQWidget@@PBDI@Z$30 100249c4 f   dialog.obj
 0001:000239ce       __unwindfunclet$??0dialogBase@@QAE@PAVQWidget@@PBDI@Z$31 100249ce f   dialog.obj
 0001:000239d8       __unwindfunclet$??0dialogBase@@QAE@PAVQWidget@@PBDI@Z$32 100249d8 f   dialog.obj
 0001:000239e2       __unwindfunclet$??0dialogBase@@QAE@PAVQWidget@@PBDI@Z$33 100249e2 f   dialog.obj
 0001:000239ec       __unwindfunclet$??0dialogBase@@QAE@PAVQWidget@@PBDI@Z$34 100249ec f   dialog.obj
 0001:000239f6       __unwindfunclet$??0dialogBase@@QAE@PAVQWidget@@PBDI@Z$35 100249f6 f   dialog.obj
 0001:00023a00       __unwindfunclet$??0dialogBase@@QAE@PAVQWidget@@PBDI@Z$36 10024a00 f   dialog.obj
 0001:00023a0a       __unwindfunclet$??0dialogBase@@QAE@PAVQWidget@@PBDI@Z$37 10024a0a f   dialog.obj
 0001:00023a14       __unwindfunclet$??0dialogBase@@QAE@PAVQWidget@@PBDI@Z$38 10024a14 f   dialog.obj
 0001:00023a1e       __unwindfunclet$??0dialogBase@@QAE@PAVQWidget@@PBDI@Z$39 10024a1e f   dialog.obj
 0001:00023a28       __unwindfunclet$??0dialogBase@@QAE@PAVQWidget@@PBDI@Z$40 10024a28 f   dialog.obj
 0001:00023a32       __unwindfunclet$??0dialogBase@@QAE@PAVQWidget@@PBDI@Z$41 10024a32 f   dialog.obj
 0001:00023a3c       __unwindfunclet$??0dialogBase@@QAE@PAVQWidget@@PBDI@Z$42 10024a3c f   dialog.obj
 0001:00023a46       __unwindfunclet$??0dialogBase@@QAE@PAVQWidget@@PBDI@Z$43 10024a46 f   dialog.obj
 0001:00023a4f       __unwindfunclet$??0dialogBase@@QAE@PAVQWidget@@PBDI@Z$44 10024a4f f   dialog.obj
 0001:00023a59       __unwindfunclet$??0dialogBase@@QAE@PAVQWidget@@PBDI@Z$45 10024a59 f   dialog.obj
 0001:00023a63       __unwindfunclet$??0dialogBase@@QAE@PAVQWidget@@PBDI@Z$46 10024a63 f   dialog.obj
 0001:00023a6d       __unwindfunclet$??0dialogBase@@QAE@PAVQWidget@@PBDI@Z$47 10024a6d f   dialog.obj
 0001:00023a77       __unwindfunclet$??0dialogBase@@QAE@PAVQWidget@@PBDI@Z$48 10024a77 f   dialog.obj
 0001:00023a81       __unwindfunclet$??0dialogBase@@QAE@PAVQWidget@@PBDI@Z$49 10024a81 f   dialog.obj
 0001:00023a8b       __unwindfunclet$??0dialogBase@@QAE@PAVQWidget@@PBDI@Z$50 10024a8b f   dialog.obj
 0001:00023a95       __unwindfunclet$??0dialogBase@@QAE@PAVQWidget@@PBDI@Z$51 10024a95 f   dialog.obj
 0001:00023a9f       __unwindfunclet$??0dialogBase@@QAE@PAVQWidget@@PBDI@Z$52 10024a9f f   dialog.obj
 0001:00023aa9       __unwindfunclet$??0dialogBase@@QAE@PAVQWidget@@PBDI@Z$53 10024aa9 f   dialog.obj
 0001:00023ab3       __unwindfunclet$??0dialogBase@@QAE@PAVQWidget@@PBDI@Z$54 10024ab3 f   dialog.obj
 0001:00023abd       __unwindfunclet$??0dialogBase@@QAE@PAVQWidget@@PBDI@Z$55 10024abd f   dialog.obj
 0001:00023ac7       __unwindfunclet$??0dialogBase@@QAE@PAVQWidget@@PBDI@Z$56 10024ac7 f   dialog.obj
 0001:00023ad1       __unwindfunclet$??0dialogBase@@QAE@PAVQWidget@@PBDI@Z$57 10024ad1 f   dialog.obj
 0001:00023ada       __unwindfunclet$??0dialogBase@@QAE@PAVQWidget@@PBDI@Z$58 10024ada f   dialog.obj
 0001:00023ae3       __unwindfunclet$??0dialogBase@@QAE@PAVQWidget@@PBDI@Z$59 10024ae3 f   dialog.obj
 0001:00023aec       __unwindfunclet$??0dialogBase@@QAE@PAVQWidget@@PBDI@Z$60 10024aec f   dialog.obj
 0001:00023af5       __unwindfunclet$??0dialogBase@@QAE@PAVQWidget@@PBDI@Z$61 10024af5 f   dialog.obj
 0001:00023afe       __unwindfunclet$??0dialogBase@@QAE@PAVQWidget@@PBDI@Z$62 10024afe f   dialog.obj
 0001:00023b07       __unwindfunclet$??0dialogBase@@QAE@PAVQWidget@@PBDI@Z$63 10024b07 f   dialog.obj
 0001:00023b10       __unwindfunclet$??0dialogBase@@QAE@PAVQWidget@@PBDI@Z$64 10024b10 f   dialog.obj
 0001:00023b19       __unwindfunclet$??0dialogBase@@QAE@PAVQWidget@@PBDI@Z$65 10024b19 f   dialog.obj
 0001:00023b22       __unwindfunclet$??0dialogBase@@QAE@PAVQWidget@@PBDI@Z$66 10024b22 f   dialog.obj
 0001:00023b2b       __unwindfunclet$??0dialogBase@@QAE@PAVQWidget@@PBDI@Z$67 10024b2b f   dialog.obj
 0001:00023b34       __unwindfunclet$??0dialogBase@@QAE@PAVQWidget@@PBDI@Z$68 10024b34 f   dialog.obj
 0001:00023b3e       __unwindfunclet$??0dialogBase@@QAE@PAVQWidget@@PBDI@Z$69 10024b3e f   dialog.obj
 0001:00023b48       __unwindfunclet$??0dialogBase@@QAE@PAVQWidget@@PBDI@Z$70 10024b48 f   dialog.obj
 0001:00023b52       __unwindfunclet$??0dialogBase@@QAE@PAVQWidget@@PBDI@Z$71 10024b52 f   dialog.obj
 0001:00023b5c       __unwindfunclet$??0dialogBase@@QAE@PAVQWidget@@PBDI@Z$72 10024b5c f   dialog.obj
 0001:00023b66       __unwindfunclet$??0dialogBase@@QAE@PAVQWidget@@PBDI@Z$73 10024b66 f   dialog.obj
 0001:00023b70       __unwindfunclet$??0dialogBase@@QAE@PAVQWidget@@PBDI@Z$74 10024b70 f   dialog.obj
 0001:00023b7a       __unwindfunclet$??0dialogBase@@QAE@PAVQWidget@@PBDI@Z$75 10024b7a f   dialog.obj
 0001:00023b84       __unwindfunclet$??0dialogBase@@QAE@PAVQWidget@@PBDI@Z$76 10024b84 f   dialog.obj
 0001:00023b8e       __unwindfunclet$??0dialogBase@@QAE@PAVQWidget@@PBDI@Z$77 10024b8e f   dialog.obj
 0001:00023b98       __unwindfunclet$??0dialogBase@@QAE@PAVQWidget@@PBDI@Z$78 10024b98 f   dialog.obj
 0001:00023ba2       __unwindfunclet$??0dialogBase@@QAE@PAVQWidget@@PBDI@Z$79 10024ba2 f   dialog.obj
 0001:00023bac       __unwindfunclet$??0dialogBase@@QAE@PAVQWidget@@PBDI@Z$80 10024bac f   dialog.obj
 0001:00023bb6       __unwindfunclet$??0dialogBase@@QAE@PAVQWidget@@PBDI@Z$81 10024bb6 f   dialog.obj
 0001:00023bc0       __unwindfunclet$??0dialogBase@@QAE@PAVQWidget@@PBDI@Z$82 10024bc0 f   dialog.obj
 0001:00023bca       __unwindfunclet$??0dialogBase@@QAE@PAVQWidget@@PBDI@Z$83 10024bca f   dialog.obj
 0001:00023bd4       __unwindfunclet$??0dialogBase@@QAE@PAVQWidget@@PBDI@Z$84 10024bd4 f   dialog.obj
 0001:00023bde       __unwindfunclet$??0dialogBase@@QAE@PAVQWidget@@PBDI@Z$85 10024bde f   dialog.obj
 0001:00023be8       __unwindfunclet$??0dialogBase@@QAE@PAVQWidget@@PBDI@Z$86 10024be8 f   dialog.obj
 0001:00023bf2       __unwindfunclet$??0dialogBase@@QAE@PAVQWidget@@PBDI@Z$87 10024bf2 f   dialog.obj
 0001:00023bfc       __unwindfunclet$??0dialogBase@@QAE@PAVQWidget@@PBDI@Z$88 10024bfc f   dialog.obj
 0001:00023c06       __unwindfunclet$??0dialogBase@@QAE@PAVQWidget@@PBDI@Z$89 10024c06 f   dialog.obj
 0001:00023c10       __unwindfunclet$??0dialogBase@@QAE@PAVQWidget@@PBDI@Z$90 10024c10 f   dialog.obj
 0001:00023c1a       __unwindfunclet$??0dialogBase@@QAE@PAVQWidget@@PBDI@Z$91 10024c1a f   dialog.obj
 0001:00023c24       __unwindfunclet$??0dialogBase@@QAE@PAVQWidget@@PBDI@Z$92 10024c24 f   dialog.obj
 0001:00023c2e       __unwindfunclet$??0dialogBase@@QAE@PAVQWidget@@PBDI@Z$93 10024c2e f   dialog.obj
 0001:00023c38       __unwindfunclet$??0dialogBase@@QAE@PAVQWidget@@PBDI@Z$94 10024c38 f   dialog.obj
 0001:00023c42       __unwindfunclet$??0dialogBase@@QAE@PAVQWidget@@PBDI@Z$95 10024c42 f   dialog.obj
 0001:00023c4c       __unwindfunclet$??0dialogBase@@QAE@PAVQWidget@@PBDI@Z$96 10024c4c f   dialog.obj
 0001:00023c56       __unwindfunclet$??0dialogBase@@QAE@PAVQWidget@@PBDI@Z$97 10024c56 f   dialog.obj
 0001:00023c60       __unwindfunclet$??0dialogBase@@QAE@PAVQWidget@@PBDI@Z$98 10024c60 f   dialog.obj
 0001:00023c6a       __unwindfunclet$??0dialogBase@@QAE@PAVQWidget@@PBDI@Z$99 10024c6a f   dialog.obj
 0001:00023c74       __unwindfunclet$??0dialogBase@@QAE@PAVQWidget@@PBDI@Z$100 10024c74 f   dialog.obj
 0001:00023c7e       __unwindfunclet$??0dialogBase@@QAE@PAVQWidget@@PBDI@Z$101 10024c7e f   dialog.obj
 0001:00023c88       __unwindfunclet$??0dialogBase@@QAE@PAVQWidget@@PBDI@Z$102 10024c88 f   dialog.obj
 0001:00023c92       __unwindfunclet$??0dialogBase@@QAE@PAVQWidget@@PBDI@Z$103 10024c92 f   dialog.obj
 0001:00023c9c       __unwindfunclet$??0dialogBase@@QAE@PAVQWidget@@PBDI@Z$104 10024c9c f   dialog.obj
 0001:00023ca6       __unwindfunclet$??0dialogBase@@QAE@PAVQWidget@@PBDI@Z$105 10024ca6 f   dialog.obj
 0001:00023cb0       __unwindfunclet$??0dialogBase@@QAE@PAVQWidget@@PBDI@Z$106 10024cb0 f   dialog.obj
 0001:00023cba       __unwindfunclet$??0dialogBase@@QAE@PAVQWidget@@PBDI@Z$107 10024cba f   dialog.obj
 0001:00023cc4       __unwindfunclet$??0dialogBase@@QAE@PAVQWidget@@PBDI@Z$108 10024cc4 f   dialog.obj
 0001:00023cce       __unwindfunclet$??0dialogBase@@QAE@PAVQWidget@@PBDI@Z$109 10024cce f   dialog.obj
 0001:00023cd8       __unwindfunclet$??0dialogBase@@QAE@PAVQWidget@@PBDI@Z$110 10024cd8 f   dialog.obj
 0001:00023ce2       __unwindfunclet$??0dialogBase@@QAE@PAVQWidget@@PBDI@Z$111 10024ce2 f   dialog.obj
 0001:00023ceb       __unwindfunclet$??0dialogBase@@QAE@PAVQWidget@@PBDI@Z$112 10024ceb f   dialog.obj
 0001:00023cf5       __unwindfunclet$??0dialogBase@@QAE@PAVQWidget@@PBDI@Z$113 10024cf5 f   dialog.obj
 0001:00023cff       __unwindfunclet$??0dialogBase@@QAE@PAVQWidget@@PBDI@Z$114 10024cff f   dialog.obj
 0001:00023d09       __unwindfunclet$??0dialogBase@@QAE@PAVQWidget@@PBDI@Z$115 10024d09 f   dialog.obj
 0001:00023d13       __unwindfunclet$??0dialogBase@@QAE@PAVQWidget@@PBDI@Z$116 10024d13 f   dialog.obj
 0001:00023d1d       __unwindfunclet$??0dialogBase@@QAE@PAVQWidget@@PBDI@Z$117 10024d1d f   dialog.obj
 0001:00023d27       __unwindfunclet$??0dialogBase@@QAE@PAVQWidget@@PBDI@Z$118 10024d27 f   dialog.obj
 0001:00023d31       __unwindfunclet$??0dialogBase@@QAE@PAVQWidget@@PBDI@Z$119 10024d31 f   dialog.obj
 0001:00023d3b       __unwindfunclet$??0dialogBase@@QAE@PAVQWidget@@PBDI@Z$120 10024d3b f   dialog.obj
 0001:00023d45       __unwindfunclet$??0dialogBase@@QAE@PAVQWidget@@PBDI@Z$121 10024d45 f   dialog.obj
 0001:00023d4f       __unwindfunclet$??0dialogBase@@QAE@PAVQWidget@@PBDI@Z$122 10024d4f f   dialog.obj
 0001:00023d59       __unwindfunclet$??0dialogBase@@QAE@PAVQWidget@@PBDI@Z$123 10024d59 f   dialog.obj
 0001:00023d63       __unwindfunclet$??0dialogBase@@QAE@PAVQWidget@@PBDI@Z$124 10024d63 f   dialog.obj
 0001:00023d6d       __unwindfunclet$??0dialogBase@@QAE@PAVQWidget@@PBDI@Z$125 10024d6d f   dialog.obj
 0001:00023d77       __unwindfunclet$??0dialogBase@@QAE@PAVQWidget@@PBDI@Z$126 10024d77 f   dialog.obj
 0001:00023d81       __unwindfunclet$??0dialogBase@@QAE@PAVQWidget@@PBDI@Z$127 10024d81 f   dialog.obj
 0001:00023d8b       __unwindfunclet$??0dialogBase@@QAE@PAVQWidget@@PBDI@Z$128 10024d8b f   dialog.obj
 0001:00023d95       __unwindfunclet$??0dialogBase@@QAE@PAVQWidget@@PBDI@Z$129 10024d95 f   dialog.obj
 0001:00023d9f       __unwindfunclet$??0dialogBase@@QAE@PAVQWidget@@PBDI@Z$130 10024d9f f   dialog.obj
 0001:00023da9       __unwindfunclet$??0dialogBase@@QAE@PAVQWidget@@PBDI@Z$131 10024da9 f   dialog.obj
 0001:00023db3       __unwindfunclet$??0dialogBase@@QAE@PAVQWidget@@PBDI@Z$132 10024db3 f   dialog.obj
 0001:00023dbd       __unwindfunclet$??0dialogBase@@QAE@PAVQWidget@@PBDI@Z$133 10024dbd f   dialog.obj
 0001:00023dc7       __unwindfunclet$??0dialogBase@@QAE@PAVQWidget@@PBDI@Z$134 10024dc7 f   dialog.obj
 0001:00023dd1       __unwindfunclet$??0dialogBase@@QAE@PAVQWidget@@PBDI@Z$135 10024dd1 f   dialog.obj
 0001:00023ddb       __unwindfunclet$??0dialogBase@@QAE@PAVQWidget@@PBDI@Z$136 10024ddb f   dialog.obj
 0001:00023de5       __unwindfunclet$??0dialogBase@@QAE@PAVQWidget@@PBDI@Z$137 10024de5 f   dialog.obj
 0001:00023def       __unwindfunclet$??0dialogBase@@QAE@PAVQWidget@@PBDI@Z$138 10024def f   dialog.obj
 0001:00023df9       __unwindfunclet$??0dialogBase@@QAE@PAVQWidget@@PBDI@Z$139 10024df9 f   dialog.obj
 0001:00023e03       __unwindfunclet$??0dialogBase@@QAE@PAVQWidget@@PBDI@Z$140 10024e03 f   dialog.obj
 0001:00023e0d       __unwindfunclet$??0dialogBase@@QAE@PAVQWidget@@PBDI@Z$141 10024e0d f   dialog.obj
 0001:00023e17       __unwindfunclet$??0dialogBase@@QAE@PAVQWidget@@PBDI@Z$142 10024e17 f   dialog.obj
 0001:00023e21       __unwindfunclet$??0dialogBase@@QAE@PAVQWidget@@PBDI@Z$143 10024e21 f   dialog.obj
 0001:00023e2b       __unwindfunclet$??0dialogBase@@QAE@PAVQWidget@@PBDI@Z$144 10024e2b f   dialog.obj
 0001:00023e35       __unwindfunclet$??0dialogBase@@QAE@PAVQWidget@@PBDI@Z$145 10024e35 f   dialog.obj
 0001:00023e3f       __unwindfunclet$??0dialogBase@@QAE@PAVQWidget@@PBDI@Z$146 10024e3f f   dialog.obj
 0001:00023e49       __unwindfunclet$??0dialogBase@@QAE@PAVQWidget@@PBDI@Z$147 10024e49 f   dialog.obj
 0001:00023e53       __unwindfunclet$??0dialogBase@@QAE@PAVQWidget@@PBDI@Z$148 10024e53 f   dialog.obj
 0001:00023e5d       __unwindfunclet$??0dialogBase@@QAE@PAVQWidget@@PBDI@Z$149 10024e5d f   dialog.obj
 0001:00023e67       __unwindfunclet$??0dialogBase@@QAE@PAVQWidget@@PBDI@Z$150 10024e67 f   dialog.obj
 0001:00023e70       __unwindfunclet$??0dialogBase@@QAE@PAVQWidget@@PBDI@Z$151 10024e70 f   dialog.obj
 0001:00023e7a       __unwindfunclet$??0dialogBase@@QAE@PAVQWidget@@PBDI@Z$152 10024e7a f   dialog.obj
 0001:00023e84       __unwindfunclet$??0dialogBase@@QAE@PAVQWidget@@PBDI@Z$153 10024e84 f   dialog.obj
 0001:00023e8e       __unwindfunclet$??0dialogBase@@QAE@PAVQWidget@@PBDI@Z$154 10024e8e f   dialog.obj
 0001:00023e98       __unwindfunclet$??0dialogBase@@QAE@PAVQWidget@@PBDI@Z$155 10024e98 f   dialog.obj
 0001:00023ea2       __unwindfunclet$??0dialogBase@@QAE@PAVQWidget@@PBDI@Z$156 10024ea2 f   dialog.obj
 0001:00023eac       __unwindfunclet$??0dialogBase@@QAE@PAVQWidget@@PBDI@Z$157 10024eac f   dialog.obj
 0001:00023eb6       __unwindfunclet$??0dialogBase@@QAE@PAVQWidget@@PBDI@Z$158 10024eb6 f   dialog.obj
 0001:00023ec0       __unwindfunclet$??0dialogBase@@QAE@PAVQWidget@@PBDI@Z$159 10024ec0 f   dialog.obj
 0001:00023eca       __unwindfunclet$??0dialogBase@@QAE@PAVQWidget@@PBDI@Z$160 10024eca f   dialog.obj
 0001:00023ed4       __unwindfunclet$??0dialogBase@@QAE@PAVQWidget@@PBDI@Z$161 10024ed4 f   dialog.obj
 0001:00023ede       __unwindfunclet$??0dialogBase@@QAE@PAVQWidget@@PBDI@Z$162 10024ede f   dialog.obj
 0001:00023ee8       __unwindfunclet$??0dialogBase@@QAE@PAVQWidget@@PBDI@Z$163 10024ee8 f   dialog.obj
 0001:00023ef2       __unwindfunclet$??0dialogBase@@QAE@PAVQWidget@@PBDI@Z$164 10024ef2 f   dialog.obj
 0001:00023efc       __unwindfunclet$??0dialogBase@@QAE@PAVQWidget@@PBDI@Z$165 10024efc f   dialog.obj
 0001:00023f06       __unwindfunclet$??0dialogBase@@QAE@PAVQWidget@@PBDI@Z$166 10024f06 f   dialog.obj
 0001:00023f10       __unwindfunclet$??0dialogBase@@QAE@PAVQWidget@@PBDI@Z$167 10024f10 f   dialog.obj
 0001:00023f1a       __unwindfunclet$??0dialogBase@@QAE@PAVQWidget@@PBDI@Z$168 10024f1a f   dialog.obj
 0001:00023f24       __unwindfunclet$??0dialogBase@@QAE@PAVQWidget@@PBDI@Z$169 10024f24 f   dialog.obj
 0001:00023f2e       __unwindfunclet$??0dialogBase@@QAE@PAVQWidget@@PBDI@Z$170 10024f2e f   dialog.obj
 0001:00023f38       __unwindfunclet$??0dialogBase@@QAE@PAVQWidget@@PBDI@Z$171 10024f38 f   dialog.obj
 0001:00023f42       __unwindfunclet$??0dialogBase@@QAE@PAVQWidget@@PBDI@Z$172 10024f42 f   dialog.obj
 0001:00023f4c       __unwindfunclet$??0dialogBase@@QAE@PAVQWidget@@PBDI@Z$173 10024f4c f   dialog.obj
 0001:00023f56       __unwindfunclet$??0dialogBase@@QAE@PAVQWidget@@PBDI@Z$174 10024f56 f   dialog.obj
 0001:00023f60       __unwindfunclet$??0dialogBase@@QAE@PAVQWidget@@PBDI@Z$175 10024f60 f   dialog.obj
 0001:00023f6a       __unwindfunclet$??0dialogBase@@QAE@PAVQWidget@@PBDI@Z$176 10024f6a f   dialog.obj
 0001:00023f73       __unwindfunclet$??0dialogBase@@QAE@PAVQWidget@@PBDI@Z$177 10024f73 f   dialog.obj
 0001:00023f7c       __unwindfunclet$??0dialogBase@@QAE@PAVQWidget@@PBDI@Z$178 10024f7c f   dialog.obj
 0001:00023f86       __unwindfunclet$??0dialogBase@@QAE@PAVQWidget@@PBDI@Z$179 10024f86 f   dialog.obj
 0001:00023f90       __unwindfunclet$??0dialogBase@@QAE@PAVQWidget@@PBDI@Z$180 10024f90 f   dialog.obj
 0001:00023f9a       __unwindfunclet$??0dialogBase@@QAE@PAVQWidget@@PBDI@Z$181 10024f9a f   dialog.obj
 0001:00023fa4       __unwindfunclet$??0dialogBase@@QAE@PAVQWidget@@PBDI@Z$182 10024fa4 f   dialog.obj
 0001:00023fae       __unwindfunclet$??0dialogBase@@QAE@PAVQWidget@@PBDI@Z$183 10024fae f   dialog.obj
 0001:00023fb8       __unwindfunclet$??0dialogBase@@QAE@PAVQWidget@@PBDI@Z$184 10024fb8 f   dialog.obj
 0001:00023fc2       __unwindfunclet$??0dialogBase@@QAE@PAVQWidget@@PBDI@Z$185 10024fc2 f   dialog.obj
 0001:00023fcc       __unwindfunclet$??0dialogBase@@QAE@PAVQWidget@@PBDI@Z$186 10024fcc f   dialog.obj
 0001:00023fd6       __unwindfunclet$??0dialogBase@@QAE@PAVQWidget@@PBDI@Z$187 10024fd6 f   dialog.obj
 0001:00023fe0       __unwindfunclet$??0dialogBase@@QAE@PAVQWidget@@PBDI@Z$188 10024fe0 f   dialog.obj
 0001:00023fea       __unwindfunclet$??0dialogBase@@QAE@PAVQWidget@@PBDI@Z$189 10024fea f   dialog.obj
 0001:00023ff4       __unwindfunclet$??0dialogBase@@QAE@PAVQWidget@@PBDI@Z$190 10024ff4 f   dialog.obj
 0001:00023ffe       __unwindfunclet$??0dialogBase@@QAE@PAVQWidget@@PBDI@Z$191 10024ffe f   dialog.obj
 0001:00024008       __unwindfunclet$??0dialogBase@@QAE@PAVQWidget@@PBDI@Z$192 10025008 f   dialog.obj
 0001:00024012       __unwindfunclet$??0dialogBase@@QAE@PAVQWidget@@PBDI@Z$193 10025012 f   dialog.obj
 0001:0002401b       __unwindfunclet$??0dialogBase@@QAE@PAVQWidget@@PBDI@Z$194 1002501b f   dialog.obj
 0001:00024025       __unwindfunclet$??0dialogBase@@QAE@PAVQWidget@@PBDI@Z$195 10025025 f   dialog.obj
 0001:0002402e       __ehhandler$??0dialogBase@@QAE@PAVQWidget@@PBDI@Z 1002502e f   dialog.obj
 0001:00024049       __unwindfunclet$?languageChange@dialogBase@@MAEXXZ$0 10025049 f   dialog.obj
 0001:00024052       __unwindfunclet$?languageChange@dialogBase@@MAEXXZ$1 10025052 f   dialog.obj
 0001:0002405b       __unwindfunclet$?languageChange@dialogBase@@MAEXXZ$2 1002505b f   dialog.obj
 0001:00024064       __unwindfunclet$?languageChange@dialogBase@@MAEXXZ$3 10025064 f   dialog.obj
 0001:0002406d       __unwindfunclet$?languageChange@dialogBase@@MAEXXZ$4 1002506d f   dialog.obj
 0001:00024076       __unwindfunclet$?languageChange@dialogBase@@MAEXXZ$5 10025076 f   dialog.obj
 0001:0002407f       __unwindfunclet$?languageChange@dialogBase@@MAEXXZ$6 1002507f f   dialog.obj
 0001:00024088       __unwindfunclet$?languageChange@dialogBase@@MAEXXZ$7 10025088 f   dialog.obj
 0001:00024091       __unwindfunclet$?languageChange@dialogBase@@MAEXXZ$8 10025091 f   dialog.obj
 0001:0002409a       __unwindfunclet$?languageChange@dialogBase@@MAEXXZ$9 1002509a f   dialog.obj
 0001:000240a3       __unwindfunclet$?languageChange@dialogBase@@MAEXXZ$10 100250a3 f   dialog.obj
 0001:000240ac       __unwindfunclet$?languageChange@dialogBase@@MAEXXZ$11 100250ac f   dialog.obj
 0001:000240b5       __unwindfunclet$?languageChange@dialogBase@@MAEXXZ$12 100250b5 f   dialog.obj
 0001:000240be       __unwindfunclet$?languageChange@dialogBase@@MAEXXZ$13 100250be f   dialog.obj
 0001:000240c7       __unwindfunclet$?languageChange@dialogBase@@MAEXXZ$14 100250c7 f   dialog.obj
 0001:000240d0       __unwindfunclet$?languageChange@dialogBase@@MAEXXZ$15 100250d0 f   dialog.obj
 0001:000240d9       __unwindfunclet$?languageChange@dialogBase@@MAEXXZ$16 100250d9 f   dialog.obj
 0001:000240e2       __unwindfunclet$?languageChange@dialogBase@@MAEXXZ$17 100250e2 f   dialog.obj
 0001:000240eb       __unwindfunclet$?languageChange@dialogBase@@MAEXXZ$18 100250eb f   dialog.obj
 0001:000240f4       __unwindfunclet$?languageChange@dialogBase@@MAEXXZ$19 100250f4 f   dialog.obj
 0001:000240fd       __unwindfunclet$?languageChange@dialogBase@@MAEXXZ$20 100250fd f   dialog.obj
 0001:00024106       __unwindfunclet$?languageChange@dialogBase@@MAEXXZ$21 10025106 f   dialog.obj
 0001:0002410f       __unwindfunclet$?languageChange@dialogBase@@MAEXXZ$22 1002510f f   dialog.obj
 0001:00024118       __unwindfunclet$?languageChange@dialogBase@@MAEXXZ$23 10025118 f   dialog.obj
 0001:00024121       __unwindfunclet$?languageChange@dialogBase@@MAEXXZ$24 10025121 f   dialog.obj
 0001:0002412a       __unwindfunclet$?languageChange@dialogBase@@MAEXXZ$25 1002512a f   dialog.obj
 0001:00024133       __unwindfunclet$?languageChange@dialogBase@@MAEXXZ$26 10025133 f   dialog.obj
 0001:0002413c       __unwindfunclet$?languageChange@dialogBase@@MAEXXZ$27 1002513c f   dialog.obj
 0001:00024145       __unwindfunclet$?languageChange@dialogBase@@MAEXXZ$28 10025145 f   dialog.obj
 0001:0002414e       __unwindfunclet$?languageChange@dialogBase@@MAEXXZ$29 1002514e f   dialog.obj
 0001:00024157       __unwindfunclet$?languageChange@dialogBase@@MAEXXZ$30 10025157 f   dialog.obj
 0001:00024160       __unwindfunclet$?languageChange@dialogBase@@MAEXXZ$31 10025160 f   dialog.obj
 0001:00024169       __unwindfunclet$?languageChange@dialogBase@@MAEXXZ$32 10025169 f   dialog.obj
 0001:00024172       __unwindfunclet$?languageChange@dialogBase@@MAEXXZ$33 10025172 f   dialog.obj
 0001:0002417b       __unwindfunclet$?languageChange@dialogBase@@MAEXXZ$34 1002517b f   dialog.obj
 0001:00024184       __unwindfunclet$?languageChange@dialogBase@@MAEXXZ$35 10025184 f   dialog.obj
 0001:0002418d       __unwindfunclet$?languageChange@dialogBase@@MAEXXZ$36 1002518d f   dialog.obj
 0001:00024196       __unwindfunclet$?languageChange@dialogBase@@MAEXXZ$37 10025196 f   dialog.obj
 0001:0002419f       __unwindfunclet$?languageChange@dialogBase@@MAEXXZ$38 1002519f f   dialog.obj
 0001:000241a8       __unwindfunclet$?languageChange@dialogBase@@MAEXXZ$39 100251a8 f   dialog.obj
 0001:000241b1       __unwindfunclet$?languageChange@dialogBase@@MAEXXZ$40 100251b1 f   dialog.obj
 0001:000241ba       __unwindfunclet$?languageChange@dialogBase@@MAEXXZ$41 100251ba f   dialog.obj
 0001:000241c3       __unwindfunclet$?languageChange@dialogBase@@MAEXXZ$42 100251c3 f   dialog.obj
 0001:000241cc       __unwindfunclet$?languageChange@dialogBase@@MAEXXZ$43 100251cc f   dialog.obj
 0001:000241d5       __unwindfunclet$?languageChange@dialogBase@@MAEXXZ$44 100251d5 f   dialog.obj
 0001:000241de       __unwindfunclet$?languageChange@dialogBase@@MAEXXZ$45 100251de f   dialog.obj
 0001:000241e7       __unwindfunclet$?languageChange@dialogBase@@MAEXXZ$46 100251e7 f   dialog.obj
 0001:000241f0       __unwindfunclet$?languageChange@dialogBase@@MAEXXZ$47 100251f0 f   dialog.obj
 0001:000241f9       __unwindfunclet$?languageChange@dialogBase@@MAEXXZ$48 100251f9 f   dialog.obj
 0001:00024202       __unwindfunclet$?languageChange@dialogBase@@MAEXXZ$49 10025202 f   dialog.obj
 0001:0002420b       __unwindfunclet$?languageChange@dialogBase@@MAEXXZ$50 1002520b f   dialog.obj
 0001:00024214       __unwindfunclet$?languageChange@dialogBase@@MAEXXZ$51 10025214 f   dialog.obj
 0001:0002421d       __unwindfunclet$?languageChange@dialogBase@@MAEXXZ$52 1002521d f   dialog.obj
 0001:00024226       __unwindfunclet$?languageChange@dialogBase@@MAEXXZ$53 10025226 f   dialog.obj
 0001:0002422f       __unwindfunclet$?languageChange@dialogBase@@MAEXXZ$54 1002522f f   dialog.obj
 0001:00024238       __unwindfunclet$?languageChange@dialogBase@@MAEXXZ$55 10025238 f   dialog.obj
 0001:00024241       __unwindfunclet$?languageChange@dialogBase@@MAEXXZ$56 10025241 f   dialog.obj
 0001:0002424a       __unwindfunclet$?languageChange@dialogBase@@MAEXXZ$57 1002524a f   dialog.obj
 0001:00024253       __unwindfunclet$?languageChange@dialogBase@@MAEXXZ$58 10025253 f   dialog.obj
 0001:0002425c       __unwindfunclet$?languageChange@dialogBase@@MAEXXZ$59 1002525c f   dialog.obj
 0001:00024265       __unwindfunclet$?languageChange@dialogBase@@MAEXXZ$60 10025265 f   dialog.obj
 0001:0002426e       __unwindfunclet$?languageChange@dialogBase@@MAEXXZ$61 1002526e f   dialog.obj
 0001:00024277       __unwindfunclet$?languageChange@dialogBase@@MAEXXZ$62 10025277 f   dialog.obj
 0001:00024280       __unwindfunclet$?languageChange@dialogBase@@MAEXXZ$63 10025280 f   dialog.obj
 0001:00024289       __unwindfunclet$?languageChange@dialogBase@@MAEXXZ$64 10025289 f   dialog.obj
 0001:00024295       __unwindfunclet$?languageChange@dialogBase@@MAEXXZ$65 10025295 f   dialog.obj
 0001:0002429e       __unwindfunclet$?languageChange@dialogBase@@MAEXXZ$66 1002529e f   dialog.obj
 0001:000242aa       __unwindfunclet$?languageChange@dialogBase@@MAEXXZ$67 100252aa f   dialog.obj
 0001:000242b3       __unwindfunclet$?languageChange@dialogBase@@MAEXXZ$68 100252b3 f   dialog.obj
 0001:000242bf       __unwindfunclet$?languageChange@dialogBase@@MAEXXZ$69 100252bf f   dialog.obj
 0001:000242c8       __unwindfunclet$?languageChange@dialogBase@@MAEXXZ$70 100252c8 f   dialog.obj
 0001:000242d4       __unwindfunclet$?languageChange@dialogBase@@MAEXXZ$71 100252d4 f   dialog.obj
 0001:000242dd       __unwindfunclet$?languageChange@dialogBase@@MAEXXZ$72 100252dd f   dialog.obj
 0001:000242e9       __unwindfunclet$?languageChange@dialogBase@@MAEXXZ$73 100252e9 f   dialog.obj
 0001:000242f2       __unwindfunclet$?languageChange@dialogBase@@MAEXXZ$74 100252f2 f   dialog.obj
 0001:000242fe       __unwindfunclet$?languageChange@dialogBase@@MAEXXZ$75 100252fe f   dialog.obj
 0001:00024307       __unwindfunclet$?languageChange@dialogBase@@MAEXXZ$76 10025307 f   dialog.obj
 0001:00024313       __unwindfunclet$?languageChange@dialogBase@@MAEXXZ$77 10025313 f   dialog.obj
 0001:0002431c       __unwindfunclet$?languageChange@dialogBase@@MAEXXZ$78 1002531c f   dialog.obj
 0001:00024328       __unwindfunclet$?languageChange@dialogBase@@MAEXXZ$79 10025328 f   dialog.obj
 0001:00024331       __unwindfunclet$?languageChange@dialogBase@@MAEXXZ$80 10025331 f   dialog.obj
 0001:0002433d       __unwindfunclet$?languageChange@dialogBase@@MAEXXZ$81 1002533d f   dialog.obj
 0001:00024346       __unwindfunclet$?languageChange@dialogBase@@MAEXXZ$82 10025346 f   dialog.obj
 0001:00024352       __unwindfunclet$?languageChange@dialogBase@@MAEXXZ$83 10025352 f   dialog.obj
 0001:0002435b       __unwindfunclet$?languageChange@dialogBase@@MAEXXZ$84 1002535b f   dialog.obj
 0001:00024367       __unwindfunclet$?languageChange@dialogBase@@MAEXXZ$85 10025367 f   dialog.obj
 0001:00024370       __unwindfunclet$?languageChange@dialogBase@@MAEXXZ$86 10025370 f   dialog.obj
 0001:0002437c       __unwindfunclet$?languageChange@dialogBase@@MAEXXZ$87 1002537c f   dialog.obj
 0001:00024385       __unwindfunclet$?languageChange@dialogBase@@MAEXXZ$88 10025385 f   dialog.obj
 0001:00024391       __unwindfunclet$?languageChange@dialogBase@@MAEXXZ$89 10025391 f   dialog.obj
 0001:0002439a       __unwindfunclet$?languageChange@dialogBase@@MAEXXZ$90 1002539a f   dialog.obj
 0001:000243a6       __unwindfunclet$?languageChange@dialogBase@@MAEXXZ$91 100253a6 f   dialog.obj
 0001:000243b2       __unwindfunclet$?languageChange@dialogBase@@MAEXXZ$92 100253b2 f   dialog.obj
 0001:000243be       __unwindfunclet$?languageChange@dialogBase@@MAEXXZ$93 100253be f   dialog.obj
 0001:000243ca       __unwindfunclet$?languageChange@dialogBase@@MAEXXZ$94 100253ca f   dialog.obj
 0001:000243d3       __unwindfunclet$?languageChange@dialogBase@@MAEXXZ$95 100253d3 f   dialog.obj
 0001:000243df       __unwindfunclet$?languageChange@dialogBase@@MAEXXZ$96 100253df f   dialog.obj
 0001:000243e8       __unwindfunclet$?languageChange@dialogBase@@MAEXXZ$97 100253e8 f   dialog.obj
 0001:000243f1       __unwindfunclet$?languageChange@dialogBase@@MAEXXZ$98 100253f1 f   dialog.obj
 0001:000243fa       __unwindfunclet$?languageChange@dialogBase@@MAEXXZ$99 100253fa f   dialog.obj
 0001:00024403       __unwindfunclet$?languageChange@dialogBase@@MAEXXZ$100 10025403 f   dialog.obj
 0001:0002440c       __unwindfunclet$?languageChange@dialogBase@@MAEXXZ$101 1002540c f   dialog.obj
 0001:00024415       __unwindfunclet$?languageChange@dialogBase@@MAEXXZ$102 10025415 f   dialog.obj
 0001:0002441e       __unwindfunclet$?languageChange@dialogBase@@MAEXXZ$103 1002541e f   dialog.obj
 0001:00024427       __unwindfunclet$?languageChange@dialogBase@@MAEXXZ$104 10025427 f   dialog.obj
 0001:00024430       __unwindfunclet$?languageChange@dialogBase@@MAEXXZ$105 10025430 f   dialog.obj
 0001:00024439       __unwindfunclet$?languageChange@dialogBase@@MAEXXZ$106 10025439 f   dialog.obj
 0001:00024442       __unwindfunclet$?languageChange@dialogBase@@MAEXXZ$107 10025442 f   dialog.obj
 0001:0002444b       __unwindfunclet$?languageChange@dialogBase@@MAEXXZ$108 1002544b f   dialog.obj
 0001:00024454       __unwindfunclet$?languageChange@dialogBase@@MAEXXZ$109 10025454 f   dialog.obj
 0001:00024460       __unwindfunclet$?languageChange@dialogBase@@MAEXXZ$110 10025460 f   dialog.obj
 0001:0002446c       __unwindfunclet$?languageChange@dialogBase@@MAEXXZ$111 1002546c f   dialog.obj
 0001:00024478       __unwindfunclet$?languageChange@dialogBase@@MAEXXZ$112 10025478 f   dialog.obj
 0001:00024484       __unwindfunclet$?languageChange@dialogBase@@MAEXXZ$113 10025484 f   dialog.obj
 0001:00024490       __unwindfunclet$?languageChange@dialogBase@@MAEXXZ$114 10025490 f   dialog.obj
 0001:0002449c       __unwindfunclet$?languageChange@dialogBase@@MAEXXZ$115 1002549c f   dialog.obj
 0001:000244a8       __unwindfunclet$?languageChange@dialogBase@@MAEXXZ$116 100254a8 f   dialog.obj
 0001:000244b4       __unwindfunclet$?languageChange@dialogBase@@MAEXXZ$117 100254b4 f   dialog.obj
 0001:000244c0       __unwindfunclet$?languageChange@dialogBase@@MAEXXZ$118 100254c0 f   dialog.obj
 0001:000244cc       __unwindfunclet$?languageChange@dialogBase@@MAEXXZ$119 100254cc f   dialog.obj
 0001:000244d8       __unwindfunclet$?languageChange@dialogBase@@MAEXXZ$120 100254d8 f   dialog.obj
 0001:000244e4       __unwindfunclet$?languageChange@dialogBase@@MAEXXZ$121 100254e4 f   dialog.obj
 0001:000244f0       __unwindfunclet$?languageChange@dialogBase@@MAEXXZ$122 100254f0 f   dialog.obj
 0001:000244fc       __unwindfunclet$?languageChange@dialogBase@@MAEXXZ$123 100254fc f   dialog.obj
 0001:00024508       __unwindfunclet$?languageChange@dialogBase@@MAEXXZ$124 10025508 f   dialog.obj
 0001:00024514       __unwindfunclet$?languageChange@dialogBase@@MAEXXZ$125 10025514 f   dialog.obj
 0001:00024520       __unwindfunclet$?languageChange@dialogBase@@MAEXXZ$126 10025520 f   dialog.obj
 0001:0002452c       __unwindfunclet$?languageChange@dialogBase@@MAEXXZ$127 1002552c f   dialog.obj
 0001:00024538       __ehhandler$?languageChange@dialogBase@@MAEXXZ 10025538 f   dialog.obj
 0001:00024556       __unwindfunclet$??0manage_tempBase@@QAE@PAVQWidget@@PBD_NI@Z$0 10025556 f   manage_temp.obj
 0001:0002455f       __unwindfunclet$??0manage_tempBase@@QAE@PAVQWidget@@PBD_NI@Z$1 1002555f f   manage_temp.obj
 0001:00024569       __unwindfunclet$??0manage_tempBase@@QAE@PAVQWidget@@PBD_NI@Z$2 10025569 f   manage_temp.obj
 0001:00024573       __unwindfunclet$??0manage_tempBase@@QAE@PAVQWidget@@PBD_NI@Z$3 10025573 f   manage_temp.obj
 0001:0002457d       __unwindfunclet$??0manage_tempBase@@QAE@PAVQWidget@@PBD_NI@Z$4 1002557d f   manage_temp.obj
 0001:00024587       __unwindfunclet$??0manage_tempBase@@QAE@PAVQWidget@@PBD_NI@Z$5 10025587 f   manage_temp.obj
 0001:00024591       __unwindfunclet$??0manage_tempBase@@QAE@PAVQWidget@@PBD_NI@Z$6 10025591 f   manage_temp.obj
 0001:0002459b       __unwindfunclet$??0manage_tempBase@@QAE@PAVQWidget@@PBD_NI@Z$7 1002559b f   manage_temp.obj
 0001:000245a5       __unwindfunclet$??0manage_tempBase@@QAE@PAVQWidget@@PBD_NI@Z$8 100255a5 f   manage_temp.obj
 0001:000245af       __unwindfunclet$??0manage_tempBase@@QAE@PAVQWidget@@PBD_NI@Z$9 100255af f   manage_temp.obj
 0001:000245b9       __unwindfunclet$??0manage_tempBase@@QAE@PAVQWidget@@PBD_NI@Z$10 100255b9 f   manage_temp.obj
 0001:000245c3       __unwindfunclet$??0manage_tempBase@@QAE@PAVQWidget@@PBD_NI@Z$11 100255c3 f   manage_temp.obj
 0001:000245cd       __unwindfunclet$??0manage_tempBase@@QAE@PAVQWidget@@PBD_NI@Z$12 100255cd f   manage_temp.obj
 0001:000245d6       __unwindfunclet$??0manage_tempBase@@QAE@PAVQWidget@@PBD_NI@Z$13 100255d6 f   manage_temp.obj
 0001:000245df       __unwindfunclet$??0manage_tempBase@@QAE@PAVQWidget@@PBD_NI@Z$14 100255df f   manage_temp.obj
 0001:000245e8       __unwindfunclet$??0manage_tempBase@@QAE@PAVQWidget@@PBD_NI@Z$15 100255e8 f   manage_temp.obj
 0001:000245f1       __unwindfunclet$??0manage_tempBase@@QAE@PAVQWidget@@PBD_NI@Z$16 100255f1 f   manage_temp.obj
 0001:000245fa       __unwindfunclet$??0manage_tempBase@@QAE@PAVQWidget@@PBD_NI@Z$17 100255fa f   manage_temp.obj
 0001:00024603       __unwindfunclet$??0manage_tempBase@@QAE@PAVQWidget@@PBD_NI@Z$18 10025603 f   manage_temp.obj
 0001:0002460c       __unwindfunclet$??0manage_tempBase@@QAE@PAVQWidget@@PBD_NI@Z$19 1002560c f   manage_temp.obj
 0001:00024615       __unwindfunclet$??0manage_tempBase@@QAE@PAVQWidget@@PBD_NI@Z$20 10025615 f   manage_temp.obj
 0001:0002461e       __unwindfunclet$??0manage_tempBase@@QAE@PAVQWidget@@PBD_NI@Z$21 1002561e f   manage_temp.obj
 0001:00024627       __unwindfunclet$??0manage_tempBase@@QAE@PAVQWidget@@PBD_NI@Z$22 10025627 f   manage_temp.obj
 0001:00024631       __unwindfunclet$??0manage_tempBase@@QAE@PAVQWidget@@PBD_NI@Z$23 10025631 f   manage_temp.obj
 0001:0002463b       __unwindfunclet$??0manage_tempBase@@QAE@PAVQWidget@@PBD_NI@Z$24 1002563b f   manage_temp.obj
 0001:00024645       __unwindfunclet$??0manage_tempBase@@QAE@PAVQWidget@@PBD_NI@Z$25 10025645 f   manage_temp.obj
 0001:0002464f       __unwindfunclet$??0manage_tempBase@@QAE@PAVQWidget@@PBD_NI@Z$26 1002564f f   manage_temp.obj
 0001:00024659       __unwindfunclet$??0manage_tempBase@@QAE@PAVQWidget@@PBD_NI@Z$27 10025659 f   manage_temp.obj
 0001:00024663       __unwindfunclet$??0manage_tempBase@@QAE@PAVQWidget@@PBD_NI@Z$28 10025663 f   manage_temp.obj
 0001:0002466d       __unwindfunclet$??0manage_tempBase@@QAE@PAVQWidget@@PBD_NI@Z$29 1002566d f   manage_temp.obj
 0001:00024677       __unwindfunclet$??0manage_tempBase@@QAE@PAVQWidget@@PBD_NI@Z$30 10025677 f   manage_temp.obj
 0001:00024681       __unwindfunclet$??0manage_tempBase@@QAE@PAVQWidget@@PBD_NI@Z$31 10025681 f   manage_temp.obj
 0001:0002468b       __unwindfunclet$??0manage_tempBase@@QAE@PAVQWidget@@PBD_NI@Z$32 1002568b f   manage_temp.obj
 0001:00024695       __unwindfunclet$??0manage_tempBase@@QAE@PAVQWidget@@PBD_NI@Z$33 10025695 f   manage_temp.obj
 0001:0002469f       __unwindfunclet$??0manage_tempBase@@QAE@PAVQWidget@@PBD_NI@Z$34 1002569f f   manage_temp.obj
 0001:000246a9       __unwindfunclet$??0manage_tempBase@@QAE@PAVQWidget@@PBD_NI@Z$35 100256a9 f   manage_temp.obj
 0001:000246b3       __unwindfunclet$??0manage_tempBase@@QAE@PAVQWidget@@PBD_NI@Z$36 100256b3 f   manage_temp.obj
 0001:000246bd       __unwindfunclet$??0manage_tempBase@@QAE@PAVQWidget@@PBD_NI@Z$37 100256bd f   manage_temp.obj
 0001:000246c7       __unwindfunclet$??0manage_tempBase@@QAE@PAVQWidget@@PBD_NI@Z$38 100256c7 f   manage_temp.obj
 0001:000246d1       __unwindfunclet$??0manage_tempBase@@QAE@PAVQWidget@@PBD_NI@Z$39 100256d1 f   manage_temp.obj
 0001:000246db       __unwindfunclet$??0manage_tempBase@@QAE@PAVQWidget@@PBD_NI@Z$40 100256db f   manage_temp.obj
 0001:000246e5       __unwindfunclet$??0manage_tempBase@@QAE@PAVQWidget@@PBD_NI@Z$41 100256e5 f   manage_temp.obj
 0001:000246ef       __unwindfunclet$??0manage_tempBase@@QAE@PAVQWidget@@PBD_NI@Z$42 100256ef f   manage_temp.obj
 0001:000246f9       __unwindfunclet$??0manage_tempBase@@QAE@PAVQWidget@@PBD_NI@Z$43 100256f9 f   manage_temp.obj
 0001:00024703       __unwindfunclet$??0manage_tempBase@@QAE@PAVQWidget@@PBD_NI@Z$44 10025703 f   manage_temp.obj
 0001:0002470d       __unwindfunclet$??0manage_tempBase@@QAE@PAVQWidget@@PBD_NI@Z$45 1002570d f   manage_temp.obj
 0001:00024717       __unwindfunclet$??0manage_tempBase@@QAE@PAVQWidget@@PBD_NI@Z$46 10025717 f   manage_temp.obj
 0001:00024721       __unwindfunclet$??0manage_tempBase@@QAE@PAVQWidget@@PBD_NI@Z$47 10025721 f   manage_temp.obj
 0001:0002472b       __unwindfunclet$??0manage_tempBase@@QAE@PAVQWidget@@PBD_NI@Z$48 1002572b f   manage_temp.obj
 0001:00024735       __unwindfunclet$??0manage_tempBase@@QAE@PAVQWidget@@PBD_NI@Z$49 10025735 f   manage_temp.obj
 0001:0002473f       __unwindfunclet$??0manage_tempBase@@QAE@PAVQWidget@@PBD_NI@Z$50 1002573f f   manage_temp.obj
 0001:00024749       __unwindfunclet$??0manage_tempBase@@QAE@PAVQWidget@@PBD_NI@Z$51 10025749 f   manage_temp.obj
 0001:00024753       __unwindfunclet$??0manage_tempBase@@QAE@PAVQWidget@@PBD_NI@Z$52 10025753 f   manage_temp.obj
 0001:0002475d       __unwindfunclet$??0manage_tempBase@@QAE@PAVQWidget@@PBD_NI@Z$53 1002575d f   manage_temp.obj
 0001:00024767       __unwindfunclet$??0manage_tempBase@@QAE@PAVQWidget@@PBD_NI@Z$54 10025767 f   manage_temp.obj
 0001:00024771       __unwindfunclet$??0manage_tempBase@@QAE@PAVQWidget@@PBD_NI@Z$55 10025771 f   manage_temp.obj
 0001:0002477b       __unwindfunclet$??0manage_tempBase@@QAE@PAVQWidget@@PBD_NI@Z$56 1002577b f   manage_temp.obj
 0001:00024785       __unwindfunclet$??0manage_tempBase@@QAE@PAVQWidget@@PBD_NI@Z$57 10025785 f   manage_temp.obj
 0001:0002478f       __unwindfunclet$??0manage_tempBase@@QAE@PAVQWidget@@PBD_NI@Z$58 1002578f f   manage_temp.obj
 0001:00024799       __unwindfunclet$??0manage_tempBase@@QAE@PAVQWidget@@PBD_NI@Z$59 10025799 f   manage_temp.obj
 0001:000247a3       __unwindfunclet$??0manage_tempBase@@QAE@PAVQWidget@@PBD_NI@Z$60 100257a3 f   manage_temp.obj
 0001:000247ac       __unwindfunclet$??0manage_tempBase@@QAE@PAVQWidget@@PBD_NI@Z$61 100257ac f   manage_temp.obj
 0001:000247b6       __unwindfunclet$??0manage_tempBase@@QAE@PAVQWidget@@PBD_NI@Z$62 100257b6 f   manage_temp.obj
 0001:000247c0       __unwindfunclet$??0manage_tempBase@@QAE@PAVQWidget@@PBD_NI@Z$63 100257c0 f   manage_temp.obj
 0001:000247ca       __unwindfunclet$??0manage_tempBase@@QAE@PAVQWidget@@PBD_NI@Z$64 100257ca f   manage_temp.obj
 0001:000247d3       __unwindfunclet$??0manage_tempBase@@QAE@PAVQWidget@@PBD_NI@Z$65 100257d3 f   manage_temp.obj
 0001:000247dc       __unwindfunclet$??0manage_tempBase@@QAE@PAVQWidget@@PBD_NI@Z$66 100257dc f   manage_temp.obj
 0001:000247e6       __unwindfunclet$??0manage_tempBase@@QAE@PAVQWidget@@PBD_NI@Z$67 100257e6 f   manage_temp.obj
 0001:000247f0       __unwindfunclet$??0manage_tempBase@@QAE@PAVQWidget@@PBD_NI@Z$68 100257f0 f   manage_temp.obj
 0001:000247fa       __unwindfunclet$??0manage_tempBase@@QAE@PAVQWidget@@PBD_NI@Z$69 100257fa f   manage_temp.obj
 0001:00024804       __unwindfunclet$??0manage_tempBase@@QAE@PAVQWidget@@PBD_NI@Z$70 10025804 f   manage_temp.obj
 0001:0002480e       __unwindfunclet$??0manage_tempBase@@QAE@PAVQWidget@@PBD_NI@Z$71 1002580e f   manage_temp.obj
 0001:00024818       __unwindfunclet$??0manage_tempBase@@QAE@PAVQWidget@@PBD_NI@Z$72 10025818 f   manage_temp.obj
 0001:00024821       __unwindfunclet$??0manage_tempBase@@QAE@PAVQWidget@@PBD_NI@Z$73 10025821 f   manage_temp.obj
 0001:0002482b       __unwindfunclet$??0manage_tempBase@@QAE@PAVQWidget@@PBD_NI@Z$74 1002582b f   manage_temp.obj
 0001:00024835       __unwindfunclet$??0manage_tempBase@@QAE@PAVQWidget@@PBD_NI@Z$75 10025835 f   manage_temp.obj
 0001:0002483f       __unwindfunclet$??0manage_tempBase@@QAE@PAVQWidget@@PBD_NI@Z$76 1002583f f   manage_temp.obj
 0001:00024849       __ehhandler$??0manage_tempBase@@QAE@PAVQWidget@@PBD_NI@Z 10025849 f   manage_temp.obj
 0001:00024864       __unwindfunclet$?languageChange@manage_tempBase@@MAEXXZ$0 10025864 f   manage_temp.obj
 0001:0002486d       __unwindfunclet$?languageChange@manage_tempBase@@MAEXXZ$1 1002586d f   manage_temp.obj
 0001:00024876       __unwindfunclet$?languageChange@manage_tempBase@@MAEXXZ$2 10025876 f   manage_temp.obj
 0001:0002487f       __unwindfunclet$?languageChange@manage_tempBase@@MAEXXZ$3 1002587f f   manage_temp.obj
 0001:00024888       __unwindfunclet$?languageChange@manage_tempBase@@MAEXXZ$4 10025888 f   manage_temp.obj
 0001:00024891       __unwindfunclet$?languageChange@manage_tempBase@@MAEXXZ$5 10025891 f   manage_temp.obj
 0001:0002489a       __unwindfunclet$?languageChange@manage_tempBase@@MAEXXZ$6 1002589a f   manage_temp.obj
 0001:000248a3       __unwindfunclet$?languageChange@manage_tempBase@@MAEXXZ$7 100258a3 f   manage_temp.obj
 0001:000248ac       __unwindfunclet$?languageChange@manage_tempBase@@MAEXXZ$8 100258ac f   manage_temp.obj
 0001:000248b5       __unwindfunclet$?languageChange@manage_tempBase@@MAEXXZ$9 100258b5 f   manage_temp.obj
 0001:000248be       __unwindfunclet$?languageChange@manage_tempBase@@MAEXXZ$10 100258be f   manage_temp.obj
 0001:000248c7       __unwindfunclet$?languageChange@manage_tempBase@@MAEXXZ$11 100258c7 f   manage_temp.obj
 0001:000248d0       __unwindfunclet$?languageChange@manage_tempBase@@MAEXXZ$12 100258d0 f   manage_temp.obj
 0001:000248d9       __unwindfunclet$?languageChange@manage_tempBase@@MAEXXZ$13 100258d9 f   manage_temp.obj
 0001:000248e2       __unwindfunclet$?languageChange@manage_tempBase@@MAEXXZ$14 100258e2 f   manage_temp.obj
 0001:000248eb       __unwindfunclet$?languageChange@manage_tempBase@@MAEXXZ$15 100258eb f   manage_temp.obj
 0001:000248f4       __unwindfunclet$?languageChange@manage_tempBase@@MAEXXZ$16 100258f4 f   manage_temp.obj
 0001:000248fd       __unwindfunclet$?languageChange@manage_tempBase@@MAEXXZ$17 100258fd f   manage_temp.obj
 0001:00024906       __unwindfunclet$?languageChange@manage_tempBase@@MAEXXZ$18 10025906 f   manage_temp.obj
 0001:0002490f       __unwindfunclet$?languageChange@manage_tempBase@@MAEXXZ$19 1002590f f   manage_temp.obj
 0001:00024918       __unwindfunclet$?languageChange@manage_tempBase@@MAEXXZ$20 10025918 f   manage_temp.obj
 0001:00024921       __unwindfunclet$?languageChange@manage_tempBase@@MAEXXZ$21 10025921 f   manage_temp.obj
 0001:0002492a       __unwindfunclet$?languageChange@manage_tempBase@@MAEXXZ$22 1002592a f   manage_temp.obj
 0001:00024933       __unwindfunclet$?languageChange@manage_tempBase@@MAEXXZ$23 10025933 f   manage_temp.obj
 0001:0002493c       __unwindfunclet$?languageChange@manage_tempBase@@MAEXXZ$24 1002593c f   manage_temp.obj
 0001:00024945       __unwindfunclet$?languageChange@manage_tempBase@@MAEXXZ$25 10025945 f   manage_temp.obj
 0001:0002494e       __unwindfunclet$?languageChange@manage_tempBase@@MAEXXZ$26 1002594e f   manage_temp.obj
 0001:00024957       __unwindfunclet$?languageChange@manage_tempBase@@MAEXXZ$27 10025957 f   manage_temp.obj
 0001:00024960       __unwindfunclet$?languageChange@manage_tempBase@@MAEXXZ$28 10025960 f   manage_temp.obj
 0001:00024969       __unwindfunclet$?languageChange@manage_tempBase@@MAEXXZ$29 10025969 f   manage_temp.obj
 0001:00024972       __unwindfunclet$?languageChange@manage_tempBase@@MAEXXZ$30 10025972 f   manage_temp.obj
 0001:0002497b       __unwindfunclet$?languageChange@manage_tempBase@@MAEXXZ$31 1002597b f   manage_temp.obj
 0001:00024984       __unwindfunclet$?languageChange@manage_tempBase@@MAEXXZ$32 10025984 f   manage_temp.obj
 0001:0002498d       __unwindfunclet$?languageChange@manage_tempBase@@MAEXXZ$33 1002598d f   manage_temp.obj
 0001:00024996       __unwindfunclet$?languageChange@manage_tempBase@@MAEXXZ$34 10025996 f   manage_temp.obj
 0001:0002499f       __unwindfunclet$?languageChange@manage_tempBase@@MAEXXZ$35 1002599f f   manage_temp.obj
 0001:000249a8       __unwindfunclet$?languageChange@manage_tempBase@@MAEXXZ$36 100259a8 f   manage_temp.obj
 0001:000249b1       __unwindfunclet$?languageChange@manage_tempBase@@MAEXXZ$37 100259b1 f   manage_temp.obj
 0001:000249ba       __unwindfunclet$?languageChange@manage_tempBase@@MAEXXZ$38 100259ba f   manage_temp.obj
 0001:000249c3       __unwindfunclet$?languageChange@manage_tempBase@@MAEXXZ$39 100259c3 f   manage_temp.obj
 0001:000249cc       __unwindfunclet$?languageChange@manage_tempBase@@MAEXXZ$40 100259cc f   manage_temp.obj
 0001:000249d5       __unwindfunclet$?languageChange@manage_tempBase@@MAEXXZ$41 100259d5 f   manage_temp.obj
 0001:000249de       __unwindfunclet$?languageChange@manage_tempBase@@MAEXXZ$42 100259de f   manage_temp.obj
 0001:000249e7       __unwindfunclet$?languageChange@manage_tempBase@@MAEXXZ$43 100259e7 f   manage_temp.obj
 0001:000249f0       __unwindfunclet$?languageChange@manage_tempBase@@MAEXXZ$44 100259f0 f   manage_temp.obj
 0001:000249f9       __unwindfunclet$?languageChange@manage_tempBase@@MAEXXZ$45 100259f9 f   manage_temp.obj
 0001:00024a02       __unwindfunclet$?languageChange@manage_tempBase@@MAEXXZ$46 10025a02 f   manage_temp.obj
 0001:00024a0b       __unwindfunclet$?languageChange@manage_tempBase@@MAEXXZ$47 10025a0b f   manage_temp.obj
 0001:00024a14       __unwindfunclet$?languageChange@manage_tempBase@@MAEXXZ$48 10025a14 f   manage_temp.obj
 0001:00024a1d       __unwindfunclet$?languageChange@manage_tempBase@@MAEXXZ$49 10025a1d f   manage_temp.obj
 0001:00024a26       __unwindfunclet$?languageChange@manage_tempBase@@MAEXXZ$50 10025a26 f   manage_temp.obj
 0001:00024a2f       __unwindfunclet$?languageChange@manage_tempBase@@MAEXXZ$51 10025a2f f   manage_temp.obj
 0001:00024a38       __unwindfunclet$?languageChange@manage_tempBase@@MAEXXZ$52 10025a38 f   manage_temp.obj
 0001:00024a41       __unwindfunclet$?languageChange@manage_tempBase@@MAEXXZ$53 10025a41 f   manage_temp.obj
 0001:00024a4a       __unwindfunclet$?languageChange@manage_tempBase@@MAEXXZ$54 10025a4a f   manage_temp.obj
 0001:00024a53       __unwindfunclet$?languageChange@manage_tempBase@@MAEXXZ$55 10025a53 f   manage_temp.obj
 0001:00024a5c       __ehhandler$?languageChange@manage_tempBase@@MAEXXZ 10025a5c f   manage_temp.obj
 0001:00024a77       __unwindfunclet$?command@alm_db_output@@IAEXVQString@@0@Z$0 10025a77 f   moc_alm_db_output.obj
 0001:00024a80       __unwindfunclet$?command@alm_db_output@@IAEXVQString@@0@Z$1 10025a80 f   moc_alm_db_output.obj
 0001:00024a89       __unwindfunclet$?command@alm_db_output@@IAEXVQString@@0@Z$2 10025a89 f   moc_alm_db_output.obj
 0001:00024a9d       __ehhandler$?command@alm_db_output@@IAEXVQString@@0@Z 10025a9d f   moc_alm_db_output.obj
 0001:00024ac2       __unwindfunclet$?qt_emit@alm_db_output@@UAE_NHPAUQUObject@@@Z$0 10025ac2 f   moc_alm_db_output.obj
 0001:00024acb       __ehhandler$?qt_emit@alm_db_output@@UAE_NHPAUQUObject@@@Z 10025acb f   moc_alm_db_output.obj
 0001:00024ae6       __unwindfunclet$?itemChanged@dialog@@QAEXH@Z$0 10025ae6 f   moc_dialogimpl.obj
 0001:00024ae6       __unwindfunclet$?setUnknownDefaultText@manage_temp@@QAEXXZ$0 10025ae6 f   moc_dialogimpl.obj
 0001:00024ae6       __unwindfunclet$?menuNewFile@alm_db_output@@AAEXXZ$0 10025ae6 f   moc_dialogimpl.obj
 0001:00024ae6       __unwindfunclet$?setAckDefaultText@manage_temp@@QAEXXZ$0 10025ae6 f   moc_dialogimpl.obj
 0001:00024ae6       __unwindfunclet$?qt_invoke@dialog@@UAE_NHPAUQUObject@@@Z$0 10025ae6 f   moc_dialogimpl.obj
 0001:00024ae6       __unwindfunclet$?setOkDefaultText@manage_temp@@QAEXXZ$0 10025ae6 f   moc_dialogimpl.obj
 0001:00024ae6       __unwindfunclet$?setFailDefaultText@manage_temp@@QAEXXZ$0 10025ae6 f   moc_dialogimpl.obj
 0001:00024ae6       __unwindfunclet$?setIgnoreDefaultText@manage_temp@@QAEXXZ$0 10025ae6 f   moc_dialogimpl.obj
 0001:00024ae6       __unwindfunclet$?setLatchedDefaultText@manage_temp@@QAEXXZ$0 10025ae6 f   moc_dialogimpl.obj
 0001:00024ae6       __unwindfunclet$?getDbase@dbConnection@@QAEPAVQSqlDatabase@@XZ$0 10025ae6 f   moc_dialogimpl.obj
 0001:00024aef       __ehhandler$?getDbase@dbConnection@@QAEPAVQSqlDatabase@@XZ 10025aef f   moc_dialogimpl.obj
 0001:00024aef       __ehhandler$?menuNewFile@alm_db_output@@AAEXXZ 10025aef f   moc_dialogimpl.obj
 0001:00024aef       __ehhandler$?setLatchedDefaultText@manage_temp@@QAEXXZ 10025aef f   moc_dialogimpl.obj
 0001:00024aef       __ehhandler$?setIgnoreDefaultText@manage_temp@@QAEXXZ 10025aef f   moc_dialogimpl.obj
 0001:00024aef       __ehhandler$?setAckDefaultText@manage_temp@@QAEXXZ 10025aef f   moc_dialogimpl.obj
 0001:00024aef       __ehhandler$?setOkDefaultText@manage_temp@@QAEXXZ 10025aef f   moc_dialogimpl.obj
 0001:00024aef       __ehhandler$?qt_invoke@dialog@@UAE_NHPAUQUObject@@@Z 10025aef f   moc_dialogimpl.obj
 0001:00024aef       __ehhandler$?setUnknownDefaultText@manage_temp@@QAEXXZ 10025aef f   moc_dialogimpl.obj
 0001:00024aef       __ehhandler$?itemChanged@dialog@@QAEXH@Z 10025aef f   moc_dialogimpl.obj
 0001:00024aef       __ehhandler$?setFailDefaultText@manage_temp@@QAEXXZ 10025aef f   moc_dialogimpl.obj
 0001:00024b0a       __unwindfunclet$?loadState@cfg_Settings@@SA?AVQString@@ABV2@@Z$0 10025b0a f   cfg_widgets001:cfg_Settings.obj
 0001:00024b13       __unwindfunclet$?loadState@cfg_Settings@@SA?AVQString@@ABV2@@Z$1 10025b13 f   cfg_widgets001:cfg_Settings.obj
 0001:00024b1c       __unwindfunclet$?loadState@cfg_Settings@@SA?AVQString@@ABV2@@Z$2 10025b1c f   cfg_widgets001:cfg_Settings.obj
 0001:00024b25       __unwindfunclet$?loadState@cfg_Settings@@SA?AVQString@@ABV2@@Z$3 10025b25 f   cfg_widgets001:cfg_Settings.obj
 0001:00024b3f       __ehhandler$?loadState@cfg_Settings@@SA?AVQString@@ABV2@@Z 10025b3f f   cfg_widgets001:cfg_Settings.obj
 0001:00024b5a       __unwindfunclet$?loadState@cfg_Settings@@SAXAAVQPoint@@AAVQSize@@AA_NABVQString@@@Z$0 10025b5a f   cfg_widgets001:cfg_Settings.obj
 0001:00024b63       __unwindfunclet$?loadState@cfg_Settings@@SAXAAVQPoint@@AAVQSize@@AA_NABVQString@@@Z$1 10025b63 f   cfg_widgets001:cfg_Settings.obj
 0001:00024b6c       __ehhandler$?loadState@cfg_Settings@@SAXAAVQPoint@@AAVQSize@@AA_NABVQString@@@Z 10025b6c f   cfg_widgets001:cfg_Settings.obj
 0001:00024b87       __unwindfunclet$?loadState@cfg_Settings@@SAXQAVQListView@@ABVQString@@@Z$0 10025b87 f   cfg_widgets001:cfg_Settings.obj
 0001:00024b87       __unwindfunclet$?loadState@cfg_Settings@@SAXQAVQTable@@ABVQString@@@Z$0 10025b87 f   cfg_widgets001:cfg_Settings.obj
 0001:00024b90       __unwindfunclet$?loadState@cfg_Settings@@SAXQAVQListView@@ABVQString@@@Z$1 10025b90 f   cfg_widgets001:cfg_Settings.obj
 0001:00024b90       __unwindfunclet$?loadState@cfg_Settings@@SAXQAVQTable@@ABVQString@@@Z$1 10025b90 f   cfg_widgets001:cfg_Settings.obj
 0001:00024b99       __ehhandler$?loadState@cfg_Settings@@SAXQAVQListView@@ABVQString@@@Z 10025b99 f   cfg_widgets001:cfg_Settings.obj
 0001:00024b99       __ehhandler$?loadState@cfg_Settings@@SAXQAVQTable@@ABVQString@@@Z 10025b99 f   cfg_widgets001:cfg_Settings.obj
 0001:00024bb4       __unwindfunclet$?loadState@cfg_Settings@@SAXQAVQSplitter@@ABVQString@@@Z$0 10025bb4 f   cfg_widgets001:cfg_Settings.obj
 0001:00024bbd       __unwindfunclet$?loadState@cfg_Settings@@SAXQAVQSplitter@@ABVQString@@@Z$1 10025bbd f   cfg_widgets001:cfg_Settings.obj
 0001:00024bc6       __unwindfunclet$?loadState@cfg_Settings@@SAXQAVQSplitter@@ABVQString@@@Z$2 10025bc6 f   cfg_widgets001:cfg_Settings.obj
 0001:00024bcf       __ehhandler$?loadState@cfg_Settings@@SAXQAVQSplitter@@ABVQString@@@Z 10025bcf f   cfg_widgets001:cfg_Settings.obj
 0001:00024bea       __unwindfunclet$?saveState@cfg_Settings@@SAXABVQPoint@@ABVQSize@@AB_NABVQString@@@Z$0 10025bea f   cfg_widgets001:cfg_Settings.obj
 0001:00024bf3       __unwindfunclet$?saveState@cfg_Settings@@SAXABVQPoint@@ABVQSize@@AB_NABVQString@@@Z$1 10025bf3 f   cfg_widgets001:cfg_Settings.obj
 0001:00024bfc       __unwindfunclet$?saveState@cfg_Settings@@SAXABVQPoint@@ABVQSize@@AB_NABVQString@@@Z$2 10025bfc f   cfg_widgets001:cfg_Settings.obj
 0001:00024c05       __unwindfunclet$?saveState@cfg_Settings@@SAXABVQPoint@@ABVQSize@@AB_NABVQString@@@Z$3 10025c05 f   cfg_widgets001:cfg_Settings.obj
 0001:00024c0e       __unwindfunclet$?saveState@cfg_Settings@@SAXABVQPoint@@ABVQSize@@AB_NABVQString@@@Z$4 10025c0e f   cfg_widgets001:cfg_Settings.obj
 0001:00024c17       __unwindfunclet$?saveState@cfg_Settings@@SAXABVQPoint@@ABVQSize@@AB_NABVQString@@@Z$5 10025c17 f   cfg_widgets001:cfg_Settings.obj
 0001:00024c20       __unwindfunclet$?saveState@cfg_Settings@@SAXABVQPoint@@ABVQSize@@AB_NABVQString@@@Z$6 10025c20 f   cfg_widgets001:cfg_Settings.obj
 0001:00024c29       __ehhandler$?saveState@cfg_Settings@@SAXABVQPoint@@ABVQSize@@AB_NABVQString@@@Z 10025c29 f   cfg_widgets001:cfg_Settings.obj
 0001:00024c44       __unwindfunclet$?saveState@cfg_Settings@@SAXABVQString@@0@Z$0 10025c44 f   cfg_widgets001:cfg_Settings.obj
 0001:00024c4d       __unwindfunclet$?saveState@cfg_Settings@@SAXABVQString@@0@Z$1 10025c4d f   cfg_widgets001:cfg_Settings.obj
 0001:00024c56       __unwindfunclet$?saveState@cfg_Settings@@SAXABVQString@@0@Z$2 10025c56 f   cfg_widgets001:cfg_Settings.obj
 0001:00024c5f       __ehhandler$?saveState@cfg_Settings@@SAXABVQString@@0@Z 10025c5f f   cfg_widgets001:cfg_Settings.obj
 0001:00024c7a       __unwindfunclet$?saveState@cfg_Settings@@SAXQBVQListView@@ABVQString@@@Z$0 10025c7a f   cfg_widgets001:cfg_Settings.obj
 0001:00024c7a       __unwindfunclet$?saveState@cfg_Settings@@SAXQBVQTable@@ABVQString@@@Z$0 10025c7a f   cfg_widgets001:cfg_Settings.obj
 0001:00024c83       __unwindfunclet$?saveState@cfg_Settings@@SAXQBVQTable@@ABVQString@@@Z$1 10025c83 f   cfg_widgets001:cfg_Settings.obj
 0001:00024c83       __unwindfunclet$?saveState@cfg_Settings@@SAXQBVQListView@@ABVQString@@@Z$1 10025c83 f   cfg_widgets001:cfg_Settings.obj
 0001:00024c8c       __unwindfunclet$?saveState@cfg_Settings@@SAXQBVQListView@@ABVQString@@@Z$2 10025c8c f   cfg_widgets001:cfg_Settings.obj
 0001:00024c8c       __unwindfunclet$?saveState@cfg_Settings@@SAXQBVQTable@@ABVQString@@@Z$2 10025c8c f   cfg_widgets001:cfg_Settings.obj
 0001:00024c95       __unwindfunclet$?saveState@cfg_Settings@@SAXQBVQListView@@ABVQString@@@Z$3 10025c95 f   cfg_widgets001:cfg_Settings.obj
 0001:00024c95       __unwindfunclet$?saveState@cfg_Settings@@SAXQBVQTable@@ABVQString@@@Z$3 10025c95 f   cfg_widgets001:cfg_Settings.obj
 0001:00024c9e       __ehhandler$?saveState@cfg_Settings@@SAXQBVQListView@@ABVQString@@@Z 10025c9e f   cfg_widgets001:cfg_Settings.obj
 0001:00024c9e       __ehhandler$?saveState@cfg_Settings@@SAXQBVQTable@@ABVQString@@@Z 10025c9e f   cfg_widgets001:cfg_Settings.obj
 0001:00024cb9       __unwindfunclet$?saveState@cfg_Settings@@SAXQBVQSplitter@@ABVQString@@@Z$0 10025cb9 f   cfg_widgets001:cfg_Settings.obj
 0001:00024cc2       __unwindfunclet$?saveState@cfg_Settings@@SAXQBVQSplitter@@ABVQString@@@Z$1 10025cc2 f   cfg_widgets001:cfg_Settings.obj
 0001:00024ccb       __unwindfunclet$?saveState@cfg_Settings@@SAXQBVQSplitter@@ABVQString@@@Z$2 10025ccb f   cfg_widgets001:cfg_Settings.obj
 0001:00024cd4       __unwindfunclet$?saveState@cfg_Settings@@SAXQBVQSplitter@@ABVQString@@@Z$3 10025cd4 f   cfg_widgets001:cfg_Settings.obj
 0001:00024cdd       __ehhandler$?saveState@cfg_Settings@@SAXQBVQSplitter@@ABVQString@@@Z 10025cdd f   cfg_widgets001:cfg_Settings.obj
 0001:00024d00       __unwindfunclet$??0Document_BncsSystem@@QAE@XZ$0 10025d00 f   config_alarm_utilities:Document.obj
 0001:00024d09       __unwindfunclet$??0Document_BncsSystem@@QAE@XZ$1 10025d09 f   config_alarm_utilities:Document.obj
 0001:00024d11       __ehhandler$??0Document_BncsSystem@@QAE@XZ 10025d11 f   config_alarm_utilities:Document.obj
 0001:00024d30       __unwindfunclet$?load@Document_BncsSystem@@QAE_NXZ$0 10025d30 f   config_alarm_utilities:Document.obj
 0001:00024d3c       __unwindfunclet$?load@Document_BncsSystem@@QAE_NXZ$1 10025d3c f   config_alarm_utilities:Document.obj
 0001:00024d48       __ehhandler$?load@Document_BncsSystem@@QAE_NXZ 10025d48 f   config_alarm_utilities:Document.obj
 0001:00024d70       __unwindfunclet$??0Loaders@@QAE@XZ$0 10025d70 f   config_alarm_utilities:Loaders.obj
 0001:00024d7b       __ehhandler$??0Loaders@@QAE@XZ 10025d7b f   config_alarm_utilities:Loaders.obj
 0001:00024da0       __unwindfunclet$??0FileLoad@@IAE@ABVQString@@@Z$0 10025da0 f   config_alarm_utilities:Loaders.obj
 0001:00024da0       __unwindfunclet$??1FileLoad@@UAE@XZ$0 10025da0 f   config_alarm_utilities:Loaders.obj
 0001:00024dac       __ehhandler$??1FileLoad@@UAE@XZ 10025dac f   config_alarm_utilities:Loaders.obj
 0001:00024dac       __ehhandler$??0FileLoad@@IAE@ABVQString@@@Z 10025dac f   config_alarm_utilities:Loaders.obj
 0001:00024dd0       __unwindfunclet$??1Loaders@@UAE@XZ$0 10025dd0 f   config_alarm_utilities:Loaders.obj
 0001:00024ddb       __unwindfunclet$??1Loaders@@UAE@XZ$1 10025ddb f   config_alarm_utilities:Loaders.obj
 0001:00024de6       __unwindfunclet$??1Loaders@@UAE@XZ$2 10025de6 f   config_alarm_utilities:Loaders.obj
 0001:00024def       __unwindfunclet$??1Loaders@@UAE@XZ$3 10025def f   config_alarm_utilities:Loaders.obj
 0001:00024df8       __ehhandler$??1Loaders@@UAE@XZ 10025df8 f   config_alarm_utilities:Loaders.obj
 0001:00024e20       __unwindfunclet$??_G?$QPtrList@VFileLoad@@@@UAEPAXI@Z$0 10025e20 f   config_alarm_utilities:Loaders.obj
 0001:00024e20       __unwindfunclet$??1?$QPtrList@VFileLoad@@@@UAE@XZ$0 10025e20 f   config_alarm_utilities:Loaders.obj
 0001:00024e20       __unwindfunclet$??_G?$QPtrList@VDirLoad@@@@UAEPAXI@Z$0 10025e20 f   config_alarm_utilities:Loaders.obj
 0001:00024e20       __unwindfunclet$??1?$QPtrList@VDirLoad@@@@UAE@XZ$0 10025e20 f   config_alarm_utilities:Loaders.obj
 0001:00024e29       __ehhandler$??1?$QPtrList@VDirLoad@@@@UAE@XZ 10025e29 f   config_alarm_utilities:Loaders.obj
 0001:00024e29       __ehhandler$??1?$QPtrList@VFileLoad@@@@UAE@XZ 10025e29 f   config_alarm_utilities:Loaders.obj
 0001:00024e29       __ehhandler$??_G?$QPtrList@VFileLoad@@@@UAEPAXI@Z 10025e29 f   config_alarm_utilities:Loaders.obj
 0001:00024e29       __ehhandler$??_G?$QPtrList@VDirLoad@@@@UAEPAXI@Z 10025e29 f   config_alarm_utilities:Loaders.obj
 0001:00024e50       __unwindfunclet$?matches@FileLoad@@QAE_NABVQString@@@Z$0 10025e50 f   config_alarm_utilities:Loaders.obj
 0001:00024e59       __unwindfunclet$?matches@FileLoad@@QAE_NABVQString@@@Z$1 10025e59 f   config_alarm_utilities:Loaders.obj
 0001:00024e62       __unwindfunclet$?matches@FileLoad@@QAE_NABVQString@@@Z$2 10025e62 f   config_alarm_utilities:Loaders.obj
 0001:00024e6b       __ehhandler$?matches@FileLoad@@QAE_NABVQString@@@Z 10025e6b f   config_alarm_utilities:Loaders.obj
 0001:00024e90       __unwindfunclet$?request@FileLoad@@QAEXPAVISendCommand@@@Z$0 10025e90 f   config_alarm_utilities:Loaders.obj
 0001:00024e99       __unwindfunclet$?request@FileLoad@@QAEXPAVISendCommand@@@Z$1 10025e99 f   config_alarm_utilities:Loaders.obj
 0001:00024ea2       __ehhandler$?request@FileLoad@@QAEXPAVISendCommand@@@Z 10025ea2 f   config_alarm_utilities:Loaders.obj
 0001:00024ec0       ??__F?_Generic_object@?$_Error_objects@H@std@@2V_Generic_error_category@2@A@@YAXXZ 10025ec0 f   alm_db_output.obj
 0001:00024ecb       ??__F?_Iostream_object@?$_Error_objects@H@std@@2V_Iostream_error_category@2@A@@YAXXZ 10025ecb f   alm_db_output.obj
 0001:00024ed6       ??__F?_System_object@?$_Error_objects@H@std@@2V_System_error_category@2@A@@YAXXZ 10025ed6 f   alm_db_output.obj
 0001:00024ee1       ??__FcleanUp_setDefaultsBase@@YAXXZ 10025ee1 f   moc_setdefaults.obj
 0001:00024eec       ??__FcleanUp_setDefaults@@YAXXZ 10025eec f   moc_setdefaultsimpl.obj
 0001:00024ef7       ??__FcleanUp_alm_db_output@@YAXXZ 10025ef7 f   moc_alm_db_output.obj
 0001:00024f02       ??__FcleanUp_dialogBase@@YAXXZ 10025f02 f   moc_dialog.obj
 0001:00024f0d       ??__FcleanUp_dialog@@YAXXZ 10025f0d f   moc_dialogimpl.obj
 0001:00024f18       ??__FcleanUp_manage_tempBase@@YAXXZ 10025f18 f   moc_manage_temp.obj
 0001:00024f23       ??__FcleanUp_manage_temp@@YAXXZ 10025f23 f   moc_manage_tempimpl.obj
 0001:00024f30       ??__F?sm_sSystemFolder@Document@@1VQString@@A@@YAXXZ 10025f30 f   config_alarm_utilities:Document.obj
 0002:00001680       ?_Generic_object$initializer$@?$_Error_objects@H@std@@2P6AXXZA 10027680     alm_db_output.obj
 0002:00001684       ?_Iostream_object$initializer$@?$_Error_objects@H@std@@2P6AXXZA 10027684     alm_db_output.obj
 0002:00001688       ?_System_object$initializer$@?$_Error_objects@H@std@@2P6AXXZA 10027688     alm_db_output.obj
 0002:0000168c       _cleanUp_setDefaultsBase$initializer$ 1002768c     moc_setdefaults.obj
 0002:00001690       _cleanUp_setDefaults$initializer$ 10027690     moc_setdefaultsimpl.obj
 0002:00001694       _cleanUp_alm_db_output$initializer$ 10027694     moc_alm_db_output.obj
 0002:00001698       _cleanUp_dialogBase$initializer$ 10027698     moc_dialog.obj
 0002:0000169c       _cleanUp_dialog$initializer$ 1002769c     moc_dialogimpl.obj
 0002:000016a0       _cleanUp_manage_tempBase$initializer$ 100276a0     moc_manage_temp.obj
 0002:000016a4       _cleanUp_manage_temp$initializer$ 100276a4     moc_manage_tempimpl.obj
 0002:000016a8       ?sm_sSystemFolder$initializer$@Document@@1P6AXXZA 100276a8     config_alarm_utilities:Document.obj
 0002:000016b4       _pcinit                    100276b4     MSVCRT:crtdll.obj
 0002:000016b8       _pinit                     100276b8     MSVCRT:atonexit.obj
 0002:0000509c       ?slot_0@?3??staticMetaObject@setDefaultsBase@@SAPAVQMetaObject@@XZ@4UQUMethod@@B 1002b09c     moc_setdefaults.obj
 0002:000050b8       ?slot_tbl@?3??staticMetaObject@setDefaultsBase@@SAPAVQMetaObject@@XZ@4QBUQMetaData@@B 1002b0b8     moc_setdefaults.obj
 0002:00008ce8       ?slot_0@?3??staticMetaObject@alm_db_output@@SAPAVQMetaObject@@XZ@4UQUMethod@@B 1002ece8     moc_alm_db_output.obj
 0002:00008cfc       ?slot_1@?3??staticMetaObject@alm_db_output@@SAPAVQMetaObject@@XZ@4UQUMethod@@B 1002ecfc     moc_alm_db_output.obj
 0002:00008d2c       ?slot_2@?3??staticMetaObject@alm_db_output@@SAPAVQMetaObject@@XZ@4UQUMethod@@B 1002ed2c     moc_alm_db_output.obj
 0002:00008d38       ?slot_3@?3??staticMetaObject@alm_db_output@@SAPAVQMetaObject@@XZ@4UQUMethod@@B 1002ed38     moc_alm_db_output.obj
 0002:00008d54       ?slot_4@?3??staticMetaObject@alm_db_output@@SAPAVQMetaObject@@XZ@4UQUMethod@@B 1002ed54     moc_alm_db_output.obj
 0002:00008d70       ?slot_5@?3??staticMetaObject@alm_db_output@@SAPAVQMetaObject@@XZ@4UQUMethod@@B 1002ed70     moc_alm_db_output.obj
 0002:00008d8c       ?slot_6@?3??staticMetaObject@alm_db_output@@SAPAVQMetaObject@@XZ@4UQUMethod@@B 1002ed8c     moc_alm_db_output.obj
 0002:00008dac       ?slot_7@?3??staticMetaObject@alm_db_output@@SAPAVQMetaObject@@XZ@4UQUMethod@@B 1002edac     moc_alm_db_output.obj
 0002:00008dc4       ?slot_8@?3??staticMetaObject@alm_db_output@@SAPAVQMetaObject@@XZ@4UQUMethod@@B 1002edc4     moc_alm_db_output.obj
 0002:00008de0       ?slot_9@?3??staticMetaObject@alm_db_output@@SAPAVQMetaObject@@XZ@4UQUMethod@@B 1002ede0     moc_alm_db_output.obj
 0002:00008e00       ?slot_10@?3??staticMetaObject@alm_db_output@@SAPAVQMetaObject@@XZ@4UQUMethod@@B 1002ee00     moc_alm_db_output.obj
 0002:00008e18       ?slot_11@?3??staticMetaObject@alm_db_output@@SAPAVQMetaObject@@XZ@4UQUMethod@@B 1002ee18     moc_alm_db_output.obj
 0002:00008e30       ?slot_12@?3??staticMetaObject@alm_db_output@@SAPAVQMetaObject@@XZ@4UQUMethod@@B 1002ee30     moc_alm_db_output.obj
 0002:00008e6c       ?slot_13@?3??staticMetaObject@alm_db_output@@SAPAVQMetaObject@@XZ@4UQUMethod@@B 1002ee6c     moc_alm_db_output.obj
 0002:00008e88       ?slot_14@?3??staticMetaObject@alm_db_output@@SAPAVQMetaObject@@XZ@4UQUMethod@@B 1002ee88     moc_alm_db_output.obj
 0002:00008ea8       ?slot_15@?3??staticMetaObject@alm_db_output@@SAPAVQMetaObject@@XZ@4UQUMethod@@B 1002eea8     moc_alm_db_output.obj
 0002:00008ec8       ?slot_16@?3??staticMetaObject@alm_db_output@@SAPAVQMetaObject@@XZ@4UQUMethod@@B 1002eec8     moc_alm_db_output.obj
 0002:00008ee4       ?slot_17@?3??staticMetaObject@alm_db_output@@SAPAVQMetaObject@@XZ@4UQUMethod@@B 1002eee4     moc_alm_db_output.obj
 0002:00008f00       ?slot_18@?3??staticMetaObject@alm_db_output@@SAPAVQMetaObject@@XZ@4UQUMethod@@B 1002ef00     moc_alm_db_output.obj
 0002:00008f1c       ?slot_19@?3??staticMetaObject@alm_db_output@@SAPAVQMetaObject@@XZ@4UQUMethod@@B 1002ef1c     moc_alm_db_output.obj
 0002:00008f38       ?slot_20@?3??staticMetaObject@alm_db_output@@SAPAVQMetaObject@@XZ@4UQUMethod@@B 1002ef38     moc_alm_db_output.obj
 0002:00008f58       ?slot_tbl@?3??staticMetaObject@alm_db_output@@SAPAVQMetaObject@@XZ@4QBUQMetaData@@B 1002ef58     moc_alm_db_output.obj
 0002:0000921c       ?signal_0@?3??staticMetaObject@alm_db_output@@SAPAVQMetaObject@@XZ@4UQUMethod@@B 1002f21c     moc_alm_db_output.obj
 0002:00009230       ?signal_tbl@?3??staticMetaObject@alm_db_output@@SAPAVQMetaObject@@XZ@4QBUQMetaData@@B 1002f230     moc_alm_db_output.obj
 0002:00009278       ?slot_0@?3??staticMetaObject@dialogBase@@SAPAVQMetaObject@@XZ@4UQUMethod@@B 1002f278     moc_dialog.obj
 0002:0000928c       ?slot_1@?3??staticMetaObject@dialogBase@@SAPAVQMetaObject@@XZ@4UQUMethod@@B 1002f28c     moc_dialog.obj
 0002:00009298       ?slot_tbl@?3??staticMetaObject@dialogBase@@SAPAVQMetaObject@@XZ@4QBUQMetaData@@B 1002f298     moc_dialog.obj
 0002:000092bc       ?slot_0@?3??staticMetaObject@dialog@@SAPAVQMetaObject@@XZ@4UQUMethod@@B 1002f2bc     moc_dialogimpl.obj
 0002:000092c8       ?slot_1@?3??staticMetaObject@dialog@@SAPAVQMetaObject@@XZ@4UQUMethod@@B 1002f2c8     moc_dialogimpl.obj
 0002:000092e8       ?slot_2@?3??staticMetaObject@dialog@@SAPAVQMetaObject@@XZ@4UQUMethod@@B 1002f2e8     moc_dialogimpl.obj
 0002:000092fc       ?slot_3@?3??staticMetaObject@dialog@@SAPAVQMetaObject@@XZ@4UQUMethod@@B 1002f2fc     moc_dialogimpl.obj
 0002:00009310       ?slot_4@?3??staticMetaObject@dialog@@SAPAVQMetaObject@@XZ@4UQUMethod@@B 1002f310     moc_dialogimpl.obj
 0002:0000932c       ?slot_5@?3??staticMetaObject@dialog@@SAPAVQMetaObject@@XZ@4UQUMethod@@B 1002f32c     moc_dialogimpl.obj
 0002:00009358       ?slot_6@?3??staticMetaObject@dialog@@SAPAVQMetaObject@@XZ@4UQUMethod@@B 1002f358     moc_dialogimpl.obj
 0002:00009374       ?slot_7@?3??staticMetaObject@dialog@@SAPAVQMetaObject@@XZ@4UQUMethod@@B 1002f374     moc_dialogimpl.obj
 0002:0000938c       ?slot_8@?3??staticMetaObject@dialog@@SAPAVQMetaObject@@XZ@4UQUMethod@@B 1002f38c     moc_dialogimpl.obj
 0002:000093a4       ?slot_9@?3??staticMetaObject@dialog@@SAPAVQMetaObject@@XZ@4UQUMethod@@B 1002f3a4     moc_dialogimpl.obj
 0002:000093bc       ?slot_10@?3??staticMetaObject@dialog@@SAPAVQMetaObject@@XZ@4UQUMethod@@B 1002f3bc     moc_dialogimpl.obj
 0002:000093e0       ?slot_11@?3??staticMetaObject@dialog@@SAPAVQMetaObject@@XZ@4UQUMethod@@B 1002f3e0     moc_dialogimpl.obj
 0002:00009400       ?slot_12@?3??staticMetaObject@dialog@@SAPAVQMetaObject@@XZ@4UQUMethod@@B 1002f400     moc_dialogimpl.obj
 0002:00009420       ?slot_13@?3??staticMetaObject@dialog@@SAPAVQMetaObject@@XZ@4UQUMethod@@B 1002f420     moc_dialogimpl.obj
 0002:00009440       ?slot_14@?3??staticMetaObject@dialog@@SAPAVQMetaObject@@XZ@4UQUMethod@@B 1002f440     moc_dialogimpl.obj
 0002:0000945c       ?slot_15@?3??staticMetaObject@dialog@@SAPAVQMetaObject@@XZ@4UQUMethod@@B 1002f45c     moc_dialogimpl.obj
 0002:00009478       ?slot_16@?3??staticMetaObject@dialog@@SAPAVQMetaObject@@XZ@4UQUMethod@@B 1002f478     moc_dialogimpl.obj
 0002:0000949c       ?slot_17@?3??staticMetaObject@dialog@@SAPAVQMetaObject@@XZ@4UQUMethod@@B 1002f49c     moc_dialogimpl.obj
 0002:000094bc       ?slot_18@?3??staticMetaObject@dialog@@SAPAVQMetaObject@@XZ@4UQUMethod@@B 1002f4bc     moc_dialogimpl.obj
 0002:000094dc       ?slot_19@?3??staticMetaObject@dialog@@SAPAVQMetaObject@@XZ@4UQUMethod@@B 1002f4dc     moc_dialogimpl.obj
 0002:00009508       ?slot_20@?3??staticMetaObject@dialog@@SAPAVQMetaObject@@XZ@4UQUMethod@@B 1002f508     moc_dialogimpl.obj
 0002:00009524       ?slot_21@?3??staticMetaObject@dialog@@SAPAVQMetaObject@@XZ@4UQUMethod@@B 1002f524     moc_dialogimpl.obj
 0002:00009544       ?slot_22@?3??staticMetaObject@dialog@@SAPAVQMetaObject@@XZ@4UQUMethod@@B 1002f544     moc_dialogimpl.obj
 0002:00009560       ?slot_23@?3??staticMetaObject@dialog@@SAPAVQMetaObject@@XZ@4UQUMethod@@B 1002f560     moc_dialogimpl.obj
 0002:00009580       ?slot_24@?3??staticMetaObject@dialog@@SAPAVQMetaObject@@XZ@4UQUMethod@@B 1002f580     moc_dialogimpl.obj
 0002:000095a0       ?slot_25@?3??staticMetaObject@dialog@@SAPAVQMetaObject@@XZ@4UQUMethod@@B 1002f5a0     moc_dialogimpl.obj
 0002:000095c0       ?slot_26@?3??staticMetaObject@dialog@@SAPAVQMetaObject@@XZ@4UQUMethod@@B 1002f5c0     moc_dialogimpl.obj
 0002:000095e4       ?slot_27@?3??staticMetaObject@dialog@@SAPAVQMetaObject@@XZ@4UQUMethod@@B 1002f5e4     moc_dialogimpl.obj
 0002:00009608       ?slot_28@?3??staticMetaObject@dialog@@SAPAVQMetaObject@@XZ@4UQUMethod@@B 1002f608     moc_dialogimpl.obj
 0002:0000962c       ?slot_29@?3??staticMetaObject@dialog@@SAPAVQMetaObject@@XZ@4UQUMethod@@B 1002f62c     moc_dialogimpl.obj
 0002:0000964c       ?slot_30@?3??staticMetaObject@dialog@@SAPAVQMetaObject@@XZ@4UQUMethod@@B 1002f64c     moc_dialogimpl.obj
 0002:00009668       ?slot_31@?3??staticMetaObject@dialog@@SAPAVQMetaObject@@XZ@4UQUMethod@@B 1002f668     moc_dialogimpl.obj
 0002:00009688       ?slot_tbl@?3??staticMetaObject@dialog@@SAPAVQMetaObject@@XZ@4QBUQMetaData@@B 1002f688     moc_dialogimpl.obj
 0002:00009a9c       ?signal_0@?3??staticMetaObject@dialog@@SAPAVQMetaObject@@XZ@4UQUMethod@@B 1002fa9c     moc_dialogimpl.obj
 0002:00009ab8       ?signal_tbl@?3??staticMetaObject@dialog@@SAPAVQMetaObject@@XZ@4QBUQMetaData@@B 1002fab8     moc_dialogimpl.obj
 0002:00009ad4       ?slot_0@?3??staticMetaObject@manage_tempBase@@SAPAVQMetaObject@@XZ@4UQUMethod@@B 1002fad4     moc_manage_temp.obj
 0002:00009ae0       ?slot_tbl@?3??staticMetaObject@manage_tempBase@@SAPAVQMetaObject@@XZ@4QBUQMetaData@@B 1002fae0     moc_manage_temp.obj
 0002:00009af8       ?slot_0@?3??staticMetaObject@manage_temp@@SAPAVQMetaObject@@XZ@4UQUMethod@@B 1002faf8     moc_manage_tempimpl.obj
 0002:00009b0c       ?slot_1@?3??staticMetaObject@manage_temp@@SAPAVQMetaObject@@XZ@4UQUMethod@@B 1002fb0c     moc_manage_tempimpl.obj
 0002:00009b28       ?slot_2@?3??staticMetaObject@manage_temp@@SAPAVQMetaObject@@XZ@4UQUMethod@@B 1002fb28     moc_manage_tempimpl.obj
 0002:00009b44       ?slot_3@?3??staticMetaObject@manage_temp@@SAPAVQMetaObject@@XZ@4UQUMethod@@B 1002fb44     moc_manage_tempimpl.obj
 0002:00009b50       ?slot_4@?3??staticMetaObject@manage_temp@@SAPAVQMetaObject@@XZ@4UQUMethod@@B 1002fb50     moc_manage_tempimpl.obj
 0002:00009b74       ?slot_5@?3??staticMetaObject@manage_temp@@SAPAVQMetaObject@@XZ@4UQUMethod@@B 1002fb74     moc_manage_tempimpl.obj
 0002:00009b94       ?slot_6@?3??staticMetaObject@manage_temp@@SAPAVQMetaObject@@XZ@4UQUMethod@@B 1002fb94     moc_manage_tempimpl.obj
 0002:00009ba0       ?slot_7@?3??staticMetaObject@manage_temp@@SAPAVQMetaObject@@XZ@4UQUMethod@@B 1002fba0     moc_manage_tempimpl.obj
 0002:00009bac       ?slot_8@?3??staticMetaObject@manage_temp@@SAPAVQMetaObject@@XZ@4UQUMethod@@B 1002fbac     moc_manage_tempimpl.obj
 0002:00009bd0       ?slot_9@?3??staticMetaObject@manage_temp@@SAPAVQMetaObject@@XZ@4UQUMethod@@B 1002fbd0     moc_manage_tempimpl.obj
 0002:00009bdc       ?slot_10@?3??staticMetaObject@manage_temp@@SAPAVQMetaObject@@XZ@4UQUMethod@@B 1002fbdc     moc_manage_tempimpl.obj
 0002:00009be8       ?slot_11@?3??staticMetaObject@manage_temp@@SAPAVQMetaObject@@XZ@4UQUMethod@@B 1002fbe8     moc_manage_tempimpl.obj
 0002:00009bf4       ?slot_12@?3??staticMetaObject@manage_temp@@SAPAVQMetaObject@@XZ@4UQUMethod@@B 1002fbf4     moc_manage_tempimpl.obj
 0002:00009c00       ?slot_13@?3??staticMetaObject@manage_temp@@SAPAVQMetaObject@@XZ@4UQUMethod@@B 1002fc00     moc_manage_tempimpl.obj
 0002:00009c0c       ?slot_14@?3??staticMetaObject@manage_temp@@SAPAVQMetaObject@@XZ@4UQUMethod@@B 1002fc0c     moc_manage_tempimpl.obj
 0002:00009c18       ?slot_15@?3??staticMetaObject@manage_temp@@SAPAVQMetaObject@@XZ@4UQUMethod@@B 1002fc18     moc_manage_tempimpl.obj
 0002:00009c24       ?slot_16@?3??staticMetaObject@manage_temp@@SAPAVQMetaObject@@XZ@4UQUMethod@@B 1002fc24     moc_manage_tempimpl.obj
 0002:00009c44       ?slot_17@?3??staticMetaObject@manage_temp@@SAPAVQMetaObject@@XZ@4UQUMethod@@B 1002fc44     moc_manage_tempimpl.obj
 0002:00009c50       ?slot_18@?3??staticMetaObject@manage_temp@@SAPAVQMetaObject@@XZ@4UQUMethod@@B 1002fc50     moc_manage_tempimpl.obj
 0002:00009c70       ?slot_19@?3??staticMetaObject@manage_temp@@SAPAVQMetaObject@@XZ@4UQUMethod@@B 1002fc70     moc_manage_tempimpl.obj
 0002:00009c94       ?slot_20@?3??staticMetaObject@manage_temp@@SAPAVQMetaObject@@XZ@4UQUMethod@@B 1002fc94     moc_manage_tempimpl.obj
 0002:00009cb8       ?slot_21@?3??staticMetaObject@manage_temp@@SAPAVQMetaObject@@XZ@4UQUMethod@@B 1002fcb8     moc_manage_tempimpl.obj
 0002:00009ce0       ?slot_tbl@?3??staticMetaObject@manage_temp@@SAPAVQMetaObject@@XZ@4QBUQMetaData@@B 1002fce0     moc_manage_tempimpl.obj
 0002:00009ffc       _GS_ExceptionPointers      1002fffc     MSVCRT:gs_report.obj
 0002:0000bfb0       __catchsym$?_Copy@?$basic_string@DU?$char_traits@D@std@@V?$allocator@D@2@@std@@QAEXII@Z$5 10031fb0     alm_db_output.obj
 0002:0000bfc0       __catchsym$?_Copy@?$basic_string@DU?$char_traits@D@std@@V?$allocator@D@2@@std@@QAEXII@Z$4 10031fc0     alm_db_output.obj
 0002:0000bfd0       __unwindtable$?_Copy@?$basic_string@DU?$char_traits@D@std@@V?$allocator@D@2@@std@@QAEXII@Z 10031fd0     alm_db_output.obj
 0002:0000bff0       __ehfuncinfo$?_Copy@?$basic_string@DU?$char_traits@D@std@@V?$allocator@D@2@@std@@QAEXII@Z 10031ff0     alm_db_output.obj
 0002:0000c014       __tryblocktable$?_Copy@?$basic_string@DU?$char_traits@D@std@@V?$allocator@D@2@@std@@QAEXII@Z 10032014     alm_db_output.obj
 0002:0000c03c       __unwindtable$??1QDockWindowList@@UAE@XZ 1003203c     alm_db_output.obj
 0002:0000c04c       __ehfuncinfo$??1QDockWindowList@@UAE@XZ 1003204c     alm_db_output.obj
 0002:0000c070       __unwindtable$??1QPopupMenuList@@UAE@XZ 10032070     alm_db_output.obj
 0002:0000c078       __ehfuncinfo$??1QPopupMenuList@@UAE@XZ 10032078     alm_db_output.obj
 0002:0000c09c       __unwindtable$??0config_plugin_base@@QAE@ABVQString@@00@Z 1003209c     alm_db_output.obj
 0002:0000c0bc       __ehfuncinfo$??0config_plugin_base@@QAE@ABVQString@@00@Z 100320bc     alm_db_output.obj
 0002:0000c0e0       __unwindtable$??1config_plugin_base@@UAE@XZ 100320e0     alm_db_output.obj
 0002:0000c0f8       __ehfuncinfo$??1config_plugin_base@@UAE@XZ 100320f8     alm_db_output.obj
 0002:0000c11c       __unwindtable$?about@config_plugin_base@@UAE?AVQString@@XZ 1003211c     alm_db_output.obj
 0002:0000c12c       __ehfuncinfo$?about@config_plugin_base@@UAE?AVQString@@XZ 1003212c     alm_db_output.obj
 0002:0000c150       __ehfuncinfo$??0alm_db_output@@QAE@ABVQString@@00@Z 10032150     alm_db_output.obj
 0002:0000c174       __unwindtable$??0alm_db_output@@QAE@ABVQString@@00@Z 10032174     alm_db_output.obj
 0002:0000c38c       __ehfuncinfo$??1alm_db_output@@UAE@XZ 1003238c     alm_db_output.obj
 0002:0000c3b0       __unwindtable$??1alm_db_output@@UAE@XZ 100323b0     alm_db_output.obj
 0002:0000c428       __unwindtable$?toolbars@alm_db_output@@UAE?AVQDockWindowList@@XZ 10032428     alm_db_output.obj
 0002:0000c430       __ehfuncinfo$?toolbars@alm_db_output@@UAE?AVQDockWindowList@@XZ 10032430     alm_db_output.obj
 0002:0000c454       __unwindtable$?menus@alm_db_output@@UAE?AVQPopupMenuList@@XZ 10032454     alm_db_output.obj
 0002:0000c45c       __ehfuncinfo$?menus@alm_db_output@@UAE?AVQPopupMenuList@@XZ 1003245c     alm_db_output.obj
 0002:0000c480       __unwindtable$?reply@alm_db_output@@UAEXPAVresponse@@@Z 10032480     alm_db_output.obj
 0002:0000c488       __ehfuncinfo$?reply@alm_db_output@@UAEXPAVresponse@@@Z 10032488     alm_db_output.obj
 0002:0000c4ac       __ehfuncinfo$?navigate@alm_db_output@@UAEXABVQString@@0@Z 100324ac     alm_db_output.obj
 0002:0000c4d0       __unwindtable$?navigate@alm_db_output@@UAEXABVQString@@0@Z 100324d0     alm_db_output.obj
 0002:0000c558       __unwindtable$?activate@alm_db_output@@UAEX_N@Z 10032558     alm_db_output.obj
 0002:0000c570       __ehfuncinfo$?activate@alm_db_output@@UAEX_N@Z 10032570     alm_db_output.obj
 0002:0000c594       __unwindtable$?closeEvent@alm_db_output@@UAEXPAVQCloseEvent@@@Z 10032594     alm_db_output.obj
 0002:0000c59c       __ehfuncinfo$?closeEvent@alm_db_output@@UAEXPAVQCloseEvent@@@Z 1003259c     alm_db_output.obj
 0002:0000c5c0       __unwindtable$?about@alm_db_output@@UAE?AVQString@@XZ 100325c0     alm_db_output.obj
 0002:0000c5c8       __ehfuncinfo$?about@alm_db_output@@UAE?AVQString@@XZ 100325c8     alm_db_output.obj
 0002:0000c5ec       __unwindtable$?sendCommand@alm_db_output@@UAEXABVQString@@0@Z 100325ec     alm_db_output.obj
 0002:0000c5f4       __ehfuncinfo$?sendCommand@alm_db_output@@UAEXABVQString@@0@Z 100325f4     alm_db_output.obj
 0002:0000c618       __ehfuncinfo$?pasteSelectedProcs@alm_db_output@@AAEX_N@Z 10032618     alm_db_output.obj
 0002:0000c63c       __unwindtable$?pasteSelectedProcs@alm_db_output@@AAEX_N@Z 1003263c     alm_db_output.obj
 0002:0000c6cc       __ehfuncinfo$?pasteOptions@alm_db_output@@AAEXXZ 100326cc     alm_db_output.obj
 0002:0000c6f0       __unwindtable$?pasteOptions@alm_db_output@@AAEXXZ 100326f0     alm_db_output.obj
 0002:0000c718       __ehfuncinfo$?copyToClipBoard@alm_db_output@@AAEXXZ 10032718     alm_db_output.obj
 0002:0000c73c       __unwindtable$?copyToClipBoard@alm_db_output@@AAEXXZ 1003273c     alm_db_output.obj
 0002:0000c7a4       __ehfuncinfo$?editSelectedProcs@alm_db_output@@AAEXXZ 100327a4     alm_db_output.obj
 0002:0000c7c8       __unwindtable$?editSelectedProcs@alm_db_output@@AAEXXZ 100327c8     alm_db_output.obj
 0002:0000c928       __unwindtable$?menuDeleteFile@alm_db_output@@AAEXXZ 10032928     alm_db_output.obj
 0002:0000c940       __ehfuncinfo$?menuDeleteFile@alm_db_output@@AAEXXZ 10032940     alm_db_output.obj
 0002:0000c964       __ehfuncinfo$?menuDuplicateFile@alm_db_output@@AAEXXZ 10032964     alm_db_output.obj
 0002:0000c988       __unwindtable$?menuDuplicateFile@alm_db_output@@AAEXXZ 10032988     alm_db_output.obj
 0002:0000c9f0       __unwindtable$?markDirty@alm_db_output@@AAEXXZ 100329f0     alm_db_output.obj
 0002:0000c9f0       __unwindtable$?EditProcess@alm_db_output@@AAEXXZ 100329f0     alm_db_output.obj
 0002:0000c9f0       __unwindtable$?apply@alm_db_output@@EAEXXZ 100329f0     alm_db_output.obj
 0002:0000c9f8       __ehfuncinfo$?EditProcess@alm_db_output@@AAEXXZ 100329f8     alm_db_output.obj
 0002:0000c9f8       __ehfuncinfo$?apply@alm_db_output@@EAEXXZ 100329f8     alm_db_output.obj
 0002:0000c9f8       __ehfuncinfo$?markDirty@alm_db_output@@AAEXXZ 100329f8     alm_db_output.obj
 0002:0000ca1c       __ehfuncinfo$?renameModule@alm_db_output@@AAEXPAVQListViewItem@@HABVQString@@@Z 10032a1c     alm_db_output.obj
 0002:0000ca40       __unwindtable$?renameModule@alm_db_output@@AAEXPAVQListViewItem@@HABVQString@@@Z 10032a40     alm_db_output.obj
 0002:0000ca68       __ehfuncinfo$?selectFile@alm_db_output@@AAEXPAVQListViewItem@@@Z 10032a68     alm_db_output.obj
 0002:0000ca8c       __unwindtable$?selectFile@alm_db_output@@AAEXPAVQListViewItem@@@Z 10032a8c     alm_db_output.obj
 0002:0000cacc       __ehfuncinfo$?selectSystem@alm_db_output@@AAEXABVQString@@@Z 10032acc     alm_db_output.obj
 0002:0000caf0       __unwindtable$?selectSystem@alm_db_output@@AAEXABVQString@@@Z 10032af0     alm_db_output.obj
 0002:0000cbb0       __ehfuncinfo$?filterChange@alm_db_output@@AAEXXZ 10032bb0     alm_db_output.obj
 0002:0000cbd4       __unwindtable$?filterChange@alm_db_output@@AAEXXZ 10032bd4     alm_db_output.obj
 0002:0000cbfc       __ehfuncinfo$?templateProcess@alm_db_output@@AAEXXZ 10032bfc     alm_db_output.obj
 0002:0000cc20       __unwindtable$?templateProcess@alm_db_output@@AAEXXZ 10032c20     alm_db_output.obj
 0002:0000cd10       __unwindtable$?useAltId@alm_db_output@@AAE?AVQString@@V2@ABV2@_N@Z 10032d10     alm_db_output.obj
 0002:0000cd28       __ehfuncinfo$?useAltId@alm_db_output@@AAE?AVQString@@V2@ABV2@_N@Z 10032d28     alm_db_output.obj
 0002:0000cd4c       __unwindtable$?addProcSetting@alm_db_output@@AAEXPAVcProcess@@ABVQString@@@Z 10032d4c     alm_db_output.obj
 0002:0000cd5c       __ehfuncinfo$?addProcSetting@alm_db_output@@AAEXPAVcProcess@@ABVQString@@@Z 10032d5c     alm_db_output.obj
 0002:0000cd80       __ehfuncinfo$?decodeSystem@alm_db_output@@AAEXABVQString@@@Z 10032d80     alm_db_output.obj
 0002:0000cda4       __unwindtable$?decodeSystem@alm_db_output@@AAEXABVQString@@@Z 10032da4     alm_db_output.obj
 0002:0000cddc       __ehfuncinfo$?updateFileList@alm_db_output@@AAEXXZ 10032ddc     alm_db_output.obj
 0002:0000ce00       __unwindtable$?updateFileList@alm_db_output@@AAEXXZ 10032e00     alm_db_output.obj
 0002:0000d010       __ehfuncinfo$?loadFile@alm_db_output@@AAE_NABVQString@@@Z 10033010     alm_db_output.obj
 0002:0000d034       __unwindtable$?loadFile@alm_db_output@@AAE_NABVQString@@@Z 10033034     alm_db_output.obj
 0002:0000d10c       __ehfuncinfo$?saveFile@alm_db_output@@AAE_NPAVcOutputFile@@@Z 1003310c     alm_db_output.obj
 0002:0000d130       __unwindtable$?saveFile@alm_db_output@@AAE_NPAVcOutputFile@@@Z 10033130     alm_db_output.obj
 0002:0000d370       __ehfuncinfo$?newFile@alm_db_output@@AAEXABVQString@@@Z 10033370     alm_db_output.obj
 0002:0000d394       __unwindtable$?newFile@alm_db_output@@AAEXABVQString@@@Z 10033394     alm_db_output.obj
 0002:0000d424       __ehfuncinfo$?AllocateCfgFileName@alm_db_output@@AAEXAAVQString@@0AAH@Z 10033424     alm_db_output.obj
 0002:0000d448       __unwindtable$?AllocateCfgFileName@alm_db_output@@AAEXAAVQString@@0AAH@Z 10033448     alm_db_output.obj
 0002:0000d490       __unwindtable$?allocateSystemName@alm_db_output@@AAEXAAVQString@@@Z 10033490     alm_db_output.obj
 0002:0000d4a8       __ehfuncinfo$?allocateSystemName@alm_db_output@@AAEXAAVQString@@@Z 100334a8     alm_db_output.obj
 0002:0000d4cc       __ehfuncinfo$?loadProcesses@alm_db_output@@AAE_NABVQString@@@Z 100334cc     alm_db_output.obj
 0002:0000d4f0       __unwindtable$?loadProcesses@alm_db_output@@AAE_NABVQString@@@Z 100334f0     alm_db_output.obj
 0002:0000d5e8       __unwindtable$?selectProcess@alm_db_output@@AAEXABVQString@@@Z 100335e8     alm_db_output.obj
 0002:0000d5f8       __ehfuncinfo$?selectProcess@alm_db_output@@AAEXABVQString@@@Z 100335f8     alm_db_output.obj
 0002:0000d61c       __ehfuncinfo$?updateList@alm_db_output@@AAEXXZ 1003361c     alm_db_output.obj
 0002:0000d640       __unwindtable$?updateList@alm_db_output@@AAEXXZ 10033640     alm_db_output.obj
 0002:0000d668       __unwindtable$?doUpload@alm_db_output@@AAEXPAVresponse@@@Z 10033668     alm_db_output.obj
 0002:0000d670       __ehfuncinfo$?doUpload@alm_db_output@@AAEXPAVresponse@@@Z 10033670     alm_db_output.obj
 0002:0000d694       __ehfuncinfo$?doLock@alm_db_output@@AAEXPAVresponse@@@Z 10033694     alm_db_output.obj
 0002:0000d6b8       __unwindtable$?doLock@alm_db_output@@AAEXPAVresponse@@@Z 100336b8     alm_db_output.obj
 0002:0000d760       __unwindtable$?doDownload@alm_db_output@@AAEXPAVresponse@@@Z 10033760     alm_db_output.obj
 0002:0000d770       __ehfuncinfo$?doDownload@alm_db_output@@AAEXPAVresponse@@@Z 10033770     alm_db_output.obj
 0002:0000d794       __ehfuncinfo$?doDone@alm_db_output@@AAEXPAVresponse@@@Z 10033794     alm_db_output.obj
 0002:0000d7b8       __unwindtable$?doDone@alm_db_output@@AAEXPAVresponse@@@Z 100337b8     alm_db_output.obj
 0002:0000d8a0       __ehfuncinfo$?doDownloadRead@alm_db_output@@AAEXPAVresponse@@@Z 100338a0     alm_db_output.obj
 0002:0000d8c4       __unwindtable$?doDownloadRead@alm_db_output@@AAEXPAVresponse@@@Z 100338c4     alm_db_output.obj
 0002:0000d9cc       __unwindtable$??0FileLoad_BncsSystem@alm_db_output@@QAE@PAV1@@Z 100339cc     alm_db_output.obj
 0002:0000d9ec       __ehfuncinfo$??0FileLoad_BncsSystem@alm_db_output@@QAE@PAV1@@Z 100339ec     alm_db_output.obj
 0002:0000da10       __unwindtable$??1FileLoad_BncsSystem@alm_db_output@@UAE@XZ 10033a10     alm_db_output.obj
 0002:0000da18       __ehfuncinfo$??1FileLoad_BncsSystem@alm_db_output@@UAE@XZ 10033a18     alm_db_output.obj
 0002:0000da3c       __unwindtable$??1?$QDict@VQAction@@@@UAE@XZ 10033a3c     alm_db_output.obj
 0002:0000da44       __ehfuncinfo$??1?$QDict@VQAction@@@@UAE@XZ 10033a44     alm_db_output.obj
 0002:0000da68       __unwindtable$??1?$QPtrList@VcOutputFile@@@@UAE@XZ 10033a68     alm_db_output.obj
 0002:0000da68       __unwindtable$??1?$QPtrList@VQPopupMenu@@@@UAE@XZ 10033a68     alm_db_output.obj
 0002:0000da68       __unwindtable$??1?$QPtrList@VcProcess@@@@UAE@XZ 10033a68     alm_db_output.obj
 0002:0000da70       __ehfuncinfo$??1?$QPtrList@VcOutputFile@@@@UAE@XZ 10033a70     alm_db_output.obj
 0002:0000da70       __ehfuncinfo$??1?$QPtrList@VQPopupMenu@@@@UAE@XZ 10033a70     alm_db_output.obj
 0002:0000da70       __ehfuncinfo$??1?$QPtrList@VcProcess@@@@UAE@XZ 10033a70     alm_db_output.obj
 0002:0000da94       __unwindtable$?copy@?$QMapPrivate@VQString@@PAVcProcess@@@@QAEPAU?$QMapNode@VQString@@PAVcProcess@@@@PAU2@@Z 10033a94     alm_db_output.obj
 0002:0000da94       __unwindtable$??0?$QMapPrivate@VQString@@PAVcProcess@@@@QAE@PBV0@@Z 10033a94     alm_db_output.obj
 0002:0000da9c       __ehfuncinfo$??0?$QMapPrivate@VQString@@PAVcProcess@@@@QAE@PBV0@@Z 10033a9c     alm_db_output.obj
 0002:0000da9c       __ehfuncinfo$?copy@?$QMapPrivate@VQString@@PAVcProcess@@@@QAEPAU?$QMapNode@VQString@@PAVcProcess@@@@PAU2@@Z 10033a9c     alm_db_output.obj
 0002:0000dac0       __unwindtable$??0?$QMapNode@VQString@@PAVcProcess@@@@QAE@ABU0@@Z 10033ac0     alm_db_output.obj
 0002:0000dac0       __unwindtable$??0?$QMapNode@VQString@@PAVcProcess@@@@QAE@ABVQString@@@Z 10033ac0     alm_db_output.obj
 0002:0000dac8       __ehfuncinfo$??0?$QMapNode@VQString@@PAVcProcess@@@@QAE@ABU0@@Z 10033ac8     alm_db_output.obj
 0002:0000dac8       __ehfuncinfo$??0?$QMapNode@VQString@@PAVcProcess@@@@QAE@ABVQString@@@Z 10033ac8     alm_db_output.obj
 0002:0000daec       __unwindtable$??1cOutputFile@@UAE@XZ 10033aec     cOutputFile.obj
 0002:0000daec       __unwindtable$??0cOutputFile@@QAE@XZ 10033aec     cOutputFile.obj
 0002:0000dafc       __ehfuncinfo$??1cOutputFile@@UAE@XZ 10033afc     cOutputFile.obj
 0002:0000dafc       __ehfuncinfo$??0cOutputFile@@QAE@XZ 10033afc     cOutputFile.obj
 0002:0000db20       __ehfuncinfo$??0cProcess@@QAE@VQString@@@Z 10033b20     cProcess.obj
 0002:0000db44       __unwindtable$??0cProcess@@QAE@VQString@@@Z 10033b44     cProcess.obj
 0002:0000db94       __ehfuncinfo$??1cProcess@@UAE@XZ 10033b94     cProcess.obj
 0002:0000dbb8       __unwindtable$??1cProcess@@UAE@XZ 10033bb8     cProcess.obj
 0002:0000dbf8       __ehfuncinfo$??0dbConnection@@QAE@XZ 10033bf8     DBCONNECTION.obj
 0002:0000dc1c       __unwindtable$??0dbConnection@@QAE@XZ 10033c1c     DBCONNECTION.obj
 0002:0000dc6c       __ehfuncinfo$??1dbConnection@@UAE@XZ 10033c6c     DBCONNECTION.obj
 0002:0000dc90       __unwindtable$??1dbConnection@@UAE@XZ 10033c90     DBCONNECTION.obj
 0002:0000dcc8       __ehfuncinfo$?run@dbConnection@@UAEXXZ 10033cc8     DBCONNECTION.obj
 0002:0000dcec       __unwindtable$?run@dbConnection@@UAEXXZ 10033cec     DBCONNECTION.obj
 0002:0000dd44       __ehfuncinfo$?lastError@dbConnection@@QAE?AVQString@@XZ 10033d44     DBCONNECTION.obj
 0002:0000dd68       __unwindtable$?lastError@dbConnection@@QAE?AVQString@@XZ 10033d68     DBCONNECTION.obj
 0002:0000dde0       __ehfuncinfo$??0dialog@@QAE@PAVIGetDocuments@@PAVQWidget@@PBDI@Z 10033de0     dialogimpl.obj
 0002:0000de04       __unwindtable$??0dialog@@QAE@PAVIGetDocuments@@PAVQWidget@@PBDI@Z 10033e04     dialogimpl.obj
 0002:0000dfa4       __ehfuncinfo$??1dialog@@UAE@XZ 10033fa4     dialogimpl.obj
 0002:0000dfc8       __unwindtable$??1dialog@@UAE@XZ 10033fc8     dialogimpl.obj
 0002:0000e1a8       __ehfuncinfo$?saveProcess@dialog@@QAE_NPAVcProcess@@@Z 100341a8     dialogimpl.obj
 0002:0000e1cc       __unwindtable$?saveProcess@dialog@@QAE_NPAVcProcess@@@Z 100341cc     dialogimpl.obj
 0002:0000e20c       __unwindtable$?dbToolsStart@dialog@@QAEXXZ 1003420c     dialogimpl.obj
 0002:0000e224       __ehfuncinfo$?dbToolsStart@dialog@@QAEXXZ 10034224     dialogimpl.obj
 0002:0000e248       __ehfuncinfo$?getSep@dialog@@QAE?AVQString@@H@Z 10034248     dialogimpl.obj
 0002:0000e26c       __unwindtable$?getSep@dialog@@QAE?AVQString@@H@Z 1003426c     dialogimpl.obj
 0002:0000e29c       __ehfuncinfo$?itemChanged@dialog@@QAEXABVQString@@@Z 1003429c     dialogimpl.obj
 0002:0000e2c0       __unwindtable$?itemChanged@dialog@@QAEXABVQString@@@Z 100342c0     dialogimpl.obj
 0002:0000e300       __unwindtable$?dbDriverChanged@dialog@@QAEXABVQString@@@Z 10034300     dialogimpl.obj
 0002:0000e300       __unwindtable$?dbDriverChanged_reserve@dialog@@QAEXABVQString@@@Z 10034300     dialogimpl.obj
 0002:0000e310       __ehfuncinfo$?dbDriverChanged_reserve@dialog@@QAEXABVQString@@@Z 10034310     dialogimpl.obj
 0002:0000e310       __ehfuncinfo$?dbDriverChanged@dialog@@QAEXABVQString@@@Z 10034310     dialogimpl.obj
 0002:0000e334       __unwindtable$?copyData@dialog@@QAEXXZ 10034334     dialogimpl.obj
 0002:0000e34c       __ehfuncinfo$?copyData@dialog@@QAEXXZ 1003434c     dialogimpl.obj
 0002:0000e370       __ehfuncinfo$?pasteData@dialog@@QAEXXZ 10034370     dialogimpl.obj
 0002:0000e394       __unwindtable$?pasteData@dialog@@QAEXXZ 10034394     dialogimpl.obj
 0002:0000e41c       __ehfuncinfo$?dbEditStart@dialog@@QAEXXZ 1003441c     dialogimpl.obj
 0002:0000e440       __unwindtable$?dbEditStart@dialog@@QAEXXZ 10034440     dialogimpl.obj
 0002:0000e468       __unwindtable$?fillDataTable@dialog@@QAEXXZ 10034468     dialogimpl.obj
 0002:0000e478       __ehfuncinfo$?fillDataTable@dialog@@QAEXXZ 10034478     dialogimpl.obj
 0002:0000e49c       __unwindtable$?clearAllProcesses@dialog@@QAEXXZ 1003449c     dialogimpl.obj
 0002:0000e49c       __unwindtable$?clearAllLogs@dialog@@QAEXXZ 1003449c     dialogimpl.obj
 0002:0000e4bc       __ehfuncinfo$?clearAllLogs@dialog@@QAEXXZ 100344bc     dialogimpl.obj
 0002:0000e4bc       __ehfuncinfo$?clearAllProcesses@dialog@@QAEXXZ 100344bc     dialogimpl.obj
 0002:0000e4e0       __ehfuncinfo$?clearProcessesBefore@dialog@@QAEXXZ 100344e0     dialogimpl.obj
 0002:0000e4e0       __ehfuncinfo$?clearLogsBefore@dialog@@QAEXXZ 100344e0     dialogimpl.obj
 0002:0000e504       __unwindtable$?clearProcessesBefore@dialog@@QAEXXZ 10034504     dialogimpl.obj
 0002:0000e504       __unwindtable$?clearLogsBefore@dialog@@QAEXXZ 10034504     dialogimpl.obj
 0002:0000e52c       __ehfuncinfo$?createNewLogTable@dialog@@QAEXXZ 1003452c     dialogimpl.obj
 0002:0000e550       __unwindtable$?createNewLogTable@dialog@@QAEXXZ 10034550     dialogimpl.obj
 0002:0000e628       __ehfuncinfo$?createNewProcTable@dialog@@QAEXXZ 10034628     dialogimpl.obj
 0002:0000e64c       __unwindtable$?createNewProcTable@dialog@@QAEXXZ 1003464c     dialogimpl.obj
 0002:0000e714       __ehfuncinfo$?dbToolUpdate@dialog@@QAEXXZ 10034714     dialogimpl.obj
 0002:0000e738       __unwindtable$?dbToolUpdate@dialog@@QAEXXZ 10034738     dialogimpl.obj
 0002:0000e7a8       __ehfuncinfo$?setAllDefaultText@dialog@@QAEXXZ 100347a8     dialogimpl.obj
 0002:0000e7cc       __unwindtable$?setAllDefaultText@dialog@@QAEXXZ 100347cc     dialogimpl.obj
 0002:0000e804       __ehfuncinfo$?clearAllText@dialog@@QAEXXZ 10034804     dialogimpl.obj
 0002:0000e828       __unwindtable$?clearAllText@dialog@@QAEXXZ 10034828     dialogimpl.obj
 0002:0000e860       __unwindtable$?setAckDefaultText@dialog@@QAEXXZ 10034860     dialogimpl.obj
 0002:0000e860       __unwindtable$?setLatchedDefaultText@dialog@@QAEXXZ 10034860     dialogimpl.obj
 0002:0000e860       __unwindtable$?setIgnoreDefaultText@dialog@@QAEXXZ 10034860     dialogimpl.obj
 0002:0000e860       __unwindtable$?setOkDefaultText@dialog@@QAEXXZ 10034860     dialogimpl.obj
 0002:0000e860       __unwindtable$?setFailDefaultText@dialog@@QAEXXZ 10034860     dialogimpl.obj
 0002:0000e860       __unwindtable$?setUnknownDefaultText@dialog@@QAEXXZ 10034860     dialogimpl.obj
 0002:0000e870       __ehfuncinfo$?setIgnoreDefaultText@dialog@@QAEXXZ 10034870     dialogimpl.obj
 0002:0000e870       __ehfuncinfo$?setUnknownDefaultText@dialog@@QAEXXZ 10034870     dialogimpl.obj
 0002:0000e870       __ehfuncinfo$?setOkDefaultText@dialog@@QAEXXZ 10034870     dialogimpl.obj
 0002:0000e870       __ehfuncinfo$?setFailDefaultText@dialog@@QAEXXZ 10034870     dialogimpl.obj
 0002:0000e870       __ehfuncinfo$?setLatchedDefaultText@dialog@@QAEXXZ 10034870     dialogimpl.obj
 0002:0000e870       __ehfuncinfo$?setAckDefaultText@dialog@@QAEXXZ 10034870     dialogimpl.obj
 0002:0000e894       __unwindtable$?setGroupDefaultText@dialog@@QAEXXZ 10034894     dialogimpl.obj
 0002:0000e894       __unwindtable$?procSelection@alm_db_output@@AAEXXZ 10034894     dialogimpl.obj
 0002:0000e8a4       __ehfuncinfo$?setGroupDefaultText@dialog@@QAEXXZ 100348a4     dialogimpl.obj
 0002:0000e8a4       __ehfuncinfo$?procSelection@alm_db_output@@AAEXXZ 100348a4     dialogimpl.obj
 0002:0000e8c8       __ehfuncinfo$?dbStartConnect@dialog@@AAEXXZ 100348c8     dialogimpl.obj
 0002:0000e8ec       __unwindtable$?dbStartConnect@dialog@@AAEXXZ 100348ec     dialogimpl.obj
 0002:0000e954       __ehfuncinfo$?useAltId@dialog@@AAE?AVQString@@V2@0_N@Z 10034954     dialogimpl.obj
 0002:0000e978       __unwindtable$?useAltId@dialog@@AAE?AVQString@@V2@0_N@Z 10034978     dialogimpl.obj
 0002:0000e9a8       __unwindtable$?connectDb@dialog@@AAEPAVQSqlDatabase@@XZ 100349a8     dialogimpl.obj
 0002:0000e9c8       __ehfuncinfo$?connectDb@dialog@@AAEPAVQSqlDatabase@@XZ 100349c8     dialogimpl.obj
 0002:0000e9ec       __ehfuncinfo$?defaultText@dialog@@AAE?AVQString@@W4AlarmStates@Alarms@@@Z 100349ec     dialogimpl.obj
 0002:0000ea10       __unwindtable$?defaultText@dialog@@AAE?AVQString@@W4AlarmStates@Alarms@@@Z 10034a10     dialogimpl.obj
 0002:0000ea90       __ehfuncinfo$??0manage_temp@@QAE@QAV?$QMap@VQString@@PAVcProcess@@@@PAVdialog@@@Z 10034a90     manage_tempimpl.obj
 0002:0000eab4       __unwindtable$??0manage_temp@@QAE@QAV?$QMap@VQString@@PAVcProcess@@@@PAVdialog@@@Z 10034ab4     manage_tempimpl.obj
 0002:0000eb0c       __ehfuncinfo$??1manage_temp@@UAE@XZ 10034b0c     manage_tempimpl.obj
 0002:0000eb30       __unwindtable$??1manage_temp@@UAE@XZ 10034b30     manage_tempimpl.obj
 0002:0000eb88       __unwindtable$?levelChanged@dialog@@QAEXH@Z 10034b88     manage_tempimpl.obj
 0002:0000eb88       __unwindtable$?setDefaultGroup@manage_temp@@QAEXVQString@@@Z 10034b88     manage_tempimpl.obj
 0002:0000eb90       __ehfuncinfo$?levelChanged@dialog@@QAEXH@Z 10034b90     manage_tempimpl.obj
 0002:0000eb90       __ehfuncinfo$?setDefaultGroup@manage_temp@@QAEXVQString@@@Z 10034b90     manage_tempimpl.obj
 0002:0000ebb4       __ehfuncinfo$?setProcess@manage_temp@@AAEXPAVQListViewItem@@@Z 10034bb4     manage_tempimpl.obj
 0002:0000ebd8       __unwindtable$?setProcess@manage_temp@@AAEXPAVQListViewItem@@@Z 10034bd8     manage_tempimpl.obj
 0002:0000ec08       __ehfuncinfo$?defaultText@manage_temp@@AAE?AVQString@@W4AlarmStates@Alarms@@@Z 10034c08     manage_tempimpl.obj
 0002:0000ec2c       __unwindtable$?defaultText@manage_temp@@AAE?AVQString@@W4AlarmStates@Alarms@@@Z 10034c2c     manage_tempimpl.obj
 0002:0000ed0c       __ehfuncinfo$?prefixChanged@manage_temp@@QAEXABVQString@@@Z 10034d0c     manage_tempimpl.obj
 0002:0000ed30       __unwindtable$?prefixChanged@manage_temp@@QAEXABVQString@@@Z 10034d30     manage_tempimpl.obj
 0002:0000ede0       __ehfuncinfo$?selectProcess@manage_temp@@QAEXPAVQListViewItem@@@Z 10034de0     manage_tempimpl.obj
 0002:0000ee04       __unwindtable$?selectProcess@manage_temp@@QAEXPAVQListViewItem@@@Z 10034e04     manage_tempimpl.obj
 0002:0000ee4c       __unwindtable$?setAllParamsDefaultText@manage_temp@@QAEXXZ 10034e4c     manage_tempimpl.obj
 0002:0000ee4c       __unwindtable$?clearAllParamsText@manage_temp@@QAEXXZ 10034e4c     manage_tempimpl.obj
 0002:0000ee5c       __ehfuncinfo$?setAllParamsDefaultText@manage_temp@@QAEXXZ 10034e5c     manage_tempimpl.obj
 0002:0000ee5c       __ehfuncinfo$?clearAllParamsText@manage_temp@@QAEXXZ 10034e5c     manage_tempimpl.obj
 0002:0000ee80       __ehfuncinfo$?resetDefaults@dialog@@QAEXXZ 10034e80     manage_tempimpl.obj
 0002:0000ee80       __ehfuncinfo$?setAllDefaultText@manage_temp@@QAEXXZ 10034e80     manage_tempimpl.obj
 0002:0000eea4       __unwindtable$?setAllDefaultText@manage_temp@@QAEXXZ 10034ea4     manage_tempimpl.obj
 0002:0000eea4       __unwindtable$?resetDefaults@dialog@@QAEXXZ 10034ea4     manage_tempimpl.obj
 0002:0000eed4       __ehfuncinfo$?clearAllText@manage_temp@@QAEXXZ 10034ed4     manage_tempimpl.obj
 0002:0000eef8       __unwindtable$?clearAllText@manage_temp@@QAEXXZ 10034ef8     manage_tempimpl.obj
 0002:0000ef38       __unwindtable$?setDeviceDefaultText@manage_temp@@QAEXXZ 10034f38     manage_tempimpl.obj
 0002:0000ef48       __ehfuncinfo$?setDeviceDefaultText@manage_temp@@QAEXXZ 10034f48     manage_tempimpl.obj
 0002:0000ef6c       __ehfuncinfo$?itemChanged@manage_temp@@QAEXXZ 10034f6c     manage_tempimpl.obj
 0002:0000ef90       __unwindtable$?itemChanged@manage_temp@@QAEXXZ 10034f90     manage_tempimpl.obj
 0002:0000efd8       __unwindtable$?keys@plugindesc@@UAE?AVQStringList@@ABVQString@@0@Z 10034fd8     plugindesc.obj
 0002:0000efe8       __ehfuncinfo$?keys@plugindesc@@UAE?AVQStringList@@ABVQString@@0@Z 10034fe8     plugindesc.obj
 0002:0000f00c       __unwindtable$??4?$QGuardedPtr@VQDockWindow@@@@QAEAAV0@PAVQDockWindow@@@Z 1003500c     plugindesc.obj
 0002:0000f00c       __unwindtable$?insert@?$QMapPrivate@VQString@@PAVcProcess@@@@QAE?AV?$QMapIterator@VQString@@PAVcProcess@@@@PAUQMapNodeBase@@0ABVQString@@@Z 1003500c     plugindesc.obj
 0002:0000f00c       __unwindtable$?detachInternal@?$QMap@VQString@@PAVcProcess@@@@AAEXXZ 1003500c     plugindesc.obj
 0002:0000f00c       __unwindtable$??0?$QGuardedPtr@VQDockWindow@@@@QAE@XZ 1003500c     plugindesc.obj
 0002:0000f00c       __unwindtable$?clear@?$QMap@VQString@@PAVcProcess@@@@QAEXXZ 1003500c     plugindesc.obj
 0002:0000f00c       __unwindtable$??0?$QMapPrivate@VQString@@PAVcProcess@@@@QAE@XZ 1003500c     plugindesc.obj
 0002:0000f00c       __unwindtable$?create@plugindesc@@UAEPAVconfig_plugin_base@@ABVQString@@00@Z 1003500c     plugindesc.obj
 0002:0000f00c       __unwindtable$??4?$QGuardedPtr@VQPopupMenu@@@@QAEAAV0@PAVQPopupMenu@@@Z 1003500c     plugindesc.obj
 0002:0000f00c       __unwindtable$??0?$QGuardedPtr@VQPopupMenu@@@@QAE@XZ 1003500c     plugindesc.obj
 0002:0000f00c       __unwindtable$??0?$QMap@VQString@@PAVcProcess@@@@QAE@XZ 1003500c     plugindesc.obj
 0002:0000f014       __ehfuncinfo$??0?$QMap@VQString@@PAVcProcess@@@@QAE@XZ 10035014     plugindesc.obj
 0002:0000f014       __ehfuncinfo$?create@plugindesc@@UAEPAVconfig_plugin_base@@ABVQString@@00@Z 10035014     plugindesc.obj
 0002:0000f014       __ehfuncinfo$?clear@?$QMap@VQString@@PAVcProcess@@@@QAEXXZ 10035014     plugindesc.obj
 0002:0000f014       __ehfuncinfo$??0?$QGuardedPtr@VQDockWindow@@@@QAE@XZ 10035014     plugindesc.obj
 0002:0000f014       __ehfuncinfo$??0?$QMapPrivate@VQString@@PAVcProcess@@@@QAE@XZ 10035014     plugindesc.obj
 0002:0000f014       __ehfuncinfo$??4?$QGuardedPtr@VQPopupMenu@@@@QAEAAV0@PAVQPopupMenu@@@Z 10035014     plugindesc.obj
 0002:0000f014       __ehfuncinfo$?detachInternal@?$QMap@VQString@@PAVcProcess@@@@AAEXXZ 10035014     plugindesc.obj
 0002:0000f014       __ehfuncinfo$??0?$QGuardedPtr@VQPopupMenu@@@@QAE@XZ 10035014     plugindesc.obj
 0002:0000f014       __ehfuncinfo$?insert@?$QMapPrivate@VQString@@PAVcProcess@@@@QAE?AV?$QMapIterator@VQString@@PAVcProcess@@@@PAUQMapNodeBase@@0ABVQString@@@Z 10035014     plugindesc.obj
 0002:0000f014       __ehfuncinfo$??4?$QGuardedPtr@VQDockWindow@@@@QAEAAV0@PAVQDockWindow@@@Z 10035014     plugindesc.obj
 0002:0000f038       __ehfuncinfo$??0setDefaultsBase@@QAE@PAVQWidget@@PBD_NI@Z 10035038     setdefaults.obj
 0002:0000f05c       __unwindtable$??0setDefaultsBase@@QAE@PAVQWidget@@PBD_NI@Z 1003505c     setdefaults.obj
 0002:0000f21c       __ehfuncinfo$?languageChange@setDefaultsBase@@MAEXXZ 1003521c     setdefaults.obj
 0002:0000f240       __unwindtable$?languageChange@setDefaultsBase@@MAEXXZ 10035240     setdefaults.obj
 0002:0000f3a0       __ehfuncinfo$??0setDefaults@@QAE@PAVQWidget@@PBD_NI@Z 100353a0     setdefaultsimpl.obj
 0002:0000f3c4       __unwindtable$??0setDefaults@@QAE@PAVQWidget@@PBD_NI@Z 100353c4     setdefaultsimpl.obj
 0002:0000f3fc       __ehfuncinfo$??0dialogBase@@QAE@PAVQWidget@@PBDI@Z 100353fc     dialog.obj
 0002:0000f420       __unwindtable$??0dialogBase@@QAE@PAVQWidget@@PBDI@Z 10035420     dialog.obj
 0002:0000fa40       __ehfuncinfo$?languageChange@dialogBase@@MAEXXZ 10035a40     dialog.obj
 0002:0000fa64       __unwindtable$?languageChange@dialogBase@@MAEXXZ 10035a64     dialog.obj
 0002:0000fe64       __ehfuncinfo$??0manage_tempBase@@QAE@PAVQWidget@@PBD_NI@Z 10035e64     manage_temp.obj
 0002:0000fe88       __unwindtable$??0manage_tempBase@@QAE@PAVQWidget@@PBD_NI@Z 10035e88     manage_temp.obj
 0002:000100f0       __ehfuncinfo$?languageChange@manage_tempBase@@MAEXXZ 100360f0     manage_temp.obj
 0002:00010114       __unwindtable$?languageChange@manage_tempBase@@MAEXXZ 10036114     manage_temp.obj
 0002:000102d4       __unwindtable$?qt_emit@alm_db_output@@UAE_NHPAUQUObject@@@Z 100362d4     moc_alm_db_output.obj
 0002:000102dc       __ehfuncinfo$?qt_emit@alm_db_output@@UAE_NHPAUQUObject@@@Z 100362dc     moc_alm_db_output.obj
 0002:00010300       __unwindtable$?command@alm_db_output@@IAEXVQString@@0@Z 10036300     moc_alm_db_output.obj
 0002:00010318       __ehfuncinfo$?command@alm_db_output@@IAEXVQString@@0@Z 10036318     moc_alm_db_output.obj
 0002:0001033c       __unwindtable$?setUnknownDefaultText@manage_temp@@QAEXXZ 1003633c     moc_dialogimpl.obj
 0002:0001033c       __unwindtable$?setOkDefaultText@manage_temp@@QAEXXZ 1003633c     moc_dialogimpl.obj
 0002:0001033c       __unwindtable$?setLatchedDefaultText@manage_temp@@QAEXXZ 1003633c     moc_dialogimpl.obj
 0002:0001033c       __unwindtable$?menuNewFile@alm_db_output@@AAEXXZ 1003633c     moc_dialogimpl.obj
 0002:0001033c       __unwindtable$?setAckDefaultText@manage_temp@@QAEXXZ 1003633c     moc_dialogimpl.obj
 0002:0001033c       __unwindtable$?setIgnoreDefaultText@manage_temp@@QAEXXZ 1003633c     moc_dialogimpl.obj
 0002:0001033c       __unwindtable$?getDbase@dbConnection@@QAEPAVQSqlDatabase@@XZ 1003633c     moc_dialogimpl.obj
 0002:0001033c       __unwindtable$?setFailDefaultText@manage_temp@@QAEXXZ 1003633c     moc_dialogimpl.obj
 0002:0001033c       __unwindtable$?qt_invoke@dialog@@UAE_NHPAUQUObject@@@Z 1003633c     moc_dialogimpl.obj
 0002:0001033c       __unwindtable$?itemChanged@dialog@@QAEXH@Z 1003633c     moc_dialogimpl.obj
 0002:00010344       __ehfuncinfo$?setFailDefaultText@manage_temp@@QAEXXZ 10036344     moc_dialogimpl.obj
 0002:00010344       __ehfuncinfo$?itemChanged@dialog@@QAEXH@Z 10036344     moc_dialogimpl.obj
 0002:00010344       __ehfuncinfo$?setLatchedDefaultText@manage_temp@@QAEXXZ 10036344     moc_dialogimpl.obj
 0002:00010344       __ehfuncinfo$?qt_invoke@dialog@@UAE_NHPAUQUObject@@@Z 10036344     moc_dialogimpl.obj
 0002:00010344       __ehfuncinfo$?menuNewFile@alm_db_output@@AAEXXZ 10036344     moc_dialogimpl.obj
 0002:00010344       __ehfuncinfo$?getDbase@dbConnection@@QAEPAVQSqlDatabase@@XZ 10036344     moc_dialogimpl.obj
 0002:00010344       __ehfuncinfo$?setUnknownDefaultText@manage_temp@@QAEXXZ 10036344     moc_dialogimpl.obj
 0002:00010344       __ehfuncinfo$?setOkDefaultText@manage_temp@@QAEXXZ 10036344     moc_dialogimpl.obj
 0002:00010344       __ehfuncinfo$?setIgnoreDefaultText@manage_temp@@QAEXXZ 10036344     moc_dialogimpl.obj
 0002:00010344       __ehfuncinfo$?setAckDefaultText@manage_temp@@QAEXXZ 10036344     moc_dialogimpl.obj
 0002:00010368       __unwindtable$?saveState@cfg_Settings@@SAXABVQString@@0@Z 10036368     cfg_widgets001:cfg_Settings.obj
 0002:00010380       __ehfuncinfo$?saveState@cfg_Settings@@SAXABVQString@@0@Z 10036380     cfg_widgets001:cfg_Settings.obj
 0002:000103a4       __ehfuncinfo$?saveState@cfg_Settings@@SAXQBVQListView@@ABVQString@@@Z 100363a4     cfg_widgets001:cfg_Settings.obj
 0002:000103a4       __ehfuncinfo$?saveState@cfg_Settings@@SAXQBVQTable@@ABVQString@@@Z 100363a4     cfg_widgets001:cfg_Settings.obj
 0002:000103c8       __unwindtable$?saveState@cfg_Settings@@SAXQBVQListView@@ABVQString@@@Z 100363c8     cfg_widgets001:cfg_Settings.obj
 0002:000103c8       __unwindtable$?saveState@cfg_Settings@@SAXQBVQTable@@ABVQString@@@Z 100363c8     cfg_widgets001:cfg_Settings.obj
 0002:000103f0       __unwindtable$?saveState@cfg_Settings@@SAXQBVQSplitter@@ABVQString@@@Z 100363f0     cfg_widgets001:cfg_Settings.obj
 0002:00010410       __ehfuncinfo$?saveState@cfg_Settings@@SAXQBVQSplitter@@ABVQString@@@Z 10036410     cfg_widgets001:cfg_Settings.obj
 0002:00010434       __ehfuncinfo$?saveState@cfg_Settings@@SAXABVQPoint@@ABVQSize@@AB_NABVQString@@@Z 10036434     cfg_widgets001:cfg_Settings.obj
 0002:00010458       __unwindtable$?saveState@cfg_Settings@@SAXABVQPoint@@ABVQSize@@AB_NABVQString@@@Z 10036458     cfg_widgets001:cfg_Settings.obj
 0002:00010490       __unwindtable$?loadState@cfg_Settings@@SA?AVQString@@ABV2@@Z 10036490     cfg_widgets001:cfg_Settings.obj
 0002:000104b0       __ehfuncinfo$?loadState@cfg_Settings@@SA?AVQString@@ABV2@@Z 100364b0     cfg_widgets001:cfg_Settings.obj
 0002:000104d4       __unwindtable$?loadState@cfg_Settings@@SAXQAVQListView@@ABVQString@@@Z 100364d4     cfg_widgets001:cfg_Settings.obj
 0002:000104d4       __unwindtable$?loadState@cfg_Settings@@SAXQAVQTable@@ABVQString@@@Z 100364d4     cfg_widgets001:cfg_Settings.obj
 0002:000104e4       __ehfuncinfo$?loadState@cfg_Settings@@SAXQAVQTable@@ABVQString@@@Z 100364e4     cfg_widgets001:cfg_Settings.obj
 0002:000104e4       __ehfuncinfo$?loadState@cfg_Settings@@SAXQAVQListView@@ABVQString@@@Z 100364e4     cfg_widgets001:cfg_Settings.obj
 0002:00010508       __unwindtable$?loadState@cfg_Settings@@SAXQAVQSplitter@@ABVQString@@@Z 10036508     cfg_widgets001:cfg_Settings.obj
 0002:00010520       __ehfuncinfo$?loadState@cfg_Settings@@SAXQAVQSplitter@@ABVQString@@@Z 10036520     cfg_widgets001:cfg_Settings.obj
 0002:00010544       __unwindtable$?loadState@cfg_Settings@@SAXAAVQPoint@@AAVQSize@@AA_NABVQString@@@Z 10036544     cfg_widgets001:cfg_Settings.obj
 0002:00010554       __ehfuncinfo$?loadState@cfg_Settings@@SAXAAVQPoint@@AAVQSize@@AA_NABVQString@@@Z 10036554     cfg_widgets001:cfg_Settings.obj
 0002:00010578       __unwindtable$??0Document_BncsSystem@@QAE@XZ 10036578     config_alarm_utilities:Document.obj
 0002:00010590       __ehfuncinfo$??0Document_BncsSystem@@QAE@XZ 10036590     config_alarm_utilities:Document.obj
 0002:000105b4       __unwindtable$?load@Document_BncsSystem@@QAE_NXZ 100365b4     config_alarm_utilities:Document.obj
 0002:000105cc       __ehfuncinfo$?load@Document_BncsSystem@@QAE_NXZ 100365cc     config_alarm_utilities:Document.obj
 0002:000105f0       __unwindtable$??0FileLoad@@IAE@ABVQString@@@Z 100365f0     config_alarm_utilities:Loaders.obj
 0002:000105f0       __unwindtable$??1FileLoad@@UAE@XZ 100365f0     config_alarm_utilities:Loaders.obj
 0002:000105f8       __ehfuncinfo$??0FileLoad@@IAE@ABVQString@@@Z 100365f8     config_alarm_utilities:Loaders.obj
 0002:000105f8       __ehfuncinfo$??1FileLoad@@UAE@XZ 100365f8     config_alarm_utilities:Loaders.obj
 0002:0001061c       __unwindtable$?matches@FileLoad@@QAE_NABVQString@@@Z 1003661c     config_alarm_utilities:Loaders.obj
 0002:00010634       __ehfuncinfo$?matches@FileLoad@@QAE_NABVQString@@@Z 10036634     config_alarm_utilities:Loaders.obj
 0002:00010658       __unwindtable$?request@FileLoad@@QAEXPAVISendCommand@@@Z 10036658     config_alarm_utilities:Loaders.obj
 0002:00010668       __ehfuncinfo$?request@FileLoad@@QAEXPAVISendCommand@@@Z 10036668     config_alarm_utilities:Loaders.obj
 0002:0001068c       __unwindtable$??0Loaders@@QAE@XZ 1003668c     config_alarm_utilities:Loaders.obj
 0002:00010694       __ehfuncinfo$??0Loaders@@QAE@XZ 10036694     config_alarm_utilities:Loaders.obj
 0002:000106b8       __unwindtable$??1Loaders@@UAE@XZ 100366b8     config_alarm_utilities:Loaders.obj
 0002:000106d8       __ehfuncinfo$??1Loaders@@UAE@XZ 100366d8     config_alarm_utilities:Loaders.obj
 0002:000106fc       __unwindtable$??1?$QPtrList@VFileLoad@@@@UAE@XZ 100366fc     config_alarm_utilities:Loaders.obj
 0002:000106fc       __unwindtable$??_G?$QPtrList@VFileLoad@@@@UAEPAXI@Z 100366fc     config_alarm_utilities:Loaders.obj
 0002:000106fc       __unwindtable$??_G?$QPtrList@VDirLoad@@@@UAEPAXI@Z 100366fc     config_alarm_utilities:Loaders.obj
 0002:000106fc       __unwindtable$??1?$QPtrList@VDirLoad@@@@UAE@XZ 100366fc     config_alarm_utilities:Loaders.obj
 0002:00010704       __ehfuncinfo$??1?$QPtrList@VFileLoad@@@@UAE@XZ 10036704     config_alarm_utilities:Loaders.obj
 0002:00010704       __ehfuncinfo$??1?$QPtrList@VDirLoad@@@@UAE@XZ 10036704     config_alarm_utilities:Loaders.obj
 0002:00010704       __ehfuncinfo$??_G?$QPtrList@VDirLoad@@@@UAEPAXI@Z 10036704     config_alarm_utilities:Loaders.obj
 0002:00010704       __ehfuncinfo$??_G?$QPtrList@VFileLoad@@@@UAEPAXI@Z 10036704     config_alarm_utilities:Loaders.obj
 0002:00010728       __sehtable$__onexit        10036728     MSVCRT:atonexit.obj
 0002:00010748       __sehtable$??_L@YGXPAXIHP6EX0@Z1@Z 10036748     MSVCRT:ehvecctr.obj
 0002:00010768       __sehtable$??_M@YGXPAXIHP6EX0@Z@Z 10036768     MSVCRT:ehvecdtr.obj
 0002:00010788       __sehtable$?__ArrayUnwind@@YGXPAXIHP6EX0@Z@Z 10036788     MSVCRT:ehvecdtr.obj
 0002:000107a8       __sehtable$___DllMainCRTStartup 100367a8     MSVCRT:crtdll.obj
 0002:000107d0       __sehtable$__IsNonwritableInCurrentImage 100367d0     MSVCRT:pesect.obj
 0002:000107f0       .edata                     100367f0     config_alm_db_output.exp
 0002:00010818       rgpv                       10036818     config_alm_db_output.exp
 0002:0001081c       rgszName                   1003681c     config_alm_db_output.exp
 0002:00010820       rgwOrd                     10036820     config_alm_db_output.exp
 0002:00010822       szName                     10036822     config_alm_db_output.exp
 0002:0001083b       $N00001                    1003683b     config_alm_db_output.exp
 0002:0001fd62       .idata$6                   10045d62     qt-mt323:qt-mt323.dll
 0002:0001ff48       .idata$6                   10045f48     alm_sys_select:alm_sys_select.dll
 0002:0001ff7c       .idata$6                   10045f7c     config_icons:config_icons.dll
 0002:0001ffaa       .idata$6                   10045faa     kernel32:KERNEL32.dll
 0002:00020052       .idata$6                   10046052     msvcprt:MSVCP120.dll
 0002:000200fc       .idata$6                   100460fc     MSVCRT:MSVCR120.dll
 0003:00000010       _filesave                  10047010     plugindesc.obj
 0003:0000005c       ?param_slot_2@?3??staticMetaObject@alm_db_output@@SAPAVQMetaObject@@XZ@4QBUQUParameter@@B 1004705c     moc_alm_db_output.obj
 0003:0000006c       ?param_slot_13@?3??staticMetaObject@alm_db_output@@SAPAVQMetaObject@@XZ@4QBUQUParameter@@B 1004706c     moc_alm_db_output.obj
 0003:0000009c       ?param_slot_15@?3??staticMetaObject@alm_db_output@@SAPAVQMetaObject@@XZ@4QBUQUParameter@@B 1004709c     moc_alm_db_output.obj
 0003:000000cc       ?param_slot_18@?3??staticMetaObject@alm_db_output@@SAPAVQMetaObject@@XZ@4QBUQUParameter@@B 100470cc     moc_alm_db_output.obj
 0003:000000dc       ?param_slot_2@?3??staticMetaObject@dialog@@SAPAVQMetaObject@@XZ@4QBUQUParameter@@B 100470dc     moc_dialogimpl.obj
 0003:000000ec       ?param_slot_3@?3??staticMetaObject@dialog@@SAPAVQMetaObject@@XZ@4QBUQUParameter@@B 100470ec     moc_dialogimpl.obj
 0003:000000fc       ?param_slot_4@?3??staticMetaObject@dialog@@SAPAVQMetaObject@@XZ@4QBUQUParameter@@B 100470fc     moc_dialogimpl.obj
 0003:0000010c       ?param_slot_5@?3??staticMetaObject@dialog@@SAPAVQMetaObject@@XZ@4QBUQUParameter@@B 1004710c     moc_dialogimpl.obj
 0003:0000011c       ?param_slot_6@?3??staticMetaObject@dialog@@SAPAVQMetaObject@@XZ@4QBUQUParameter@@B 1004711c     moc_dialogimpl.obj
 0003:0000012c       ?param_slot_11@?3??staticMetaObject@dialog@@SAPAVQMetaObject@@XZ@4QBUQUParameter@@B 1004712c     moc_dialogimpl.obj
 0003:0000013c       ?param_slot_12@?3??staticMetaObject@dialog@@SAPAVQMetaObject@@XZ@4QBUQUParameter@@B 1004713c     moc_dialogimpl.obj
 0003:0000014c       ?param_slot_20@?3??staticMetaObject@dialog@@SAPAVQMetaObject@@XZ@4QBUQUParameter@@B 1004714c     moc_dialogimpl.obj
 0003:0000015c       ?param_slot_1@?3??staticMetaObject@manage_temp@@SAPAVQMetaObject@@XZ@4QBUQUParameter@@B 1004715c     moc_manage_tempimpl.obj
 0003:0000016c       ?param_slot_3@?3??staticMetaObject@manage_temp@@SAPAVQMetaObject@@XZ@4QBUQUParameter@@B 1004716c     moc_manage_tempimpl.obj
 0003:00000ba8       _allocator_arg             10047ba8     alm_db_output.obj
 0003:00000ba9       _piecewise_construct       10047ba9     alm_db_output.obj
 0003:00000bb4       ?bLoaded@?1??loadProcesses@alm_db_output@@AAE_NABVQString@@@Z@4_NA 10047bb4     alm_db_output.obj
 0003:00000bb8       ?iCount@?1???0dbConnection@@QAE@XZ@4HA 10047bb8     DBCONNECTION.obj
 0003:00000bc0       _cleanUp_setDefaultsBase   10047bc0     moc_setdefaults.obj
 0003:00000bc8       _cleanUp_setDefaults       10047bc8     moc_setdefaultsimpl.obj
 0003:00000bd0       _cleanUp_alm_db_output     10047bd0     moc_alm_db_output.obj
 0003:00000bd4       ?$S1@?3??staticMetaObject@alm_db_output@@SAPAVQMetaObject@@XZ@4IA 10047bd4     moc_alm_db_output.obj
 0003:00000bd8       ?param_slot_14@?3??staticMetaObject@alm_db_output@@SAPAVQMetaObject@@XZ@4QBUQUParameter@@B 10047bd8     moc_alm_db_output.obj
 0003:00000be8       ?param_signal_0@?3??staticMetaObject@alm_db_output@@SAPAVQMetaObject@@XZ@4QBUQUParameter@@B 10047be8     moc_alm_db_output.obj
 0003:00000c0c       _cleanUp_dialogBase        10047c0c     moc_dialog.obj
 0003:00000c14       _cleanUp_dialog            10047c14     moc_dialogimpl.obj
 0003:00000c18       ?$S1@?3??staticMetaObject@dialog@@SAPAVQMetaObject@@XZ@4IA 10047c18     moc_dialogimpl.obj
 0003:00000c20       _cleanUp_manage_tempBase   10047c20     moc_manage_temp.obj
 0003:00000c28       _cleanUp_manage_temp       10047c28     moc_manage_tempimpl.obj
 0003:00000c2c       ?$S1@?3??staticMetaObject@manage_temp@@SAPAVQMetaObject@@XZ@4IA 10047c2c     moc_manage_tempimpl.obj
 0003:00000c30       ?param_slot_2@?3??staticMetaObject@manage_temp@@SAPAVQMetaObject@@XZ@4QBUQUParameter@@B 10047c30     moc_manage_tempimpl.obj
 0003:00000c44       ___proc_attached           10047c44     MSVCRT:crtdll.obj
 0003:00000c48       _GS_ExceptionRecord        10047c48     MSVCRT:gs_report.obj
 0003:00000c98       _GS_ContextRecord          10047c98     MSVCRT:gs_report.obj
 0003:00000f64       _DebuggerWasPresent        10047f64     MSVCRT:gs_report.obj
 0004:000000a0       $R000000                   100480a0     version.res
 0004:00000550       $R0004B0                   10048550     version.res
